 testPlugin

 Timestamp is 614c801b (Thu Sep 23 13:24:43 2021)

 Preferred load address is 10000000

 Start         Length     Name                   Class
 0001:00000000 00000311H .text$di                CODE
 0001:00000320 00019bccH .text$mn                CODE
 0001:00019ef0 000042b4H .text$x                 CODE
 0001:0001e1b0 0000010bH .text$yd                CODE
 0002:00000000 000012a0H .idata$5                DATA
 0002:000012a0 00000004H .CRT$XCA                DATA
 0002:000012a4 0000005cH .CRT$XCU                DATA
 0002:00001300 00000004H .CRT$XCZ                DATA
 0002:00001304 00000004H .CRT$XIA                DATA
 0002:00001308 00000004H .CRT$XIAA               DATA
 0002:0000130c 00000004H .CRT$XIC                DATA
 0002:00001310 00000004H .CRT$XIZ                DATA
 0002:00001320 0000b6c0H .rdata                  DATA
 0002:0000c9e0 00001bd4H .rdata$r                DATA
 0002:0000e5b4 00000004H .rtc$IAA                DATA
 0002:0000e5b8 00000004H .rtc$IZZ                DATA
 0002:0000e5bc 00000004H .rtc$TAA                DATA
 0002:0000e5c0 00000004H .rtc$TZZ                DATA
 0002:0000e5c8 00003becH .xdata$x                DATA
 0002:000121c0 00000568H .edata                  DATA
 0002:00012728 00000050H .idata$2                DATA
 0002:00012778 00000014H .idata$3                DATA
 0002:0001278c 000012a0H .idata$4                DATA
 0002:00013a2c 0000c12cH .idata$6                DATA
 0003:00000000 00000ec4H .data                   DATA
 0003:00000ec4 0000087cH .data$r                 DATA
 0003:00001740 0000054cH .bss                    DATA
 0004:00000000 000000a0H .rsrc$01                DATA
 0004:000000a0 00000608H .rsrc$02                DATA

  Address         Publics by Value              Rva+Base       Lib:Object

 0000:00000000       ___safe_se_handler_table   00000000     <absolute>
 0000:00000000       ___safe_se_handler_count   00000000     <absolute>
 0000:00000000       ___guard_fids_table        00000000     <absolute>
 0000:00000000       ___guard_fids_count        00000000     <absolute>
 0000:00000000       ___guard_flags             00000000     <absolute>
 0000:00000000       ___ImageBase               10000000     <linker-defined>
 0001:00000320       ??0dialog@@QAE@PAVQWidget@@PBDI@Z 10001320 f   dialogimpl.obj
 0001:00000348       ??1dialog@@UAE@XZ          10001348 f   dialogimpl.obj
 0001:0000035a       ??_Edialog@@WCI@AEPAXI@Z   1000135a f i dialogimpl.obj
 0001:00000362       ??_Gdialog@@UAEPAXI@Z      10001362 f i dialogimpl.obj
 0001:00000362       ??_Edialog@@UAEPAXI@Z      10001362 f i dialogimpl.obj
 0001:00000381       ?metaObject@dialog@@UBEPAVQMetaObject@@XZ 10001381 f i dialogimpl.obj
 0001:00000386       ??0fileDrop@@QAE@PAVQWidget@@PBD@Z 10001386 f   fileDrop.obj
 0001:000003e5       ??1fileDrop@@UAE@XZ        100013e5 f   fileDrop.obj
 0001:000003f8       ??_EfileDrop@@WCI@AEPAXI@Z 100013f8 f i fileDrop.obj
 0001:00000400       ??_EfileDrop@@UAEPAXI@Z    10001400 f i fileDrop.obj
 0001:00000400       ??_GfileDrop@@UAEPAXI@Z    10001400 f i fileDrop.obj
 0001:0000041f       ?cbChanged@fileDrop@@QAEXXZ 1000141f f   fileDrop.obj
 0001:00000445       ?contextMenuEvent@fileDrop@@UAEXPAVQContextMenuEvent@@@Z 10001445 f   fileDrop.obj
 0001:00000566       ?dragEnterEvent@fileDrop@@UAEXPAVQDragEnterEvent@@@Z 10001566 f   fileDrop.obj
 0001:00000599       ?dropEvent@fileDrop@@UAEXPAVQDropEvent@@@Z 10001599 f   fileDrop.obj
 0001:0000063f       ?metaObject@fileDrop@@UBEPAVQMetaObject@@XZ 1000163f f i fileDrop.obj
 0001:00000644       ??0?$QGuardedPtr@VQDockWindow@@@@QAE@XZ 10001644 f i fileManager.obj
 0001:00000644       ??0?$QGuardedPtr@VQPopupMenu@@@@QAE@XZ 10001644 f i fileManager.obj
 0001:00000685       ??0config_plugin_base@@QAE@ABVQString@@00@Z 10001685 f i fileManager.obj
 0001:00000712       ??0fileManager@@QAE@ABVQString@@00@Z 10001712 f   fileManager.obj
 0001:00000aa3       ??1?$QGuardedPtr@VQPopupMenu@@@@QAE@XZ 10001aa3 f i fileManager.obj
 0001:00000aa3       ??1?$QGuardedPtr@VQDockWindow@@@@QAE@XZ 10001aa3 f i fileManager.obj
 0001:00000aa8       ??1?$QPtrList@VQPopupMenu@@@@UAE@XZ 10001aa8 f i fileManager.obj
 0001:00000adb       ??1QDockWindowList@@UAE@XZ 10001adb f i fileManager.obj
 0001:00000b24       ??1QPopupMenuList@@UAE@XZ  10001b24 f i fileManager.obj
 0001:00000b56       ??1config_plugin_base@@UAE@XZ 10001b56 f i fileManager.obj
 0001:00000bb0       ??1fileManager@@UAE@XZ     10001bb0 f   fileManager.obj
 0001:00000c61       ??_EQLabel@@WCI@AEPAXI@Z   10001c61 f i fileManager.obj
 0001:00000c69       ??_EQListView@@WCI@AEPAXI@Z 10001c69 f i fileManager.obj
 0001:00000c71       ??_EQSplitter@@WCI@AEPAXI@Z 10001c71 f i fileManager.obj
 0001:00000c79       ??_EQVBoxLayout@@WCI@AEPAXI@Z 10001c79 f i fileManager.obj
 0001:00000c81       ??_Econfig_plugin_base@@WCI@AEPAXI@Z 10001c81 f i fileManager.obj
 0001:00000c89       ??_EfileManager@@WCI@AEPAXI@Z 10001c89 f i fileManager.obj
 0001:00000c91       ??_G?$QPtrList@VQPopupMenu@@@@UAEPAXI@Z 10001c91 f i fileManager.obj
 0001:00000c91       ??_E?$QPtrList@VQPopupMenu@@@@UAEPAXI@Z 10001c91 f i fileManager.obj
 0001:00000cb0       ??_GQDockWindowList@@UAEPAXI@Z 10001cb0 f i fileManager.obj
 0001:00000cb0       ??_EQDockWindowList@@UAEPAXI@Z 10001cb0 f i fileManager.obj
 0001:00000ccf       ??_GQGuardedPtrPrivate@@UAEPAXI@Z 10001ccf f i fileManager.obj
 0001:00000ccf       ??_EQGuardedPtrPrivate@@UAEPAXI@Z 10001ccf f i fileManager.obj
 0001:00000cef       ??_GQLabel@@UAEPAXI@Z      10001cef f i fileManager.obj
 0001:00000cef       ??_EQLabel@@UAEPAXI@Z      10001cef f i fileManager.obj
 0001:00000d0f       ??_GQListView@@UAEPAXI@Z   10001d0f f i fileManager.obj
 0001:00000d0f       ??_EQListView@@UAEPAXI@Z   10001d0f f i fileManager.obj
 0001:00000d2f       ??_GQListViewItem@@UAEPAXI@Z 10001d2f f i fileManager.obj
 0001:00000d2f       ??_EQListViewItem@@UAEPAXI@Z 10001d2f f i fileManager.obj
 0001:00000d4f       ??_EQPopupMenuList@@UAEPAXI@Z 10001d4f f i fileManager.obj
 0001:00000d4f       ??_GQPopupMenuList@@UAEPAXI@Z 10001d4f f i fileManager.obj
 0001:00000d6e       ??_EQSplitter@@UAEPAXI@Z   10001d6e f i fileManager.obj
 0001:00000d6e       ??_GQSplitter@@UAEPAXI@Z   10001d6e f i fileManager.obj
 0001:00000d8e       ??_GQVBoxLayout@@UAEPAXI@Z 10001d8e f i fileManager.obj
 0001:00000d8e       ??_EQVBoxLayout@@UAEPAXI@Z 10001d8e f i fileManager.obj
 0001:00000dae       ??_Econfig_plugin_base@@UAEPAXI@Z 10001dae f i fileManager.obj
 0001:00000dae       ??_Gconfig_plugin_base@@UAEPAXI@Z 10001dae f i fileManager.obj
 0001:00000dcd       ??_EfileManager@@UAEPAXI@Z 10001dcd f i fileManager.obj
 0001:00000dcd       ??_GfileManager@@UAEPAXI@Z 10001dcd f i fileManager.obj
 0001:00000dec       ?about@config_plugin_base@@UAE?AVQString@@XZ 10001dec f i fileManager.obj
 0001:00000e42       ?activate@fileManager@@UAEX_N@Z 10001e42 f   fileManager.obj
 0001:00000e8c       ?apply@fileManager@@UAEXXZ 10001e8c f   fileManager.obj
 0001:00000e99       ?clear@?$QPtrList@VQPopupMenu@@@@UAEXXZ 10001e99 f i fileManager.obj
 0001:00000ea0       ?deinit@pluginBase@@MAEXPAVQCloseEvent@@@Z 10001ea0 f i pluginBase:pluginBase.obj
 0001:00000ea0       ?deinit@testPluginFromBase@@MAEXPAVQCloseEvent@@@Z 10001ea0 f i testPluginFromBase.obj
 0001:00000ea0       ?closeEvent@config_plugin_base@@UAEXPAVQCloseEvent@@@Z 10001ea0 f i fileManager.obj
 0001:00000ea0       ?closeEvent@fileManager@@UAEXPAVQCloseEvent@@@Z 10001ea0 f i fileManager.obj
 0001:00000eae       ?copyFile@fileManager@@AAEXABVQString@@0@Z 10001eae f   fileManager.obj
 0001:0000101e       ?count@?$QPtrList@VQPopupMenu@@@@UBEIXZ 1000201e f i fileManager.obj
 0001:00001022       ?deref@?$QGuardedPtr@VQPopupMenu@@@@AAEXXZ 10002022 f i fileManager.obj
 0001:00001022       ?deref@?$QGuardedPtr@VQDockWindow@@@@AAEXXZ 10002022 f i fileManager.obj
 0001:00001037       ?dirChanged@fileManager@@QAEXPAVQListViewItem@@@Z 10002037 f   fileManager.obj
 0001:000010fd       ?doFileList@fileManager@@QAEXVQStringList@@@Z 100020fd f   fileManager.obj
 0001:000012ce       ?isDirty@fileManager@@UAE_NXZ 100022ce f   fileManager.obj
 0001:000012d5       ?lviFind@fileManager@@AAEPAVQListViewItem@@PAV2@ABVQString@@@Z 100022d5 f   fileManager.obj
 0001:00001337       ?menus@config_plugin_base@@UAE?AVQPopupMenuList@@XZ 10002337 f   fileManager.obj
 0001:00001337       ?menus@fileManager@@UAE?AVQPopupMenuList@@XZ 10002337 f   fileManager.obj
 0001:0000135a       ?metaObject@fileManager@@UBEPAVQMetaObject@@XZ 1000235a f i fileManager.obj
 0001:0000135f       ?navigate@config_plugin_base@@UAEXABVQString@@0@Z 1000235f f i fileManager.obj
 0001:00001362       ?navigate@fileManager@@UAEXABVQString@@0@Z 10002362 f   fileManager.obj
 0001:00001362       ?navigate@workstationEditor@@UAEXABVQString@@0@Z 10002362 f   workstationEditor.obj
 0001:0000138b       ?reply@fileManager@@UAEXPAVresponse@@@Z 1000238b f   fileManager.obj
 0001:00001e64       ?dragMoveEvent@fileDrop@@UAEXPAVQDragMoveEvent@@@Z 10002e64 f   fileDrop.obj
 0001:00001e64       ?reply@config_plugin_base@@UAEXPAVresponse@@@Z 10002e64 f   fileManager.obj
 0001:00001e64       ?resizeEvent@fileManager@@UAEXPAVQResizeEvent@@@Z 10002e64 f   fileManager.obj
 0001:00001e64       ?activate@config_plugin_base@@UAEX_N@Z 10002e64 f   fileManager.obj
 0001:00001e64       ?dragLeaveEvent@fileDrop@@UAEXPAVQDragLeaveEvent@@@Z 10002e64 f   fileDrop.obj
 0001:00001e67       ?timerEvent@fileManager@@EAEXPAVQTimerEvent@@@Z 10002e67 f   fileManager.obj
 0001:00001ec7       ?toolbars@config_plugin_base@@UAE?AVQDockWindowList@@XZ 10002ec7 f i fileManager.obj
 0001:00001ec7       ?toolbars@fileManager@@UAE?AVQDockWindowList@@XZ 10002ec7 f i fileManager.obj
 0001:00001eeb       ??0fromBaseDialogBase@@QAE@PAVQWidget@@PBDI@Z 10002eeb f   frombasedialog.obj
 0001:0000337c       ??1fromBaseDialogBase@@UAE@XZ 1000437c f   frombasedialog.obj
 0001:0000338f       ??_EQGroupBox@@WCI@AEPAXI@Z 1000438f f i frombasedialog.obj
 0001:00003397       ??_EQHBoxLayout@@WCI@AEPAXI@Z 10004397 f i frombasedialog.obj
 0001:0000339f       ??_EQLineEdit@@WCI@AEPAXI@Z 1000439f f i frombasedialog.obj
 0001:000033a7       ??_EQListBox@@WCI@AEPAXI@Z 100043a7 f i frombasedialog.obj
 0001:000033af       ??_EQPushButton@@WCI@AEPAXI@Z 100043af f i frombasedialog.obj
 0001:000033b7       ??_EQFrame@@WCI@AEPAXI@Z   100043b7 f i frombasedialog.obj
 0001:000033b7       ??_EQWidget@@WCI@AEPAXI@Z  100043b7 f i frombasedialog.obj
 0001:000033bf       ??_EfromBaseDialogBase@@WCI@AEPAXI@Z 100043bf f i frombasedialog.obj
 0001:000033c7       ??_EQGroupBox@@UAEPAXI@Z   100043c7 f i frombasedialog.obj
 0001:000033c7       ??_GQGroupBox@@UAEPAXI@Z   100043c7 f i frombasedialog.obj
 0001:000033e7       ??_GQHBoxLayout@@UAEPAXI@Z 100043e7 f i frombasedialog.obj
 0001:000033e7       ??_EQHBoxLayout@@UAEPAXI@Z 100043e7 f i frombasedialog.obj
 0001:00003407       ??_EQLineEdit@@UAEPAXI@Z   10004407 f i frombasedialog.obj
 0001:00003407       ??_GQLineEdit@@UAEPAXI@Z   10004407 f i frombasedialog.obj
 0001:00003427       ??_GQListBox@@UAEPAXI@Z    10004427 f i frombasedialog.obj
 0001:00003427       ??_EQListBox@@UAEPAXI@Z    10004427 f i frombasedialog.obj
 0001:00003447       ??_EQPushButton@@UAEPAXI@Z 10004447 f i frombasedialog.obj
 0001:00003447       ??_GQPushButton@@UAEPAXI@Z 10004447 f i frombasedialog.obj
 0001:00003467       ??_EQSpacerItem@@UAEPAXI@Z 10004467 f i frombasedialog.obj
 0001:00003467       ??_GQSpacerItem@@UAEPAXI@Z 10004467 f i frombasedialog.obj
 0001:00003487       ??_GQFrame@@UAEPAXI@Z      10004487 f i frombasedialog.obj
 0001:00003487       ??_EQWidget@@UAEPAXI@Z     10004487 f i frombasedialog.obj
 0001:00003487       ??_EQFrame@@UAEPAXI@Z      10004487 f i frombasedialog.obj
 0001:00003487       ??_GQWidget@@UAEPAXI@Z     10004487 f i frombasedialog.obj
 0001:000034a7       ??_EfromBaseDialogBase@@UAEPAXI@Z 100044a7 f i frombasedialog.obj
 0001:000034a7       ??_GfromBaseDialogBase@@UAEPAXI@Z 100044a7 f i frombasedialog.obj
 0001:000034c6       ?languageChange@fromBaseDialogBase@@MAEXXZ 100044c6 f   frombasedialog.obj
 0001:000039b0       ?metaObject@fromBaseDialogBase@@UBEPAVQMetaObject@@XZ 100049b0 f i frombasedialog.obj
 0001:000039b5       ??0fromBaseDialog@@QAE@PAVQWidget@@PBD_NI@Z 100049b5 f   frombasedialogimpl.obj
 0001:000039dd       ??1fromBaseDialog@@UAE@XZ  100049dd f   frombasedialogimpl.obj
 0001:000039ef       ??_EfromBaseDialog@@WCI@AEPAXI@Z 100049ef f i frombasedialogimpl.obj
 0001:000039f7       ??_GfromBaseDialog@@UAEPAXI@Z 100049f7 f i frombasedialogimpl.obj
 0001:000039f7       ??_EfromBaseDialog@@UAEPAXI@Z 100049f7 f i frombasedialogimpl.obj
 0001:00003a16       ?metaObject@fromBaseDialog@@UBEPAVQMetaObject@@XZ 10004a16 f i frombasedialogimpl.obj
 0001:00003a1b       ??0launchCustomTable@@QAE@PAVQWidget@@PBD@Z 10004a1b f   launchCustomTable.obj
 0001:00003b62       ??1cfg_Table@@UAE@XZ       10004b62 f i launchCustomTable.obj
 0001:00003b68       ??1launchCustomTable@@UAE@XZ 10004b68 f   launchCustomTable.obj
 0001:00003b7b       ??_ElaunchCustomTable@@WCI@AEPAXI@Z 10004b7b f i launchCustomTable.obj
 0001:00003b83       ??_ElaunchCustomTable@@UAEPAXI@Z 10004b83 f i launchCustomTable.obj
 0001:00003b83       ??_GlaunchCustomTable@@UAEPAXI@Z 10004b83 f i launchCustomTable.obj
 0001:00003ba2       ?endEdit@launchCustomTable@@QAEXXZ 10004ba2 f   launchCustomTable.obj
 0001:00003be7       ?metaObject@cfg_Table@@UBEPAVQMetaObject@@XZ 10004be7 f i launchCustomTable.obj
 0001:00003bed       ??0launchEditor@@QAE@ABVQString@@00@Z 10004bed f   launchEditor.obj
 0001:00004585       ??1?$QDict@VQAction@@@@UAE@XZ 10005585 f i launchEditor.obj
 0001:000045b8       ??1launchEditor@@UAE@XZ    100055b8 f   launchEditor.obj
 0001:0000469c       ??4?$QGuardedPtr@VQPopupMenu@@@@QAEAAV0@PAVQPopupMenu@@@Z 1000569c f i launchEditor.obj
 0001:0000469c       ??4?$QGuardedPtr@VQDockWindow@@@@QAEAAV0@PAVQDockWindow@@@Z 1000569c f i launchEditor.obj
 0001:000046fa       ??_EQDockWindow@@WCI@AEPAXI@Z 100056fa f i launchEditor.obj
 0001:00004702       ??_EQPopupMenu@@WCI@AEPAXI@Z 10005702 f i launchEditor.obj
 0001:0000470a       ??_EQPopupMenu@@WIM@AEPAXI@Z 1000570a f i launchEditor.obj
 0001:00004715       ??_EQToolBar@@WCI@AEPAXI@Z 10005715 f i launchEditor.obj
 0001:0000471d       ??_ElaunchEditor@@WCI@AEPAXI@Z 1000571d f i launchEditor.obj
 0001:00004725       ??_G?$QDict@VQAction@@@@UAEPAXI@Z 10005725 f i launchEditor.obj
 0001:00004725       ??_E?$QDict@VQAction@@@@UAEPAXI@Z 10005725 f i launchEditor.obj
 0001:00004744       ??_EQAction@@UAEPAXI@Z     10005744 f i launchEditor.obj
 0001:00004744       ??_GQAction@@UAEPAXI@Z     10005744 f i launchEditor.obj
 0001:00004764       ??_EQDockWindow@@UAEPAXI@Z 10005764 f i launchEditor.obj
 0001:00004764       ??_GQDockWindow@@UAEPAXI@Z 10005764 f i launchEditor.obj
 0001:00004784       ??_EQPopupMenu@@UAEPAXI@Z  10005784 f i launchEditor.obj
 0001:00004784       ??_GQPopupMenu@@UAEPAXI@Z  10005784 f i launchEditor.obj
 0001:000047a4       ??_GQToolBar@@UAEPAXI@Z    100057a4 f i launchEditor.obj
 0001:000047a4       ??_EQToolBar@@UAEPAXI@Z    100057a4 f i launchEditor.obj
 0001:000047c4       ??_ElaunchEditor@@UAEPAXI@Z 100057c4 f i launchEditor.obj
 0001:000047c4       ??_GlaunchEditor@@UAEPAXI@Z 100057c4 f i launchEditor.obj
 0001:000047e3       ?about@launchEditor@@UAE?AVQString@@XZ 100057e3 f   launchEditor.obj
 0001:0000488b       ?activate@launchEditor@@UAEX_N@Z 1000588b f   launchEditor.obj
 0001:00004a28       ?apply@launchEditor@@UAEXXZ 10005a28 f   launchEditor.obj
 0001:00004a77       ?clear@?$QDict@VQAction@@@@UAEXXZ 10005a77 f i launchEditor.obj
 0001:00004a7d       ?closeEvent@launchEditor@@UAEXPAVQCloseEvent@@@Z 10005a7d f   launchEditor.obj
 0001:00004ae3       ?count@?$QDict@VQAction@@@@UBEIXZ 10005ae3 f i launchEditor.obj
 0001:00004ae7       ?deleteItem@?$QPtrList@VQPopupMenu@@@@EAEXPAX@Z 10005ae7 f i fileManager.obj
 0001:00004ae7       ?deleteItem@?$QDict@VQAction@@@@EAEXPAX@Z 10005ae7 f i launchEditor.obj
 0001:00004b02       ?isDirty@launchEditor@@UAE_NXZ 10005b02 f   launchEditor.obj
 0001:00004b0f       ?metaObject@launchEditor@@UBEPAVQMetaObject@@XZ 10005b0f f i launchEditor.obj
 0001:00004b14       ?navigate@launchEditor@@UAEXABVQString@@0@Z 10005b14 f   launchEditor.obj
 0001:00004b7b       ?navigateToWs@launchEditor@@AAEXH@Z 10005b7b f   launchEditor.obj
 0001:00004bff       ?navigateWSEditor@launchEditor@@AAEXXZ 10005bff f   launchEditor.obj
 0001:00004c41       ?reply@launchEditor@@UAEXPAVresponse@@@Z 10005c41 f   launchEditor.obj
 0001:00004f86       ?textStatus@response@@QAE?AVQString@@W4status@1@@Z 10005f86 f i launchEditor.obj
 0001:00004fd5       ?toolbars@launchEditor@@UAE?AVQDockWindowList@@XZ 10005fd5 f   launchEditor.obj
 0001:0000502d       ?workstationChanged@launchEditor@@AAEXPAVQListViewItem@@@Z 1000602d f   launchEditor.obj
 0001:000050dd       ??0launchEditorDlg@@QAE@ABVQString@@PAVQWidget@@PBDI@Z 100060dd f   launcheditordlgimpl.obj
 0001:00005386       ??1launchEditorDlg@@UAE@XZ 10006386 f   launcheditordlgimpl.obj
 0001:000053c5       ??_ElaunchEditorDlg@@WCI@AEPAXI@Z 100063c5 f i launcheditordlgimpl.obj
 0001:000053cd       ??_EQCheckTableItem@@UAEPAXI@Z 100063cd f i launcheditordlgimpl.obj
 0001:000053cd       ??_GQCheckTableItem@@UAEPAXI@Z 100063cd f i launcheditordlgimpl.obj
 0001:000053ed       ??_ElaunchEditorDlg@@UAEPAXI@Z 100063ed f i launcheditordlgimpl.obj
 0001:000053ed       ??_GlaunchEditorDlg@@UAEPAXI@Z 100063ed f i launcheditordlgimpl.obj
 0001:0000540c       ?createLaunchElement@launchEditorDlg@@QAE?AVQDomElement@@ABVQString@@AAVQDomDocument@@@Z 1000640c f   launcheditordlgimpl.obj
 0001:00005825       ?csiValueChanged@launchEditorDlg@@QAEXABVQString@@@Z 10006825 f   launcheditordlgimpl.obj
 0001:00005870       ?doAdd@launchEditorDlg@@QAEXXZ 10006870 f   launcheditordlgimpl.obj
 0001:00005a34       ?doDuplicate@launchEditorDlg@@QAEXXZ 10006a34 f   launcheditordlgimpl.obj
 0001:00005c29       ?doMoveDown@launchEditorDlg@@QAEXXZ 10006c29 f   launcheditordlgimpl.obj
 0001:00005cee       ?doMoveUp@launchEditorDlg@@QAEXXZ 10006cee f   launcheditordlgimpl.obj
 0001:00005d92       ?doRemove@launchEditorDlg@@QAEXXZ 10006d92 f   launcheditordlgimpl.obj
 0001:00005def       ?load@launchEditorDlg@@QAE_NABVQString@@H@Z 10006def f   launcheditordlgimpl.obj
 0001:0000658b       ?metaObject@launchEditorDlg@@UBEPAVQMetaObject@@XZ 1000758b f i launcheditordlgimpl.obj
 0001:00006590       ?rebootoptionchanged@launchEditorDlg@@QAEXXZ 10007590 f   launcheditordlgimpl.obj
 0001:000065d9       ?save@launchEditorDlg@@QAEXH@Z 100075d9 f   launcheditordlgimpl.obj
 0001:000069df       ?tableValueChanged@launchEditorDlg@@QAEXHH@Z 100079df f   launcheditordlgimpl.obj
 0001:00006a47       ??_Gconfig_plugin_desc_base@@UAEPAXI@Z 10007a47 f i plugindesc.obj
 0001:00006a47       ??_Eplugindesc@@UAEPAXI@Z  10007a47 f i plugindesc.obj
 0001:00006a47       ??_Gplugindesc@@UAEPAXI@Z  10007a47 f i plugindesc.obj
 0001:00006a47       ??_Econfig_plugin_desc_base@@UAEPAXI@Z 10007a47 f i plugindesc.obj
 0001:00006a67       ?create@plugindesc@@UAEPAVconfig_plugin_base@@ABVQString@@00@Z 10007a67 f   plugindesc.obj
 0001:00006b97       ?keys@plugindesc@@UAE?AVQStringList@@ABVQString@@0@Z 10007b97 f   plugindesc.obj
 0001:00006cc3       ?pixmap@plugindesc@@UAE?AVQPixmap@@ABVQString@@@Z 10007cc3 f   plugindesc.obj
 0001:00006d2f       _load_bncs_config_plugin_desc 10007d2f f   plugindesc.obj
 0001:00006d45       ??0testPlugin@@QAE@ABVQString@@00@Z 10007d45 f   testPlugin.obj
 0001:0000820c       ??1testPlugin@@UAE@XZ      1000920c f   testPlugin.obj
 0001:000082ac       ??_EtestPlugin@@WCI@AEPAXI@Z 100092ac f i testPlugin.obj
 0001:000082b4       ??_GtestPlugin@@UAEPAXI@Z  100092b4 f i testPlugin.obj
 0001:000082b4       ??_EtestPlugin@@UAEPAXI@Z  100092b4 f i testPlugin.obj
 0001:000082d3       ?activate@testPlugin@@UAEX_N@Z 100092d3 f   testPlugin.obj
 0001:00008349       ?apply@testPlugin@@UAEXXZ  10009349 f   testPlugin.obj
 0001:000083ab       ?checkoutDir@testPlugin@@AAEXXZ 100093ab f   testPlugin.obj
 0001:000083f5       ?checkoutFile@testPlugin@@AAEXXZ 100093f5 f   testPlugin.obj
 0001:0000843f       ?closeEvent@testPlugin@@UAEXPAVQCloseEvent@@@Z 1000943f f   testPlugin.obj
 0001:000085bf       ?db@testPlugin@@AAEXVQString@@@Z 100095bf f   testPlugin.obj
 0001:000085f9       ?dbClear@testPlugin@@AAEXXZ 100095f9 f   testPlugin.obj
 0001:00008608       ?dir@testPlugin@@AAEXXZ    10009608 f   testPlugin.obj
 0001:00008652       ?doDirty@testPlugin@@AAEXXZ 10009652 f   testPlugin.obj
 0001:0000869b       ?doHelp@testPlugin@@AAEXXZ 1000969b f   testPlugin.obj
 0001:000086e5       ?doNavigate@testPlugin@@AAEXXZ 100096e5 f   testPlugin.obj
 0001:0000872f       ?downloadDir@testPlugin@@AAEXXZ 1000972f f   testPlugin.obj
 0001:00008779       ?downloadFile@testPlugin@@AAEXXZ 10009779 f   testPlugin.obj
 0001:000087c3       ?isDirty@testPlugin@@UAE_NXZ 100097c3 f   testPlugin.obj
 0001:000087ca       ?lockFile@testPlugin@@AAEXXZ 100097ca f   testPlugin.obj
 0001:00008814       ?menus@testPlugin@@UAE?AVQPopupMenuList@@XZ 10009814 f   testPlugin.obj
 0001:00008873       ?metaObject@testPlugin@@UBEPAVQMetaObject@@XZ 10009873 f i testPlugin.obj
 0001:00008878       ?navigate@testPlugin@@UAEXABVQString@@0@Z 10009878 f   testPlugin.obj
 0001:000088e1       ?reply@testPlugin@@UAEXPAVresponse@@@Z 100098e1 f   testPlugin.obj
 0001:00008a71       ?toolbars@testPlugin@@UAE?AVQDockWindowList@@XZ 10009a71 f   testPlugin.obj
 0001:00008ade       ?unlockDir@testPlugin@@AAEXXZ 10009ade f   testPlugin.obj
 0001:00008b28       ?unlockFile@testPlugin@@AAEXXZ 10009b28 f   testPlugin.obj
 0001:00008b72       ?uploadDir@testPlugin@@AAEXXZ 10009b72 f   testPlugin.obj
 0001:00008bbc       ?uploadFile@testPlugin@@AAEXXZ 10009bbc f   testPlugin.obj
 0001:00008c06       ??0testPluginFromBase@@QAE@ABVQString@@00@Z 10009c06 f   testPluginFromBase.obj
 0001:00009940       ??1testPluginFromBase@@UAE@XZ 1000a940 f   testPluginFromBase.obj
 0001:00009952       ??_EtestPluginFromBase@@WCI@AEPAXI@Z 1000a952 f i testPluginFromBase.obj
 0001:0000995a       ??_EtestPluginFromBase@@UAEPAXI@Z 1000a95a f i testPluginFromBase.obj
 0001:0000995a       ??_GtestPluginFromBase@@UAEPAXI@Z 1000a95a f i testPluginFromBase.obj
 0001:00009979       ?checkoutDirS@testPluginFromBase@@AAEXXZ 1000a979 f   testPluginFromBase.obj
 0001:00009ae2       ?checkoutFileS@testPluginFromBase@@AAEXXZ 1000aae2 f   testPluginFromBase.obj
 0001:00009c30       ?db@testPluginFromBase@@AAEXVQString@@@Z 1000ac30 f   testPluginFromBase.obj
 0001:00009c6a       ?dbClearS@testPluginFromBase@@AAEXXZ 1000ac6a f   testPluginFromBase.obj
 0001:00009c79       ?dirS@testPluginFromBase@@AAEXXZ 1000ac79 f   testPluginFromBase.obj
 0001:00009e5d       ?doCleanS@testPluginFromBase@@AAEXXZ 1000ae5d f   testPluginFromBase.obj
 0001:00009f0a       ?doDirtyS@testPluginFromBase@@AAEXXZ 1000af0a f   testPluginFromBase.obj
 0001:00009fc0       ?init@pluginBase@@MAEXXZ   1000afc0 f   pluginBase:pluginBase.obj
 0001:00009fc0       ?apply@config_plugin_base@@UAEXXZ 1000afc0 f   fileManager.obj
 0001:00009fc0       ?doNavigateS@testPluginFromBase@@AAEXXZ 1000afc0 f   testPluginFromBase.obj
 0001:00009fc0       ?doHelpS@testPluginFromBase@@AAEXXZ 1000afc0 f   testPluginFromBase.obj
 0001:00009fc1       ?downloadDirS@testPluginFromBase@@AAEXXZ 1000afc1 f   testPluginFromBase.obj
 0001:0000a12a       ?downloadFileS@testPluginFromBase@@AAEXXZ 1000b12a f   testPluginFromBase.obj
 0001:0000a278       ?init@testPluginFromBase@@MAEXXZ 1000b278 f   testPluginFromBase.obj
 0001:0000a2e8       ?lastError@configFile@@QAE?AVQString@@XZ 1000b2e8 f i testPluginFromBase.obj
 0001:0000a306       ?loadFile@testPluginFromBase@@MAEXVQString@@@Z 1000b306 f   testPluginFromBase.obj
 0001:0000a365       ?lockFileS@testPluginFromBase@@AAEXXZ 1000b365 f   testPluginFromBase.obj
 0001:0000a4b3       ?metaObject@testPluginFromBase@@UBEPAVQMetaObject@@XZ 1000b4b3 f i testPluginFromBase.obj
 0001:0000a4b8       ?saveFile@testPluginFromBase@@MAEXVQString@@@Z 1000b4b8 f   testPluginFromBase.obj
 0001:0000a517       ?unlockDirS@testPluginFromBase@@AAEXXZ 1000b517 f   testPluginFromBase.obj
 0001:0000a680       ?unlockFileS@testPluginFromBase@@AAEXXZ 1000b680 f   testPluginFromBase.obj
 0001:0000a7ce       ?uploadDirS@testPluginFromBase@@AAEXXZ 1000b7ce f   testPluginFromBase.obj
 0001:0000a937       ?uploadFileS@testPluginFromBase@@AAEXXZ 1000b937 f   testPluginFromBase.obj
 0001:0000aa85       ??0workstationCustomTable@@QAE@PAVQWidget@@PBD@Z 1000ba85 f   workstationCustomTable.obj
 0001:0000abb1       ??1workstationCustomTable@@UAE@XZ 1000bbb1 f   workstationCustomTable.obj
 0001:0000abc4       ??_EworkstationCustomTable@@WCI@AEPAXI@Z 1000bbc4 f i workstationCustomTable.obj
 0001:0000abcc       ??_EworkstationCustomTable@@UAEPAXI@Z 1000bbcc f i workstationCustomTable.obj
 0001:0000abcc       ??_GworkstationCustomTable@@UAEPAXI@Z 1000bbcc f i workstationCustomTable.obj
 0001:0000abeb       ?destroyed@workstationCustomTable@@QAEXXZ 1000bbeb f   workstationCustomTable.obj
 0001:0000abf8       ?metaObject@workstationCustomTable@@UBEPAVQMetaObject@@XZ 1000bbf8 f i workstationCustomTable.obj
 0001:0000abfd       ?sortColumn@workstationCustomTable@@QAEXHHH@Z 1000bbfd f   workstationCustomTable.obj
 0001:0000ac23       ??0workstationDockWindow@@QAE@PAVQWidget@@PBDI@Z 1000bc23 f   workstationdockwindowimpl.obj
 0001:0000ad59       ??1workstationDockWindow@@UAE@XZ 1000bd59 f   workstationdockwindowimpl.obj
 0001:0000ad6b       ??_EworkstationDockWindow@@WCI@AEPAXI@Z 1000bd6b f i workstationdockwindowimpl.obj
 0001:0000ad73       ??_GworkstationDockWindow@@UAEPAXI@Z 1000bd73 f i workstationdockwindowimpl.obj
 0001:0000ad73       ??_EworkstationDockWindow@@UAEPAXI@Z 1000bd73 f i workstationdockwindowimpl.obj
 0001:0000ad92       ?clearSelection@workstationDockWindow@@QAEXXZ 1000bd92 f   workstationdockwindowimpl.obj
 0001:0000ad9d       ?findItem@workstationDockWindow@@QAEPAVQListViewItem@@ABVQString@@H@Z 1000bd9d f   workstationdockwindowimpl.obj
 0001:0000adb5       ?load@workstationDockWindow@@QAEXABVQString@@@Z 1000bdb5 f   workstationdockwindowimpl.obj
 0001:0000adc1       ?metaObject@workstationDockWindow@@UBEPAVQMetaObject@@XZ 1000bdc1 f i workstationdockwindowimpl.obj
 0001:0000adc6       ?setSelected@workstationDockWindow@@QAEXPAVQListViewItem@@_N@Z 1000bdc6 f   workstationdockwindowimpl.obj
 0001:0000add5       ??0workstationEditor@@QAE@ABVQString@@00@Z 1000bdd5 f   workstationEditor.obj
 0001:0000b414       ??1workstationEditor@@UAE@XZ 1000c414 f   workstationEditor.obj
 0001:0000b4c4       ??_EworkstationEditor@@WCI@AEPAXI@Z 1000c4c4 f i workstationEditor.obj
 0001:0000b4cc       ??_GworkstationEditor@@UAEPAXI@Z 1000c4cc f i workstationEditor.obj
 0001:0000b4cc       ??_EworkstationEditor@@UAEPAXI@Z 1000c4cc f i workstationEditor.obj
 0001:0000b4eb       ?about@workstationEditor@@UAE?AVQString@@XZ 1000c4eb f   workstationEditor.obj
 0001:0000b593       ?activate@workstationEditor@@UAEX_N@Z 1000c593 f   workstationEditor.obj
 0001:0000b6fb       ?apply@workstationEditor@@UAEXXZ 1000c6fb f   workstationEditor.obj
 0001:0000b7eb       ?closeEvent@workstationEditor@@UAEXPAVQCloseEvent@@@Z 1000c7eb f   workstationEditor.obj
 0001:0000b8c1       ?inc@?$QMapIterator@VQString@@H@@AAEHXZ 1000c8c1 f i workstationEditor.obj
 0001:0000b8f2       ?isDirty@workstationEditor@@UAE_NXZ 1000c8f2 f   workstationEditor.obj
 0001:0000b8ff       ?menus@workstationEditor@@UAE?AVQPopupMenuList@@XZ 1000c8ff f   workstationEditor.obj
 0001:0000b8ff       ?menus@launchEditor@@UAE?AVQPopupMenuList@@XZ 1000c8ff f   launchEditor.obj
 0001:0000b949       ?metaObject@workstationEditor@@UBEPAVQMetaObject@@XZ 1000c949 f i workstationEditor.obj
 0001:0000b94e       ?reply@workstationEditor@@UAEXPAVresponse@@@Z 1000c94e f   workstationEditor.obj
 0001:0000bcaf       ?resizeEvent@testPlugin@@UAEXPAVQResizeEvent@@@Z 1000ccaf f   testPlugin.obj
 0001:0000bcaf       ?resizeEvent@launchEditor@@UAEXPAVQResizeEvent@@@Z 1000ccaf f   launchEditor.obj
 0001:0000bcaf       ?resizeEvent@workstationEditor@@UAEXPAVQResizeEvent@@@Z 1000ccaf f   workstationEditor.obj
 0001:0000bce4       ?toolbars@workstationEditor@@UAE?AVQDockWindowList@@XZ 1000cce4 f   workstationEditor.obj
 0001:0000bd2e       ??0workstationEditorDlg@@QAE@ABVQString@@PAVQWidget@@PBDI@Z 1000cd2e f   workstationeditordlgimpl.obj
 0001:0000be5e       ??1workstationEditorDlg@@UAE@XZ 1000ce5e f   workstationeditordlgimpl.obj
 0001:0000be9d       ??_EworkstationEditorDlg@@WCI@AEPAXI@Z 1000ce9d f i workstationeditordlgimpl.obj
 0001:0000bea5       ??_EworkstationEditorDlg@@UAEPAXI@Z 1000cea5 f i workstationeditordlgimpl.obj
 0001:0000bea5       ??_GworkstationEditorDlg@@UAEPAXI@Z 1000cea5 f i workstationeditordlgimpl.obj
 0001:0000bec4       ?doAdd@workstationEditorDlg@@AAEXXZ 1000cec4 f   workstationeditordlgimpl.obj
 0001:0000c226       ?doRemove@workstationEditorDlg@@AAEXXZ 1000d226 f   workstationeditordlgimpl.obj
 0001:0000c2bf       ?load@workstationEditorDlg@@QAE_NABVQString@@@Z 1000d2bf f   workstationeditordlgimpl.obj
 0001:0000c6d0       ?metaObject@workstationEditorDlg@@UBEPAVQMetaObject@@XZ 1000d6d0 f i workstationeditordlgimpl.obj
 0001:0000c6d5       ?newBNCSSystemIni@workstationEditorDlg@@AAEXH_N0@Z 1000d6d5 f   workstationeditordlgimpl.obj
 0001:0000cafd       ?save@workstationEditorDlg@@QAEXXZ 1000dafd f   workstationeditordlgimpl.obj
 0001:0000cd5b       ?tableValueChanged@workstationEditorDlg@@AAEXHH@Z 1000dd5b f   workstationeditordlgimpl.obj
 0001:0000cdb4       ?toXML@@YA?AVQString@@ABV1@@Z 1000ddb4 f   workstationeditordlgimpl.obj
 0001:0000cf4e       ??0workstationEditorNewWsDlg@@QAE@ABVQString@@PAVQWidget@@PBD_NI@Z 1000df4e f   workstationeditornewwsdlgimpl.obj
 0001:0000cfbf       ??1workstationEditorNewWsDlg@@UAE@XZ 1000dfbf f   workstationeditornewwsdlgimpl.obj
 0001:0000d011       ??_EworkstationEditorNewWsDlg@@WCI@AEPAXI@Z 1000e011 f i workstationeditornewwsdlgimpl.obj
 0001:0000d019       ??_GworkstationEditorNewWsDlg@@UAEPAXI@Z 1000e019 f i workstationeditornewwsdlgimpl.obj
 0001:0000d019       ??_EworkstationEditorNewWsDlg@@UAEPAXI@Z 1000e019 f i workstationeditornewwsdlgimpl.obj
 0001:0000d038       ?accept@workstationEditorNewWsDlg@@UAEXXZ 1000e038 f   workstationeditornewwsdlgimpl.obj
 0001:0000d1f4       ?loadUsers@workstationEditorNewWsDlg@@AAEXXZ 1000e1f4 f   workstationeditornewwsdlgimpl.obj
 0001:0000d3cc       ?metaObject@workstationEditorNewWsDlg@@UBEPAVQMetaObject@@XZ 1000e3cc f i workstationeditornewwsdlgimpl.obj
 0001:0000d3d1       ?setExistingWs@workstationEditorNewWsDlg@@QAEXABVQStringList@@@Z 1000e3d1 f   workstationeditornewwsdlgimpl.obj
 0001:0000d3e1       ??0workstationUserTableItem@@QAE@ABVQString@@PAVQTable@@W4EditType@QTableItem@@0@Z 1000e3e1 f   workstationUserTableItem.obj
 0001:0000d42e       ??1workstationUserTableItem@@UAE@XZ 1000e42e f   workstationUserTableItem.obj
 0001:0000d464       ??_EQComboBox@@WCI@AEPAXI@Z 1000e464 f i workstationUserTableItem.obj
 0001:0000d46c       ??_GQComboBox@@UAEPAXI@Z   1000e46c f i workstationUserTableItem.obj
 0001:0000d46c       ??_EQComboBox@@UAEPAXI@Z   1000e46c f i workstationUserTableItem.obj
 0001:0000d48c       ??_EworkstationUserTableItem@@UAEPAXI@Z 1000e48c f i workstationUserTableItem.obj
 0001:0000d48c       ??_GworkstationUserTableItem@@UAEPAXI@Z 1000e48c f i workstationUserTableItem.obj
 0001:0000d4ab       ?createEditor@workstationUserTableItem@@UBEPAVQWidget@@XZ 1000e4ab f   workstationUserTableItem.obj
 0001:0000d735       ?setContentFromEditor@workstationUserTableItem@@UAEXPAVQWidget@@@Z 1000e735 f   workstationUserTableItem.obj
 0001:0000d790       ?createDirectory@xfer@@QAEXAAVQString@@@Z 1000e790 f   xfer.obj
 0001:0000d8bb       ?setFileDate@xfer@@QAE_NABVQString@@AAVQDateTime@@@Z 1000e8bb f   xfer.obj
 0001:0000da29       ??0xml_listview@@QAE@PAVQWidget@@PBDI@Z 1000ea29 f   xml_listview.obj
 0001:0000da8c       ??1xml_listview@@UAE@XZ    1000ea8c f   xml_listview.obj
 0001:0000dacc       ??_Exml_listview@@WCI@AEPAXI@Z 1000eacc f i xml_listview.obj
 0001:0000dad4       ??_Exml_listview@@UAEPAXI@Z 1000ead4 f i xml_listview.obj
 0001:0000dad4       ??_Gxml_listview@@UAEPAXI@Z 1000ead4 f i xml_listview.obj
 0001:0000daf3       ?addColumns@xml_listview@@QAEXAAVQStringList@@0@Z 1000eaf3 f   xml_listview.obj
 0001:0000db56       ?load@xml_listview@@QAEXABVQString@@@Z 1000eb56 f   xml_listview.obj
 0001:0000e970       ?metaObject@xml_listview@@UBEPAVQMetaObject@@XZ 1000f970 f i xml_listview.obj
 0001:0000e975       ?startDrag@xml_listview@@UAEXXZ 1000f975 f   xml_listview.obj
 0001:0000e991       ??0dialogBase@@QAE@PAVQWidget@@PBDI@Z 1000f991 f   dialog.obj
 0001:0000fd48       ??1dialogBase@@UAE@XZ      10010d48 f   dialog.obj
 0001:0000fd5b       ??_EdialogBase@@WCI@AEPAXI@Z 10010d5b f i dialog.obj
 0001:0000fd63       ??_EdialogBase@@UAEPAXI@Z  10010d63 f i dialog.obj
 0001:0000fd63       ??_GdialogBase@@UAEPAXI@Z  10010d63 f i dialog.obj
 0001:0000fd82       ?languageChange@dialogBase@@MAEXXZ 10010d82 f   dialog.obj
 0001:00010237       ?metaObject@dialogBase@@UBEPAVQMetaObject@@XZ 10011237 f i dialog.obj
 0001:0001023c       ??0launchEditorDlgBase@@QAE@PAVQWidget@@PBDI@Z 1001123c f   launcheditordlg.obj
 0001:00010c57       ??1launchEditorDlgBase@@UAE@XZ 10011c57 f   launcheditordlg.obj
 0001:00010c97       ??_ElaunchEditorDlgBase@@WCI@AEPAXI@Z 10011c97 f i launcheditordlg.obj
 0001:00010c9f       ??_GlaunchEditorDlgBase@@UAEPAXI@Z 10011c9f f i launcheditordlg.obj
 0001:00010c9f       ??_ElaunchEditorDlgBase@@UAEPAXI@Z 10011c9f f i launcheditordlg.obj
 0001:00010cbe       ?languageChange@launchEditorDlgBase@@MAEXXZ 10011cbe f   launcheditordlg.obj
 0001:000114b6       ?metaObject@launchEditorDlgBase@@UBEPAVQMetaObject@@XZ 100124b6 f i launcheditordlg.obj
 0001:000114bb       ?className@dialogBase@@UBEPBDXZ 100124bb f   moc_dialog.obj
 0001:000114c1       ?qt_cast@dialogBase@@UAEPAXPBD@Z 100124c1 f   moc_dialog.obj
 0001:000114ef       ?qt_invoke@dialogBase@@UAE_NHPAUQUObject@@@Z 100124ef f   moc_dialog.obj
 0001:00011521       ?staticMetaObject@dialogBase@@SAPAVQMetaObject@@XZ 10012521 f   moc_dialog.obj
 0001:0001156b       ?tr@dialogBase@@SA?AVQString@@PBD0@Z 1001256b f   moc_dialog.obj
 0001:000115ae       ?className@dialog@@UBEPBDXZ 100125ae f   moc_dialogimpl.obj
 0001:000115b4       ?qt_cast@dialog@@UAEPAXPBD@Z 100125b4 f   moc_dialogimpl.obj
 0001:000115e1       ?qt_invoke@dialog@@UAE_NHPAUQUObject@@@Z 100125e1 f   moc_dialogimpl.obj
 0001:000115ea       ?staticMetaObject@dialog@@SAPAVQMetaObject@@XZ 100125ea f   moc_dialogimpl.obj
 0001:0001162e       ?className@fileDrop@@UBEPBDXZ 1001262e f   moc_fileDrop.obj
 0001:00011634       ?fileList@fileDrop@@IAEXVQStringList@@@Z 10012634 f   moc_fileDrop.obj
 0001:000116d0       ?qt_cast@fileDrop@@UAEPAXPBD@Z 100126d0 f   moc_fileDrop.obj
 0001:000116fe       ?qt_emit@fileDrop@@UAE_NHPAUQUObject@@@Z 100126fe f   moc_fileDrop.obj
 0001:0001173e       ?qt_invoke@fileDrop@@UAE_NHPAUQUObject@@@Z 1001273e f   moc_fileDrop.obj
 0001:0001176d       ?staticMetaObject@fileDrop@@SAPAVQMetaObject@@XZ 1001276d f   moc_fileDrop.obj
 0001:000117eb       ?className@fileManager@@UBEPBDXZ 100127eb f   moc_fileManager.obj
 0001:000117f1       ?command@fileManager@@IAEXVQString@@0@Z 100127f1 f   moc_fileManager.obj
 0001:000118b1       ?qt_cast@fileManager@@UAEPAXPBD@Z 100128b1 f   moc_fileManager.obj
 0001:000118df       ?qt_emit@fileManager@@UAE_NHPAUQUObject@@@Z 100128df f   moc_fileManager.obj
 0001:00011943       ?qt_invoke@fileManager@@UAE_NHPAUQUObject@@@Z 10012943 f   moc_fileManager.obj
 0001:00011998       ?staticMetaObject@fileManager@@SAPAVQMetaObject@@XZ 10012998 f   moc_fileManager.obj
 0001:00011a85       ?className@fromBaseDialogBase@@UBEPBDXZ 10012a85 f   moc_frombasedialog.obj
 0001:00011a8b       ?qt_cast@fromBaseDialogBase@@UAEPAXPBD@Z 10012a8b f   moc_frombasedialog.obj
 0001:00011ab9       ?qt_emit@workstationEditorDlgBase@@UAE_NHPAUQUObject@@@Z 10012ab9 f   moc_workstationeditordlg.obj
 0001:00011ab9       ?qt_emit@dialogBase@@UAE_NHPAUQUObject@@@Z 10012ab9 f   moc_dialog.obj
 0001:00011ab9       ?qt_emit@workstationDockWindowBase@@UAE_NHPAUQUObject@@@Z 10012ab9 f   moc_workstationdockwindow.obj
 0001:00011ab9       ?qt_emit@fromBaseDialogBase@@UAE_NHPAUQUObject@@@Z 10012ab9 f   moc_frombasedialog.obj
 0001:00011ab9       ?qt_emit@launchEditorDlgBase@@UAE_NHPAUQUObject@@@Z 10012ab9 f   moc_launcheditordlg.obj
 0001:00011ac3       ?qt_invoke@fromBaseDialogBase@@UAE_NHPAUQUObject@@@Z 10012ac3 f   moc_frombasedialog.obj
 0001:00011af5       ?staticMetaObject@fromBaseDialogBase@@SAPAVQMetaObject@@XZ 10012af5 f   moc_frombasedialog.obj
 0001:00011b3f       ?tr@fromBaseDialogBase@@SA?AVQString@@PBD0@Z 10012b3f f   moc_frombasedialog.obj
 0001:00011b82       ?className@fromBaseDialog@@UBEPBDXZ 10012b82 f   moc_frombasedialogimpl.obj
 0001:00011b88       ?qt_cast@fromBaseDialog@@UAEPAXPBD@Z 10012b88 f   moc_frombasedialogimpl.obj
 0001:00011bb5       ?qt_emit@fromBaseDialog@@UAE_NHPAUQUObject@@@Z 10012bb5 f   moc_frombasedialogimpl.obj
 0001:00011bb5       ?qt_emit@dialog@@UAE_NHPAUQUObject@@@Z 10012bb5 f   moc_dialogimpl.obj
 0001:00011bbe       ?qt_invoke@fromBaseDialog@@UAE_NHPAUQUObject@@@Z 10012bbe f   moc_frombasedialogimpl.obj
 0001:00011bc7       ?qt_property@fromBaseDialog@@UAE_NHHPAVQVariant@@@Z 10012bc7 f   moc_frombasedialogimpl.obj
 0001:00011bc7       ?qt_property@testPluginFromBase@@UAE_NHHPAVQVariant@@@Z 10012bc7 f   moc_testPluginFromBase.obj
 0001:00011bc7       ?qt_property@launchEditorDlg@@UAE_NHHPAVQVariant@@@Z 10012bc7 f   moc_launcheditordlgimpl.obj
 0001:00011bc7       ?qt_property@dialog@@UAE_NHHPAVQVariant@@@Z 10012bc7 f   moc_dialogimpl.obj
 0001:00011bc7       ?qt_property@workstationDockWindow@@UAE_NHHPAVQVariant@@@Z 10012bc7 f   moc_workstationdockwindowimpl.obj
 0001:00011bc7       ?qt_property@workstationEditorDlg@@UAE_NHHPAVQVariant@@@Z 10012bc7 f   moc_workstationeditordlgimpl.obj
 0001:00011bd0       ?staticMetaObject@fromBaseDialog@@SAPAVQMetaObject@@XZ 10012bd0 f   moc_frombasedialogimpl.obj
 0001:00011c14       ?className@launchEditor@@UBEPBDXZ 10012c14 f   moc_launchEditor.obj
 0001:00011c1a       ?command@launchEditor@@IAEXVQString@@0@Z 10012c1a f   moc_launchEditor.obj
 0001:00011cda       ?qt_cast@launchEditor@@UAEPAXPBD@Z 10012cda f   moc_launchEditor.obj
 0001:00011d08       ?qt_emit@launchEditor@@UAE_NHPAUQUObject@@@Z 10012d08 f   moc_launchEditor.obj
 0001:00011d6c       ?qt_invoke@launchEditor@@UAE_NHPAUQUObject@@@Z 10012d6c f   moc_launchEditor.obj
 0001:00011db0       ?qt_property@launchEditor@@UAE_NHHPAVQVariant@@@Z 10012db0 f   moc_launchEditor.obj
 0001:00011db0       ?qt_property@workstationEditorDlgBase@@UAE_NHHPAVQVariant@@@Z 10012db0 f   moc_workstationeditordlg.obj
 0001:00011db0       ?qt_property@pluginBase@@UAE_NHHPAVQVariant@@@Z 10012db0 f   pluginBase:moc_pluginBase.obj
 0001:00011db0       ?qt_property@fromBaseDialogBase@@UAE_NHHPAVQVariant@@@Z 10012db0 f   moc_frombasedialog.obj
 0001:00011db0       ?qt_property@testPlugin@@UAE_NHHPAVQVariant@@@Z 10012db0 f   moc_testPlugin.obj
 0001:00011db0       ?qt_property@workstationDockWindowBase@@UAE_NHHPAVQVariant@@@Z 10012db0 f   moc_workstationdockwindow.obj
 0001:00011db0       ?qt_property@launchEditorDlgBase@@UAE_NHHPAVQVariant@@@Z 10012db0 f   moc_launcheditordlg.obj
 0001:00011db0       ?qt_property@workstationEditor@@UAE_NHHPAVQVariant@@@Z 10012db0 f   moc_workstationeditor.obj
 0001:00011db0       ?qt_property@fileManager@@UAE_NHHPAVQVariant@@@Z 10012db0 f   moc_fileManager.obj
 0001:00011db0       ?qt_property@dialogBase@@UAE_NHHPAVQVariant@@@Z 10012db0 f   moc_dialog.obj
 0001:00011dba       ?staticMetaObject@launchEditor@@SAPAVQMetaObject@@XZ 10012dba f   moc_launchEditor.obj
 0001:00011e7f       ?className@launchEditorDlgBase@@UBEPBDXZ 10012e7f f   moc_launcheditordlg.obj
 0001:00011e85       ?qt_cast@launchEditorDlgBase@@UAEPAXPBD@Z 10012e85 f   moc_launcheditordlg.obj
 0001:00011eb3       ?qt_invoke@launchEditorDlgBase@@UAE_NHPAUQUObject@@@Z 10012eb3 f   moc_launcheditordlg.obj
 0001:00011ee5       ?staticMetaObject@launchEditorDlgBase@@SAPAVQMetaObject@@XZ 10012ee5 f   moc_launcheditordlg.obj
 0001:00011f2f       ?tr@launchEditorDlgBase@@SA?AVQString@@PBD0@Z 10012f2f f   moc_launcheditordlg.obj
 0001:00011f72       ?className@launchEditorDlg@@UBEPBDXZ 10012f72 f   moc_launcheditordlgimpl.obj
 0001:00011f78       ?command@launchEditorDlg@@IAEXVQString@@0@Z 10012f78 f   moc_launcheditordlgimpl.obj
 0001:00012038       ?qt_cast@launchEditorDlg@@UAEPAXPBD@Z 10013038 f   moc_launcheditordlgimpl.obj
 0001:00012065       ?qt_emit@launchEditorDlg@@UAE_NHPAUQUObject@@@Z 10013065 f   moc_launcheditordlgimpl.obj
 0001:000120c8       ?qt_invoke@launchEditorDlg@@UAE_NHPAUQUObject@@@Z 100130c8 f   moc_launcheditordlgimpl.obj
 0001:00012170       ?staticMetaObject@launchEditorDlg@@SAPAVQMetaObject@@XZ 10013170 f   moc_launcheditordlgimpl.obj
 0001:0001226c       ?className@testPlugin@@UBEPBDXZ 1001326c f   moc_testPlugin.obj
 0001:00012272       ?command@testPlugin@@IAEXVQString@@0@Z 10013272 f   moc_testPlugin.obj
 0001:00012332       ?qt_cast@testPlugin@@UAEPAXPBD@Z 10013332 f   moc_testPlugin.obj
 0001:00012360       ?qt_emit@testPlugin@@UAE_NHPAUQUObject@@@Z 10013360 f   moc_testPlugin.obj
 0001:000123c4       ?qt_invoke@testPlugin@@UAE_NHPAUQUObject@@@Z 100133c4 f   moc_testPlugin.obj
 0001:000124b0       ?staticMetaObject@testPlugin@@SAPAVQMetaObject@@XZ 100134b0 f   moc_testPlugin.obj
 0001:0001254a       ?className@testPluginFromBase@@UBEPBDXZ 1001354a f   moc_testPluginFromBase.obj
 0001:00012550       ?qt_cast@testPluginFromBase@@UAEPAXPBD@Z 10013550 f   moc_testPluginFromBase.obj
 0001:0001257d       ?qt_emit@testPluginFromBase@@UAE_NHPAUQUObject@@@Z 1001357d f   moc_testPluginFromBase.obj
 0001:00012586       ?qt_invoke@testPluginFromBase@@UAE_NHPAUQUObject@@@Z 10013586 f   moc_testPluginFromBase.obj
 0001:0001267e       ?staticMetaObject@testPluginFromBase@@SAPAVQMetaObject@@XZ 1001367e f   moc_testPluginFromBase.obj
 0001:000126c7       ?className@workstationCustomTable@@UBEPBDXZ 100136c7 f   moc_workstationCustomTable.obj
 0001:000126cd       ?qt_cast@workstationCustomTable@@UAEPAXPBD@Z 100136cd f   moc_workstationCustomTable.obj
 0001:000126fa       ?qt_emit@workstationCustomTable@@UAE_NHPAUQUObject@@@Z 100136fa f   moc_workstationCustomTable.obj
 0001:00012703       ?qt_invoke@workstationCustomTable@@UAE_NHPAUQUObject@@@Z 10013703 f   moc_workstationCustomTable.obj
 0001:00012765       ?qt_property@workstationCustomTable@@UAE_NHHPAVQVariant@@@Z 10013765 f   moc_workstationCustomTable.obj
 0001:0001276e       ?staticMetaObject@workstationCustomTable@@SAPAVQMetaObject@@XZ 1001376e f   moc_workstationCustomTable.obj
 0001:00012880       ?className@workstationDockWindowBase@@UBEPBDXZ 10013880 f   moc_workstationdockwindow.obj
 0001:00012886       ?qt_cast@workstationDockWindowBase@@UAEPAXPBD@Z 10013886 f   moc_workstationdockwindow.obj
 0001:000128b4       ?qt_invoke@workstationDockWindowBase@@UAE_NHPAUQUObject@@@Z 100138b4 f   moc_workstationdockwindow.obj
 0001:000128e6       ?staticMetaObject@workstationDockWindowBase@@SAPAVQMetaObject@@XZ 100138e6 f   moc_workstationdockwindow.obj
 0001:00012930       ?tr@workstationDockWindowBase@@SA?AVQString@@PBD0@Z 10013930 f   moc_workstationdockwindow.obj
 0001:00012973       ?className@workstationDockWindow@@UBEPBDXZ 10013973 f   moc_workstationdockwindowimpl.obj
 0001:00012979       ?qt_cast@workstationDockWindow@@UAEPAXPBD@Z 10013979 f   moc_workstationdockwindowimpl.obj
 0001:000129a6       ?qt_emit@workstationDockWindow@@UAE_NHPAUQUObject@@@Z 100139a6 f   moc_workstationdockwindowimpl.obj
 0001:000129da       ?qt_invoke@workstationDockWindow@@UAE_NHPAUQUObject@@@Z 100139da f   moc_workstationdockwindowimpl.obj
 0001:000129e3       ?selectionChanged@workstationDockWindow@@IAEXPAVQListViewItem@@@Z 100139e3 f   moc_workstationdockwindowimpl.obj
 0001:00012a6e       ?staticMetaObject@workstationDockWindow@@SAPAVQMetaObject@@XZ 10013a6e f   moc_workstationdockwindowimpl.obj
 0001:00012ae7       ?className@workstationEditor@@UBEPBDXZ 10013ae7 f   moc_workstationeditor.obj
 0001:00012aed       ?command@workstationEditor@@IAEXVQString@@0@Z 10013aed f   moc_workstationeditor.obj
 0001:00012bad       ?qt_cast@workstationEditor@@UAEPAXPBD@Z 10013bad f   moc_workstationeditor.obj
 0001:00012bdb       ?qt_emit@workstationEditor@@UAE_NHPAUQUObject@@@Z 10013bdb f   moc_workstationeditor.obj
 0001:00012c3f       ?staticMetaObject@workstationEditor@@SAPAVQMetaObject@@XZ 10013c3f f   moc_workstationeditor.obj
 0001:00012cd4       ?className@workstationEditorDlgBase@@UBEPBDXZ 10013cd4 f   moc_workstationeditordlg.obj
 0001:00012cda       ?qt_cast@workstationEditorDlgBase@@UAEPAXPBD@Z 10013cda f   moc_workstationeditordlg.obj
 0001:00012d08       ?qt_invoke@workstationEditorDlgBase@@UAE_NHPAUQUObject@@@Z 10013d08 f   moc_workstationeditordlg.obj
 0001:00012d3a       ?staticMetaObject@workstationEditorDlgBase@@SAPAVQMetaObject@@XZ 10013d3a f   moc_workstationeditordlg.obj
 0001:00012d84       ?tr@workstationEditorDlgBase@@SA?AVQString@@PBD0@Z 10013d84 f   moc_workstationeditordlg.obj
 0001:00012dc7       ?className@workstationEditorDlg@@UBEPBDXZ 10013dc7 f   moc_workstationeditordlgimpl.obj
 0001:00012dcd       ?command@workstationEditorDlg@@IAEXVQString@@0@Z 10013dcd f   moc_workstationeditordlgimpl.obj
 0001:00012e8d       ?qt_cast@workstationEditorDlg@@UAEPAXPBD@Z 10013e8d f   moc_workstationeditordlgimpl.obj
 0001:00012eba       ?qt_emit@workstationEditorDlg@@UAE_NHPAUQUObject@@@Z 10013eba f   moc_workstationeditordlgimpl.obj
 0001:00012f1d       ?qt_invoke@workstationEditorDlg@@UAE_NHPAUQUObject@@@Z 10013f1d f   moc_workstationeditordlgimpl.obj
 0001:00012f6d       ?staticMetaObject@workstationEditorDlg@@SAPAVQMetaObject@@XZ 10013f6d f   moc_workstationeditordlgimpl.obj
 0001:0001304a       ?className@workstationEditorNewWsDlgBase@@UBEPBDXZ 1001404a f   moc_workstationeditornewwsdlg.obj
 0001:00013050       ?qt_cast@workstationEditorNewWsDlgBase@@UAEPAXPBD@Z 10014050 f   moc_workstationeditornewwsdlg.obj
 0001:0001307e       ?qt_emit@workstationEditorNewWsDlgBase@@UAE_NHPAUQUObject@@@Z 1001407e f   moc_workstationeditornewwsdlg.obj
 0001:00013088       ?qt_invoke@workstationEditorNewWsDlgBase@@UAE_NHPAUQUObject@@@Z 10014088 f   moc_workstationeditornewwsdlg.obj
 0001:000130ba       ?qt_property@workstationEditorNewWsDlgBase@@UAE_NHHPAVQVariant@@@Z 100140ba f   moc_workstationeditornewwsdlg.obj
 0001:000130c4       ?staticMetaObject@workstationEditorNewWsDlgBase@@SAPAVQMetaObject@@XZ 100140c4 f   moc_workstationeditornewwsdlg.obj
 0001:0001310e       ?tr@workstationEditorNewWsDlgBase@@SA?AVQString@@PBD0@Z 1001410e f   moc_workstationeditornewwsdlg.obj
 0001:00013151       ?className@workstationEditorNewWsDlg@@UBEPBDXZ 10014151 f   moc_workstationeditornewwsdlgimpl.obj
 0001:00013157       ?qt_cast@workstationEditorNewWsDlg@@UAEPAXPBD@Z 10014157 f   moc_workstationeditornewwsdlgimpl.obj
 0001:00013184       ?qt_emit@workstationEditorNewWsDlg@@UAE_NHPAUQUObject@@@Z 10014184 f   moc_workstationeditornewwsdlgimpl.obj
 0001:0001318d       ?qt_invoke@workstationEditorNewWsDlg@@UAE_NHPAUQUObject@@@Z 1001418d f   moc_workstationeditornewwsdlgimpl.obj
 0001:00013196       ?qt_property@workstationEditorNewWsDlg@@UAE_NHHPAVQVariant@@@Z 10014196 f   moc_workstationeditornewwsdlgimpl.obj
 0001:0001319f       ?staticMetaObject@workstationEditorNewWsDlg@@SAPAVQMetaObject@@XZ 1001419f f   moc_workstationeditornewwsdlgimpl.obj
 0001:000131e3       ?className@xml_listview@@UBEPBDXZ 100141e3 f   moc_xml_listview.obj
 0001:000131e9       ?qt_cast@xml_listview@@UAEPAXPBD@Z 100141e9 f   moc_xml_listview.obj
 0001:00013217       ?qt_emit@xml_listview@@UAE_NHPAUQUObject@@@Z 10014217 f   moc_xml_listview.obj
 0001:0001324c       ?qt_invoke@xml_listview@@UAE_NHPAUQUObject@@@Z 1001424c f   moc_xml_listview.obj
 0001:00013256       ?qt_property@xml_listview@@UAE_NHHPAVQVariant@@@Z 10014256 f   moc_xml_listview.obj
 0001:00013256       ?qt_property@fileDrop@@UAE_NHHPAVQVariant@@@Z 10014256 f   moc_fileDrop.obj
 0001:00013260       ?startDrag@xml_listview@@IAEXPAVQListViewItem@@@Z 10014260 f   moc_xml_listview.obj
 0001:000132eb       ?staticMetaObject@xml_listview@@SAPAVQMetaObject@@XZ 100142eb f   moc_xml_listview.obj
 0001:00013365       ??0workstationDockWindowBase@@QAE@PAVQWidget@@PBDI@Z 10014365 f   workstationdockwindow.obj
 0001:0001357d       ??1workstationDockWindowBase@@UAE@XZ 1001457d f   workstationdockwindow.obj
 0001:000135bd       ??_EQTabWidget@@WCI@AEPAXI@Z 100145bd f i workstationdockwindow.obj
 0001:000135c5       ??_EworkstationDockWindowBase@@WCI@AEPAXI@Z 100145c5 f i workstationdockwindow.obj
 0001:000135cd       ??_EQTabWidget@@UAEPAXI@Z  100145cd f i workstationdockwindow.obj
 0001:000135cd       ??_GQTabWidget@@UAEPAXI@Z  100145cd f i workstationdockwindow.obj
 0001:000135ed       ??_GworkstationDockWindowBase@@UAEPAXI@Z 100145ed f i workstationdockwindow.obj
 0001:000135ed       ??_EworkstationDockWindowBase@@UAEPAXI@Z 100145ed f i workstationdockwindow.obj
 0001:0001360c       ?languageChange@workstationDockWindowBase@@MAEXXZ 1001460c f   workstationdockwindow.obj
 0001:00013683       ?metaObject@workstationDockWindowBase@@UBEPAVQMetaObject@@XZ 10014683 f i workstationdockwindow.obj
 0001:00013688       ??0workstationEditorDlgBase@@QAE@PAVQWidget@@PBDI@Z 10014688 f   workstationeditordlg.obj
 0001:0001396e       ??1workstationEditorDlgBase@@UAE@XZ 1001496e f   workstationeditordlg.obj
 0001:000139ae       ??_EworkstationEditorDlgBase@@WCI@AEPAXI@Z 100149ae f i workstationeditordlg.obj
 0001:000139b6       ??_EworkstationEditorDlgBase@@UAEPAXI@Z 100149b6 f i workstationeditordlg.obj
 0001:000139b6       ??_GworkstationEditorDlgBase@@UAEPAXI@Z 100149b6 f i workstationeditordlg.obj
 0001:000139d5       ?languageChange@workstationEditorDlgBase@@MAEXXZ 100149d5 f   workstationeditordlg.obj
 0001:00013b6d       ?metaObject@workstationEditorDlgBase@@UBEPAVQMetaObject@@XZ 10014b6d f i workstationeditordlg.obj
 0001:00013b72       ??0workstationEditorNewWsDlgBase@@QAE@PAVQWidget@@PBD_NI@Z 10014b72 f   workstationeditornewwsdlg.obj
 0001:000144f5       ??1workstationEditorNewWsDlgBase@@UAE@XZ 100154f5 f   workstationeditornewwsdlg.obj
 0001:00014508       ??_EQButtonGroup@@WCI@AEPAXI@Z 10015508 f i workstationeditornewwsdlg.obj
 0001:00014510       ??_EQCheckBox@@WCI@AEPAXI@Z 10015510 f i launcheditordlg.obj
 0001:00014510       ??_EQRadioButton@@WCI@AEPAXI@Z 10015510 f i workstationeditornewwsdlg.obj
 0001:00014518       ??_EworkstationEditorNewWsDlgBase@@WCI@AEPAXI@Z 10015518 f i workstationeditornewwsdlg.obj
 0001:00014520       ??_GQButtonGroup@@UAEPAXI@Z 10015520 f i workstationeditornewwsdlg.obj
 0001:00014520       ??_EQButtonGroup@@UAEPAXI@Z 10015520 f i workstationeditornewwsdlg.obj
 0001:00014540       ??_GQCheckBox@@UAEPAXI@Z   10015540 f i launcheditordlg.obj
 0001:00014540       ??_EQCheckBox@@UAEPAXI@Z   10015540 f i launcheditordlg.obj
 0001:00014540       ??_GQRadioButton@@UAEPAXI@Z 10015540 f i workstationeditornewwsdlg.obj
 0001:00014540       ??_EQRadioButton@@UAEPAXI@Z 10015540 f i workstationeditornewwsdlg.obj
 0001:00014560       ??_EworkstationEditorNewWsDlgBase@@UAEPAXI@Z 10015560 f i workstationeditornewwsdlg.obj
 0001:00014560       ??_GworkstationEditorNewWsDlgBase@@UAEPAXI@Z 10015560 f i workstationeditornewwsdlg.obj
 0001:0001457f       ?languageChange@workstationEditorNewWsDlgBase@@MAEXXZ 1001557f f   workstationeditornewwsdlg.obj
 0001:000147da       ?metaObject@workstationEditorNewWsDlgBase@@UBEPAVQMetaObject@@XZ 100157da f i workstationeditornewwsdlg.obj
 0001:000147df       ??0cfg_Table@@QAE@ABV0@@Z  100157df f i cfg_widgets001:moc_cfg_Table.obj
 0001:00014811       ??4cfg_Table@@QAEAAV0@ABV0@@Z 10015811 f i cfg_widgets001:moc_cfg_Table.obj
 0001:00014836       ??_Ecfg_Table@@UAEPAXI@Z   10015836 f i cfg_widgets001:moc_cfg_Table.obj
 0001:00014884       ??_Ecfg_Table@@WCI@AEPAXI@Z 10015884 f i cfg_widgets001:moc_cfg_Table.obj
 0001:0001488c       ??_Fcfg_Table@@QAEXXZ      1001588c f i cfg_widgets001:moc_cfg_Table.obj
 0001:00014896       ?className@cfg_Table@@UBEPBDXZ 10015896 f   cfg_widgets001:moc_cfg_Table.obj
 0001:0001489c       ?clipboardDataValid@cfg_Table@@IAEX_N@Z 1001589c f   cfg_widgets001:moc_cfg_Table.obj
 0001:000148bc       ?dataPasted@cfg_Table@@IAEXXZ 100158bc f   cfg_widgets001:moc_cfg_Table.obj
 0001:000148d1       ?qObject@cfg_Table@@QAEPAVQObject@@XZ 100158d1 f i cfg_widgets001:moc_cfg_Table.obj
 0001:000148d4       ?qt_cast@cfg_Table@@UAEPAXPBD@Z 100158d4 f   cfg_widgets001:moc_cfg_Table.obj
 0001:00014902       ?qt_emit@cfg_Table@@UAE_NHPAUQUObject@@@Z 10015902 f   cfg_widgets001:moc_cfg_Table.obj
 0001:00014946       ?qt_invoke@cfg_Table@@UAE_NHPAUQUObject@@@Z 10015946 f   cfg_widgets001:moc_cfg_Table.obj
 0001:000149a0       ?qt_property@cfg_Table@@UAE_NHHPAVQVariant@@@Z 100159a0 f   cfg_widgets001:moc_cfg_Table.obj
 0001:000149aa       ?qt_static_property@cfg_Table@@SA_NPAVQObject@@HHPAVQVariant@@@Z 100159aa f   cfg_widgets001:moc_cfg_Table.obj
 0001:000149aa       ?isDirty@config_plugin_base@@UAE_NXZ 100159aa f   fileManager.obj
 0001:000149aa       ?validate@config_plugin_base@@UAE_NXZ 100159aa f   fileManager.obj
 0001:000149ad       ?staticMetaObject@cfg_Table@@SAPAVQMetaObject@@XZ 100159ad f   cfg_widgets001:moc_cfg_Table.obj
 0001:00014a2c       ?tr@cfg_Table@@SA?AVQString@@PBD0@Z 10015a2c f   cfg_widgets001:moc_cfg_Table.obj
 0001:00014a6f       ?trUtf8@cfg_Table@@SA?AVQString@@PBD0@Z 10015a6f f   cfg_widgets001:moc_cfg_Table.obj
 0001:00014ab2       ??0cfg_Table@@QAE@PAVQWidget@@PBD@Z 10015ab2 f   cfg_widgets001:cfg_Table.obj
 0001:00014b0c       ??_EQStringList@@QAEPAXI@Z 10015b0c f i cfg_widgets001:cfg_Table.obj
 0001:00014b58       ?clipBoardDataChanged@cfg_Table@@IAEXXZ 10015b58 f   cfg_widgets001:cfg_Table.obj
 0001:00014bac       ?copyToClipboard@cfg_Table@@QAEXXZ 10015bac f   cfg_widgets001:cfg_Table.obj
 0001:00014cbb       ?deleteItems@cfg_Table@@QAEXXZ 10015cbb f   cfg_widgets001:cfg_Table.obj
 0001:00014d47       ?fillUndoBuffer@cfg_Table@@AAEXXZ 10015d47 f   cfg_widgets001:cfg_Table.obj
 0001:00014ebc       ?pasteClipboard@cfg_Table@@QAEXXZ 10015ebc f   cfg_widgets001:cfg_Table.obj
 0001:000152af       ?undoPaste@cfg_Table@@QAEXXZ 100162af f   cfg_widgets001:cfg_Table.obj
 0001:000153e1       ?validateRow@cfg_Table@@MAEHH@Z 100163e1 f   cfg_widgets001:cfg_Table.obj
 0001:000153f4       ?adjustSize@QWidget@@UAEXXZ 100163f4 f   qt-mt323:qt-mt323.dll
 0001:000153fa       ?checkConnectArgs@QObject@@MAE_NPBDPBV1@0@Z 100163fa f   qt-mt323:qt-mt323.dll
 0001:00015400       ?childEvent@QObject@@MAEXPAVQChildEvent@@@Z 10016400 f   qt-mt323:qt-mt323.dll
 0001:00015406       ?close@QWidget@@UAE_N_N@Z  10016406 f   qt-mt323:qt-mt323.dll
 0001:0001540c       ?closeEvent@QWidget@@MAEXPAVQCloseEvent@@@Z 1001640c f   qt-mt323:qt-mt323.dll
 0001:00015412       ?cmd@QPaintDevice@@MAE_NHPAVQPainter@@PATQPDevCmdParam@@@Z 10016412 f   qt-mt323:qt-mt323.dll
 0001:00015418       ?connectNotify@QObject@@MAEXPBD@Z 10016418 f   qt-mt323:qt-mt323.dll
 0001:0001541e       ?contextMenuEvent@QWidget@@MAEXPAVQContextMenuEvent@@@Z 1001641e f   qt-mt323:qt-mt323.dll
 0001:00015424       ?create@QWidget@@MAEXPAUHWND__@@_N1@Z 10016424 f   qt-mt323:qt-mt323.dll
 0001:0001542a       ?customEvent@QObject@@MAEXPAVQCustomEvent@@@Z 1001642a f   qt-mt323:qt-mt323.dll
 0001:00015430       ?customWhatsThis@QWidget@@UBE_NXZ 10016430 f   qt-mt323:qt-mt323.dll
 0001:00015436       ?destroy@QWidget@@MAEX_N0@Z 10016436 f   qt-mt323:qt-mt323.dll
 0001:0001543c       ?disconnectNotify@QObject@@MAEXPBD@Z 1001643c f   qt-mt323:qt-mt323.dll
 0001:00015442       ?dragEnterEvent@QWidget@@MAEXPAVQDragEnterEvent@@@Z 10016442 f   qt-mt323:qt-mt323.dll
 0001:00015448       ?dragLeaveEvent@QWidget@@MAEXPAVQDragLeaveEvent@@@Z 10016448 f   qt-mt323:qt-mt323.dll
 0001:0001544e       ?dragMoveEvent@QWidget@@MAEXPAVQDragMoveEvent@@@Z 1001644e f   qt-mt323:qt-mt323.dll
 0001:00015454       ?dropEvent@QWidget@@MAEXPAVQDropEvent@@@Z 10016454 f   qt-mt323:qt-mt323.dll
 0001:0001545a       ?enabledChange@QWidget@@MAEX_N@Z 1001645a f   qt-mt323:qt-mt323.dll
 0001:00015460       ?enterEvent@QWidget@@MAEXPAVQEvent@@@Z 10016460 f   qt-mt323:qt-mt323.dll
 0001:00015466       ?event@QWidget@@MAE_NPAVQEvent@@@Z 10016466 f   qt-mt323:qt-mt323.dll
 0001:0001546c       ?eventFilter@QObject@@UAE_NPAV1@PAVQEvent@@@Z 1001646c f   qt-mt323:qt-mt323.dll
 0001:00015472       ?focusInEvent@QWidget@@MAEXPAVQFocusEvent@@@Z 10016472 f   qt-mt323:qt-mt323.dll
 0001:00015478       ?focusNextPrevChild@QWidget@@MAE_N_N@Z 10016478 f   qt-mt323:qt-mt323.dll
 0001:0001547e       ?focusOutEvent@QWidget@@MAEXPAVQFocusEvent@@@Z 1001647e f   qt-mt323:qt-mt323.dll
 0001:00015484       ?fontChange@QWidget@@MAEXABVQFont@@@Z 10016484 f   qt-mt323:qt-mt323.dll
 0001:0001548a       ?fontInf@QPaintDevice@@MBEHPAVQFont@@H@Z 1001648a f   qt-mt323:qt-mt323.dll
 0001:00015490       ?fontMet@QPaintDevice@@MBEHPAVQFont@@HPBDH@Z 10016490 f   qt-mt323:qt-mt323.dll
 0001:00015496       ?handle@QPaintDevice@@UBEPAUHDC__@@XZ 10016496 f   qt-mt323:qt-mt323.dll
 0001:0001549c       ?heightForWidth@QWidget@@UBEHH@Z 1001649c f   qt-mt323:qt-mt323.dll
 0001:000154a2       ?hide@QWidget@@UAEXXZ      100164a2 f   qt-mt323:qt-mt323.dll
 0001:000154a8       ?hideEvent@QWidget@@MAEXPAVQHideEvent@@@Z 100164a8 f   qt-mt323:qt-mt323.dll
 0001:000154ae       ?imComposeEvent@QWidget@@MAEXPAVQIMEvent@@@Z 100164ae f   qt-mt323:qt-mt323.dll
 0001:000154b4       ?imEndEvent@QWidget@@MAEXPAVQIMEvent@@@Z 100164b4 f   qt-mt323:qt-mt323.dll
 0001:000154ba       ?imStartEvent@QWidget@@MAEXPAVQIMEvent@@@Z 100164ba f   qt-mt323:qt-mt323.dll
 0001:000154c0       ?insertChild@QObject@@UAEXPAV1@@Z 100164c0 f   qt-mt323:qt-mt323.dll
 0001:000154c6       ?keyPressEvent@QWidget@@MAEXPAVQKeyEvent@@@Z 100164c6 f   qt-mt323:qt-mt323.dll
 0001:000154cc       ?keyReleaseEvent@QWidget@@MAEXPAVQKeyEvent@@@Z 100164cc f   qt-mt323:qt-mt323.dll
 0001:000154d2       ?leaveEvent@QWidget@@MAEXPAVQEvent@@@Z 100164d2 f   qt-mt323:qt-mt323.dll
 0001:000154d8       ?metric@QWidget@@MBEHH@Z   100164d8 f   qt-mt323:qt-mt323.dll
 0001:000154de       ?minimumSizeHint@QWidget@@UBE?AVQSize@@XZ 100164de f   qt-mt323:qt-mt323.dll
 0001:000154e4       ?mouseDoubleClickEvent@QWidget@@MAEXPAVQMouseEvent@@@Z 100164e4 f   qt-mt323:qt-mt323.dll
 0001:000154ea       ?mouseMoveEvent@QWidget@@MAEXPAVQMouseEvent@@@Z 100164ea f   qt-mt323:qt-mt323.dll
 0001:000154f0       ?mousePressEvent@QWidget@@MAEXPAVQMouseEvent@@@Z 100164f0 f   qt-mt323:qt-mt323.dll
 0001:000154f6       ?mouseReleaseEvent@QWidget@@MAEXPAVQMouseEvent@@@Z 100164f6 f   qt-mt323:qt-mt323.dll
 0001:000154fc       ?move@QWidget@@UAEXHH@Z    100164fc f   qt-mt323:qt-mt323.dll
 0001:00015502       ?moveEvent@QWidget@@MAEXPAVQMoveEvent@@@Z 10016502 f   qt-mt323:qt-mt323.dll
 0001:00015508       ?paintEvent@QWidget@@MAEXPAVQPaintEvent@@@Z 10016508 f   qt-mt323:qt-mt323.dll
 0001:0001550e       ?paletteChange@QWidget@@MAEXABVQPalette@@@Z 1001650e f   qt-mt323:qt-mt323.dll
 0001:00015514       ?polish@QWidget@@UAEXXZ    10016514 f   qt-mt323:qt-mt323.dll
 0001:0001551a       ?property@QObject@@UBE?AVQVariant@@PBD@Z 1001651a f   qt-mt323:qt-mt323.dll
 0001:00015520       ?removeChild@QObject@@UAEXPAV1@@Z 10016520 f   qt-mt323:qt-mt323.dll
 0001:00015526       ?reparent@QWidget@@UAEXPAV1@IABVQPoint@@_N@Z 10016526 f   qt-mt323:qt-mt323.dll
 0001:0001552c       ?resize@QWidget@@UAEXHH@Z  1001652c f   qt-mt323:qt-mt323.dll
 0001:00015532       ?resizeEvent@QWidget@@MAEXPAVQResizeEvent@@@Z 10016532 f   qt-mt323:qt-mt323.dll
 0001:00015538       ?resolution@QPaintDevice@@UBEHXZ 10016538 f   qt-mt323:qt-mt323.dll
 0001:0001553e       ?setAcceptDrops@QWidget@@UAEX_N@Z 1001653e f   qt-mt323:qt-mt323.dll
 0001:00015544       ?setActiveWindow@QWidget@@UAEXXZ 10016544 f   qt-mt323:qt-mt323.dll
 0001:0001554a       ?setAutoMask@QWidget@@UAEX_N@Z 1001654a f   qt-mt323:qt-mt323.dll
 0001:00015550       ?setBackgroundColor@QWidget@@UAEXABVQColor@@@Z 10016550 f   qt-mt323:qt-mt323.dll
 0001:00015556       ?setBackgroundMode@QWidget@@UAEXW4BackgroundMode@Qt@@@Z 10016556 f   qt-mt323:qt-mt323.dll
 0001:0001555c       ?setBackgroundOrigin@QWidget@@UAEXW4BackgroundOrigin@1@@Z 1001655c f   qt-mt323:qt-mt323.dll
 0001:00015562       ?setBackgroundPixmap@QWidget@@UAEXABVQPixmap@@@Z 10016562 f   qt-mt323:qt-mt323.dll
 0001:00015568       ?setCaption@QWidget@@UAEXABVQString@@@Z 10016568 f   qt-mt323:qt-mt323.dll
 0001:0001556e       ?setCursor@QWidget@@UAEXABVQCursor@@@Z 1001656e f   qt-mt323:qt-mt323.dll
 0001:00015574       ?setEnabled@QWidget@@UAEX_N@Z 10016574 f   qt-mt323:qt-mt323.dll
 0001:0001557a       ?setEraseColor@QWidget@@UAEXABVQColor@@@Z 1001657a f   qt-mt323:qt-mt323.dll
 0001:00015580       ?setErasePixmap@QWidget@@UAEXABVQPixmap@@@Z 10016580 f   qt-mt323:qt-mt323.dll
 0001:00015586       ?setFocus@QWidget@@UAEXXZ  10016586 f   qt-mt323:qt-mt323.dll
 0001:0001558c       ?setFocusPolicy@QWidget@@UAEXW4FocusPolicy@1@@Z 1001658c f   qt-mt323:qt-mt323.dll
 0001:00015592       ?setFocusProxy@QWidget@@UAEXPAV1@@Z 10016592 f   qt-mt323:qt-mt323.dll
 0001:00015598       ?setFont@QWidget@@UAEXABVQFont@@@Z 10016598 f   qt-mt323:qt-mt323.dll
 0001:0001559e       ?setGeometry@QWidget@@UAEXABVQRect@@@Z 1001659e f   qt-mt323:qt-mt323.dll
 0001:000155a4       ?setGeometry@QWidget@@UAEXHHHH@Z 100165a4 f   qt-mt323:qt-mt323.dll
 0001:000155aa       ?setIcon@QWidget@@UAEXABVQPixmap@@@Z 100165aa f   qt-mt323:qt-mt323.dll
 0001:000155b0       ?setIconText@QWidget@@UAEXABVQString@@@Z 100165b0 f   qt-mt323:qt-mt323.dll
 0001:000155b6       ?setKeyCompression@QWidget@@MAEX_N@Z 100165b6 f   qt-mt323:qt-mt323.dll
 0001:000155bc       ?setMask@QWidget@@UAEXABVQBitmap@@@Z 100165bc f   qt-mt323:qt-mt323.dll
 0001:000155c2       ?setMask@QWidget@@UAEXABVQRegion@@@Z 100165c2 f   qt-mt323:qt-mt323.dll
 0001:000155c8       ?setMaximumSize@QWidget@@UAEXHH@Z 100165c8 f   qt-mt323:qt-mt323.dll
 0001:000155ce       ?setMicroFocusHint@QWidget@@MAEXHHHH_NPAVQFont@@@Z 100165ce f   qt-mt323:qt-mt323.dll
 0001:000155d4       ?setMinimumSize@QWidget@@UAEXHH@Z 100165d4 f   qt-mt323:qt-mt323.dll
 0001:000155da       ?setMouseTracking@QWidget@@UAEX_N@Z 100165da f   qt-mt323:qt-mt323.dll
 0001:000155e0       ?setName@QWidget@@UAEXPBD@Z 100165e0 f   qt-mt323:qt-mt323.dll
 0001:000155e6       ?setPalette@QWidget@@UAEXABVQPalette@@@Z 100165e6 f   qt-mt323:qt-mt323.dll
 0001:000155ec       ?setPaletteBackgroundColor@QWidget@@UAEXABVQColor@@@Z 100165ec f   qt-mt323:qt-mt323.dll
 0001:000155f2       ?setPaletteBackgroundPixmap@QWidget@@UAEXABVQPixmap@@@Z 100165f2 f   qt-mt323:qt-mt323.dll
 0001:000155f8       ?setProperty@QObject@@UAE_NPBDABVQVariant@@@Z 100165f8 f   qt-mt323:qt-mt323.dll
 0001:000155fe       ?setResolution@QPaintDevice@@UAEXH@Z 100165fe f   qt-mt323:qt-mt323.dll
 0001:00015604       ?setSizeIncrement@QWidget@@UAEXHH@Z 10016604 f   qt-mt323:qt-mt323.dll
 0001:0001560a       ?setSizePolicy@QWidget@@UAEXVQSizePolicy@@@Z 1001660a f   qt-mt323:qt-mt323.dll
 0001:00015610       ?setUpdatesEnabled@QWidget@@UAEX_N@Z 10016610 f   qt-mt323:qt-mt323.dll
 0001:00015616       ?setWFlags@QWidget@@MAEXI@Z 10016616 f   qt-mt323:qt-mt323.dll
 0001:0001561c       ?setWState@QWidget@@MAEXI@Z 1001661c f   qt-mt323:qt-mt323.dll
 0001:00015622       ?show@QWidget@@UAEXXZ      10016622 f   qt-mt323:qt-mt323.dll
 0001:00015628       ?showEvent@QWidget@@MAEXPAVQShowEvent@@@Z 10016628 f   qt-mt323:qt-mt323.dll
 0001:0001562e       ?showMaximized@QWidget@@UAEXXZ 1001662e f   qt-mt323:qt-mt323.dll
 0001:00015634       ?showMinimized@QWidget@@UAEXXZ 10016634 f   qt-mt323:qt-mt323.dll
 0001:0001563a       ?showNormal@QWidget@@UAEXXZ 1001663a f   qt-mt323:qt-mt323.dll
 0001:00015640       ?sizeHint@QWidget@@UBE?AVQSize@@XZ 10016640 f   qt-mt323:qt-mt323.dll
 0001:00015646       ?sizePolicy@QWidget@@UBE?AVQSizePolicy@@XZ 10016646 f   qt-mt323:qt-mt323.dll
 0001:0001564c       ?styleChange@QWidget@@MAEXAAVQStyle@@@Z 1001664c f   qt-mt323:qt-mt323.dll
 0001:00015652       ?tabletEvent@QWidget@@MAEXPAVQTabletEvent@@@Z 10016652 f   qt-mt323:qt-mt323.dll
 0001:00015658       ?timerEvent@QObject@@MAEXPAVQTimerEvent@@@Z 10016658 f   qt-mt323:qt-mt323.dll
 0001:0001565e       ?unsetCursor@QWidget@@UAEXXZ 1001665e f   qt-mt323:qt-mt323.dll
 0001:00015664       ?updateMask@QWidget@@MAEXXZ 10016664 f   qt-mt323:qt-mt323.dll
 0001:0001566a       ?wheelEvent@QWidget@@MAEXPAVQWheelEvent@@@Z 1001666a f   qt-mt323:qt-mt323.dll
 0001:00015670       ?winEvent@QWidget@@MAE_NPAUtagMSG@@@Z 10016670 f   qt-mt323:qt-mt323.dll
 0001:00015676       ?windowActivationChange@QWidget@@MAEX_N@Z 10016676 f   qt-mt323:qt-mt323.dll
 0001:0001567c       ?addChild@QScrollView@@UAEXPAVQWidget@@HH@Z 1001667c f   qt-mt323:qt-mt323.dll
 0001:00015682       ?addColumn@QListView@@UAEHABVQIconSet@@ABVQString@@H@Z 10016682 f   qt-mt323:qt-mt323.dll
 0001:00015688       ?addColumn@QListView@@UAEHABVQString@@H@Z 10016688 f   qt-mt323:qt-mt323.dll
 0001:0001568e       ?clear@QListView@@UAEXXZ   1001668e f   qt-mt323:qt-mt323.dll
 0001:00015694       ?clearSelection@QListView@@UAEXXZ 10016694 f   qt-mt323:qt-mt323.dll
 0001:0001569a       ?contentsContextMenuEvent@QListView@@MAEXPAVQContextMenuEvent@@@Z 1001669a f   qt-mt323:qt-mt323.dll
 0001:000156a0       ?contentsDragEnterEvent@QListView@@MAEXPAVQDragEnterEvent@@@Z 100166a0 f   qt-mt323:qt-mt323.dll
 0001:000156a6       ?contentsDragLeaveEvent@QListView@@MAEXPAVQDragLeaveEvent@@@Z 100166a6 f   qt-mt323:qt-mt323.dll
 0001:000156ac       ?contentsDragMoveEvent@QListView@@MAEXPAVQDragMoveEvent@@@Z 100166ac f   qt-mt323:qt-mt323.dll
 0001:000156b2       ?contentsDropEvent@QListView@@MAEXPAVQDropEvent@@@Z 100166b2 f   qt-mt323:qt-mt323.dll
 0001:000156b8       ?contentsMouseDoubleClickEvent@QListView@@MAEXPAVQMouseEvent@@@Z 100166b8 f   qt-mt323:qt-mt323.dll
 0001:000156be       ?contentsMouseMoveEvent@QListView@@MAEXPAVQMouseEvent@@@Z 100166be f   qt-mt323:qt-mt323.dll
 0001:000156c4       ?contentsMousePressEvent@QListView@@MAEXPAVQMouseEvent@@@Z 100166c4 f   qt-mt323:qt-mt323.dll
 0001:000156ca       ?contentsMouseReleaseEvent@QListView@@MAEXPAVQMouseEvent@@@Z 100166ca f   qt-mt323:qt-mt323.dll
 0001:000156d0       ?contentsWheelEvent@QScrollView@@MAEXPAVQWheelEvent@@@Z 100166d0 f   qt-mt323:qt-mt323.dll
 0001:000156d6       ?dragObject@QListView@@MAEPAVQDragObject@@XZ 100166d6 f   qt-mt323:qt-mt323.dll
 0001:000156dc       ?drawContents@QScrollView@@EAEXPAVQPainter@@@Z 100166dc f   qt-mt323:qt-mt323.dll
 0001:000156e2       ?drawContents@QScrollView@@MAEXPAVQPainter@@HHHH@Z 100166e2 f   qt-mt323:qt-mt323.dll
 0001:000156e8       ?drawContentsOffset@QListView@@MAEXPAVQPainter@@HHHHHH@Z 100166e8 f   qt-mt323:qt-mt323.dll
 0001:000156ee       ?drawFrame@QFrame@@MAEXPAVQPainter@@@Z 100166ee f   qt-mt323:qt-mt323.dll
 0001:000156f4       ?eventFilter@QListView@@UAE_NPAVQObject@@PAVQEvent@@@Z 100166f4 f   qt-mt323:qt-mt323.dll
 0001:000156fa       ?focusInEvent@QListView@@MAEXPAVQFocusEvent@@@Z 100166fa f   qt-mt323:qt-mt323.dll
 0001:00015700       ?focusNextPrevChild@QScrollView@@MAE_N_N@Z 10016700 f   qt-mt323:qt-mt323.dll
 0001:00015706       ?focusOutEvent@QListView@@MAEXPAVQFocusEvent@@@Z 10016706 f   qt-mt323:qt-mt323.dll
 0001:0001570c       ?fontChange@QScrollView@@MAEXABVQFont@@@Z 1001670c f   qt-mt323:qt-mt323.dll
 0001:00015712       ?frameChanged@QScrollView@@MAEXXZ 10016712 f   qt-mt323:qt-mt323.dll
 0001:00015718       ?insertItem@QListView@@UAEXPAVQListViewItem@@@Z 10016718 f   qt-mt323:qt-mt323.dll
 0001:0001571e       ?invertSelection@QListView@@UAEXXZ 1001671e f   qt-mt323:qt-mt323.dll
 0001:00015724       ?keyPressEvent@QListView@@MAEXPAVQKeyEvent@@@Z 10016724 f   qt-mt323:qt-mt323.dll
 0001:0001572a       ?minimumSizeHint@QListView@@UBE?AVQSize@@XZ 1001672a f   qt-mt323:qt-mt323.dll
 0001:00015730       ?mouseDoubleClickEvent@QScrollView@@MAEXPAVQMouseEvent@@@Z 10016730 f   qt-mt323:qt-mt323.dll
 0001:00015736       ?mouseMoveEvent@QScrollView@@MAEXPAVQMouseEvent@@@Z 10016736 f   qt-mt323:qt-mt323.dll
 0001:0001573c       ?mousePressEvent@QScrollView@@MAEXPAVQMouseEvent@@@Z 1001673c f   qt-mt323:qt-mt323.dll
 0001:00015742       ?mouseReleaseEvent@QScrollView@@MAEXPAVQMouseEvent@@@Z 10016742 f   qt-mt323:qt-mt323.dll
 0001:00015748       ?moveChild@QScrollView@@UAEXPAVQWidget@@HH@Z 10016748 f   qt-mt323:qt-mt323.dll
 0001:0001574e       ?paintEmptyArea@QListView@@MAEXPAVQPainter@@ABVQRect@@@Z 1001674e f   qt-mt323:qt-mt323.dll
 0001:00015754       ?paintEvent@QFrame@@MAEXPAVQPaintEvent@@@Z 10016754 f   qt-mt323:qt-mt323.dll
 0001:0001575a       ?removeChild@QScrollView@@UAEXPAVQObject@@@Z 1001675a f   qt-mt323:qt-mt323.dll
 0001:00015760       ?removeColumn@QListView@@UAEXH@Z 10016760 f   qt-mt323:qt-mt323.dll
 0001:00015766       ?removeItem@QListView@@UAEXPAVQListViewItem@@@Z 10016766 f   qt-mt323:qt-mt323.dll
 0001:0001576c       ?resize@QScrollView@@UAEXHH@Z 1001676c f   qt-mt323:qt-mt323.dll
 0001:00015772       ?resizeContents@QScrollView@@UAEXHH@Z 10016772 f   qt-mt323:qt-mt323.dll
 0001:00015778       ?resizeEvent@QListView@@MAEXPAVQResizeEvent@@@Z 10016778 f   qt-mt323:qt-mt323.dll
 0001:0001577e       ?selectAll@QListView@@UAEX_N@Z 1001677e f   qt-mt323:qt-mt323.dll
 0001:00015784       ?setAllColumnsShowFocus@QListView@@UAEX_N@Z 10016784 f   qt-mt323:qt-mt323.dll
 0001:0001578a       ?setColumnAlignment@QListView@@UAEXHH@Z 1001678a f   qt-mt323:qt-mt323.dll
 0001:00015790       ?setColumnText@QListView@@UAEXHABVQIconSet@@ABVQString@@@Z 10016790 f   qt-mt323:qt-mt323.dll
 0001:00015796       ?setColumnText@QListView@@UAEXHABVQString@@@Z 10016796 f   qt-mt323:qt-mt323.dll
 0001:0001579c       ?setColumnWidth@QListView@@UAEXHH@Z 1001679c f   qt-mt323:qt-mt323.dll
 0001:000157a2       ?setColumnWidthMode@QListView@@UAEXHW4WidthMode@1@@Z 100167a2 f   qt-mt323:qt-mt323.dll
 0001:000157a8       ?setContentsPos@QListView@@UAEXHH@Z 100167a8 f   qt-mt323:qt-mt323.dll
 0001:000157ae       ?setCornerWidget@QScrollView@@UAEXPAVQWidget@@@Z 100167ae f   qt-mt323:qt-mt323.dll
 0001:000157b4       ?setCurrentItem@QListView@@UAEXPAVQListViewItem@@@Z 100167b4 f   qt-mt323:qt-mt323.dll
 0001:000157ba       ?setDefaultRenameAction@QListView@@UAEXW4RenameAction@1@@Z 100167ba f   qt-mt323:qt-mt323.dll
 0001:000157c0       ?setDragAutoScroll@QScrollView@@UAEX_N@Z 100167c0 f   qt-mt323:qt-mt323.dll
 0001:000157c6       ?setEnabled@QScrollView@@UAEX_N@Z 100167c6 f   qt-mt323:qt-mt323.dll
 0001:000157cc       ?setFont@QListView@@UAEXABVQFont@@@Z 100167cc f   qt-mt323:qt-mt323.dll
 0001:000157d2       ?setFrameRect@QFrame@@UAEXABVQRect@@@Z 100167d2 f   qt-mt323:qt-mt323.dll
 0001:000157d8       ?setFrameStyle@QFrame@@UAEXH@Z 100167d8 f   qt-mt323:qt-mt323.dll
 0001:000157de       ?setHBarGeometry@QScrollView@@MAEXAAVQScrollBar@@HHHH@Z 100167de f   qt-mt323:qt-mt323.dll
 0001:000157e4       ?setHScrollBarMode@QScrollView@@UAEXW4ScrollBarMode@1@@Z 100167e4 f   qt-mt323:qt-mt323.dll
 0001:000157ea       ?setItemMargin@QListView@@UAEXH@Z 100167ea f   qt-mt323:qt-mt323.dll
 0001:000157f0       ?setLineWidth@QFrame@@UAEXH@Z 100167f0 f   qt-mt323:qt-mt323.dll
 0001:000157f6       ?setMargin@QFrame@@UAEXH@Z 100167f6 f   qt-mt323:qt-mt323.dll
 0001:000157fc       ?setMargins@QScrollView@@MAEXHHHH@Z 100167fc f   qt-mt323:qt-mt323.dll
 0001:00015802       ?setMidLineWidth@QFrame@@UAEXH@Z 10016802 f   qt-mt323:qt-mt323.dll
 0001:00015808       ?setMultiSelection@QListView@@UAEX_N@Z 10016808 f   qt-mt323:qt-mt323.dll
 0001:0001580e       ?setOpen@QListView@@UAEXPAVQListViewItem@@_N@Z 1001680e f   qt-mt323:qt-mt323.dll
 0001:00015814       ?setPalette@QListView@@UAEXABVQPalette@@@Z 10016814 f   qt-mt323:qt-mt323.dll
 0001:0001581a       ?setResizeMode@QListView@@UAEXW4ResizeMode@1@@Z 1001681a f   qt-mt323:qt-mt323.dll
 0001:00015820       ?setResizePolicy@QScrollView@@UAEXW4ResizePolicy@1@@Z 10016820 f   qt-mt323:qt-mt323.dll
 0001:00015826       ?setRootIsDecorated@QListView@@UAEX_N@Z 10016826 f   qt-mt323:qt-mt323.dll
 0001:0001582c       ?setSelected@QListView@@UAEXPAVQListViewItem@@_N@Z 1001682c f   qt-mt323:qt-mt323.dll
 0001:00015832       ?setShowSortIndicator@QListView@@UAEX_N@Z 10016832 f   qt-mt323:qt-mt323.dll
 0001:00015838       ?setShowToolTips@QListView@@UAEX_N@Z 10016838 f   qt-mt323:qt-mt323.dll
 0001:0001583e       ?setSorting@QListView@@UAEXH_N@Z 1001683e f   qt-mt323:qt-mt323.dll
 0001:00015844       ?setTreeStepSize@QListView@@UAEXH@Z 10016844 f   qt-mt323:qt-mt323.dll
 0001:0001584a       ?setVBarGeometry@QScrollView@@MAEXAAVQScrollBar@@HHHH@Z 1001684a f   qt-mt323:qt-mt323.dll
 0001:00015850       ?setVScrollBarMode@QScrollView@@UAEXW4ScrollBarMode@1@@Z 10016850 f   qt-mt323:qt-mt323.dll
 0001:00015856       ?show@QListView@@UAEXXZ    10016856 f   qt-mt323:qt-mt323.dll
 0001:0001585c       ?showEvent@QListView@@MAEXPAVQShowEvent@@@Z 1001685c f   qt-mt323:qt-mt323.dll
 0001:00015862       ?sizeHint@QListView@@UBE?AVQSize@@XZ 10016862 f   qt-mt323:qt-mt323.dll
 0001:00015868       ?sort@QListView@@UAEXXZ    10016868 f   qt-mt323:qt-mt323.dll
 0001:0001586e       ?startDrag@QListView@@MAEXXZ 1001686e f   qt-mt323:qt-mt323.dll
 0001:00015874       ?styleChange@QListView@@MAEXAAVQStyle@@@Z 10016874 f   qt-mt323:qt-mt323.dll
 0001:0001587a       ?takeItem@QListView@@UAEXPAVQListViewItem@@@Z 1001687a f   qt-mt323:qt-mt323.dll
 0001:00015880       ?viewportContextMenuEvent@QScrollView@@MAEXPAVQContextMenuEvent@@@Z 10016880 f   qt-mt323:qt-mt323.dll
 0001:00015886       ?viewportDragEnterEvent@QScrollView@@MAEXPAVQDragEnterEvent@@@Z 10016886 f   qt-mt323:qt-mt323.dll
 0001:0001588c       ?viewportDragLeaveEvent@QScrollView@@MAEXPAVQDragLeaveEvent@@@Z 1001688c f   qt-mt323:qt-mt323.dll
 0001:00015892       ?viewportDragMoveEvent@QScrollView@@MAEXPAVQDragMoveEvent@@@Z 10016892 f   qt-mt323:qt-mt323.dll
 0001:00015898       ?viewportDropEvent@QScrollView@@MAEXPAVQDropEvent@@@Z 10016898 f   qt-mt323:qt-mt323.dll
 0001:0001589e       ?viewportMouseDoubleClickEvent@QScrollView@@MAEXPAVQMouseEvent@@@Z 1001689e f   qt-mt323:qt-mt323.dll
 0001:000158a4       ?viewportMouseMoveEvent@QScrollView@@MAEXPAVQMouseEvent@@@Z 100168a4 f   qt-mt323:qt-mt323.dll
 0001:000158aa       ?viewportMousePressEvent@QScrollView@@MAEXPAVQMouseEvent@@@Z 100168aa f   qt-mt323:qt-mt323.dll
 0001:000158b0       ?viewportMouseReleaseEvent@QScrollView@@MAEXPAVQMouseEvent@@@Z 100168b0 f   qt-mt323:qt-mt323.dll
 0001:000158b6       ?viewportPaintEvent@QScrollView@@MAEXPAVQPaintEvent@@@Z 100168b6 f   qt-mt323:qt-mt323.dll
 0001:000158bc       ?viewportResizeEvent@QListView@@MAEXPAVQResizeEvent@@@Z 100168bc f   qt-mt323:qt-mt323.dll
 0001:000158c2       ?viewportWheelEvent@QScrollView@@MAEXPAVQWheelEvent@@@Z 100168c2 f   qt-mt323:qt-mt323.dll
 0001:000158c8       ?wheelEvent@QScrollView@@MAEXPAVQWheelEvent@@@Z 100168c8 f   qt-mt323:qt-mt323.dll
 0001:000158ce       ?windowActivationChange@QListView@@MAEX_N@Z 100168ce f   qt-mt323:qt-mt323.dll
 0001:000158d4       ?acceptDrop@QListViewItem@@UBE_NPBVQMimeSource@@@Z 100168d4 f   qt-mt323:qt-mt323.dll
 0001:000158da       ?activate@QListViewItem@@MAEXXZ 100168da f   qt-mt323:qt-mt323.dll
 0001:000158e0       ?addItem@QBoxLayout@@UAEXPAVQLayoutItem@@@Z 100168e0 f   qt-mt323:qt-mt323.dll
 0001:000158e6       ?cancelRename@QListViewItem@@MAEXH@Z 100168e6 f   qt-mt323:qt-mt323.dll
 0001:000158ec       ?childEvent@QLayout@@MAEXPAVQChildEvent@@@Z 100168ec f   qt-mt323:qt-mt323.dll
 0001:000158f2       ?childEvent@QSplitter@@MAEXPAVQChildEvent@@@Z 100168f2 f   qt-mt323:qt-mt323.dll
 0001:000158f8       ?className@QGuardedPtrPrivate@@UBEPBDXZ 100168f8 f   qt-mt323:qt-mt323.dll
 0001:000158fe       ?className@QLabel@@UBEPBDXZ 100168fe f   qt-mt323:qt-mt323.dll
 0001:00015904       ?className@QListView@@UBEPBDXZ 10016904 f   qt-mt323:qt-mt323.dll
 0001:0001590a       ?className@QSplitter@@UBEPBDXZ 1001690a f   qt-mt323:qt-mt323.dll
 0001:00015910       ?className@QVBoxLayout@@UBEPBDXZ 10016910 f   qt-mt323:qt-mt323.dll
 0001:00015916       ?className@QWidget@@UBEPBDXZ 10016916 f   qt-mt323:qt-mt323.dll
 0001:0001591c       ?clear@?$QPtrList@VQDockWindow@@@@UAEXXZ 1001691c f   qt-mt323:qt-mt323.dll
 0001:00015922       ?compare@QListViewItem@@UBEHPAV1@H_N@Z 10016922 f   qt-mt323:qt-mt323.dll
 0001:00015928       ?compareItems@QGList@@MAEHPAX0@Z 10016928 f   qt-mt323:qt-mt323.dll
 0001:0001592e       ?contextMenuEvent@QScrollView@@MAEXPAVQContextMenuEvent@@@Z 1001692e f   qt-mt323:qt-mt323.dll
 0001:00015934       ?count@?$QPtrList@VQDockWindow@@@@UBEIXZ 10016934 f   qt-mt323:qt-mt323.dll
 0001:0001593a       ?deleteItem@?$QPtrList@VQDockWindow@@@@EAEXPAX@Z 1001693a f   qt-mt323:qt-mt323.dll
 0001:00015940       ?dragEntered@QListViewItem@@MAEXXZ 10016940 f   qt-mt323:qt-mt323.dll
 0001:00015946       ?dragLeft@QListViewItem@@MAEXXZ 10016946 f   qt-mt323:qt-mt323.dll
 0001:0001594c       ?drawContents@QFrame@@MAEXPAVQPainter@@@Z 1001694c f   qt-mt323:qt-mt323.dll
 0001:00015952       ?drawContents@QLabel@@MAEXPAVQPainter@@@Z 10016952 f   qt-mt323:qt-mt323.dll
 0001:00015958       ?drawSplitter@QSplitter@@MAEXPAVQPainter@@HHHH@Z 10016958 f   qt-mt323:qt-mt323.dll
 0001:0001595e       ?dropped@QListViewItem@@MAEXPAVQDropEvent@@@Z 1001695e f   qt-mt323:qt-mt323.dll
 0001:00015964       ?enforceSortOrder@QListViewItem@@MBEXXZ 10016964 f   qt-mt323:qt-mt323.dll
 0001:0001596a       ?event@QObject@@UAE_NPAVQEvent@@@Z 1001696a f   qt-mt323:qt-mt323.dll
 0001:00015970       ?event@QSplitter@@MAE_NPAVQEvent@@@Z 10016970 f   qt-mt323:qt-mt323.dll
 0001:00015976       ?eventFilter@QLayout@@MAE_NPAVQObject@@PAVQEvent@@@Z 10016976 f   qt-mt323:qt-mt323.dll
 0001:0001597c       ?expanding@QBoxLayout@@UBE?AW4ExpandData@QSizePolicy@@XZ 1001697c f   qt-mt323:qt-mt323.dll
 0001:00015982       ?fontChange@QLabel@@MAEXABVQFont@@@Z 10016982 f   qt-mt323:qt-mt323.dll
 0001:00015988       ?frameChanged@QFrame@@MAEXXZ 10016988 f   qt-mt323:qt-mt323.dll
 0001:0001598e       ?geometry@QLayout@@UBE?AVQRect@@XZ 1001698e f   qt-mt323:qt-mt323.dll
 0001:00015994       ?hasHeightForWidth@QBoxLayout@@UBE_NXZ 10016994 f   qt-mt323:qt-mt323.dll
 0001:0001599a       ?heightForWidth@QBoxLayout@@UBEHH@Z 1001699a f   qt-mt323:qt-mt323.dll
 0001:000159a0       ?heightForWidth@QLabel@@UBEHH@Z 100169a0 f   qt-mt323:qt-mt323.dll
 0001:000159a6       ?insertItem@QListViewItem@@UAEXPAV1@@Z 100169a6 f   qt-mt323:qt-mt323.dll
 0001:000159ac       ?invalidate@QBoxLayout@@UAEXXZ 100169ac f   qt-mt323:qt-mt323.dll
 0001:000159b2       ?invalidateHeight@QListViewItem@@UAEXXZ 100169b2 f   qt-mt323:qt-mt323.dll
 0001:000159b8       ?isEmpty@QLayout@@UBE_NXZ  100169b8 f   qt-mt323:qt-mt323.dll
 0001:000159be       ?iterator@QBoxLayout@@UAE?AVQLayoutIterator@@XZ 100169be f   qt-mt323:qt-mt323.dll
 0001:000159c4       ?key@QListViewItem@@UBE?AVQString@@H_N@Z 100169c4 f   qt-mt323:qt-mt323.dll
 0001:000159ca       ?layout@QLayout@@UAEPAV1@XZ 100169ca f   qt-mt323:qt-mt323.dll
 0001:000159d0       ?maximumSize@QBoxLayout@@UBE?AVQSize@@XZ 100169d0 f   qt-mt323:qt-mt323.dll
 0001:000159d6       ?metaObject@QGuardedPtrPrivate@@UBEPAVQMetaObject@@XZ 100169d6 f   qt-mt323:qt-mt323.dll
 0001:000159dc       ?metaObject@QLabel@@UBEPAVQMetaObject@@XZ 100169dc f   qt-mt323:qt-mt323.dll
 0001:000159e2       ?metaObject@QListView@@UBEPAVQMetaObject@@XZ 100169e2 f   qt-mt323:qt-mt323.dll
 0001:000159e8       ?metaObject@QSplitter@@UBEPAVQMetaObject@@XZ 100169e8 f   qt-mt323:qt-mt323.dll
 0001:000159ee       ?metaObject@QVBoxLayout@@UBEPAVQMetaObject@@XZ 100169ee f   qt-mt323:qt-mt323.dll
 0001:000159f4       ?metaObject@QWidget@@UBEPAVQMetaObject@@XZ 100169f4 f   qt-mt323:qt-mt323.dll
 0001:000159fa       ?minimumSize@QBoxLayout@@UBE?AVQSize@@XZ 100169fa f   qt-mt323:qt-mt323.dll
 0001:00015a00       ?minimumSizeHint@QLabel@@UBE?AVQSize@@XZ 10016a00 f   qt-mt323:qt-mt323.dll
 0001:00015a06       ?minimumSizeHint@QSplitter@@UBE?AVQSize@@XZ 10016a06 f   qt-mt323:qt-mt323.dll
 0001:00015a0c       ?newItem@QPtrCollection@@MAEPAXPAX@Z 10016a0c f   qt-mt323:qt-mt323.dll
 0001:00015a12       ?okRename@QListViewItem@@MAEXH@Z 10016a12 f   qt-mt323:qt-mt323.dll
 0001:00015a18       ?paintBranches@QListViewItem@@UAEXPAVQPainter@@ABVQColorGroup@@HHH@Z 10016a18 f   qt-mt323:qt-mt323.dll
 0001:00015a1e       ?paintCell@QListViewItem@@UAEXPAVQPainter@@ABVQColorGroup@@HHH@Z 10016a1e f   qt-mt323:qt-mt323.dll
 0001:00015a24       ?paintFocus@QListViewItem@@UAEXPAVQPainter@@ABVQColorGroup@@ABVQRect@@@Z 10016a24 f   qt-mt323:qt-mt323.dll
 0001:00015a2a       ?pixmap@QListViewItem@@UBEPBVQPixmap@@H@Z 10016a2a f   qt-mt323:qt-mt323.dll
 0001:00015a30       ?qt_cast@QGuardedPtrPrivate@@UAEPAXPBD@Z 10016a30 f   qt-mt323:qt-mt323.dll
 0001:00015a36       ?qt_cast@QLabel@@UAEPAXPBD@Z 10016a36 f   qt-mt323:qt-mt323.dll
 0001:00015a3c       ?qt_cast@QListView@@UAEPAXPBD@Z 10016a3c f   qt-mt323:qt-mt323.dll
 0001:00015a42       ?qt_cast@QSplitter@@UAEPAXPBD@Z 10016a42 f   qt-mt323:qt-mt323.dll
 0001:00015a48       ?qt_cast@QVBoxLayout@@UAEPAXPBD@Z 10016a48 f   qt-mt323:qt-mt323.dll
 0001:00015a4e       ?qt_cast@QWidget@@UAEPAXPBD@Z 10016a4e f   qt-mt323:qt-mt323.dll
 0001:00015a54       ?qt_emit@QGuardedPtrPrivate@@UAE_NHPAUQUObject@@@Z 10016a54 f   qt-mt323:qt-mt323.dll
 0001:00015a5a       ?qt_emit@QLabel@@UAE_NHPAUQUObject@@@Z 10016a5a f   qt-mt323:qt-mt323.dll
 0001:00015a60       ?qt_emit@QListView@@UAE_NHPAUQUObject@@@Z 10016a60 f   qt-mt323:qt-mt323.dll
 0001:00015a66       ?qt_emit@QSplitter@@UAE_NHPAUQUObject@@@Z 10016a66 f   qt-mt323:qt-mt323.dll
 0001:00015a6c       ?qt_emit@QVBoxLayout@@UAE_NHPAUQUObject@@@Z 10016a6c f   qt-mt323:qt-mt323.dll
 0001:00015a72       ?qt_emit@QWidget@@UAE_NHPAUQUObject@@@Z 10016a72 f   qt-mt323:qt-mt323.dll
 0001:00015a78       ?qt_invoke@QGuardedPtrPrivate@@UAE_NHPAUQUObject@@@Z 10016a78 f   qt-mt323:qt-mt323.dll
 0001:00015a7e       ?qt_invoke@QLabel@@UAE_NHPAUQUObject@@@Z 10016a7e f   qt-mt323:qt-mt323.dll
 0001:00015a84       ?qt_invoke@QListView@@UAE_NHPAUQUObject@@@Z 10016a84 f   qt-mt323:qt-mt323.dll
 0001:00015a8a       ?qt_invoke@QSplitter@@UAE_NHPAUQUObject@@@Z 10016a8a f   qt-mt323:qt-mt323.dll
 0001:00015a90       ?qt_invoke@QVBoxLayout@@UAE_NHPAUQUObject@@@Z 10016a90 f   qt-mt323:qt-mt323.dll
 0001:00015a96       ?qt_invoke@QWidget@@UAE_NHPAUQUObject@@@Z 10016a96 f   qt-mt323:qt-mt323.dll
 0001:00015a9c       ?qt_property@QGuardedPtrPrivate@@UAE_NHHPAVQVariant@@@Z 10016a9c f   qt-mt323:qt-mt323.dll
 0001:00015aa2       ?qt_property@QLabel@@UAE_NHHPAVQVariant@@@Z 10016aa2 f   qt-mt323:qt-mt323.dll
 0001:00015aa8       ?qt_property@QListView@@UAE_NHHPAVQVariant@@@Z 10016aa8 f   qt-mt323:qt-mt323.dll
 0001:00015aae       ?qt_property@QSplitter@@UAE_NHHPAVQVariant@@@Z 10016aae f   qt-mt323:qt-mt323.dll
 0001:00015ab4       ?qt_property@QVBoxLayout@@UAE_NHHPAVQVariant@@@Z 10016ab4 f   qt-mt323:qt-mt323.dll
 0001:00015aba       ?qt_property@QWidget@@UAE_NHHPAVQVariant@@@Z 10016aba f   qt-mt323:qt-mt323.dll
 0001:00015ac0       ?read@QGList@@MAEAAVQDataStream@@AAV2@AAPAX@Z 10016ac0 f   qt-mt323:qt-mt323.dll
 0001:00015ac6       ?removeItem@QListViewItem@@UAEXPAV1@@Z 10016ac6 f   qt-mt323:qt-mt323.dll
 0001:00015acc       ?resizeEvent@QLabel@@MAEXPAVQResizeEvent@@@Z 10016acc f   qt-mt323:qt-mt323.dll
 0001:00015ad2       ?resizeEvent@QSplitter@@MAEXPAVQResizeEvent@@@Z 10016ad2 f   qt-mt323:qt-mt323.dll
 0001:00015ad8       ?rtti@QListViewItem@@UBEHXZ 10016ad8 f   qt-mt323:qt-mt323.dll
 0001:00015ade       ?setAlignment@QLabel@@UAEXH@Z 10016ade f   qt-mt323:qt-mt323.dll
 0001:00015ae4       ?setAlignment@QLayoutItem@@UAEXH@Z 10016ae4 f   qt-mt323:qt-mt323.dll
 0001:00015aea       ?setAutoAdd@QLayout@@UAEX_N@Z 10016aea f   qt-mt323:qt-mt323.dll
 0001:00015af0       ?setAutoResize@QLabel@@UAEX_N@Z 10016af0 f   qt-mt323:qt-mt323.dll
 0001:00015af6       ?setBuddy@QLabel@@UAEXPAVQWidget@@@Z 10016af6 f   qt-mt323:qt-mt323.dll
 0001:00015afc       ?setDragEnabled@QListViewItem@@UAEX_N@Z 10016afc f   qt-mt323:qt-mt323.dll
 0001:00015b02       ?setDropEnabled@QListViewItem@@UAEX_N@Z 10016b02 f   qt-mt323:qt-mt323.dll
 0001:00015b08       ?setEnabled@QListViewItem@@UAEX_N@Z 10016b08 f   qt-mt323:qt-mt323.dll
 0001:00015b0e       ?setExpandable@QListViewItem@@UAEX_N@Z 10016b0e f   qt-mt323:qt-mt323.dll
 0001:00015b14       ?setFont@QLabel@@UAEXABVQFont@@@Z 10016b14 f   qt-mt323:qt-mt323.dll
 0001:00015b1a       ?setGeometry@QBoxLayout@@UAEXABVQRect@@@Z 10016b1a f   qt-mt323:qt-mt323.dll
 0001:00015b20       ?setHeight@QListViewItem@@MAEXH@Z 10016b20 f   qt-mt323:qt-mt323.dll
 0001:00015b26       ?setMargin@QLayout@@UAEXH@Z 10016b26 f   qt-mt323:qt-mt323.dll
 0001:00015b2c       ?setMenuBar@QLayout@@UAEXPAVQMenuBar@@@Z 10016b2c f   qt-mt323:qt-mt323.dll
 0001:00015b32       ?setMovie@QLabel@@UAEXABVQMovie@@@Z 10016b32 f   qt-mt323:qt-mt323.dll
 0001:00015b38       ?setMultiLinesEnabled@QListViewItem@@UAEX_N@Z 10016b38 f   qt-mt323:qt-mt323.dll
 0001:00015b3e       ?setName@QObject@@UAEXPBD@Z 10016b3e f   qt-mt323:qt-mt323.dll
 0001:00015b44       ?setNum@QLabel@@UAEXH@Z    10016b44 f   qt-mt323:qt-mt323.dll
 0001:00015b4a       ?setNum@QLabel@@UAEXN@Z    10016b4a f   qt-mt323:qt-mt323.dll
 0001:00015b50       ?setOpaqueResize@QSplitter@@UAEX_N@Z 10016b50 f   qt-mt323:qt-mt323.dll
 0001:00015b56       ?setOpen@QListViewItem@@UAEX_N@Z 10016b56 f   qt-mt323:qt-mt323.dll
 0001:00015b5c       ?setOrientation@QSplitter@@UAEXW4Orientation@Qt@@@Z 10016b5c f   qt-mt323:qt-mt323.dll
 0001:00015b62       ?setPicture@QLabel@@UAEXABVQPicture@@@Z 10016b62 f   qt-mt323:qt-mt323.dll
 0001:00015b68       ?setPixmap@QLabel@@UAEXABVQPixmap@@@Z 10016b68 f   qt-mt323:qt-mt323.dll
 0001:00015b6e       ?setPixmap@QListViewItem@@UAEXHABVQPixmap@@@Z 10016b6e f   qt-mt323:qt-mt323.dll
 0001:00015b74       ?setRenameEnabled@QListViewItem@@UAEXH_N@Z 10016b74 f   qt-mt323:qt-mt323.dll
 0001:00015b7a       ?setResizeMode@QSplitter@@UAEXPAVQWidget@@W4ResizeMode@1@@Z 10016b7a f   qt-mt323:qt-mt323.dll
 0001:00015b80       ?setRubberband@QSplitter@@MAEXH@Z 10016b80 f   qt-mt323:qt-mt323.dll
 0001:00015b86       ?setSelectable@QListViewItem@@UAEX_N@Z 10016b86 f   qt-mt323:qt-mt323.dll
 0001:00015b8c       ?setSelected@QListViewItem@@UAEX_N@Z 10016b8c f   qt-mt323:qt-mt323.dll
 0001:00015b92       ?setSpacing@QLayout@@UAEXH@Z 10016b92 f   qt-mt323:qt-mt323.dll
 0001:00015b98       ?setText@QLabel@@UAEXABVQString@@@Z 10016b98 f   qt-mt323:qt-mt323.dll
 0001:00015b9e       ?setText@QListViewItem@@UAEXHABVQString@@@Z 10016b9e f   qt-mt323:qt-mt323.dll
 0001:00015ba4       ?setup@QListViewItem@@UAEXXZ 10016ba4 f   qt-mt323:qt-mt323.dll
 0001:00015baa       ?sizeHint@QBoxLayout@@UBE?AVQSize@@XZ 10016baa f   qt-mt323:qt-mt323.dll
 0001:00015bb0       ?sizeHint@QLabel@@UBE?AVQSize@@XZ 10016bb0 f   qt-mt323:qt-mt323.dll
 0001:00015bb6       ?sizeHint@QSplitter@@UBE?AVQSize@@XZ 10016bb6 f   qt-mt323:qt-mt323.dll
 0001:00015bbc       ?sort@QListViewItem@@UAEXXZ 10016bbc f   qt-mt323:qt-mt323.dll
 0001:00015bc2       ?sortChildItems@QListViewItem@@UAEXH_N@Z 10016bc2 f   qt-mt323:qt-mt323.dll
 0001:00015bc8       ?spacerItem@QLayoutItem@@UAEPAVQSpacerItem@@XZ 10016bc8 f   qt-mt323:qt-mt323.dll
 0001:00015bce       ?startRename@QListViewItem@@UAEXH@Z 10016bce f   qt-mt323:qt-mt323.dll
 0001:00015bd4       ?styleChange@QFrame@@MAEXAAVQStyle@@@Z 10016bd4 f   qt-mt323:qt-mt323.dll
 0001:00015bda       ?styleChange@QSplitter@@MAEXAAVQStyle@@@Z 10016bda f   qt-mt323:qt-mt323.dll
 0001:00015be0       ?takeItem@QListViewItem@@UAEXPAV1@@Z 10016be0 f   qt-mt323:qt-mt323.dll
 0001:00015be6       ?text@QListViewItem@@UBE?AVQString@@H@Z 10016be6 f   qt-mt323:qt-mt323.dll
 0001:00015bec       ?widget@QLayoutItem@@UAEPAVQWidget@@XZ 10016bec f   qt-mt323:qt-mt323.dll
 0001:00015bf2       ?width@QListViewItem@@UBEHABVQFontMetrics@@PBVQListView@@H@Z 10016bf2 f   qt-mt323:qt-mt323.dll
 0001:00015bf8       ?write@QGList@@MBEAAVQDataStream@@AAV2@PAX@Z 10016bf8 f   qt-mt323:qt-mt323.dll
 0001:00015bfe       ?childEvent@QGroupBox@@MAEXPAVQChildEvent@@@Z 10016bfe f   qt-mt323:qt-mt323.dll
 0001:00015c04       ?className@QFrame@@UBEPBDXZ 10016c04 f   qt-mt323:qt-mt323.dll
 0001:00015c0a       ?className@QGroupBox@@UBEPBDXZ 10016c0a f   qt-mt323:qt-mt323.dll
 0001:00015c10       ?className@QHBoxLayout@@UBEPBDXZ 10016c10 f   qt-mt323:qt-mt323.dll
 0001:00015c16       ?className@QLineEdit@@UBEPBDXZ 10016c16 f   qt-mt323:qt-mt323.dll
 0001:00015c1c       ?className@QListBox@@UBEPBDXZ 10016c1c f   qt-mt323:qt-mt323.dll
 0001:00015c22       ?className@QPushButton@@UBEPBDXZ 10016c22 f   qt-mt323:qt-mt323.dll
 0001:00015c28       ?clear@QLineEdit@@UAEXXZ   10016c28 f   qt-mt323:qt-mt323.dll
 0001:00015c2e       ?clearSelection@QListBox@@UAEXXZ 10016c2e f   qt-mt323:qt-mt323.dll
 0001:00015c34       ?clearValidator@QLineEdit@@UAEXXZ 10016c34 f   qt-mt323:qt-mt323.dll
 0001:00015c3a       ?contentsContextMenuEvent@QListBox@@MAEXPAVQContextMenuEvent@@@Z 10016c3a f   qt-mt323:qt-mt323.dll
 0001:00015c40       ?contentsDragEnterEvent@QScrollView@@MAEXPAVQDragEnterEvent@@@Z 10016c40 f   qt-mt323:qt-mt323.dll
 0001:00015c46       ?contentsDragLeaveEvent@QScrollView@@MAEXPAVQDragLeaveEvent@@@Z 10016c46 f   qt-mt323:qt-mt323.dll
 0001:00015c4c       ?contentsDragMoveEvent@QScrollView@@MAEXPAVQDragMoveEvent@@@Z 10016c4c f   qt-mt323:qt-mt323.dll
 0001:00015c52       ?contentsDropEvent@QScrollView@@MAEXPAVQDropEvent@@@Z 10016c52 f   qt-mt323:qt-mt323.dll
 0001:00015c58       ?contentsMouseDoubleClickEvent@QScrollView@@MAEXPAVQMouseEvent@@@Z 10016c58 f   qt-mt323:qt-mt323.dll
 0001:00015c5e       ?contentsMouseMoveEvent@QScrollView@@MAEXPAVQMouseEvent@@@Z 10016c5e f   qt-mt323:qt-mt323.dll
 0001:00015c64       ?contentsMousePressEvent@QScrollView@@MAEXPAVQMouseEvent@@@Z 10016c64 f   qt-mt323:qt-mt323.dll
 0001:00015c6a       ?contentsMouseReleaseEvent@QScrollView@@MAEXPAVQMouseEvent@@@Z 10016c6a f   qt-mt323:qt-mt323.dll
 0001:00015c70       ?contextMenuEvent@QLineEdit@@MAEXPAVQContextMenuEvent@@@Z 10016c70 f   qt-mt323:qt-mt323.dll
 0001:00015c76       ?copy@QLineEdit@@UBEXXZ    10016c76 f   qt-mt323:qt-mt323.dll
 0001:00015c7c       ?createPopupMenu@QLineEdit@@MAEPAVQPopupMenu@@XZ 10016c7c f   qt-mt323:qt-mt323.dll
 0001:00015c82       ?cut@QLineEdit@@UAEXXZ     10016c82 f   qt-mt323:qt-mt323.dll
 0001:00015c88       ?deselect@QLineEdit@@UAEXXZ 10016c88 f   qt-mt323:qt-mt323.dll
 0001:00015c8e       ?dragEnterEvent@QLineEdit@@MAEXPAVQDragEnterEvent@@@Z 10016c8e f   qt-mt323:qt-mt323.dll
 0001:00015c94       ?dragLeaveEvent@QLineEdit@@MAEXPAVQDragLeaveEvent@@@Z 10016c94 f   qt-mt323:qt-mt323.dll
 0001:00015c9a       ?dragMoveEvent@QLineEdit@@MAEXPAVQDragMoveEvent@@@Z 10016c9a f   qt-mt323:qt-mt323.dll
 0001:00015ca0       ?drawButton@QPushButton@@MAEXPAVQPainter@@@Z 10016ca0 f   qt-mt323:qt-mt323.dll
 0001:00015ca6       ?drawButtonLabel@QPushButton@@MAEXPAVQPainter@@@Z 10016ca6 f   qt-mt323:qt-mt323.dll
 0001:00015cac       ?drawContents@QLineEdit@@MAEXPAVQPainter@@@Z 10016cac f   qt-mt323:qt-mt323.dll
 0001:00015cb2       ?drawContentsOffset@QScrollView@@MAEXPAVQPainter@@HHHHHH@Z 10016cb2 f   qt-mt323:qt-mt323.dll
 0001:00015cb8       ?dropEvent@QLineEdit@@MAEXPAVQDropEvent@@@Z 10016cb8 f   qt-mt323:qt-mt323.dll
 0001:00015cbe       ?enabledChange@QButton@@MAEX_N@Z 10016cbe f   qt-mt323:qt-mt323.dll
 0001:00015cc4       ?ensureCurrentVisible@QListBox@@UAEXXZ 10016cc4 f   qt-mt323:qt-mt323.dll
 0001:00015cca       ?event@QGroupBox@@MAE_NPAVQEvent@@@Z 10016cca f   qt-mt323:qt-mt323.dll
 0001:00015cd0       ?event@QLineEdit@@MAE_NPAVQEvent@@@Z 10016cd0 f   qt-mt323:qt-mt323.dll
 0001:00015cd6       ?eventFilter@QListBox@@MAE_NPAVQObject@@PAVQEvent@@@Z 10016cd6 f   qt-mt323:qt-mt323.dll
 0001:00015cdc       ?expanding@QSpacerItem@@UBE?AW4ExpandData@QSizePolicy@@XZ 10016cdc f   qt-mt323:qt-mt323.dll
 0001:00015ce2       ?focusInEvent@QGroupBox@@MAEXPAVQFocusEvent@@@Z 10016ce2 f   qt-mt323:qt-mt323.dll
 0001:00015ce8       ?focusInEvent@QLineEdit@@MAEXPAVQFocusEvent@@@Z 10016ce8 f   qt-mt323:qt-mt323.dll
 0001:00015cee       ?focusInEvent@QListBox@@MAEXPAVQFocusEvent@@@Z 10016cee f   qt-mt323:qt-mt323.dll
 0001:00015cf4       ?focusInEvent@QPushButton@@MAEXPAVQFocusEvent@@@Z 10016cf4 f   qt-mt323:qt-mt323.dll
 0001:00015cfa       ?focusOutEvent@QLineEdit@@MAEXPAVQFocusEvent@@@Z 10016cfa f   qt-mt323:qt-mt323.dll
 0001:00015d00       ?focusOutEvent@QListBox@@MAEXPAVQFocusEvent@@@Z 10016d00 f   qt-mt323:qt-mt323.dll
 0001:00015d06       ?focusOutEvent@QPushButton@@MAEXPAVQFocusEvent@@@Z 10016d06 f   qt-mt323:qt-mt323.dll
 0001:00015d0c       ?fontChange@QGroupBox@@MAEXABVQFont@@@Z 10016d0c f   qt-mt323:qt-mt323.dll
 0001:00015d12       ?geometry@QSpacerItem@@UBE?AVQRect@@XZ 10016d12 f   qt-mt323:qt-mt323.dll
 0001:00015d18       ?hasHeightForWidth@QLayoutItem@@UBE_NXZ 10016d18 f   qt-mt323:qt-mt323.dll
 0001:00015d1e       ?heightForWidth@QLayoutItem@@UBEHH@Z 10016d1e f   qt-mt323:qt-mt323.dll
 0001:00015d24       ?hitButton@QButton@@MBE_NABVQPoint@@@Z 10016d24 f   qt-mt323:qt-mt323.dll
 0001:00015d2a       ?imComposeEvent@QLineEdit@@MAEXPAVQIMEvent@@@Z 10016d2a f   qt-mt323:qt-mt323.dll
 0001:00015d30       ?imEndEvent@QLineEdit@@MAEXPAVQIMEvent@@@Z 10016d30 f   qt-mt323:qt-mt323.dll
 0001:00015d36       ?imStartEvent@QLineEdit@@MAEXPAVQIMEvent@@@Z 10016d36 f   qt-mt323:qt-mt323.dll
 0001:00015d3c       ?insert@QLineEdit@@UAEXABVQString@@@Z 10016d3c f   qt-mt323:qt-mt323.dll
 0001:00015d42       ?invalidate@QLayoutItem@@UAEXXZ 10016d42 f   qt-mt323:qt-mt323.dll
 0001:00015d48       ?invertSelection@QListBox@@UAEXXZ 10016d48 f   qt-mt323:qt-mt323.dll
 0001:00015d4e       ?isEmpty@QSpacerItem@@UBE_NXZ 10016d4e f   qt-mt323:qt-mt323.dll
 0001:00015d54       ?iterator@QLayoutItem@@UAE?AVQLayoutIterator@@XZ 10016d54 f   qt-mt323:qt-mt323.dll
 0001:00015d5a       ?keyPressEvent@QButton@@MAEXPAVQKeyEvent@@@Z 10016d5a f   qt-mt323:qt-mt323.dll
 0001:00015d60       ?keyPressEvent@QLineEdit@@MAEXPAVQKeyEvent@@@Z 10016d60 f   qt-mt323:qt-mt323.dll
 0001:00015d66       ?keyPressEvent@QListBox@@MAEXPAVQKeyEvent@@@Z 10016d66 f   qt-mt323:qt-mt323.dll
 0001:00015d6c       ?keyReleaseEvent@QButton@@MAEXPAVQKeyEvent@@@Z 10016d6c f   qt-mt323:qt-mt323.dll
 0001:00015d72       ?layout@QLayoutItem@@UAEPAVQLayout@@XZ 10016d72 f   qt-mt323:qt-mt323.dll
 0001:00015d78       ?maximumSize@QSpacerItem@@UBE?AVQSize@@XZ 10016d78 f   qt-mt323:qt-mt323.dll
 0001:00015d7e       ?metaObject@QFrame@@UBEPAVQMetaObject@@XZ 10016d7e f   qt-mt323:qt-mt323.dll
 0001:00015d84       ?metaObject@QGroupBox@@UBEPAVQMetaObject@@XZ 10016d84 f   qt-mt323:qt-mt323.dll
 0001:00015d8a       ?metaObject@QHBoxLayout@@UBEPAVQMetaObject@@XZ 10016d8a f   qt-mt323:qt-mt323.dll
 0001:00015d90       ?metaObject@QLineEdit@@UBEPAVQMetaObject@@XZ 10016d90 f   qt-mt323:qt-mt323.dll
 0001:00015d96       ?metaObject@QListBox@@UBEPAVQMetaObject@@XZ 10016d96 f   qt-mt323:qt-mt323.dll
 0001:00015d9c       ?metaObject@QPushButton@@UBEPAVQMetaObject@@XZ 10016d9c f   qt-mt323:qt-mt323.dll
 0001:00015da2       ?minimumSize@QSpacerItem@@UBE?AVQSize@@XZ 10016da2 f   qt-mt323:qt-mt323.dll
 0001:00015da8       ?minimumSizeHint@QLineEdit@@UBE?AVQSize@@XZ 10016da8 f   qt-mt323:qt-mt323.dll
 0001:00015dae       ?minimumSizeHint@QListBox@@UBE?AVQSize@@XZ 10016dae f   qt-mt323:qt-mt323.dll
 0001:00015db4       ?mouseDoubleClickEvent@QLineEdit@@MAEXPAVQMouseEvent@@@Z 10016db4 f   qt-mt323:qt-mt323.dll
 0001:00015dba       ?mouseDoubleClickEvent@QListBox@@MAEXPAVQMouseEvent@@@Z 10016dba f   qt-mt323:qt-mt323.dll
 0001:00015dc0       ?mouseMoveEvent@QButton@@MAEXPAVQMouseEvent@@@Z 10016dc0 f   qt-mt323:qt-mt323.dll
 0001:00015dc6       ?mouseMoveEvent@QLineEdit@@MAEXPAVQMouseEvent@@@Z 10016dc6 f   qt-mt323:qt-mt323.dll
 0001:00015dcc       ?mouseMoveEvent@QListBox@@MAEXPAVQMouseEvent@@@Z 10016dcc f   qt-mt323:qt-mt323.dll
 0001:00015dd2       ?mousePressEvent@QButton@@MAEXPAVQMouseEvent@@@Z 10016dd2 f   qt-mt323:qt-mt323.dll
 0001:00015dd8       ?mousePressEvent@QLineEdit@@MAEXPAVQMouseEvent@@@Z 10016dd8 f   qt-mt323:qt-mt323.dll
 0001:00015dde       ?mousePressEvent@QListBox@@MAEXPAVQMouseEvent@@@Z 10016dde f   qt-mt323:qt-mt323.dll
 0001:00015de4       ?mouseReleaseEvent@QButton@@MAEXPAVQMouseEvent@@@Z 10016de4 f   qt-mt323:qt-mt323.dll
 0001:00015dea       ?mouseReleaseEvent@QLineEdit@@MAEXPAVQMouseEvent@@@Z 10016dea f   qt-mt323:qt-mt323.dll
 0001:00015df0       ?mouseReleaseEvent@QListBox@@MAEXPAVQMouseEvent@@@Z 10016df0 f   qt-mt323:qt-mt323.dll
 0001:00015df6       ?move@QPushButton@@UAEXHH@Z 10016df6 f   qt-mt323:qt-mt323.dll
 0001:00015dfc       ?paintCell@QListBox@@MAEXPAVQPainter@@HH@Z 10016dfc f   qt-mt323:qt-mt323.dll
 0001:00015e02       ?paintEvent@QButton@@MAEXPAVQPaintEvent@@@Z 10016e02 f   qt-mt323:qt-mt323.dll
 0001:00015e08       ?paintEvent@QGroupBox@@MAEXPAVQPaintEvent@@@Z 10016e08 f   qt-mt323:qt-mt323.dll
 0001:00015e0e       ?paste@QLineEdit@@UAEXXZ   10016e0e f   qt-mt323:qt-mt323.dll
 0001:00015e14       ?qt_cast@QFrame@@UAEPAXPBD@Z 10016e14 f   qt-mt323:qt-mt323.dll
 0001:00015e1a       ?qt_cast@QGroupBox@@UAEPAXPBD@Z 10016e1a f   qt-mt323:qt-mt323.dll
 0001:00015e20       ?qt_cast@QHBoxLayout@@UAEPAXPBD@Z 10016e20 f   qt-mt323:qt-mt323.dll
 0001:00015e26       ?qt_cast@QLineEdit@@UAEPAXPBD@Z 10016e26 f   qt-mt323:qt-mt323.dll
 0001:00015e2c       ?qt_cast@QListBox@@UAEPAXPBD@Z 10016e2c f   qt-mt323:qt-mt323.dll
 0001:00015e32       ?qt_cast@QPushButton@@UAEPAXPBD@Z 10016e32 f   qt-mt323:qt-mt323.dll
 0001:00015e38       ?qt_emit@QFrame@@UAE_NHPAUQUObject@@@Z 10016e38 f   qt-mt323:qt-mt323.dll
 0001:00015e3e       ?qt_emit@QGroupBox@@UAE_NHPAUQUObject@@@Z 10016e3e f   qt-mt323:qt-mt323.dll
 0001:00015e44       ?qt_emit@QHBoxLayout@@UAE_NHPAUQUObject@@@Z 10016e44 f   qt-mt323:qt-mt323.dll
 0001:00015e4a       ?qt_emit@QLineEdit@@UAE_NHPAUQUObject@@@Z 10016e4a f   qt-mt323:qt-mt323.dll
 0001:00015e50       ?qt_emit@QListBox@@UAE_NHPAUQUObject@@@Z 10016e50 f   qt-mt323:qt-mt323.dll
 0001:00015e56       ?qt_emit@QPushButton@@UAE_NHPAUQUObject@@@Z 10016e56 f   qt-mt323:qt-mt323.dll
 0001:00015e5c       ?qt_invoke@QFrame@@UAE_NHPAUQUObject@@@Z 10016e5c f   qt-mt323:qt-mt323.dll
 0001:00015e62       ?qt_invoke@QGroupBox@@UAE_NHPAUQUObject@@@Z 10016e62 f   qt-mt323:qt-mt323.dll
 0001:00015e68       ?qt_invoke@QHBoxLayout@@UAE_NHPAUQUObject@@@Z 10016e68 f   qt-mt323:qt-mt323.dll
 0001:00015e6e       ?qt_invoke@QLineEdit@@UAE_NHPAUQUObject@@@Z 10016e6e f   qt-mt323:qt-mt323.dll
 0001:00015e74       ?qt_invoke@QListBox@@UAE_NHPAUQUObject@@@Z 10016e74 f   qt-mt323:qt-mt323.dll
 0001:00015e7a       ?qt_invoke@QPushButton@@UAE_NHPAUQUObject@@@Z 10016e7a f   qt-mt323:qt-mt323.dll
 0001:00015e80       ?qt_property@QFrame@@UAE_NHHPAVQVariant@@@Z 10016e80 f   qt-mt323:qt-mt323.dll
 0001:00015e86       ?qt_property@QGroupBox@@UAE_NHHPAVQVariant@@@Z 10016e86 f   qt-mt323:qt-mt323.dll
 0001:00015e8c       ?qt_property@QHBoxLayout@@UAE_NHHPAVQVariant@@@Z 10016e8c f   qt-mt323:qt-mt323.dll
 0001:00015e92       ?qt_property@QLineEdit@@UAE_NHHPAVQVariant@@@Z 10016e92 f   qt-mt323:qt-mt323.dll
 0001:00015e98       ?qt_property@QListBox@@UAE_NHHPAVQVariant@@@Z 10016e98 f   qt-mt323:qt-mt323.dll
 0001:00015e9e       ?qt_property@QPushButton@@UAE_NHHPAVQVariant@@@Z 10016e9e f   qt-mt323:qt-mt323.dll
 0001:00015ea4       ?redo@QLineEdit@@UAEXXZ    10016ea4 f   qt-mt323:qt-mt323.dll
 0001:00015eaa       ?resize@QPushButton@@UAEXHH@Z 10016eaa f   qt-mt323:qt-mt323.dll
 0001:00015eb0       ?resizeEvent@QFrame@@MAEXPAVQResizeEvent@@@Z 10016eb0 f   qt-mt323:qt-mt323.dll
 0001:00015eb6       ?resizeEvent@QGroupBox@@MAEXPAVQResizeEvent@@@Z 10016eb6 f   qt-mt323:qt-mt323.dll
 0001:00015ebc       ?resizeEvent@QLineEdit@@MAEXPAVQResizeEvent@@@Z 10016ebc f   qt-mt323:qt-mt323.dll
 0001:00015ec2       ?resizeEvent@QListBox@@MAEXPAVQResizeEvent@@@Z 10016ec2 f   qt-mt323:qt-mt323.dll
 0001:00015ec8       ?resizeEvent@QPushButton@@MAEXPAVQResizeEvent@@@Z 10016ec8 f   qt-mt323:qt-mt323.dll
 0001:00015ece       ?selectAll@QLineEdit@@UAEXXZ 10016ece f   qt-mt323:qt-mt323.dll
 0001:00015ed4       ?selectAll@QListBox@@UAEX_N@Z 10016ed4 f   qt-mt323:qt-mt323.dll
 0001:00015eda       ?setAccel@QButton@@UAEXABVQKeySequence@@@Z 10016eda f   qt-mt323:qt-mt323.dll
 0001:00015ee0       ?setAlignment@QGroupBox@@UAEXH@Z 10016ee0 f   qt-mt323:qt-mt323.dll
 0001:00015ee6       ?setAlignment@QLineEdit@@UAEXH@Z 10016ee6 f   qt-mt323:qt-mt323.dll
 0001:00015eec       ?setAutoDefault@QPushButton@@UAEX_N@Z 10016eec f   qt-mt323:qt-mt323.dll
 0001:00015ef2       ?setAutoRepeat@QButton@@UAEX_N@Z 10016ef2 f   qt-mt323:qt-mt323.dll
 0001:00015ef8       ?setBottomItem@QListBox@@UAEXH@Z 10016ef8 f   qt-mt323:qt-mt323.dll
 0001:00015efe       ?setColumnLayout@QGroupBox@@UAEXHW4Orientation@Qt@@@Z 10016efe f   qt-mt323:qt-mt323.dll
 0001:00015f04       ?setColumnMode@QListBox@@UAEXH@Z 10016f04 f   qt-mt323:qt-mt323.dll
 0001:00015f0a       ?setColumnMode@QListBox@@UAEXW4LayoutMode@1@@Z 10016f0a f   qt-mt323:qt-mt323.dll
 0001:00015f10       ?setContentsPos@QScrollView@@UAEXHH@Z 10016f10 f   qt-mt323:qt-mt323.dll
 0001:00015f16       ?setCurrentItem@QListBox@@UAEXH@Z 10016f16 f   qt-mt323:qt-mt323.dll
 0001:00015f1c       ?setCurrentItem@QListBox@@UAEXPAVQListBoxItem@@@Z 10016f1c f   qt-mt323:qt-mt323.dll
 0001:00015f22       ?setCursorPosition@QLineEdit@@UAEXH@Z 10016f22 f   qt-mt323:qt-mt323.dll
 0001:00015f28       ?setDefault@QPushButton@@UAEX_N@Z 10016f28 f   qt-mt323:qt-mt323.dll
 0001:00015f2e       ?setDown@QButton@@UAEX_N@Z 10016f2e f   qt-mt323:qt-mt323.dll
 0001:00015f34       ?setDragEnabled@QLineEdit@@UAEX_N@Z 10016f34 f   qt-mt323:qt-mt323.dll
 0001:00015f3a       ?setEchoMode@QLineEdit@@UAEXW4EchoMode@1@@Z 10016f3a f   qt-mt323:qt-mt323.dll
 0001:00015f40       ?setEnabled@QGroupBox@@UAEX_N@Z 10016f40 f   qt-mt323:qt-mt323.dll
 0001:00015f46       ?setFont@QLineEdit@@UAEXABVQFont@@@Z 10016f46 f   qt-mt323:qt-mt323.dll
 0001:00015f4c       ?setFont@QListBox@@UAEXABVQFont@@@Z 10016f4c f   qt-mt323:qt-mt323.dll
 0001:00015f52       ?setFrame@QLineEdit@@UAEX_N@Z 10016f52 f   qt-mt323:qt-mt323.dll
 0001:00015f58       ?setGeometry@QPushButton@@UAEXABVQRect@@@Z 10016f58 f   qt-mt323:qt-mt323.dll
 0001:00015f5e       ?setGeometry@QPushButton@@UAEXHHHH@Z 10016f5e f   qt-mt323:qt-mt323.dll
 0001:00015f64       ?setGeometry@QSpacerItem@@UAEXABVQRect@@@Z 10016f64 f   qt-mt323:qt-mt323.dll
 0001:00015f6a       ?setGroup@QButton@@EAEXPAVQButtonGroup@@@Z 10016f6a f   qt-mt323:qt-mt323.dll
 0001:00015f70       ?setIsMenuButton@QPushButton@@UAEX_N@Z 10016f70 f   qt-mt323:qt-mt323.dll
 0001:00015f76       ?setMaxLength@QLineEdit@@UAEXH@Z 10016f76 f   qt-mt323:qt-mt323.dll
 0001:00015f7c       ?setOn@QPushButton@@UAEX_N@Z 10016f7c f   qt-mt323:qt-mt323.dll
 0001:00015f82       ?setPalette@QLineEdit@@UAEXABVQPalette@@@Z 10016f82 f   qt-mt323:qt-mt323.dll
 0001:00015f88       ?setPixmap@QButton@@UAEXABVQPixmap@@@Z 10016f88 f   qt-mt323:qt-mt323.dll
 0001:00015f8e       ?setReadOnly@QLineEdit@@UAEX_N@Z 10016f8e f   qt-mt323:qt-mt323.dll
 0001:00015f94       ?setRowMode@QListBox@@UAEXH@Z 10016f94 f   qt-mt323:qt-mt323.dll
 0001:00015f9a       ?setRowMode@QListBox@@UAEXW4LayoutMode@1@@Z 10016f9a f   qt-mt323:qt-mt323.dll
 0001:00015fa0       ?setSelected@QListBox@@UAEXPAVQListBoxItem@@_N@Z 10016fa0 f   qt-mt323:qt-mt323.dll
 0001:00015fa6       ?setSelection@QLineEdit@@UAEXHH@Z 10016fa6 f   qt-mt323:qt-mt323.dll
 0001:00015fac       ?setSelectionMode@QListBox@@UAEXW4SelectionMode@1@@Z 10016fac f   qt-mt323:qt-mt323.dll
 0001:00015fb2       ?setState@QButton@@MAEXW4ToggleState@1@@Z 10016fb2 f   qt-mt323:qt-mt323.dll
 0001:00015fb8       ?setText@QButton@@UAEXABVQString@@@Z 10016fb8 f   qt-mt323:qt-mt323.dll
 0001:00015fbe       ?setText@QLineEdit@@UAEXABVQString@@@Z 10016fbe f   qt-mt323:qt-mt323.dll
 0001:00015fc4       ?setTitle@QGroupBox@@UAEXABVQString@@@Z 10016fc4 f   qt-mt323:qt-mt323.dll
 0001:00015fca       ?setToggleType@QButton@@MAEXW4ToggleType@1@@Z 10016fca f   qt-mt323:qt-mt323.dll
 0001:00015fd0       ?setTopItem@QListBox@@UAEXH@Z 10016fd0 f   qt-mt323:qt-mt323.dll
 0001:00015fd6       ?setValidator@QLineEdit@@UAEXPBVQValidator@@@Z 10016fd6 f   qt-mt323:qt-mt323.dll
 0001:00015fdc       ?setVariableHeight@QListBox@@UAEX_N@Z 10016fdc f   qt-mt323:qt-mt323.dll
 0001:00015fe2       ?setVariableWidth@QListBox@@UAEX_N@Z 10016fe2 f   qt-mt323:qt-mt323.dll
 0001:00015fe8       ?show@QScrollView@@UAEXXZ  10016fe8 f   qt-mt323:qt-mt323.dll
 0001:00015fee       ?showEvent@QListBox@@MAEXPAVQShowEvent@@@Z 10016fee f   qt-mt323:qt-mt323.dll
 0001:00015ff4       ?sizeHint@QFrame@@UBE?AVQSize@@XZ 10016ff4 f   qt-mt323:qt-mt323.dll
 0001:00015ffa       ?sizeHint@QGroupBox@@UBE?AVQSize@@XZ 10016ffa f   qt-mt323:qt-mt323.dll
 0001:00016000       ?sizeHint@QLineEdit@@UBE?AVQSize@@XZ 10017000 f   qt-mt323:qt-mt323.dll
 0001:00016006       ?sizeHint@QListBox@@UBE?AVQSize@@XZ 10017006 f   qt-mt323:qt-mt323.dll
 0001:0001600c       ?sizeHint@QPushButton@@UBE?AVQSize@@XZ 1001700c f   qt-mt323:qt-mt323.dll
 0001:00016012       ?sizeHint@QSpacerItem@@UBE?AVQSize@@XZ 10017012 f   qt-mt323:qt-mt323.dll
 0001:00016018       ?spacerItem@QSpacerItem@@UAEPAV1@XZ 10017018 f   qt-mt323:qt-mt323.dll
 0001:0001601e       ?styleChange@QScrollView@@UAEXAAVQStyle@@@Z 1001701e f   qt-mt323:qt-mt323.dll
 0001:00016024       ?undo@QLineEdit@@UAEXXZ    10017024 f   qt-mt323:qt-mt323.dll
 0001:0001602a       ?updateMask@QPushButton@@MAEXXZ 1001702a f   qt-mt323:qt-mt323.dll
 0001:00016030       ?viewportPaintEvent@QListBox@@UAEXPAVQPaintEvent@@@Z 10017030 f   qt-mt323:qt-mt323.dll
 0001:00016036       ?viewportResizeEvent@QScrollView@@MAEXPAVQResizeEvent@@@Z 10017036 f   qt-mt323:qt-mt323.dll
 0001:0001603c       ?windowActivationChange@QLineEdit@@MAEX_N@Z 1001703c f   qt-mt323:qt-mt323.dll
 0001:00016042       ?windowActivationChange@QListBox@@MAEX_N@Z 10017042 f   qt-mt323:qt-mt323.dll
 0001:00016048       ?setSelectionMode@QTable@@UAEXW4SelectionMode@1@@Z 10017048 f   qt-mt323:qt-mt323.dll
 0001:0001604e       ?insertColumns@QTable@@UAEXHH@Z 1001704e f   qt-mt323:qt-mt323.dll
 0001:00016054       ?endEdit@QTable@@MAEXHH_N0@Z 10017054 f   qt-mt323:qt-mt323.dll
 0001:0001605a       ?activateNextCell@QTable@@MAEXXZ 1001705a f   qt-mt323:qt-mt323.dll
 0001:00016060       ?addSelection@QTable@@UAEHABVQTableSelection@@@Z 10017060 f   qt-mt323:qt-mt323.dll
 0001:00016066       ?adjustColumn@QTable@@UAEXH@Z 10017066 f   qt-mt323:qt-mt323.dll
 0001:0001606c       ?adjustRow@QTable@@UAEXH@Z 1001706c f   qt-mt323:qt-mt323.dll
 0001:00016072       ?beginEdit@QTable@@MAEPAVQWidget@@HH_N@Z 10017072 f   qt-mt323:qt-mt323.dll
 0001:00016078       ?cellGeometry@QTable@@UBE?AVQRect@@HH@Z 10017078 f   qt-mt323:qt-mt323.dll
 0001:0001607e       ?cellRect@QTable@@UBE?AVQRect@@HH@Z 1001707e f   qt-mt323:qt-mt323.dll
 0001:00016084       ?cellWidget@QTable@@UBEPAVQWidget@@HH@Z 10017084 f   qt-mt323:qt-mt323.dll
 0001:0001608a       ?clearCell@QTable@@UAEXHH@Z 1001708a f   qt-mt323:qt-mt323.dll
 0001:00016090       ?clearCellWidget@QTable@@UAEXHH@Z 10017090 f   qt-mt323:qt-mt323.dll
 0001:00016096       ?columnAt@QTable@@UBEHH@Z  10017096 f   qt-mt323:qt-mt323.dll
 0001:0001609c       ?columnClicked@QTable@@MAEXH@Z 1001709c f   qt-mt323:qt-mt323.dll
 0001:000160a2       ?columnIndexChanged@QTable@@MAEXHHH@Z 100170a2 f   qt-mt323:qt-mt323.dll
 0001:000160a8       ?columnPos@QTable@@UBEHH@Z 100170a8 f   qt-mt323:qt-mt323.dll
 0001:000160ae       ?columnWidth@QTable@@UBEHH@Z 100170ae f   qt-mt323:qt-mt323.dll
 0001:000160b4       ?columnWidthChanged@QTable@@MAEXH@Z 100170b4 f   qt-mt323:qt-mt323.dll
 0001:000160ba       ?contentsContextMenuEvent@QTable@@MAEXPAVQContextMenuEvent@@@Z 100170ba f   qt-mt323:qt-mt323.dll
 0001:000160c0       ?contentsDragEnterEvent@QTable@@MAEXPAVQDragEnterEvent@@@Z 100170c0 f   qt-mt323:qt-mt323.dll
 0001:000160c6       ?contentsDragLeaveEvent@QTable@@MAEXPAVQDragLeaveEvent@@@Z 100170c6 f   qt-mt323:qt-mt323.dll
 0001:000160cc       ?contentsDragMoveEvent@QTable@@MAEXPAVQDragMoveEvent@@@Z 100170cc f   qt-mt323:qt-mt323.dll
 0001:000160d2       ?contentsDropEvent@QTable@@MAEXPAVQDropEvent@@@Z 100170d2 f   qt-mt323:qt-mt323.dll
 0001:000160d8       ?contentsMouseDoubleClickEvent@QTable@@MAEXPAVQMouseEvent@@@Z 100170d8 f   qt-mt323:qt-mt323.dll
 0001:000160de       ?contentsMouseMoveEvent@QTable@@MAEXPAVQMouseEvent@@@Z 100170de f   qt-mt323:qt-mt323.dll
 0001:000160e4       ?contentsMousePressEvent@QTable@@MAEXPAVQMouseEvent@@@Z 100170e4 f   qt-mt323:qt-mt323.dll
 0001:000160ea       ?contentsMouseReleaseEvent@QTable@@MAEXPAVQMouseEvent@@@Z 100170ea f   qt-mt323:qt-mt323.dll
 0001:000160f0       ?createEditor@QTable@@MBEPAVQWidget@@HH_N@Z 100170f0 f   qt-mt323:qt-mt323.dll
 0001:000160f6       ?currentSelection@QTable@@UBEHXZ 100170f6 f   qt-mt323:qt-mt323.dll
 0001:000160fc       ?dragObject@QTable@@MAEPAVQDragObject@@XZ 100170fc f   qt-mt323:qt-mt323.dll
 0001:00016102       ?drawContents@QTable@@EAEXPAVQPainter@@@Z 10017102 f   qt-mt323:qt-mt323.dll
 0001:00016108       ?drawContents@QTable@@MAEXPAVQPainter@@HHHH@Z 10017108 f   qt-mt323:qt-mt323.dll
 0001:0001610e       ?editCell@QTable@@UAEXHH_N@Z 1001710e f   qt-mt323:qt-mt323.dll
 0001:00016114       ?eventFilter@QTable@@UAE_NPAVQObject@@PAVQEvent@@@Z 10017114 f   qt-mt323:qt-mt323.dll
 0001:0001611a       ?focusInEvent@QTable@@MAEXPAVQFocusEvent@@@Z 1001711a f   qt-mt323:qt-mt323.dll
 0001:00016120       ?focusOutEvent@QTable@@MAEXPAVQFocusEvent@@@Z 10017120 f   qt-mt323:qt-mt323.dll
 0001:00016126       ?hideColumn@QTable@@UAEXH@Z 10017126 f   qt-mt323:qt-mt323.dll
 0001:0001612c       ?hideRow@QTable@@UAEXH@Z   1001712c f   qt-mt323:qt-mt323.dll
 0001:00016132       ?insertRows@QTable@@UAEXHH@Z 10017132 f   qt-mt323:qt-mt323.dll
 0001:00016138       ?insertWidget@QTable@@MAEXHHPAVQWidget@@@Z 10017138 f   qt-mt323:qt-mt323.dll
 0001:0001613e       ?item@QTable@@UBEPAVQTableItem@@HH@Z 1001713e f   qt-mt323:qt-mt323.dll
 0001:00016144       ?keyPressEvent@QTable@@MAEXPAVQKeyEvent@@@Z 10017144 f   qt-mt323:qt-mt323.dll
 0001:0001614a       ?minimumSizeHint@QScrollView@@UBE?AVQSize@@XZ 1001714a f   qt-mt323:qt-mt323.dll
 0001:00016150       ?numCols@QTable@@UBEHXZ    10017150 f   qt-mt323:qt-mt323.dll
 0001:00016156       ?numRows@QTable@@UBEHXZ    10017156 f   qt-mt323:qt-mt323.dll
 0001:0001615c       ?paintCell@QTable@@UAEXPAVQPainter@@HHABVQRect@@_N@Z 1001715c f   qt-mt323:qt-mt323.dll
 0001:00016162       ?paintCell@QTable@@UAEXPAVQPainter@@HHABVQRect@@_NABVQColorGroup@@@Z 10017162 f   qt-mt323:qt-mt323.dll
 0001:00016168       ?paintEmptyArea@QTable@@MAEXPAVQPainter@@HHHH@Z 10017168 f   qt-mt323:qt-mt323.dll
 0001:0001616e       ?paintEvent@QTable@@MAEXPAVQPaintEvent@@@Z 1001716e f   qt-mt323:qt-mt323.dll
 0001:00016174       ?paintFocus@QTable@@UAEXPAVQPainter@@ABVQRect@@@Z 10017174 f   qt-mt323:qt-mt323.dll
 0001:0001617a       ?pixmap@QTable@@UBE?AVQPixmap@@HH@Z 1001717a f   qt-mt323:qt-mt323.dll
 0001:00016180       ?removeColumn@QTable@@UAEXH@Z 10017180 f   qt-mt323:qt-mt323.dll
 0001:00016186       ?removeColumns@QTable@@UAEXABV?$QMemArray@H@@@Z 10017186 f   qt-mt323:qt-mt323.dll
 0001:0001618c       ?removeRow@QTable@@UAEXH@Z 1001718c f   qt-mt323:qt-mt323.dll
 0001:00016192       ?removeRows@QTable@@UAEXABV?$QMemArray@H@@@Z 10017192 f   qt-mt323:qt-mt323.dll
 0001:00016198       ?removeSelection@QTable@@UAEXABVQTableSelection@@@Z 10017198 f   qt-mt323:qt-mt323.dll
 0001:0001619e       ?removeSelection@QTable@@UAEXH@Z 1001719e f   qt-mt323:qt-mt323.dll
 0001:000161a4       ?resizeData@QTable@@MAEXH@Z 100171a4 f   qt-mt323:qt-mt323.dll
 0001:000161aa       ?resizeEvent@QScrollView@@MAEXPAVQResizeEvent@@@Z 100171aa f   qt-mt323:qt-mt323.dll
 0001:000161b0       ?rowAt@QTable@@UBEHH@Z     100171b0 f   qt-mt323:qt-mt323.dll
 0001:000161b6       ?rowHeight@QTable@@UBEHH@Z 100171b6 f   qt-mt323:qt-mt323.dll
 0001:000161bc       ?rowHeightChanged@QTable@@MAEXH@Z 100171bc f   qt-mt323:qt-mt323.dll
 0001:000161c2       ?rowIndexChanged@QTable@@MAEXHHH@Z 100171c2 f   qt-mt323:qt-mt323.dll
 0001:000161c8       ?rowPos@QTable@@UBEHH@Z    100171c8 f   qt-mt323:qt-mt323.dll
 0001:000161ce       ?setCellContentFromEditor@QTable@@MAEXHH@Z 100171ce f   qt-mt323:qt-mt323.dll
 0001:000161d4       ?setCellWidget@QTable@@UAEXHHPAVQWidget@@@Z 100171d4 f   qt-mt323:qt-mt323.dll
 0001:000161da       ?setColumnMovingEnabled@QTable@@UAEX_N@Z 100171da f   qt-mt323:qt-mt323.dll
 0001:000161e0       ?setColumnReadOnly@QTable@@UAEXH_N@Z 100171e0 f   qt-mt323:qt-mt323.dll
 0001:000161e6       ?setColumnStretchable@QTable@@UAEXH_N@Z 100171e6 f   qt-mt323:qt-mt323.dll
 0001:000161ec       ?setColumnWidth@QTable@@UAEXHH@Z 100171ec f   qt-mt323:qt-mt323.dll
 0001:000161f2       ?setCurrentCell@QTable@@UAEXHH@Z 100171f2 f   qt-mt323:qt-mt323.dll
 0001:000161f8       ?setDragEnabled@QTable@@UAEX_N@Z 100171f8 f   qt-mt323:qt-mt323.dll
 0001:000161fe       ?setEnabled@QTable@@UAEX_N@Z 100171fe f   qt-mt323:qt-mt323.dll
 0001:00016204       ?setFocusStyle@QTable@@UAEXW4FocusStyle@1@@Z 10017204 f   qt-mt323:qt-mt323.dll
 0001:0001620a       ?setItem@QTable@@UAEXHHPAVQTableItem@@@Z 1001720a f   qt-mt323:qt-mt323.dll
 0001:00016210       ?setLeftMargin@QTable@@UAEXH@Z 10017210 f   qt-mt323:qt-mt323.dll
 0001:00016216       ?setNumCols@QTable@@UAEXH@Z 10017216 f   qt-mt323:qt-mt323.dll
 0001:0001621c       ?setNumRows@QTable@@UAEXH@Z 1001721c f   qt-mt323:qt-mt323.dll
 0001:00016222       ?setPixmap@QTable@@UAEXHHABVQPixmap@@@Z 10017222 f   qt-mt323:qt-mt323.dll
 0001:00016228       ?setReadOnly@QTable@@UAEX_N@Z 10017228 f   qt-mt323:qt-mt323.dll
 0001:0001622e       ?setRowHeight@QTable@@UAEXHH@Z 1001722e f   qt-mt323:qt-mt323.dll
 0001:00016234       ?setRowMovingEnabled@QTable@@UAEX_N@Z 10017234 f   qt-mt323:qt-mt323.dll
 0001:0001623a       ?setRowReadOnly@QTable@@UAEXH_N@Z 1001723a f   qt-mt323:qt-mt323.dll
 0001:00016240       ?setRowStretchable@QTable@@UAEXH_N@Z 10017240 f   qt-mt323:qt-mt323.dll
 0001:00016246       ?setShowGrid@QTable@@UAEX_N@Z 10017246 f   qt-mt323:qt-mt323.dll
 0001:0001624c       ?setSorting@QTable@@UAEX_N@Z 1001724c f   qt-mt323:qt-mt323.dll
 0001:00016252       ?setText@QTable@@UAEXHHABVQString@@@Z 10017252 f   qt-mt323:qt-mt323.dll
 0001:00016258       ?setTopMargin@QTable@@UAEXH@Z 10017258 f   qt-mt323:qt-mt323.dll
 0001:0001625e       ?showColumn@QTable@@UAEXH@Z 1001725e f   qt-mt323:qt-mt323.dll
 0001:00016264       ?showEvent@QTable@@MAEXPAVQShowEvent@@@Z 10017264 f   qt-mt323:qt-mt323.dll
 0001:0001626a       ?showRow@QTable@@UAEXH@Z   1001726a f   qt-mt323:qt-mt323.dll
 0001:00016270       ?sizeHint@QTable@@UBE?AVQSize@@XZ 10017270 f   qt-mt323:qt-mt323.dll
 0001:00016276       ?sortColumn@QTable@@UAEXH_N0@Z 10017276 f   qt-mt323:qt-mt323.dll
 0001:0001627c       ?startDrag@QTable@@MAEXXZ  1001727c f   qt-mt323:qt-mt323.dll
 0001:00016282       ?swapCells@QTable@@UAEXHHHH@Z 10017282 f   qt-mt323:qt-mt323.dll
 0001:00016288       ?swapColumns@QTable@@UAEXHH_N@Z 10017288 f   qt-mt323:qt-mt323.dll
 0001:0001628e       ?swapRows@QTable@@UAEXHH_N@Z 1001728e f   qt-mt323:qt-mt323.dll
 0001:00016294       ?takeItem@QTable@@UAEXPAVQTableItem@@@Z 10017294 f   qt-mt323:qt-mt323.dll
 0001:0001629a       ?text@QTable@@UBE?AVQString@@HH@Z 1001729a f   qt-mt323:qt-mt323.dll
 0001:000162a0       ?viewportResizeEvent@QTable@@MAEXPAVQResizeEvent@@@Z 100172a0 f   qt-mt323:qt-mt323.dll
 0001:000162a6       ?windowActivationChange@QTable@@MAEX_N@Z 100172a6 f   qt-mt323:qt-mt323.dll
 0001:000162ac       ?activateItemAt@QPopupMenu@@UAEXH@Z 100172ac f   qt-mt323:qt-mt323.dll
 0001:000162b2       ?addTo@QAction@@UAE_NPAVQWidget@@@Z 100172b2 f   qt-mt323:qt-mt323.dll
 0001:000162b8       ?addedTo@QAction@@MAEXHPAVQPopupMenu@@@Z 100172b8 f   qt-mt323:qt-mt323.dll
 0001:000162be       ?addedTo@QAction@@MAEXPAVQWidget@@0@Z 100172be f   qt-mt323:qt-mt323.dll
 0001:000162c4       ?className@QAction@@UBEPBDXZ 100172c4 f   qt-mt323:qt-mt323.dll
 0001:000162ca       ?className@QDockWindow@@UBEPBDXZ 100172ca f   qt-mt323:qt-mt323.dll
 0001:000162d0       ?className@QPopupMenu@@UBEPBDXZ 100172d0 f   qt-mt323:qt-mt323.dll
 0001:000162d6       ?className@QToolBar@@UBEPBDXZ 100172d6 f   qt-mt323:qt-mt323.dll
 0001:000162dc       ?clear@QToolBar@@UAEXXZ    100172dc f   qt-mt323:qt-mt323.dll
 0001:000162e2       ?closeEvent@QPopupMenu@@MAEXPAVQCloseEvent@@@Z 100172e2 f   qt-mt323:qt-mt323.dll
 0001:000162e8       ?contextMenuEvent@QDockWindow@@MAEXPAVQContextMenuEvent@@@Z 100172e8 f   qt-mt323:qt-mt323.dll
 0001:000162ee       ?customWhatsThis@QPopupMenu@@UBE_NXZ 100172ee f   qt-mt323:qt-mt323.dll
 0001:000162f4       ?dock@QDockWindow@@UAEXXZ  100172f4 f   qt-mt323:qt-mt323.dll
 0001:000162fa       ?drawContents@QDockWindow@@MAEXPAVQPainter@@@Z 100172fa f   qt-mt323:qt-mt323.dll
 0001:00016300       ?drawContents@QPopupMenu@@MAEXPAVQPainter@@@Z 10017300 f   qt-mt323:qt-mt323.dll
 0001:00016306       ?drawFrame@QDockWindow@@MAEXPAVQPainter@@@Z 10017306 f   qt-mt323:qt-mt323.dll
 0001:0001630c       ?enabledChange@QPopupMenu@@MAEX_N@Z 1001730c f   qt-mt323:qt-mt323.dll
 0001:00016312       ?event@QDockWindow@@MAE_NPAVQEvent@@@Z 10017312 f   qt-mt323:qt-mt323.dll
 0001:00016318       ?event@QToolBar@@UAE_NPAVQEvent@@@Z 10017318 f   qt-mt323:qt-mt323.dll
 0001:0001631e       ?eventFilter@QDockWindow@@UAE_NPAVQObject@@PAVQEvent@@@Z 1001731e f   qt-mt323:qt-mt323.dll
 0001:00016324       ?focusInEvent@QPopupMenu@@MAEXPAVQFocusEvent@@@Z 10017324 f   qt-mt323:qt-mt323.dll
 0001:0001632a       ?focusNextPrevChild@QPopupMenu@@MAE_N_N@Z 1001732a f   qt-mt323:qt-mt323.dll
 0001:00016330       ?focusOutEvent@QPopupMenu@@MAEXPAVQFocusEvent@@@Z 10017330 f   qt-mt323:qt-mt323.dll
 0001:00016336       ?frameChanged@QPopupMenu@@EAEXXZ 10017336 f   qt-mt323:qt-mt323.dll
 0001:0001633c       ?hide@QPopupMenu@@UAEXXZ   1001733c f   qt-mt323:qt-mt323.dll
 0001:00016342       ?hide@QToolBar@@UAEXXZ     10017342 f   qt-mt323:qt-mt323.dll
 0001:00016348       ?hideEvent@QDockWindow@@MAEXPAVQHideEvent@@@Z 10017348 f   qt-mt323:qt-mt323.dll
 0001:0001634e       ?keyPressEvent@QPopupMenu@@MAEXPAVQKeyEvent@@@Z 1001734e f   qt-mt323:qt-mt323.dll
 0001:00016354       ?leaveEvent@QPopupMenu@@MAEXPAVQEvent@@@Z 10017354 f   qt-mt323:qt-mt323.dll
 0001:0001635a       ?menuContentsChanged@QPopupMenu@@EAEXXZ 1001735a f   qt-mt323:qt-mt323.dll
 0001:00016360       ?menuDelPopup@QPopupMenu@@EAEXPAV1@@Z 10017360 f   qt-mt323:qt-mt323.dll
 0001:00016366       ?menuInsPopup@QPopupMenu@@EAEXPAV1@@Z 10017366 f   qt-mt323:qt-mt323.dll
 0001:0001636c       ?menuStateChanged@QPopupMenu@@EAEXXZ 1001736c f   qt-mt323:qt-mt323.dll
 0001:00016372       ?metaObject@QAction@@UBEPAVQMetaObject@@XZ 10017372 f   qt-mt323:qt-mt323.dll
 0001:00016378       ?metaObject@QDockWindow@@UBEPAVQMetaObject@@XZ 10017378 f   qt-mt323:qt-mt323.dll
 0001:0001637e       ?metaObject@QPopupMenu@@UBEPAVQMetaObject@@XZ 1001737e f   qt-mt323:qt-mt323.dll
 0001:00016384       ?metaObject@QToolBar@@UBEPAVQMetaObject@@XZ 10017384 f   qt-mt323:qt-mt323.dll
 0001:0001638a       ?minimumSizeHint@QDockWindow@@UBE?AVQSize@@XZ 1001738a f   qt-mt323:qt-mt323.dll
 0001:00016390       ?minimumSizeHint@QToolBar@@UBE?AVQSize@@XZ 10017390 f   qt-mt323:qt-mt323.dll
 0001:00016396       ?mouseMoveEvent@QPopupMenu@@MAEXPAVQMouseEvent@@@Z 10017396 f   qt-mt323:qt-mt323.dll
 0001:0001639c       ?mousePressEvent@QPopupMenu@@MAEXPAVQMouseEvent@@@Z 1001739c f   qt-mt323:qt-mt323.dll
 0001:000163a2       ?mouseReleaseEvent@QPopupMenu@@MAEXPAVQMouseEvent@@@Z 100173a2 f   qt-mt323:qt-mt323.dll
 0001:000163a8       ?paintEvent@QPopupMenu@@MAEXPAVQPaintEvent@@@Z 100173a8 f   qt-mt323:qt-mt323.dll
 0001:000163ae       ?qt_cast@QAction@@UAEPAXPBD@Z 100173ae f   qt-mt323:qt-mt323.dll
 0001:000163b4       ?qt_cast@QDockWindow@@UAEPAXPBD@Z 100173b4 f   qt-mt323:qt-mt323.dll
 0001:000163ba       ?qt_cast@QPopupMenu@@UAEPAXPBD@Z 100173ba f   qt-mt323:qt-mt323.dll
 0001:000163c0       ?qt_cast@QToolBar@@UAEPAXPBD@Z 100173c0 f   qt-mt323:qt-mt323.dll
 0001:000163c6       ?qt_emit@QAction@@UAE_NHPAUQUObject@@@Z 100173c6 f   qt-mt323:qt-mt323.dll
 0001:000163cc       ?qt_emit@QDockWindow@@UAE_NHPAUQUObject@@@Z 100173cc f   qt-mt323:qt-mt323.dll
 0001:000163d2       ?qt_emit@QPopupMenu@@UAE_NHPAUQUObject@@@Z 100173d2 f   qt-mt323:qt-mt323.dll
 0001:000163d8       ?qt_emit@QToolBar@@UAE_NHPAUQUObject@@@Z 100173d8 f   qt-mt323:qt-mt323.dll
 0001:000163de       ?qt_invoke@QAction@@UAE_NHPAUQUObject@@@Z 100173de f   qt-mt323:qt-mt323.dll
 0001:000163e4       ?qt_invoke@QDockWindow@@UAE_NHPAUQUObject@@@Z 100173e4 f   qt-mt323:qt-mt323.dll
 0001:000163ea       ?qt_invoke@QPopupMenu@@UAE_NHPAUQUObject@@@Z 100173ea f   qt-mt323:qt-mt323.dll
 0001:000163f0       ?qt_invoke@QToolBar@@UAE_NHPAUQUObject@@@Z 100173f0 f   qt-mt323:qt-mt323.dll
 0001:000163f6       ?qt_property@QAction@@UAE_NHHPAVQVariant@@@Z 100173f6 f   qt-mt323:qt-mt323.dll
 0001:000163fc       ?qt_property@QDockWindow@@UAE_NHHPAVQVariant@@@Z 100173fc f   qt-mt323:qt-mt323.dll
 0001:00016402       ?qt_property@QPopupMenu@@UAE_NHHPAVQVariant@@@Z 10017402 f   qt-mt323:qt-mt323.dll
 0001:00016408       ?qt_property@QToolBar@@UAE_NHHPAVQVariant@@@Z 10017408 f   qt-mt323:qt-mt323.dll
 0001:0001640e       ?read@QGDict@@MAEAAVQDataStream@@AAV2@AAPAX@Z 1001740e f   qt-mt323:qt-mt323.dll
 0001:00016414       ?removeFrom@QAction@@UAE_NPAVQWidget@@@Z 10017414 f   qt-mt323:qt-mt323.dll
 0001:0001641a       ?resizeEvent@QDockWindow@@MAEXPAVQResizeEvent@@@Z 1001741a f   qt-mt323:qt-mt323.dll
 0001:00016420       ?resizeEvent@QToolBar@@MAEXPAVQResizeEvent@@@Z 10017420 f   qt-mt323:qt-mt323.dll
 0001:00016426       ?setAccel@QAction@@UAEXABVQKeySequence@@@Z 10017426 f   qt-mt323:qt-mt323.dll
 0001:0001642c       ?setActiveItem@QPopupMenu@@UAEXH@Z 1001742c f   qt-mt323:qt-mt323.dll
 0001:00016432       ?setCaption@QDockWindow@@UAEXABVQString@@@Z 10017432 f   qt-mt323:qt-mt323.dll
 0001:00016438       ?setCheckable@QPopupMenu@@UAEX_N@Z 10017438 f   qt-mt323:qt-mt323.dll
 0001:0001643e       ?setCloseMode@QDockWindow@@UAEXH@Z 1001743e f   qt-mt323:qt-mt323.dll
 0001:00016444       ?setEnabled@QAction@@UAEX_N@Z 10017444 f   qt-mt323:qt-mt323.dll
 0001:0001644a       ?setFirstItemActive@QPopupMenu@@EAEXXZ 1001744a f   qt-mt323:qt-mt323.dll
 0001:00016450       ?setFixedExtentHeight@QDockWindow@@UAEXH@Z 10017450 f   qt-mt323:qt-mt323.dll
 0001:00016456       ?setFixedExtentWidth@QDockWindow@@UAEXH@Z 10017456 f   qt-mt323:qt-mt323.dll
 0001:0001645c       ?setFont@QPopupMenu@@UAEXABVQFont@@@Z 1001745c f   qt-mt323:qt-mt323.dll
 0001:00016462       ?setHorizontallyStretchable@QDockWindow@@UAEX_N@Z 10017462 f   qt-mt323:qt-mt323.dll
 0001:00016468       ?setIconSet@QAction@@UAEXABVQIconSet@@@Z 10017468 f   qt-mt323:qt-mt323.dll
 0001:0001646e       ?setId@QMenuData@@UAEXHH@Z 1001746e f   qt-mt323:qt-mt323.dll
 0001:00016474       ?setLabel@QToolBar@@UAEXABVQString@@@Z 10017474 f   qt-mt323:qt-mt323.dll
 0001:0001647a       ?setMenuText@QAction@@UAEXABVQString@@@Z 1001747a f   qt-mt323:qt-mt323.dll
 0001:00016480       ?setMinimumSize@QToolBar@@UAEXHH@Z 10017480 f   qt-mt323:qt-mt323.dll
 0001:00016486       ?setMovingEnabled@QDockWindow@@UAEX_N@Z 10017486 f   qt-mt323:qt-mt323.dll
 0001:0001648c       ?setNewLine@QDockWindow@@UAEX_N@Z 1001748c f   qt-mt323:qt-mt323.dll
 0001:00016492       ?setOffset@QDockWindow@@UAEXH@Z 10017492 f   qt-mt323:qt-mt323.dll
 0001:00016498       ?setOn@QAction@@UAEX_N@Z   10017498 f   qt-mt323:qt-mt323.dll
 0001:0001649e       ?setOpaqueMoving@QDockWindow@@UAEX_N@Z 1001749e f   qt-mt323:qt-mt323.dll
 0001:000164a4       ?setOrientation@QDockWindow@@UAEXW4Orientation@Qt@@@Z 100174a4 f   qt-mt323:qt-mt323.dll
 0001:000164aa       ?setOrientation@QToolBar@@UAEXW4Orientation@Qt@@@Z 100174aa f   qt-mt323:qt-mt323.dll
 0001:000164b0       ?setResizeEnabled@QDockWindow@@UAEX_N@Z 100174b0 f   qt-mt323:qt-mt323.dll
 0001:000164b6       ?setStatusTip@QAction@@UAEXABVQString@@@Z 100174b6 f   qt-mt323:qt-mt323.dll
 0001:000164bc       ?setStretchableWidget@QToolBar@@UAEXPAVQWidget@@@Z 100174bc f   qt-mt323:qt-mt323.dll
 0001:000164c2       ?setText@QAction@@UAEXABVQString@@@Z 100174c2 f   qt-mt323:qt-mt323.dll
 0001:000164c8       ?setToggleAction@QAction@@UAEX_N@Z 100174c8 f   qt-mt323:qt-mt323.dll
 0001:000164ce       ?setToolTip@QAction@@UAEXABVQString@@@Z 100174ce f   qt-mt323:qt-mt323.dll
 0001:000164d4       ?setVerticallyStretchable@QDockWindow@@UAEX_N@Z 100174d4 f   qt-mt323:qt-mt323.dll
 0001:000164da       ?setWhatsThis@QAction@@UAEXABVQString@@@Z 100174da f   qt-mt323:qt-mt323.dll
 0001:000164e0       ?setWidget@QDockWindow@@UAEXPAVQWidget@@@Z 100174e0 f   qt-mt323:qt-mt323.dll
 0001:000164e6       ?show@QPopupMenu@@UAEXXZ   100174e6 f   qt-mt323:qt-mt323.dll
 0001:000164ec       ?show@QToolBar@@UAEXXZ     100174ec f   qt-mt323:qt-mt323.dll
 0001:000164f2       ?showEvent@QDockWindow@@MAEXPAVQShowEvent@@@Z 100174f2 f   qt-mt323:qt-mt323.dll
 0001:000164f8       ?sizeHint@QDockWindow@@UBE?AVQSize@@XZ 100174f8 f   qt-mt323:qt-mt323.dll
 0001:000164fe       ?sizeHint@QPopupMenu@@UBE?AVQSize@@XZ 100174fe f   qt-mt323:qt-mt323.dll
 0001:00016504       ?styleChange@QPopupMenu@@MAEXAAVQStyle@@@Z 10017504 f   qt-mt323:qt-mt323.dll
 0001:0001650a       ?styleChange@QToolBar@@MAEXAAVQStyle@@@Z 1001750a f   qt-mt323:qt-mt323.dll
 0001:00016510       ?timerEvent@QPopupMenu@@MAEXPAVQTimerEvent@@@Z 10017510 f   qt-mt323:qt-mt323.dll
 0001:00016516       ?undock@QDockWindow@@UAEXPAVQWidget@@@Z 10017516 f   qt-mt323:qt-mt323.dll
 0001:0001651c       ?undock@QDockWindow@@UAEXXZ 1001751c f   qt-mt323:qt-mt323.dll
 0001:00016522       ?updateItem@QPopupMenu@@UAEXH@Z 10017522 f   qt-mt323:qt-mt323.dll
 0001:00016528       ?write@QGDict@@MBEAAVQDataStream@@AAV2@PAX@Z 10017528 f   qt-mt323:qt-mt323.dll
 0001:0001652e       ?alignment@QTableItem@@UBEHXZ 1001752e f   qt-mt323:qt-mt323.dll
 0001:00016534       ?createEditor@QCheckTableItem@@UBEPAVQWidget@@XZ 10017534 f   qt-mt323:qt-mt323.dll
 0001:0001653a       ?key@QTableItem@@UBE?AVQString@@XZ 1001753a f   qt-mt323:qt-mt323.dll
 0001:00016540       ?paint@QCheckTableItem@@UAEXPAVQPainter@@ABVQColorGroup@@ABVQRect@@_N@Z 10017540 f   qt-mt323:qt-mt323.dll
 0001:00016546       ?pixmap@QTableItem@@UBE?AVQPixmap@@XZ 10017546 f   qt-mt323:qt-mt323.dll
 0001:0001654c       ?rtti@QCheckTableItem@@UBEHXZ 1001754c f   qt-mt323:qt-mt323.dll
 0001:00016552       ?setChecked@QCheckTableItem@@UAEX_N@Z 10017552 f   qt-mt323:qt-mt323.dll
 0001:00016558       ?setCol@QTableItem@@UAEXH@Z 10017558 f   qt-mt323:qt-mt323.dll
 0001:0001655e       ?setContentFromEditor@QCheckTableItem@@UAEXPAVQWidget@@@Z 1001755e f   qt-mt323:qt-mt323.dll
 0001:00016564       ?setEnabled@QTableItem@@UAEX_N@Z 10017564 f   qt-mt323:qt-mt323.dll
 0001:0001656a       ?setPixmap@QTableItem@@UAEXABVQPixmap@@@Z 1001756a f   qt-mt323:qt-mt323.dll
 0001:00016570       ?setReplaceable@QTableItem@@UAEX_N@Z 10017570 f   qt-mt323:qt-mt323.dll
 0001:00016576       ?setRow@QTableItem@@UAEXH@Z 10017576 f   qt-mt323:qt-mt323.dll
 0001:0001657c       ?setSpan@QTableItem@@UAEXHH@Z 1001757c f   qt-mt323:qt-mt323.dll
 0001:00016582       ?setText@QCheckTableItem@@UAEXABVQString@@@Z 10017582 f   qt-mt323:qt-mt323.dll
 0001:00016588       ?setWordWrap@QTableItem@@UAEX_N@Z 10017588 f   qt-mt323:qt-mt323.dll
 0001:0001658e       ?sizeHint@QCheckTableItem@@UBE?AVQSize@@XZ 1001758e f   qt-mt323:qt-mt323.dll
 0001:00016594       ?text@QTableItem@@UBE?AVQString@@XZ 10017594 f   qt-mt323:qt-mt323.dll
 0001:0001659a       ?accept@QDialog@@MAEXXZ    1001759a f   qt-mt323:qt-mt323.dll
 0001:000165a0       ?closeEvent@QDialog@@MAEXPAVQCloseEvent@@@Z 100175a0 f   qt-mt323:qt-mt323.dll
 0001:000165a6       ?contextMenuEvent@QDialog@@MAEXPAVQContextMenuEvent@@@Z 100175a6 f   qt-mt323:qt-mt323.dll
 0001:000165ac       ?done@QDialog@@MAEXH@Z     100175ac f   qt-mt323:qt-mt323.dll
 0001:000165b2       ?eventFilter@QDialog@@MAE_NPAVQObject@@PAVQEvent@@@Z 100175b2 f   qt-mt323:qt-mt323.dll
 0001:000165b8       ?hide@QDialog@@UAEXXZ      100175b8 f   qt-mt323:qt-mt323.dll
 0001:000165be       ?keyPressEvent@QDialog@@MAEXPAVQKeyEvent@@@Z 100175be f   qt-mt323:qt-mt323.dll
 0001:000165c4       ?minimumSizeHint@QDialog@@UBE?AVQSize@@XZ 100175c4 f   qt-mt323:qt-mt323.dll
 0001:000165ca       ?move@QDialog@@UAEXHH@Z    100175ca f   qt-mt323:qt-mt323.dll
 0001:000165d0       ?reject@QDialog@@MAEXXZ    100175d0 f   qt-mt323:qt-mt323.dll
 0001:000165d6       ?resize@QDialog@@UAEXHH@Z  100175d6 f   qt-mt323:qt-mt323.dll
 0001:000165dc       ?resizeEvent@QDialog@@MAEXPAVQResizeEvent@@@Z 100175dc f   qt-mt323:qt-mt323.dll
 0001:000165e2       ?setGeometry@QDialog@@UAEXABVQRect@@@Z 100175e2 f   qt-mt323:qt-mt323.dll
 0001:000165e8       ?setGeometry@QDialog@@UAEXHHHH@Z 100175e8 f   qt-mt323:qt-mt323.dll
 0001:000165ee       ?show@QDialog@@UAEXXZ      100175ee f   qt-mt323:qt-mt323.dll
 0001:000165f4       ?sizeHint@QDialog@@UBE?AVQSize@@XZ 100175f4 f   qt-mt323:qt-mt323.dll
 0001:000165fa       ?className@QComboBox@@UBEPBDXZ 100175fa f   qt-mt323:qt-mt323.dll
 0001:00016600       ?eventFilter@QComboBox@@UAE_NPAVQObject@@PAVQEvent@@@Z 10017600 f   qt-mt323:qt-mt323.dll
 0001:00016606       ?focusInEvent@QComboBox@@MAEXPAVQFocusEvent@@@Z 10017606 f   qt-mt323:qt-mt323.dll
 0001:0001660c       ?focusOutEvent@QComboBox@@MAEXPAVQFocusEvent@@@Z 1001760c f   qt-mt323:qt-mt323.dll
 0001:00016612       ?keyPressEvent@QComboBox@@MAEXPAVQKeyEvent@@@Z 10017612 f   qt-mt323:qt-mt323.dll
 0001:00016618       ?metaObject@QComboBox@@UBEPAVQMetaObject@@XZ 10017618 f   qt-mt323:qt-mt323.dll
 0001:0001661e       ?mouseDoubleClickEvent@QComboBox@@MAEXPAVQMouseEvent@@@Z 1001761e f   qt-mt323:qt-mt323.dll
 0001:00016624       ?mouseMoveEvent@QComboBox@@MAEXPAVQMouseEvent@@@Z 10017624 f   qt-mt323:qt-mt323.dll
 0001:0001662a       ?mousePressEvent@QComboBox@@MAEXPAVQMouseEvent@@@Z 1001762a f   qt-mt323:qt-mt323.dll
 0001:00016630       ?mouseReleaseEvent@QComboBox@@MAEXPAVQMouseEvent@@@Z 10017630 f   qt-mt323:qt-mt323.dll
 0001:00016636       ?paint@QTableItem@@UAEXPAVQPainter@@ABVQColorGroup@@ABVQRect@@_N@Z 10017636 f   qt-mt323:qt-mt323.dll
 0001:0001663c       ?paintEvent@QComboBox@@MAEXPAVQPaintEvent@@@Z 1001763c f   qt-mt323:qt-mt323.dll
 0001:00016642       ?popup@QComboBox@@UAEXXZ   10017642 f   qt-mt323:qt-mt323.dll
 0001:00016648       ?qt_cast@QComboBox@@UAEPAXPBD@Z 10017648 f   qt-mt323:qt-mt323.dll
 0001:0001664e       ?qt_emit@QComboBox@@UAE_NHPAUQUObject@@@Z 1001764e f   qt-mt323:qt-mt323.dll
 0001:00016654       ?qt_invoke@QComboBox@@UAE_NHPAUQUObject@@@Z 10017654 f   qt-mt323:qt-mt323.dll
 0001:0001665a       ?qt_property@QComboBox@@UAE_NHHPAVQVariant@@@Z 1001765a f   qt-mt323:qt-mt323.dll
 0001:00016660       ?resizeEvent@QComboBox@@MAEXPAVQResizeEvent@@@Z 10017660 f   qt-mt323:qt-mt323.dll
 0001:00016666       ?rtti@QTableItem@@UBEHXZ   10017666 f   qt-mt323:qt-mt323.dll
 0001:0001666c       ?setAutoCompletion@QComboBox@@UAEX_N@Z 1001766c f   qt-mt323:qt-mt323.dll
 0001:00016672       ?setAutoResize@QComboBox@@UAEX_N@Z 10017672 f   qt-mt323:qt-mt323.dll
 0001:00016678       ?setCurrentItem@QComboBox@@UAEXH@Z 10017678 f   qt-mt323:qt-mt323.dll
 0001:0001667e       ?setCurrentText@QComboBox@@UAEXABVQString@@@Z 1001767e f   qt-mt323:qt-mt323.dll
 0001:00016684       ?setEditText@QComboBox@@UAEXABVQString@@@Z 10017684 f   qt-mt323:qt-mt323.dll
 0001:0001668a       ?setEnabled@QComboBox@@UAEX_N@Z 1001768a f   qt-mt323:qt-mt323.dll
 0001:00016690       ?setFont@QComboBox@@UAEXABVQFont@@@Z 10017690 f   qt-mt323:qt-mt323.dll
 0001:00016696       ?setInsertionPolicy@QComboBox@@UAEXW4Policy@1@@Z 10017696 f   qt-mt323:qt-mt323.dll
 0001:0001669c       ?setLineEdit@QComboBox@@UAEXPAVQLineEdit@@@Z 1001769c f   qt-mt323:qt-mt323.dll
 0001:000166a2       ?setListBox@QComboBox@@UAEXPAVQListBox@@@Z 100176a2 f   qt-mt323:qt-mt323.dll
 0001:000166a8       ?setMaxCount@QComboBox@@UAEXH@Z 100176a8 f   qt-mt323:qt-mt323.dll
 0001:000166ae       ?setPalette@QComboBox@@UAEXABVQPalette@@@Z 100176ae f   qt-mt323:qt-mt323.dll
 0001:000166b4       ?setSizeLimit@QComboBox@@UAEXH@Z 100176b4 f   qt-mt323:qt-mt323.dll
 0001:000166ba       ?setText@QTableItem@@UAEXABVQString@@@Z 100176ba f   qt-mt323:qt-mt323.dll
 0001:000166c0       ?setValidator@QComboBox@@UAEXPBVQValidator@@@Z 100176c0 f   qt-mt323:qt-mt323.dll
 0001:000166c6       ?sizeHint@QComboBox@@UBE?AVQSize@@XZ 100176c6 f   qt-mt323:qt-mt323.dll
 0001:000166cc       ?sizeHint@QTableItem@@UBE?AVQSize@@XZ 100176cc f   qt-mt323:qt-mt323.dll
 0001:000166d2       ?styleChange@QComboBox@@MAEXAAVQStyle@@@Z 100176d2 f   qt-mt323:qt-mt323.dll
 0001:000166d8       ?updateMask@QComboBox@@MAEXXZ 100176d8 f   qt-mt323:qt-mt323.dll
 0001:000166de       ?wheelEvent@QComboBox@@MAEXPAVQWheelEvent@@@Z 100176de f   qt-mt323:qt-mt323.dll
 0001:000166e4       ?className@QCheckBox@@UBEPBDXZ 100176e4 f   qt-mt323:qt-mt323.dll
 0001:000166ea       ?drawButton@QCheckBox@@MAEXPAVQPainter@@@Z 100176ea f   qt-mt323:qt-mt323.dll
 0001:000166f0       ?drawButtonLabel@QCheckBox@@MAEXPAVQPainter@@@Z 100176f0 f   qt-mt323:qt-mt323.dll
 0001:000166f6       ?focusInEvent@QButton@@MAEXPAVQFocusEvent@@@Z 100176f6 f   qt-mt323:qt-mt323.dll
 0001:000166fc       ?focusOutEvent@QButton@@MAEXPAVQFocusEvent@@@Z 100176fc f   qt-mt323:qt-mt323.dll
 0001:00016702       ?hitButton@QCheckBox@@MBE_NABVQPoint@@@Z 10017702 f   qt-mt323:qt-mt323.dll
 0001:00016708       ?metaObject@QCheckBox@@UBEPAVQMetaObject@@XZ 10017708 f   qt-mt323:qt-mt323.dll
 0001:0001670e       ?qt_cast@QCheckBox@@UAEPAXPBD@Z 1001770e f   qt-mt323:qt-mt323.dll
 0001:00016714       ?qt_emit@QCheckBox@@UAE_NHPAUQUObject@@@Z 10017714 f   qt-mt323:qt-mt323.dll
 0001:0001671a       ?qt_invoke@QCheckBox@@UAE_NHPAUQUObject@@@Z 1001771a f   qt-mt323:qt-mt323.dll
 0001:00016720       ?qt_property@QCheckBox@@UAE_NHHPAVQVariant@@@Z 10017720 f   qt-mt323:qt-mt323.dll
 0001:00016726       ?resizeEvent@QCheckBox@@MAEXPAVQResizeEvent@@@Z 10017726 f   qt-mt323:qt-mt323.dll
 0001:0001672c       ?sizeHint@QCheckBox@@UBE?AVQSize@@XZ 1001772c f   qt-mt323:qt-mt323.dll
 0001:00016732       ?updateMask@QCheckBox@@MAEXXZ 10017732 f   qt-mt323:qt-mt323.dll
 0001:00016738       ?addTab@QTabWidget@@UAEXPAVQWidget@@ABVQIconSet@@ABVQString@@@Z 10017738 f   qt-mt323:qt-mt323.dll
 0001:0001673e       ?addTab@QTabWidget@@UAEXPAVQWidget@@ABVQString@@@Z 1001773e f   qt-mt323:qt-mt323.dll
 0001:00016744       ?addTab@QTabWidget@@UAEXPAVQWidget@@PAVQTab@@@Z 10017744 f   qt-mt323:qt-mt323.dll
 0001:0001674a       ?className@QTabWidget@@UBEPBDXZ 1001774a f   qt-mt323:qt-mt323.dll
 0001:00016750       ?eventFilter@QTabWidget@@MAE_NPAVQObject@@PAVQEvent@@@Z 10017750 f   qt-mt323:qt-mt323.dll
 0001:00016756       ?insertTab@QTabWidget@@UAEXPAVQWidget@@ABVQIconSet@@ABVQString@@H@Z 10017756 f   qt-mt323:qt-mt323.dll
 0001:0001675c       ?insertTab@QTabWidget@@UAEXPAVQWidget@@ABVQString@@H@Z 1001775c f   qt-mt323:qt-mt323.dll
 0001:00016762       ?insertTab@QTabWidget@@UAEXPAVQWidget@@PAVQTab@@H@Z 10017762 f   qt-mt323:qt-mt323.dll
 0001:00016768       ?metaObject@QTabWidget@@UBEPAVQMetaObject@@XZ 10017768 f   qt-mt323:qt-mt323.dll
 0001:0001676e       ?minimumSizeHint@QTabWidget@@UBE?AVQSize@@XZ 1001776e f   qt-mt323:qt-mt323.dll
 0001:00016774       ?qt_cast@QTabWidget@@UAEPAXPBD@Z 10017774 f   qt-mt323:qt-mt323.dll
 0001:0001677a       ?qt_emit@QTabWidget@@UAE_NHPAUQUObject@@@Z 1001777a f   qt-mt323:qt-mt323.dll
 0001:00016780       ?qt_invoke@QTabWidget@@UAE_NHPAUQUObject@@@Z 10017780 f   qt-mt323:qt-mt323.dll
 0001:00016786       ?qt_property@QTabWidget@@UAE_NHHPAVQVariant@@@Z 10017786 f   qt-mt323:qt-mt323.dll
 0001:0001678c       ?removePage@QTabWidget@@UAEXPAVQWidget@@@Z 1001778c f   qt-mt323:qt-mt323.dll
 0001:00016792       ?resizeEvent@QTabWidget@@MAEXPAVQResizeEvent@@@Z 10017792 f   qt-mt323:qt-mt323.dll
 0001:00016798       ?showEvent@QTabWidget@@MAEXPAVQShowEvent@@@Z 10017798 f   qt-mt323:qt-mt323.dll
 0001:0001679e       ?showPage@QTabWidget@@UAEXPAVQWidget@@@Z 1001779e f   qt-mt323:qt-mt323.dll
 0001:000167a4       ?sizeHint@QTabWidget@@UBE?AVQSize@@XZ 100177a4 f   qt-mt323:qt-mt323.dll
 0001:000167aa       ?styleChange@QTabWidget@@MAEXAAVQStyle@@@Z 100177aa f   qt-mt323:qt-mt323.dll
 0001:000167b0       ?updateMask@QTabWidget@@MAEXXZ 100177b0 f   qt-mt323:qt-mt323.dll
 0001:000167b6       ?className@QButtonGroup@@UBEPBDXZ 100177b6 f   qt-mt323:qt-mt323.dll
 0001:000167bc       ?className@QRadioButton@@UBEPBDXZ 100177bc f   qt-mt323:qt-mt323.dll
 0001:000167c2       ?drawButton@QRadioButton@@MAEXPAVQPainter@@@Z 100177c2 f   qt-mt323:qt-mt323.dll
 0001:000167c8       ?drawButtonLabel@QRadioButton@@MAEXPAVQPainter@@@Z 100177c8 f   qt-mt323:qt-mt323.dll
 0001:000167ce       ?event@QButtonGroup@@MAE_NPAVQEvent@@@Z 100177ce f   qt-mt323:qt-mt323.dll
 0001:000167d4       ?hitButton@QRadioButton@@MBE_NABVQPoint@@@Z 100177d4 f   qt-mt323:qt-mt323.dll
 0001:000167da       ?metaObject@QButtonGroup@@UBEPAVQMetaObject@@XZ 100177da f   qt-mt323:qt-mt323.dll
 0001:000167e0       ?metaObject@QRadioButton@@UBEPAVQMetaObject@@XZ 100177e0 f   qt-mt323:qt-mt323.dll
 0001:000167e6       ?moveFocus@QButtonGroup@@UAEXH@Z 100177e6 f   qt-mt323:qt-mt323.dll
 0001:000167ec       ?qt_cast@QButtonGroup@@UAEPAXPBD@Z 100177ec f   qt-mt323:qt-mt323.dll
 0001:000167f2       ?qt_cast@QRadioButton@@UAEPAXPBD@Z 100177f2 f   qt-mt323:qt-mt323.dll
 0001:000167f8       ?qt_emit@QButtonGroup@@UAE_NHPAUQUObject@@@Z 100177f8 f   qt-mt323:qt-mt323.dll
 0001:000167fe       ?qt_emit@QRadioButton@@UAE_NHPAUQUObject@@@Z 100177fe f   qt-mt323:qt-mt323.dll
 0001:00016804       ?qt_invoke@QButtonGroup@@UAE_NHPAUQUObject@@@Z 10017804 f   qt-mt323:qt-mt323.dll
 0001:0001680a       ?qt_invoke@QRadioButton@@UAE_NHPAUQUObject@@@Z 1001780a f   qt-mt323:qt-mt323.dll
 0001:00016810       ?qt_property@QButtonGroup@@UAE_NHHPAVQVariant@@@Z 10017810 f   qt-mt323:qt-mt323.dll
 0001:00016816       ?qt_property@QRadioButton@@UAE_NHHPAVQVariant@@@Z 10017816 f   qt-mt323:qt-mt323.dll
 0001:0001681c       ?resizeEvent@QRadioButton@@MAEXPAVQResizeEvent@@@Z 1001781c f   qt-mt323:qt-mt323.dll
 0001:00016822       ?setButton@QButtonGroup@@UAEXH@Z 10017822 f   qt-mt323:qt-mt323.dll
 0001:00016828       ?setChecked@QRadioButton@@UAEX_N@Z 10017828 f   qt-mt323:qt-mt323.dll
 0001:0001682e       ?setExclusive@QButtonGroup@@UAEX_N@Z 1001782e f   qt-mt323:qt-mt323.dll
 0001:00016834       ?setRadioButtonExclusive@QButtonGroup@@UAEX_N@Z 10017834 f   qt-mt323:qt-mt323.dll
 0001:0001683a       ?sizeHint@QRadioButton@@UBE?AVQSize@@XZ 1001783a f   qt-mt323:qt-mt323.dll
 0001:00016840       ?updateMask@QRadioButton@@MAEXXZ 10017840 f   qt-mt323:qt-mt323.dll
 0001:00016850       ??0configFile@@QAE@PAVpluginBase@@VQString@@_N@Z 10017850 f   pluginBase:configFile.obj
 0001:00016940       ??1configFile@@UAE@XZ      10017940 f i pluginBase:configFile.obj
 0001:000169c0       ??BconfigFile@@QAE?AVQFileInfo@@XZ 100179c0 f   pluginBase:configFile.obj
 0001:00016a30       ??_GconfigFile@@UAEPAXI@Z  10017a30 f i pluginBase:configFile.obj
 0001:00016a30       ??_EconfigFile@@UAEPAXI@Z  10017a30 f i pluginBase:configFile.obj
 0001:00016ac0       ?checkout@configFile@@QAE_N_N@Z 10017ac0 f   pluginBase:configFile.obj
 0001:00016b70       ?dirList@configFile@@QAE_NAAVQStringList@@@Z 10017b70 f   pluginBase:configFile.obj
 0001:00016de0       ?download@configFile@@QAE_N_N@Z 10017de0 f   pluginBase:configFile.obj
 0001:00016e90       ?getLocalPath@configFile@@QAE?AVQString@@XZ 10017e90 f   pluginBase:configFile.obj
 0001:00016f70       ?getModTime@configFile@@QAE?AVQDateTime@@XZ 10017f70 f   pluginBase:configFile.obj
 0001:00017060       ?isPending@configFile@@QAE_NH@Z 10018060 f i pluginBase:configFile.obj
 0001:000170b0       ?lock@configFile@@QAE_N_N@Z 100180b0 f   pluginBase:configFile.obj
 0001:000171d0       ?metaObject@configFile@@UBEPAVQMetaObject@@XZ 100181d0 f i pluginBase:configFile.obj
 0001:000171e0       ?needsReload@configFile@@QAE_NXZ 100181e0 f   pluginBase:configFile.obj
 0001:00017210       ?rememberModTime@configFile@@QAEXXZ 10018210 f   pluginBase:configFile.obj
 0001:00017240       ?reply@configFile@@MAEXPAVresponse@@@Z 10018240 f   pluginBase:configFile.obj
 0001:00017410       ?sendCommand@configFile@@IAEXVQString@@@Z 10018410 f   pluginBase:configFile.obj
 0001:00017490       ?setClean@configFile@@QAE_NXZ 10018490 f   pluginBase:configFile.obj
 0001:000174e0       ?setDirty@configFile@@QAE_NXZ 100184e0 f   pluginBase:configFile.obj
 0001:00017590       ?timerEvent@configFile@@MAEXPAVQTimerEvent@@@Z 10018590 f   pluginBase:configFile.obj
 0001:00017630       ?unlock@configFile@@QAE_N_N@Z 10018630 f   pluginBase:configFile.obj
 0001:00017740       ?upload@configFile@@QAE_N_N@Z 10018740 f   pluginBase:configFile.obj
 0001:000177f0       ??0?$QMapNode@VQString@@VconfigFile@@@@QAE@ABU0@@Z 100187f0 f i pluginBase:pluginBase.obj
 0001:00017880       ??0?$QMapPrivate@VQString@@VconfigFile@@@@QAE@PBV0@@Z 10018880 f i pluginBase:pluginBase.obj
 0001:000179a0       ??0?$QMapPrivate@VQString@@VconfigFile@@@@QAE@XZ 100189a0 f i pluginBase:pluginBase.obj
 0001:00017a50       ??0pluginBase@@QAE@ABVQString@@00@Z 10018a50 f   pluginBase:pluginBase.obj
 0001:00017b10       ??1?$QMap@VQString@@VconfigFile@@@@QAE@XZ 10018b10 f i pluginBase:pluginBase.obj
 0001:00017b80       ??1?$QMapNode@VQString@@VconfigFile@@@@QAE@XZ 10018b80 f i pluginBase:pluginBase.obj
 0001:00017c10       ??1pluginBase@@UAE@XZ      10018c10 f   pluginBase:pluginBase.obj
 0001:00017e50       ??4configFile@@QAEAAV0@ABV0@@Z 10018e50 f i pluginBase:pluginBase.obj
 0001:00017f00       ??A?$QMap@VQString@@VconfigFile@@@@QAEAAVconfigFile@@ABVQString@@@Z 10018f00 f i pluginBase:pluginBase.obj
 0001:00018015       ??_EpluginBase@@WCI@AEPAXI@Z 10019015 f i pluginBase:pluginBase.obj
 0001:00018020       ??_GpluginBase@@UAEPAXI@Z  10019020 f i pluginBase:pluginBase.obj
 0001:00018020       ??_EpluginBase@@UAEPAXI@Z  10019020 f i pluginBase:pluginBase.obj
 0001:00018050       ?activate@pluginBase@@EAEX_N@Z 10019050 f   pluginBase:pluginBase.obj
 0001:00018090       ?addMenu@pluginBase@@QAEXPAVQPopupMenu@@@Z 10019090 f   pluginBase:pluginBase.obj
 0001:000180a0       ?addToolbar@pluginBase@@QAEXPAVQDockWindow@@@Z 100190a0 f   pluginBase:pluginBase.obj
 0001:000180b0       ?apply@pluginBase@@EAEXXZ  100190b0 f   pluginBase:pluginBase.obj
 0001:000180c0       ?clear@?$QMapPrivate@VQString@@VconfigFile@@@@QAEXPAU?$QMapNode@VQString@@VconfigFile@@@@@Z 100190c0 f i pluginBase:pluginBase.obj
 0001:00018180       ?closeEvent@pluginBase@@EAEXPAVQCloseEvent@@@Z 10019180 f   pluginBase:pluginBase.obj
 0001:000181c0       ?copy@?$QMapPrivate@VQString@@VconfigFile@@@@QAEPAU?$QMapNode@VQString@@VconfigFile@@@@PAU2@@Z 100191c0 f i pluginBase:pluginBase.obj
 0001:00018290       ?dec@?$QMapIterator@VQString@@VconfigFile@@@@AAEHXZ 10019290 f i pluginBase:pluginBase.obj
 0001:000182f0       ?doLoadFile@pluginBase@@QAEXAAVconfigFile@@@Z 100192f0 f   pluginBase:pluginBase.obj
 0001:00018320       ?file@pluginBase@@QAEAAVconfigFile@@VQString@@@Z 10019320 f   pluginBase:pluginBase.obj
 0001:00018470       ?find@?$QMapPrivate@VQString@@VconfigFile@@@@QBE?AV?$QMapConstIterator@VQString@@VconfigFile@@@@ABVQString@@@Z 10019470 f i pluginBase:pluginBase.obj
 0001:000184f0       ?insert@?$QMap@VQString@@VconfigFile@@@@QAE?AV?$QMapIterator@VQString@@VconfigFile@@@@ABVQString@@ABVconfigFile@@_N@Z 100194f0 f i pluginBase:pluginBase.obj
 0001:00018590       ?insert@?$QMapPrivate@VQString@@VconfigFile@@@@QAE?AV?$QMapIterator@VQString@@VconfigFile@@@@PAUQMapNodeBase@@0ABVQString@@@Z 10019590 f i pluginBase:pluginBase.obj
 0001:000186a0       ?insertSingle@?$QMapPrivate@VQString@@VconfigFile@@@@QAE?AV?$QMapIterator@VQString@@VconfigFile@@@@ABVQString@@@Z 100196a0 f i pluginBase:pluginBase.obj
 0001:00018760       ?isDirty@pluginBase@@EAE_NXZ 10019760 f   pluginBase:pluginBase.obj
 0001:00018880       ?saveFile@pluginBase@@MAEXVQString@@@Z 10019880 f i pluginBase:pluginBase.obj
 0001:00018880       ?loadFile@pluginBase@@MAEXVQString@@@Z 10019880 f i pluginBase:pluginBase.obj
 0001:00018890       ?loadModdedFiles@pluginBase@@AAEXXZ 10019890 f   pluginBase:pluginBase.obj
 0001:000189c0       ?menus@pluginBase@@EAE?AVQPopupMenuList@@XZ 100199c0 f   pluginBase:pluginBase.obj
 0001:000189f0       ?metaObject@pluginBase@@UBEPAVQMetaObject@@XZ 100199f0 f i pluginBase:pluginBase.obj
 0001:00018a00       ?relativeName@configFile@@QAE?AVQString@@XZ 10019a00 f i pluginBase:pluginBase.obj
 0001:00018a30       ?releaseAllLocks@pluginBase@@AAEXXZ 10019a30 f   pluginBase:pluginBase.obj
 0001:00018b50       ?reply@pluginBase@@EAEXPAVresponse@@@Z 10019b50 f   pluginBase:pluginBase.obj
 0001:00018b80       ?saveAllFiles@pluginBase@@AAEXXZ 10019b80 f   pluginBase:pluginBase.obj
 0001:00018cb0       ?sendCommand@pluginBase@@AAEXVQString@@0@Z 10019cb0 f   pluginBase:pluginBase.obj
 0001:00018d40       ?toolbars@pluginBase@@EAE?AVQDockWindowList@@XZ 10019d40 f   pluginBase:pluginBase.obj
 0001:00018d70       ?uploadAllFiles@pluginBase@@AAEXXZ 10019d70 f   pluginBase:pluginBase.obj
 0001:00018e90       ?waitForAllFiles@pluginBase@@QAE_NXZ 10019e90 f   pluginBase:pluginBase.obj
 0001:00018fd0       ?className@pluginBase@@UBEPBDXZ 10019fd0 f   pluginBase:moc_pluginBase.obj
 0001:00018fe0       ?command@pluginBase@@IAEXVQString@@0@Z 10019fe0 f   pluginBase:moc_pluginBase.obj
 0001:000190e0       ?qt_cast@pluginBase@@UAEPAXPBD@Z 1001a0e0 f   pluginBase:moc_pluginBase.obj
 0001:00019140       ?qt_emit@pluginBase@@UAE_NHPAUQUObject@@@Z 1001a140 f   pluginBase:moc_pluginBase.obj
 0001:000191e0       ?qt_invoke@pluginBase@@UAE_NHPAUQUObject@@@Z 1001a1e0 f   pluginBase:moc_pluginBase.obj
 0001:000191e0       ?qt_invoke@workstationEditor@@UAE_NHPAUQUObject@@@Z 1001a1e0 f   moc_workstationeditor.obj
 0001:000191f0       ?staticMetaObject@pluginBase@@SAPAVQMetaObject@@XZ 1001a1f0 f   pluginBase:moc_pluginBase.obj
 0001:000192a0       ?className@configFile@@UBEPBDXZ 1001a2a0 f   pluginBase:moc_configFile.obj
 0001:000192b0       ?qt_cast@configFile@@UAEPAXPBD@Z 1001a2b0 f   pluginBase:moc_configFile.obj
 0001:00019310       ?qt_emit@configFile@@UAE_NHPAUQUObject@@@Z 1001a310 f   pluginBase:moc_configFile.obj
 0001:00019320       ?qt_invoke@configFile@@UAE_NHPAUQUObject@@@Z 1001a320 f   pluginBase:moc_configFile.obj
 0001:00019330       ?qt_property@configFile@@UAE_NHHPAVQVariant@@@Z 1001a330 f   pluginBase:moc_configFile.obj
 0001:00019340       ?staticMetaObject@configFile@@SAPAVQMetaObject@@XZ 1001a340 f   pluginBase:moc_configFile.obj
 0001:0001938e       ??3@YAXPAX@Z               1001a38e f   MSVCRT:MSVCR120.dll
 0001:00019394       ??_Etype_info@@UAEPAXI@Z   1001a394 f i MSVCRT:ti_inst.obj
 0001:000193de       @__security_check_cookie@4 1001a3de f   MSVCRT:secchk.obj
 0001:000193ed       __EH_epilog3               1001a3ed f   MSVCRT:ehprolg3.obj
 0001:00019401       __EH_epilog3_GS            1001a401 f   MSVCRT:ehprolg3.obj
 0001:00019410       __EH_prolog3               1001a410 f   MSVCRT:ehprolg3.obj
 0001:00019443       __EH_prolog3_GS            1001a443 f   MSVCRT:ehprolg3.obj
 0001:0001947a       ___CxxFrameHandler3        1001a47a f   MSVCRT:MSVCR120.dll
 0001:00019480       ??2@YAPAXI@Z               1001a480 f   MSVCRT:MSVCR120.dll
 0001:00019490       __chkstk                   1001a490 f   MSVCRT:chkstk.obj
 0001:00019490       __alloca_probe             1001a490 f   MSVCRT:chkstk.obj
 0001:000194bc       __purecall                 1001a4bc f   MSVCRT:MSVCR120.dll
 0001:000194c2       ___atonexitinit            1001a4c2 f   MSVCRT:atonexit.obj
 0001:000194fe       __onexit                   1001a4fe f   MSVCRT:atonexit.obj
 0001:000195a7       _atexit                    1001a5a7 f   MSVCRT:atonexit.obj
 0001:000195bc       ??_L@YGXPAXIHP6EX0@Z1@Z    1001a5bc f   MSVCRT:ehvecctr.obj
 0001:0001961e       ??_M@YGXPAXIHP6EX0@Z@Z     1001a61e f   MSVCRT:ehvecdtr.obj
 0001:0001968d       ?__ArrayUnwind@@YGXPAXIHP6EX0@Z@Z 1001a68d f   MSVCRT:ehvecdtr.obj
 0001:00019737       __CRT_INIT@12              1001a737 f   MSVCRT:crtdll.obj
 0001:0001992e       __DllMainCRTStartup@12     1001a92e f   MSVCRT:crtdll.obj
 0001:00019a84       _getenv                    1001aa84 f   MSVCRT:MSVCR120.dll
 0001:00019a8a       ??1type_info@@UAE@XZ       1001aa8a f   MSVCRT:MSVCR120.dll
 0001:00019a90       ___raise_securityfailure   1001aa90 f   MSVCRT:gs_report.obj
 0001:00019acd       ___report_gsfailure        1001aacd f   MSVCRT:gs_report.obj
 0001:00019bc8       __lock                     1001abc8 f   MSVCRT:MSVCR120.dll
 0001:00019bce       __unlock                   1001abce f   MSVCRT:MSVCR120.dll
 0001:00019bd4       ___dllonexit               1001abd4 f   MSVCRT:MSVCR120.dll
 0001:00019be0       __SEH_prolog4              1001abe0 f   MSVCRT:sehprolg4.obj
 0001:00019c25       __SEH_epilog4              1001ac25 f   MSVCRT:sehprolg4.obj
 0001:00019c39       __except_handler4          1001ac39 f   MSVCRT:chandler4gs.obj
 0001:00019c5c       ?terminate@@YAXXZ          1001ac5c f   MSVCRT:MSVCR120.dll
 0001:00019c62       ___CppXcptFilter           1001ac62 f   MSVCRT:MSVCR120.dll
 0001:00019c68       __amsg_exit                1001ac68 f   MSVCRT:MSVCR120.dll
 0001:00019c70       __FindPESection            1001ac70 f   MSVCRT:pesect.obj
 0001:00019cc0       __IsNonwritableInCurrentImage 1001acc0 f   MSVCRT:pesect.obj
 0001:00019d80       __ValidateImageBase        1001ad80 f   MSVCRT:pesect.obj
 0001:00019db1       ___security_init_cookie    1001adb1 f   MSVCRT:gs_support.obj
 0001:00019e4d       _DllMain@12                1001ae4d f   MSVCRT:dllmain.obj
 0001:00019e6f       __RTC_Initialize           1001ae6f f   MSVCRT:initsect.obj
 0001:00019e8f       __RTC_Terminate            1001ae8f f   MSVCRT:initsect.obj
 0001:00019eb0       __initterm                 1001aeb0 f   MSVCRT:MSVCR120.dll
 0001:00019eb6       __initterm_e               1001aeb6 f   MSVCRT:MSVCR120.dll
 0001:00019ebc       ___clean_type_info_names   1001aebc f   MSVCRT:tncleanup.obj
 0001:00019ec8       __crt_debugger_hook        1001aec8 f   MSVCRT:MSVCR120.dll
 0001:00019ece       ___crtUnhandledException   1001aece f   MSVCRT:MSVCR120.dll
 0001:00019ed4       ___crtTerminateProcess     1001aed4 f   MSVCRT:MSVCR120.dll
 0001:00019eda       __except_handler4_common   1001aeda f   MSVCRT:MSVCR120.dll
 0001:00019ee0       ___clean_type_info_names_internal 1001aee0 f   MSVCRT:MSVCR120.dll
 0001:00019ee6       _IsProcessorFeaturePresent@4 1001aee6 f   kernel32:KERNEL32.dll
 0002:00000000       __imp__DisableThreadLibraryCalls@4 10020000     kernel32:KERNEL32.dll
 0002:00000004       __imp__SetFileTime@16      10020004     kernel32:KERNEL32.dll
 0002:00000008       __imp__GetSystemTimeAsFileTime@4 10020008     kernel32:KERNEL32.dll
 0002:0000000c       __imp__GetCurrentThreadId@0 1002000c     kernel32:KERNEL32.dll
 0002:00000010       __imp__GetCurrentProcessId@0 10020010     kernel32:KERNEL32.dll
 0002:00000014       __imp__QueryPerformanceCounter@4 10020014     kernel32:KERNEL32.dll
 0002:00000018       __imp__IsProcessorFeaturePresent@4 10020018     kernel32:KERNEL32.dll
 0002:0000001c       __imp__IsDebuggerPresent@0 1002001c     kernel32:KERNEL32.dll
 0002:00000020       __imp__DecodePointer@4     10020020     kernel32:KERNEL32.dll
 0002:00000024       __imp__EncodePointer@4     10020024     kernel32:KERNEL32.dll
 0002:00000028       __imp__CloseHandle@4       10020028     kernel32:KERNEL32.dll
 0002:0000002c       __imp__SystemTimeToFileTime@8 1002002c     kernel32:KERNEL32.dll
 0002:00000030       __imp__LocalFileTimeToFileTime@8 10020030     kernel32:KERNEL32.dll
 0002:00000034       __imp__CreateFileA@28      10020034     kernel32:KERNEL32.dll
 0002:00000038       __imp__WritePrivateProfileStringA@16 10020038     kernel32:KERNEL32.dll
 0002:0000003c       \177KERNEL32_NULL_THUNK_DATA 1002003c     kernel32:KERNEL32.dll
 0002:00000040       __imp___initterm_e         10020040     MSVCRT:MSVCR120.dll
 0002:00000044       __imp___initterm           10020044     MSVCRT:MSVCR120.dll
 0002:00000048       __imp___malloc_crt         10020048     MSVCRT:MSVCR120.dll
 0002:0000004c       __imp__free                1002004c     MSVCRT:MSVCR120.dll
 0002:00000050       __imp___amsg_exit          10020050     MSVCRT:MSVCR120.dll
 0002:00000054       __imp____CppXcptFilter     10020054     MSVCRT:MSVCR120.dll
 0002:00000058       __imp___onexit             10020058     MSVCRT:MSVCR120.dll
 0002:0000005c       __imp____dllonexit         1002005c     MSVCRT:MSVCR120.dll
 0002:00000060       __imp___calloc_crt         10020060     MSVCRT:MSVCR120.dll
 0002:00000064       __imp___unlock             10020064     MSVCRT:MSVCR120.dll
 0002:00000068       __imp___lock               10020068     MSVCRT:MSVCR120.dll
 0002:0000006c       __imp_??1type_info@@UAE@XZ 1002006c     MSVCRT:MSVCR120.dll
 0002:00000070       __imp__getenv              10020070     MSVCRT:MSVCR120.dll
 0002:00000074       __imp___purecall           10020074     MSVCRT:MSVCR120.dll
 0002:00000078       __imp_??2@YAPAXI@Z         10020078     MSVCRT:MSVCR120.dll
 0002:0000007c       __imp____CxxFrameHandler3  1002007c     MSVCRT:MSVCR120.dll
 0002:00000080       __imp_??3@YAXPAX@Z         10020080     MSVCRT:MSVCR120.dll
 0002:00000084       __imp___crt_debugger_hook  10020084     MSVCRT:MSVCR120.dll
 0002:00000088       __imp____crtUnhandledException 10020088     MSVCRT:MSVCR120.dll
 0002:0000008c       __imp____crtTerminateProcess 1002008c     MSVCRT:MSVCR120.dll
 0002:00000090       __imp___except_handler4_common 10020090     MSVCRT:MSVCR120.dll
 0002:00000094       __imp____clean_type_info_names_internal 10020094     MSVCRT:MSVCR120.dll
 0002:00000098       __imp_?terminate@@YAXXZ    10020098     MSVCRT:MSVCR120.dll
 0002:0000009c       \177MSVCR120_NULL_THUNK_DATA 1002009c     MSVCRT:MSVCR120.dll
 0002:000000a0       __imp_?fnConfig_icons@@YAPAPBDPBD@Z 100200a0     config_icons:config_icons.dll
 0002:000000a4       \177config_icons_NULL_THUNK_DATA 100200a4     config_icons:config_icons.dll
 0002:000000a8       __imp_?move@QWidget@@UAEXHH@Z 100200a8     qt-mt323:qt-mt323.dll
 0002:000000ac       __imp_?moveEvent@QWidget@@MAEXPAVQMoveEvent@@@Z 100200ac     qt-mt323:qt-mt323.dll
 0002:000000b0       __imp_?paintEvent@QWidget@@MAEXPAVQPaintEvent@@@Z 100200b0     qt-mt323:qt-mt323.dll
 0002:000000b4       __imp_?paletteChange@QWidget@@MAEXABVQPalette@@@Z 100200b4     qt-mt323:qt-mt323.dll
 0002:000000b8       __imp_?polish@QWidget@@UAEXXZ 100200b8     qt-mt323:qt-mt323.dll
 0002:000000bc       __imp_?property@QObject@@UBE?AVQVariant@@PBD@Z 100200bc     qt-mt323:qt-mt323.dll
 0002:000000c0       __imp_?removeChild@QObject@@UAEXPAV1@@Z 100200c0     qt-mt323:qt-mt323.dll
 0002:000000c4       __imp_?reparent@QWidget@@UAEXPAV1@IABVQPoint@@_N@Z 100200c4     qt-mt323:qt-mt323.dll
 0002:000000c8       __imp_?resize@QWidget@@UAEXHH@Z 100200c8     qt-mt323:qt-mt323.dll
 0002:000000cc       __imp_?resizeEvent@QWidget@@MAEXPAVQResizeEvent@@@Z 100200cc     qt-mt323:qt-mt323.dll
 0002:000000d0       __imp_?resolution@QPaintDevice@@UBEHXZ 100200d0     qt-mt323:qt-mt323.dll
 0002:000000d4       __imp_?setAcceptDrops@QWidget@@UAEX_N@Z 100200d4     qt-mt323:qt-mt323.dll
 0002:000000d8       __imp_?setActiveWindow@QWidget@@UAEXXZ 100200d8     qt-mt323:qt-mt323.dll
 0002:000000dc       __imp_?setAutoMask@QWidget@@UAEX_N@Z 100200dc     qt-mt323:qt-mt323.dll
 0002:000000e0       __imp_?setBackgroundColor@QWidget@@UAEXABVQColor@@@Z 100200e0     qt-mt323:qt-mt323.dll
 0002:000000e4       __imp_?setBackgroundMode@QWidget@@UAEXW4BackgroundMode@Qt@@@Z 100200e4     qt-mt323:qt-mt323.dll
 0002:000000e8       __imp_?setBackgroundOrigin@QWidget@@UAEXW4BackgroundOrigin@1@@Z 100200e8     qt-mt323:qt-mt323.dll
 0002:000000ec       __imp_?setBackgroundPixmap@QWidget@@UAEXABVQPixmap@@@Z 100200ec     qt-mt323:qt-mt323.dll
 0002:000000f0       __imp_?setCaption@QWidget@@UAEXABVQString@@@Z 100200f0     qt-mt323:qt-mt323.dll
 0002:000000f4       __imp_?setCursor@QWidget@@UAEXABVQCursor@@@Z 100200f4     qt-mt323:qt-mt323.dll
 0002:000000f8       __imp_?setEnabled@QWidget@@UAEX_N@Z 100200f8     qt-mt323:qt-mt323.dll
 0002:000000fc       __imp_?setEraseColor@QWidget@@UAEXABVQColor@@@Z 100200fc     qt-mt323:qt-mt323.dll
 0002:00000100       __imp_?setErasePixmap@QWidget@@UAEXABVQPixmap@@@Z 10020100     qt-mt323:qt-mt323.dll
 0002:00000104       __imp_?setFocus@QWidget@@UAEXXZ 10020104     qt-mt323:qt-mt323.dll
 0002:00000108       __imp_?setFocusPolicy@QWidget@@UAEXW4FocusPolicy@1@@Z 10020108     qt-mt323:qt-mt323.dll
 0002:0000010c       __imp_?setFocusProxy@QWidget@@UAEXPAV1@@Z 1002010c     qt-mt323:qt-mt323.dll
 0002:00000110       __imp_?setFont@QWidget@@UAEXABVQFont@@@Z 10020110     qt-mt323:qt-mt323.dll
 0002:00000114       __imp_?setGeometry@QWidget@@UAEXABVQRect@@@Z 10020114     qt-mt323:qt-mt323.dll
 0002:00000118       __imp_?setGeometry@QWidget@@UAEXHHHH@Z 10020118     qt-mt323:qt-mt323.dll
 0002:0000011c       __imp_?setIcon@QWidget@@UAEXABVQPixmap@@@Z 1002011c     qt-mt323:qt-mt323.dll
 0002:00000120       __imp_?setIconText@QWidget@@UAEXABVQString@@@Z 10020120     qt-mt323:qt-mt323.dll
 0002:00000124       __imp_?setKeyCompression@QWidget@@MAEX_N@Z 10020124     qt-mt323:qt-mt323.dll
 0002:00000128       __imp_?setMask@QWidget@@UAEXABVQBitmap@@@Z 10020128     qt-mt323:qt-mt323.dll
 0002:0000012c       __imp_?setMask@QWidget@@UAEXABVQRegion@@@Z 1002012c     qt-mt323:qt-mt323.dll
 0002:00000130       __imp_?setMaximumSize@QWidget@@UAEXHH@Z 10020130     qt-mt323:qt-mt323.dll
 0002:00000134       __imp_?setMicroFocusHint@QWidget@@MAEXHHHH_NPAVQFont@@@Z 10020134     qt-mt323:qt-mt323.dll
 0002:00000138       __imp_?setMinimumSize@QWidget@@UAEXHH@Z 10020138     qt-mt323:qt-mt323.dll
 0002:0000013c       __imp_?setMouseTracking@QWidget@@UAEX_N@Z 1002013c     qt-mt323:qt-mt323.dll
 0002:00000140       __imp_?setName@QWidget@@UAEXPBD@Z 10020140     qt-mt323:qt-mt323.dll
 0002:00000144       __imp_?setPalette@QWidget@@UAEXABVQPalette@@@Z 10020144     qt-mt323:qt-mt323.dll
 0002:00000148       __imp_?setPaletteBackgroundColor@QWidget@@UAEXABVQColor@@@Z 10020148     qt-mt323:qt-mt323.dll
 0002:0000014c       __imp_?setPaletteBackgroundPixmap@QWidget@@UAEXABVQPixmap@@@Z 1002014c     qt-mt323:qt-mt323.dll
 0002:00000150       __imp_?setProperty@QObject@@UAE_NPBDABVQVariant@@@Z 10020150     qt-mt323:qt-mt323.dll
 0002:00000154       __imp_?setResolution@QPaintDevice@@UAEXH@Z 10020154     qt-mt323:qt-mt323.dll
 0002:00000158       __imp_?setSizeIncrement@QWidget@@UAEXHH@Z 10020158     qt-mt323:qt-mt323.dll
 0002:0000015c       __imp_?setSizePolicy@QWidget@@UAEXVQSizePolicy@@@Z 1002015c     qt-mt323:qt-mt323.dll
 0002:00000160       __imp_?setUpdatesEnabled@QWidget@@UAEX_N@Z 10020160     qt-mt323:qt-mt323.dll
 0002:00000164       __imp_?setWFlags@QWidget@@MAEXI@Z 10020164     qt-mt323:qt-mt323.dll
 0002:00000168       __imp_?setWState@QWidget@@MAEXI@Z 10020168     qt-mt323:qt-mt323.dll
 0002:0000016c       __imp_?show@QWidget@@UAEXXZ 1002016c     qt-mt323:qt-mt323.dll
 0002:00000170       __imp_?showEvent@QWidget@@MAEXPAVQShowEvent@@@Z 10020170     qt-mt323:qt-mt323.dll
 0002:00000174       __imp_?showMaximized@QWidget@@UAEXXZ 10020174     qt-mt323:qt-mt323.dll
 0002:00000178       __imp_?showMinimized@QWidget@@UAEXXZ 10020178     qt-mt323:qt-mt323.dll
 0002:0000017c       __imp_?showNormal@QWidget@@UAEXXZ 1002017c     qt-mt323:qt-mt323.dll
 0002:00000180       __imp_?sizeHint@QWidget@@UBE?AVQSize@@XZ 10020180     qt-mt323:qt-mt323.dll
 0002:00000184       __imp_?sizePolicy@QWidget@@UBE?AVQSizePolicy@@XZ 10020184     qt-mt323:qt-mt323.dll
 0002:00000188       __imp_?styleChange@QWidget@@MAEXAAVQStyle@@@Z 10020188     qt-mt323:qt-mt323.dll
 0002:0000018c       __imp_?tabletEvent@QWidget@@MAEXPAVQTabletEvent@@@Z 1002018c     qt-mt323:qt-mt323.dll
 0002:00000190       __imp_?timerEvent@QObject@@MAEXPAVQTimerEvent@@@Z 10020190     qt-mt323:qt-mt323.dll
 0002:00000194       __imp_?unsetCursor@QWidget@@UAEXXZ 10020194     qt-mt323:qt-mt323.dll
 0002:00000198       __imp_?updateMask@QWidget@@MAEXXZ 10020198     qt-mt323:qt-mt323.dll
 0002:0000019c       __imp_?wheelEvent@QWidget@@MAEXPAVQWheelEvent@@@Z 1002019c     qt-mt323:qt-mt323.dll
 0002:000001a0       __imp_?winEvent@QWidget@@MAE_NPAUtagMSG@@@Z 100201a0     qt-mt323:qt-mt323.dll
 0002:000001a4       __imp_?windowActivationChange@QWidget@@MAEX_N@Z 100201a4     qt-mt323:qt-mt323.dll
 0002:000001a8       __imp_?qDebug@@YAXPBDZZ    100201a8     qt-mt323:qt-mt323.dll
 0002:000001ac       __imp_??0QString@@QAE@PBD@Z 100201ac     qt-mt323:qt-mt323.dll
 0002:000001b0       __imp_??1QString@@QAE@XZ   100201b0     qt-mt323:qt-mt323.dll
 0002:000001b4       __imp_??8@YA_NABVQString@@PBD@Z 100201b4     qt-mt323:qt-mt323.dll
 0002:000001b8       __imp_?connect@QObject@@SA_NPBV1@PBD01@Z 100201b8     qt-mt323:qt-mt323.dll
 0002:000001bc       __imp_??0QStringList@@QAE@XZ 100201bc     qt-mt323:qt-mt323.dll
 0002:000001c0       __imp_??0QStringList@@QAE@ABV0@@Z 100201c0     qt-mt323:qt-mt323.dll
 0002:000001c4       __imp_??1QStringList@@QAE@XZ 100201c4     qt-mt323:qt-mt323.dll
 0002:000001c8       __imp_??0QListView@@QAE@PAVQWidget@@PBDI@Z 100201c8     qt-mt323:qt-mt323.dll
 0002:000001cc       __imp_??1QListView@@UAE@XZ 100201cc     qt-mt323:qt-mt323.dll
 0002:000001d0       __imp_?clipboard@QApplication@@SAPAVQClipboard@@XZ 100201d0     qt-mt323:qt-mt323.dll
 0002:000001d4       __imp_?data@QClipboard@@QBEPAVQMimeSource@@XZ 100201d4     qt-mt323:qt-mt323.dll
 0002:000001d8       __imp_?canDecode@QUriDrag@@SA_NPBVQMimeSource@@@Z 100201d8     qt-mt323:qt-mt323.dll
 0002:000001dc       __imp_?decodeLocalFiles@QUriDrag@@SA_NPBVQMimeSource@@AAVQStringList@@@Z 100201dc     qt-mt323:qt-mt323.dll
 0002:000001e0       __imp_?insertItem@QMenuData@@QAEHABVQString@@HH@Z 100201e0     qt-mt323:qt-mt323.dll
 0002:000001e4       __imp_??0QPopupMenu@@QAE@PAVQWidget@@PBD@Z 100201e4     qt-mt323:qt-mt323.dll
 0002:000001e8       __imp_??1QPopupMenu@@UAE@XZ 100201e8     qt-mt323:qt-mt323.dll
 0002:000001ec       __imp_?exec@QPopupMenu@@QAEHABVQPoint@@H@Z 100201ec     qt-mt323:qt-mt323.dll
 0002:000001f0       __imp_?addChild@QScrollView@@UAEXPAVQWidget@@HH@Z 100201f0     qt-mt323:qt-mt323.dll
 0002:000001f4       __imp_?addColumn@QListView@@UAEHABVQIconSet@@ABVQString@@H@Z 100201f4     qt-mt323:qt-mt323.dll
 0002:000001f8       __imp_?addColumn@QListView@@UAEHABVQString@@H@Z 100201f8     qt-mt323:qt-mt323.dll
 0002:000001fc       __imp_?clear@QListView@@UAEXXZ 100201fc     qt-mt323:qt-mt323.dll
 0002:00000200       __imp_?clearSelection@QListView@@UAEXXZ 10020200     qt-mt323:qt-mt323.dll
 0002:00000204       __imp_?contentsContextMenuEvent@QListView@@MAEXPAVQContextMenuEvent@@@Z 10020204     qt-mt323:qt-mt323.dll
 0002:00000208       __imp_?contentsDragEnterEvent@QListView@@MAEXPAVQDragEnterEvent@@@Z 10020208     qt-mt323:qt-mt323.dll
 0002:0000020c       __imp_?contentsDragLeaveEvent@QListView@@MAEXPAVQDragLeaveEvent@@@Z 1002020c     qt-mt323:qt-mt323.dll
 0002:00000210       __imp_?contentsDragMoveEvent@QListView@@MAEXPAVQDragMoveEvent@@@Z 10020210     qt-mt323:qt-mt323.dll
 0002:00000214       __imp_?contentsDropEvent@QListView@@MAEXPAVQDropEvent@@@Z 10020214     qt-mt323:qt-mt323.dll
 0002:00000218       __imp_?contentsMouseDoubleClickEvent@QListView@@MAEXPAVQMouseEvent@@@Z 10020218     qt-mt323:qt-mt323.dll
 0002:0000021c       __imp_?contentsMouseMoveEvent@QListView@@MAEXPAVQMouseEvent@@@Z 1002021c     qt-mt323:qt-mt323.dll
 0002:00000220       __imp_?contentsMousePressEvent@QListView@@MAEXPAVQMouseEvent@@@Z 10020220     qt-mt323:qt-mt323.dll
 0002:00000224       __imp_?contentsMouseReleaseEvent@QListView@@MAEXPAVQMouseEvent@@@Z 10020224     qt-mt323:qt-mt323.dll
 0002:00000228       __imp_?contentsWheelEvent@QScrollView@@MAEXPAVQWheelEvent@@@Z 10020228     qt-mt323:qt-mt323.dll
 0002:0000022c       __imp_?dragObject@QListView@@MAEPAVQDragObject@@XZ 1002022c     qt-mt323:qt-mt323.dll
 0002:00000230       __imp_?drawContents@QScrollView@@EAEXPAVQPainter@@@Z 10020230     qt-mt323:qt-mt323.dll
 0002:00000234       __imp_?drawContents@QScrollView@@MAEXPAVQPainter@@HHHH@Z 10020234     qt-mt323:qt-mt323.dll
 0002:00000238       __imp_?drawContentsOffset@QListView@@MAEXPAVQPainter@@HHHHHH@Z 10020238     qt-mt323:qt-mt323.dll
 0002:0000023c       __imp_?drawFrame@QFrame@@MAEXPAVQPainter@@@Z 1002023c     qt-mt323:qt-mt323.dll
 0002:00000240       __imp_?eventFilter@QListView@@UAE_NPAVQObject@@PAVQEvent@@@Z 10020240     qt-mt323:qt-mt323.dll
 0002:00000244       __imp_?focusInEvent@QListView@@MAEXPAVQFocusEvent@@@Z 10020244     qt-mt323:qt-mt323.dll
 0002:00000248       __imp_?focusNextPrevChild@QScrollView@@MAE_N_N@Z 10020248     qt-mt323:qt-mt323.dll
 0002:0000024c       __imp_?focusOutEvent@QListView@@MAEXPAVQFocusEvent@@@Z 1002024c     qt-mt323:qt-mt323.dll
 0002:00000250       __imp_?fontChange@QScrollView@@MAEXABVQFont@@@Z 10020250     qt-mt323:qt-mt323.dll
 0002:00000254       __imp_?frameChanged@QScrollView@@MAEXXZ 10020254     qt-mt323:qt-mt323.dll
 0002:00000258       __imp_?insertItem@QListView@@UAEXPAVQListViewItem@@@Z 10020258     qt-mt323:qt-mt323.dll
 0002:0000025c       __imp_?invertSelection@QListView@@UAEXXZ 1002025c     qt-mt323:qt-mt323.dll
 0002:00000260       __imp_?keyPressEvent@QListView@@MAEXPAVQKeyEvent@@@Z 10020260     qt-mt323:qt-mt323.dll
 0002:00000264       __imp_?minimumSizeHint@QListView@@UBE?AVQSize@@XZ 10020264     qt-mt323:qt-mt323.dll
 0002:00000268       __imp_?mouseDoubleClickEvent@QScrollView@@MAEXPAVQMouseEvent@@@Z 10020268     qt-mt323:qt-mt323.dll
 0002:0000026c       __imp_?mouseMoveEvent@QScrollView@@MAEXPAVQMouseEvent@@@Z 1002026c     qt-mt323:qt-mt323.dll
 0002:00000270       __imp_?mousePressEvent@QScrollView@@MAEXPAVQMouseEvent@@@Z 10020270     qt-mt323:qt-mt323.dll
 0002:00000274       __imp_?mouseReleaseEvent@QScrollView@@MAEXPAVQMouseEvent@@@Z 10020274     qt-mt323:qt-mt323.dll
 0002:00000278       __imp_?moveChild@QScrollView@@UAEXPAVQWidget@@HH@Z 10020278     qt-mt323:qt-mt323.dll
 0002:0000027c       __imp_?paintEmptyArea@QListView@@MAEXPAVQPainter@@ABVQRect@@@Z 1002027c     qt-mt323:qt-mt323.dll
 0002:00000280       __imp_?paintEvent@QFrame@@MAEXPAVQPaintEvent@@@Z 10020280     qt-mt323:qt-mt323.dll
 0002:00000284       __imp_?removeChild@QScrollView@@UAEXPAVQObject@@@Z 10020284     qt-mt323:qt-mt323.dll
 0002:00000288       __imp_?removeColumn@QListView@@UAEXH@Z 10020288     qt-mt323:qt-mt323.dll
 0002:0000028c       __imp_?removeItem@QListView@@UAEXPAVQListViewItem@@@Z 1002028c     qt-mt323:qt-mt323.dll
 0002:00000290       __imp_?resize@QScrollView@@UAEXHH@Z 10020290     qt-mt323:qt-mt323.dll
 0002:00000294       __imp_?resizeContents@QScrollView@@UAEXHH@Z 10020294     qt-mt323:qt-mt323.dll
 0002:00000298       __imp_?resizeEvent@QListView@@MAEXPAVQResizeEvent@@@Z 10020298     qt-mt323:qt-mt323.dll
 0002:0000029c       __imp_?selectAll@QListView@@UAEX_N@Z 1002029c     qt-mt323:qt-mt323.dll
 0002:000002a0       __imp_?setAllColumnsShowFocus@QListView@@UAEX_N@Z 100202a0     qt-mt323:qt-mt323.dll
 0002:000002a4       __imp_?setColumnAlignment@QListView@@UAEXHH@Z 100202a4     qt-mt323:qt-mt323.dll
 0002:000002a8       __imp_?setColumnText@QListView@@UAEXHABVQIconSet@@ABVQString@@@Z 100202a8     qt-mt323:qt-mt323.dll
 0002:000002ac       __imp_?setColumnText@QListView@@UAEXHABVQString@@@Z 100202ac     qt-mt323:qt-mt323.dll
 0002:000002b0       __imp_?setColumnWidth@QListView@@UAEXHH@Z 100202b0     qt-mt323:qt-mt323.dll
 0002:000002b4       __imp_?setColumnWidthMode@QListView@@UAEXHW4WidthMode@1@@Z 100202b4     qt-mt323:qt-mt323.dll
 0002:000002b8       __imp_?setContentsPos@QListView@@UAEXHH@Z 100202b8     qt-mt323:qt-mt323.dll
 0002:000002bc       __imp_?setCornerWidget@QScrollView@@UAEXPAVQWidget@@@Z 100202bc     qt-mt323:qt-mt323.dll
 0002:000002c0       __imp_?setCurrentItem@QListView@@UAEXPAVQListViewItem@@@Z 100202c0     qt-mt323:qt-mt323.dll
 0002:000002c4       __imp_?setDefaultRenameAction@QListView@@UAEXW4RenameAction@1@@Z 100202c4     qt-mt323:qt-mt323.dll
 0002:000002c8       __imp_?setDragAutoScroll@QScrollView@@UAEX_N@Z 100202c8     qt-mt323:qt-mt323.dll
 0002:000002cc       __imp_?setEnabled@QScrollView@@UAEX_N@Z 100202cc     qt-mt323:qt-mt323.dll
 0002:000002d0       __imp_?setFont@QListView@@UAEXABVQFont@@@Z 100202d0     qt-mt323:qt-mt323.dll
 0002:000002d4       __imp_?setFrameRect@QFrame@@UAEXABVQRect@@@Z 100202d4     qt-mt323:qt-mt323.dll
 0002:000002d8       __imp_?setFrameStyle@QFrame@@UAEXH@Z 100202d8     qt-mt323:qt-mt323.dll
 0002:000002dc       __imp_?setHBarGeometry@QScrollView@@MAEXAAVQScrollBar@@HHHH@Z 100202dc     qt-mt323:qt-mt323.dll
 0002:000002e0       __imp_?setHScrollBarMode@QScrollView@@UAEXW4ScrollBarMode@1@@Z 100202e0     qt-mt323:qt-mt323.dll
 0002:000002e4       __imp_?setItemMargin@QListView@@UAEXH@Z 100202e4     qt-mt323:qt-mt323.dll
 0002:000002e8       __imp_?setLineWidth@QFrame@@UAEXH@Z 100202e8     qt-mt323:qt-mt323.dll
 0002:000002ec       __imp_?setMargin@QFrame@@UAEXH@Z 100202ec     qt-mt323:qt-mt323.dll
 0002:000002f0       __imp_?setMargins@QScrollView@@MAEXHHHH@Z 100202f0     qt-mt323:qt-mt323.dll
 0002:000002f4       __imp_?setMidLineWidth@QFrame@@UAEXH@Z 100202f4     qt-mt323:qt-mt323.dll
 0002:000002f8       __imp_?setMultiSelection@QListView@@UAEX_N@Z 100202f8     qt-mt323:qt-mt323.dll
 0002:000002fc       __imp_?setOpen@QListView@@UAEXPAVQListViewItem@@_N@Z 100202fc     qt-mt323:qt-mt323.dll
 0002:00000300       __imp_?setPalette@QListView@@UAEXABVQPalette@@@Z 10020300     qt-mt323:qt-mt323.dll
 0002:00000304       __imp_?setResizeMode@QListView@@UAEXW4ResizeMode@1@@Z 10020304     qt-mt323:qt-mt323.dll
 0002:00000308       __imp_?setResizePolicy@QScrollView@@UAEXW4ResizePolicy@1@@Z 10020308     qt-mt323:qt-mt323.dll
 0002:0000030c       __imp_?setRootIsDecorated@QListView@@UAEX_N@Z 1002030c     qt-mt323:qt-mt323.dll
 0002:00000310       __imp_?setSelected@QListView@@UAEXPAVQListViewItem@@_N@Z 10020310     qt-mt323:qt-mt323.dll
 0002:00000314       __imp_?setShowSortIndicator@QListView@@UAEX_N@Z 10020314     qt-mt323:qt-mt323.dll
 0002:00000318       __imp_?setShowToolTips@QListView@@UAEX_N@Z 10020318     qt-mt323:qt-mt323.dll
 0002:0000031c       __imp_?setSorting@QListView@@UAEXH_N@Z 1002031c     qt-mt323:qt-mt323.dll
 0002:00000320       __imp_?setTreeStepSize@QListView@@UAEXH@Z 10020320     qt-mt323:qt-mt323.dll
 0002:00000324       __imp_?setVBarGeometry@QScrollView@@MAEXAAVQScrollBar@@HHHH@Z 10020324     qt-mt323:qt-mt323.dll
 0002:00000328       __imp_?setVScrollBarMode@QScrollView@@UAEXW4ScrollBarMode@1@@Z 10020328     qt-mt323:qt-mt323.dll
 0002:0000032c       __imp_?show@QListView@@UAEXXZ 1002032c     qt-mt323:qt-mt323.dll
 0002:00000330       __imp_?showEvent@QListView@@MAEXPAVQShowEvent@@@Z 10020330     qt-mt323:qt-mt323.dll
 0002:00000334       __imp_?sizeHint@QListView@@UBE?AVQSize@@XZ 10020334     qt-mt323:qt-mt323.dll
 0002:00000338       __imp_?sort@QListView@@UAEXXZ 10020338     qt-mt323:qt-mt323.dll
 0002:0000033c       __imp_?startDrag@QListView@@MAEXXZ 1002033c     qt-mt323:qt-mt323.dll
 0002:00000340       __imp_?styleChange@QListView@@MAEXAAVQStyle@@@Z 10020340     qt-mt323:qt-mt323.dll
 0002:00000344       __imp_?takeItem@QListView@@UAEXPAVQListViewItem@@@Z 10020344     qt-mt323:qt-mt323.dll
 0002:00000348       __imp_?viewportContextMenuEvent@QScrollView@@MAEXPAVQContextMenuEvent@@@Z 10020348     qt-mt323:qt-mt323.dll
 0002:0000034c       __imp_?viewportDragEnterEvent@QScrollView@@MAEXPAVQDragEnterEvent@@@Z 1002034c     qt-mt323:qt-mt323.dll
 0002:00000350       __imp_?viewportDragLeaveEvent@QScrollView@@MAEXPAVQDragLeaveEvent@@@Z 10020350     qt-mt323:qt-mt323.dll
 0002:00000354       __imp_?viewportDragMoveEvent@QScrollView@@MAEXPAVQDragMoveEvent@@@Z 10020354     qt-mt323:qt-mt323.dll
 0002:00000358       __imp_?viewportDropEvent@QScrollView@@MAEXPAVQDropEvent@@@Z 10020358     qt-mt323:qt-mt323.dll
 0002:0000035c       __imp_?viewportMouseDoubleClickEvent@QScrollView@@MAEXPAVQMouseEvent@@@Z 1002035c     qt-mt323:qt-mt323.dll
 0002:00000360       __imp_?viewportMouseMoveEvent@QScrollView@@MAEXPAVQMouseEvent@@@Z 10020360     qt-mt323:qt-mt323.dll
 0002:00000364       __imp_?viewportMousePressEvent@QScrollView@@MAEXPAVQMouseEvent@@@Z 10020364     qt-mt323:qt-mt323.dll
 0002:00000368       __imp_?viewportMouseReleaseEvent@QScrollView@@MAEXPAVQMouseEvent@@@Z 10020368     qt-mt323:qt-mt323.dll
 0002:0000036c       __imp_?viewportPaintEvent@QScrollView@@MAEXPAVQPaintEvent@@@Z 1002036c     qt-mt323:qt-mt323.dll
 0002:00000370       __imp_?viewportResizeEvent@QListView@@MAEXPAVQResizeEvent@@@Z 10020370     qt-mt323:qt-mt323.dll
 0002:00000374       __imp_?viewportWheelEvent@QScrollView@@MAEXPAVQWheelEvent@@@Z 10020374     qt-mt323:qt-mt323.dll
 0002:00000378       __imp_?wheelEvent@QScrollView@@MAEXPAVQWheelEvent@@@Z 10020378     qt-mt323:qt-mt323.dll
 0002:0000037c       __imp_?windowActivationChange@QListView@@MAEX_N@Z 1002037c     qt-mt323:qt-mt323.dll
 0002:00000380       __imp_??0QString@@QAE@XZ   10020380     qt-mt323:qt-mt323.dll
 0002:00000384       __imp_??0QString@@QAE@ABV0@@Z 10020384     qt-mt323:qt-mt323.dll
 0002:00000388       __imp_??4QString@@QAEAAV0@ABV0@@Z 10020388     qt-mt323:qt-mt323.dll
 0002:0000038c       __imp_?truncate@QString@@QAEXI@Z 1002038c     qt-mt323:qt-mt323.dll
 0002:00000390       __imp_?contains@QString@@QBEHPBD_N@Z 10020390     qt-mt323:qt-mt323.dll
 0002:00000394       __imp_?insert@QString@@QAEAAV1@IABV1@@Z 10020394     qt-mt323:qt-mt323.dll
 0002:00000398       __imp_?prepend@QString@@QAEAAV1@PBD@Z 10020398     qt-mt323:qt-mt323.dll
 0002:0000039c       __imp_?ascii@QString@@QBEPBDXZ 1002039c     qt-mt323:qt-mt323.dll
 0002:000003a0       __imp_??8@YA_NABVQString@@0@Z 100203a0     qt-mt323:qt-mt323.dll
 0002:000003a4       __imp_??H@YA?BVQString@@ABV0@0@Z 100203a4     qt-mt323:qt-mt323.dll
 0002:000003a8       __imp_??H@YA?BVQString@@ABV0@PBD@Z 100203a8     qt-mt323:qt-mt323.dll
 0002:000003ac       __imp_??H@YA?BVQString@@PBDABV0@@Z 100203ac     qt-mt323:qt-mt323.dll
 0002:000003b0       __imp_?begin@?$QValueList@VQString@@@@QAE?AV?$QValueListIterator@VQString@@@@XZ 100203b0     qt-mt323:qt-mt323.dll
 0002:000003b4       __imp_??A?$QValueList@VQString@@@@QAEAAVQString@@I@Z 100203b4     qt-mt323:qt-mt323.dll
 0002:000003b8       __imp_?detachInternal@?$QValueList@VQString@@@@AAEXXZ 100203b8     qt-mt323:qt-mt323.dll
 0002:000003bc       __imp_??0QGList@@IAE@XZ    100203bc     qt-mt323:qt-mt323.dll
 0002:000003c0       __imp_??0QGList@@IAE@ABV0@@Z 100203c0     qt-mt323:qt-mt323.dll
 0002:000003c4       __imp_??1QGList@@MAE@XZ    100203c4     qt-mt323:qt-mt323.dll
 0002:000003c8       __imp_?clear@QGList@@MAEXXZ 100203c8     qt-mt323:qt-mt323.dll
 0002:000003cc       __imp_?startTimer@QObject@@QAEHH@Z 100203cc     qt-mt323:qt-mt323.dll
 0002:000003d0       __imp_?killTimer@QObject@@QAEXH@Z 100203d0     qt-mt323:qt-mt323.dll
 0002:000003d4       __imp_?split@QStringList@@SA?AV1@ABVQString@@0_N@Z 100203d4     qt-mt323:qt-mt323.dll
 0002:000003d8       __imp_??0QWidget@@QAE@PAV0@PBDI@Z 100203d8     qt-mt323:qt-mt323.dll
 0002:000003dc       __imp_??1QWidget@@UAE@XZ   100203dc     qt-mt323:qt-mt323.dll
 0002:000003e0       __imp_?update@QWidget@@QAEXXZ 100203e0     qt-mt323:qt-mt323.dll
 0002:000003e4       __imp_?information@QMessageBox@@SAHPAVQWidget@@ABVQString@@1111HH@Z 100203e4     qt-mt323:qt-mt323.dll
 0002:000003e8       __imp_??0QPixmap@@QAE@QAPBD@Z 100203e8     qt-mt323:qt-mt323.dll
 0002:000003ec       __imp_??1QPixmap@@UAE@XZ   100203ec     qt-mt323:qt-mt323.dll
 0002:000003f0       __imp_?addWidget@QBoxLayout@@QAEXPAVQWidget@@HH@Z 100203f0     qt-mt323:qt-mt323.dll
 0002:000003f4       __imp_??0QVBoxLayout@@QAE@PAVQWidget@@HHPBD@Z 100203f4     qt-mt323:qt-mt323.dll
 0002:000003f8       __imp_??1QVBoxLayout@@UAE@XZ 100203f8     qt-mt323:qt-mt323.dll
 0002:000003fc       __imp_??0QLabel@@QAE@PAVQWidget@@PBDI@Z 100203fc     qt-mt323:qt-mt323.dll
 0002:00000400       __imp_??1QLabel@@UAE@XZ    10020400     qt-mt323:qt-mt323.dll
 0002:00000404       __imp_??0QListViewItem@@QAE@PAVQListView@@VQString@@1111111@Z 10020404     qt-mt323:qt-mt323.dll
 0002:00000408       __imp_??0QListViewItem@@QAE@PAV0@VQString@@1111111@Z 10020408     qt-mt323:qt-mt323.dll
 0002:0000040c       __imp_??1QListViewItem@@UAE@XZ 1002040c     qt-mt323:qt-mt323.dll
 0002:00000410       __imp_?firstChild@QListViewItem@@QBEPAV1@XZ 10020410     qt-mt323:qt-mt323.dll
 0002:00000414       __imp_?parent@QListViewItem@@QBEPAV1@XZ 10020414     qt-mt323:qt-mt323.dll
 0002:00000418       __imp_?findItem@QListView@@QBEPAVQListViewItem@@ABVQString@@HI@Z 10020418     qt-mt323:qt-mt323.dll
 0002:0000041c       __imp_??1?$QPtrList@VQDockWindow@@@@UAE@XZ 1002041c     qt-mt323:qt-mt323.dll
 0002:00000420       __imp_??0QFile@@QAE@ABVQString@@@Z 10020420     qt-mt323:qt-mt323.dll
 0002:00000424       __imp_??1QFile@@UAE@XZ     10020424     qt-mt323:qt-mt323.dll
 0002:00000428       __imp_?open@QFile@@UAE_NH@Z 10020428     qt-mt323:qt-mt323.dll
 0002:0000042c       __imp_?readBlock@QFile@@UAEJPADK@Z 1002042c     qt-mt323:qt-mt323.dll
 0002:00000430       __imp_?writeBlock@QFile@@UAEJPBDK@Z 10020430     qt-mt323:qt-mt323.dll
 0002:00000434       __imp_??4QDomNode@@QAEAAV0@ABV0@@Z 10020434     qt-mt323:qt-mt323.dll
 0002:00000438       __imp_??1QDomNode@@UAE@XZ  10020438     qt-mt323:qt-mt323.dll
 0002:0000043c       __imp_?firstChild@QDomNode@@UBE?AV1@XZ 1002043c     qt-mt323:qt-mt323.dll
 0002:00000440       __imp_?nextSibling@QDomNode@@UBE?AV1@XZ 10020440     qt-mt323:qt-mt323.dll
 0002:00000444       __imp_?isNull@QDomNode@@QBE_NXZ 10020444     qt-mt323:qt-mt323.dll
 0002:00000448       __imp_?toElement@QDomNode@@QAE?AVQDomElement@@XZ 10020448     qt-mt323:qt-mt323.dll
 0002:0000044c       __imp_??0QDomDocument@@QAE@ABVQString@@@Z 1002044c     qt-mt323:qt-mt323.dll
 0002:00000450       __imp_??1QDomDocument@@UAE@XZ 10020450     qt-mt323:qt-mt323.dll
 0002:00000454       __imp_?documentElement@QDomDocument@@QBE?AVQDomElement@@XZ 10020454     qt-mt323:qt-mt323.dll
 0002:00000458       __imp_?setContent@QDomDocument@@QAE_NABVQString@@PAV2@PAH2@Z 10020458     qt-mt323:qt-mt323.dll
 0002:0000045c       __imp_??1QDomElement@@UAE@XZ 1002045c     qt-mt323:qt-mt323.dll
 0002:00000460       __imp_?attribute@QDomElement@@QBE?AVQString@@ABV2@0@Z 10020460     qt-mt323:qt-mt323.dll
 0002:00000464       __imp_?add@QToolTip@@SAXPAVQWidget@@ABVQString@@@Z 10020464     qt-mt323:qt-mt323.dll
 0002:00000468       __imp_?toString@QDateTime@@QBE?AVQString@@ABV2@@Z 10020468     qt-mt323:qt-mt323.dll
 0002:0000046c       __imp_?fromString@QDateTime@@SA?AV1@ABVQString@@W4DateFormat@Qt@@@Z 1002046c     qt-mt323:qt-mt323.dll
 0002:00000470       __imp_??0QFileInfo@@QAE@ABVQString@@@Z 10020470     qt-mt323:qt-mt323.dll
 0002:00000474       __imp_??1QFileInfo@@QAE@XZ 10020474     qt-mt323:qt-mt323.dll
 0002:00000478       __imp_?exists@QFileInfo@@QBE_NXZ 10020478     qt-mt323:qt-mt323.dll
 0002:0000047c       __imp_?fileName@QFileInfo@@QBE?AVQString@@XZ 1002047c     qt-mt323:qt-mt323.dll
 0002:00000480       __imp_?absFilePath@QFileInfo@@QBE?AVQString@@XZ 10020480     qt-mt323:qt-mt323.dll
 0002:00000484       __imp_?lastModified@QFileInfo@@QBE?AVQDateTime@@XZ 10020484     qt-mt323:qt-mt323.dll
 0002:00000488       __imp_?add@QWhatsThis@@SAXPAVQWidget@@ABVQString@@@Z 10020488     qt-mt323:qt-mt323.dll
 0002:0000048c       __imp_??0QSplitter@@QAE@PAVQWidget@@PBD@Z 1002048c     qt-mt323:qt-mt323.dll
 0002:00000490       __imp_??1QSplitter@@UAE@XZ 10020490     qt-mt323:qt-mt323.dll
 0002:00000494       __imp_??0QGuardedPtrPrivate@@QAE@PAVQObject@@@Z 10020494     qt-mt323:qt-mt323.dll
 0002:00000498       __imp_??1QGuardedPtrPrivate@@UAE@XZ 10020498     qt-mt323:qt-mt323.dll
 0002:0000049c       __imp_?acceptDrop@QListViewItem@@UBE_NPBVQMimeSource@@@Z 1002049c     qt-mt323:qt-mt323.dll
 0002:000004a0       __imp_?activate@QListViewItem@@MAEXXZ 100204a0     qt-mt323:qt-mt323.dll
 0002:000004a4       __imp_?addItem@QBoxLayout@@UAEXPAVQLayoutItem@@@Z 100204a4     qt-mt323:qt-mt323.dll
 0002:000004a8       __imp_?cancelRename@QListViewItem@@MAEXH@Z 100204a8     qt-mt323:qt-mt323.dll
 0002:000004ac       __imp_?childEvent@QLayout@@MAEXPAVQChildEvent@@@Z 100204ac     qt-mt323:qt-mt323.dll
 0002:000004b0       __imp_?childEvent@QSplitter@@MAEXPAVQChildEvent@@@Z 100204b0     qt-mt323:qt-mt323.dll
 0002:000004b4       __imp_?className@QGuardedPtrPrivate@@UBEPBDXZ 100204b4     qt-mt323:qt-mt323.dll
 0002:000004b8       __imp_?className@QLabel@@UBEPBDXZ 100204b8     qt-mt323:qt-mt323.dll
 0002:000004bc       __imp_?className@QListView@@UBEPBDXZ 100204bc     qt-mt323:qt-mt323.dll
 0002:000004c0       __imp_?className@QSplitter@@UBEPBDXZ 100204c0     qt-mt323:qt-mt323.dll
 0002:000004c4       __imp_?className@QVBoxLayout@@UBEPBDXZ 100204c4     qt-mt323:qt-mt323.dll
 0002:000004c8       __imp_?className@QWidget@@UBEPBDXZ 100204c8     qt-mt323:qt-mt323.dll
 0002:000004cc       __imp_?clear@?$QPtrList@VQDockWindow@@@@UAEXXZ 100204cc     qt-mt323:qt-mt323.dll
 0002:000004d0       __imp_?compare@QListViewItem@@UBEHPAV1@H_N@Z 100204d0     qt-mt323:qt-mt323.dll
 0002:000004d4       __imp_?compareItems@QGList@@MAEHPAX0@Z 100204d4     qt-mt323:qt-mt323.dll
 0002:000004d8       __imp_?contextMenuEvent@QScrollView@@MAEXPAVQContextMenuEvent@@@Z 100204d8     qt-mt323:qt-mt323.dll
 0002:000004dc       __imp_?count@?$QPtrList@VQDockWindow@@@@UBEIXZ 100204dc     qt-mt323:qt-mt323.dll
 0002:000004e0       __imp_?deleteItem@?$QPtrList@VQDockWindow@@@@EAEXPAX@Z 100204e0     qt-mt323:qt-mt323.dll
 0002:000004e4       __imp_?dragEntered@QListViewItem@@MAEXXZ 100204e4     qt-mt323:qt-mt323.dll
 0002:000004e8       __imp_?dragLeft@QListViewItem@@MAEXXZ 100204e8     qt-mt323:qt-mt323.dll
 0002:000004ec       __imp_?drawContents@QFrame@@MAEXPAVQPainter@@@Z 100204ec     qt-mt323:qt-mt323.dll
 0002:000004f0       __imp_?drawContents@QLabel@@MAEXPAVQPainter@@@Z 100204f0     qt-mt323:qt-mt323.dll
 0002:000004f4       __imp_?drawSplitter@QSplitter@@MAEXPAVQPainter@@HHHH@Z 100204f4     qt-mt323:qt-mt323.dll
 0002:000004f8       __imp_?dropped@QListViewItem@@MAEXPAVQDropEvent@@@Z 100204f8     qt-mt323:qt-mt323.dll
 0002:000004fc       __imp_?enforceSortOrder@QListViewItem@@MBEXXZ 100204fc     qt-mt323:qt-mt323.dll
 0002:00000500       __imp_?event@QObject@@UAE_NPAVQEvent@@@Z 10020500     qt-mt323:qt-mt323.dll
 0002:00000504       __imp_?event@QSplitter@@MAE_NPAVQEvent@@@Z 10020504     qt-mt323:qt-mt323.dll
 0002:00000508       __imp_?eventFilter@QLayout@@MAE_NPAVQObject@@PAVQEvent@@@Z 10020508     qt-mt323:qt-mt323.dll
 0002:0000050c       __imp_?expanding@QBoxLayout@@UBE?AW4ExpandData@QSizePolicy@@XZ 1002050c     qt-mt323:qt-mt323.dll
 0002:00000510       __imp_?fontChange@QLabel@@MAEXABVQFont@@@Z 10020510     qt-mt323:qt-mt323.dll
 0002:00000514       __imp_?frameChanged@QFrame@@MAEXXZ 10020514     qt-mt323:qt-mt323.dll
 0002:00000518       __imp_?geometry@QLayout@@UBE?AVQRect@@XZ 10020518     qt-mt323:qt-mt323.dll
 0002:0000051c       __imp_?hasHeightForWidth@QBoxLayout@@UBE_NXZ 1002051c     qt-mt323:qt-mt323.dll
 0002:00000520       __imp_?heightForWidth@QBoxLayout@@UBEHH@Z 10020520     qt-mt323:qt-mt323.dll
 0002:00000524       __imp_?heightForWidth@QLabel@@UBEHH@Z 10020524     qt-mt323:qt-mt323.dll
 0002:00000528       __imp_?insertItem@QListViewItem@@UAEXPAV1@@Z 10020528     qt-mt323:qt-mt323.dll
 0002:0000052c       __imp_?invalidate@QBoxLayout@@UAEXXZ 1002052c     qt-mt323:qt-mt323.dll
 0002:00000530       __imp_?invalidateHeight@QListViewItem@@UAEXXZ 10020530     qt-mt323:qt-mt323.dll
 0002:00000534       __imp_?isEmpty@QLayout@@UBE_NXZ 10020534     qt-mt323:qt-mt323.dll
 0002:00000538       __imp_?iterator@QBoxLayout@@UAE?AVQLayoutIterator@@XZ 10020538     qt-mt323:qt-mt323.dll
 0002:0000053c       __imp_?key@QListViewItem@@UBE?AVQString@@H_N@Z 1002053c     qt-mt323:qt-mt323.dll
 0002:00000540       __imp_?layout@QLayout@@UAEPAV1@XZ 10020540     qt-mt323:qt-mt323.dll
 0002:00000544       __imp_?maximumSize@QBoxLayout@@UBE?AVQSize@@XZ 10020544     qt-mt323:qt-mt323.dll
 0002:00000548       __imp_?metaObject@QGuardedPtrPrivate@@UBEPAVQMetaObject@@XZ 10020548     qt-mt323:qt-mt323.dll
 0002:0000054c       __imp_?metaObject@QLabel@@UBEPAVQMetaObject@@XZ 1002054c     qt-mt323:qt-mt323.dll
 0002:00000550       __imp_?metaObject@QListView@@UBEPAVQMetaObject@@XZ 10020550     qt-mt323:qt-mt323.dll
 0002:00000554       __imp_?metaObject@QSplitter@@UBEPAVQMetaObject@@XZ 10020554     qt-mt323:qt-mt323.dll
 0002:00000558       __imp_?metaObject@QVBoxLayout@@UBEPAVQMetaObject@@XZ 10020558     qt-mt323:qt-mt323.dll
 0002:0000055c       __imp_?metaObject@QWidget@@UBEPAVQMetaObject@@XZ 1002055c     qt-mt323:qt-mt323.dll
 0002:00000560       __imp_?minimumSize@QBoxLayout@@UBE?AVQSize@@XZ 10020560     qt-mt323:qt-mt323.dll
 0002:00000564       __imp_?minimumSizeHint@QLabel@@UBE?AVQSize@@XZ 10020564     qt-mt323:qt-mt323.dll
 0002:00000568       __imp_?minimumSizeHint@QSplitter@@UBE?AVQSize@@XZ 10020568     qt-mt323:qt-mt323.dll
 0002:0000056c       __imp_?newItem@QPtrCollection@@MAEPAXPAX@Z 1002056c     qt-mt323:qt-mt323.dll
 0002:00000570       __imp_?okRename@QListViewItem@@MAEXH@Z 10020570     qt-mt323:qt-mt323.dll
 0002:00000574       __imp_?paintBranches@QListViewItem@@UAEXPAVQPainter@@ABVQColorGroup@@HHH@Z 10020574     qt-mt323:qt-mt323.dll
 0002:00000578       __imp_?paintCell@QListViewItem@@UAEXPAVQPainter@@ABVQColorGroup@@HHH@Z 10020578     qt-mt323:qt-mt323.dll
 0002:0000057c       __imp_?paintFocus@QListViewItem@@UAEXPAVQPainter@@ABVQColorGroup@@ABVQRect@@@Z 1002057c     qt-mt323:qt-mt323.dll
 0002:00000580       __imp_?pixmap@QListViewItem@@UBEPBVQPixmap@@H@Z 10020580     qt-mt323:qt-mt323.dll
 0002:00000584       __imp_?qt_cast@QGuardedPtrPrivate@@UAEPAXPBD@Z 10020584     qt-mt323:qt-mt323.dll
 0002:00000588       __imp_?qt_cast@QLabel@@UAEPAXPBD@Z 10020588     qt-mt323:qt-mt323.dll
 0002:0000058c       __imp_?qt_cast@QListView@@UAEPAXPBD@Z 1002058c     qt-mt323:qt-mt323.dll
 0002:00000590       __imp_?qt_cast@QSplitter@@UAEPAXPBD@Z 10020590     qt-mt323:qt-mt323.dll
 0002:00000594       __imp_?qt_cast@QVBoxLayout@@UAEPAXPBD@Z 10020594     qt-mt323:qt-mt323.dll
 0002:00000598       __imp_?qt_cast@QWidget@@UAEPAXPBD@Z 10020598     qt-mt323:qt-mt323.dll
 0002:0000059c       __imp_?qt_emit@QGuardedPtrPrivate@@UAE_NHPAUQUObject@@@Z 1002059c     qt-mt323:qt-mt323.dll
 0002:000005a0       __imp_?qt_emit@QLabel@@UAE_NHPAUQUObject@@@Z 100205a0     qt-mt323:qt-mt323.dll
 0002:000005a4       __imp_?qt_emit@QListView@@UAE_NHPAUQUObject@@@Z 100205a4     qt-mt323:qt-mt323.dll
 0002:000005a8       __imp_?qt_emit@QSplitter@@UAE_NHPAUQUObject@@@Z 100205a8     qt-mt323:qt-mt323.dll
 0002:000005ac       __imp_?qt_emit@QVBoxLayout@@UAE_NHPAUQUObject@@@Z 100205ac     qt-mt323:qt-mt323.dll
 0002:000005b0       __imp_?qt_emit@QWidget@@UAE_NHPAUQUObject@@@Z 100205b0     qt-mt323:qt-mt323.dll
 0002:000005b4       __imp_?qt_invoke@QGuardedPtrPrivate@@UAE_NHPAUQUObject@@@Z 100205b4     qt-mt323:qt-mt323.dll
 0002:000005b8       __imp_?qt_invoke@QLabel@@UAE_NHPAUQUObject@@@Z 100205b8     qt-mt323:qt-mt323.dll
 0002:000005bc       __imp_?qt_invoke@QListView@@UAE_NHPAUQUObject@@@Z 100205bc     qt-mt323:qt-mt323.dll
 0002:000005c0       __imp_?qt_invoke@QSplitter@@UAE_NHPAUQUObject@@@Z 100205c0     qt-mt323:qt-mt323.dll
 0002:000005c4       __imp_?qt_invoke@QVBoxLayout@@UAE_NHPAUQUObject@@@Z 100205c4     qt-mt323:qt-mt323.dll
 0002:000005c8       __imp_?qt_invoke@QWidget@@UAE_NHPAUQUObject@@@Z 100205c8     qt-mt323:qt-mt323.dll
 0002:000005cc       __imp_?qt_property@QGuardedPtrPrivate@@UAE_NHHPAVQVariant@@@Z 100205cc     qt-mt323:qt-mt323.dll
 0002:000005d0       __imp_?qt_property@QLabel@@UAE_NHHPAVQVariant@@@Z 100205d0     qt-mt323:qt-mt323.dll
 0002:000005d4       __imp_?qt_property@QListView@@UAE_NHHPAVQVariant@@@Z 100205d4     qt-mt323:qt-mt323.dll
 0002:000005d8       __imp_?qt_property@QSplitter@@UAE_NHHPAVQVariant@@@Z 100205d8     qt-mt323:qt-mt323.dll
 0002:000005dc       __imp_?qt_property@QVBoxLayout@@UAE_NHHPAVQVariant@@@Z 100205dc     qt-mt323:qt-mt323.dll
 0002:000005e0       __imp_?qt_property@QWidget@@UAE_NHHPAVQVariant@@@Z 100205e0     qt-mt323:qt-mt323.dll
 0002:000005e4       __imp_?read@QGList@@MAEAAVQDataStream@@AAV2@AAPAX@Z 100205e4     qt-mt323:qt-mt323.dll
 0002:000005e8       __imp_?removeItem@QListViewItem@@UAEXPAV1@@Z 100205e8     qt-mt323:qt-mt323.dll
 0002:000005ec       __imp_?resizeEvent@QLabel@@MAEXPAVQResizeEvent@@@Z 100205ec     qt-mt323:qt-mt323.dll
 0002:000005f0       __imp_?resizeEvent@QSplitter@@MAEXPAVQResizeEvent@@@Z 100205f0     qt-mt323:qt-mt323.dll
 0002:000005f4       __imp_?rtti@QListViewItem@@UBEHXZ 100205f4     qt-mt323:qt-mt323.dll
 0002:000005f8       __imp_?setAlignment@QLabel@@UAEXH@Z 100205f8     qt-mt323:qt-mt323.dll
 0002:000005fc       __imp_?setAlignment@QLayoutItem@@UAEXH@Z 100205fc     qt-mt323:qt-mt323.dll
 0002:00000600       __imp_?setAutoAdd@QLayout@@UAEX_N@Z 10020600     qt-mt323:qt-mt323.dll
 0002:00000604       __imp_?setAutoResize@QLabel@@UAEX_N@Z 10020604     qt-mt323:qt-mt323.dll
 0002:00000608       __imp_?setBuddy@QLabel@@UAEXPAVQWidget@@@Z 10020608     qt-mt323:qt-mt323.dll
 0002:0000060c       __imp_?setDragEnabled@QListViewItem@@UAEX_N@Z 1002060c     qt-mt323:qt-mt323.dll
 0002:00000610       __imp_?setDropEnabled@QListViewItem@@UAEX_N@Z 10020610     qt-mt323:qt-mt323.dll
 0002:00000614       __imp_?setEnabled@QListViewItem@@UAEX_N@Z 10020614     qt-mt323:qt-mt323.dll
 0002:00000618       __imp_?setExpandable@QListViewItem@@UAEX_N@Z 10020618     qt-mt323:qt-mt323.dll
 0002:0000061c       __imp_?setFont@QLabel@@UAEXABVQFont@@@Z 1002061c     qt-mt323:qt-mt323.dll
 0002:00000620       __imp_?setGeometry@QBoxLayout@@UAEXABVQRect@@@Z 10020620     qt-mt323:qt-mt323.dll
 0002:00000624       __imp_?setHeight@QListViewItem@@MAEXH@Z 10020624     qt-mt323:qt-mt323.dll
 0002:00000628       __imp_?setMargin@QLayout@@UAEXH@Z 10020628     qt-mt323:qt-mt323.dll
 0002:0000062c       __imp_?setMenuBar@QLayout@@UAEXPAVQMenuBar@@@Z 1002062c     qt-mt323:qt-mt323.dll
 0002:00000630       __imp_?setMovie@QLabel@@UAEXABVQMovie@@@Z 10020630     qt-mt323:qt-mt323.dll
 0002:00000634       __imp_?setMultiLinesEnabled@QListViewItem@@UAEX_N@Z 10020634     qt-mt323:qt-mt323.dll
 0002:00000638       __imp_?setName@QObject@@UAEXPBD@Z 10020638     qt-mt323:qt-mt323.dll
 0002:0000063c       __imp_?setNum@QLabel@@UAEXH@Z 1002063c     qt-mt323:qt-mt323.dll
 0002:00000640       __imp_?setNum@QLabel@@UAEXN@Z 10020640     qt-mt323:qt-mt323.dll
 0002:00000644       __imp_?setOpaqueResize@QSplitter@@UAEX_N@Z 10020644     qt-mt323:qt-mt323.dll
 0002:00000648       __imp_?setOpen@QListViewItem@@UAEX_N@Z 10020648     qt-mt323:qt-mt323.dll
 0002:0000064c       __imp_?setOrientation@QSplitter@@UAEXW4Orientation@Qt@@@Z 1002064c     qt-mt323:qt-mt323.dll
 0002:00000650       __imp_?setPicture@QLabel@@UAEXABVQPicture@@@Z 10020650     qt-mt323:qt-mt323.dll
 0002:00000654       __imp_?setPixmap@QLabel@@UAEXABVQPixmap@@@Z 10020654     qt-mt323:qt-mt323.dll
 0002:00000658       __imp_?setPixmap@QListViewItem@@UAEXHABVQPixmap@@@Z 10020658     qt-mt323:qt-mt323.dll
 0002:0000065c       __imp_?setRenameEnabled@QListViewItem@@UAEXH_N@Z 1002065c     qt-mt323:qt-mt323.dll
 0002:00000660       __imp_?setResizeMode@QSplitter@@UAEXPAVQWidget@@W4ResizeMode@1@@Z 10020660     qt-mt323:qt-mt323.dll
 0002:00000664       __imp_?setRubberband@QSplitter@@MAEXH@Z 10020664     qt-mt323:qt-mt323.dll
 0002:00000668       __imp_?setSelectable@QListViewItem@@UAEX_N@Z 10020668     qt-mt323:qt-mt323.dll
 0002:0000066c       __imp_?setSelected@QListViewItem@@UAEX_N@Z 1002066c     qt-mt323:qt-mt323.dll
 0002:00000670       __imp_?setSpacing@QLayout@@UAEXH@Z 10020670     qt-mt323:qt-mt323.dll
 0002:00000674       __imp_?setText@QLabel@@UAEXABVQString@@@Z 10020674     qt-mt323:qt-mt323.dll
 0002:00000678       __imp_?setText@QListViewItem@@UAEXHABVQString@@@Z 10020678     qt-mt323:qt-mt323.dll
 0002:0000067c       __imp_?setup@QListViewItem@@UAEXXZ 1002067c     qt-mt323:qt-mt323.dll
 0002:00000680       __imp_?sizeHint@QBoxLayout@@UBE?AVQSize@@XZ 10020680     qt-mt323:qt-mt323.dll
 0002:00000684       __imp_?sizeHint@QLabel@@UBE?AVQSize@@XZ 10020684     qt-mt323:qt-mt323.dll
 0002:00000688       __imp_?sizeHint@QSplitter@@UBE?AVQSize@@XZ 10020688     qt-mt323:qt-mt323.dll
 0002:0000068c       __imp_?sort@QListViewItem@@UAEXXZ 1002068c     qt-mt323:qt-mt323.dll
 0002:00000690       __imp_?sortChildItems@QListViewItem@@UAEXH_N@Z 10020690     qt-mt323:qt-mt323.dll
 0002:00000694       __imp_?spacerItem@QLayoutItem@@UAEPAVQSpacerItem@@XZ 10020694     qt-mt323:qt-mt323.dll
 0002:00000698       __imp_?startRename@QListViewItem@@UAEXH@Z 10020698     qt-mt323:qt-mt323.dll
 0002:0000069c       __imp_?styleChange@QFrame@@MAEXAAVQStyle@@@Z 1002069c     qt-mt323:qt-mt323.dll
 0002:000006a0       __imp_?styleChange@QSplitter@@MAEXAAVQStyle@@@Z 100206a0     qt-mt323:qt-mt323.dll
 0002:000006a4       __imp_?takeItem@QListViewItem@@UAEXPAV1@@Z 100206a4     qt-mt323:qt-mt323.dll
 0002:000006a8       __imp_?text@QListViewItem@@UBE?AVQString@@H@Z 100206a8     qt-mt323:qt-mt323.dll
 0002:000006ac       __imp_?widget@QLayoutItem@@UAEPAVQWidget@@XZ 100206ac     qt-mt323:qt-mt323.dll
 0002:000006b0       __imp_?width@QListViewItem@@UBEHABVQFontMetrics@@PBVQListView@@H@Z 100206b0     qt-mt323:qt-mt323.dll
 0002:000006b4       __imp_?write@QGList@@MBEAAVQDataStream@@AAV2@PAX@Z 100206b4     qt-mt323:qt-mt323.dll
 0002:000006b8       __imp_?null@QString@@2V1@A 100206b8     qt-mt323:qt-mt323.dll
 0002:000006bc       __imp_??_7?$QPtrList@VQDockWindow@@@@6B@ 100206bc     qt-mt323:qt-mt323.dll
 0002:000006c0       __imp_?setMinimumSize@QWidget@@QAEXABVQSize@@@Z 100206c0     qt-mt323:qt-mt323.dll
 0002:000006c4       __imp_?resize@QWidget@@QAEXABVQSize@@@Z 100206c4     qt-mt323:qt-mt323.dll
 0002:000006c8       __imp_??0QPushButton@@QAE@PAVQWidget@@PBD@Z 100206c8     qt-mt323:qt-mt323.dll
 0002:000006cc       __imp_??1QPushButton@@UAE@XZ 100206cc     qt-mt323:qt-mt323.dll
 0002:000006d0       __imp_??0QFrame@@QAE@PAVQWidget@@PBDI@Z 100206d0     qt-mt323:qt-mt323.dll
 0002:000006d4       __imp_?setFrameShape@QFrame@@QAEXW4Shape@1@@Z 100206d4     qt-mt323:qt-mt323.dll
 0002:000006d8       __imp_?setFrameShadow@QFrame@@QAEXW4Shadow@1@@Z 100206d8     qt-mt323:qt-mt323.dll
 0002:000006dc       __imp_??0QListBox@@QAE@PAVQWidget@@PBDI@Z 100206dc     qt-mt323:qt-mt323.dll
 0002:000006e0       __imp_??1QListBox@@UAE@XZ  100206e0     qt-mt323:qt-mt323.dll
 0002:000006e4       __imp_??0QGroupBox@@QAE@PAVQWidget@@PBD@Z 100206e4     qt-mt323:qt-mt323.dll
 0002:000006e8       __imp_??1QGroupBox@@UAE@XZ 100206e8     qt-mt323:qt-mt323.dll
 0002:000006ec       __imp_??0QLineEdit@@QAE@PAVQWidget@@PBD@Z 100206ec     qt-mt323:qt-mt323.dll
 0002:000006f0       __imp_??1QLineEdit@@UAE@XZ 100206f0     qt-mt323:qt-mt323.dll
 0002:000006f4       __imp_??1QLayoutItem@@UAE@XZ 100206f4     qt-mt323:qt-mt323.dll
 0002:000006f8       __imp_??0QSpacerItem@@QAE@HHW4SizeType@QSizePolicy@@0@Z 100206f8     qt-mt323:qt-mt323.dll
 0002:000006fc       __imp_?addLayout@QBoxLayout@@QAEXPAVQLayout@@H@Z 100206fc     qt-mt323:qt-mt323.dll
 0002:00000700       __imp_??0QHBoxLayout@@QAE@PAVQWidget@@HHPBD@Z 10020700     qt-mt323:qt-mt323.dll
 0002:00000704       __imp_??1QHBoxLayout@@UAE@XZ 10020704     qt-mt323:qt-mt323.dll
 0002:00000708       __imp_??0QVBoxLayout@@QAE@PAVQLayout@@HPBD@Z 10020708     qt-mt323:qt-mt323.dll
 0002:0000070c       __imp_?childEvent@QGroupBox@@MAEXPAVQChildEvent@@@Z 1002070c     qt-mt323:qt-mt323.dll
 0002:00000710       __imp_?className@QFrame@@UBEPBDXZ 10020710     qt-mt323:qt-mt323.dll
 0002:00000714       __imp_?className@QGroupBox@@UBEPBDXZ 10020714     qt-mt323:qt-mt323.dll
 0002:00000718       __imp_?className@QHBoxLayout@@UBEPBDXZ 10020718     qt-mt323:qt-mt323.dll
 0002:0000071c       __imp_?className@QLineEdit@@UBEPBDXZ 1002071c     qt-mt323:qt-mt323.dll
 0002:00000720       __imp_?className@QListBox@@UBEPBDXZ 10020720     qt-mt323:qt-mt323.dll
 0002:00000724       __imp_?className@QPushButton@@UBEPBDXZ 10020724     qt-mt323:qt-mt323.dll
 0002:00000728       __imp_?clear@QLineEdit@@UAEXXZ 10020728     qt-mt323:qt-mt323.dll
 0002:0000072c       __imp_?clearSelection@QListBox@@UAEXXZ 1002072c     qt-mt323:qt-mt323.dll
 0002:00000730       __imp_?clearValidator@QLineEdit@@UAEXXZ 10020730     qt-mt323:qt-mt323.dll
 0002:00000734       __imp_?contentsContextMenuEvent@QListBox@@MAEXPAVQContextMenuEvent@@@Z 10020734     qt-mt323:qt-mt323.dll
 0002:00000738       __imp_?contentsDragEnterEvent@QScrollView@@MAEXPAVQDragEnterEvent@@@Z 10020738     qt-mt323:qt-mt323.dll
 0002:0000073c       __imp_?contentsDragLeaveEvent@QScrollView@@MAEXPAVQDragLeaveEvent@@@Z 1002073c     qt-mt323:qt-mt323.dll
 0002:00000740       __imp_?contentsDragMoveEvent@QScrollView@@MAEXPAVQDragMoveEvent@@@Z 10020740     qt-mt323:qt-mt323.dll
 0002:00000744       __imp_?contentsDropEvent@QScrollView@@MAEXPAVQDropEvent@@@Z 10020744     qt-mt323:qt-mt323.dll
 0002:00000748       __imp_?contentsMouseDoubleClickEvent@QScrollView@@MAEXPAVQMouseEvent@@@Z 10020748     qt-mt323:qt-mt323.dll
 0002:0000074c       __imp_?contentsMouseMoveEvent@QScrollView@@MAEXPAVQMouseEvent@@@Z 1002074c     qt-mt323:qt-mt323.dll
 0002:00000750       __imp_?contentsMousePressEvent@QScrollView@@MAEXPAVQMouseEvent@@@Z 10020750     qt-mt323:qt-mt323.dll
 0002:00000754       __imp_?contentsMouseReleaseEvent@QScrollView@@MAEXPAVQMouseEvent@@@Z 10020754     qt-mt323:qt-mt323.dll
 0002:00000758       __imp_?contextMenuEvent@QLineEdit@@MAEXPAVQContextMenuEvent@@@Z 10020758     qt-mt323:qt-mt323.dll
 0002:0000075c       __imp_?copy@QLineEdit@@UBEXXZ 1002075c     qt-mt323:qt-mt323.dll
 0002:00000760       __imp_?createPopupMenu@QLineEdit@@MAEPAVQPopupMenu@@XZ 10020760     qt-mt323:qt-mt323.dll
 0002:00000764       __imp_?cut@QLineEdit@@UAEXXZ 10020764     qt-mt323:qt-mt323.dll
 0002:00000768       __imp_?deselect@QLineEdit@@UAEXXZ 10020768     qt-mt323:qt-mt323.dll
 0002:0000076c       __imp_?dragEnterEvent@QLineEdit@@MAEXPAVQDragEnterEvent@@@Z 1002076c     qt-mt323:qt-mt323.dll
 0002:00000770       __imp_?dragLeaveEvent@QLineEdit@@MAEXPAVQDragLeaveEvent@@@Z 10020770     qt-mt323:qt-mt323.dll
 0002:00000774       __imp_?dragMoveEvent@QLineEdit@@MAEXPAVQDragMoveEvent@@@Z 10020774     qt-mt323:qt-mt323.dll
 0002:00000778       __imp_?drawButton@QPushButton@@MAEXPAVQPainter@@@Z 10020778     qt-mt323:qt-mt323.dll
 0002:0000077c       __imp_?drawButtonLabel@QPushButton@@MAEXPAVQPainter@@@Z 1002077c     qt-mt323:qt-mt323.dll
 0002:00000780       __imp_?drawContents@QLineEdit@@MAEXPAVQPainter@@@Z 10020780     qt-mt323:qt-mt323.dll
 0002:00000784       __imp_?drawContentsOffset@QScrollView@@MAEXPAVQPainter@@HHHHHH@Z 10020784     qt-mt323:qt-mt323.dll
 0002:00000788       __imp_?dropEvent@QLineEdit@@MAEXPAVQDropEvent@@@Z 10020788     qt-mt323:qt-mt323.dll
 0002:0000078c       __imp_?enabledChange@QButton@@MAEX_N@Z 1002078c     qt-mt323:qt-mt323.dll
 0002:00000790       __imp_?ensureCurrentVisible@QListBox@@UAEXXZ 10020790     qt-mt323:qt-mt323.dll
 0002:00000794       __imp_?event@QGroupBox@@MAE_NPAVQEvent@@@Z 10020794     qt-mt323:qt-mt323.dll
 0002:00000798       __imp_?event@QLineEdit@@MAE_NPAVQEvent@@@Z 10020798     qt-mt323:qt-mt323.dll
 0002:0000079c       __imp_?eventFilter@QListBox@@MAE_NPAVQObject@@PAVQEvent@@@Z 1002079c     qt-mt323:qt-mt323.dll
 0002:000007a0       __imp_?expanding@QSpacerItem@@UBE?AW4ExpandData@QSizePolicy@@XZ 100207a0     qt-mt323:qt-mt323.dll
 0002:000007a4       __imp_?focusInEvent@QGroupBox@@MAEXPAVQFocusEvent@@@Z 100207a4     qt-mt323:qt-mt323.dll
 0002:000007a8       __imp_?focusInEvent@QLineEdit@@MAEXPAVQFocusEvent@@@Z 100207a8     qt-mt323:qt-mt323.dll
 0002:000007ac       __imp_?focusInEvent@QListBox@@MAEXPAVQFocusEvent@@@Z 100207ac     qt-mt323:qt-mt323.dll
 0002:000007b0       __imp_?focusInEvent@QPushButton@@MAEXPAVQFocusEvent@@@Z 100207b0     qt-mt323:qt-mt323.dll
 0002:000007b4       __imp_?focusOutEvent@QLineEdit@@MAEXPAVQFocusEvent@@@Z 100207b4     qt-mt323:qt-mt323.dll
 0002:000007b8       __imp_?focusOutEvent@QListBox@@MAEXPAVQFocusEvent@@@Z 100207b8     qt-mt323:qt-mt323.dll
 0002:000007bc       __imp_?focusOutEvent@QPushButton@@MAEXPAVQFocusEvent@@@Z 100207bc     qt-mt323:qt-mt323.dll
 0002:000007c0       __imp_?fontChange@QGroupBox@@MAEXABVQFont@@@Z 100207c0     qt-mt323:qt-mt323.dll
 0002:000007c4       __imp_?geometry@QSpacerItem@@UBE?AVQRect@@XZ 100207c4     qt-mt323:qt-mt323.dll
 0002:000007c8       __imp_?hasHeightForWidth@QLayoutItem@@UBE_NXZ 100207c8     qt-mt323:qt-mt323.dll
 0002:000007cc       __imp_?heightForWidth@QLayoutItem@@UBEHH@Z 100207cc     qt-mt323:qt-mt323.dll
 0002:000007d0       __imp_?hitButton@QButton@@MBE_NABVQPoint@@@Z 100207d0     qt-mt323:qt-mt323.dll
 0002:000007d4       __imp_?imComposeEvent@QLineEdit@@MAEXPAVQIMEvent@@@Z 100207d4     qt-mt323:qt-mt323.dll
 0002:000007d8       __imp_?imEndEvent@QLineEdit@@MAEXPAVQIMEvent@@@Z 100207d8     qt-mt323:qt-mt323.dll
 0002:000007dc       __imp_?imStartEvent@QLineEdit@@MAEXPAVQIMEvent@@@Z 100207dc     qt-mt323:qt-mt323.dll
 0002:000007e0       __imp_?insert@QLineEdit@@UAEXABVQString@@@Z 100207e0     qt-mt323:qt-mt323.dll
 0002:000007e4       __imp_?invalidate@QLayoutItem@@UAEXXZ 100207e4     qt-mt323:qt-mt323.dll
 0002:000007e8       __imp_?invertSelection@QListBox@@UAEXXZ 100207e8     qt-mt323:qt-mt323.dll
 0002:000007ec       __imp_?isEmpty@QSpacerItem@@UBE_NXZ 100207ec     qt-mt323:qt-mt323.dll
 0002:000007f0       __imp_?iterator@QLayoutItem@@UAE?AVQLayoutIterator@@XZ 100207f0     qt-mt323:qt-mt323.dll
 0002:000007f4       __imp_?keyPressEvent@QButton@@MAEXPAVQKeyEvent@@@Z 100207f4     qt-mt323:qt-mt323.dll
 0002:000007f8       __imp_?keyPressEvent@QLineEdit@@MAEXPAVQKeyEvent@@@Z 100207f8     qt-mt323:qt-mt323.dll
 0002:000007fc       __imp_?keyPressEvent@QListBox@@MAEXPAVQKeyEvent@@@Z 100207fc     qt-mt323:qt-mt323.dll
 0002:00000800       __imp_?keyReleaseEvent@QButton@@MAEXPAVQKeyEvent@@@Z 10020800     qt-mt323:qt-mt323.dll
 0002:00000804       __imp_?layout@QLayoutItem@@UAEPAVQLayout@@XZ 10020804     qt-mt323:qt-mt323.dll
 0002:00000808       __imp_?maximumSize@QSpacerItem@@UBE?AVQSize@@XZ 10020808     qt-mt323:qt-mt323.dll
 0002:0000080c       __imp_?metaObject@QFrame@@UBEPAVQMetaObject@@XZ 1002080c     qt-mt323:qt-mt323.dll
 0002:00000810       __imp_?metaObject@QGroupBox@@UBEPAVQMetaObject@@XZ 10020810     qt-mt323:qt-mt323.dll
 0002:00000814       __imp_?metaObject@QHBoxLayout@@UBEPAVQMetaObject@@XZ 10020814     qt-mt323:qt-mt323.dll
 0002:00000818       __imp_?metaObject@QLineEdit@@UBEPAVQMetaObject@@XZ 10020818     qt-mt323:qt-mt323.dll
 0002:0000081c       __imp_?metaObject@QListBox@@UBEPAVQMetaObject@@XZ 1002081c     qt-mt323:qt-mt323.dll
 0002:00000820       __imp_?metaObject@QPushButton@@UBEPAVQMetaObject@@XZ 10020820     qt-mt323:qt-mt323.dll
 0002:00000824       __imp_?minimumSize@QSpacerItem@@UBE?AVQSize@@XZ 10020824     qt-mt323:qt-mt323.dll
 0002:00000828       __imp_?minimumSizeHint@QLineEdit@@UBE?AVQSize@@XZ 10020828     qt-mt323:qt-mt323.dll
 0002:0000082c       __imp_?minimumSizeHint@QListBox@@UBE?AVQSize@@XZ 1002082c     qt-mt323:qt-mt323.dll
 0002:00000830       __imp_?mouseDoubleClickEvent@QLineEdit@@MAEXPAVQMouseEvent@@@Z 10020830     qt-mt323:qt-mt323.dll
 0002:00000834       __imp_?mouseDoubleClickEvent@QListBox@@MAEXPAVQMouseEvent@@@Z 10020834     qt-mt323:qt-mt323.dll
 0002:00000838       __imp_?mouseMoveEvent@QButton@@MAEXPAVQMouseEvent@@@Z 10020838     qt-mt323:qt-mt323.dll
 0002:0000083c       __imp_?mouseMoveEvent@QLineEdit@@MAEXPAVQMouseEvent@@@Z 1002083c     qt-mt323:qt-mt323.dll
 0002:00000840       __imp_?mouseMoveEvent@QListBox@@MAEXPAVQMouseEvent@@@Z 10020840     qt-mt323:qt-mt323.dll
 0002:00000844       __imp_?mousePressEvent@QButton@@MAEXPAVQMouseEvent@@@Z 10020844     qt-mt323:qt-mt323.dll
 0002:00000848       __imp_?mousePressEvent@QLineEdit@@MAEXPAVQMouseEvent@@@Z 10020848     qt-mt323:qt-mt323.dll
 0002:0000084c       __imp_?mousePressEvent@QListBox@@MAEXPAVQMouseEvent@@@Z 1002084c     qt-mt323:qt-mt323.dll
 0002:00000850       __imp_?mouseReleaseEvent@QButton@@MAEXPAVQMouseEvent@@@Z 10020850     qt-mt323:qt-mt323.dll
 0002:00000854       __imp_?mouseReleaseEvent@QLineEdit@@MAEXPAVQMouseEvent@@@Z 10020854     qt-mt323:qt-mt323.dll
 0002:00000858       __imp_?mouseReleaseEvent@QListBox@@MAEXPAVQMouseEvent@@@Z 10020858     qt-mt323:qt-mt323.dll
 0002:0000085c       __imp_?move@QPushButton@@UAEXHH@Z 1002085c     qt-mt323:qt-mt323.dll
 0002:00000860       __imp_?paintCell@QListBox@@MAEXPAVQPainter@@HH@Z 10020860     qt-mt323:qt-mt323.dll
 0002:00000864       __imp_?paintEvent@QButton@@MAEXPAVQPaintEvent@@@Z 10020864     qt-mt323:qt-mt323.dll
 0002:00000868       __imp_?paintEvent@QGroupBox@@MAEXPAVQPaintEvent@@@Z 10020868     qt-mt323:qt-mt323.dll
 0002:0000086c       __imp_?paste@QLineEdit@@UAEXXZ 1002086c     qt-mt323:qt-mt323.dll
 0002:00000870       __imp_?qt_cast@QFrame@@UAEPAXPBD@Z 10020870     qt-mt323:qt-mt323.dll
 0002:00000874       __imp_?qt_cast@QGroupBox@@UAEPAXPBD@Z 10020874     qt-mt323:qt-mt323.dll
 0002:00000878       __imp_?qt_cast@QHBoxLayout@@UAEPAXPBD@Z 10020878     qt-mt323:qt-mt323.dll
 0002:0000087c       __imp_?qt_cast@QLineEdit@@UAEPAXPBD@Z 1002087c     qt-mt323:qt-mt323.dll
 0002:00000880       __imp_?qt_cast@QListBox@@UAEPAXPBD@Z 10020880     qt-mt323:qt-mt323.dll
 0002:00000884       __imp_?qt_cast@QPushButton@@UAEPAXPBD@Z 10020884     qt-mt323:qt-mt323.dll
 0002:00000888       __imp_?qt_emit@QFrame@@UAE_NHPAUQUObject@@@Z 10020888     qt-mt323:qt-mt323.dll
 0002:0000088c       __imp_?qt_emit@QGroupBox@@UAE_NHPAUQUObject@@@Z 1002088c     qt-mt323:qt-mt323.dll
 0002:00000890       __imp_?qt_emit@QHBoxLayout@@UAE_NHPAUQUObject@@@Z 10020890     qt-mt323:qt-mt323.dll
 0002:00000894       __imp_?qt_emit@QLineEdit@@UAE_NHPAUQUObject@@@Z 10020894     qt-mt323:qt-mt323.dll
 0002:00000898       __imp_?qt_emit@QListBox@@UAE_NHPAUQUObject@@@Z 10020898     qt-mt323:qt-mt323.dll
 0002:0000089c       __imp_?qt_emit@QPushButton@@UAE_NHPAUQUObject@@@Z 1002089c     qt-mt323:qt-mt323.dll
 0002:000008a0       __imp_?qt_invoke@QFrame@@UAE_NHPAUQUObject@@@Z 100208a0     qt-mt323:qt-mt323.dll
 0002:000008a4       __imp_?qt_invoke@QGroupBox@@UAE_NHPAUQUObject@@@Z 100208a4     qt-mt323:qt-mt323.dll
 0002:000008a8       __imp_?qt_invoke@QHBoxLayout@@UAE_NHPAUQUObject@@@Z 100208a8     qt-mt323:qt-mt323.dll
 0002:000008ac       __imp_?qt_invoke@QLineEdit@@UAE_NHPAUQUObject@@@Z 100208ac     qt-mt323:qt-mt323.dll
 0002:000008b0       __imp_?qt_invoke@QListBox@@UAE_NHPAUQUObject@@@Z 100208b0     qt-mt323:qt-mt323.dll
 0002:000008b4       __imp_?qt_invoke@QPushButton@@UAE_NHPAUQUObject@@@Z 100208b4     qt-mt323:qt-mt323.dll
 0002:000008b8       __imp_?qt_property@QFrame@@UAE_NHHPAVQVariant@@@Z 100208b8     qt-mt323:qt-mt323.dll
 0002:000008bc       __imp_?qt_property@QGroupBox@@UAE_NHHPAVQVariant@@@Z 100208bc     qt-mt323:qt-mt323.dll
 0002:000008c0       __imp_?qt_property@QHBoxLayout@@UAE_NHHPAVQVariant@@@Z 100208c0     qt-mt323:qt-mt323.dll
 0002:000008c4       __imp_?qt_property@QLineEdit@@UAE_NHHPAVQVariant@@@Z 100208c4     qt-mt323:qt-mt323.dll
 0002:000008c8       __imp_?qt_property@QListBox@@UAE_NHHPAVQVariant@@@Z 100208c8     qt-mt323:qt-mt323.dll
 0002:000008cc       __imp_?qt_property@QPushButton@@UAE_NHHPAVQVariant@@@Z 100208cc     qt-mt323:qt-mt323.dll
 0002:000008d0       __imp_?redo@QLineEdit@@UAEXXZ 100208d0     qt-mt323:qt-mt323.dll
 0002:000008d4       __imp_?resize@QPushButton@@UAEXHH@Z 100208d4     qt-mt323:qt-mt323.dll
 0002:000008d8       __imp_?resizeEvent@QFrame@@MAEXPAVQResizeEvent@@@Z 100208d8     qt-mt323:qt-mt323.dll
 0002:000008dc       __imp_?resizeEvent@QGroupBox@@MAEXPAVQResizeEvent@@@Z 100208dc     qt-mt323:qt-mt323.dll
 0002:000008e0       __imp_?resizeEvent@QLineEdit@@MAEXPAVQResizeEvent@@@Z 100208e0     qt-mt323:qt-mt323.dll
 0002:000008e4       __imp_?resizeEvent@QListBox@@MAEXPAVQResizeEvent@@@Z 100208e4     qt-mt323:qt-mt323.dll
 0002:000008e8       __imp_?resizeEvent@QPushButton@@MAEXPAVQResizeEvent@@@Z 100208e8     qt-mt323:qt-mt323.dll
 0002:000008ec       __imp_?selectAll@QLineEdit@@UAEXXZ 100208ec     qt-mt323:qt-mt323.dll
 0002:000008f0       __imp_?selectAll@QListBox@@UAEX_N@Z 100208f0     qt-mt323:qt-mt323.dll
 0002:000008f4       __imp_?setAccel@QButton@@UAEXABVQKeySequence@@@Z 100208f4     qt-mt323:qt-mt323.dll
 0002:000008f8       __imp_?setAlignment@QGroupBox@@UAEXH@Z 100208f8     qt-mt323:qt-mt323.dll
 0002:000008fc       __imp_?setAlignment@QLineEdit@@UAEXH@Z 100208fc     qt-mt323:qt-mt323.dll
 0002:00000900       __imp_?setAutoDefault@QPushButton@@UAEX_N@Z 10020900     qt-mt323:qt-mt323.dll
 0002:00000904       __imp_?setAutoRepeat@QButton@@UAEX_N@Z 10020904     qt-mt323:qt-mt323.dll
 0002:00000908       __imp_?setBottomItem@QListBox@@UAEXH@Z 10020908     qt-mt323:qt-mt323.dll
 0002:0000090c       __imp_?setColumnLayout@QGroupBox@@UAEXHW4Orientation@Qt@@@Z 1002090c     qt-mt323:qt-mt323.dll
 0002:00000910       __imp_?setColumnMode@QListBox@@UAEXH@Z 10020910     qt-mt323:qt-mt323.dll
 0002:00000914       __imp_?setColumnMode@QListBox@@UAEXW4LayoutMode@1@@Z 10020914     qt-mt323:qt-mt323.dll
 0002:00000918       __imp_?setContentsPos@QScrollView@@UAEXHH@Z 10020918     qt-mt323:qt-mt323.dll
 0002:0000091c       __imp_?setCurrentItem@QListBox@@UAEXH@Z 1002091c     qt-mt323:qt-mt323.dll
 0002:00000920       __imp_?setCurrentItem@QListBox@@UAEXPAVQListBoxItem@@@Z 10020920     qt-mt323:qt-mt323.dll
 0002:00000924       __imp_?setCursorPosition@QLineEdit@@UAEXH@Z 10020924     qt-mt323:qt-mt323.dll
 0002:00000928       __imp_?setDefault@QPushButton@@UAEX_N@Z 10020928     qt-mt323:qt-mt323.dll
 0002:0000092c       __imp_?setDown@QButton@@UAEX_N@Z 1002092c     qt-mt323:qt-mt323.dll
 0002:00000930       __imp_?setDragEnabled@QLineEdit@@UAEX_N@Z 10020930     qt-mt323:qt-mt323.dll
 0002:00000934       __imp_?setEchoMode@QLineEdit@@UAEXW4EchoMode@1@@Z 10020934     qt-mt323:qt-mt323.dll
 0002:00000938       __imp_?setEnabled@QGroupBox@@UAEX_N@Z 10020938     qt-mt323:qt-mt323.dll
 0002:0000093c       __imp_?setFont@QLineEdit@@UAEXABVQFont@@@Z 1002093c     qt-mt323:qt-mt323.dll
 0002:00000940       __imp_?setFont@QListBox@@UAEXABVQFont@@@Z 10020940     qt-mt323:qt-mt323.dll
 0002:00000944       __imp_?setFrame@QLineEdit@@UAEX_N@Z 10020944     qt-mt323:qt-mt323.dll
 0002:00000948       __imp_?setGeometry@QPushButton@@UAEXABVQRect@@@Z 10020948     qt-mt323:qt-mt323.dll
 0002:0000094c       __imp_?setGeometry@QPushButton@@UAEXHHHH@Z 1002094c     qt-mt323:qt-mt323.dll
 0002:00000950       __imp_?mouseReleaseEvent@QWidget@@MAEXPAVQMouseEvent@@@Z 10020950     qt-mt323:qt-mt323.dll
 0002:00000954       __imp_?setGroup@QButton@@EAEXPAVQButtonGroup@@@Z 10020954     qt-mt323:qt-mt323.dll
 0002:00000958       __imp_?setIsMenuButton@QPushButton@@UAEX_N@Z 10020958     qt-mt323:qt-mt323.dll
 0002:0000095c       __imp_?setMaxLength@QLineEdit@@UAEXH@Z 1002095c     qt-mt323:qt-mt323.dll
 0002:00000960       __imp_?setOn@QPushButton@@UAEX_N@Z 10020960     qt-mt323:qt-mt323.dll
 0002:00000964       __imp_?setPalette@QLineEdit@@UAEXABVQPalette@@@Z 10020964     qt-mt323:qt-mt323.dll
 0002:00000968       __imp_?setPixmap@QButton@@UAEXABVQPixmap@@@Z 10020968     qt-mt323:qt-mt323.dll
 0002:0000096c       __imp_?setReadOnly@QLineEdit@@UAEX_N@Z 1002096c     qt-mt323:qt-mt323.dll
 0002:00000970       __imp_?setRowMode@QListBox@@UAEXH@Z 10020970     qt-mt323:qt-mt323.dll
 0002:00000974       __imp_?setRowMode@QListBox@@UAEXW4LayoutMode@1@@Z 10020974     qt-mt323:qt-mt323.dll
 0002:00000978       __imp_?setSelected@QListBox@@UAEXPAVQListBoxItem@@_N@Z 10020978     qt-mt323:qt-mt323.dll
 0002:0000097c       __imp_?setSelection@QLineEdit@@UAEXHH@Z 1002097c     qt-mt323:qt-mt323.dll
 0002:00000980       __imp_?setSelectionMode@QListBox@@UAEXW4SelectionMode@1@@Z 10020980     qt-mt323:qt-mt323.dll
 0002:00000984       __imp_?setState@QButton@@MAEXW4ToggleState@1@@Z 10020984     qt-mt323:qt-mt323.dll
 0002:00000988       __imp_?setText@QButton@@UAEXABVQString@@@Z 10020988     qt-mt323:qt-mt323.dll
 0002:0000098c       __imp_?setText@QLineEdit@@UAEXABVQString@@@Z 1002098c     qt-mt323:qt-mt323.dll
 0002:00000990       __imp_?setTitle@QGroupBox@@UAEXABVQString@@@Z 10020990     qt-mt323:qt-mt323.dll
 0002:00000994       __imp_?setToggleType@QButton@@MAEXW4ToggleType@1@@Z 10020994     qt-mt323:qt-mt323.dll
 0002:00000998       __imp_?setTopItem@QListBox@@UAEXH@Z 10020998     qt-mt323:qt-mt323.dll
 0002:0000099c       __imp_?setValidator@QLineEdit@@UAEXPBVQValidator@@@Z 1002099c     qt-mt323:qt-mt323.dll
 0002:000009a0       __imp_?setVariableHeight@QListBox@@UAEX_N@Z 100209a0     qt-mt323:qt-mt323.dll
 0002:000009a4       __imp_?setVariableWidth@QListBox@@UAEX_N@Z 100209a4     qt-mt323:qt-mt323.dll
 0002:000009a8       __imp_?show@QScrollView@@UAEXXZ 100209a8     qt-mt323:qt-mt323.dll
 0002:000009ac       __imp_?showEvent@QListBox@@MAEXPAVQShowEvent@@@Z 100209ac     qt-mt323:qt-mt323.dll
 0002:000009b0       __imp_?sizeHint@QFrame@@UBE?AVQSize@@XZ 100209b0     qt-mt323:qt-mt323.dll
 0002:000009b4       __imp_?sizeHint@QGroupBox@@UBE?AVQSize@@XZ 100209b4     qt-mt323:qt-mt323.dll
 0002:000009b8       __imp_?sizeHint@QLineEdit@@UBE?AVQSize@@XZ 100209b8     qt-mt323:qt-mt323.dll
 0002:000009bc       __imp_?sizeHint@QListBox@@UBE?AVQSize@@XZ 100209bc     qt-mt323:qt-mt323.dll
 0002:000009c0       __imp_?sizeHint@QPushButton@@UBE?AVQSize@@XZ 100209c0     qt-mt323:qt-mt323.dll
 0002:000009c4       __imp_?sizeHint@QSpacerItem@@UBE?AVQSize@@XZ 100209c4     qt-mt323:qt-mt323.dll
 0002:000009c8       __imp_?spacerItem@QSpacerItem@@UAEPAV1@XZ 100209c8     qt-mt323:qt-mt323.dll
 0002:000009cc       __imp_?styleChange@QScrollView@@UAEXAAVQStyle@@@Z 100209cc     qt-mt323:qt-mt323.dll
 0002:000009d0       __imp_?undo@QLineEdit@@UAEXXZ 100209d0     qt-mt323:qt-mt323.dll
 0002:000009d4       __imp_?updateMask@QPushButton@@MAEXXZ 100209d4     qt-mt323:qt-mt323.dll
 0002:000009d8       __imp_?viewportPaintEvent@QListBox@@UAEXPAVQPaintEvent@@@Z 100209d8     qt-mt323:qt-mt323.dll
 0002:000009dc       __imp_?viewportResizeEvent@QScrollView@@MAEXPAVQResizeEvent@@@Z 100209dc     qt-mt323:qt-mt323.dll
 0002:000009e0       __imp_?windowActivationChange@QLineEdit@@MAEX_N@Z 100209e0     qt-mt323:qt-mt323.dll
 0002:000009e4       __imp_?windowActivationChange@QListBox@@MAEX_N@Z 100209e4     qt-mt323:qt-mt323.dll
 0002:000009e8       __imp_??6?$QValueList@VQString@@@@QAEAAV0@ABVQString@@@Z 100209e8     qt-mt323:qt-mt323.dll
 0002:000009ec       __imp_??1QTable@@UAE@XZ    100209ec     qt-mt323:qt-mt323.dll
 0002:000009f0       __imp_?setSelectionMode@QTable@@UAEXW4SelectionMode@1@@Z 100209f0     qt-mt323:qt-mt323.dll
 0002:000009f4       __imp_?insertColumns@QTable@@UAEXHH@Z 100209f4     qt-mt323:qt-mt323.dll
 0002:000009f8       __imp_?setColumnLabels@QTable@@QAEXABVQStringList@@@Z 100209f8     qt-mt323:qt-mt323.dll
 0002:000009fc       __imp_?endEdit@QTable@@MAEXHH_N0@Z 100209fc     qt-mt323:qt-mt323.dll
 0002:00000a00       __imp_?isEditing@QTable@@IBE_NXZ 10020a00     qt-mt323:qt-mt323.dll
 0002:00000a04       __imp_?currEditRow@QTable@@IBEHXZ 10020a04     qt-mt323:qt-mt323.dll
 0002:00000a08       __imp_?currEditCol@QTable@@IBEHXZ 10020a08     qt-mt323:qt-mt323.dll
 0002:00000a0c       __imp_?activateNextCell@QTable@@MAEXXZ 10020a0c     qt-mt323:qt-mt323.dll
 0002:00000a10       __imp_?addSelection@QTable@@UAEHABVQTableSelection@@@Z 10020a10     qt-mt323:qt-mt323.dll
 0002:00000a14       __imp_?adjustColumn@QTable@@UAEXH@Z 10020a14     qt-mt323:qt-mt323.dll
 0002:00000a18       __imp_?adjustRow@QTable@@UAEXH@Z 10020a18     qt-mt323:qt-mt323.dll
 0002:00000a1c       __imp_?beginEdit@QTable@@MAEPAVQWidget@@HH_N@Z 10020a1c     qt-mt323:qt-mt323.dll
 0002:00000a20       __imp_?cellGeometry@QTable@@UBE?AVQRect@@HH@Z 10020a20     qt-mt323:qt-mt323.dll
 0002:00000a24       __imp_?cellRect@QTable@@UBE?AVQRect@@HH@Z 10020a24     qt-mt323:qt-mt323.dll
 0002:00000a28       __imp_?cellWidget@QTable@@UBEPAVQWidget@@HH@Z 10020a28     qt-mt323:qt-mt323.dll
 0002:00000a2c       __imp_?clearCell@QTable@@UAEXHH@Z 10020a2c     qt-mt323:qt-mt323.dll
 0002:00000a30       __imp_?clearCellWidget@QTable@@UAEXHH@Z 10020a30     qt-mt323:qt-mt323.dll
 0002:00000a34       __imp_?columnAt@QTable@@UBEHH@Z 10020a34     qt-mt323:qt-mt323.dll
 0002:00000a38       __imp_?columnClicked@QTable@@MAEXH@Z 10020a38     qt-mt323:qt-mt323.dll
 0002:00000a3c       __imp_?columnIndexChanged@QTable@@MAEXHHH@Z 10020a3c     qt-mt323:qt-mt323.dll
 0002:00000a40       __imp_?columnPos@QTable@@UBEHH@Z 10020a40     qt-mt323:qt-mt323.dll
 0002:00000a44       __imp_?columnWidth@QTable@@UBEHH@Z 10020a44     qt-mt323:qt-mt323.dll
 0002:00000a48       __imp_?columnWidthChanged@QTable@@MAEXH@Z 10020a48     qt-mt323:qt-mt323.dll
 0002:00000a4c       __imp_?contentsContextMenuEvent@QTable@@MAEXPAVQContextMenuEvent@@@Z 10020a4c     qt-mt323:qt-mt323.dll
 0002:00000a50       __imp_?contentsDragEnterEvent@QTable@@MAEXPAVQDragEnterEvent@@@Z 10020a50     qt-mt323:qt-mt323.dll
 0002:00000a54       __imp_?contentsDragLeaveEvent@QTable@@MAEXPAVQDragLeaveEvent@@@Z 10020a54     qt-mt323:qt-mt323.dll
 0002:00000a58       __imp_?contentsDragMoveEvent@QTable@@MAEXPAVQDragMoveEvent@@@Z 10020a58     qt-mt323:qt-mt323.dll
 0002:00000a5c       __imp_?contentsDropEvent@QTable@@MAEXPAVQDropEvent@@@Z 10020a5c     qt-mt323:qt-mt323.dll
 0002:00000a60       __imp_?contentsMouseDoubleClickEvent@QTable@@MAEXPAVQMouseEvent@@@Z 10020a60     qt-mt323:qt-mt323.dll
 0002:00000a64       __imp_?contentsMouseMoveEvent@QTable@@MAEXPAVQMouseEvent@@@Z 10020a64     qt-mt323:qt-mt323.dll
 0002:00000a68       __imp_?contentsMousePressEvent@QTable@@MAEXPAVQMouseEvent@@@Z 10020a68     qt-mt323:qt-mt323.dll
 0002:00000a6c       __imp_?contentsMouseReleaseEvent@QTable@@MAEXPAVQMouseEvent@@@Z 10020a6c     qt-mt323:qt-mt323.dll
 0002:00000a70       __imp_?createEditor@QTable@@MBEPAVQWidget@@HH_N@Z 10020a70     qt-mt323:qt-mt323.dll
 0002:00000a74       __imp_?currentSelection@QTable@@UBEHXZ 10020a74     qt-mt323:qt-mt323.dll
 0002:00000a78       __imp_?dragObject@QTable@@MAEPAVQDragObject@@XZ 10020a78     qt-mt323:qt-mt323.dll
 0002:00000a7c       __imp_?drawContents@QTable@@EAEXPAVQPainter@@@Z 10020a7c     qt-mt323:qt-mt323.dll
 0002:00000a80       __imp_?drawContents@QTable@@MAEXPAVQPainter@@HHHH@Z 10020a80     qt-mt323:qt-mt323.dll
 0002:00000a84       __imp_?editCell@QTable@@UAEXHH_N@Z 10020a84     qt-mt323:qt-mt323.dll
 0002:00000a88       __imp_?eventFilter@QTable@@UAE_NPAVQObject@@PAVQEvent@@@Z 10020a88     qt-mt323:qt-mt323.dll
 0002:00000a8c       __imp_?focusInEvent@QTable@@MAEXPAVQFocusEvent@@@Z 10020a8c     qt-mt323:qt-mt323.dll
 0002:00000a90       __imp_?focusOutEvent@QTable@@MAEXPAVQFocusEvent@@@Z 10020a90     qt-mt323:qt-mt323.dll
 0002:00000a94       __imp_?hideColumn@QTable@@UAEXH@Z 10020a94     qt-mt323:qt-mt323.dll
 0002:00000a98       __imp_?hideRow@QTable@@UAEXH@Z 10020a98     qt-mt323:qt-mt323.dll
 0002:00000a9c       __imp_?insertRows@QTable@@UAEXHH@Z 10020a9c     qt-mt323:qt-mt323.dll
 0002:00000aa0       __imp_?insertWidget@QTable@@MAEXHHPAVQWidget@@@Z 10020aa0     qt-mt323:qt-mt323.dll
 0002:00000aa4       __imp_?item@QTable@@UBEPAVQTableItem@@HH@Z 10020aa4     qt-mt323:qt-mt323.dll
 0002:00000aa8       __imp_?keyPressEvent@QTable@@MAEXPAVQKeyEvent@@@Z 10020aa8     qt-mt323:qt-mt323.dll
 0002:00000aac       __imp_?minimumSizeHint@QScrollView@@UBE?AVQSize@@XZ 10020aac     qt-mt323:qt-mt323.dll
 0002:00000ab0       __imp_?numCols@QTable@@UBEHXZ 10020ab0     qt-mt323:qt-mt323.dll
 0002:00000ab4       __imp_?numRows@QTable@@UBEHXZ 10020ab4     qt-mt323:qt-mt323.dll
 0002:00000ab8       __imp_?paintCell@QTable@@UAEXPAVQPainter@@HHABVQRect@@_N@Z 10020ab8     qt-mt323:qt-mt323.dll
 0002:00000abc       __imp_?paintCell@QTable@@UAEXPAVQPainter@@HHABVQRect@@_NABVQColorGroup@@@Z 10020abc     qt-mt323:qt-mt323.dll
 0002:00000ac0       __imp_?paintEmptyArea@QTable@@MAEXPAVQPainter@@HHHH@Z 10020ac0     qt-mt323:qt-mt323.dll
 0002:00000ac4       __imp_?paintEvent@QTable@@MAEXPAVQPaintEvent@@@Z 10020ac4     qt-mt323:qt-mt323.dll
 0002:00000ac8       __imp_?paintFocus@QTable@@UAEXPAVQPainter@@ABVQRect@@@Z 10020ac8     qt-mt323:qt-mt323.dll
 0002:00000acc       __imp_?pixmap@QTable@@UBE?AVQPixmap@@HH@Z 10020acc     qt-mt323:qt-mt323.dll
 0002:00000ad0       __imp_?removeColumn@QTable@@UAEXH@Z 10020ad0     qt-mt323:qt-mt323.dll
 0002:00000ad4       __imp_?removeColumns@QTable@@UAEXABV?$QMemArray@H@@@Z 10020ad4     qt-mt323:qt-mt323.dll
 0002:00000ad8       __imp_?removeRow@QTable@@UAEXH@Z 10020ad8     qt-mt323:qt-mt323.dll
 0002:00000adc       __imp_?removeRows@QTable@@UAEXABV?$QMemArray@H@@@Z 10020adc     qt-mt323:qt-mt323.dll
 0002:00000ae0       __imp_?removeSelection@QTable@@UAEXABVQTableSelection@@@Z 10020ae0     qt-mt323:qt-mt323.dll
 0002:00000ae4       __imp_?removeSelection@QTable@@UAEXH@Z 10020ae4     qt-mt323:qt-mt323.dll
 0002:00000ae8       __imp_?resizeData@QTable@@MAEXH@Z 10020ae8     qt-mt323:qt-mt323.dll
 0002:00000aec       __imp_?resizeEvent@QScrollView@@MAEXPAVQResizeEvent@@@Z 10020aec     qt-mt323:qt-mt323.dll
 0002:00000af0       __imp_?rowAt@QTable@@UBEHH@Z 10020af0     qt-mt323:qt-mt323.dll
 0002:00000af4       __imp_?rowHeight@QTable@@UBEHH@Z 10020af4     qt-mt323:qt-mt323.dll
 0002:00000af8       __imp_?rowHeightChanged@QTable@@MAEXH@Z 10020af8     qt-mt323:qt-mt323.dll
 0002:00000afc       __imp_?rowIndexChanged@QTable@@MAEXHHH@Z 10020afc     qt-mt323:qt-mt323.dll
 0002:00000b00       __imp_?rowPos@QTable@@UBEHH@Z 10020b00     qt-mt323:qt-mt323.dll
 0002:00000b04       __imp_?setCellContentFromEditor@QTable@@MAEXHH@Z 10020b04     qt-mt323:qt-mt323.dll
 0002:00000b08       __imp_?setCellWidget@QTable@@UAEXHHPAVQWidget@@@Z 10020b08     qt-mt323:qt-mt323.dll
 0002:00000b0c       __imp_?setColumnMovingEnabled@QTable@@UAEX_N@Z 10020b0c     qt-mt323:qt-mt323.dll
 0002:00000b10       __imp_?setColumnReadOnly@QTable@@UAEXH_N@Z 10020b10     qt-mt323:qt-mt323.dll
 0002:00000b14       __imp_?setColumnStretchable@QTable@@UAEXH_N@Z 10020b14     qt-mt323:qt-mt323.dll
 0002:00000b18       __imp_?setColumnWidth@QTable@@UAEXHH@Z 10020b18     qt-mt323:qt-mt323.dll
 0002:00000b1c       __imp_?setCurrentCell@QTable@@UAEXHH@Z 10020b1c     qt-mt323:qt-mt323.dll
 0002:00000b20       __imp_?setDragEnabled@QTable@@UAEX_N@Z 10020b20     qt-mt323:qt-mt323.dll
 0002:00000b24       __imp_?setEnabled@QTable@@UAEX_N@Z 10020b24     qt-mt323:qt-mt323.dll
 0002:00000b28       __imp_?setFocusStyle@QTable@@UAEXW4FocusStyle@1@@Z 10020b28     qt-mt323:qt-mt323.dll
 0002:00000b2c       __imp_?setItem@QTable@@UAEXHHPAVQTableItem@@@Z 10020b2c     qt-mt323:qt-mt323.dll
 0002:00000b30       __imp_?setLeftMargin@QTable@@UAEXH@Z 10020b30     qt-mt323:qt-mt323.dll
 0002:00000b34       __imp_?setNumCols@QTable@@UAEXH@Z 10020b34     qt-mt323:qt-mt323.dll
 0002:00000b38       __imp_?setNumRows@QTable@@UAEXH@Z 10020b38     qt-mt323:qt-mt323.dll
 0002:00000b3c       __imp_?setPixmap@QTable@@UAEXHHABVQPixmap@@@Z 10020b3c     qt-mt323:qt-mt323.dll
 0002:00000b40       __imp_?setReadOnly@QTable@@UAEX_N@Z 10020b40     qt-mt323:qt-mt323.dll
 0002:00000b44       __imp_?setRowHeight@QTable@@UAEXHH@Z 10020b44     qt-mt323:qt-mt323.dll
 0002:00000b48       __imp_?setRowMovingEnabled@QTable@@UAEX_N@Z 10020b48     qt-mt323:qt-mt323.dll
 0002:00000b4c       __imp_?setRowReadOnly@QTable@@UAEXH_N@Z 10020b4c     qt-mt323:qt-mt323.dll
 0002:00000b50       __imp_?setRowStretchable@QTable@@UAEXH_N@Z 10020b50     qt-mt323:qt-mt323.dll
 0002:00000b54       __imp_?setShowGrid@QTable@@UAEX_N@Z 10020b54     qt-mt323:qt-mt323.dll
 0002:00000b58       __imp_?setSorting@QTable@@UAEX_N@Z 10020b58     qt-mt323:qt-mt323.dll
 0002:00000b5c       __imp_?setText@QTable@@UAEXHHABVQString@@@Z 10020b5c     qt-mt323:qt-mt323.dll
 0002:00000b60       __imp_?setTopMargin@QTable@@UAEXH@Z 10020b60     qt-mt323:qt-mt323.dll
 0002:00000b64       __imp_?showColumn@QTable@@UAEXH@Z 10020b64     qt-mt323:qt-mt323.dll
 0002:00000b68       __imp_?showEvent@QTable@@MAEXPAVQShowEvent@@@Z 10020b68     qt-mt323:qt-mt323.dll
 0002:00000b6c       __imp_?showRow@QTable@@UAEXH@Z 10020b6c     qt-mt323:qt-mt323.dll
 0002:00000b70       __imp_?sizeHint@QTable@@UBE?AVQSize@@XZ 10020b70     qt-mt323:qt-mt323.dll
 0002:00000b74       __imp_?sortColumn@QTable@@UAEXH_N0@Z 10020b74     qt-mt323:qt-mt323.dll
 0002:00000b78       __imp_?startDrag@QTable@@MAEXXZ 10020b78     qt-mt323:qt-mt323.dll
 0002:00000b7c       __imp_?swapCells@QTable@@UAEXHHHH@Z 10020b7c     qt-mt323:qt-mt323.dll
 0002:00000b80       __imp_?swapColumns@QTable@@UAEXHH_N@Z 10020b80     qt-mt323:qt-mt323.dll
 0002:00000b84       __imp_?swapRows@QTable@@UAEXHH_N@Z 10020b84     qt-mt323:qt-mt323.dll
 0002:00000b88       __imp_?takeItem@QTable@@UAEXPAVQTableItem@@@Z 10020b88     qt-mt323:qt-mt323.dll
 0002:00000b8c       __imp_?text@QTable@@UBE?AVQString@@HH@Z 10020b8c     qt-mt323:qt-mt323.dll
 0002:00000b90       __imp_?viewportResizeEvent@QTable@@MAEXPAVQResizeEvent@@@Z 10020b90     qt-mt323:qt-mt323.dll
 0002:00000b94       __imp_?windowActivationChange@QTable@@MAEX_N@Z 10020b94     qt-mt323:qt-mt323.dll
 0002:00000b98       __imp_?arg@QString@@QBE?AV1@HHH@Z 10020b98     qt-mt323:qt-mt323.dll
 0002:00000b9c       __imp_?arg@QString@@QBE?AV1@ABV1@H@Z 10020b9c     qt-mt323:qt-mt323.dll
 0002:00000ba0       __imp_?toInt@QString@@QBEHPA_NH@Z 10020ba0     qt-mt323:qt-mt323.dll
 0002:00000ba4       __imp_?append@QGList@@IAEXPAX@Z 10020ba4     qt-mt323:qt-mt323.dll
 0002:00000ba8       __imp_?rect@QWidget@@QBE?AVQRect@@XZ 10020ba8     qt-mt323:qt-mt323.dll
 0002:00000bac       __imp_??0QKeySequence@@QAE@H@Z 10020bac     qt-mt323:qt-mt323.dll
 0002:00000bb0       __imp_??0QIconSet@@QAE@ABVQPixmap@@W4Size@0@@Z 10020bb0     qt-mt323:qt-mt323.dll
 0002:00000bb4       __imp_??1QIconSet@@UAE@XZ  10020bb4     qt-mt323:qt-mt323.dll
 0002:00000bb8       __imp_??0QAction@@QAE@ABVQString@@ABVQIconSet@@0VQKeySequence@@PAVQObject@@PBD_N@Z 10020bb8     qt-mt323:qt-mt323.dll
 0002:00000bbc       __imp_??1QAction@@UAE@XZ   10020bbc     qt-mt323:qt-mt323.dll
 0002:00000bc0       __imp_??0QDockWindow@@QAE@PAVQWidget@@PBDI@Z 10020bc0     qt-mt323:qt-mt323.dll
 0002:00000bc4       __imp_??1QDockWindow@@UAE@XZ 10020bc4     qt-mt323:qt-mt323.dll
 0002:00000bc8       __imp_??0QToolBar@@QAE@PAVQMainWindow@@PBD@Z 10020bc8     qt-mt323:qt-mt323.dll
 0002:00000bcc       __imp_??1QToolBar@@UAE@XZ  10020bcc     qt-mt323:qt-mt323.dll
 0002:00000bd0       __imp_??9QDateTime@@QBE_NABV0@@Z 10020bd0     qt-mt323:qt-mt323.dll
 0002:00000bd4       __imp_?reconnect@QGuardedPtrPrivate@@QAEXPAVQObject@@@Z 10020bd4     qt-mt323:qt-mt323.dll
 0002:00000bd8       __imp_?look_string@QGDict@@QAEPAXABVQString@@PAXH@Z 10020bd8     qt-mt323:qt-mt323.dll
 0002:00000bdc       __imp_??0QGDict@@IAE@IW4KeyType@0@_N1@Z 10020bdc     qt-mt323:qt-mt323.dll
 0002:00000be0       __imp_??1QGDict@@MAE@XZ    10020be0     qt-mt323:qt-mt323.dll
 0002:00000be4       __imp_?clear@QGDict@@MAEXXZ 10020be4     qt-mt323:qt-mt323.dll
 0002:00000be8       __imp_?activateItemAt@QPopupMenu@@UAEXH@Z 10020be8     qt-mt323:qt-mt323.dll
 0002:00000bec       __imp_?addTo@QAction@@UAE_NPAVQWidget@@@Z 10020bec     qt-mt323:qt-mt323.dll
 0002:00000bf0       __imp_?addedTo@QAction@@MAEXHPAVQPopupMenu@@@Z 10020bf0     qt-mt323:qt-mt323.dll
 0002:00000bf4       __imp_?addedTo@QAction@@MAEXPAVQWidget@@0@Z 10020bf4     qt-mt323:qt-mt323.dll
 0002:00000bf8       __imp_?className@QAction@@UBEPBDXZ 10020bf8     qt-mt323:qt-mt323.dll
 0002:00000bfc       __imp_?className@QDockWindow@@UBEPBDXZ 10020bfc     qt-mt323:qt-mt323.dll
 0002:00000c00       __imp_?className@QPopupMenu@@UBEPBDXZ 10020c00     qt-mt323:qt-mt323.dll
 0002:00000c04       __imp_?className@QToolBar@@UBEPBDXZ 10020c04     qt-mt323:qt-mt323.dll
 0002:00000c08       __imp_?clear@QToolBar@@UAEXXZ 10020c08     qt-mt323:qt-mt323.dll
 0002:00000c0c       __imp_?closeEvent@QPopupMenu@@MAEXPAVQCloseEvent@@@Z 10020c0c     qt-mt323:qt-mt323.dll
 0002:00000c10       __imp_?contextMenuEvent@QDockWindow@@MAEXPAVQContextMenuEvent@@@Z 10020c10     qt-mt323:qt-mt323.dll
 0002:00000c14       __imp_?customWhatsThis@QPopupMenu@@UBE_NXZ 10020c14     qt-mt323:qt-mt323.dll
 0002:00000c18       __imp_?dock@QDockWindow@@UAEXXZ 10020c18     qt-mt323:qt-mt323.dll
 0002:00000c1c       __imp_?drawContents@QDockWindow@@MAEXPAVQPainter@@@Z 10020c1c     qt-mt323:qt-mt323.dll
 0002:00000c20       __imp_?drawContents@QPopupMenu@@MAEXPAVQPainter@@@Z 10020c20     qt-mt323:qt-mt323.dll
 0002:00000c24       __imp_?drawFrame@QDockWindow@@MAEXPAVQPainter@@@Z 10020c24     qt-mt323:qt-mt323.dll
 0002:00000c28       __imp_?enabledChange@QPopupMenu@@MAEX_N@Z 10020c28     qt-mt323:qt-mt323.dll
 0002:00000c2c       __imp_?event@QDockWindow@@MAE_NPAVQEvent@@@Z 10020c2c     qt-mt323:qt-mt323.dll
 0002:00000c30       __imp_?event@QToolBar@@UAE_NPAVQEvent@@@Z 10020c30     qt-mt323:qt-mt323.dll
 0002:00000c34       __imp_?eventFilter@QDockWindow@@UAE_NPAVQObject@@PAVQEvent@@@Z 10020c34     qt-mt323:qt-mt323.dll
 0002:00000c38       __imp_?focusInEvent@QPopupMenu@@MAEXPAVQFocusEvent@@@Z 10020c38     qt-mt323:qt-mt323.dll
 0002:00000c3c       __imp_?focusNextPrevChild@QPopupMenu@@MAE_N_N@Z 10020c3c     qt-mt323:qt-mt323.dll
 0002:00000c40       __imp_?focusOutEvent@QPopupMenu@@MAEXPAVQFocusEvent@@@Z 10020c40     qt-mt323:qt-mt323.dll
 0002:00000c44       __imp_?frameChanged@QPopupMenu@@EAEXXZ 10020c44     qt-mt323:qt-mt323.dll
 0002:00000c48       __imp_?hide@QPopupMenu@@UAEXXZ 10020c48     qt-mt323:qt-mt323.dll
 0002:00000c4c       __imp_?hide@QToolBar@@UAEXXZ 10020c4c     qt-mt323:qt-mt323.dll
 0002:00000c50       __imp_?hideEvent@QDockWindow@@MAEXPAVQHideEvent@@@Z 10020c50     qt-mt323:qt-mt323.dll
 0002:00000c54       __imp_?keyPressEvent@QPopupMenu@@MAEXPAVQKeyEvent@@@Z 10020c54     qt-mt323:qt-mt323.dll
 0002:00000c58       __imp_?leaveEvent@QPopupMenu@@MAEXPAVQEvent@@@Z 10020c58     qt-mt323:qt-mt323.dll
 0002:00000c5c       __imp_?menuContentsChanged@QPopupMenu@@EAEXXZ 10020c5c     qt-mt323:qt-mt323.dll
 0002:00000c60       __imp_?menuDelPopup@QPopupMenu@@EAEXPAV1@@Z 10020c60     qt-mt323:qt-mt323.dll
 0002:00000c64       __imp_?menuInsPopup@QPopupMenu@@EAEXPAV1@@Z 10020c64     qt-mt323:qt-mt323.dll
 0002:00000c68       __imp_?menuStateChanged@QPopupMenu@@EAEXXZ 10020c68     qt-mt323:qt-mt323.dll
 0002:00000c6c       __imp_?metaObject@QAction@@UBEPAVQMetaObject@@XZ 10020c6c     qt-mt323:qt-mt323.dll
 0002:00000c70       __imp_?metaObject@QDockWindow@@UBEPAVQMetaObject@@XZ 10020c70     qt-mt323:qt-mt323.dll
 0002:00000c74       __imp_?metaObject@QPopupMenu@@UBEPAVQMetaObject@@XZ 10020c74     qt-mt323:qt-mt323.dll
 0002:00000c78       __imp_?metaObject@QToolBar@@UBEPAVQMetaObject@@XZ 10020c78     qt-mt323:qt-mt323.dll
 0002:00000c7c       __imp_?minimumSizeHint@QDockWindow@@UBE?AVQSize@@XZ 10020c7c     qt-mt323:qt-mt323.dll
 0002:00000c80       __imp_?minimumSizeHint@QToolBar@@UBE?AVQSize@@XZ 10020c80     qt-mt323:qt-mt323.dll
 0002:00000c84       __imp_?mouseMoveEvent@QPopupMenu@@MAEXPAVQMouseEvent@@@Z 10020c84     qt-mt323:qt-mt323.dll
 0002:00000c88       __imp_?mousePressEvent@QPopupMenu@@MAEXPAVQMouseEvent@@@Z 10020c88     qt-mt323:qt-mt323.dll
 0002:00000c8c       __imp_?mouseReleaseEvent@QPopupMenu@@MAEXPAVQMouseEvent@@@Z 10020c8c     qt-mt323:qt-mt323.dll
 0002:00000c90       __imp_?paintEvent@QPopupMenu@@MAEXPAVQPaintEvent@@@Z 10020c90     qt-mt323:qt-mt323.dll
 0002:00000c94       __imp_?qt_cast@QAction@@UAEPAXPBD@Z 10020c94     qt-mt323:qt-mt323.dll
 0002:00000c98       __imp_?qt_cast@QDockWindow@@UAEPAXPBD@Z 10020c98     qt-mt323:qt-mt323.dll
 0002:00000c9c       __imp_?qt_cast@QPopupMenu@@UAEPAXPBD@Z 10020c9c     qt-mt323:qt-mt323.dll
 0002:00000ca0       __imp_?qt_cast@QToolBar@@UAEPAXPBD@Z 10020ca0     qt-mt323:qt-mt323.dll
 0002:00000ca4       __imp_?qt_emit@QAction@@UAE_NHPAUQUObject@@@Z 10020ca4     qt-mt323:qt-mt323.dll
 0002:00000ca8       __imp_?qt_emit@QDockWindow@@UAE_NHPAUQUObject@@@Z 10020ca8     qt-mt323:qt-mt323.dll
 0002:00000cac       __imp_?qt_emit@QPopupMenu@@UAE_NHPAUQUObject@@@Z 10020cac     qt-mt323:qt-mt323.dll
 0002:00000cb0       __imp_?qt_emit@QToolBar@@UAE_NHPAUQUObject@@@Z 10020cb0     qt-mt323:qt-mt323.dll
 0002:00000cb4       __imp_?qt_invoke@QAction@@UAE_NHPAUQUObject@@@Z 10020cb4     qt-mt323:qt-mt323.dll
 0002:00000cb8       __imp_?qt_invoke@QDockWindow@@UAE_NHPAUQUObject@@@Z 10020cb8     qt-mt323:qt-mt323.dll
 0002:00000cbc       __imp_?qt_invoke@QPopupMenu@@UAE_NHPAUQUObject@@@Z 10020cbc     qt-mt323:qt-mt323.dll
 0002:00000cc0       __imp_?qt_invoke@QToolBar@@UAE_NHPAUQUObject@@@Z 10020cc0     qt-mt323:qt-mt323.dll
 0002:00000cc4       __imp_?qt_property@QAction@@UAE_NHHPAVQVariant@@@Z 10020cc4     qt-mt323:qt-mt323.dll
 0002:00000cc8       __imp_?qt_property@QDockWindow@@UAE_NHHPAVQVariant@@@Z 10020cc8     qt-mt323:qt-mt323.dll
 0002:00000ccc       __imp_?qt_property@QPopupMenu@@UAE_NHHPAVQVariant@@@Z 10020ccc     qt-mt323:qt-mt323.dll
 0002:00000cd0       __imp_?qt_property@QToolBar@@UAE_NHHPAVQVariant@@@Z 10020cd0     qt-mt323:qt-mt323.dll
 0002:00000cd4       __imp_?read@QGDict@@MAEAAVQDataStream@@AAV2@AAPAX@Z 10020cd4     qt-mt323:qt-mt323.dll
 0002:00000cd8       __imp_?removeFrom@QAction@@UAE_NPAVQWidget@@@Z 10020cd8     qt-mt323:qt-mt323.dll
 0002:00000cdc       __imp_?resizeEvent@QDockWindow@@MAEXPAVQResizeEvent@@@Z 10020cdc     qt-mt323:qt-mt323.dll
 0002:00000ce0       __imp_?resizeEvent@QToolBar@@MAEXPAVQResizeEvent@@@Z 10020ce0     qt-mt323:qt-mt323.dll
 0002:00000ce4       __imp_?setAccel@QAction@@UAEXABVQKeySequence@@@Z 10020ce4     qt-mt323:qt-mt323.dll
 0002:00000ce8       __imp_?setActiveItem@QPopupMenu@@UAEXH@Z 10020ce8     qt-mt323:qt-mt323.dll
 0002:00000cec       __imp_?setCaption@QDockWindow@@UAEXABVQString@@@Z 10020cec     qt-mt323:qt-mt323.dll
 0002:00000cf0       __imp_?setCheckable@QPopupMenu@@UAEX_N@Z 10020cf0     qt-mt323:qt-mt323.dll
 0002:00000cf4       __imp_?setCloseMode@QDockWindow@@UAEXH@Z 10020cf4     qt-mt323:qt-mt323.dll
 0002:00000cf8       __imp_?setEnabled@QAction@@UAEX_N@Z 10020cf8     qt-mt323:qt-mt323.dll
 0002:00000cfc       __imp_?setFirstItemActive@QPopupMenu@@EAEXXZ 10020cfc     qt-mt323:qt-mt323.dll
 0002:00000d00       __imp_?setFixedExtentHeight@QDockWindow@@UAEXH@Z 10020d00     qt-mt323:qt-mt323.dll
 0002:00000d04       __imp_?setFixedExtentWidth@QDockWindow@@UAEXH@Z 10020d04     qt-mt323:qt-mt323.dll
 0002:00000d08       __imp_?setFont@QPopupMenu@@UAEXABVQFont@@@Z 10020d08     qt-mt323:qt-mt323.dll
 0002:00000d0c       __imp_?setHorizontallyStretchable@QDockWindow@@UAEX_N@Z 10020d0c     qt-mt323:qt-mt323.dll
 0002:00000d10       __imp_?setIconSet@QAction@@UAEXABVQIconSet@@@Z 10020d10     qt-mt323:qt-mt323.dll
 0002:00000d14       __imp_?setId@QMenuData@@UAEXHH@Z 10020d14     qt-mt323:qt-mt323.dll
 0002:00000d18       __imp_?setLabel@QToolBar@@UAEXABVQString@@@Z 10020d18     qt-mt323:qt-mt323.dll
 0002:00000d1c       __imp_?setMenuText@QAction@@UAEXABVQString@@@Z 10020d1c     qt-mt323:qt-mt323.dll
 0002:00000d20       __imp_?setMinimumSize@QToolBar@@UAEXHH@Z 10020d20     qt-mt323:qt-mt323.dll
 0002:00000d24       __imp_?setMovingEnabled@QDockWindow@@UAEX_N@Z 10020d24     qt-mt323:qt-mt323.dll
 0002:00000d28       __imp_?setNewLine@QDockWindow@@UAEX_N@Z 10020d28     qt-mt323:qt-mt323.dll
 0002:00000d2c       __imp_?setOffset@QDockWindow@@UAEXH@Z 10020d2c     qt-mt323:qt-mt323.dll
 0002:00000d30       __imp_?setOn@QAction@@UAEX_N@Z 10020d30     qt-mt323:qt-mt323.dll
 0002:00000d34       __imp_?setOpaqueMoving@QDockWindow@@UAEX_N@Z 10020d34     qt-mt323:qt-mt323.dll
 0002:00000d38       __imp_?setOrientation@QDockWindow@@UAEXW4Orientation@Qt@@@Z 10020d38     qt-mt323:qt-mt323.dll
 0002:00000d3c       __imp_?setOrientation@QToolBar@@UAEXW4Orientation@Qt@@@Z 10020d3c     qt-mt323:qt-mt323.dll
 0002:00000d40       __imp_?setResizeEnabled@QDockWindow@@UAEX_N@Z 10020d40     qt-mt323:qt-mt323.dll
 0002:00000d44       __imp_?setStatusTip@QAction@@UAEXABVQString@@@Z 10020d44     qt-mt323:qt-mt323.dll
 0002:00000d48       __imp_?setStretchableWidget@QToolBar@@UAEXPAVQWidget@@@Z 10020d48     qt-mt323:qt-mt323.dll
 0002:00000d4c       __imp_?setText@QAction@@UAEXABVQString@@@Z 10020d4c     qt-mt323:qt-mt323.dll
 0002:00000d50       __imp_?setToggleAction@QAction@@UAEX_N@Z 10020d50     qt-mt323:qt-mt323.dll
 0002:00000d54       __imp_?setToolTip@QAction@@UAEXABVQString@@@Z 10020d54     qt-mt323:qt-mt323.dll
 0002:00000d58       __imp_?setVerticallyStretchable@QDockWindow@@UAEX_N@Z 10020d58     qt-mt323:qt-mt323.dll
 0002:00000d5c       __imp_?setWhatsThis@QAction@@UAEXABVQString@@@Z 10020d5c     qt-mt323:qt-mt323.dll
 0002:00000d60       __imp_?setWidget@QDockWindow@@UAEXPAVQWidget@@@Z 10020d60     qt-mt323:qt-mt323.dll
 0002:00000d64       __imp_?show@QPopupMenu@@UAEXXZ 10020d64     qt-mt323:qt-mt323.dll
 0002:00000d68       __imp_?show@QToolBar@@UAEXXZ 10020d68     qt-mt323:qt-mt323.dll
 0002:00000d6c       __imp_?showEvent@QDockWindow@@MAEXPAVQShowEvent@@@Z 10020d6c     qt-mt323:qt-mt323.dll
 0002:00000d70       __imp_?sizeHint@QDockWindow@@UBE?AVQSize@@XZ 10020d70     qt-mt323:qt-mt323.dll
 0002:00000d74       __imp_?sizeHint@QPopupMenu@@UBE?AVQSize@@XZ 10020d74     qt-mt323:qt-mt323.dll
 0002:00000d78       __imp_?styleChange@QPopupMenu@@MAEXAAVQStyle@@@Z 10020d78     qt-mt323:qt-mt323.dll
 0002:00000d7c       __imp_?styleChange@QToolBar@@MAEXAAVQStyle@@@Z 10020d7c     qt-mt323:qt-mt323.dll
 0002:00000d80       __imp_?timerEvent@QPopupMenu@@MAEXPAVQTimerEvent@@@Z 10020d80     qt-mt323:qt-mt323.dll
 0002:00000d84       __imp_?undock@QDockWindow@@UAEXPAVQWidget@@@Z 10020d84     qt-mt323:qt-mt323.dll
 0002:00000d88       __imp_?undock@QDockWindow@@UAEXXZ 10020d88     qt-mt323:qt-mt323.dll
 0002:00000d8c       __imp_?updateItem@QPopupMenu@@UAEXH@Z 10020d8c     qt-mt323:qt-mt323.dll
 0002:00000d90       __imp_?write@QGDict@@MBEAAVQDataStream@@AAV2@PAX@Z 10020d90     qt-mt323:qt-mt323.dll
 0002:00000d94       __imp_?lower@QString@@QBE?AV1@XZ 10020d94     qt-mt323:qt-mt323.dll
 0002:00000d98       __imp_??0QTextStream@@QAE@PAVQIODevice@@@Z 10020d98     qt-mt323:qt-mt323.dll
 0002:00000d9c       __imp_??1QTextStream@@UAE@XZ 10020d9c     qt-mt323:qt-mt323.dll
 0002:00000da0       __imp_??6QTextStream@@QAEAAV0@ABVQString@@@Z 10020da0     qt-mt323:qt-mt323.dll
 0002:00000da4       __imp_?blockSignals@QObject@@QAEX_N@Z 10020da4     qt-mt323:qt-mt323.dll
 0002:00000da8       __imp_?updateContents@QScrollView@@QAEXXZ 10020da8     qt-mt323:qt-mt323.dll
 0002:00000dac       __imp_??0QTableSelection@@QAE@HHHH@Z 10020dac     qt-mt323:qt-mt323.dll
 0002:00000db0       __imp_??1QTableItem@@UAE@XZ 10020db0     qt-mt323:qt-mt323.dll
 0002:00000db4       __imp_??0QCheckTableItem@@QAE@PAVQTable@@ABVQString@@@Z 10020db4     qt-mt323:qt-mt323.dll
 0002:00000db8       __imp_?isChecked@QCheckTableItem@@QBE_NXZ 10020db8     qt-mt323:qt-mt323.dll
 0002:00000dbc       __imp_?clearSelection@QTable@@QAEX_N@Z 10020dbc     qt-mt323:qt-mt323.dll
 0002:00000dc0       __imp_?currentText@QComboBox@@QBE?AVQString@@XZ 10020dc0     qt-mt323:qt-mt323.dll
 0002:00000dc4       __imp_?setChecked@QCheckBox@@QAEX_N@Z 10020dc4     qt-mt323:qt-mt323.dll
 0002:00000dc8       __imp_?setIconSet@QPushButton@@QAEXABVQIconSet@@@Z 10020dc8     qt-mt323:qt-mt323.dll
 0002:00000dcc       __imp_?replaceChild@QDomNode@@UAE?AV1@ABV1@0@Z 10020dcc     qt-mt323:qt-mt323.dll
 0002:00000dd0       __imp_?appendChild@QDomNode@@UAE?AV1@ABV1@@Z 10020dd0     qt-mt323:qt-mt323.dll
 0002:00000dd4       __imp_?createElement@QDomDocument@@QAE?AVQDomElement@@ABVQString@@@Z 10020dd4     qt-mt323:qt-mt323.dll
 0002:00000dd8       __imp_?setContent@QDomDocument@@QAE_NPAVQIODevice@@PAVQString@@PAH2@Z 10020dd8     qt-mt323:qt-mt323.dll
 0002:00000ddc       __imp_?toString@QDomDocument@@QBE?AVQString@@XZ 10020ddc     qt-mt323:qt-mt323.dll
 0002:00000de0       __imp_?setAttribute@QDomElement@@QAEXABVQString@@0@Z 10020de0     qt-mt323:qt-mt323.dll
 0002:00000de4       __imp_?close@QFile@@UAEXXZ 10020de4     qt-mt323:qt-mt323.dll
 0002:00000de8       __imp_?alignment@QTableItem@@UBEHXZ 10020de8     qt-mt323:qt-mt323.dll
 0002:00000dec       __imp_?createEditor@QCheckTableItem@@UBEPAVQWidget@@XZ 10020dec     qt-mt323:qt-mt323.dll
 0002:00000df0       __imp_?key@QTableItem@@UBE?AVQString@@XZ 10020df0     qt-mt323:qt-mt323.dll
 0002:00000df4       __imp_?paint@QCheckTableItem@@UAEXPAVQPainter@@ABVQColorGroup@@ABVQRect@@_N@Z 10020df4     qt-mt323:qt-mt323.dll
 0002:00000df8       __imp_?pixmap@QTableItem@@UBE?AVQPixmap@@XZ 10020df8     qt-mt323:qt-mt323.dll
 0002:00000dfc       __imp_?rtti@QCheckTableItem@@UBEHXZ 10020dfc     qt-mt323:qt-mt323.dll
 0002:00000e00       __imp_?setChecked@QCheckTableItem@@UAEX_N@Z 10020e00     qt-mt323:qt-mt323.dll
 0002:00000e04       __imp_?setCol@QTableItem@@UAEXH@Z 10020e04     qt-mt323:qt-mt323.dll
 0002:00000e08       __imp_?setContentFromEditor@QCheckTableItem@@UAEXPAVQWidget@@@Z 10020e08     qt-mt323:qt-mt323.dll
 0002:00000e0c       __imp_?setEnabled@QTableItem@@UAEX_N@Z 10020e0c     qt-mt323:qt-mt323.dll
 0002:00000e10       __imp_?setPixmap@QTableItem@@UAEXABVQPixmap@@@Z 10020e10     qt-mt323:qt-mt323.dll
 0002:00000e14       __imp_?setReplaceable@QTableItem@@UAEX_N@Z 10020e14     qt-mt323:qt-mt323.dll
 0002:00000e18       __imp_?setRow@QTableItem@@UAEXH@Z 10020e18     qt-mt323:qt-mt323.dll
 0002:00000e1c       __imp_?setSpan@QTableItem@@UAEXHH@Z 10020e1c     qt-mt323:qt-mt323.dll
 0002:00000e20       __imp_?setText@QCheckTableItem@@UAEXABVQString@@@Z 10020e20     qt-mt323:qt-mt323.dll
 0002:00000e24       __imp_?setWordWrap@QTableItem@@UAEX_N@Z 10020e24     qt-mt323:qt-mt323.dll
 0002:00000e28       __imp_?sizeHint@QCheckTableItem@@UBE?AVQSize@@XZ 10020e28     qt-mt323:qt-mt323.dll
 0002:00000e2c       __imp_?text@QTableItem@@UBE?AVQString@@XZ 10020e2c     qt-mt323:qt-mt323.dll
 0002:00000e30       __imp_??4QString@@QAEAAV0@PBD@Z 10020e30     qt-mt323:qt-mt323.dll
 0002:00000e34       __imp_?sprintf@QString@@QAAAAV1@PBDZZ 10020e34     qt-mt323:qt-mt323.dll
 0002:00000e38       __imp_?replace@QString@@QAEAAV1@ABV1@0@Z 10020e38     qt-mt323:qt-mt323.dll
 0002:00000e3c       __imp_??6QTextStream@@QAEAAV0@PBD@Z 10020e3c     qt-mt323:qt-mt323.dll
 0002:00000e40       __imp_??0QPixmap@@QAE@XZ   10020e40     qt-mt323:qt-mt323.dll
 0002:00000e44       __imp_?text@QLineEdit@@QBE?AVQString@@XZ 10020e44     qt-mt323:qt-mt323.dll
 0002:00000e48       __imp_?insertItem@QListBox@@QAEXABVQString@@H@Z 10020e48     qt-mt323:qt-mt323.dll
 0002:00000e4c       __imp_?clear@QListBox@@QAEXXZ 10020e4c     qt-mt323:qt-mt323.dll
 0002:00000e50       __imp_?readLine@QFile@@UAEJPADK@Z 10020e50     qt-mt323:qt-mt323.dll
 0002:00000e54       __imp_?insertSeparator@QMenuData@@QAEHH@Z 10020e54     qt-mt323:qt-mt323.dll
 0002:00000e58       __imp_?horizontalHeader@QTable@@QBEPAVQHeader@@XZ 10020e58     qt-mt323:qt-mt323.dll
 0002:00000e5c       __imp_??9@YA_NABVQString@@PBD@Z 10020e5c     qt-mt323:qt-mt323.dll
 0002:00000e60       __imp_??0?$QMap@VQString@@H@@QAE@XZ 10020e60     qt-mt323:qt-mt323.dll
 0002:00000e64       __imp_??1?$QMap@VQString@@H@@QAE@XZ 10020e64     qt-mt323:qt-mt323.dll
 0002:00000e68       __imp_?begin@?$QMap@VQString@@H@@QAE?AV?$QMapIterator@VQString@@H@@XZ 10020e68     qt-mt323:qt-mt323.dll
 0002:00000e6c       __imp_?end@?$QMap@VQString@@H@@QAE?AV?$QMapIterator@VQString@@H@@XZ 10020e6c     qt-mt323:qt-mt323.dll
 0002:00000e70       __imp_??A?$QMap@VQString@@H@@QAEAAHABVQString@@@Z 10020e70     qt-mt323:qt-mt323.dll
 0002:00000e74       __imp_?clear@?$QMap@VQString@@H@@QAEXXZ 10020e74     qt-mt323:qt-mt323.dll
 0002:00000e78       __imp_?rightJustify@QString@@QBE?AV1@IVQChar@@_N@Z 10020e78     qt-mt323:qt-mt323.dll
 0002:00000e7c       __imp_?exec@QDialog@@QAEHXZ 10020e7c     qt-mt323:qt-mt323.dll
 0002:00000e80       __imp_??YQString@@QAEAAV0@PBD@Z 10020e80     qt-mt323:qt-mt323.dll
 0002:00000e84       __imp_??4QStringList@@QAEAAV0@ABV0@@Z 10020e84     qt-mt323:qt-mt323.dll
 0002:00000e88       __imp_?accept@QDialog@@MAEXXZ 10020e88     qt-mt323:qt-mt323.dll
 0002:00000e8c       __imp_?insertItem@QComboBox@@QAEXABVQString@@H@Z 10020e8c     qt-mt323:qt-mt323.dll
 0002:00000e90       __imp_?closeEvent@QDialog@@MAEXPAVQCloseEvent@@@Z 10020e90     qt-mt323:qt-mt323.dll
 0002:00000e94       __imp_?contextMenuEvent@QDialog@@MAEXPAVQContextMenuEvent@@@Z 10020e94     qt-mt323:qt-mt323.dll
 0002:00000e98       __imp_?done@QDialog@@MAEXH@Z 10020e98     qt-mt323:qt-mt323.dll
 0002:00000e9c       __imp_?eventFilter@QDialog@@MAE_NPAVQObject@@PAVQEvent@@@Z 10020e9c     qt-mt323:qt-mt323.dll
 0002:00000ea0       __imp_?hide@QDialog@@UAEXXZ 10020ea0     qt-mt323:qt-mt323.dll
 0002:00000ea4       __imp_?keyPressEvent@QDialog@@MAEXPAVQKeyEvent@@@Z 10020ea4     qt-mt323:qt-mt323.dll
 0002:00000ea8       __imp_?minimumSizeHint@QDialog@@UBE?AVQSize@@XZ 10020ea8     qt-mt323:qt-mt323.dll
 0002:00000eac       __imp_?move@QDialog@@UAEXHH@Z 10020eac     qt-mt323:qt-mt323.dll
 0002:00000eb0       __imp_?reject@QDialog@@MAEXXZ 10020eb0     qt-mt323:qt-mt323.dll
 0002:00000eb4       __imp_?resize@QDialog@@UAEXHH@Z 10020eb4     qt-mt323:qt-mt323.dll
 0002:00000eb8       __imp_?resizeEvent@QDialog@@MAEXPAVQResizeEvent@@@Z 10020eb8     qt-mt323:qt-mt323.dll
 0002:00000ebc       __imp_?setGeometry@QDialog@@UAEXABVQRect@@@Z 10020ebc     qt-mt323:qt-mt323.dll
 0002:00000ec0       __imp_?setGeometry@QDialog@@UAEXHHHH@Z 10020ec0     qt-mt323:qt-mt323.dll
 0002:00000ec4       __imp_?show@QDialog@@UAEXXZ 10020ec4     qt-mt323:qt-mt323.dll
 0002:00000ec8       __imp_?sizeHint@QDialog@@UBE?AVQSize@@XZ 10020ec8     qt-mt323:qt-mt323.dll
 0002:00000ecc       __imp_?inherits@QObject@@QBE_NPBD@Z 10020ecc     qt-mt323:qt-mt323.dll
 0002:00000ed0       __imp_?viewport@QScrollView@@QBEPAVQWidget@@XZ 10020ed0     qt-mt323:qt-mt323.dll
 0002:00000ed4       __imp_??0QTableItem@@QAE@PAVQTable@@W4EditType@0@ABVQString@@@Z 10020ed4     qt-mt323:qt-mt323.dll
 0002:00000ed8       __imp_?setContentFromEditor@QTableItem@@UAEXPAVQWidget@@@Z 10020ed8     qt-mt323:qt-mt323.dll
 0002:00000edc       __imp_??0QComboBox@@QAE@PAVQWidget@@PBD@Z 10020edc     qt-mt323:qt-mt323.dll
 0002:00000ee0       __imp_??1QComboBox@@UAE@XZ 10020ee0     qt-mt323:qt-mt323.dll
 0002:00000ee4       __imp_?className@QComboBox@@UBEPBDXZ 10020ee4     qt-mt323:qt-mt323.dll
 0002:00000ee8       __imp_?eventFilter@QComboBox@@UAE_NPAVQObject@@PAVQEvent@@@Z 10020ee8     qt-mt323:qt-mt323.dll
 0002:00000eec       __imp_?focusInEvent@QComboBox@@MAEXPAVQFocusEvent@@@Z 10020eec     qt-mt323:qt-mt323.dll
 0002:00000ef0       __imp_?focusOutEvent@QComboBox@@MAEXPAVQFocusEvent@@@Z 10020ef0     qt-mt323:qt-mt323.dll
 0002:00000ef4       __imp_?keyPressEvent@QComboBox@@MAEXPAVQKeyEvent@@@Z 10020ef4     qt-mt323:qt-mt323.dll
 0002:00000ef8       __imp_?metaObject@QComboBox@@UBEPAVQMetaObject@@XZ 10020ef8     qt-mt323:qt-mt323.dll
 0002:00000efc       __imp_?mouseDoubleClickEvent@QComboBox@@MAEXPAVQMouseEvent@@@Z 10020efc     qt-mt323:qt-mt323.dll
 0002:00000f00       __imp_?mouseMoveEvent@QComboBox@@MAEXPAVQMouseEvent@@@Z 10020f00     qt-mt323:qt-mt323.dll
 0002:00000f04       __imp_?mousePressEvent@QComboBox@@MAEXPAVQMouseEvent@@@Z 10020f04     qt-mt323:qt-mt323.dll
 0002:00000f08       __imp_?mouseReleaseEvent@QComboBox@@MAEXPAVQMouseEvent@@@Z 10020f08     qt-mt323:qt-mt323.dll
 0002:00000f0c       __imp_?paint@QTableItem@@UAEXPAVQPainter@@ABVQColorGroup@@ABVQRect@@_N@Z 10020f0c     qt-mt323:qt-mt323.dll
 0002:00000f10       __imp_?paintEvent@QComboBox@@MAEXPAVQPaintEvent@@@Z 10020f10     qt-mt323:qt-mt323.dll
 0002:00000f14       __imp_?popup@QComboBox@@UAEXXZ 10020f14     qt-mt323:qt-mt323.dll
 0002:00000f18       __imp_?qt_cast@QComboBox@@UAEPAXPBD@Z 10020f18     qt-mt323:qt-mt323.dll
 0002:00000f1c       __imp_?qt_emit@QComboBox@@UAE_NHPAUQUObject@@@Z 10020f1c     qt-mt323:qt-mt323.dll
 0002:00000f20       __imp_?qt_invoke@QComboBox@@UAE_NHPAUQUObject@@@Z 10020f20     qt-mt323:qt-mt323.dll
 0002:00000f24       __imp_?qt_property@QComboBox@@UAE_NHHPAVQVariant@@@Z 10020f24     qt-mt323:qt-mt323.dll
 0002:00000f28       __imp_?resizeEvent@QComboBox@@MAEXPAVQResizeEvent@@@Z 10020f28     qt-mt323:qt-mt323.dll
 0002:00000f2c       __imp_?rtti@QTableItem@@UBEHXZ 10020f2c     qt-mt323:qt-mt323.dll
 0002:00000f30       __imp_?setAutoCompletion@QComboBox@@UAEX_N@Z 10020f30     qt-mt323:qt-mt323.dll
 0002:00000f34       __imp_?setAutoResize@QComboBox@@UAEX_N@Z 10020f34     qt-mt323:qt-mt323.dll
 0002:00000f38       __imp_?setCurrentItem@QComboBox@@UAEXH@Z 10020f38     qt-mt323:qt-mt323.dll
 0002:00000f3c       __imp_?setCurrentText@QComboBox@@UAEXABVQString@@@Z 10020f3c     qt-mt323:qt-mt323.dll
 0002:00000f40       __imp_?setEditText@QComboBox@@UAEXABVQString@@@Z 10020f40     qt-mt323:qt-mt323.dll
 0002:00000f44       __imp_?setEnabled@QComboBox@@UAEX_N@Z 10020f44     qt-mt323:qt-mt323.dll
 0002:00000f48       __imp_?setFont@QComboBox@@UAEXABVQFont@@@Z 10020f48     qt-mt323:qt-mt323.dll
 0002:00000f4c       __imp_?setInsertionPolicy@QComboBox@@UAEXW4Policy@1@@Z 10020f4c     qt-mt323:qt-mt323.dll
 0002:00000f50       __imp_?setLineEdit@QComboBox@@UAEXPAVQLineEdit@@@Z 10020f50     qt-mt323:qt-mt323.dll
 0002:00000f54       __imp_?setListBox@QComboBox@@UAEXPAVQListBox@@@Z 10020f54     qt-mt323:qt-mt323.dll
 0002:00000f58       __imp_?setMaxCount@QComboBox@@UAEXH@Z 10020f58     qt-mt323:qt-mt323.dll
 0002:00000f5c       __imp_?setPalette@QComboBox@@UAEXABVQPalette@@@Z 10020f5c     qt-mt323:qt-mt323.dll
 0002:00000f60       __imp_?setSizeLimit@QComboBox@@UAEXH@Z 10020f60     qt-mt323:qt-mt323.dll
 0002:00000f64       __imp_?setText@QTableItem@@UAEXABVQString@@@Z 10020f64     qt-mt323:qt-mt323.dll
 0002:00000f68       __imp_?setValidator@QComboBox@@UAEXPBVQValidator@@@Z 10020f68     qt-mt323:qt-mt323.dll
 0002:00000f6c       __imp_?sizeHint@QComboBox@@UBE?AVQSize@@XZ 10020f6c     qt-mt323:qt-mt323.dll
 0002:00000f70       __imp_?sizeHint@QTableItem@@UBE?AVQSize@@XZ 10020f70     qt-mt323:qt-mt323.dll
 0002:00000f74       __imp_?styleChange@QComboBox@@MAEXAAVQStyle@@@Z 10020f74     qt-mt323:qt-mt323.dll
 0002:00000f78       __imp_?updateMask@QComboBox@@MAEXXZ 10020f78     qt-mt323:qt-mt323.dll
 0002:00000f7c       __imp_?wheelEvent@QComboBox@@MAEXPAVQWheelEvent@@@Z 10020f7c     qt-mt323:qt-mt323.dll
 0002:00000f80       __imp_??YQString@@QAEAAV0@ABV0@@Z 10020f80     qt-mt323:qt-mt323.dll
 0002:00000f84       __imp_?year@QDate@@QBEHXZ  10020f84     qt-mt323:qt-mt323.dll
 0002:00000f88       __imp_?month@QDate@@QBEHXZ 10020f88     qt-mt323:qt-mt323.dll
 0002:00000f8c       __imp_?day@QDate@@QBEHXZ   10020f8c     qt-mt323:qt-mt323.dll
 0002:00000f90       __imp_?hour@QTime@@QBEHXZ  10020f90     qt-mt323:qt-mt323.dll
 0002:00000f94       __imp_?minute@QTime@@QBEHXZ 10020f94     qt-mt323:qt-mt323.dll
 0002:00000f98       __imp_?second@QTime@@QBEHXZ 10020f98     qt-mt323:qt-mt323.dll
 0002:00000f9c       __imp_?dirPath@QFileInfo@@QBE?AVQString@@_N@Z 10020f9c     qt-mt323:qt-mt323.dll
 0002:00000fa0       __imp_?convertToAbs@QFileInfo@@QAE_NXZ 10020fa0     qt-mt323:qt-mt323.dll
 0002:00000fa4       __imp_??0QDir@@QAE@XZ      10020fa4     qt-mt323:qt-mt323.dll
 0002:00000fa8       __imp_??1QDir@@UAE@XZ      10020fa8     qt-mt323:qt-mt323.dll
 0002:00000fac       __imp_?mkdir@QDir@@UBE_NABVQString@@_N@Z 10020fac     qt-mt323:qt-mt323.dll
 0002:00000fb0       __imp_?setContent@QDomDocument@@QAE_NPAVQIODevice@@_NPAVQString@@PAH3@Z 10020fb0     qt-mt323:qt-mt323.dll
 0002:00000fb4       __imp_?selectedItem@QListView@@QBEPAVQListViewItem@@XZ 10020fb4     qt-mt323:qt-mt323.dll
 0002:00000fb8       __imp_?updateContents@QListView@@IAEXXZ 10020fb8     qt-mt323:qt-mt323.dll
 0002:00000fbc       __imp_??1QFont@@QAE@XZ     10020fbc     qt-mt323:qt-mt323.dll
 0002:00000fc0       __imp_?setWeight@QFont@@QAEXH@Z 10020fc0     qt-mt323:qt-mt323.dll
 0002:00000fc4       __imp_?font@QWidget@@QBE?AVQFont@@XZ 10020fc4     qt-mt323:qt-mt323.dll
 0002:00000fc8       __imp_??1QButton@@UAE@XZ   10020fc8     qt-mt323:qt-mt323.dll
 0002:00000fcc       __imp_??0QComboBox@@QAE@_NPAVQWidget@@PBD@Z 10020fcc     qt-mt323:qt-mt323.dll
 0002:00000fd0       __imp_?setEditable@QComboBox@@QAEX_N@Z 10020fd0     qt-mt323:qt-mt323.dll
 0002:00000fd4       __imp_?clear@QComboBox@@QAEXXZ 10020fd4     qt-mt323:qt-mt323.dll
 0002:00000fd8       __imp_??0QCheckBox@@QAE@PAVQWidget@@PBD@Z 10020fd8     qt-mt323:qt-mt323.dll
 0002:00000fdc       __imp_?className@QCheckBox@@UBEPBDXZ 10020fdc     qt-mt323:qt-mt323.dll
 0002:00000fe0       __imp_?drawButton@QCheckBox@@MAEXPAVQPainter@@@Z 10020fe0     qt-mt323:qt-mt323.dll
 0002:00000fe4       __imp_?drawButtonLabel@QCheckBox@@MAEXPAVQPainter@@@Z 10020fe4     qt-mt323:qt-mt323.dll
 0002:00000fe8       __imp_?focusInEvent@QButton@@MAEXPAVQFocusEvent@@@Z 10020fe8     qt-mt323:qt-mt323.dll
 0002:00000fec       __imp_?focusOutEvent@QButton@@MAEXPAVQFocusEvent@@@Z 10020fec     qt-mt323:qt-mt323.dll
 0002:00000ff0       __imp_?hitButton@QCheckBox@@MBE_NABVQPoint@@@Z 10020ff0     qt-mt323:qt-mt323.dll
 0002:00000ff4       __imp_?metaObject@QCheckBox@@UBEPAVQMetaObject@@XZ 10020ff4     qt-mt323:qt-mt323.dll
 0002:00000ff8       __imp_?qt_cast@QCheckBox@@UAEPAXPBD@Z 10020ff8     qt-mt323:qt-mt323.dll
 0002:00000ffc       __imp_?qt_emit@QCheckBox@@UAE_NHPAUQUObject@@@Z 10020ffc     qt-mt323:qt-mt323.dll
 0002:00001000       __imp_?qt_invoke@QCheckBox@@UAE_NHPAUQUObject@@@Z 10021000     qt-mt323:qt-mt323.dll
 0002:00001004       __imp_?qt_property@QCheckBox@@UAE_NHHPAVQVariant@@@Z 10021004     qt-mt323:qt-mt323.dll
 0002:00001008       __imp_?resizeEvent@QCheckBox@@MAEXPAVQResizeEvent@@@Z 10021008     qt-mt323:qt-mt323.dll
 0002:0000100c       __imp_?sizeHint@QCheckBox@@UBE?AVQSize@@XZ 1002100c     qt-mt323:qt-mt323.dll
 0002:00001010       __imp_?updateMask@QCheckBox@@MAEXXZ 10021010     qt-mt323:qt-mt323.dll
 0002:00001014       __imp_?qstrcmp@@YAHPBD0@Z  10021014     qt-mt323:qt-mt323.dll
 0002:00001018       __imp_?fromLatin1@QString@@SA?AV1@PBDH@Z 10021018     qt-mt323:qt-mt323.dll
 0002:0000101c       __imp_?fromUtf8@QString@@SA?AV1@PBDH@Z 1002101c     qt-mt323:qt-mt323.dll
 0002:00001020       __imp_?staticMetaObject@QWidget@@SAPAVQMetaObject@@XZ 10021020     qt-mt323:qt-mt323.dll
 0002:00001024       __imp_?new_metaobject@QMetaObject@@SAPAV1@PBDPAV1@QBUQMetaData@@H2HQBVQMetaProperty@@HQBUQMetaEnum@@HQBUQClassInfo@@H@Z 10021024     qt-mt323:qt-mt323.dll
 0002:00001028       __imp_??0QMetaObjectCleanUp@@QAE@PBDP6APAVQMetaObject@@XZ@Z 10021028     qt-mt323:qt-mt323.dll
 0002:0000102c       __imp_??1QMetaObjectCleanUp@@QAE@XZ 1002102c     qt-mt323:qt-mt323.dll
 0002:00001030       __imp_?setMetaObject@QMetaObjectCleanUp@@QAEXAAPAVQMetaObject@@@Z 10021030     qt-mt323:qt-mt323.dll
 0002:00001034       __imp_?translate@QApplication@@QBE?AVQString@@PBD00W4Encoding@1@@Z 10021034     qt-mt323:qt-mt323.dll
 0002:00001038       __imp_?qApp@@3PAVQApplication@@A 10021038     qt-mt323:qt-mt323.dll
 0002:0000103c       __imp_?receivers@QObject@@IBEPAVQConnectionList@@H@Z 1002103c     qt-mt323:qt-mt323.dll
 0002:00001040       __imp_?activate_signal@QObject@@IAEXPAVQConnectionList@@PAUQUObject@@@Z 10021040     qt-mt323:qt-mt323.dll
 0002:00001044       __imp_?staticMetaObject@QListView@@SAPAVQMetaObject@@XZ 10021044     qt-mt323:qt-mt323.dll
 0002:00001048       __imp_??0QUObject@@QAE@XZ  10021048     qt-mt323:qt-mt323.dll
 0002:0000104c       __imp_??1QUObject@@QAE@XZ  1002104c     qt-mt323:qt-mt323.dll
 0002:00001050       __imp_?set@QUType_varptr@@QAEXPAUQUObject@@PBX@Z 10021050     qt-mt323:qt-mt323.dll
 0002:00001054       __imp_?static_QUType_varptr@@3UQUType_varptr@@A 10021054     qt-mt323:qt-mt323.dll
 0002:00001058       __imp_?set@QUType_QString@@QAEXPAUQUObject@@ABVQString@@@Z 10021058     qt-mt323:qt-mt323.dll
 0002:0000105c       __imp_?static_QUType_ptr@@3UQUType_ptr@@A 1002105c     qt-mt323:qt-mt323.dll
 0002:00001060       __imp_?static_QUType_QString@@3UQUType_QString@@A 10021060     qt-mt323:qt-mt323.dll
 0002:00001064       __imp_?static_QUType_int@@3UQUType_int@@A 10021064     qt-mt323:qt-mt323.dll
 0002:00001068       __imp_?set@QUType_ptr@@QAEXPAUQUObject@@PBX@Z 10021068     qt-mt323:qt-mt323.dll
 0002:0000106c       __imp_?qt_cast@QDialog@@UAEPAXPBD@Z 1002106c     qt-mt323:qt-mt323.dll
 0002:00001070       __imp_?qt_invoke@QDialog@@UAE_NHPAUQUObject@@@Z 10021070     qt-mt323:qt-mt323.dll
 0002:00001074       __imp_?qt_emit@QDialog@@UAE_NHPAUQUObject@@@Z 10021074     qt-mt323:qt-mt323.dll
 0002:00001078       __imp_?qt_property@QDialog@@UAE_NHHPAVQVariant@@@Z 10021078     qt-mt323:qt-mt323.dll
 0002:0000107c       __imp_?staticMetaObject@QDialog@@SAPAVQMetaObject@@XZ 1002107c     qt-mt323:qt-mt323.dll
 0002:00001080       __imp_??0QTabWidget@@QAE@PAVQWidget@@PBDI@Z 10021080     qt-mt323:qt-mt323.dll
 0002:00001084       __imp_??1QTabWidget@@UAE@XZ 10021084     qt-mt323:qt-mt323.dll
 0002:00001088       __imp_?changeTab@QTabWidget@@QAEXPAVQWidget@@ABVQString@@@Z 10021088     qt-mt323:qt-mt323.dll
 0002:0000108c       __imp_?addTab@QTabWidget@@UAEXPAVQWidget@@ABVQIconSet@@ABVQString@@@Z 1002108c     qt-mt323:qt-mt323.dll
 0002:00001090       __imp_?addTab@QTabWidget@@UAEXPAVQWidget@@ABVQString@@@Z 10021090     qt-mt323:qt-mt323.dll
 0002:00001094       __imp_?addTab@QTabWidget@@UAEXPAVQWidget@@PAVQTab@@@Z 10021094     qt-mt323:qt-mt323.dll
 0002:00001098       __imp_?className@QTabWidget@@UBEPBDXZ 10021098     qt-mt323:qt-mt323.dll
 0002:0000109c       __imp_?eventFilter@QTabWidget@@MAE_NPAVQObject@@PAVQEvent@@@Z 1002109c     qt-mt323:qt-mt323.dll
 0002:000010a0       __imp_?insertTab@QTabWidget@@UAEXPAVQWidget@@ABVQIconSet@@ABVQString@@H@Z 100210a0     qt-mt323:qt-mt323.dll
 0002:000010a4       __imp_?insertTab@QTabWidget@@UAEXPAVQWidget@@ABVQString@@H@Z 100210a4     qt-mt323:qt-mt323.dll
 0002:000010a8       __imp_?insertTab@QTabWidget@@UAEXPAVQWidget@@PAVQTab@@H@Z 100210a8     qt-mt323:qt-mt323.dll
 0002:000010ac       __imp_?metaObject@QTabWidget@@UBEPAVQMetaObject@@XZ 100210ac     qt-mt323:qt-mt323.dll
 0002:000010b0       __imp_?minimumSizeHint@QTabWidget@@UBE?AVQSize@@XZ 100210b0     qt-mt323:qt-mt323.dll
 0002:000010b4       __imp_?qt_cast@QTabWidget@@UAEPAXPBD@Z 100210b4     qt-mt323:qt-mt323.dll
 0002:000010b8       __imp_?qt_emit@QTabWidget@@UAE_NHPAUQUObject@@@Z 100210b8     qt-mt323:qt-mt323.dll
 0002:000010bc       __imp_?qt_invoke@QTabWidget@@UAE_NHPAUQUObject@@@Z 100210bc     qt-mt323:qt-mt323.dll
 0002:000010c0       __imp_?qt_property@QTabWidget@@UAE_NHHPAVQVariant@@@Z 100210c0     qt-mt323:qt-mt323.dll
 0002:000010c4       __imp_?removePage@QTabWidget@@UAEXPAVQWidget@@@Z 100210c4     qt-mt323:qt-mt323.dll
 0002:000010c8       __imp_?resizeEvent@QTabWidget@@MAEXPAVQResizeEvent@@@Z 100210c8     qt-mt323:qt-mt323.dll
 0002:000010cc       __imp_?showEvent@QTabWidget@@MAEXPAVQShowEvent@@@Z 100210cc     qt-mt323:qt-mt323.dll
 0002:000010d0       __imp_?showPage@QTabWidget@@UAEXPAVQWidget@@@Z 100210d0     qt-mt323:qt-mt323.dll
 0002:000010d4       __imp_?sizeHint@QTabWidget@@UBE?AVQSize@@XZ 100210d4     qt-mt323:qt-mt323.dll
 0002:000010d8       __imp_?styleChange@QTabWidget@@MAEXAAVQStyle@@@Z 100210d8     qt-mt323:qt-mt323.dll
 0002:000010dc       __imp_?updateMask@QTabWidget@@MAEXXZ 100210dc     qt-mt323:qt-mt323.dll
 0002:000010e0       __imp_?setMaximumSize@QWidget@@QAEXABVQSize@@@Z 100210e0     qt-mt323:qt-mt323.dll
 0002:000010e4       __imp_??0QDialog@@QAE@PAVQWidget@@PBD_NI@Z 100210e4     qt-mt323:qt-mt323.dll
 0002:000010e8       __imp_??1QDialog@@UAE@XZ   100210e8     qt-mt323:qt-mt323.dll
 0002:000010ec       __imp_?resize@QDialog@@QAEXABVQSize@@@Z 100210ec     qt-mt323:qt-mt323.dll
 0002:000010f0       __imp_?setSizeGripEnabled@QDialog@@QAEX_N@Z 100210f0     qt-mt323:qt-mt323.dll
 0002:000010f4       __imp_??0QButtonGroup@@QAE@PAVQWidget@@PBD@Z 100210f4     qt-mt323:qt-mt323.dll
 0002:000010f8       __imp_??1QButtonGroup@@UAE@XZ 100210f8     qt-mt323:qt-mt323.dll
 0002:000010fc       __imp_??0QRadioButton@@QAE@PAVQWidget@@PBD@Z 100210fc     qt-mt323:qt-mt323.dll
 0002:00001100       __imp_?className@QButtonGroup@@UBEPBDXZ 10021100     qt-mt323:qt-mt323.dll
 0002:00001104       __imp_?className@QRadioButton@@UBEPBDXZ 10021104     qt-mt323:qt-mt323.dll
 0002:00001108       __imp_?drawButton@QRadioButton@@MAEXPAVQPainter@@@Z 10021108     qt-mt323:qt-mt323.dll
 0002:0000110c       __imp_?drawButtonLabel@QRadioButton@@MAEXPAVQPainter@@@Z 1002110c     qt-mt323:qt-mt323.dll
 0002:00001110       __imp_?event@QButtonGroup@@MAE_NPAVQEvent@@@Z 10021110     qt-mt323:qt-mt323.dll
 0002:00001114       __imp_?hitButton@QRadioButton@@MBE_NABVQPoint@@@Z 10021114     qt-mt323:qt-mt323.dll
 0002:00001118       __imp_?metaObject@QButtonGroup@@UBEPAVQMetaObject@@XZ 10021118     qt-mt323:qt-mt323.dll
 0002:0000111c       __imp_?metaObject@QRadioButton@@UBEPAVQMetaObject@@XZ 1002111c     qt-mt323:qt-mt323.dll
 0002:00001120       __imp_?moveFocus@QButtonGroup@@UAEXH@Z 10021120     qt-mt323:qt-mt323.dll
 0002:00001124       __imp_?qt_cast@QButtonGroup@@UAEPAXPBD@Z 10021124     qt-mt323:qt-mt323.dll
 0002:00001128       __imp_?qt_cast@QRadioButton@@UAEPAXPBD@Z 10021128     qt-mt323:qt-mt323.dll
 0002:0000112c       __imp_?qt_emit@QButtonGroup@@UAE_NHPAUQUObject@@@Z 1002112c     qt-mt323:qt-mt323.dll
 0002:00001130       __imp_?qt_emit@QRadioButton@@UAE_NHPAUQUObject@@@Z 10021130     qt-mt323:qt-mt323.dll
 0002:00001134       __imp_?qt_invoke@QButtonGroup@@UAE_NHPAUQUObject@@@Z 10021134     qt-mt323:qt-mt323.dll
 0002:00001138       __imp_?qt_invoke@QRadioButton@@UAE_NHPAUQUObject@@@Z 10021138     qt-mt323:qt-mt323.dll
 0002:0000113c       __imp_?qt_property@QButtonGroup@@UAE_NHHPAVQVariant@@@Z 1002113c     qt-mt323:qt-mt323.dll
 0002:00001140       __imp_?qt_property@QRadioButton@@UAE_NHHPAVQVariant@@@Z 10021140     qt-mt323:qt-mt323.dll
 0002:00001144       __imp_?resizeEvent@QRadioButton@@MAEXPAVQResizeEvent@@@Z 10021144     qt-mt323:qt-mt323.dll
 0002:00001148       __imp_?setButton@QButtonGroup@@UAEXH@Z 10021148     qt-mt323:qt-mt323.dll
 0002:0000114c       __imp_?setChecked@QRadioButton@@UAEX_N@Z 1002114c     qt-mt323:qt-mt323.dll
 0002:00001150       __imp_?setExclusive@QButtonGroup@@UAEX_N@Z 10021150     qt-mt323:qt-mt323.dll
 0002:00001154       __imp_?setRadioButtonExclusive@QButtonGroup@@UAEX_N@Z 10021154     qt-mt323:qt-mt323.dll
 0002:00001158       __imp_?sizeHint@QRadioButton@@UBE?AVQSize@@XZ 10021158     qt-mt323:qt-mt323.dll
 0002:0000115c       __imp_?updateMask@QRadioButton@@MAEXXZ 1002115c     qt-mt323:qt-mt323.dll
 0002:00001160       __imp_?activate_signal@QObject@@IAEXH@Z 10021160     qt-mt323:qt-mt323.dll
 0002:00001164       __imp_?activate_signal_bool@QObject@@IAEXH_N@Z 10021164     qt-mt323:qt-mt323.dll
 0002:00001168       __imp_?qt_cast@QTable@@UAEPAXPBD@Z 10021168     qt-mt323:qt-mt323.dll
 0002:0000116c       __imp_?qt_invoke@QTable@@UAE_NHPAUQUObject@@@Z 1002116c     qt-mt323:qt-mt323.dll
 0002:00001170       __imp_?qt_emit@QTable@@UAE_NHPAUQUObject@@@Z 10021170     qt-mt323:qt-mt323.dll
 0002:00001174       __imp_?qt_property@QTable@@UAE_NHHPAVQVariant@@@Z 10021174     qt-mt323:qt-mt323.dll
 0002:00001178       __imp_?staticMetaObject@QTable@@SAPAVQMetaObject@@XZ 10021178     qt-mt323:qt-mt323.dll
 0002:0000117c       __imp_??0QTable@@QAE@ABV0@@Z 1002117c     qt-mt323:qt-mt323.dll
 0002:00001180       __imp_??4QTable@@QAEAAV0@ABV0@@Z 10021180     qt-mt323:qt-mt323.dll
 0002:00001184       __imp_?static_QUType_bool@@3UQUType_bool@@A 10021184     qt-mt323:qt-mt323.dll
 0002:00001188       __imp_?append@?$QValueList@VQString@@@@QAE?AV?$QValueListIterator@VQString@@@@ABVQString@@@Z 10021188     qt-mt323:qt-mt323.dll
 0002:0000118c       __imp_??0QTable@@QAE@PAVQWidget@@PBD@Z 1002118c     qt-mt323:qt-mt323.dll
 0002:00001190       __imp_?numSelections@QTable@@QBEHXZ 10021190     qt-mt323:qt-mt323.dll
 0002:00001194       __imp_?selection@QTable@@QBE?AVQTableSelection@@H@Z 10021194     qt-mt323:qt-mt323.dll
 0002:00001198       __imp_?text@QClipboard@@QBE?AVQString@@XZ 10021198     qt-mt323:qt-mt323.dll
 0002:0000119c       __imp_?setText@QClipboard@@QAEXABVQString@@@Z 1002119c     qt-mt323:qt-mt323.dll
 0002:000011a0       __imp_?warning@QMessageBox@@SAHPAVQWidget@@ABVQString@@1111HH@Z 100211a0     qt-mt323:qt-mt323.dll
 0002:000011a4       __imp_?mousePressEvent@QWidget@@MAEXPAVQMouseEvent@@@Z 100211a4     qt-mt323:qt-mt323.dll
 0002:000011a8       __imp_?mouseMoveEvent@QWidget@@MAEXPAVQMouseEvent@@@Z 100211a8     qt-mt323:qt-mt323.dll
 0002:000011ac       __imp_?mouseDoubleClickEvent@QWidget@@MAEXPAVQMouseEvent@@@Z 100211ac     qt-mt323:qt-mt323.dll
 0002:000011b0       __imp_?minimumSizeHint@QWidget@@UBE?AVQSize@@XZ 100211b0     qt-mt323:qt-mt323.dll
 0002:000011b4       __imp_?metric@QWidget@@MBEHH@Z 100211b4     qt-mt323:qt-mt323.dll
 0002:000011b8       __imp_?leaveEvent@QWidget@@MAEXPAVQEvent@@@Z 100211b8     qt-mt323:qt-mt323.dll
 0002:000011bc       __imp_?keyReleaseEvent@QWidget@@MAEXPAVQKeyEvent@@@Z 100211bc     qt-mt323:qt-mt323.dll
 0002:000011c0       __imp_?keyPressEvent@QWidget@@MAEXPAVQKeyEvent@@@Z 100211c0     qt-mt323:qt-mt323.dll
 0002:000011c4       __imp_?insertChild@QObject@@UAEXPAV1@@Z 100211c4     qt-mt323:qt-mt323.dll
 0002:000011c8       __imp_?imStartEvent@QWidget@@MAEXPAVQIMEvent@@@Z 100211c8     qt-mt323:qt-mt323.dll
 0002:000011cc       __imp_?imEndEvent@QWidget@@MAEXPAVQIMEvent@@@Z 100211cc     qt-mt323:qt-mt323.dll
 0002:000011d0       __imp_?imComposeEvent@QWidget@@MAEXPAVQIMEvent@@@Z 100211d0     qt-mt323:qt-mt323.dll
 0002:000011d4       __imp_?hideEvent@QWidget@@MAEXPAVQHideEvent@@@Z 100211d4     qt-mt323:qt-mt323.dll
 0002:000011d8       __imp_?hide@QWidget@@UAEXXZ 100211d8     qt-mt323:qt-mt323.dll
 0002:000011dc       __imp_?heightForWidth@QWidget@@UBEHH@Z 100211dc     qt-mt323:qt-mt323.dll
 0002:000011e0       __imp_?handle@QPaintDevice@@UBEPAUHDC__@@XZ 100211e0     qt-mt323:qt-mt323.dll
 0002:000011e4       __imp_?fontMet@QPaintDevice@@MBEHPAVQFont@@HPBDH@Z 100211e4     qt-mt323:qt-mt323.dll
 0002:000011e8       __imp_?fontInf@QPaintDevice@@MBEHPAVQFont@@H@Z 100211e8     qt-mt323:qt-mt323.dll
 0002:000011ec       __imp_?fontChange@QWidget@@MAEXABVQFont@@@Z 100211ec     qt-mt323:qt-mt323.dll
 0002:000011f0       __imp_?focusOutEvent@QWidget@@MAEXPAVQFocusEvent@@@Z 100211f0     qt-mt323:qt-mt323.dll
 0002:000011f4       __imp_?focusNextPrevChild@QWidget@@MAE_N_N@Z 100211f4     qt-mt323:qt-mt323.dll
 0002:000011f8       __imp_?focusInEvent@QWidget@@MAEXPAVQFocusEvent@@@Z 100211f8     qt-mt323:qt-mt323.dll
 0002:000011fc       __imp_?eventFilter@QObject@@UAE_NPAV1@PAVQEvent@@@Z 100211fc     qt-mt323:qt-mt323.dll
 0002:00001200       __imp_?event@QWidget@@MAE_NPAVQEvent@@@Z 10021200     qt-mt323:qt-mt323.dll
 0002:00001204       __imp_?enterEvent@QWidget@@MAEXPAVQEvent@@@Z 10021204     qt-mt323:qt-mt323.dll
 0002:00001208       __imp_?enabledChange@QWidget@@MAEX_N@Z 10021208     qt-mt323:qt-mt323.dll
 0002:0000120c       __imp_?dropEvent@QWidget@@MAEXPAVQDropEvent@@@Z 1002120c     qt-mt323:qt-mt323.dll
 0002:00001210       __imp_?dragMoveEvent@QWidget@@MAEXPAVQDragMoveEvent@@@Z 10021210     qt-mt323:qt-mt323.dll
 0002:00001214       __imp_?dragLeaveEvent@QWidget@@MAEXPAVQDragLeaveEvent@@@Z 10021214     qt-mt323:qt-mt323.dll
 0002:00001218       __imp_?dragEnterEvent@QWidget@@MAEXPAVQDragEnterEvent@@@Z 10021218     qt-mt323:qt-mt323.dll
 0002:0000121c       __imp_?disconnectNotify@QObject@@MAEXPBD@Z 1002121c     qt-mt323:qt-mt323.dll
 0002:00001220       __imp_?destroy@QWidget@@MAEX_N0@Z 10021220     qt-mt323:qt-mt323.dll
 0002:00001224       __imp_?customWhatsThis@QWidget@@UBE_NXZ 10021224     qt-mt323:qt-mt323.dll
 0002:00001228       __imp_?customEvent@QObject@@MAEXPAVQCustomEvent@@@Z 10021228     qt-mt323:qt-mt323.dll
 0002:0000122c       __imp_?create@QWidget@@MAEXPAUHWND__@@_N1@Z 1002122c     qt-mt323:qt-mt323.dll
 0002:00001230       __imp_??0QObject@@QAE@PAV0@PBD@Z 10021230     qt-mt323:qt-mt323.dll
 0002:00001234       __imp_??1QObject@@UAE@XZ   10021234     qt-mt323:qt-mt323.dll
 0002:00001238       __imp_??0QDate@@QAE@HHH@Z  10021238     qt-mt323:qt-mt323.dll
 0002:0000123c       __imp_??0QDateTime@@QAE@ABVQDate@@@Z 1002123c     qt-mt323:qt-mt323.dll
 0002:00001240       __imp_??OQDateTime@@QBE_NABV0@@Z 10021240     qt-mt323:qt-mt323.dll
 0002:00001244       __imp_??0QFileInfo@@QAE@ABV0@@Z 10021244     qt-mt323:qt-mt323.dll
 0002:00001248       __imp_?eventLoop@QApplication@@SAPAVQEventLoop@@XZ 10021248     qt-mt323:qt-mt323.dll
 0002:0000124c       __imp_??M@YA_NABVQString@@0@Z 1002124c     qt-mt323:qt-mt323.dll
 0002:00001250       __imp_?rebalance@QMapPrivateBase@@QAEXPAUQMapNodeBase@@AAPAU2@@Z 10021250     qt-mt323:qt-mt323.dll
 0002:00001254       __imp_??4QObject@@QAEAAV0@ABV0@@Z 10021254     qt-mt323:qt-mt323.dll
 0002:00001258       __imp_?begin@?$QPtrList@VQDockWindow@@@@QAE?AV?$QPtrListStdIterator@VQDockWindow@@@@XZ 10021258     qt-mt323:qt-mt323.dll
 0002:0000125c       __imp_?end@?$QPtrList@VQDockWindow@@@@QAE?AV?$QPtrListStdIterator@VQDockWindow@@@@XZ 1002125c     qt-mt323:qt-mt323.dll
 0002:00001260       __imp_?null@QChar@@2V1@A   10021260     qt-mt323:qt-mt323.dll
 0002:00001264       __imp_?qt_cast@QObject@@UAEPAXPBD@Z 10021264     qt-mt323:qt-mt323.dll
 0002:00001268       __imp_?qt_invoke@QObject@@UAE_NHPAUQUObject@@@Z 10021268     qt-mt323:qt-mt323.dll
 0002:0000126c       __imp_?qt_emit@QObject@@UAE_NHPAUQUObject@@@Z 1002126c     qt-mt323:qt-mt323.dll
 0002:00001270       __imp_?qt_property@QObject@@UAE_NHHPAVQVariant@@@Z 10021270     qt-mt323:qt-mt323.dll
 0002:00001274       __imp_?staticMetaObject@QObject@@SAPAVQMetaObject@@XZ 10021274     qt-mt323:qt-mt323.dll
 0002:00001278       __imp_?contextMenuEvent@QWidget@@MAEXPAVQContextMenuEvent@@@Z 10021278     qt-mt323:qt-mt323.dll
 0002:0000127c       __imp_?connectNotify@QObject@@MAEXPBD@Z 1002127c     qt-mt323:qt-mt323.dll
 0002:00001280       __imp_?cmd@QPaintDevice@@MAE_NHPAVQPainter@@PATQPDevCmdParam@@@Z 10021280     qt-mt323:qt-mt323.dll
 0002:00001284       __imp_?closeEvent@QWidget@@MAEXPAVQCloseEvent@@@Z 10021284     qt-mt323:qt-mt323.dll
 0002:00001288       __imp_?close@QWidget@@UAE_N_N@Z 10021288     qt-mt323:qt-mt323.dll
 0002:0000128c       __imp_?childEvent@QObject@@MAEXPAVQChildEvent@@@Z 1002128c     qt-mt323:qt-mt323.dll
 0002:00001290       __imp_?checkConnectArgs@QObject@@MAE_NPBDPBV1@0@Z 10021290     qt-mt323:qt-mt323.dll
 0002:00001294       __imp_?adjustSize@QWidget@@UAEXXZ 10021294     qt-mt323:qt-mt323.dll
 0002:00001298       __imp_?setGeometry@QSpacerItem@@UAEXABVQRect@@@Z 10021298     qt-mt323:qt-mt323.dll
 0002:0000129c       \177qt-mt323_NULL_THUNK_DATA 1002129c     qt-mt323:qt-mt323.dll
 0002:000012a0       ___xc_a                    100212a0     MSVCRT:cinitexe.obj
 0002:00001300       ___xc_z                    10021300     MSVCRT:cinitexe.obj
 0002:00001304       ___xi_a                    10021304     MSVCRT:cinitexe.obj
 0002:00001310       ___xi_z                    10021310     MSVCRT:cinitexe.obj
 0002:00001324       ??_7dialog@@6BQObject@@@   10021324     dialogimpl.obj
 0002:000014dc       ??_7dialog@@6BQPaintDevice@@@ 100214dc     dialogimpl.obj
 0002:00001500       ??_7fileDrop@@6BQObject@@@ 10021500     fileDrop.obj
 0002:000017e4       ??_7fileDrop@@6BQPaintDevice@@@ 100217e4     fileDrop.obj
 0002:00001804       ??_C@_0N@KKJBDLGM@1cbChanged?$CI?$CJ?$AA@ 10021804     fileDrop.obj
 0002:00001814       ??_C@_0P@GLIODLHI@2dataChanged?$CI?$CJ?$AA@ 10021814     fileDrop.obj
 0002:00001824       ??_C@_0O@ILGLPLAE@drop?5event?5?$CFs?$AA@ 10021824     fileDrop.obj
 0002:00001834       ??_C@_0O@OKOFBKJK@text?1uri?9list?$AA@ 10021834     fileDrop.obj
 0002:00001844       ??_C@_0BF@NBOHNFFI@clipboard?5format?3?5?$CFs?$AA@ 10021844     fileDrop.obj
 0002:0000185c       ??_C@_05NEBJFIEK@Paste?$AA@ 1002185c     fileDrop.obj
 0002:00001864       ??_C@_09IACAPMLJ@15?513?58?51?$AA@ 10021864     fileManager.obj
 0002:00001870       ??_C@_0M@HIKHPPPO@a?5c?5?$CD000000?$AA@ 10021870     fileManager.obj
 0002:0000187c       ??_C@_0M@GPNFCLCG@?$CD?5c?5?$CD9c9c00?$AA@ 1002187c     fileManager.obj
 0002:00001888       ??_C@_0M@JJBPMLBF@e?5c?5?$CDcece63?$AA@ 10021888     fileManager.obj
 0002:00001894       ??_C@_0M@FPMNAHCM@b?5c?5?$CDf7f7f7?$AA@ 10021894     fileManager.obj
 0002:000018a0       ??_C@_0M@ILMKFOIF@f?5c?5?$CDffce9c?$AA@ 100218a0     fileManager.obj
 0002:000018ac       ??_C@_0M@LNKEOAIE@d?5c?5?$CDffff9c?$AA@ 100218ac     fileManager.obj
 0002:000018b8       ??_C@_0M@POENAFOL@c?5c?5?$CDffffce?$AA@ 100218b8     fileManager.obj
 0002:000018c4       ??_C@_08IMFNEMJ@?4?5c?5none?$AA@ 100218c4     fileManager.obj
 0002:000018d0       ??_C@_0BA@CIENNFAI@?4?4?$CD?$CD?$CD?$CD?$CDa?4?4?4?4?4?4?4?$AA@ 100218d0     fileManager.obj
 0002:000018e0       ??_C@_0BA@GNHHMKN@?4?$CDbccdd?$CDa?4?4?4?4?4?4?$AA@ 100218e0     fileManager.obj
 0002:000018f0       ??_C@_0BA@PKJOLHEE@?$CDeeeeeee?$CD?$CD?$CD?$CD?$CD?$CD?4?$AA@ 100218f0     fileManager.obj
 0002:00001900       ??_C@_0BA@MGMHLGDO@?$CDcccccccccccdea?$AA@ 10021900     fileManager.obj
 0002:00001910       ??_C@_0BA@MPCJIDKO@?$CDcddddddddddfea?$AA@ 10021910     fileManager.obj
 0002:00001920       ??_C@_0BA@IIHPAJGM@?$CDcdddddddfdfdea?$AA@ 10021920     fileManager.obj
 0002:00001930       ??_C@_0BA@ICOBCCKF@?$CDcddddddddfdfea?$AA@ 10021930     fileManager.obj
 0002:00001940       ??_C@_0BA@KGIJCBOK@?$CDcdddddfdfdfdea?$AA@ 10021940     fileManager.obj
 0002:00001950       ??_C@_0BA@MAMECFNI@?$CDcddddddfdfdfea?$AA@ 10021950     fileManager.obj
 0002:00001960       ??_C@_0BA@FEOMFAKA@?$CDcdddfdfdfdffea?$AA@ 10021960     fileManager.obj
 0002:00001970       ??_C@_0BA@LDKEPMLH@?$CDcfdfdfdfdfffea?$AA@ 10021970     fileManager.obj
 0002:00001980       ??_C@_0BA@IBIMNNKM@?$CDeeeeeeeeeeeeea?$AA@ 10021980     fileManager.obj
 0002:00001990       ??_C@_0BA@KKAIFHCE@?4aaaaaaaaaaaaaa?$AA@ 10021990     fileManager.obj
 0002:000019a0       ??_C@_0CD@BFGBAEB@?5?5?5?514?5?5?5?514?5?5?5?5?5?5?5?54?5?5?5?5?5?5?5?5?5?5?5@ 100219a0     fileManager.obj
 0002:000019c4       ??_C@_0M@EKMPMHDK@?4?5c?5?$CD040404?$AA@ 100219c4     fileManager.obj
 0002:000019d0       ??_C@_0M@NBLJLJNN@?$CD?5c?5?$CD808304?$AA@ 100219d0     fileManager.obj
 0002:000019dc       ??_C@_0M@EAFJJBBG@a?5c?5?$CDbfc2bf?$AA@ 100219dc     fileManager.obj
 0002:000019e8       ??_C@_08PBKCALNO@b?5c?5None?$AA@ 100219e8     fileManager.obj
 0002:000019f4       ??_C@_0P@HFKAALMG@?4?4?4?4?4?4?4?4?4?4?4?4?4?4?$AA@ 100219f4     fileManager.obj
 0002:00001a04       ??_C@_0P@LGBCEGMD@?4?$CD?4aaaaaaaa?4a?4?$AA@ 10021a04     fileManager.obj
 0002:00001a14       ??_C@_0P@MNNEIMDO@?4?$CD?4aaaaaaaa?4?4?4?$AA@ 10021a14     fileManager.obj
 0002:00001a24       ??_C@_0P@MFAMBPGN@?4?$CD?4aaaaaaaa?4?$CD?4?$AA@ 10021a24     fileManager.obj
 0002:00001a34       ??_C@_0P@HPMEFAGN@?4?$CD?$CD?4?4?4?4?4?4?4?4?$CD?$CD?4?$AA@ 10021a34     fileManager.obj
 0002:00001a44       ??_C@_0P@JAJCNDBN@?4?$CD?$CD?$CD?$CD?$CD?$CD?$CD?$CD?$CD?$CD?$CD?$CD?4?$AA@ 10021a44     fileManager.obj
 0002:00001a54       ??_C@_0P@INKOIILA@?4?$CD?$CD?4?4?4?4?4?4?4?4?4?$CD?4?$AA@ 10021a54     fileManager.obj
 0002:00001a64       ??_C@_0P@KJADPPJB@?4?$CD?$CD?4?4?4?4?4?4aa?4?$CD?4?$AA@ 10021a64     fileManager.obj
 0002:00001a74       ??_C@_0P@PKKONJFP@b?4?4?4?4?4?4?4?4?4?4?4?4?4?$AA@ 10021a74     fileManager.obj
 0002:00001a84       ??_C@_09KDLGOOHH@16?516?54?51?$AA@ 10021a84     fileManager.obj
 0002:00001a90       ??_C@_0M@KEPPNGJB@?$CD?5c?5?$CD000000?$AA@ 10021a90     fileManager.obj
 0002:00001a9c       ??_C@_0M@BCKHMLG@b?5c?5?$CD000080?$AA@ 10021a9c     fileManager.obj
 0002:00001aa8       ??_C@_0M@DPJAAKFM@a?5c?5?$CDffffff?$AA@ 10021aa8     fileManager.obj
 0002:00001ab4       ??_C@_0BB@DDKGLOCG@?4?4?4?4?4?4?4?4?4?4?4?4?4?4?4?4?$AA@ 10021ab4     fileManager.obj
 0002:00001ac8       ??_C@_0BB@GDAPNCLP@?4?$CD?$CD?$CD?$CD?$CD?$CD?4?4?4?4?4?4?4?4?4?$AA@ 10021ac8     fileManager.obj
 0002:00001adc       ??_C@_0BB@FFNCKNDA@?4?$CDaaaa?$CD?$CD?4?4?4?4?4?4?4?4?$AA@ 10021adc     fileManager.obj
 0002:00001af0       ??_C@_0BB@DONCJNPK@?4?$CDaaaa?$CDa?$CD?4?4?4?4?4?4?4?$AA@ 10021af0     fileManager.obj
 0002:00001b04       ??_C@_0BB@HJAKJBPB@?4?$CDa?$CD?$CDa?$CDbbbbbb?4?4?4?$AA@ 10021b04     fileManager.obj
 0002:00001b18       ??_C@_0BB@FLJEJCPD@?4?$CDaaaaabaaaabb?4?4?$AA@ 10021b18     fileManager.obj
 0002:00001b2c       ??_C@_0BB@BPNLNHEE@?4?$CDa?$CD?$CD?$CD?$CDbaaaabab?4?$AA@ 10021b2c     fileManager.obj
 0002:00001b40       ??_C@_0BB@MGPEEHJO@?4?$CDaaaaaba?$CD?$CDabbbb?$AA@ 10021b40     fileManager.obj
 0002:00001b54       ??_C@_0BB@GPBBDME@?4?$CDa?$CD?$CD?$CD?$CDbaaaaaaab?$AA@ 10021b54     fileManager.obj
 0002:00001b68       ??_C@_0BB@MABJBMAB@?4?$CDaaaaaba?$CD?$CD?$CD?$CD?$CDab?$AA@ 10021b68     fileManager.obj
 0002:00001b7c       ??_C@_0BB@GEIMNJCI@?4?$CD?$CD?$CD?$CD?$CD?$CDbaaaaaaab?$AA@ 10021b7c     fileManager.obj
 0002:00001b90       ??_C@_0BB@NNLHCEIJ@?4?4?4?4?4?4?4ba?$CD?$CD?$CD?$CD?$CDab?$AA@ 10021b90     fileManager.obj
 0002:00001ba4       ??_C@_0BB@DECFLFLB@?4?4?4?4?4?4?4baaaaaaab?$AA@ 10021ba4     fileManager.obj
 0002:00001bb8       ??_C@_0BB@GDAIINMD@?4?4?4?4?4?4?4bbbbbbbbb?$AA@ 10021bb8     fileManager.obj
 0002:00001bcc       ??_C@_09OJGAFBMP@16?516?58?51?$AA@ 10021bcc     fileManager.obj
 0002:00001bd8       ??_C@_0M@HFLCJFDJ@e?5c?5?$CD000080?$AA@ 10021bd8     fileManager.obj
 0002:00001be4       ??_C@_0M@JHADGEMH@c?5c?5?$CD808000?$AA@ 10021be4     fileManager.obj
 0002:00001bf0       ??_C@_0M@CLFHJBA@b?5c?5?$CD808080?$AA@ 10021bf0     fileManager.obj
 0002:00001bfc       ??_C@_0M@MHLPHELG@d?5c?5?$CDd4d0c8?$AA@ 10021bfc     fileManager.obj
 0002:00001c08       ??_C@_0M@LLEAKCIM@a?5c?5?$CDffff00?$AA@ 10021c08     fileManager.obj
 0002:00001c14       ??_C@_0M@ELAIODND@f?5c?5?$CDffffff?$AA@ 10021c14     fileManager.obj
 0002:00001c20       ??_C@_0BB@GHIGIKBH@?4?4?4?4?4?4?$CD?$CD?$CD?$CD?4?4?4?4?4?4?$AA@ 10021c20     fileManager.obj
 0002:00001c34       ??_C@_0BB@EIGJHLLO@?4?4?$CD?$CD?$CD?$CD?$CDaa?$CD?$CD?$CD?$CD?$CD?4?4?$AA@ 10021c34     fileManager.obj
 0002:00001c48       ??_C@_0BB@GFDBAPPE@?4?$CDbcb?$CDa?$CD?$CDa?$CDcbc?$CD?4?$AA@ 10021c48     fileManager.obj
 0002:00001c5c       ??_C@_0BB@JBCPPMEE@?4?$CDcb?$CDdddddd?$CDcb?$CD?4?$AA@ 10021c5c     fileManager.obj
 0002:00001c70       ??_C@_0BB@OPOOCIAI@?4?$CDbc?$CD?$CD?$CD?$CD?$CD?$CD?$CD?$CDbc?$CD?4?$AA@ 10021c70     fileManager.obj
 0002:00001c84       ??_C@_0BB@EEBHCOMC@?4?$CDcbcbcbcbcbcb?$CD?4?$AA@ 10021c84     fileManager.obj
 0002:00001c98       ??_C@_0BB@BABPPNAH@?4?$CDbcbcbeeeeeee?$CD?4?$AA@ 10021c98     fileManager.obj
 0002:00001cac       ??_C@_0BB@IAJPFFAE@?4?$CDcbcbcefffffee?4?$AA@ 10021cac     fileManager.obj
 0002:00001cc0       ??_C@_0BB@DCBNANCH@?4?$CDbcbcbefffffefe?$AA@ 10021cc0     fileManager.obj
 0002:00001cd4       ??_C@_0BB@KKOBKMBK@?4?$CDcbcbcefeeefeee?$AA@ 10021cd4     fileManager.obj
 0002:00001ce8       ??_C@_0BB@CAKIKCMJ@?4?$CDbcbcbefffffffe?$AA@ 10021ce8     fileManager.obj
 0002:00001cfc       ??_C@_0BB@OPAHGIJD@?4?$CDcbcbcefeeeeefe?$AA@ 10021cfc     fileManager.obj
 0002:00001d10       ??_C@_0BB@FMOFIOAF@?4?4?$CD?$CD?$CD?$CD?$CDefffffffe?$AA@ 10021d10     fileManager.obj
 0002:00001d24       ??_C@_0BB@FCCLJILH@?4?4?4?4?4?4?4eeeeeeeee?$AA@ 10021d24     fileManager.obj
 0002:00001d38       ??_C@_09DOGBNGMO@16?516?53?51?$AA@ 10021d38     fileManager.obj
 0002:00001d44       ??_C@_0M@KKOMIHCJ@?$CD?5c?5?$CD000080?$AA@ 10021d44     fileManager.obj
 0002:00001d50       ??_C@_0M@HFCLKLOA@a?5c?5?$CD808080?$AA@ 10021d50     fileManager.obj
 0002:00001d5c       ??_C@_0BB@DDMLBOGJ@?4?4?4?4?4?4?4?$CD?$CD?$CD?$CDa?4?4?4?4?$AA@ 10021d5c     fileManager.obj
 0002:00001d70       ??_C@_0BB@JOKGMNA@?4?$CD?4?4?4?$CD?$CD?4?4?4?4?$CDa?4?4?4?$AA@ 10021d70     fileManager.obj
 0002:00001d84       ??_C@_0BB@HJFOCKLM@?4?$CD?$CD?4?$CD?4?4?4?4?4?4?4?$CD?4?4?4?$AA@ 10021d84     fileManager.obj
 0002:00001d98       ??_C@_0BB@IJIIDKJJ@?4?$CD?$CD?$CD?4?4?4?4?4?4?4?4?$CD?4?4?4?$AA@ 10021d98     fileManager.obj
 0002:00001dac       ??_C@_0BB@MOKEFKOH@?4?$CD?$CD?$CD?$CD?4?4?4?4?4?4?4?$CD?4?4?4?$AA@ 10021dac     fileManager.obj
 0002:00001dc0       ??_C@_0BB@MOKGEDPO@?4?$CD?$CD?$CD?$CD?$CD?4?4?4?4?4?$CDa?4?4?4?$AA@ 10021dc0     fileManager.obj
 0002:00001dd4       ??_C@_0BB@DNHLKIGI@?4?4?4?4?4?4?4?4?4?4a?$CD?4?4?4?4?$AA@ 10021dd4     fileManager.obj
 0002:00001dec       ??_SQVBoxLayout@@6BQObject@@@ 10021dec     fileManager.obj
 0002:00001e54       ??_SQVBoxLayout@@6BQLayoutItem@@@ 10021e54     fileManager.obj
 0002:00001e9c       ??_SQLabel@@6BQObject@@@   10021e9c     fileManager.obj
 0002:00002094       ??_SQLabel@@6BQPaintDevice@@@ 10022094     fileManager.obj
 0002:000020bc       ??_SQListViewItem@@6B@     100220bc     fileManager.obj
 0002:0000215c       ??_SQListView@@6BQObject@@@ 1002215c     fileManager.obj
 0002:00002440       ??_SQListView@@6BQPaintDevice@@@ 10022440     fileManager.obj
 0002:00002464       ??_SQSplitter@@6BQObject@@@ 10022464     fileManager.obj
 0002:0000264c       ??_SQSplitter@@6BQPaintDevice@@@ 1002264c     fileManager.obj
 0002:00002674       ??_SQGuardedPtrPrivate@@6B@ 10022674     fileManager.obj
 0002:000026c8       ??_7QDockWindowList@@6B@   100226c8     fileManager.obj
 0002:000026ec       ??_7?$QPtrList@VQPopupMenu@@@@6B@ 100226ec     fileManager.obj
 0002:00002710       ??_7QPopupMenuList@@6B@    10022710     fileManager.obj
 0002:00002734       ??_7config_plugin_base@@6BQObject@@@ 10022734     fileManager.obj
 0002:0000290c       ??_7config_plugin_base@@6BQPaintDevice@@@ 1002290c     fileManager.obj
 0002:00002930       ??_C@_0EB@GNDACMDJ@?$CC?5?9?5the?5author?5should?5have?5defin@ 10022930     fileManager.obj
 0002:00002974       ??_C@_0CH@BDPDPLDP@This?5is?5the?5default?5?$CCAbout?$CC?5text@ 10022974     fileManager.obj
 0002:000029a0       ??_7fileManager@@6BQObject@@@ 100229a0     fileManager.obj
 0002:00002b78       ??_7fileManager@@6BQPaintDevice@@@ 10022b78     fileManager.obj
 0002:00002b98       ??_C@_0BD@KAKJEBEP@fileManager?5path?5?3?$AA@ 10022b98     fileManager.obj
 0002:00002bac       ??_C@_0DI@IJJKAFPF@DON?8T?5USE?5THIS?5UNLESS?5YOU?5REALLY@ 10022bac     fileManager.obj
 0002:00002be8       ??_C@_0EM@MMDFMPPO@?$DMh1?5text?$DN?$CCred?$CC?$DODON?8T?5USE?5THIS?5UN@ 10022be8     fileManager.obj
 0002:00002c38       ??_C@_0BEL@MMAFIFFO@?$DMh1?$DOProof?5of?5concept?5file?5manage@ 10022c38     fileManager.obj
 0002:00002d84       ??_C@_0M@EIENEKNL@Directories?$AA@ 10022d84     fileManager.obj
 0002:00002d90       ??_C@_04PBAHLACE@File?$AA@ 10022d90     fileManager.obj
 0002:00002d98       ??_C@_04EBKMHHBE@Size?$AA@ 10022d98     fileManager.obj
 0002:00002da0       ??_C@_04FMEGDJGD@Date?$AA@ 10022da0     fileManager.obj
 0002:00002da8       ??_C@_0BP@DLOLLDHI@1dirChanged?$CI?5QListViewItem?5?$CK?5?$CJ?$AA@ 10022da8     fileManager.obj
 0002:00002dc8       ??_C@_0BM@LNFFBMAG@2clicked?$CI?5QListViewItem?5?$CK?5?$CJ?$AA@ 10022dc8     fileManager.obj
 0002:00002de4       ??_C@_0BL@EPJPGGJG@1doFileList?$CI?5QStringList?5?$CJ?$AA@ 10022de4     fileManager.obj
 0002:00002e00       ??_C@_0BJ@DOHBJGPH@2fileList?$CI?5QStringList?5?$CJ?$AA@ 10022e00     fileManager.obj
 0002:00002e1c       ??_C@_04MKMCLCOO@lock?$AA@ 10022e1c     fileManager.obj
 0002:00002e24       ??_C@_0BF@HJDLHOKO@Configuration?5Plugin?$AA@ 10022e24     fileManager.obj
 0002:00002e3c       ??_C@_01KMDKNFGN@?1?$AA@   10022e3c     fileManager.obj
 0002:00002e40       ??_C@_0L@CIKGEHEG@uploadFile?$AA@ 10022e40     fileManager.obj
 0002:00002e4c       ??_C@_06BNCCALCL@unlock?$AA@ 10022e4c     fileManager.obj
 0002:00002e54       ??_C@_0P@CDOMPBPE@Starting?5timer?$AA@ 10022e54     fileManager.obj
 0002:00002e64       ??_C@_03DAPAKLGM@dir?$AA@  10022e64     fileManager.obj
 0002:00002e68       ??_C@_0L@IINBHNNO@mydocument?$AA@ 10022e68     fileManager.obj
 0002:00002e74       ??_C@_04JNIHBGGH@date?$AA@ 10022e74     fileManager.obj
 0002:00002e7c       ??_C@_04MEMAJGDJ@name?$AA@ 10022e7c     fileManager.obj
 0002:00002e84       ??_C@_0BB@IMDJJABM@dd?1MM?1yyyy?5hh?3mm?$AA@ 10022e84     fileManager.obj
 0002:00002e98       ??_C@_04IAGNFIBA@size?$AA@ 10022e98     fileManager.obj
 0002:00002ea0       ??_C@_0CO@DMDPGOMC@Being?5asked?5to?5navigate?5to?5?$CFs?5wi@ 10022ea0     fileManager.obj
 0002:00002ece       ??_C@_00CNPNBAHC@?$AA@     10022ece     fileManager.obj
 0002:00002ed0       ??_C@_0BD@GPFAPHEJ@fileManager?3?3apply?$AA@ 10022ed0     fileManager.obj
 0002:00002ee4       ??_C@_04MKEOLIJC@?5to?5?$AA@ 10022ee4     fileManager.obj
 0002:00002eec       ??_C@_0BD@BBIIOIAM@copying?5file?5from?5?$AA@ 10022eec     fileManager.obj
 0002:00002f00       ??_C@_0DJ@LPNHIDPB@void?5fileManager?3?3timerEvent?$CI?5QT@ 10022f00     fileManager.obj
 0002:00002f44       ??_SQWidget@@6BQObject@@@  10022f44     frombasedialog.obj
 0002:000030f8       ??_SQWidget@@6BQPaintDevice@@@ 100230f8     frombasedialog.obj
 0002:0000311c       ??_7fromBaseDialogBase@@6BQObject@@@ 1002311c     frombasedialog.obj
 0002:000032d4       ??_7fromBaseDialogBase@@6BQPaintDevice@@@ 100232d4     frombasedialog.obj
 0002:000032fc       ??_SQPushButton@@6BQObject@@@ 100232fc     frombasedialog.obj
 0002:000034ec       ??_SQPushButton@@6BQPaintDevice@@@ 100234ec     frombasedialog.obj
 0002:00003514       ??_SQFrame@@6BQObject@@@   10023514     frombasedialog.obj
 0002:000036e8       ??_SQFrame@@6BQPaintDevice@@@ 100236e8     frombasedialog.obj
 0002:0000370c       ??_SQListBox@@6BQObject@@@ 1002370c     frombasedialog.obj
 0002:000039b4       ??_SQListBox@@6BQPaintDevice@@@ 100239b4     frombasedialog.obj
 0002:000039dc       ??_SQGroupBox@@6BQObject@@@ 100239dc     frombasedialog.obj
 0002:00003bbc       ??_SQGroupBox@@6BQPaintDevice@@@ 10023bbc     frombasedialog.obj
 0002:00003be4       ??_SQLineEdit@@6BQObject@@@ 10023be4     frombasedialog.obj
 0002:00003e0c       ??_SQLineEdit@@6BQPaintDevice@@@ 10023e0c     frombasedialog.obj
 0002:00003e34       ??_SQSpacerItem@@6B@       10023e34     frombasedialog.obj
 0002:00003e7c       ??_SQHBoxLayout@@6BQObject@@@ 10023e7c     frombasedialog.obj
 0002:00003ee4       ??_SQHBoxLayout@@6BQLayoutItem@@@ 10023ee4     frombasedialog.obj
 0002:00003f24       ??_C@_0BD@FOLDOIBO@fromBaseDialogBase?$AA@ 10023f24     frombasedialog.obj
 0002:00003f38       ??_C@_0N@CJBMCOMC@textLabel1_4?$AA@ 10023f38     frombasedialog.obj
 0002:00003f48       ??_C@_07LDCEANHD@layout4?$AA@ 10023f48     frombasedialog.obj
 0002:00003f50       ??_C@_02BIKLEMDE@db?$AA@   10023f50     frombasedialog.obj
 0002:00003f54       ??_C@_07PMGFJLLE@layout3?$AA@ 10023f54     frombasedialog.obj
 0002:00003f5c       ??_C@_07FPLPIMMH@dbClear?$AA@ 10023f5c     frombasedialog.obj
 0002:00003f64       ??_C@_07KKDPDMDC@layout5?$AA@ 10023f64     frombasedialog.obj
 0002:00003f6c       ??_C@_09EIIPLPDF@layout5_2?$AA@ 10023f6c     frombasedialog.obj
 0002:00003f78       ??_C@_09JAGLPBKP@groupBox1?$AA@ 10023f78     frombasedialog.obj
 0002:00003f84       ??_C@_0N@EHHLDFOB@checkoutFile?$AA@ 10023f84     frombasedialog.obj
 0002:00003f94       ??_C@_0N@LJNCPLAD@downloadFile?$AA@ 10023f94     frombasedialog.obj
 0002:00003fa4       ??_C@_08BNOEHPNM@editFile?$AA@ 10023fa4     frombasedialog.obj
 0002:00003fb0       ??_C@_0L@HHAIFFOB@unlockFile?$AA@ 10023fb0     frombasedialog.obj
 0002:00003fbc       ??_C@_0M@HLAAGANF@groupBox2_2?$AA@ 10023fbc     frombasedialog.obj
 0002:00003fc8       ??_C@_08LKNNDKNB@lockFile?$AA@ 10023fc8     frombasedialog.obj
 0002:00003fd4       ??_C@_08OHOAFCBC@editLock?$AA@ 10023fd4     frombasedialog.obj
 0002:00003fe0       ??_C@_09LLEGKCGM@groupBox2?$AA@ 10023fe0     frombasedialog.obj
 0002:00003fec       ??_C@_0M@IKGKPMGN@checkoutDir?$AA@ 10023fec     frombasedialog.obj
 0002:00003ff8       ??_C@_0M@PHLPGIPF@downloadDir?$AA@ 10023ff8     frombasedialog.obj
 0002:00004004       ??_C@_07BAPPNKJD@editDir?$AA@ 10024004     frombasedialog.obj
 0002:0000400c       ??_C@_09OHGPLKLL@uploadDir?$AA@ 1002400c     frombasedialog.obj
 0002:00004018       ??_C@_09EMPFBFIC@unlockDir?$AA@ 10024018     frombasedialog.obj
 0002:00004024       ??_C@_0O@DLGNBGPO@groupBox2_2_2?$AA@ 10024024     frombasedialog.obj
 0002:00004034       ??_C@_0M@GHLBHEIA@editDirList?$AA@ 10024034     frombasedialog.obj
 0002:00004040       ??_C@_07JIAJFOLA@layout7?$AA@ 10024040     frombasedialog.obj
 0002:00004048       ??_C@_0BA@PEHLHPPD@groupBox2_2_2_2?$AA@ 10024048     frombasedialog.obj
 0002:00004058       ??_C@_08NCKPMOJE@navigate?$AA@ 10024058     frombasedialog.obj
 0002:00004064       ??_C@_0N@FFJAKNHO@editNavigate?$AA@ 10024064     frombasedialog.obj
 0002:00004074       ??_C@_0BC@HFLLBHFE@groupBox2_2_2_2_2?$AA@ 10024074     frombasedialog.obj
 0002:00004088       ??_C@_04PCJFHION@help?$AA@ 10024088     frombasedialog.obj
 0002:00004090       ??_C@_08NPLHJIBB@editHelp?$AA@ 10024090     frombasedialog.obj
 0002:0000409c       ??_C@_0L@FOJLNNIH@dirtygroup?$AA@ 1002409c     frombasedialog.obj
 0002:000040a8       ??_C@_05CCAMFJOL@clean?$AA@ 100240a8     frombasedialog.obj
 0002:000040b0       ??_C@_05CFEJGMAI@dirty?$AA@ 100240b0     frombasedialog.obj
 0002:000040b8       ??_C@_09JBGPPANP@editDirty?$AA@ 100240b8     frombasedialog.obj
 0002:000040c4       ??_C@_08KDEPKCK@dropzone?$AA@ 100240c4     frombasedialog.obj
 0002:000040d0       ??_C@_05MLDKGAGH@Form1?$AA@ 100240d0     frombasedialog.obj
 0002:000040d8       ??_C@_0DJ@MGGNBBLL@?$DMh1?$DO?$DMp?5align?$DN?$CCcenter?$CC?$DOConfig?5Edi@ 100240d8     frombasedialog.obj
 0002:00004114       ??_C@_05MDNHABIA@Clear?$AA@ 10024114     frombasedialog.obj
 0002:0000411c       ??_C@_0O@NCENGNDK@Checkout?5?$CIRW?$CJ?$AA@ 1002411c     frombasedialog.obj
 0002:0000412c       ??_C@_0O@IOICLFGI@Download?5?$CIRO?$CJ?$AA@ 1002412c     frombasedialog.obj
 0002:0000413c       ??_C@_06GPFPJJPN@Upload?$AA@ 1002413c     frombasedialog.obj
 0002:00004144       ??_C@_06NCJPDCLH@Unlock?$AA@ 10024144     frombasedialog.obj
 0002:0000414c       ??_C@_04LADJNOK@Lock?$AA@  1002414c     frombasedialog.obj
 0002:00004154       ??_C@_09EOAFACM@Directory?$AA@ 10024154     frombasedialog.obj
 0002:00004160       ??_C@_03JAMCAEFC@Dir?$AA@  10024160     frombasedialog.obj
 0002:00004164       ??_C@_08FAFOEMDH@Navigate?$AA@ 10024164     frombasedialog.obj
 0002:00004170       ??_C@_04DDFEFHOJ@Help?$AA@ 10024170     frombasedialog.obj
 0002:00004178       ??_C@_04DNCDCIAE@Open?$AA@ 10024178     frombasedialog.obj
 0002:00004180       ??_C@_05CCOFGJDO@Dirty?$AA@ 10024180     frombasedialog.obj
 0002:00004188       ??_C@_05CFKAFMNN@Clean?$AA@ 10024188     frombasedialog.obj
 0002:00004190       __xmm@00000027000003780000000b0000000b 10024190     frombasedialog.obj
 0002:000041a0       __xmm@000001890000037800000028000001a4 100241a0     frombasedialog.obj
 0002:000041b0       __xmm@000002310000019f0000002f0000000c 100241b0     frombasedialog.obj
 0002:000041c4       ??_7fromBaseDialog@@6BQObject@@@ 100241c4     frombasedialogimpl.obj
 0002:0000437c       ??_7fromBaseDialog@@6BQPaintDevice@@@ 1002437c     frombasedialogimpl.obj
 0002:000043a0       ??_7launchCustomTable@@6BQObject@@@ 100243a0     launchCustomTable.obj
 0002:00004744       ??_7launchCustomTable@@6BQPaintDevice@@@ 10024744     launchCustomTable.obj
 0002:00004764       ??_C@_0BB@DCECNDKJ@Application?5Name?$AA@ 10024764     launchCustomTable.obj
 0002:00004778       ??_C@_0BC@IINCGMGA@Working?5Directory?$AA@ 10024778     launchCustomTable.obj
 0002:0000478c       ??_C@_09LOINMIFK@Arguments?$AA@ 1002478c     launchCustomTable.obj
 0002:00004798       ??_C@_0L@PCMONAI@Delay?5?$CImS?$CJ?$AA@ 10024798     launchCustomTable.obj
 0002:000047a4       ??_C@_0BB@GMFDKLGJ@Restart?5On?5Crash?$AA@ 100247a4     launchCustomTable.obj
 0002:000047b8       ??_C@_02GIPFHKNO@OK?$AA@   100247b8     launchEditor.obj
 0002:000047c4       ??_SQAction@@6B@           100247c4     launchEditor.obj
 0002:00004854       ??_SQDockWindow@@6BQObject@@@ 10024854     launchEditor.obj
 0002:00004a64       ??_SQDockWindow@@6BQPaintDevice@@@ 10024a64     launchEditor.obj
 0002:00004a8c       ??_SQToolBar@@6BQObject@@@ 10024a8c     launchEditor.obj
 0002:00004ca8       ??_SQToolBar@@6BQPaintDevice@@@ 10024ca8     launchEditor.obj
 0002:00004ccc       ??_SQPopupMenu@@6BQObject@@@ 10024ccc     launchEditor.obj
 0002:00004eac       ??_SQPopupMenu@@6BQPaintDevice@@@ 10024eac     launchEditor.obj
 0002:00004ed0       ??_SQPopupMenu@@6B@        10024ed0     launchEditor.obj
 0002:00004ef0       ??_C@_04OOEBCMBF@FAIL?$AA@ 10024ef0     launchEditor.obj
 0002:00004ef8       ??_C@_08OBALAKLA@READONLY?$AA@ 10024ef8     launchEditor.obj
 0002:00004f04       ??_C@_04KANDKFIK@DONE?$AA@ 10024f04     launchEditor.obj
 0002:00004f0c       ??_C@_07NFANNNEC@UNKNOWN?$AA@ 10024f0c     launchEditor.obj
 0002:00004f18       ??_7?$QDict@VQAction@@@@6B@ 10024f18     launchEditor.obj
 0002:00004f38       ??_7launchEditor@@6BQObject@@@ 10024f38     launchEditor.obj
 0002:00005110       ??_7launchEditor@@6BQPaintDevice@@@ 10025110     launchEditor.obj
 0002:00005130       ??_C@_0BE@FGANMCM@launchEditor?5path?5?3?$AA@ 10025130     launchEditor.obj
 0002:00005144       ??_C@_0BN@CEGLABJP@2command?$CI?5QString?0?5QString?5?$CJ?$AA@ 10025144     launchEditor.obj
 0002:00005164       ??_C@_0CH@MBKFDLDG@1workstationChanged?$CI?5QListViewIt@ 10025164     launchEditor.obj
 0002:0000518c       ??_C@_0CF@LFIPBHPN@2selectionChanged?$CI?5QListViewItem@ 1002518c     launchEditor.obj
 0002:000051b4       ??_C@_0BJ@JFJEEGDE@Launch?3?5Workstation?5List?$AA@ 100251b4     launchEditor.obj
 0002:000051d0       ??_C@_0M@HBIGLMLB@?1dockwindow?$AA@ 100251d0     launchEditor.obj
 0002:000051dc       ??_C@_0BG@KNDADLCE@Launch?5Editor?5Toolbar?$AA@ 100251dc     launchEditor.obj
 0002:000051f4       ??_C@_09DBJAPGHN@?1textedit?$AA@ 100251f4     launchEditor.obj
 0002:00005200       ??_C@_05LHMKEDEH@?$CGEdit?$AA@ 10025200     launchEditor.obj
 0002:00005208       ??_C@_03CLCAEGCJ@new?$AA@  10025208     launchEditor.obj
 0002:0000520c       ??_C@_04CCPFBLLC@?$CGNew?$AA@ 1002520c     launchEditor.obj
 0002:00005214       ??_C@_07EJAINBEK@filenew?$AA@ 10025214     launchEditor.obj
 0002:0000521c       ??_C@_0BA@NPMEGAC@New?5Application?$AA@ 1002521c     launchEditor.obj
 0002:0000522c       ??_C@_06FOBLBEIN@delete?$AA@ 1002522c     launchEditor.obj
 0002:00005234       ??_C@_07FGPBEGNH@?$CGDelete?$AA@ 10025234     launchEditor.obj
 0002:0000523c       ??_C@_0L@BPDPNFLB@filedelete?$AA@ 1002523c     launchEditor.obj
 0002:00005248       ??_C@_0BI@EGHAAPIP@Delete?5this?5application?$AA@ 10025248     launchEditor.obj
 0002:00005260       ??_C@_09KHIKJOBP@duplicate?$AA@ 10025260     launchEditor.obj
 0002:0000526c       ??_C@_0L@NDFJPKHF@D?$CGuplicate?$AA@ 1002526c     launchEditor.obj
 0002:00005278       ??_C@_0BL@KBLECFCO@Duplicate?5this?5application?$AA@ 10025278     launchEditor.obj
 0002:00005294       ??_C@_08GHAJENCO@1doAdd?$CI?$CJ?$AA@ 10025294     launchEditor.obj
 0002:000052a0       ??_C@_0N@KCMOKDBB@2activated?$CI?$CJ?$AA@ 100252a0     launchEditor.obj
 0002:000052b0       ??_C@_0M@BEFJDENE@1doRemove?$CI?$CJ?$AA@ 100252b0     launchEditor.obj
 0002:000052bc       ??_C@_0P@NFGMPEPE@1doDuplicate?$CI?$CJ?$AA@ 100252bc     launchEditor.obj
 0002:000052cc       ??_C@_0BJ@JHKFOCPP@deleting?5launch?5editMenu?$AA@ 100252cc     launchEditor.obj
 0002:000052e8       ??_C@_0BM@NAHHCEIA@deleting?5launch?5editToolbar?$AA@ 100252e8     launchEditor.obj
 0002:00005304       ??_C@_0BD@JGGFMPPB@deleting?5launch?5dw?$AA@ 10025304     launchEditor.obj
 0002:00005318       ??_C@_0EO@BDJLLDEB@Error?5for?5Dave?5?9?5you?5should?5neve@ 10025318     launchEditor.obj
 0002:00005368       ??_C@_0BC@HOBNKCKD@config?1launch?4xml?$AA@ 10025368     launchEditor.obj
 0002:0000537c       ??_C@_09JLEOPMAJ@?5?9?5error?$DN?$AA@ 1002537c     launchEditor.obj
 0002:00005388       ??_C@_09LBCHCBIC@?5?9?5value?$DN?$AA@ 10025388     launchEditor.obj
 0002:00005394       ??_C@_0P@ELNNACEA@?5?9?5textStatus?$DN?$AA@ 10025394     launchEditor.obj
 0002:000053a4       ??_C@_0L@LEAPMKGP@Reply?3?5op?$DN?$AA@ 100253a4     launchEditor.obj
 0002:000053b0       ??_C@_08HNIAHLMM@download?$AA@ 100253b0     launchEditor.obj
 0002:000053bc       ??_C@_0BI@MKHAAPOD@config?1workstations?4xml?$AA@ 100253bc     launchEditor.obj
 0002:000053d4       ??_C@_0BJ@NCALOKIP@?1config?1workstations?4xml?$AA@ 100253d4     launchEditor.obj
 0002:000053f0       ??_C@_0M@EBFEGAAI@Information?$AA@ 100253f0     launchEditor.obj
 0002:000053fc       ??_C@_06KAOCKAGB@upload?$AA@ 100253fc     launchEditor.obj
 0002:00005404       ??_C@_0BJ@MGIODGMN@loading?5workstations?4xml?$AA@ 10025404     launchEditor.obj
 0002:00005420       ??_C@_0BE@DMJOLDEB@workstation?5changed?$AA@ 10025420     launchEditor.obj
 0002:00005434       ??_C@_0BC@KNLOBELB@not?5on?5valid?5item?$AA@ 10025434     launchEditor.obj
 0002:00005448       ??_C@_0BG@JNFOLMDK@launch?5file?5not?5valid?$AA@ 10025448     launchEditor.obj
 0002:00005460       ??_C@_0BK@JKBCIGDB@System?1Workstations?0stuff?$AA@ 10025460     launchEditor.obj
 0002:00005480       ??_C@_0EG@BDBKIPFO@?$DMh3?$DOWorkstation?5Application?5Laun@ 10025480     launchEditor.obj
 0002:000054c8       ??_C@_08DIGPJJFJ@13?324?334?$AA@ 100254c8     launchEditor.obj
 0002:000054d4       ??_C@_0M@JEDEHNP@Sep?523?52021?$AA@ 100254d4     launchEditor.obj
 0002:000054e0       ??_C@_02PIGFKFFE@?$CF1?$AA@ 100254e0     launchEditor.obj
 0002:000054ec       ??_SQCheckTableItem@@6B@   100254ec     launcheditordlgimpl.obj
 0002:0000553c       ??_7launchEditorDlg@@6BQObject@@@ 1002553c     launcheditordlgimpl.obj
 0002:000056f4       ??_7launchEditorDlg@@6BQPaintDevice@@@ 100256f4     launcheditordlgimpl.obj
 0002:00005714       ??_C@_0BD@GOCBCOOF@1copyToClipboard?$CI?$CJ?$AA@ 10025714     launcheditordlgimpl.obj
 0002:00005728       ??_C@_0L@OELOHDKG@2clicked?$CI?$CJ?$AA@ 10025728     launcheditordlgimpl.obj
 0002:00005734       ??_C@_0BC@KJEEMEDF@1pasteClipboard?$CI?$CJ?$AA@ 10025734     launcheditordlgimpl.obj
 0002:00005748       ??_C@_02HNLLPFKA@up?$AA@   10025748     launcheditordlgimpl.obj
 0002:0000574c       ??_C@_04JMOKAGMG@down?$AA@ 1002574c     launcheditordlgimpl.obj
 0002:00005754       ??_C@_0M@NDAELMJH@1doMoveUp?$CI?$CJ?$AA@ 10025754     launcheditordlgimpl.obj
 0002:00005760       ??_C@_0O@BGGKHGH@1doMoveDown?$CI?$CJ?$AA@ 10025760     launcheditordlgimpl.obj
 0002:00005770       ??_C@_0BP@JLONLMNM@1tableValueChanged?$CI?5int?0?5int?5?$CJ?$AA@ 10025770     launcheditordlgimpl.obj
 0002:00005790       ??_C@_0BL@HPLODKLI@2valueChanged?5?$CI?5int?0?5int?5?$CJ?$AA@ 10025790     launcheditordlgimpl.obj
 0002:000057ac       ??_C@_0CE@DMGBMBGD@1csiValueChanged?$CI?5const?5QString?5@ 100257ac     launcheditordlgimpl.obj
 0002:000057d0       ??_C@_0CB@CBDIELKI@2textChanged?5?$CI?5const?5QString?5?$CG?5?$CJ@ 100257d0     launcheditordlgimpl.obj
 0002:000057f4       ??_C@_0BH@POPMNPEB@1rebootoptionchanged?$CI?$CJ?$AA@ 100257f4     launcheditordlgimpl.obj
 0002:0000580c       ??_C@_0M@LPGBGFJN@2clicked?5?$CI?$CJ?$AA@ 1002580c     launcheditordlgimpl.obj
 0002:00005818       ??_C@_0P@LBLEOAKD@trying?5to?5load?$AA@ 10025818     launcheditordlgimpl.obj
 0002:00005828       ??_C@_0M@FEGDHCCF@launch?5file?$AA@ 10025828     launcheditordlgimpl.obj
 0002:00005834       ??_C@_0BD@COFJDAMA@?2config?2launch?4xml?$AA@ 10025834     launcheditordlgimpl.obj
 0002:00005848       ??_C@_02EGCJHIOB@id?$AA@   10025848     launcheditordlgimpl.obj
 0002:0000584c       ??_C@_03BFKAHOOJ@csi?$AA@  1002584c     launcheditordlgimpl.obj
 0002:00005850       ??_C@_04LOAJBDKD@true?$AA@ 10025850     launcheditordlgimpl.obj
 0002:00005858       ??_C@_0O@BLEGCJOE@rebootoncrash?$AA@ 10025858     launcheditordlgimpl.obj
 0002:00005868       ??_C@_0L@NJNAEGOO@workingdir?$AA@ 10025868     launcheditordlgimpl.obj
 0002:00005874       ??_C@_09PBNAMLIK@arguments?$AA@ 10025874     launcheditordlgimpl.obj
 0002:00005880       ??_C@_05EKJCMADO@delay?$AA@ 10025880     launcheditordlgimpl.obj
 0002:00005888       ??_C@_0P@MHGKLOBA@restartoncrash?$AA@ 10025888     launcheditordlgimpl.obj
 0002:00005898       ??_C@_0CB@GGAKPEBL@can?8t?5read?5into?5DOM?5launch?5file?5@ 10025898     launcheditordlgimpl.obj
 0002:000058bc       ??_C@_0BI@OKPPDCEL@can?8t?5open?5launch?5file?5?$AA@ 100258bc     launcheditordlgimpl.obj
 0002:000058d4       ??_C@_0BM@CNFLJK@?$DN?$DN?$DN?$DN?$DN?$DN?$DN?$DNTable?5value?5changed?$AA@ 100258d4     launcheditordlgimpl.obj
 0002:000058f0       ??_C@_0M@DAIHPDMP@workstation?$AA@ 100258f0     launcheditordlgimpl.obj
 0002:000058fc       ??_C@_0M@MBDKLJIJ@application?$AA@ 100258fc     launcheditordlgimpl.obj
 0002:00005908       ??_C@_0CJ@IHPMIDJG@?4o?4o?$CDf?$CDA?$CDB?$CDC?$CDv?$CDk?4bQtQt?$CDD?4o?4m?$CDE?$CDB@ 10025908     plugindesc.obj
 0002:00005934       ??_C@_0CJ@NKMIADNK@?4o?$CDF?$CDG?$CDG?$CDG?$CDG?$CDG?40?4bQtQt?$CDD?4A?$CDG?$CDG?$CDG@ 10025934     plugindesc.obj
 0002:00005960       ??_C@_0CJ@FGNBBHNK@?$CDI?4h?$CDJ?$CDJ?$CDJ?$CDJ?$CDJ?4Y?$CDKQtQt?47?$CDN?$CDJ?$CDJ?$CDJ@ 10025960     plugindesc.obj
 0002:0000598c       ??_C@_0CJ@DCBNFDJK@?4a?$CDP?$CDQ?$CDQ?$CDR?$CDS?$CDS?$CDT?4pQtQt?$CDW?$CDX?$CDQ?$CDQ?$CDY@ 1002598c     plugindesc.obj
 0002:000059b8       ??_C@_0CJ@HENBALGI@?$CDr?$CD0?$CD1?$CD2?$CD3?$CD4?$CD4?4b?4pQtQt?4J?$CD5?$CD1?$CD6?$CD7@ 100259b8     plugindesc.obj
 0002:000059e4       ??_C@_0CJ@EMLENCNC@?$CDa?$CD4?$CD4?$CD4?$CD4?$CD4?$CD4?$CD4?$CD8QtQta?4?$CD4?$CD4?$CD4?$CD4@ 100259e4     plugindesc.obj
 0002:00005a10       ??_C@_0M@DCNCOAGB@20?520?5196?52?$AA@ 10025a10     plugindesc.obj
 0002:00005a1c       ??_C@_0N@EHHCJPCD@aM?5c?5?$CD0d0d06?$AA@ 10025a1c     plugindesc.obj
 0002:00005a2c       ??_C@_0N@GCGEIHOP@aF?5c?5?$CD1c1c01?$AA@ 10025a2c     plugindesc.obj
 0002:00005a3c       ??_C@_0N@JOHOGEIC@aW?5c?5?$CD232009?$AA@ 10025a3c     plugindesc.obj
 0002:00005a4c       ??_C@_0N@PFGPCACK@?$CDw?5c?5?$CD29290a?$AA@ 10025a4c     plugindesc.obj
 0002:00005a5c       ??_C@_0N@OAJCCIDI@?$CD5?5c?5?$CD464663?$AA@ 10025a5c     plugindesc.obj
 0002:00005a6c       ??_C@_0N@BEAILOKK@ap?5c?5?$CD50501e?$AA@ 10025a6c     plugindesc.obj
 0002:00005a7c       ??_C@_0N@OGBBFPGK@b?$CD?5c?5?$CD545449?$AA@ 10025a7c     plugindesc.obj
 0002:00005a8c       ??_C@_0N@LKJBINCC@aq?5c?5?$CD565600?$AA@ 10025a8c     plugindesc.obj
 0002:00005a9c       ??_C@_0N@DPAIFLGI@aw?5c?5?$CD5f5634?$AA@ 10025a9c     plugindesc.obj
 0002:00005aac       ??_C@_0N@HCFPEAFD@ae?5c?5?$CD62625a?$AA@ 10025aac     plugindesc.obj
 0002:00005abc       ??_C@_0N@LGLBLOHO@ax?5c?5?$CD646400?$AA@ 10025abc     plugindesc.obj
 0002:00005acc       ??_C@_0N@CMCIKGDI@?48?5c?5?$CD696925?$AA@ 10025acc     plugindesc.obj
 0002:00005adc       ??_C@_0N@MKADPPLN@a8?5c?5?$CD6b6904?$AA@ 10025adc     plugindesc.obj
 0002:00005aec       ??_C@_0N@FAMOPAOO@?$CDq?5c?5?$CD6d6a06?$AA@ 10025aec     plugindesc.obj
 0002:00005afc       ??_C@_0N@KAIBACEB@?4T?5c?5?$CD707041?$AA@ 10025afc     plugindesc.obj
 0002:00005b0c       ??_C@_0N@MDFEOMKE@?$CDu?5c?5?$CD717138?$AA@ 10025b0c     plugindesc.obj
 0002:00005b1c       ??_C@_0N@FGLEKGIP@?$CD4?5c?5?$CD778a94?$AA@ 10025b1c     plugindesc.obj
 0002:00005b2c       ??_C@_0N@OCNBCGKC@?$CDc?5c?5?$CD79775e?$AA@ 10025b2c     plugindesc.obj
 0002:00005b3c       ??_C@_0N@IAOAHLBM@?$CDL?5c?5?$CD7a8d95?$AA@ 10025b3c     plugindesc.obj
 0002:00005b4c       ??_C@_0N@LFLLLIGM@ba?5c?5?$CD808079?$AA@ 10025b4c     plugindesc.obj
 0002:00005b5c       ??_C@_0N@HENPEOCJ@?$CDN?5c?5?$CD87878c?$AA@ 10025b5c     plugindesc.obj
 0002:00005b6c       ??_C@_0N@NHHGIMPI@?$CDK?5c?5?$CD8d8b29?$AA@ 10025b6c     plugindesc.obj
 0002:00005b7c       ??_C@_0N@KMGPFGDD@?$CDp?5c?5?$CD8e7a5c?$AA@ 10025b7c     plugindesc.obj
 0002:00005b8c       ??_C@_0N@BAIFJPDO@?4h?5c?5?$CD8e8e94?$AA@ 10025b8c     plugindesc.obj
 0002:00005b9c       ??_C@_0N@PNJEBBII@?4b?5c?5?$CD919193?$AA@ 10025b9c     plugindesc.obj
 0002:00005bac       ??_C@_0N@LAPJFGIJ@?4F?5c?5?$CD919195?$AA@ 10025bac     plugindesc.obj
 0002:00005bbc       ??_C@_0N@KPCDOMOE@?46?5c?5?$CD927e52?$AA@ 10025bbc     plugindesc.obj
 0002:00005bcc       ??_C@_0N@KIFCMKNN@?4s?5c?5?$CD929295?$AA@ 10025bcc     plugindesc.obj
 0002:00005bdc       ??_C@_0N@PBDMMCEF@?$CDh?5c?5?$CD968061?$AA@ 10025bdc     plugindesc.obj
 0002:00005bec       ??_C@_0N@JJCJIKBD@?$CDf?5c?5?$CD968262?$AA@ 10025bec     plugindesc.obj
 0002:00005bfc       ??_C@_0N@BCFLDLB@?$CDj?5c?5?$CD978264?$AA@ 10025bfc     plugindesc.obj
 0002:00005c0c       ??_C@_0N@BDEEHAHO@?4a?5c?5?$CD9898bb?$AA@ 10025c0c     plugindesc.obj
 0002:00005c1c       ??_C@_0N@FOLNMEPO@?$CDo?5c?5?$CD999b94?$AA@ 10025c1c     plugindesc.obj
 0002:00005c2c       ??_C@_0N@HANGDLC@?$CDv?5c?5?$CD9f9f9d?$AA@ 10025c2c     plugindesc.obj
 0002:00005c3c       ??_C@_0N@LEDPNMBF@?$CDl?5c?5?$CDa08e74?$AA@ 10025c3c     plugindesc.obj
 0002:00005c4c       ??_C@_0N@ONHDOCJO@?$CD3?5c?5?$CDa6a355?$AA@ 10025c4c     plugindesc.obj
 0002:00005c5c       ??_C@_0N@BCDMEKLJ@?4n?5c?5?$CDa8a86b?$AA@ 10025c5c     plugindesc.obj
 0002:00005c6c       ??_C@_0N@LLONHBFG@?4E?5c?5?$CDababc3?$AA@ 10025c6c     plugindesc.obj
 0002:00005c7c       ??_C@_0N@LLMKPNAO@?$CDM?5c?5?$CDabadc7?$AA@ 10025c7c     plugindesc.obj
 0002:00005c8c       ??_C@_0N@GKFNCHHH@?4g?5c?5?$CDacacc5?$AA@ 10025c8c     plugindesc.obj
 0002:00005c9c       ??_C@_0N@IMANPDNA@aX?5c?5?$CDadad1b?$AA@ 10025c9c     plugindesc.obj
 0002:00005cac       ??_C@_0N@EFJPMAP@?4r?5c?5?$CDb1b1c9?$AA@ 10025cac     plugindesc.obj
 0002:00005cbc       ??_C@_0N@BDOMLGNI@?4S?5c?5?$CDb2b2c9?$AA@ 10025cbc     plugindesc.obj
 0002:00005ccc       ??_C@_0N@POFKHODM@b?4?5c?5?$CDb3b3a9?$AA@ 10025ccc     plugindesc.obj
 0002:00005cdc       ??_C@_0N@MCILNJLL@aE?5c?5?$CDb8b14a?$AA@ 10025cdc     plugindesc.obj
 0002:00005cec       ??_C@_0N@HBKCKLDA@?4U?5c?5?$CDb8b23c?$AA@ 10025cec     plugindesc.obj
 0002:00005cfc       ??_C@_0N@ELIJBPNO@?$CDk?5c?5?$CDb9c2ab?$AA@ 10025cfc     plugindesc.obj
 0002:00005d0c       ??_C@_0N@JABCLNBB@?$CDa?5c?5?$CDbaad2a?$AA@ 10025d0c     plugindesc.obj
 0002:00005d1c       ??_C@_0N@MAOCJJAB@?$CDi?5c?5?$CDbdc8b2?$AA@ 10025d1c     plugindesc.obj
 0002:00005d2c       ??_C@_0N@JECDGIF@?40?5c?5?$CDbea29a?$AA@ 10025d2c     plugindesc.obj
 0002:00005d3c       ??_C@_0N@DJKJAKHL@?42?5c?5?$CDbea39e?$AA@ 10025d3c     plugindesc.obj
 0002:00005d4c       ??_C@_0N@GELOHAEK@?4C?5c?5?$CDbfa39a?$AA@ 10025d4c     plugindesc.obj
 0002:00005d5c       ??_C@_0N@BKLBLNFI@?4N?5c?5?$CDbfa49d?$AA@ 10025d5c     plugindesc.obj
 0002:00005d6c       ??_C@_0N@HALAOCGL@?4m?5c?5?$CDbfb84d?$AA@ 10025d6c     plugindesc.obj
 0002:00005d7c       ??_C@_0N@CJMOLOPH@?4l?5c?5?$CDbfbc40?$AA@ 10025d7c     plugindesc.obj
 0002:00005d8c       ??_C@_0N@HGHLAELL@?4k?5c?5?$CDbfbc43?$AA@ 10025d8c     plugindesc.obj
 0002:00005d9c       ??_C@_0N@EGOBOKDA@?4V?5c?5?$CDbfbf3a?$AA@ 10025d9c     plugindesc.obj
 0002:00005dac       ??_C@_0N@IIOANKJO@aG?5c?5?$CDbfbf54?$AA@ 10025dac     plugindesc.obj
 0002:00005dbc       ??_C@_0N@OGJDPGMN@?$CDO?5c?5?$CDbfbf59?$AA@ 10025dbc     plugindesc.obj
 0002:00005dcc       ??_C@_0N@PEEAPOBK@?$CDx?5c?5?$CDbfbf5a?$AA@ 10025dcc     plugindesc.obj
 0002:00005ddc       ??_C@_0N@JNFPDNPL@?$CDg?5c?5?$CDbfcab5?$AA@ 10025ddc     plugindesc.obj
 0002:00005dec       ??_C@_0N@PDFFCKNG@?44?5c?5?$CDc2aaa6?$AA@ 10025dec     plugindesc.obj
 0002:00005dfc       ??_C@_0N@GPLLCAPM@?4e?5c?5?$CDc2c2d8?$AA@ 10025dfc     plugindesc.obj
 0002:00005e0c       ??_C@_0N@BFKBDNB@?$CDm?5c?5?$CDc2d6bd?$AA@ 10025e0c     plugindesc.obj
 0002:00005e1c       ??_C@_0N@FABNLLO@?4K?5c?5?$CDc3c0d2?$AA@ 10025e1c     plugindesc.obj
 0002:00005e2c       ??_C@_0N@BNAPDDM@?4A?5c?5?$CDc3c1d4?$AA@ 10025e2c     plugindesc.obj
 0002:00005e3c       ??_C@_0N@BDEAPCIN@?$CDd?5c?5?$CDc3d5bb?$AA@ 10025e3c     plugindesc.obj
 0002:00005e4c       ??_C@_0N@FNEHGFLH@?$CDn?5c?5?$CDc3d8bd?$AA@ 10025e4c     plugindesc.obj
 0002:00005e5c       ??_C@_0N@JKNAIBJB@?$CDe?5c?5?$CDc3dabd?$AA@ 10025e5c     plugindesc.obj
 0002:00005e6c       ??_C@_0N@KKKIIDOO@a7?5c?5?$CDc5b141?$AA@ 10025e6c     plugindesc.obj
 0002:00005e7c       ??_C@_0N@LOGPFING@a6?5c?5?$CDc5b541?$AA@ 10025e7c     plugindesc.obj
 0002:00005e8c       ??_C@_0N@GDPIECKN@a5?5c?5?$CDc5b741?$AA@ 10025e8c     plugindesc.obj
 0002:00005e9c       ??_C@_0N@KDDICFOL@a0?5c?5?$CDc5b841?$AA@ 10025e9c     plugindesc.obj
 0002:00005eac       ??_C@_0N@GMBKJAHO@a3?5c?5?$CDc5b941?$AA@ 10025eac     plugindesc.obj
 0002:00005ebc       ??_C@_0N@IOJICJKM@a1?5c?5?$CDc5ba41?$AA@ 10025ebc     plugindesc.obj
 0002:00005ecc       ??_C@_0N@MFONEOEE@aZ?5c?5?$CDc5bb41?$AA@ 10025ecc     plugindesc.obj
 0002:00005edc       ??_C@_0N@MKJAJINK@?4X?5c?5?$CDc5bc1d?$AA@ 10025edc     plugindesc.obj
 0002:00005eec       ??_C@_0N@NEGPGHEP@?4H?5c?5?$CDc5c10c?$AA@ 10025eec     plugindesc.obj
 0002:00005efc       ??_C@_0N@EEBOLKKG@aY?5c?5?$CDc5c241?$AA@ 10025efc     plugindesc.obj
 0002:00005f0c       ??_C@_0N@KFGCBFMF@a2?5c?5?$CDc5c341?$AA@ 10025f0c     plugindesc.obj
 0002:00005f1c       ??_C@_0N@NHIIIIJM@a4?5c?5?$CDc5c441?$AA@ 10025f1c     plugindesc.obj
 0002:00005f2c       ??_C@_0N@HPHNGLCI@az?5c?5?$CDc5c559?$AA@ 10025f2c     plugindesc.obj
 0002:00005f3c       ??_C@_0N@EPNJPMLP@aN?5c?5?$CDc9c978?$AA@ 10025f3c     plugindesc.obj
 0002:00005f4c       ??_C@_0N@IOCKFDPM@?$CD6?5c?5?$CDcaca61?$AA@ 10025f4c     plugindesc.obj
 0002:00005f5c       ??_C@_0N@HIPKBLNJ@?4j?5c?5?$CDcaca6c?$AA@ 10025f5c     plugindesc.obj
 0002:00005f6c       ??_C@_0N@HBHCFOKN@?$CDs?5c?5?$CDcaca77?$AA@ 10025f6c     plugindesc.obj
 0002:00005f7c       ??_C@_0N@BFHPAOEL@?4v?5c?5?$CDcdcd4c?$AA@ 10025f7c     plugindesc.obj
 0002:00005f8c       ??_C@_0N@HBDKIIDI@?49?5c?5?$CDcdcdcd?$AA@ 10025f8c     plugindesc.obj
 0002:00005f9c       ??_C@_0N@HHHJJDMD@?$CDb?5c?5?$CDd0b163?$AA@ 10025f9c     plugindesc.obj
 0002:00005fac       ??_C@_0N@FCNHGHFB@ad?5c?5?$CDd2b078?$AA@ 10025fac     plugindesc.obj
 0002:00005fbc       ??_C@_0N@MADOKJMH@?4P?5c?5?$CDd2bbad?$AA@ 10025fbc     plugindesc.obj
 0002:00005fcc       ??_C@_0N@NLGLODGF@?4z?5c?5?$CDd5b19c?$AA@ 10025fcc     plugindesc.obj
 0002:00005fdc       ??_C@_0N@GEGHNJC@?4J?5c?5?$CDd7b69b?$AA@ 10025fdc     plugindesc.obj
 0002:00005fec       ??_C@_0N@FAOGPLPG@?4d?5c?5?$CDd7d7e5?$AA@ 10025fec     plugindesc.obj
 0002:00005ffc       ??_C@_0N@DPDAPGEK@?4?$CD?5c?5?$CDd7d7e6?$AA@ 10025ffc     plugindesc.obj
 0002:0000600c       ??_C@_0N@DLKAPJPB@?$CDt?5c?5?$CDd8d89c?$AA@ 1002600c     plugindesc.obj
 0002:0000601c       ??_C@_0N@FAHIGJCH@?4W?5c?5?$CDdadad3?$AA@ 1002601c     plugindesc.obj
 0002:0000602c       ??_C@_0N@NCDOBMAJ@?4O?5c?5?$CDdbd0d6?$AA@ 1002602c     plugindesc.obj
 0002:0000603c       ??_C@_0N@JIKCNOLO@af?5c?5?$CDdbdba4?$AA@ 1002603c     plugindesc.obj
 0002:0000604c       ??_C@_0N@EFFFPHJM@?43?5c?5?$CDdcd0d3?$AA@ 1002604c     plugindesc.obj
 0002:0000605c       ??_C@_0N@HFLOMLGC@?41?5c?5?$CDdcd1d7?$AA@ 1002605c     plugindesc.obj
 0002:0000606c       ??_C@_0N@CHFIKHNM@aO?5c?5?$CDdcdc97?$AA@ 1002606c     plugindesc.obj
 0002:0000607c       ??_C@_0N@CJNHDMHD@?$CD?$CD?5c?5?$CDe0e0b1?$AA@ 1002607c     plugindesc.obj
 0002:0000608c       ??_C@_0N@MLBAPKLB@aL?5c?5?$CDe2d87a?$AA@ 1002608c     plugindesc.obj
 0002:0000609c       ??_C@_0N@BHLHJEM@ar?5c?5?$CDe2e26e?$AA@ 1002609c     plugindesc.obj
 0002:000060ac       ??_C@_0N@CCOEEDMF@ag?5c?5?$CDe2e2a1?$AA@ 100260ac     plugindesc.obj
 0002:000060bc       ??_C@_0N@MIIBCGOO@?45?5c?5?$CDeaf5ff?$AA@ 100260bc     plugindesc.obj
 0002:000060cc       ??_C@_0N@BDMDFABA@?4Z?5c?5?$CDeee7e1?$AA@ 100260cc     plugindesc.obj
 0002:000060dc       ??_C@_0N@PIOKCMLO@?4B?5c?5?$CDefe6de?$AA@ 100260dc     plugindesc.obj
 0002:000060ec       ??_C@_0N@DIFDHMMP@ao?5c?5?$CDf0cf89?$AA@ 100260ec     plugindesc.obj
 0002:000060fc       ??_C@_0N@FHIMFOFN@?4Y?5c?5?$CDf0faff?$AA@ 100260fc     plugindesc.obj
 0002:0000610c       ??_C@_0N@NKINOMFI@?4Q?5c?5?$CDf2ebe5?$AA@ 1002610c     plugindesc.obj
 0002:0000611c       ??_C@_0N@ILFCKLCG@?4M?5c?5?$CDf3ece6?$AA@ 1002611c     plugindesc.obj
 0002:0000612c       ??_C@_0N@LOIMCAL@?4w?5c?5?$CDf3f03d?$AA@ 1002612c     plugindesc.obj
 0002:0000613c       ??_C@_0N@PENAILCG@?$CD7?5c?5?$CDf3f3a3?$AA@ 1002613c     plugindesc.obj
 0002:0000614c       ??_C@_0N@PFDGINFC@?$CD?4?5c?5?$CDf5f5e7?$AA@ 1002614c     plugindesc.obj
 0002:0000615c       ??_C@_0N@ONIFCALO@?4p?5c?5?$CDf6f2ed?$AA@ 1002615c     plugindesc.obj
 0002:0000616c       ??_C@_0N@EDPNOBKF@av?5c?5?$CDf8df94?$AA@ 1002616c     plugindesc.obj
 0002:0000617c       ??_C@_0N@LPGGNPKF@ay?5c?5?$CDf8f8ed?$AA@ 1002617c     plugindesc.obj
 0002:0000618c       ??_C@_0N@MBJIEPGA@?4G?5c?5?$CDf8f8ee?$AA@ 1002618c     plugindesc.obj
 0002:0000619c       ??_C@_0N@KPHMDGNE@?4t?5c?5?$CDf8f8f8?$AA@ 1002619c     plugindesc.obj
 0002:000061ac       ??_C@_0N@JPOJNFEP@?4i?5c?5?$CDf9f9f1?$AA@ 100261ac     plugindesc.obj
 0002:000061bc       ??_C@_0N@BJFNDBJ@bb?5c?5?$CDf9f9f9?$AA@ 100261bc     plugindesc.obj
 0002:000061cc       ??_C@_0N@CBABMNKN@?4c?5c?5?$CDfafafa?$AA@ 100261cc     plugindesc.obj
 0002:000061dc       ??_C@_0N@IOGDCIAJ@?4q?5c?5?$CDfafaff?$AA@ 100261dc     plugindesc.obj
 0002:000061ec       ??_C@_0N@DDJCBCHB@aV?5c?5?$CDfbd097?$AA@ 100261ec     plugindesc.obj
 0002:000061fc       ??_C@_0N@KDPPJDGC@?4u?5c?5?$CDfbfbf6?$AA@ 100261fc     plugindesc.obj
 0002:0000620c       ??_C@_0N@HFONPMEB@?4R?5c?5?$CDfbfbff?$AA@ 1002620c     plugindesc.obj
 0002:0000621c       ??_C@_0N@NBBCBEOB@?4L?5c?5?$CDfcfcfd?$AA@ 1002621c     plugindesc.obj
 0002:0000622c       ??_C@_0N@OFCIAAJN@?4D?5c?5?$CDfcfcff?$AA@ 1002622c     plugindesc.obj
 0002:0000623c       ??_C@_0N@CHHECEKJ@?4o?5c?5?$CDfdfdfe?$AA@ 1002623c     plugindesc.obj
 0002:0000624c       ??_C@_0N@EDEBKFK@a9?5c?5?$CDfefefd?$AA@ 1002624c     plugindesc.obj
 0002:0000625c       ??_C@_0N@OCBAPJDL@?4f?5c?5?$CDfefeff?$AA@ 1002625c     plugindesc.obj
 0002:0000626c       ??_C@_0N@BEKBKMH@aU?5c?5?$CDffd09c?$AA@ 1002626c     plugindesc.obj
 0002:0000627c       ??_C@_0N@CCFDDBMN@aT?5c?5?$CDffd19c?$AA@ 1002627c     plugindesc.obj
 0002:0000628c       ??_C@_0N@KMGKFDAE@aR?5c?5?$CDffdc9c?$AA@ 1002628c     plugindesc.obj
 0002:0000629c       ??_C@_0N@JBKADIDE@aJ?5c?5?$CDffdf9c?$AA@ 1002629c     plugindesc.obj
 0002:000062ac       ??_C@_0N@BOEOBDO@?4y?5c?5?$CDffe25b?$AA@ 100262ac     plugindesc.obj
 0002:000062bc       ??_C@_0N@CHINDMOE@aI?5c?5?$CDffe39c?$AA@ 100262bc     plugindesc.obj
 0002:000062cc       ??_C@_0N@CEPFAFLD@aD?5c?5?$CDffe49c?$AA@ 100262cc     plugindesc.obj
 0002:000062dc       ??_C@_0N@PMPILNFN@as?5c?5?$CDffe59c?$AA@ 100262dc     plugindesc.obj
 0002:000062ec       ??_C@_0N@ECLLPHLH@?4x?5c?5?$CDffe64d?$AA@ 100262ec     plugindesc.obj
 0002:000062fc       ??_C@_0N@NECMLMJN@?4I?5c?5?$CDffe64e?$AA@ 100262fc     plugindesc.obj
 0002:0000630c       ??_C@_0N@OCFFPPEP@ac?5c?5?$CDffe69c?$AA@ 1002630c     plugindesc.obj
 0002:0000631c       ??_C@_0N@CLFAFABM@?$CDH?5c?5?$CDffe69f?$AA@ 1002631c     plugindesc.obj
 0002:0000632c       ??_C@_0N@EENEDFCM@aK?5c?5?$CDffe79c?$AA@ 1002632c     plugindesc.obj
 0002:0000633c       ??_C@_0N@HPNHKJOG@?$CDJ?5c?5?$CDffe79f?$AA@ 1002633c     plugindesc.obj
 0002:0000634c       ??_C@_0N@OBKPMAGA@au?5c?5?$CDffe89c?$AA@ 1002634c     plugindesc.obj
 0002:0000635c       ??_C@_0N@LOBOBBDI@aS?5c?5?$CDffe95b?$AA@ 1002635c     plugindesc.obj
 0002:0000636c       ??_C@_0N@CEJJOOPH@an?5c?5?$CDffe99c?$AA@ 1002636c     plugindesc.obj
 0002:0000637c       ??_C@_0N@MPBGFENF@a?$CD?5c?5?$CDffeb98?$AA@ 1002637c     plugindesc.obj
 0002:0000638c       ??_C@_0N@DLJDFNCL@aj?5c?5?$CDffeb9c?$AA@ 1002638c     plugindesc.obj
 0002:0000639c       ??_C@_0N@IGAOBLPH@?$CDF?5c?5?$CDffeb9f?$AA@ 1002639c     plugindesc.obj
 0002:000063ac       ??_C@_0N@BDJIKMDF@?$CDZ?5c?5?$CDffec98?$AA@ 100263ac     plugindesc.obj
 0002:000063bc       ??_C@_0N@PBMFKHBH@al?5c?5?$CDffed9c?$AA@ 100263bc     plugindesc.obj
 0002:000063cc       ??_C@_0N@FCEOCAPF@aH?5c?5?$CDffee9c?$AA@ 100263cc     plugindesc.obj
 0002:000063dc       ??_C@_0N@LCLDCBKL@?$CDS?5c?5?$CDffef68?$AA@ 100263dc     plugindesc.obj
 0002:000063ec       ??_C@_0N@NNFCLFIK@aA?5c?5?$CDffef9c?$AA@ 100263ec     plugindesc.obj
 0002:000063fc       ??_C@_0N@IGJCKMLN@ak?5c?5?$CDfff09c?$AA@ 100263fc     plugindesc.obj
 0002:0000640c       ??_C@_0N@DCFEBAKC@aC?5c?5?$CDfff16b?$AA@ 1002640c     plugindesc.obj
 0002:0000641c       ??_C@_0N@KDIHPBEJ@ab?5c?5?$CDfff19c?$AA@ 1002641c     plugindesc.obj
 0002:0000642c       ??_C@_0N@IDLDINAE@?$CDG?5c?5?$CDfff19f?$AA@ 1002642c     plugindesc.obj
 0002:0000643c       ??_C@_0N@JJOMNCLF@aa?5c?5?$CDfff25e?$AA@ 1002643c     plugindesc.obj
 0002:0000644c       ??_C@_0N@FABHGMNC@?$CDY?5c?5?$CDfff298?$AA@ 1002644c     plugindesc.obj
 0002:0000645c       ??_C@_0N@IEFLKENG@a?4?5c?5?$CDfff29c?$AA@ 1002645c     plugindesc.obj
 0002:0000646c       ??_C@_0N@DPHDMDBD@?47?5c?5?$CDfff34c?$AA@ 1002646c     plugindesc.obj
 0002:0000647c       ??_C@_0N@GKDJNNDG@aQ?5c?5?$CDfff39c?$AA@ 1002647c     plugindesc.obj
 0002:0000648c       ??_C@_0N@JELBIBPF@aB?5c?5?$CDfff48b?$AA@ 1002648c     plugindesc.obj
 0002:0000649c       ??_C@_0N@FOKHCIOA@?$CDV?5c?5?$CDfff49c?$AA@ 1002649c     plugindesc.obj
 0002:000064ac       ??_C@_0N@CMMOAKCG@?$CDB?5c?5?$CDfff49f?$AA@ 100264ac     plugindesc.obj
 0002:000064bc       ??_C@_0N@HNLOADOK@?$CDW?5c?5?$CDfff59c?$AA@ 100264bc     plugindesc.obj
 0002:000064cc       ??_C@_0N@PNHCBCM@?$CDC?5c?5?$CDfff59f?$AA@ 100264cc     plugindesc.obj
 0002:000064dc       ??_C@_0N@NPPKLHBM@?$CD2?5c?5?$CDfff69c?$AA@ 100264dc     plugindesc.obj
 0002:000064ec       ??_C@_0N@PHFFGGKD@?$CDI?5c?5?$CDfff69f?$AA@ 100264ec     plugindesc.obj
 0002:000064fc       ??_C@_0N@JLGPGKCH@at?5c?5?$CDfff764?$AA@ 100264fc     plugindesc.obj
 0002:0000650c       ??_C@_0N@ILHNEOOG@?$CD0?5c?5?$CDfff79c?$AA@ 1002650c     plugindesc.obj
 0002:0000651c       ??_C@_0N@OEFLHFAH@?$CDX?5c?5?$CDfff89b?$AA@ 1002651c     plugindesc.obj
 0002:0000652c       ??_C@_0N@EOLHGECB@?$CD9?5c?5?$CDfff89c?$AA@ 1002652c     plugindesc.obj
 0002:0000653c       ??_C@_0N@BCIAFMBB@?$CDE?5c?5?$CDfff89f?$AA@ 1002653c     plugindesc.obj
 0002:0000654c       ??_C@_0N@LHAHCKMC@am?5c?5?$CDfff992?$AA@ 1002654c     plugindesc.obj
 0002:0000655c       ??_C@_0N@EAPGGOKC@?$CDT?5c?5?$CDfff99c?$AA@ 1002655c     plugindesc.obj
 0002:0000656c       ??_C@_0N@DBJJHHBL@?$CDD?5c?5?$CDfff99f?$AA@ 1002656c     plugindesc.obj
 0002:0000657c       ??_C@_0N@ICLNBGIK@ah?5c?5?$CDfffa9c?$AA@ 1002657c     plugindesc.obj
 0002:0000658c       ??_C@_0N@OMALPNBJ@?$CD1?5c?5?$CDfffb9c?$AA@ 1002658c     plugindesc.obj
 0002:0000659c       ??_C@_0N@DKJBJOPL@aP?5c?5?$CDfffc9c?$AA@ 1002659c     plugindesc.obj
 0002:000065ac       ??_C@_0N@DOMHGCPC@ai?5c?5?$CDfffd5b?$AA@ 100265ac     plugindesc.obj
 0002:000065bc       ??_C@_0N@BIGDLFFI@?$CDA?5c?5?$CDffff5e?$AA@ 100265bc     plugindesc.obj
 0002:000065cc       ??_C@_0N@MIOKHOKN@?$CDQ?5c?5?$CDffff61?$AA@ 100265cc     plugindesc.obj
 0002:000065dc       ??_C@_0N@BKELGEG@?$CD8?5c?5?$CDffff74?$AA@ 100265dc     plugindesc.obj
 0002:000065ec       ??_C@_0N@EABAEKME@?$CDR?5c?5?$CDffff8f?$AA@ 100265ec     plugindesc.obj
 0002:000065fc       ??_C@_0N@EIDNDNDJ@?$CDU?5c?5?$CDffff9c?$AA@ 100265fc     plugindesc.obj
 0002:0000660c       ??_C@_0N@FPOPINPF@?$CDz?5c?5?$CDffff9f?$AA@ 1002660c     plugindesc.obj
 0002:0000661c       ??_C@_0N@DIPKLEKO@?$CDP?5c?5?$CDffffb1?$AA@ 1002661c     plugindesc.obj
 0002:0000662c       ??_C@_0N@HNJAIJD@?$CDy?5c?5?$CDffffba?$AA@ 1002662c     plugindesc.obj
 0002:0000663c       ??_C@_0CJ@JOJFFMDD@QtQtQtQtQtQtQtQtQtQtQtQtQtQtQtQt@ 1002663c     plugindesc.obj
 0002:00006668       ??_C@_0CJ@OFFKCBGA@QtQtQtQtQtQtQtQtQt?4?$CD?4a?4b?4cQtQtQt@ 10026668     plugindesc.obj
 0002:00006694       ??_C@_0CJ@MMKEFGIH@QtQtQtQtQtQtQtQt?4d?4e?4f?4g?4hQtQtQt@ 10026694     plugindesc.obj
 0002:000066c0       ??_C@_0CJ@BHLGMJOA@QtQt?4i?4j?4k?4l?4m?4n?4e?4o?4p?4q?4r?4s?4tQt@ 100266c0     plugindesc.obj
 0002:000066ec       ??_C@_0CJ@EIOGDHKO@Qt?4u?4v?4w?4x?4y?4z?4AQt?4B?4CQt?4D?4E?4FQt@ 100266ec     plugindesc.obj
 0002:00006718       ??_C@_0CJ@IEPHEIFJ@Qt?4G?4H?4I?4y?4J?4K?4L?4M?4N?4O?4P?4Q?4R?4S?4T@ 10026718     plugindesc.obj
 0002:00006744       ??_C@_0CJ@GCBMIKMF@Qt?4G?4X?4y?4z?4K?4Y?4Z?40?41?42?43?44Qt?45?4E@ 10026744     plugindesc.obj
 0002:00006770       ??_C@_0CJ@BLNHNCGJ@?$CD?4?$CD?$CD?$CDa?$CDb?$CDc?$CDd?$CDe?$CDf?$CDg?$CDh?$CDi?$CDj?$CDk?$CDl?$CDm?$CDn@ 10026770     plugindesc.obj
 0002:0000679c       ??_C@_0CJ@NNGJMAIM@?$CDs?$CDt?$CDt?$CDt?$CDt?$CDt?$CDt?$CDt?$CDt?$CDt?$CDt?$CDt?$CDt?$CDt?$CDt?$CDt@ 1002679c     plugindesc.obj
 0002:000067c8       ??_C@_0CJ@IAMGFBLP@?$CDx?$CDy?$CDz?$CDA?$CDz?$CDz?$CDz?$CDB?$CDC?$CDD?$CDE?$CDF?$CDG?$CDH?$CDI?$CDJ@ 100267c8     plugindesc.obj
 0002:000067f4       ??_C@_0CJ@CAMPKIIN@?$CDO?$CDP?$CDQ?$CDR?$CDS?$CDT?$CDU?$CDV?$CDW?$CDT?$CDX?$CDY?$CDZ?$CD0?$CD1?$CD2@ 100267f4     plugindesc.obj
 0002:00006820       ??_C@_0CJ@LHBEMEEF@?$CD6?$CD7?$CDU?$CD8?$CDU?$CDU?$CDV?$CD9?$CD0a?4a?$CD?$CDQaaab?$CDVac@ 10026820     plugindesc.obj
 0002:0000684c       ??_C@_0CJ@CDMMIPAB@afag?$CDQ?$CD8?$CDS?$CDT?$CD9ah?$CD0?$CD2aiajakalaman@ 1002684c     plugindesc.obj
 0002:00006878       ??_C@_0CJ@JAPDGGLH@afar?$CDU?$CDU?$CDU?$CDUa?4?$CD0as?$CD2?$CD0?$CDUal?$CDWatau@ 10026878     plugindesc.obj
 0002:000068a4       ??_C@_0CJ@IDJILFIC@ayaz?$CDU?$CDUaA?$CDT?$CDW?$CD9?$CD9?$CD2?$CDWauasasaBaC@ 100268a4     plugindesc.obj
 0002:000068d0       ??_C@_0CJ@LGCGMEPH@QtaG?$CDU?$CD1abaHaDaIacaHaJ?$CDWacacaKac@ 100268d0     plugindesc.obj
 0002:000068fc       ??_C@_0CJ@KCMFFCGA@QtaNaOaP?$CD2aQ?$CDW?$CDT?$CDV?$CDVanajaRaKaSaT@ 100268fc     plugindesc.obj
 0002:00006928       ??_C@_0CJ@IGAPHAKL@Qt?4GaXaYaZa0a1a2a3a4a5a3a2a1a6a7@ 10026928     plugindesc.obj
 0002:00006954       ??_C@_0CJ@MABFKAAG@Qta9b?4b?$CDb?$CDb?$CDb?$CDb?$CDb?$CDb?$CDb?$CDb?$CDb?$CDb?$CDb?$CDb?$CD@ 10026954     plugindesc.obj
 0002:00006980       ??_C@_09MGBDHDNN@18?520?58?51?$AA@ 10026980     plugindesc.obj
 0002:0000698c       ??_C@_0M@DMOCGNBA@c?5c?5?$CD840000?$AA@ 1002698c     plugindesc.obj
 0002:00006998       ??_C@_0M@HCCKGJFF@b?5c?5?$CD848484?$AA@ 10026998     plugindesc.obj
 0002:000069a4       ??_C@_0M@NNLNAJBO@e?5c?5?$CDc6c6c6?$AA@ 100269a4     plugindesc.obj
 0002:000069b0       ??_C@_0M@HKNGLPIJ@d?5c?5?$CDff0000?$AA@ 100269b0     plugindesc.obj
 0002:000069bc       ??_C@_0BD@OGGPOPDG@?4?$CDab?4?4?4cccd?4?4?4?$CDab?4?$AA@ 100269bc     plugindesc.obj
 0002:000069d0       ??_C@_0BD@PEMCIFLL@?$CDeffb?4cccdcd?4bfffb?$AA@ 100269d0     plugindesc.obj
 0002:000069e4       ??_C@_0BD@MPBCDHIE@?$CDeffbccc?$CD?$CDdcdbfff?$CD?$AA@ 100269e4     plugindesc.obj
 0002:000069f8       ??_C@_0BD@DMEHEHDG@?$CDeff?$CDcc?$CD?$CD?$CD?$CDddbfff?$CD?$AA@ 100269f8     plugindesc.obj
 0002:00006a0c       ??_C@_0BD@IIKINBDI@?$CDebfbcc?$CDef?$CDddbbfb?$CD?$AA@ 10026a0c     plugindesc.obj
 0002:00006a20       ??_C@_0BD@EPNPGGOF@?$CDeff?$CDc?$CDb?$CD?$CDb?$CDdbfbf?$CD?$AA@ 10026a20     plugindesc.obj
 0002:00006a34       ??_C@_0BD@NBJCLNPM@?$CDeffbc?$CD?$CD?$CD?$CD?$CD?$CDdbfff?$CD?$AA@ 10026a34     plugindesc.obj
 0002:00006a48       ??_C@_0BD@IPHHODIA@?$CDeff?$CDc?$CDebbf?$CDdbfff?$CD?$AA@ 10026a48     plugindesc.obj
 0002:00006a5c       ??_C@_0BD@NMKHPGOM@?$CDeffbc?$CDeeff?$CDdbfff?$CD?$AA@ 10026a5c     plugindesc.obj
 0002:00006a70       ??_C@_0BD@FNCOFIGF@?$CDeff?$CDc?$CDeeff?$CDdbbfb?$CD?$AA@ 10026a70     plugindesc.obj
 0002:00006a84       ??_C@_0BD@BFNKIHMN@?$CDbfb?$CDc?$CDeeff?$CDdbfbf?$CD?$AA@ 10026a84     plugindesc.obj
 0002:00006a98       ??_C@_0BD@BMLCEKOK@?$CDeffb?$CD?$CDeeff?$CD?$CDbfff?$CD?$AA@ 10026a98     plugindesc.obj
 0002:00006aac       ??_C@_0BD@ONNICMPO@?$CDeff?$CD?$CD?$CDe?$CD?$CDf?$CD?$CD?$CDfff?$CD?$AA@ 10026aac     plugindesc.obj
 0002:00006ac0       ??_C@_0BD@IGKEDGLC@?$CDef?$CD?$CDe?$CDe?$CD?$CDf?$CDf?$CD?$CDff?$CD?$AA@ 10026ac0     plugindesc.obj
 0002:00006ad4       ??_C@_0BD@DEBCCDJF@?$CDe?$CD?$CDee?$CDe?$CD?$CDf?$CDff?$CD?$CDf?$CD?$AA@ 10026ad4     plugindesc.obj
 0002:00006ae8       ??_C@_0BD@BLEOOIHM@?$CD?$CD?$CDeee?$CDe?$CD?$CDf?$CDfff?$CD?$CD?$CD?$AA@ 10026ae8     plugindesc.obj
 0002:00006afc       ??_C@_0BD@GMOLJMOA@?4?$CD?$CD?$CD?$CD?$CD?$CDe?$CD?$CDf?$CD?$CD?$CD?$CD?$CD?$CD?4?$AA@ 10026afc     plugindesc.obj
 0002:00006b10       ??_C@_0BD@NFMEDNCE@?$CD?$CDee?$CDe?$CD?$CD?$CD?$CD?$CD?$CDe?$CDee?$CD?$CD?$AA@ 10026b10     plugindesc.obj
 0002:00006b24       ??_C@_0BD@BBDKNHPP@?$CDee?$CDda?$CD?$CD?$CD?$CD?$CD?$CDad?$CDee?$CD?$AA@ 10026b24     plugindesc.obj
 0002:00006b38       ??_C@_0BD@HNGOLBFH@?4aacadacddcadacad?4?$AA@ 10026b38     plugindesc.obj
 0002:00006b4c       ??_C@_0M@FNAJKHBM@20?520?5130?52?$AA@ 10026b4c     plugindesc.obj
 0002:00006b58       ??_C@_0N@CGBFBHLL@?$CDo?5c?5?$CD000078?$AA@ 10026b58     plugindesc.obj
 0002:00006b68       ??_C@_0N@NADDIDBK@?$CDi?5c?5?$CD000079?$AA@ 10026b68     plugindesc.obj
 0002:00006b78       ??_C@_0N@HGLFIOOO@?$CDh?5c?5?$CD00007f?$AA@ 10026b78     plugindesc.obj
 0002:00006b88       ??_C@_0N@KIKDDBC@?$CDA?5c?5?$CD0000a5?$AA@ 10026b88     plugindesc.obj
 0002:00006b98       ??_C@_0N@OFGNPCLP@?$CDE?5c?5?$CD0000ac?$AA@ 10026b98     plugindesc.obj
 0002:00006ba8       ??_C@_0N@JNANJLCD@?$CDC?5c?5?$CD0000d0?$AA@ 10026ba8     plugindesc.obj
 0002:00006bb8       ??_C@_0N@HLNPCDAJ@?$CDB?5c?5?$CD0000d5?$AA@ 10026bb8     plugindesc.obj
 0002:00006bc8       ??_C@_0N@GAJHJBCI@?$CDy?5c?5?$CD0000f0?$AA@ 10026bc8     plugindesc.obj
 0002:00006bd8       ??_C@_0N@FHKLLOCL@?$CDu?5c?5?$CD0000f2?$AA@ 10026bd8     plugindesc.obj
 0002:00006be8       ??_C@_0N@BCNJGKBE@?$CDt?5c?5?$CD0000ff?$AA@ 10026be8     plugindesc.obj
 0002:00006bf8       ??_C@_0N@EDBOPBAA@?$CDs?5c?5?$CD0014c5?$AA@ 10026bf8     plugindesc.obj
 0002:00006c08       ??_C@_0N@JBCMDJBL@?$CDx?5c?5?$CD0014cd?$AA@ 10026c08     plugindesc.obj
 0002:00006c18       ??_C@_0N@LJNNKEAD@?$CDg?5c?5?$CD005262?$AA@ 10026c18     plugindesc.obj
 0002:00006c28       ??_C@_0N@EABIFLJG@?$CDn?5c?5?$CD005266?$AA@ 10026c28     plugindesc.obj
 0002:00006c38       ??_C@_0N@BEFKHAPK@?4u?5c?5?$CD00b6b6?$AA@ 10026c38     plugindesc.obj
 0002:00006c48       ??_C@_0N@IJELGBIK@?4r?5c?5?$CD00bdbd?$AA@ 10026c48     plugindesc.obj
 0002:00006c58       ??_C@_0N@BAOBFOID@?4q?5c?5?$CD00cccc?$AA@ 10026c58     plugindesc.obj
 0002:00006c68       ??_C@_0N@OOIOJDMA@?$CDZ?5c?5?$CD2e2e2e?$AA@ 10026c68     plugindesc.obj
 0002:00006c78       ??_C@_0N@LIJPCOKB@?$CD4?5c?5?$CD313131?$AA@ 10026c78     plugindesc.obj
 0002:00006c88       ??_C@_0N@JAPLKPLP@?4j?5c?5?$CD314949?$AA@ 10026c88     plugindesc.obj
 0002:00006c98       ??_C@_0N@NBBHIJCJ@?4i?5c?5?$CD314d4d?$AA@ 10026c98     plugindesc.obj
 0002:00006ca8       ??_C@_0N@BJCBMJFC@?4p?5c?5?$CD333333?$AA@ 10026ca8     plugindesc.obj
 0002:00006cb8       ??_C@_0N@JPNHJKA@?4s?5c?5?$CD33a6a6?$AA@ 10026cb8     plugindesc.obj
 0002:00006cc8       ??_C@_0N@ELDBGKOA@?$CD1?5c?5?$CD39d939?$AA@ 10026cc8     plugindesc.obj
 0002:00006cd8       ??_C@_0N@GNNHANNB@?$CDJ?5c?5?$CD404040?$AA@ 10026cd8     plugindesc.obj
 0002:00006ce8       ??_C@_0N@PFBIPNKP@?4R?5c?5?$CD424242?$AA@ 10026ce8     plugindesc.obj
 0002:00006cf8       ??_C@_0N@KLDKLEAE@?4K?5c?5?$CD454545?$AA@ 10026cf8     plugindesc.obj
 0002:00006d08       ??_C@_0N@KHGMHPFC@?4m?5c?5?$CD484848?$AA@ 10026d08     plugindesc.obj
 0002:00006d18       ??_C@_0N@LCNIEPCK@?$CDf?5c?5?$CD4c4c4c?$AA@ 10026d18     plugindesc.obj
 0002:00006d28       ??_C@_0N@KEJGHBHE@?4D?5c?5?$CD4e4e4e?$AA@ 10026d28     plugindesc.obj
 0002:00006d38       ??_C@_0N@PIHABEAP@?4C?5c?5?$CD525252?$AA@ 10026d38     plugindesc.obj
 0002:00006d48       ??_C@_0N@BGALNNID@?4V?5c?5?$CD527252?$AA@ 10026d48     plugindesc.obj
 0002:00006d58       ??_C@_0N@LLDHAKNF@?4Y?5c?5?$CD545454?$AA@ 10026d58     plugindesc.obj
 0002:00006d68       ??_C@_0N@FBGMGFNK@?$CDN?5c?5?$CD565656?$AA@ 10026d68     plugindesc.obj
 0002:00006d78       ??_C@_0N@HJLBMNKE@?4B?5c?5?$CD575757?$AA@ 10026d78     plugindesc.obj
 0002:00006d88       ??_C@_0N@KFBKEAHB@?4h?5c?5?$CD585858?$AA@ 10026d88     plugindesc.obj
 0002:00006d98       ??_C@_0N@OJDOAMLF@?4k?5c?5?$CD586666?$AA@ 10026d98     plugindesc.obj
 0002:00006da8       ??_C@_0N@EHMOIJHP@?4X?5c?5?$CD5a5a5a?$AA@ 10026da8     plugindesc.obj
 0002:00006db8       ??_C@_0N@MHGOGDPB@?$CDO?5c?5?$CD5b5b5b?$AA@ 10026db8     plugindesc.obj
 0002:00006dc8       ??_C@_0N@GBAAEDMJ@?$CDK?5c?5?$CD5d5d5d?$AA@ 10026dc8     plugindesc.obj
 0002:00006dd8       ??_C@_0N@GPDHAFGJ@?$CDH?5c?5?$CD606060?$AA@ 10026dd8     plugindesc.obj
 0002:00006de8       ??_C@_0N@DDEAACPO@?$CDq?5c?5?$CD626262?$AA@ 10026de8     plugindesc.obj
 0002:00006df8       ??_C@_0N@CEIANAGF@?4O?5c?5?$CD63e263?$AA@ 10026df8     plugindesc.obj
 0002:00006e08       ??_C@_0N@BADJAHNJ@?40?5c?5?$CD656565?$AA@ 10026e08     plugindesc.obj
 0002:00006e18       ??_C@_0N@GLMFBDGD@?4U?5c?5?$CD656e65?$AA@ 10026e18     plugindesc.obj
 0002:00006e28       ??_C@_0N@HKLIILC@?4Z?5c?5?$CD676767?$AA@ 10026e28     plugindesc.obj
 0002:00006e38       ??_C@_0N@OBKGCMOL@?$CDk?5c?5?$CD686868?$AA@ 10026e38     plugindesc.obj
 0002:00006e48       ??_C@_0N@FDOBGHPE@?4W?5c?5?$CD6a6b6a?$AA@ 10026e48     plugindesc.obj
 0002:00006e58       ??_C@_0N@NFAMBBOO@?43?5c?5?$CD6b6b6b?$AA@ 10026e58     plugindesc.obj
 0002:00006e68       ??_C@_0N@HLJOGGPI@?4Q?5c?5?$CD6c6c6c?$AA@ 10026e68     plugindesc.obj
 0002:00006e78       ??_C@_0N@IMICELOB@?$CDj?5c?5?$CD6c6c97?$AA@ 10026e78     plugindesc.obj
 0002:00006e88       ??_C@_0N@LCOBOHHM@?$CDv?5c?5?$CD6c6cc1?$AA@ 10026e88     plugindesc.obj
 0002:00006e98       ??_C@_0N@MJMHNGFO@?$CD7?5c?5?$CD717171?$AA@ 10026e98     plugindesc.obj
 0002:00006ea8       ??_C@_0N@MMHABJMP@?$CDe?5c?5?$CD737373?$AA@ 10026ea8     plugindesc.obj
 0002:00006eb8       ??_C@_0N@NKNIJBPP@?$CDp?5c?5?$CD73739a?$AA@ 10026eb8     plugindesc.obj
 0002:00006ec8       ??_C@_0N@MAFCNMGP@?$CDz?5c?5?$CD7373c2?$AA@ 10026ec8     plugindesc.obj
 0002:00006ed8       ??_C@_0N@KBDHNMOL@?$CD8?5c?5?$CD747474?$AA@ 10026ed8     plugindesc.obj
 0002:00006ee8       ??_C@_0N@LKFOPNGE@?$CD3?5c?5?$CD757575?$AA@ 10026ee8     plugindesc.obj
 0002:00006ef8       ??_C@_0N@PNBOBKHE@?$CD?4?5c?5?$CD777777?$AA@ 10026ef8     plugindesc.obj
 0002:00006f08       ??_C@_0N@JAMNIBDG@a?$CD?5c?5?$CD787878?$AA@ 10026f08     plugindesc.obj
 0002:00006f18       ??_C@_0N@EBIHFNLL@?4x?5c?5?$CD7bc0c0?$AA@ 10026f18     plugindesc.obj
 0002:00006f28       ??_C@_0N@ECBNLLNN@?4y?5c?5?$CD7bc2c2?$AA@ 10026f28     plugindesc.obj
 0002:00006f38       ??_C@_0N@DGIFOMJL@?$CDl?5c?5?$CD7f7f7f?$AA@ 10026f38     plugindesc.obj
 0002:00006f48       ??_C@_0N@GAMPMEDG@?$CDm?5c?5?$CD818181?$AA@ 10026f48     plugindesc.obj
 0002:00006f58       ??_C@_0N@CFKGANNG@?4T?5c?5?$CD888888?$AA@ 10026f58     plugindesc.obj
 0002:00006f68       ??_C@_0N@MMGLOLJB@?4w?5c?5?$CD8e8e8e?$AA@ 10026f68     plugindesc.obj
 0002:00006f78       ??_C@_0N@KKECMECA@?4z?5c?5?$CD8ebaba?$AA@ 10026f78     plugindesc.obj
 0002:00006f88       ??_C@_0N@EKGEFDGL@?4d?5c?5?$CD909090?$AA@ 10026f88     plugindesc.obj
 0002:00006f98       ??_C@_0N@LFMBMGOH@a?4?5c?5?$CD939393?$AA@ 10026f98     plugindesc.obj
 0002:00006fa8       ??_C@_0N@HENFGEIP@?$CDa?5c?5?$CD989898?$AA@ 10026fa8     plugindesc.obj
 0002:00006fb8       ??_C@_0N@CDGPEAFH@?$CD2?5c?5?$CD99bd99?$AA@ 10026fb8     plugindesc.obj
 0002:00006fc8       ??_C@_0N@CJDPGFGE@?4c?5c?5?$CD9a9a9a?$AA@ 10026fc8     plugindesc.obj
 0002:00006fd8       ??_C@_0N@GHGNCCAJ@?4b?5c?5?$CD9c9c9c?$AA@ 10026fd8     plugindesc.obj
 0002:00006fe8       ??_C@_0N@CLLHLKB@?$CD6?5c?5?$CD9dbc9d?$AA@ 10026fe8     plugindesc.obj
 0002:00006ff8       ??_C@_0N@KOKMALDJ@?4E?5c?5?$CD9e9e9e?$AA@ 10026ff8     plugindesc.obj
 0002:00007008       ??_C@_0N@EBHCONMB@?42?5c?5?$CD9f9f9f?$AA@ 10027008     plugindesc.obj
 0002:00007018       ??_C@_0N@OEAEDHJO@?$CDr?5c?5?$CDa4a4a4?$AA@ 10027018     plugindesc.obj
 0002:00007028       ??_C@_0N@BJECBDIM@?$CDc?5c?5?$CDa5a5a5?$AA@ 10027028     plugindesc.obj
 0002:00007038       ??_C@_0N@KMILADHD@?48?5c?5?$CDa6a6a6?$AA@ 10027038     plugindesc.obj
 0002:00007048       ??_C@_0N@OABJJJJ@?4J?5c?5?$CDa7a7a7?$AA@ 10027048     plugindesc.obj
 0002:00007058       ??_C@_0N@LBBNPALI@?4S?5c?5?$CDa8a8a8?$AA@ 10027058     plugindesc.obj
 0002:00007068       ??_C@_0N@IFIFILNL@?49?5c?5?$CDaaaaaa?$AA@ 10027068     plugindesc.obj
 0002:00007078       ??_C@_0N@NPHBDOME@?$CDd?5c?5?$CDababab?$AA@ 10027078     plugindesc.obj
 0002:00007088       ??_C@_0N@CCOGBPKI@?46?5c?5?$CDacacac?$AA@ 10027088     plugindesc.obj
 0002:00007098       ??_C@_0N@BFLGCMIL@?$CDG?5c?5?$CDadadad?$AA@ 10027098     plugindesc.obj
 0002:000070a8       ??_C@_0N@FLNGCNIA@?4t?5c?5?$CDaeaeae?$AA@ 100270a8     plugindesc.obj
 0002:000070b8       ??_C@_0N@HAGBDJOP@?4a?5c?5?$CDafafaf?$AA@ 100270b8     plugindesc.obj
 0002:000070c8       ??_C@_0N@MCACALLL@?4I?5c?5?$CDb0b0b0?$AA@ 100270c8     plugindesc.obj
 0002:000070d8       ??_C@_0N@EBJEDNPL@?4N?5c?5?$CDb1d2b1?$AA@ 100270d8     plugindesc.obj
 0002:000070e8       ??_C@_0N@JHGHKMFB@?4l?5c?5?$CDb2b2b2?$AA@ 100270e8     plugindesc.obj
 0002:000070f8       ??_C@_0N@NPALNLKE@?$CDW?5c?5?$CDb3b3b3?$AA@ 100270f8     plugindesc.obj
 0002:00007108       ??_C@_0N@DHNEPPOJ@?$CD?$CD?5c?5?$CDb4b4b4?$AA@ 10027108     plugindesc.obj
 0002:00007118       ??_C@_0N@OJJBJOEF@?$CD5?5c?5?$CDb4c4b4?$AA@ 10027118     plugindesc.obj
 0002:00007128       ??_C@_0N@JGDENJBC@?4H?5c?5?$CDb7b7b7?$AA@ 10027128     plugindesc.obj
 0002:00007138       ??_C@_0N@BGIENEDO@?$CDF?5c?5?$CDb8b8b8?$AA@ 10027138     plugindesc.obj
 0002:00007148       ??_C@_0N@EPMLNIEO@?4A?5c?5?$CDb9b9b9?$AA@ 10027148     plugindesc.obj
 0002:00007158       ??_C@_0N@HIACIEMG@?$CD0?5c?5?$CDb9c4b9?$AA@ 10027158     plugindesc.obj
 0002:00007168       ??_C@_0N@GIBODB@?4f?5c?5?$CDbbbbbb?$AA@ 10027168     plugindesc.obj
 0002:00007178       ??_C@_0N@JDCPKDOK@?$CDS?5c?5?$CDc1c1c1?$AA@ 10027178     plugindesc.obj
 0002:00007188       ??_C@_0N@JDPDAILA@?4P?5c?5?$CDc2c6c2?$AA@ 10027188     plugindesc.obj
 0002:00007198       ??_C@_0N@MBHJIAND@?4G?5c?5?$CDc4c4c4?$AA@ 10027198     plugindesc.obj
 0002:000071a8       ??_C@_0N@CICENEKD@?$CDT?5c?5?$CDc6c6c6?$AA@ 100271a8     plugindesc.obj
 0002:000071b8       ??_C@_0N@JEECOGDB@?4M?5c?5?$CDc7c7c7?$AA@ 100271b8     plugindesc.obj
 0002:000071c8       ??_C@_0N@GNFCGLAC@?41?5c?5?$CDcacaca?$AA@ 100271c8     plugindesc.obj
 0002:000071d8       ??_C@_0N@DNGDEAGB@?47?5c?5?$CDcbcbcb?$AA@ 100271d8     plugindesc.obj
 0002:000071e8       ??_C@_0N@DJNJDLLL@?4n?5c?5?$CDcdcdcd?$AA@ 100271e8     plugindesc.obj
 0002:000071f8       ??_C@_0N@HIKHOMDD@?$CDI?5c?5?$CDcecece?$AA@ 100271f8     plugindesc.obj
 0002:00007208       ??_C@_0N@FJAEGDFO@?$CDD?5c?5?$CDcfcfcf?$AA@ 10027208     plugindesc.obj
 0002:00007218       ??_C@_0N@JAPKDHIJ@?44?5c?5?$CDd0d0d0?$AA@ 10027218     plugindesc.obj
 0002:00007228       ??_C@_0N@LNALPJA@?$CDY?5c?5?$CDd1d1d1?$AA@ 10027228     plugindesc.obj
 0002:00007238       ??_C@_0N@MFEOJFBN@?$CDR?5c?5?$CDd2d2d2?$AA@ 10027238     plugindesc.obj
 0002:00007248       ??_C@_0N@GCBPEHAI@?4o?5c?5?$CDd3d3d3?$AA@ 10027248     plugindesc.obj
 0002:00007258       ??_C@_0N@BEIMCBLD@?4g?5c?5?$CDd7d7d7?$AA@ 10027258     plugindesc.obj
 0002:00007268       ??_C@_0N@KMFPPJBI@?$CDb?5c?5?$CDdbdbdb?$AA@ 10027268     plugindesc.obj
 0002:00007278       ??_C@_0N@MJGLKPGE@?45?5c?5?$CDdcdcdc?$AA@ 10027278     plugindesc.obj
 0002:00007288       ??_C@_0N@CLPONBCD@?4v?5c?5?$CDdedede?$AA@ 10027288     plugindesc.obj
 0002:00007298       ??_C@_0N@CIAFAPNO@?$CDQ?5c?5?$CDe2e2e2?$AA@ 10027298     plugindesc.obj
 0002:000072a8       ??_C@_0N@GIMLOOAN@?4?$CD?5c?5?$CDe5e5e5?$AA@ 100272a8     plugindesc.obj
 0002:000072b8       ??_C@_0N@OHPKBGHG@?4L?5c?5?$CDe7e7e7?$AA@ 100272b8     plugindesc.obj
 0002:000072c8       ??_C@_0N@OLJOJLEG@?$CDX?5c?5?$CDe9e9e9?$AA@ 100272c8     plugindesc.obj
 0002:000072d8       ??_C@_0N@HBJEJHDD@?$CDP?5c?5?$CDeaeaea?$AA@ 100272d8     plugindesc.obj
 0002:000072e8       ??_C@_0N@GPMFLNFL@?4e?5c?5?$CDececec?$AA@ 100272e8     plugindesc.obj
 0002:000072f8       ??_C@_0N@MPPJCKJF@?4F?5c?5?$CDededed?$AA@ 100272f8     plugindesc.obj
 0002:00007308       ??_C@_0N@CPJCPKPA@?$CDU?5c?5?$CDf6f6f6?$AA@ 10027308     plugindesc.obj
 0002:00007318       ??_C@_0N@PKHFBGFA@?$CDL?5c?5?$CDf8f8f8?$AA@ 10027318     plugindesc.obj
 0002:00007328       ??_C@_0N@OKKHOMMH@?$CDV?5c?5?$CDfafafa?$AA@ 10027328     plugindesc.obj
 0002:00007338       ??_C@_0N@PGNJBDN@?$CD9?5c?5?$CDfbfbfb?$AA@ 10027338     plugindesc.obj
 0002:00007348       ??_C@_0N@HDFHOOJE@?$CDw?5c?5?$CDfdfdfd?$AA@ 10027348     plugindesc.obj
 0002:00007358       ??_C@_0N@OHLCLFHA@?$CDM?5c?5?$CDfefefe?$AA@ 10027358     plugindesc.obj
 0002:00007368       ??_C@_09LMOMIOIP@Qt?5c?5none?$AA@ 10027368     plugindesc.obj
 0002:00007374       ??_C@_0CJ@OIGLBNHJ@QtQtQtQtQtQt?4?$CD?4a?4b?4b?4b?4b?4c?4d?4eQt@ 10027374     plugindesc.obj
 0002:000073a0       ??_C@_0CJ@CFDAHDL@QtQtQtQtQtQt?4f?4g?4h?4i?4j?4k?4l?4m?4nQt@ 100273a0     plugindesc.obj
 0002:000073cc       ??_C@_0CJ@DLHDCLBH@QtQtQtQtQtQt?4f?4o?4p?4q?4r?4s?4t?4m?4nQt@ 100273cc     plugindesc.obj
 0002:000073f8       ??_C@_0CJ@GHNCLIBH@QtQtQtQtQtQt?4f?4o?4p?4u?4r?4s?4t?4m?4nQt@ 100273f8     plugindesc.obj
 0002:00007424       ??_C@_0CJ@PNFGJFJD@QtQtQtQtQtQt?4f?4v?4w?4x?4y?4z?4A?4m?4nQt@ 10027424     plugindesc.obj
 0002:00007450       ??_C@_0CJ@BAFFNOIG@QtQtQtQtQtQt?4f?4B?4C?4C?4C?4C?4C?4D?4EQt@ 10027450     plugindesc.obj
 0002:0000747c       ??_C@_0CJ@DAEJIALD@QtQtQtQtQt?4F?4G?4f?4H?4H?4l?4a?4I?4J?4KQt@ 1002747c     plugindesc.obj
 0002:000074a8       ??_C@_0CJ@HNBOJK@QtQtQtQtQt?4L?4M?4N?4O?4P?4Q?4R?4D?4S?4RQt@ 100274a8     plugindesc.obj
 0002:000074d4       ??_C@_0CJ@KPCGPHGL@QtQtQtQtQt?4F?4T?4U?4V?4W?4X?4C?4Y?4Z?40Qt@ 100274d4     plugindesc.obj
 0002:00007500       ??_C@_0CJ@NMCJKKCN@QtQtQtQtQtQt?41?42?42?43?43?42?42?42?4eQt@ 10027500     plugindesc.obj
 0002:0000752c       ??_C@_0CJ@DEOJNHBL@Qt?4v?44?44?44?44?44?45Qt?46?46Qt?45?44?44?44@ 1002752c     plugindesc.obj
 0002:00007558       ??_C@_0CJ@JBLPHIMG@?4v?47?48?4b?4b?4b?49?$CD?4?$CD?$CD?$CDa?$CDa?$CDb?47?$CDc?4b?4b@ 10027558     plugindesc.obj
 0002:00007584       ??_C@_0CJ@NIONEBKK@?4o?4o?$CDf?$CDg?$CDh?$CDi?$CDj?$CDk?4D?$CDl?$CDl?$CDm?4o?4m?$CDn?$CDh@ 10027584     plugindesc.obj
 0002:000075b0       ??_C@_0CJ@MCLMGAKJ@?4o?4o?$CDf?$CDs?$CDt?$CDu?$CDv?$CDk?4T?$CDw?$CDw?4f?4o?4m?$CDx?$CDt@ 100275b0     plugindesc.obj
 0002:000075e0       ??_7config_plugin_desc_base@@6B@ 100275e0     plugindesc.obj
 0002:000075f4       ??_7plugindesc@@6B@        100275f4     plugindesc.obj
 0002:00007604       ??_C@_0BN@FDKNOOHJ@Home?1Developer?1Test?5Plugin?51?$AA@ 10027604     plugindesc.obj
 0002:00007624       ??_C@_0BN@HIIALNLK@Home?1Developer?1Test?5Plugin?52?$AA@ 10027624     plugindesc.obj
 0002:00007644       ??_C@_0BN@GBJLIMPL@Home?1Developer?1Test?5Plugin?53?$AA@ 10027644     plugindesc.obj
 0002:00007664       ??_C@_0CA@NJBAPGID@Home?1System?1Workstations?1Launch?$AA@ 10027664     plugindesc.obj
 0002:00007684       ??_C@_0CG@HDGGNOOO@Home?1System?1Workstations?1Worksta@ 10027684     plugindesc.obj
 0002:000076ac       ??_C@_0BJ@MBNGFKCP@Home?1System?1File?5Manager?$AA@ 100276ac     plugindesc.obj
 0002:000076cc       ??_7testPlugin@@6BQObject@@@ 100276cc     testPlugin.obj
 0002:000078a4       ??_7testPlugin@@6BQPaintDevice@@@ 100278a4     testPlugin.obj
 0002:000078c4       ??_C@_0BC@FBGELHEJ@testPlugin?5path?5?3?$AA@ 100278c4     testPlugin.obj
 0002:000078d8       ??_C@_0BA@BHECNFPG@1downloadFile?$CI?$CJ?$AA@ 100278d8     testPlugin.obj
 0002:000078e8       ??_C@_0O@NEJFAGCC@1uploadFile?$CI?$CJ?$AA@ 100278e8     testPlugin.obj
 0002:000078f8       ??_C@_0M@LDOJBCGK@1lockFile?$CI?$CJ?$AA@ 100278f8     testPlugin.obj
 0002:00007904       ??_C@_0O@MGGKACOK@1unlockFile?$CI?$CJ?$AA@ 10027904     testPlugin.obj
 0002:00007914       ??_C@_0N@LIDOGOCD@1unlockDir?$CI?$CJ?$AA@ 10027914     testPlugin.obj
 0002:00007924       ??_C@_0L@HDEEBEMI@1dbClear?$CI?$CJ?$AA@ 10027924     testPlugin.obj
 0002:00007930       ??_C@_0BA@HNGFFIG@1checkoutFile?$CI?$CJ?$AA@ 10027930     testPlugin.obj
 0002:00007940       ??_C@_0P@GFHEKJBN@1checkoutDir?$CI?$CJ?$AA@ 10027940     testPlugin.obj
 0002:00007950       ??_C@_0P@CLIOIDIH@1downloadDir?$CI?$CJ?$AA@ 10027950     testPlugin.obj
 0002:00007960       ??_C@_0N@PANDPGHK@1uploadDir?$CI?$CJ?$AA@ 10027960     testPlugin.obj
 0002:00007970       ??_C@_06NIOODGLD@1dir?$CI?$CJ?$AA@ 10027970     testPlugin.obj
 0002:00007978       ??_C@_0O@IFBMFLDK@1doNavigate?$CI?$CJ?$AA@ 10027978     testPlugin.obj
 0002:00007988       ??_C@_09PJDIALKE@1doHelp?$CI?$CJ?$AA@ 10027988     testPlugin.obj
 0002:00007994       ??_C@_0L@LLCEHIPB@1doDirty?$CI?$CJ?$AA@ 10027994     testPlugin.obj
 0002:000079a0       ??_C@_0BA@BALHMLMC@?2testPlugin?4sav?$AA@ 100279a0     testPlugin.obj
 0002:000079b0       ??_C@_01LIIJDEN@?$AN?$AA@  100279b0     testPlugin.obj
 0002:000079b4       ??_C@_01EEMJAFIK@?6?$AA@   100279b4     testPlugin.obj
 0002:000079b8       ??_C@_0BD@FJKLDAPM@The?5user?5level?5is?5?$AA@ 100279b8     testPlugin.obj
 0002:000079cc       ??_C@_0BF@MONACHLK@TP?3?5Workstation?5List?$AA@ 100279cc     testPlugin.obj
 0002:000079e4       ??_C@_0BB@CLGMKNED@Workstation?5List?$AA@ 100279e4     testPlugin.obj
 0002:000079f8       ??_C@_02HOGEDOAB@Id?$AA@   100279f8     testPlugin.obj
 0002:000079fc       ??_C@_04FABLJDN@Name?$AA@  100279fc     testPlugin.obj
 0002:00007a04       ??_C@_04COAGEIMF@copy?$AA@ 10027a04     testPlugin.obj
 0002:00007a0c       ??_C@_05EJNCNHFE@?$CGCopy?$AA@ 10027a0c     testPlugin.obj
 0002:00007a14       ??_C@_04OPMHGHMB@Copy?$AA@ 10027a14     testPlugin.obj
 0002:00007a1c       ??_C@_05NDLFFNHM@paste?$AA@ 10027a1c     testPlugin.obj
 0002:00007a24       ??_C@_06FENKCKDB@?$CGPaste?$AA@ 10027a24     testPlugin.obj
 0002:00007a2c       ??_C@_09MABIAGDN@selectall?$AA@ 10027a2c     testPlugin.obj
 0002:00007a38       ??_C@_0M@JHCAAOEG@Select?5?$CGAll?$AA@ 10027a38     testPlugin.obj
 0002:00007a44       ??_C@_0L@CALHPJHB@Select?5All?$AA@ 10027a44     testPlugin.obj
 0002:00007a50       ??_C@_09GACKKJAD@selectAll?$AA@ 10027a50     testPlugin.obj
 0002:00007a5c       ??_C@_04HOKNPDPJ@undo?$AA@ 10027a5c     testPlugin.obj
 0002:00007a64       ??_C@_05BJHJGMGI@?$CGUndo?$AA@ 10027a64     testPlugin.obj
 0002:00007a6c       ??_C@_04LPGMNMPN@Undo?$AA@ 10027a6c     testPlugin.obj
 0002:00007a74       ??_C@_0BA@ELAGLCLB@toolbar?5Request?$AA@ 10027a74     testPlugin.obj
 0002:00007a84       ??_C@_0N@EDFGJBJ@Menu?5Request?$AA@ 10027a84     testPlugin.obj
 0002:00007a94       ??_C@_0M@BEBFGCFG@close?5event?$AA@ 10027a94     testPlugin.obj
 0002:00007aa0       ??_C@_02PCIJFNDE@?$AN?6?$AA@ 10027aa0     testPlugin.obj
 0002:00007aa4       ??_C@_03NLJIHOMM@?5?9?5?$AA@ 10027aa4     testPlugin.obj
 0002:00007aa8       ??_C@_07KJPPILBA@Reply?3?5?$AA@ 10027aa8     testPlugin.obj
 0002:00007ab0       ??_C@_0DC@HDKLOGLE@Being?5asked?5to?5navigate?5to?5?$CC?$CFs?$CC?5@ 10027ab0     testPlugin.obj
 0002:00007ae4       ??_C@_0M@IPKBPLNA@activate?5me?$AA@ 10027ae4     testPlugin.obj
 0002:00007af0       ??_C@_0O@KDGCCNAH@deactivate?5me?$AA@ 10027af0     testPlugin.obj
 0002:00007b00       ??_C@_05KAEIDCAL@apply?$AA@ 10027b00     testPlugin.obj
 0002:00007b08       ??_C@_0BC@JOJNABEP@testPlugin?3?3apply?$AA@ 10027b08     testPlugin.obj
 0002:00007b1c       ??_C@_0BA@GNHMHBBC@syncDirDownload?$AA@ 10027b1c     testPlugin.obj
 0002:00007b2c       ??_C@_0O@JFGJGFB@syncDirUpload?$AA@ 10027b2c     testPlugin.obj
 0002:00007b40       ??_7testPluginFromBase@@6BQObject@@@ 10027b40     testPluginFromBase.obj
 0002:00007d28       ??_7testPluginFromBase@@6BQPaintDevice@@@ 10027d28     testPluginFromBase.obj
 0002:00007d48       ??_C@_0BB@KNHDMHLN@1downloadFileS?$CI?$CJ?$AA@ 10027d48     testPluginFromBase.obj
 0002:00007d5c       ??_C@_0P@CMAOAGKD@1uploadFileS?$CI?$CJ?$AA@ 10027d5c     testPluginFromBase.obj
 0002:00007d6c       ??_C@_0N@FEGOLDBF@1lockFileS?$CI?$CJ?$AA@ 10027d6c     testPluginFromBase.obj
 0002:00007d7c       ??_C@_0P@LJKDLDCF@1unlockFileS?$CI?$CJ?$AA@ 10027d7c     testPluginFromBase.obj
 0002:00007d8c       ??_C@_0O@FLGFJNFN@1unlockDirS?$CI?$CJ?$AA@ 10027d8c     testPluginFromBase.obj
 0002:00007d9c       ??_C@_0M@GMHGNMNH@1dbClearS?$CI?$CJ?$AA@ 10027d9c     testPluginFromBase.obj
 0002:00007da8       ??_C@_0BB@PNGGCCAB@1checkoutFileS?$CI?$CJ?$AA@ 10027da8     testPluginFromBase.obj
 0002:00007dbc       ??_C@_0BA@JKNJMKDB@1checkoutDirS?$CI?$CJ?$AA@ 10027dbc     testPluginFromBase.obj
 0002:00007dcc       ??_C@_0BA@IKENEKEB@1downloadDirS?$CI?$CJ?$AA@ 10027dcc     testPluginFromBase.obj
 0002:00007ddc       ??_C@_0O@EJJKJJJF@1uploadDirS?$CI?$CJ?$AA@ 10027ddc     testPluginFromBase.obj
 0002:00007dec       ??_C@_07KLAKNOEB@1dirS?$CI?$CJ?$AA@ 10027dec     testPluginFromBase.obj
 0002:00007df4       ??_C@_0P@DPDDBHKI@1doNavigateS?$CI?$CJ?$AA@ 10027df4     testPluginFromBase.obj
 0002:00007e04       ??_C@_0L@CIPIINLL@1doHelpS?$CI?$CJ?$AA@ 10027e04     testPluginFromBase.obj
 0002:00007e10       ??_C@_0M@DDLLDELD@1doDirtyS?$CI?$CJ?$AA@ 10027e10     testPluginFromBase.obj
 0002:00007e1c       ??_C@_0M@DMJICNOE@1doCleanS?$CI?$CJ?$AA@ 10027e1c     testPluginFromBase.obj
 0002:00007e28       ??_C@_03BGMCNDOO@?5OK?$AA@ 10027e28     testPluginFromBase.obj
 0002:00007e2c       ??_C@_09EIHGCJJC@Download?5?$AA@ 10027e2c     testPluginFromBase.obj
 0002:00007e38       ??_C@_07LICNECBD@?5FAIL?3?5?$AA@ 10027e38     testPluginFromBase.obj
 0002:00007e40       ??_C@_05NFFACMFJ@Lock?5?$AA@ 10027e40     testPluginFromBase.obj
 0002:00007e48       ??_C@_07FGOHPFJK@Upload?5?$AA@ 10027e48     testPluginFromBase.obj
 0002:00007e50       ??_C@_07MAFDJNLP@Unlock?5?$AA@ 10027e50     testPluginFromBase.obj
 0002:00007e58       ??_C@_0M@FCEFEINA@Unlock?5dir?5?$AA@ 10027e58     testPluginFromBase.obj
 0002:00007e64       ??_C@_0P@BHLPGIHH@Sync?5down?5dir?5?$AA@ 10027e64     testPluginFromBase.obj
 0002:00007e74       ??_C@_0N@KALCGCDI@Sync?5up?5dir?5?$AA@ 10027e74     testPluginFromBase.obj
 0002:00007e84       ??_C@_09EPNKFLLE@Checkout?5?$AA@ 10027e84     testPluginFromBase.obj
 0002:00007e90       ??_C@_0O@IHCAJIJA@Checkout?5dir?5?$AA@ 10027e90     testPluginFromBase.obj
 0002:00007ea0       ??_C@_09OMOJJJM@Dir?5list?5?$AA@ 10027ea0     testPluginFromBase.obj
 0002:00007eac       ??_C@_01GPOEFGEJ@?7?$AA@   10027eac     testPluginFromBase.obj
 0002:00007eb0       ??_C@_0N@CNAKOOCI@?$CF1?5is?5dirty?4?$AA@ 10027eb0     testPluginFromBase.obj
 0002:00007ec0       ??_C@_0CG@FALDGPOE@Dirtying?5failed?5?9?5do?5you?5have?5a?5@ 10027ec0     testPluginFromBase.obj
 0002:00007ee8       ??_C@_0N@BEAOBINP@?$CF1?5is?5clean?4?$AA@ 10027ee8     testPluginFromBase.obj
 0002:00007ef8       ??_C@_0CG@MHHODMFN@Cleaning?5failed?5?9?5do?5you?5have?5a?5@ 10027ef8     testPluginFromBase.obj
 0002:00007f20       ??_C@_0BC@BPGJHMLK@Asked?5to?5save?5?$CF1?4?$AA@ 10027f20     testPluginFromBase.obj
 0002:00007f34       ??_C@_0BE@KFIFNHGN@Asked?5to?5reload?5?$CF1?4?$AA@ 10027f34     testPluginFromBase.obj
 0002:00007f4c       ??_7workstationCustomTable@@6BQObject@@@ 10027f4c     workstationCustomTable.obj
 0002:000082f0       ??_7workstationCustomTable@@6BQPaintDevice@@@ 100282f0     workstationCustomTable.obj
 0002:00008310       ??_C@_0P@CKLAEKEC@ID?5?$CIWS?5Number?$CJ?$AA@ 10028310     workstationCustomTable.obj
 0002:00008320       ??_C@_0N@EDJNPFHL@Default?5User?$AA@ 10028320     workstationCustomTable.obj
 0002:00008330       ??_C@_0BD@PHPDBBBM@1sortColumn?$CI?5int?5?$CJ?$AA@ 10028330     workstationCustomTable.obj
 0002:00008344       ??_C@_0BA@HHAILMBL@2clicked?$CI?5int?5?$CJ?$AA@ 10028344     workstationCustomTable.obj
 0002:00008354       ??_C@_0BF@KONCIBBF@table?5item?5destroyed?$AA@ 10028354     workstationCustomTable.obj
 0002:00008370       ??_7workstationDockWindow@@6BQObject@@@ 10028370     workstationdockwindowimpl.obj
 0002:00008528       ??_7workstationDockWindow@@6BQPaintDevice@@@ 10028528     workstationdockwindowimpl.obj
 0002:0000854c       ??_7workstationEditor@@6BQObject@@@ 1002854c     workstationEditor.obj
 0002:00008724       ??_7workstationEditor@@6BQPaintDevice@@@ 10028724     workstationEditor.obj
 0002:00008744       ??_C@_0BJ@INGHKKD@workstationEditor?5path?5?3?$AA@ 10028744     workstationEditor.obj
 0002:00008760       ??_C@_0BA@PMEBAMEE@New?5Workstation?$AA@ 10028760     workstationEditor.obj
 0002:00008770       ??_C@_0BI@KPPMJODB@Delete?5this?5Workstation?$AA@ 10028770     workstationEditor.obj
 0002:00008788       ??_C@_0BB@FEGHJLOM@config?1users?4xml?$AA@ 10028788     workstationEditor.obj
 0002:000087a0       ??_C@_0EH@NBIAICCM@?$DMh3?$DOWorkstation?5Application?5Laun@ 100287a0     workstationEditor.obj
 0002:000087e8       ??_C@_08CBHEKIBI@13?324?335?$AA@ 100287e8     workstationEditor.obj
 0002:000087f8       ??_7workstationEditorDlg@@6BQObject@@@ 100287f8     workstationeditordlgimpl.obj
 0002:000089b0       ??_7workstationEditorDlg@@6BQPaintDevice@@@ 100289b0     workstationeditordlgimpl.obj
 0002:000089d0       ??_C@_0BJ@JHBMOHLN@?2config?2workstations?4xml?$AA@ 100289d0     workstationeditordlgimpl.obj
 0002:000089f0       ??_C@_0GJ@MLFBLPGP@?$DM?$DPxml?5version?$DN?$CC1?40?$CC?5encoding?$DN?$CCUT@ 100289f0     workstationeditordlgimpl.obj
 0002:00008a5c       ??_C@_06GGPOMPNM@?$CInone?$CJ?$AA@ 10028a5c     workstationeditordlgimpl.obj
 0002:00008a64       ??_C@_0BD@MKNJIFCF@?7?$DMworkstation?5id?$DN?$CC?$AA@ 10028a64     workstationeditordlgimpl.obj
 0002:00008a78       ??_C@_08LCPNEMEL@?$CC?5name?$DN?$CC?$AA@ 10028a78     workstationeditordlgimpl.obj
 0002:00008a84       ??_C@_08GEIEADAI@?$CC?5user?$DN?$CC?$AA@ 10028a84     workstationeditordlgimpl.obj
 0002:00008a90       ??_C@_05OJNDEKBN@?$CC?5?1?$DO?6?$AA@ 10028a90     workstationeditordlgimpl.obj
 0002:00008a98       ??_C@_0BA@MINDMMGO@?$DM?1workstations?$DO?$AA@ 10028a98     workstationeditordlgimpl.obj
 0002:00008aa8       ??_C@_0BM@FKDLFPIA@trying?5to?5load?5workstations?$AA@ 10028aa8     workstationeditordlgimpl.obj
 0002:00008ac4       ??_C@_04CCHAHKJA@user?$AA@ 10028ac4     workstationeditordlgimpl.obj
 0002:00008acc       ??_C@_0BN@PIFDGHFF@config?1ws?1?$CF1?1bncs_system?4ini?$AA@ 10028acc     workstationeditordlgimpl.obj
 0002:00008aec       ??_C@_0BO@JPIPFDPL@?1config?1ws?1?$CF1?1bncs_system?4ini?$AA@ 10028aec     workstationeditordlgimpl.obj
 0002:00008b0c       ??_C@_01KICIPPFI@?2?$AA@   10028b0c     workstationeditordlgimpl.obj
 0002:00008b10       ??_C@_0M@CILGCIDH@Workstation?$AA@ 10028b10     workstationeditordlgimpl.obj
 0002:00008b1c       ??_C@_07BGDMAJAE@Network?$AA@ 10028b1c     workstationeditordlgimpl.obj
 0002:00008b24       ??_C@_01GBGANLPD@0?$AA@    10028b24     workstationeditordlgimpl.obj
 0002:00008b28       ??_C@_0P@IOLOJICH@DefaultAdaptor?$AA@ 10028b28     workstationeditordlgimpl.obj
 0002:00008b38       ??_C@_07DMJBFPJJ@Channel?$AA@ 10028b38     workstationeditordlgimpl.obj
 0002:00008b40       ??_C@_01HIHLOKLC@1?$AA@    10028b40     workstationeditordlgimpl.obj
 0002:00008b44       ??_C@_0O@HMCAEAJL@NetworkEnable?$AA@ 10028b44     workstationeditordlgimpl.obj
 0002:00008b54       ??_C@_09FMACHHHI@CSIEnable?$AA@ 10028b54     workstationeditordlgimpl.obj
 0002:00008b60       ??_C@_0O@HBFIENKE@SessionEnable?$AA@ 10028b60     workstationeditordlgimpl.obj
 0002:00008b70       ??_C@_0N@DFIPDPGD@ClientEnable?$AA@ 10028b70     workstationeditordlgimpl.obj
 0002:00008b80       ??_C@_0N@CFHGKKGI@DriverEnable?$AA@ 10028b80     workstationeditordlgimpl.obj
 0002:00008b90       ??_C@_02JMHLOEOE@24?$AA@   10028b90     workstationeditordlgimpl.obj
 0002:00008b94       ??_C@_02MIGHPNDL@12?$AA@   10028b94     workstationeditordlgimpl.obj
 0002:00008b98       ??_C@_0O@DDGEDIMC@ClientBuffers?$AA@ 10028b98     workstationeditordlgimpl.obj
 0002:00008ba8       ??_C@_0O@KEKGBINP@DriverBuffers?$AA@ 10028ba8     workstationeditordlgimpl.obj
 0002:00008bb8       ??_C@_01DHDKHMHF@6?$AA@    10028bb8     workstationeditordlgimpl.obj
 0002:00008bbc       ??_C@_0P@DGCALIKD@SessionBuffers?$AA@ 10028bbc     workstationeditordlgimpl.obj
 0002:00008bcc       ??_C@_0O@NGHAPIAM@SecBuffEnable?$AA@ 10028bcc     workstationeditordlgimpl.obj
 0002:00008bdc       ??_C@_0O@CEAAPDFP@TerBuffEnable?$AA@ 10028bdc     workstationeditordlgimpl.obj
 0002:00008bec       ??_C@_0P@OGKHCCNN@LoopbackEnable?$AA@ 10028bec     workstationeditordlgimpl.obj
 0002:00008bfc       ??_C@_0M@HJFGAKIL@c?3?2csi_temp?$AA@ 10028bfc     workstationeditordlgimpl.obj
 0002:00008c08       ??_C@_0N@NHBGKGMO@TempFilePath?$AA@ 10028c08     workstationeditordlgimpl.obj
 0002:00008c18       ??_C@_0M@NNFCLJKN@KeyFilePath?$AA@ 10028c18     workstationeditordlgimpl.obj
 0002:00008c24       ??_C@_0M@FPBKNPFP@CacheEnable?$AA@ 10028c24     workstationeditordlgimpl.obj
 0002:00008c30       ??_C@_05BEHOCFPE@Cache?$AA@ 10028c30     workstationeditordlgimpl.obj
 0002:00008c38       ??_C@_04MJHCKDHM@1024?$AA@ 10028c38     workstationeditordlgimpl.obj
 0002:00008c40       ??_C@_09OEJFPKAI@CacheSize?$AA@ 10028c40     workstationeditordlgimpl.obj
 0002:00008c4c       ??_C@_02PKFBJPLJ@10?$AA@   10028c4c     workstationeditordlgimpl.obj
 0002:00008c50       ??_C@_09BDBJKAEP@CacheLife?$AA@ 10028c50     workstationeditordlgimpl.obj
 0002:00008c5c       ??_C@_0BB@LEKFHEJN@TimeServerEnable?$AA@ 10028c5c     workstationeditordlgimpl.obj
 0002:00008c70       ??_C@_0L@JAJNDELA@TimeServer?$AA@ 10028c70     workstationeditordlgimpl.obj
 0002:00008c7c       ??_C@_02PPBOIJDM@60?$AA@   10028c7c     workstationeditordlgimpl.obj
 0002:00008c80       ??_C@_0BB@JINCHM@TimeServerPeriod?$AA@ 10028c80     workstationeditordlgimpl.obj
 0002:00008c94       ??_C@_08PJGOPNMK@DiagMode?$AA@ 10028c94     workstationeditordlgimpl.obj
 0002:00008ca0       ??_C@_0M@KLCHMOKB@Diagnostics?$AA@ 10028ca0     workstationeditordlgimpl.obj
 0002:00008cac       ??_C@_0P@NDALLNJE@DiagModeExtend?$AA@ 10028cac     workstationeditordlgimpl.obj
 0002:00008cbc       ??_C@_09DAMNBEKD@DebugMode?$AA@ 10028cbc     workstationeditordlgimpl.obj
 0002:00008cc8       ??_C@_0P@CLJPELBH@ClosedownDelay?$AA@ 10028cc8     workstationeditordlgimpl.obj
 0002:00008cd8       ??_C@_04MHPHMCPO@Misc?$AA@ 10028cd8     workstationeditordlgimpl.obj
 0002:00008ce0       ??_C@_0BA@OEAMJOKB@WatchDogComPort?$AA@ 10028ce0     workstationeditordlgimpl.obj
 0002:00008cf0       ??_C@_0BG@HLJDLNAC@DisableWatchdogOnExit?$AA@ 10028cf0     workstationeditordlgimpl.obj
 0002:00008d08       ??_C@_0BA@HPIKGCJO@TxRxRetryPeriod?$AA@ 10028d08     workstationeditordlgimpl.obj
 0002:00008d18       ??_C@_06DDLNFFBN@?$CGquot?$DL?$AA@ 10028d18     workstationeditordlgimpl.obj
 0002:00008d20       ??_C@_01BJJEKLCA@?$CC?$AA@ 10028d20     workstationeditordlgimpl.obj
 0002:00008d24       ??_C@_04GJOGLFEJ@?$CGlt?$DL?$AA@ 10028d24     workstationeditordlgimpl.obj
 0002:00008d2c       ??_C@_01MNNFJEPP@?$DM?$AA@ 10028d2c     workstationeditordlgimpl.obj
 0002:00008d30       ??_C@_04LOOHDCEI@?$CGgt?$DL?$AA@ 10028d30     workstationeditordlgimpl.obj
 0002:00008d38       ??_C@_01PPODPGHN@?$DO?$AA@ 10028d38     workstationeditordlgimpl.obj
 0002:00008d3c       ??_C@_05JKJFEODM@?$CGamp?$DL?$AA@ 10028d3c     workstationeditordlgimpl.obj
 0002:00008d44       ??_C@_01HNPIGOCE@?$CG?$AA@ 10028d44     workstationeditordlgimpl.obj
 0002:00008d48       ??_C@_06PNMEMOHD@?$CGapos?$DL?$AA@ 10028d48     workstationeditordlgimpl.obj
 0002:00008d50       ??_C@_01GEODFPGF@?8?$AA@   10028d50     workstationeditordlgimpl.obj
 0002:00008d58       ??_7workstationEditorNewWsDlg@@6BQObject@@@ 10028d58     workstationeditornewwsdlgimpl.obj
 0002:00008f1c       ??_7workstationEditorNewWsDlg@@6BQPaintDevice@@@ 10028f1c     workstationeditornewwsdlgimpl.obj
 0002:00008f3c       ??_C@_0DP@PJPHHBJF@?$DMp?$DOThe?5id?5?$CIworkstation?5number?$CJ?5s@ 10028f3c     workstationeditornewwsdlgimpl.obj
 0002:00008f80       ??_C@_0FE@EJFEOKKC@?$DMp?$DOThe?5given?5id?5?$CIworkstation?5num@ 10028f80     workstationeditornewwsdlgimpl.obj
 0002:00008fd8       ??_C@_0EP@JOKPHLJC@?$DMp?$DOPlease?5enter?5even?5the?5simples@ 10028fd8     workstationeditornewwsdlgimpl.obj
 0002:00009028       ??_C@_0DJ@PJHDDNPL@?$DMh3?$DOThere?5are?5the?5following?5prob@ 10029028     workstationeditornewwsdlgimpl.obj
 0002:00009064       ??_C@_0L@CFKFHNIF@Oh?5dear?4?4?4?$AA@ 10029064     workstationeditornewwsdlgimpl.obj
 0002:00009070       ??_C@_0BC@BFIEMEJM@?2config?2users?4xml?$AA@ 10029070     workstationeditornewwsdlgimpl.obj
 0002:00009084       ??_C@_0BH@POGFMMMO@can?8t?5open?5users?5file?5?$AA@ 10029084     workstationeditornewwsdlgimpl.obj
 0002:000090a0       ??_7workstationUserTableItem@@6B@ 100290a0     workstationUserTableItem.obj
 0002:000090ec       ??_SQComboBox@@6BQObject@@@ 100290ec     workstationUserTableItem.obj
 0002:000092d0       ??_SQComboBox@@6BQPaintDevice@@@ 100292d0     workstationUserTableItem.obj
 0002:000092f0       ??_C@_0BC@NAAGCOBJ@1doValueChanged?$CI?$CJ?$AA@ 100292f0     workstationUserTableItem.obj
 0002:00009304       ??_C@_0BC@BGJFBFF@2activated?$CI?5int?5?$CJ?$AA@ 10029304     workstationUserTableItem.obj
 0002:00009318       ??_C@_0N@LIKKKKKK@1destroyed?$CI?$CJ?$AA@ 10029318     workstationUserTableItem.obj
 0002:00009328       ??_C@_0N@FGAMGGE@2destroyed?$CI?$CJ?$AA@ 10029328     workstationUserTableItem.obj
 0002:00009338       ??_C@_09IFDIHLJH@QComboBox?$AA@ 10029338     workstationUserTableItem.obj
 0002:00009344       ??_C@_0CD@PIPJCKGG@couldn?8t?5open?5file?5?$CFs?5to?5set?5dat@ 10029344     xfer.obj
 0002:0000936c       ??_7xml_listview@@6BQObject@@@ 1002936c     xml_listview.obj
 0002:00009650       ??_7xml_listview@@6BQPaintDevice@@@ 10029650     xml_listview.obj
 0002:00009670       ??_C@_02LMMGJAGL@in?$AA@   10029670     xml_listview.obj
 0002:00009674       ??_C@_0BA@FKNGFNEK@Can?8t?5open?5file?$AA@ 10029674     xml_listview.obj
 0002:00009684       ??_C@_0BB@CBMJNPGL@Can?8t?5parse?5file?$AA@ 10029684     xml_listview.obj
 0002:0000969c       ??_7dialogBase@@6BQObject@@@ 1002969c     dialog.obj
 0002:00009854       ??_7dialogBase@@6BQPaintDevice@@@ 10029854     dialog.obj
 0002:00009874       ??_C@_0L@BCEAHFEK@dialogBase?$AA@ 10029874     dialog.obj
 0002:00009880       ??_C@_0BB@NFKKNJMG@dialogBaseLayout?$AA@ 10029880     dialog.obj
 0002:00009894       ??_C@_07BPJBECHP@layout8?$AA@ 10029894     dialog.obj
 0002:0000989c       ??_C@_07GIKHDDO@layout9?$AA@ 1002989c     dialog.obj
 0002:000098a8       ??_7launchEditorDlgBase@@6BQObject@@@ 100298a8     launcheditordlg.obj
 0002:00009a60       ??_7launchEditorDlgBase@@6BQPaintDevice@@@ 10029a60     launcheditordlg.obj
 0002:00009a84       ??_SQCheckBox@@6BQObject@@@ 10029a84     launcheditordlg.obj
 0002:00009c64       ??_SQCheckBox@@6BQPaintDevice@@@ 10029c64     launcheditordlg.obj
 0002:00009c84       ??_C@_0BE@CHFGLEBE@launchEditorDlgBase?$AA@ 10029c84     launcheditordlg.obj
 0002:00009c98       ??_C@_0BK@GAIJFOBC@launchEditorDlgBaseLayout?$AA@ 10029c98     launcheditordlg.obj
 0002:00009cb4       ??_C@_0L@KGLFILOJ@textLabel1?$AA@ 10029cb4     launcheditordlg.obj
 0002:00009cc0       ??_C@_0N@HPEGIJEE@textLabel1_2?$AA@ 10029cc0     launcheditordlg.obj
 0002:00009cd0       ??_C@_04ENDCGFED@wsid?$AA@ 10029cd0     launcheditordlg.obj
 0002:00009cd8       ??_C@_0N@GGFNLIAF@textLabel1_3?$AA@ 10029cd8     launcheditordlg.obj
 0002:00009ce8       ??_C@_06DLPHCPJA@wsname?$AA@ 10029ce8     launcheditordlg.obj
 0002:00009cf0       ??_C@_0N@DAAHBPID@textLabel1_5?$AA@ 10029cf0     launcheditordlg.obj
 0002:00009d00       ??_C@_0BB@NLNIGHKI@rebootoncsicrash?$AA@ 10029d00     launcheditordlg.obj
 0002:00009d14       ??_C@_07IBBCGPPB@layout6?$AA@ 10029d14     launcheditordlg.obj
 0002:00009d1c       ??_C@_05LCLENNFI@table?$AA@ 10029d1c     launcheditordlg.obj
 0002:00009d24       ??_C@_07OFHOKKPF@layout2?$AA@ 10029d24     launcheditordlg.obj
 0002:00009d2c       ??_C@_03BDGOHNNK@add?$AA@  10029d2c     launcheditordlg.obj
 0002:00009d30       ??_C@_06LEMKAMD@remove?$AA@ 10029d30     launcheditordlg.obj
 0002:00009d38       ??_C@_06HGDPHBDI@moveup?$AA@ 10029d38     launcheditordlg.obj
 0002:00009d40       ??_C@_08MPKHEKGJ@movedown?$AA@ 10029d40     launcheditordlg.obj
 0002:00009d4c       ??_C@_0BA@PCMIOLCH@launchEditorDlg?$AA@ 10029d4c     launcheditordlg.obj
 0002:00009d60       ??_C@_0EG@OLAAFGHO@?$DMh1?$DO?$DMp?5align?$DN?$CCcenter?$CC?$DOWorkstatio@ 10029d60     launcheditordlg.obj
 0002:00009da8       ??_C@_0N@JNDMMNFO@Workstation?3?$AA@ 10029da8     launcheditordlg.obj
 0002:00009db8       ??_C@_03GKJNMMDB@ID?3?$AA@ 10029db8     launcheditordlg.obj
 0002:00009dbc       ??_C@_0BP@NDPCACKM@This?5is?5the?5workstation?5number?$AA@ 10029dbc     launcheditordlg.obj
 0002:00009ddc       ??_C@_0CG@HILNEEOK@?$DMp?$DOThis?5is?5the?5workstation?5numbe@ 10029ddc     launcheditordlg.obj
 0002:00009e04       ??_C@_0CD@KPFAEHDP@Select?5a?5workstation?5from?5the?5li@ 10029e04     launcheditordlg.obj
 0002:00009e28       ??_C@_0CE@IDFKMLLJ@This?5is?5the?5workstation?5descript@ 10029e28     launcheditordlg.obj
 0002:00009e4c       ??_C@_0CL@EANGFLDB@?$DMp?$DOThis?5is?5the?5workstation?5descr@ 10029e4c     launcheditordlg.obj
 0002:00009e78       ??_C@_0M@IOFBJEBH@CSI?5Version?$AA@ 10029e78     launcheditordlg.obj
 0002:00009e84       ??_C@_05PDFMAOIG@csi32?$AA@ 10029e84     launcheditordlg.obj
 0002:00009e8c       ??_C@_05MPMPAMM@v4csi?$AA@ 10029e8c     launcheditordlg.obj
 0002:00009e94       ??_C@_05LONMCMNM@v3csi?$AA@ 10029e94     launcheditordlg.obj
 0002:00009e9c       ??_C@_05IDLMAFGM@v2csi?$AA@ 10029e9c     launcheditordlg.obj
 0002:00009ea4       ??_C@_0DG@CIMKBJMA@Which?5CSI?5version?5to?5run?5?$CIthis?5i@ 10029ea4     launcheditordlg.obj
 0002:00009ee0       ??_C@_0KJ@GHGFNMBB@?$DMp?$DOThis?5is?5the?5CSI?5version?5to?5ru@ 10029ee0     launcheditordlg.obj
 0002:00009f8c       ??_C@_0CA@DCNMMIDN@Reboot?5workstation?5on?5CSI?5crash?$AA@ 10029f8c     launcheditordlg.obj
 0002:00009fb0       ??_C@_0HC@NOCNMLML@?$DMp?$DOThis?5should?5not?5be?5used?5as?5a?5@ 10029fb0     launcheditordlg.obj
 0002:0000a028       ??_C@_0FO@HAGHJCPN@?$DMp?$DOThe?5list?5of?5applications?5this@ 1002a028     launcheditordlg.obj
 0002:0000a088       ??_C@_0DJH@BGHNOJKA@?$DMp?$DOThis?5is?5the?5list?5of?5applicati@ 1002a088     launcheditordlg.obj
 0002:0000a420       ??_C@_03LDFMNCOE@Add?$AA@  1002a420     launcheditordlg.obj
 0002:0000a424       ??_C@_0BP@IFNAFPPO@Add?5an?5application?5to?5the?5list?$AA@ 1002a424     launcheditordlg.obj
 0002:0000a444       ??_C@_0CG@FIGHIMMB@?$DMp?$DOAdd?5an?5application?5to?5the?5lis@ 1002a444     launcheditordlg.obj
 0002:0000a46c       ??_C@_06MEPBJJFP@Remove?$AA@ 1002a46c     launcheditordlg.obj
 0002:0000a474       ??_C@_0CL@EKKHLFFN@?$DMp?$DORemove?5an?5application?5from?5th@ 1002a474     launcheditordlg.obj
 0002:0000a4a0       ??_C@_09OINHJNMP@Duplicate?$AA@ 1002a4a0     launcheditordlg.obj
 0002:0000a4ac       ??_C@_0CM@ECBLKOHJ@?$DMp?$DODuplicate?5an?5application?5in?5t@ 1002a4ac     launcheditordlg.obj
 0002:0000a4d8       ??_C@_07DMGIOHNE@Move?5Up?$AA@ 1002a4d8     launcheditordlg.obj
 0002:0000a4e0       ??_C@_0CF@FACAKFIF@?$DMp?$DOMove?5this?5item?5up?5in?5the?5list@ 1002a4e0     launcheditordlg.obj
 0002:0000a508       ??_C@_09CEAAIKKP@Move?5Down?$AA@ 1002a508     launcheditordlg.obj
 0002:0000a514       ??_C@_0CH@IFNMBHDF@?$DMp?$DOMove?5this?5item?5down?5in?5the?5li@ 1002a514     launcheditordlg.obj
 0002:0000a548       ??_C@_0P@DMEOIADN@languageChange?$AA@ 1002a548     moc_dialog.obj
 0002:0000a564       ??_C@_0BB@PFEIHPGD@languageChange?$CI?$CJ?$AA@ 1002a564     moc_dialog.obj
 0002:0000a578       ??_C@_06IOAEHBNO@dialog?$AA@ 1002a578     moc_dialogimpl.obj
 0002:0000a580       ??_C@_08ONPFHDOC@fileDrop?$AA@ 1002a580     moc_fileDrop.obj
 0002:0000a598       ??_C@_09EHKNDLFF@cbChanged?$AA@ 1002a598     moc_fileDrop.obj
 0002:0000a5b0       ??_C@_0M@ENPIPCL@cbChanged?$CI?$CJ?$AA@ 1002a5b0     moc_fileDrop.obj
 0002:0000a5bc       ??_C@_01NKEKCIAE@?$AE?$AA@ 1002a5bc     moc_fileDrop.obj
 0002:0000a5cc       ??_C@_08CLMNHHKN@fileList?$AA@ 1002a5cc     moc_fileDrop.obj
 0002:0000a5e4       ??_C@_0BG@PNNFPDKG@fileList?$CIQStringList?$CJ?$AA@ 1002a5e4     moc_fileDrop.obj
 0002:0000a5fc       ??_C@_0M@EJOCAFGP@fileManager?$AA@ 1002a5fc     moc_fileManager.obj
 0002:0000a608       ??_C@_02PFEMMEEH@li?$AA@   1002a608     moc_fileManager.obj
 0002:0000a60c       ??_C@_0O@LAFKAPIP@QListViewItem?$AA@ 1002a60c     moc_fileManager.obj
 0002:0000a628       ??_C@_0L@JEEPNFMN@dirChanged?$AA@ 1002a628     moc_fileManager.obj
 0002:0000a634       ??_C@_05DPEMMMGC@files?$AA@ 1002a634     moc_fileManager.obj
 0002:0000a648       ??_C@_0L@OEFDOKAL@doFileList?$AA@ 1002a648     moc_fileManager.obj
 0002:0000a66c       ??_C@_0BL@MNGGOFFF@dirChanged?$CIQListViewItem?$CK?$CJ?$AA@ 1002a66c     moc_fileManager.obj
 0002:0000a688       ??_C@_0BI@LOIBEOBF@doFileList?$CIQStringList?$CJ?$AA@ 1002a688     moc_fileManager.obj
 0002:0000a6ac       ??_C@_07KMMNMMFF@command?$AA@ 1002a6ac     moc_fileManager.obj
 0002:0000a6c0       ??_C@_0BJ@FEFNJDLM@command?$CIQString?0QString?$CJ?$AA@ 1002a6c0     moc_fileManager.obj
 0002:0000a6f4       ??_C@_0P@BOJJIOAA@fromBaseDialog?$AA@ 1002a6f4     moc_frombasedialogimpl.obj
 0002:0000a704       ??_C@_0N@FKCFJEKO@launchEditor?$AA@ 1002a704     moc_launchEditor.obj
 0002:0000a720       ??_C@_0BD@EJCDKKHL@workstationChanged?$AA@ 1002a720     moc_launchEditor.obj
 0002:0000a740       ??_C@_0BB@EKKGKLEJ@navigateWSEditor?$AA@ 1002a740     moc_launchEditor.obj
 0002:0000a76c       ??_C@_0CD@CJCCFBIL@workstationChanged?$CIQListViewItem@ 1002a76c     moc_launchEditor.obj
 0002:0000a790       ??_C@_0BD@BCKHEMDJ@navigateWSEditor?$CI?$CJ?$AA@ 1002a790     moc_launchEditor.obj
 0002:0000a7e0       ??_C@_0M@JIPAAGFP@doDuplicate?$AA@ 1002a7e0     moc_launcheditordlgimpl.obj
 0002:0000a7f8       ??_C@_05KLNNABIL@doAdd?$AA@ 1002a7f8     moc_launcheditordlgimpl.obj
 0002:0000a80c       ??_C@_08LHNADADA@doRemove?$AA@ 1002a80c     moc_launcheditordlgimpl.obj
 0002:0000a824       ??_C@_0L@MBPIPIML@doMoveDown?$AA@ 1002a824     moc_launcheditordlgimpl.obj
 0002:0000a83c       ??_C@_08PCOOKHCL@doMoveUp?$AA@ 1002a83c     moc_launcheditordlgimpl.obj
 0002:0000a848       ??_C@_03DMHICLNI@row?$AA@  1002a848     moc_launcheditordlgimpl.obj
 0002:0000a84c       ??_C@_03HNOLNALI@col?$AA@  1002a84c     moc_launcheditordlgimpl.obj
 0002:0000a85c       ??_C@_0BC@EKGMLGJI@tableValueChanged?$AA@ 1002a85c     moc_launcheditordlgimpl.obj
 0002:0000a87c       ??_C@_0BA@GDDILBON@csiValueChanged?$AA@ 1002a87c     moc_launcheditordlgimpl.obj
 0002:0000a898       ??_C@_0BE@POBNEEEH@rebootoptionchanged?$AA@ 1002a898     moc_launcheditordlgimpl.obj
 0002:0000a910       ??_C@_0O@KGFIPEON@doDuplicate?$CI?$CJ?$AA@ 1002a910     moc_launcheditordlgimpl.obj
 0002:0000a920       ??_C@_07NNGIFCHI@doAdd?$CI?$CJ?$AA@ 1002a920     moc_launcheditordlgimpl.obj
 0002:0000a928       ??_C@_0L@ILIHDJDM@doRemove?$CI?$CJ?$AA@ 1002a928     moc_launcheditordlgimpl.obj
 0002:0000a934       ??_C@_0N@OJHADNOA@doMoveDown?$CI?$CJ?$AA@ 1002a934     moc_launcheditordlgimpl.obj
 0002:0000a944       ??_C@_0L@EMNKLBHP@doMoveUp?$CI?$CJ?$AA@ 1002a944     moc_launcheditordlgimpl.obj
 0002:0000a950       ??_C@_0BL@NKAGANNB@tableValueChanged?$CIint?0int?$CJ?$AA@ 1002a950     moc_launcheditordlgimpl.obj
 0002:0000a96c       ??_C@_0CA@MKNFEKHK@csiValueChanged?$CIconst?5QString?$CG?$CJ?$AA@ 1002a96c     moc_launcheditordlgimpl.obj
 0002:0000a98c       ??_C@_0BG@LMJBCKOF@rebootoptionchanged?$CI?$CJ?$AA@ 1002a98c     moc_launcheditordlgimpl.obj
 0002:0000a9bc       ??_C@_0L@HLCBPADJ@testPlugin?$AA@ 1002a9bc     moc_testPlugin.obj
 0002:0000aa58       ??_C@_0L@BNDBFDDC@doNavigate?$AA@ 1002aa58     moc_testPlugin.obj
 0002:0000aa70       ??_C@_06OOEBKKPD@doHelp?$AA@ 1002aa70     moc_testPlugin.obj
 0002:0000aa84       ??_C@_07NPFKIFLJ@doDirty?$AA@ 1002aa84     moc_testPlugin.obj
 0002:0000ab38       ??_C@_0P@HDFKEJDG@downloadFile?$CI?$CJ?$AA@ 1002ab38     moc_testPlugin.obj
 0002:0000ab48       ??_C@_0L@CMDHBPIC@lockFile?$CI?$CJ?$AA@ 1002ab48     moc_testPlugin.obj
 0002:0000ab54       ??_C@_0N@DMIDJMKF@uploadFile?$CI?$CJ?$AA@ 1002ab54     moc_testPlugin.obj
 0002:0000ab64       ??_C@_0N@COHMJIGN@unlockFile?$CI?$CJ?$AA@ 1002ab64     moc_testPlugin.obj
 0002:0000ab74       ??_C@_0M@BGHANKGE@unlockDir?$CI?$CJ?$AA@ 1002ab74     moc_testPlugin.obj
 0002:0000ab80       ??_C@_09BCKNFJIO@dbClear?$CI?$CJ?$AA@ 1002ab80     moc_testPlugin.obj
 0002:0000ab8c       ??_C@_0O@FILKIDJO@downloadDir?$CI?$CJ?$AA@ 1002ab8c     moc_testPlugin.obj
 0002:0000ab9c       ??_C@_0M@FOJNECDN@uploadDir?$CI?$CJ?$AA@ 1002ab9c     moc_testPlugin.obj
 0002:0000aba8       ??_C@_0P@GDMOMJEG@checkoutFile?$CI?$CJ?$AA@ 1002aba8     moc_testPlugin.obj
 0002:0000abb8       ??_C@_0O@BGEAKJAE@checkoutDir?$CI?$CJ?$AA@ 1002abb8     moc_testPlugin.obj
 0002:0000abc8       ??_C@_05PKFEOGII@dir?$CI?$CJ?$AA@ 1002abc8     moc_testPlugin.obj
 0002:0000abd0       ??_C@_0N@GNAKMBLN@doNavigate?$CI?$CJ?$AA@ 1002abd0     moc_testPlugin.obj
 0002:0000abe0       ??_C@_08HLIKJOHK@doHelp?$CI?$CJ?$AA@ 1002abe0     moc_testPlugin.obj
 0002:0000abec       ??_C@_09NKMNDFLH@doDirty?$CI?$CJ?$AA@ 1002abec     moc_testPlugin.obj
 0002:0000ac10       ??_C@_0BD@NJPDGLIO@testPluginFromBase?$AA@ 1002ac10     moc_testPluginFromBase.obj
 0002:0000ac30       ??_C@_0O@ICGINNG@downloadFileS?$AA@ 1002ac30     moc_testPluginFromBase.obj
 0002:0000ac4c       ??_C@_09GAPIDBOP@lockFileS?$AA@ 1002ac4c     moc_testPluginFromBase.obj
 0002:0000ac64       ??_C@_0M@OABEMHF@uploadFileS?$AA@ 1002ac64     moc_testPluginFromBase.obj
 0002:0000ac7c       ??_C@_0M@EGOMNECM@unlockFileS?$AA@ 1002ac7c     moc_testPluginFromBase.obj
 0002:0000ac94       ??_C@_0L@JCGMBJIO@unlockDirS?$AA@ 1002ac94     moc_testPluginFromBase.obj
 0002:0000acac       ??_C@_08JEMJOGAI@dbClearS?$AA@ 1002acac     moc_testPluginFromBase.obj
 0002:0000acc4       ??_C@_0N@FMLGLHGM@downloadDirS?$AA@ 1002acc4     moc_testPluginFromBase.obj
 0002:0000ace0       ??_C@_0L@MNMCALCJ@uploadDirS?$AA@ 1002ace0     moc_testPluginFromBase.obj
 0002:0000acf8       ??_C@_0O@EGNMKHEM@checkoutFileS?$AA@ 1002acf8     moc_testPluginFromBase.obj
 0002:0000ad14       ??_C@_0N@KCBPHJIO@checkoutDirS?$AA@ 1002ad14     moc_testPluginFromBase.obj
 0002:0000ad30       ??_C@_04NFKCNDEP@dirS?$AA@ 1002ad30     moc_testPluginFromBase.obj
 0002:0000ad44       ??_C@_0M@FJFMGOEE@doNavigateS?$AA@ 1002ad44     moc_testPluginFromBase.obj
 0002:0000ad5c       ??_C@_07LFMMOMJL@doHelpS?$AA@ 1002ad5c     moc_testPluginFromBase.obj
 0002:0000ad70       ??_C@_08CDPEFPDK@doDirtyS?$AA@ 1002ad70     moc_testPluginFromBase.obj
 0002:0000ad88       ??_C@_08BKPAKJMN@doCleanS?$AA@ 1002ad88     moc_testPluginFromBase.obj
 0002:0000ae4c       ??_C@_0BA@DGHDBNJB@downloadFileS?$CI?$CJ?$AA@ 1002ae4c     moc_testPluginFromBase.obj
 0002:0000ae5c       ??_C@_0M@PKCAAHFC@lockFileS?$CI?$CJ?$AA@ 1002ae5c     moc_testPluginFromBase.obj
 0002:0000ae68       ??_C@_0O@FPDKAGLK@uploadFileS?$CI?$CJ?$AA@ 1002ae68     moc_testPluginFromBase.obj
 0002:0000ae78       ??_C@_0O@MKJHLDDM@unlockFileS?$CI?$CJ?$AA@ 1002ae78     moc_testPluginFromBase.obj
 0002:0000ae88       ??_C@_0N@LDHDAHNK@unlockDirS?$CI?$CJ?$AA@ 1002ae88     moc_testPluginFromBase.obj
 0002:0000ae98       ??_C@_0L@PDKINBDP@dbClearS?$CI?$CJ?$AA@ 1002ae98     moc_testPluginFromBase.obj
 0002:0000aea4       ??_C@_0P@OOFFNGIB@downloadDirS?$CI?$CJ?$AA@ 1002aea4     moc_testPluginFromBase.obj
 0002:0000aeb4       ??_C@_0N@KBIMADBC@uploadDirS?$CI?$CJ?$AA@ 1002aeb4     moc_testPluginFromBase.obj
 0002:0000aec4       ??_C@_0BA@GGGGPICN@checkoutFileS?$CI?$CJ?$AA@ 1002aec4     moc_testPluginFromBase.obj
 0002:0000aed4       ??_C@_0P@POMBFGPB@checkoutDirS?$CI?$CJ?$AA@ 1002aed4     moc_testPluginFromBase.obj
 0002:0000aee4       ??_C@_06BKCDINLF@dirS?$CI?$CJ?$AA@ 1002aee4     moc_testPluginFromBase.obj
 0002:0000aeec       ??_C@_0O@EMAHBHLB@doNavigateS?$CI?$CJ?$AA@ 1002aeec     moc_testPluginFromBase.obj
 0002:0000aefc       ??_C@_09EJBBMAPN@doHelpS?$CI?$CJ?$AA@ 1002aefc     moc_testPluginFromBase.obj
 0002:0000af08       ??_C@_0L@KMGFDJFL@doDirtyS?$CI?$CJ?$AA@ 1002af08     moc_testPluginFromBase.obj
 0002:0000af14       ??_C@_0L@KDEGCAAM@doCleanS?$CI?$CJ?$AA@ 1002af14     moc_testPluginFromBase.obj
 0002:0000af20       ??_C@_0BH@COOFPPCE@workstationCustomTable?$AA@ 1002af20     moc_workstationCustomTable.obj
 0002:0000af44       ??_C@_0L@BCAIFHPG@sortColumn?$AA@ 1002af44     moc_workstationCustomTable.obj
 0002:0000af50       ??_C@_03EFEGFOOI@asc?$AA@  1002af50     moc_workstationCustomTable.obj
 0002:0000af60       ??_C@_04BHGNNCDJ@swap?$AA@ 1002af60     moc_workstationCustomTable.obj
 0002:0000af80       ??_C@_09OMEHJBAL@destroyed?$AA@ 1002af80     moc_workstationCustomTable.obj
 0002:0000afbc       ??_C@_0BA@FENDPOLN@sortColumn?$CIint?$CJ?$AA@ 1002afbc     moc_workstationCustomTable.obj
 0002:0000afcc       ??_C@_0BE@JOPJJAHE@sortColumn?$CIint?0int?$CJ?$AA@ 1002afcc     moc_workstationCustomTable.obj
 0002:0000afe0       ??_C@_0BI@MDCPDAFE@sortColumn?$CIint?0int?0int?$CJ?$AA@ 1002afe0     moc_workstationCustomTable.obj
 0002:0000aff8       ??_C@_0M@BGOEBOON@destroyed?$CI?$CJ?$AA@ 1002aff8     moc_workstationCustomTable.obj
 0002:0000b004       ??_C@_0BK@EHDCMPCH@workstationDockWindowBase?$AA@ 1002b004     moc_workstationdockwindow.obj
 0002:0000b038       ??_C@_0BG@BHKPEAB@workstationDockWindow?$AA@ 1002b038     moc_workstationdockwindowimpl.obj
 0002:0000b05c       ??_C@_0BB@FFKPNNIH@selectionChanged?$AA@ 1002b05c     moc_workstationdockwindowimpl.obj
 0002:0000b07c       ??_C@_0CB@BHPNGIPG@selectionChanged?$CIQListViewItem?$CK?$CJ@ 1002b07c     moc_workstationdockwindowimpl.obj
 0002:0000b0a0       ??_C@_0BC@BAGEEPPC@workstationEditor?$AA@ 1002b0a0     moc_workstationeditor.obj
 0002:0000b0cc       ??_C@_0BJ@CKOABCJL@workstationEditorDlgBase?$AA@ 1002b0cc     moc_workstationeditordlg.obj
 0002:0000b100       ??_C@_0BF@PEHJFBGL@workstationEditorDlg?$AA@ 1002b100     moc_workstationeditordlgimpl.obj
 0002:0000b178       ??_C@_0BO@DAALNPEL@workstationEditorNewWsDlgBase?$AA@ 1002b178     moc_workstationeditornewwsdlg.obj
 0002:0000b1b0       ??_C@_0BK@ILOCPGJI@workstationEditorNewWsDlg?$AA@ 1002b1b0     moc_workstationeditornewwsdlgimpl.obj
 0002:0000b1cc       ??_C@_0N@JCEOKFBF@xml_listview?$AA@ 1002b1cc     moc_xml_listview.obj
 0002:0000b1e8       ??_C@_09FEKNNPNC@startDrag?$AA@ 1002b1e8     moc_xml_listview.obj
 0002:0000b200       ??_C@_0BK@DBIDNBDN@startDrag?$CIQListViewItem?$CK?$CJ?$AA@ 1002b200     moc_xml_listview.obj
 0002:0000b220       ??_7workstationDockWindowBase@@6BQObject@@@ 1002b220     workstationdockwindow.obj
 0002:0000b3d8       ??_7workstationDockWindowBase@@6BQPaintDevice@@@ 1002b3d8     workstationdockwindow.obj
 0002:0000b3fc       ??_SQTabWidget@@6BQObject@@@ 1002b3fc     workstationdockwindow.obj
 0002:0000b5d0       ??_SQTabWidget@@6BQPaintDevice@@@ 1002b5d0     workstationdockwindow.obj
 0002:0000b5f0       ??_C@_0CA@JAPGFBLL@workstationDockWindowBaseLayout?$AA@ 1002b5f0     workstationdockwindow.obj
 0002:0000b610       ??_C@_0L@NNPJCPDK@tabWidget2?$AA@ 1002b610     workstationdockwindow.obj
 0002:0000b61c       ??_C@_03CEDILPBK@tab?$AA@  1002b61c     workstationdockwindow.obj
 0002:0000b620       ??_C@_09PEOMDABK@tabLayout?$AA@ 1002b620     workstationdockwindow.obj
 0002:0000b62c       ??_C@_02DIBGMKNJ@lv?$AA@   1002b62c     workstationdockwindow.obj
 0002:0000b630       ??_C@_0N@LMIHDJBC@Workstations?$AA@ 1002b630     workstationdockwindow.obj
 0002:0000b644       ??_7workstationEditorDlgBase@@6BQObject@@@ 1002b644     workstationeditordlg.obj
 0002:0000b7fc       ??_7workstationEditorDlgBase@@6BQPaintDevice@@@ 1002b7fc     workstationeditordlg.obj
 0002:0000b81c       ??_C@_0BP@EAMJBADM@workstationEditorDlgBaseLayout?$AA@ 1002b81c     workstationeditordlg.obj
 0002:0000b83c       ??_C@_08BADCPAJD@layout10?$AA@ 1002b83c     workstationeditordlg.obj
 0002:0000b848       ??_C@_0DD@CCJBEADE@?$DMh1?$DO?$DMp?5align?$DN?$CCcenter?$CC?$DOWorkstatio@ 1002b848     workstationeditordlg.obj
 0002:0000b880       ??_7workstationEditorNewWsDlgBase@@6BQObject@@@ 1002b880     workstationeditornewwsdlg.obj
 0002:0000ba44       ??_7workstationEditorNewWsDlgBase@@6BQPaintDevice@@@ 1002ba44     workstationeditornewwsdlg.obj
 0002:0000ba6c       ??_SQButtonGroup@@6BQObject@@@ 1002ba6c     workstationeditornewwsdlg.obj
 0002:0000bc5c       ??_SQButtonGroup@@6BQPaintDevice@@@ 1002bc5c     workstationeditornewwsdlg.obj
 0002:0000bc84       ??_SQRadioButton@@6BQObject@@@ 1002bc84     workstationeditornewwsdlg.obj
 0002:0000be68       ??_SQRadioButton@@6BQPaintDevice@@@ 1002be68     workstationeditornewwsdlg.obj
 0002:0000be88       ??_C@_0CE@FDLNMAOG@workstationEditorNewWsDlgBaseLay@ 1002be88     workstationeditornewwsdlg.obj
 0002:0000beac       ??_C@_0N@OMGLLDMN@buttonGroup2?$AA@ 1002beac     workstationeditornewwsdlg.obj
 0002:0000bebc       ??_C@_0L@OCCDJBFM@layout14_2?$AA@ 1002bebc     workstationeditornewwsdlg.obj
 0002:0000bec8       ??_C@_0M@PPJNHBMP@description?$AA@ 1002bec8     workstationeditornewwsdlg.obj
 0002:0000bed4       ??_C@_09LKOFGHOI@layout8_2?$AA@ 1002bed4     workstationeditornewwsdlg.obj
 0002:0000bee0       ??_C@_0N@BGIEFLEH@buttonGroup8?$AA@ 1002bee0     workstationeditornewwsdlg.obj
 0002:0000bef0       ??_C@_06DGDLPBAN@client?$AA@ 1002bef0     workstationeditornewwsdlg.obj
 0002:0000bef8       ??_C@_06NCODBMHO@driver?$AA@ 1002bef8     workstationeditornewwsdlg.obj
 0002:0000bf00       ??_C@_04EHLGOKLJ@both?$AA@ 1002bf00     workstationeditornewwsdlg.obj
 0002:0000bf08       ??_C@_08MBPAELNK@layout19?$AA@ 1002bf08     workstationeditornewwsdlg.obj
 0002:0000bf14       ??_C@_08DKBDHOFF@buttonOk?$AA@ 1002bf14     workstationeditornewwsdlg.obj
 0002:0000bf20       ??_C@_0N@OLKBNHFJ@buttonCancel?$AA@ 1002bf20     workstationeditornewwsdlg.obj
 0002:0000bf30       ??_C@_09DMINLBG@1accept?$CI?$CJ?$AA@ 1002bf30     workstationeditornewwsdlg.obj
 0002:0000bf3c       ??_C@_09OCDCAEKE@1reject?$CI?$CJ?$AA@ 1002bf3c     workstationeditornewwsdlg.obj
 0002:0000bf48       ??_C@_0BH@MMFOGCFD@Create?5New?5Workstation?$AA@ 1002bf48     workstationeditornewwsdlg.obj
 0002:0000bf60       ??_C@_0BE@IPMACFBG@Workstation?5Details?$AA@ 1002bf60     workstationeditornewwsdlg.obj
 0002:0000bf74       ??_C@_0BI@BJDIJOJG@ID?5?$CIWorkstation?5number?$CJ?$AA@ 1002bf74     workstationeditornewwsdlg.obj
 0002:0000bf8c       ??_C@_0M@OHKMKKDH@Description?$AA@ 1002bf8c     workstationeditornewwsdlg.obj
 0002:0000bf98       ??_C@_0P@DCDMOHIO@Basic?5Settings?$AA@ 1002bf98     workstationeditornewwsdlg.obj
 0002:0000bfa8       ??_C@_06PJIGMIJB@Client?$AA@ 1002bfa8     workstationeditornewwsdlg.obj
 0002:0000bfb0       ??_C@_06BNFOCFOC@Driver?$AA@ 1002bfb0     workstationeditornewwsdlg.obj
 0002:0000bfb8       ??_C@_0BH@IKCIKBGK@Both?5Client?5and?5Driver?$AA@ 1002bfb8     workstationeditornewwsdlg.obj
 0002:0000bfd0       ??_C@_03DDKJIMDC@?$CGOK?$AA@ 1002bfd0     workstationeditornewwsdlg.obj
 0002:0000bfd4       ??_C@_07JLEKEEPN@?$CGCancel?$AA@ 1002bfd4     workstationeditornewwsdlg.obj
 0002:0000bfe0       ??_7cfg_Table@@6BQObject@@@ 1002bfe0     cfg_widgets001:moc_cfg_Table.obj
 0002:0000c384       ??_7cfg_Table@@6BQPaintDevice@@@ 1002c384     cfg_widgets001:moc_cfg_Table.obj
 0002:0000c3a4       ??_C@_09PNEKGGBK@cfg_Table?$AA@ 1002c3a4     cfg_widgets001:moc_cfg_Table.obj
 0002:0000c3bc       ??_C@_0M@MOKGOAHM@deleteItems?$AA@ 1002c3bc     cfg_widgets001:moc_cfg_Table.obj
 0002:0000c3d4       ??_C@_0BA@FJBCKEJL@copyToClipboard?$AA@ 1002c3d4     cfg_widgets001:moc_cfg_Table.obj
 0002:0000c3f0       ??_C@_09CLMPBHDI@undoPaste?$AA@ 1002c3f0     cfg_widgets001:moc_cfg_Table.obj
 0002:0000c408       ??_C@_0P@FJGFLBMO@pasteClipboard?$AA@ 1002c408     cfg_widgets001:moc_cfg_Table.obj
 0002:0000c424       ??_C@_0BF@CDBOAHLL@clipBoardDataChanged?$AA@ 1002c424     cfg_widgets001:moc_cfg_Table.obj
 0002:0000c478       ??_C@_0O@FBJIJCJH@deleteItems?$CI?$CJ?$AA@ 1002c478     cfg_widgets001:moc_cfg_Table.obj
 0002:0000c488       ??_C@_0BC@DBBGOFIB@copyToClipboard?$CI?$CJ?$AA@ 1002c488     cfg_widgets001:moc_cfg_Table.obj
 0002:0000c49c       ??_C@_0M@OGFEJKEA@undoPaste?$CI?$CJ?$AA@ 1002c49c     cfg_widgets001:moc_cfg_Table.obj
 0002:0000c4a8       ??_C@_0BB@JLAHKIAM@pasteClipboard?$CI?$CJ?$AA@ 1002c4a8     cfg_widgets001:moc_cfg_Table.obj
 0002:0000c4bc       ??_C@_0BH@OLENEJHN@clipBoardDataChanged?$CI?$CJ?$AA@ 1002c4bc     cfg_widgets001:moc_cfg_Table.obj
 0002:0000c4e0       ??_C@_0L@OIBMJOP@dataPasted?$AA@ 1002c4e0     cfg_widgets001:moc_cfg_Table.obj
 0002:0000c4f8       ??_C@_0BD@IALCIEJE@clipboardDataValid?$AA@ 1002c4f8     cfg_widgets001:moc_cfg_Table.obj
 0002:0000c524       ??_C@_0N@EJEGBDAF@dataPasted?$CI?$CJ?$AA@ 1002c524     cfg_widgets001:moc_cfg_Table.obj
 0002:0000c534       ??_C@_0BJ@FABNKMFK@clipboardDataValid?$CIbool?$CJ?$AA@ 1002c534     cfg_widgets001:moc_cfg_Table.obj
 0002:0000c550       ??_C@_0BI@DKLEEDHJ@1clipBoardDataChanged?$CI?$CJ?$AA@ 1002c550     cfg_widgets001:cfg_Table.obj
 0002:0000c568       ??_C@_0BA@NOIFKKAG@2dataChanged?5?$CI?$CJ?$AA@ 1002c568     cfg_widgets001:cfg_Table.obj
 0002:0000c578       ??_C@_03MDIDAHKD@?$CGNo?$AA@ 1002c578     cfg_widgets001:cfg_Table.obj
 0002:0000c57c       ??_C@_04ILFHLBJA@?$CGYes?$AA@ 1002c57c     cfg_widgets001:cfg_Table.obj
 0002:0000c588       ??_C@_0EG@JCAEPHHD@Selected?5Area?5does?5not?5match?4?6Do@ 1002c588     cfg_widgets001:cfg_Table.obj
 0002:0000c5d0       ??_C@_0BB@LNOIOJNO@Database?5Edtitor?$AA@ 1002c5d0     cfg_widgets001:cfg_Table.obj
 0002:0000c5e4       ??_C@_0DO@OOICEDKL@int?5cfg_Table?3?3validateRow?$CIiRow?$CJ@ 1002c5e4     cfg_widgets001:cfg_Table.obj
 0002:0000c628       ??_C@_0EE@IEHIFONC@int?5cfg_Table?3?3validateRow?$CIint?5i@ 1002c628     cfg_widgets001:cfg_Table.obj
 0002:0000c670       ??_7configFile@@6B@        1002c670     pluginBase:configFile.obj
 0002:0000c6c4       ??_C@_09DDAHAMBK@CC_SYSTEM?$AA@ 1002c6c4     pluginBase:configFile.obj
 0002:0000c6d0       ??_C@_0CE@FNJGILFO@?2BBCTechnology?2ConfigurationClie@ 1002c6d0     pluginBase:configFile.obj
 0002:0000c6f4       ??_C@_04JKHNIKCB@TEMP?$AA@ 1002c6f4     pluginBase:configFile.obj
 0002:0000c6fc       ??_C@_0CG@EMLLFHBM@Can?8t?5lock?5a?5directory?5?9?5try?5che@ 1002c6fc     pluginBase:configFile.obj
 0002:0000c724       ??_C@_07FAHBEMBB@dirList?$AA@ 1002c724     pluginBase:configFile.obj
 0002:0000c72c       ??_C@_0BF@NFLBBMAC@Operations?5timed?5out?$AA@ 1002c72c     pluginBase:configFile.obj
 0002:0000c748       ??_7pluginBase@@6BQObject@@@ 1002c748     pluginBase:pluginBase.obj
 0002:0000c930       ??_7pluginBase@@6BQPaintDevice@@@ 1002c930     pluginBase:pluginBase.obj
 0002:0000c950       ??_C@_0L@CNPGCJO@pluginBase?$AA@ 1002c950     pluginBase:moc_pluginBase.obj
 0002:0000c974       ??_C@_0L@DMICJMMP@configFile?$AA@ 1002c974     pluginBase:moc_configFile.obj
 0002:0000c984       ??_7type_info@@6B@         1002c984     MSVCRT:ti_inst.obj
 0002:0000c988       __pDefaultRawDllMain       1002c988     MSVCRT:crtdll.obj
 0002:0000c988       __pRawDllMain              1002c988     MSVCRT:crtdll.obj
 0002:0000c998       __load_config_used         1002c998     MSVCRT:loadcfg.obj
 0002:0000c9e0       ??_R4dialog@@6BQObject@@@  1002c9e0     dialogimpl.obj
 0002:0000c9f4       ??_R3dialog@@8             1002c9f4     dialogimpl.obj
 0002:0000ca04       ??_R2dialog@@8             1002ca04     dialogimpl.obj
 0002:0000ca20       ??_R1A@?0A@EA@dialog@@8    1002ca20     dialogimpl.obj
 0002:0000ca3c       ??_R1A@?0A@EA@dialogBase@@8 1002ca3c     dialogimpl.obj
 0002:0000ca58       ??_R3dialogBase@@8         1002ca58     dialogimpl.obj
 0002:0000ca68       ??_R2dialogBase@@8         1002ca68     dialogimpl.obj
 0002:0000ca80       ??_R1A@?0A@EA@QWidget@@8   1002ca80     dialogimpl.obj
 0002:0000ca9c       ??_R3QWidget@@8            1002ca9c     dialogimpl.obj
 0002:0000caac       ??_R2QWidget@@8            1002caac     dialogimpl.obj
 0002:0000cac0       ??_R1A@?0A@EA@QObject@@8   1002cac0     dialogimpl.obj
 0002:0000cadc       ??_R3QObject@@8            1002cadc     dialogimpl.obj
 0002:0000caec       ??_R2QObject@@8            1002caec     dialogimpl.obj
 0002:0000caf8       ??_R13?0A@EA@Qt@@8         1002caf8     dialogimpl.obj
 0002:0000cb14       ??_R3Qt@@8                 1002cb14     dialogimpl.obj
 0002:0000cb24       ??_R2Qt@@8                 1002cb24     dialogimpl.obj
 0002:0000cb2c       ??_R1A@?0A@EA@Qt@@8        1002cb2c     dialogimpl.obj
 0002:0000cb48       ??_R1CI@?0A@EA@QPaintDevice@@8 1002cb48     dialogimpl.obj
 0002:0000cb64       ??_R3QPaintDevice@@8       1002cb64     dialogimpl.obj
 0002:0000cb74       ??_R2QPaintDevice@@8       1002cb74     dialogimpl.obj
 0002:0000cb7c       ??_R1A@?0A@EA@QPaintDevice@@8 1002cb7c     dialogimpl.obj
 0002:0000cb98       ??_R4dialog@@6BQPaintDevice@@@ 1002cb98     dialogimpl.obj
 0002:0000cbac       ??_R4fileDrop@@6BQObject@@@ 1002cbac     fileDrop.obj
 0002:0000cbc0       ??_R3fileDrop@@8           1002cbc0     fileDrop.obj
 0002:0000cbd0       ??_R2fileDrop@@8           1002cbd0     fileDrop.obj
 0002:0000cbf4       ??_R1A@?0A@EA@fileDrop@@8  1002cbf4     fileDrop.obj
 0002:0000cc10       ??_R1A@?0A@EA@QListView@@8 1002cc10     fileDrop.obj
 0002:0000cc2c       ??_R3QListView@@8          1002cc2c     fileDrop.obj
 0002:0000cc3c       ??_R2QListView@@8          1002cc3c     fileDrop.obj
 0002:0000cc5c       ??_R1A@?0A@EA@QScrollView@@8 1002cc5c     fileDrop.obj
 0002:0000cc78       ??_R3QScrollView@@8        1002cc78     fileDrop.obj
 0002:0000cc88       ??_R2QScrollView@@8        1002cc88     fileDrop.obj
 0002:0000cca4       ??_R1A@?0A@EA@QFrame@@8    1002cca4     fileDrop.obj
 0002:0000ccc0       ??_R3QFrame@@8             1002ccc0     fileDrop.obj
 0002:0000ccd0       ??_R2QFrame@@8             1002ccd0     fileDrop.obj
 0002:0000cce8       ??_R4fileDrop@@6BQPaintDevice@@@ 1002cce8     fileDrop.obj
 0002:0000ccfc       ??_R3QShared@@8            1002ccfc     fileManager.obj
 0002:0000cd0c       ??_R2QShared@@8            1002cd0c     fileManager.obj
 0002:0000cd14       ??_R1A@?0A@EA@QShared@@8   1002cd14     fileManager.obj
 0002:0000cd30       ??_R1A@?0A@EA@QGList@@8    1002cd30     fileManager.obj
 0002:0000cd4c       ??_R3QGList@@8             1002cd4c     fileManager.obj
 0002:0000cd5c       ??_R2QGList@@8             1002cd5c     fileManager.obj
 0002:0000cd68       ??_R1A@?0A@EA@QPtrCollection@@8 1002cd68     fileManager.obj
 0002:0000cd84       ??_R3QPtrCollection@@8     1002cd84     fileManager.obj
 0002:0000cd94       ??_R2QPtrCollection@@8     1002cd94     fileManager.obj
 0002:0000cd9c       ??_R4QLabel@@6BQObject@@@  1002cd9c     fileManager.obj
 0002:0000cdb0       ??_R3QLabel@@8             1002cdb0     fileManager.obj
 0002:0000cdc0       ??_R2QLabel@@8             1002cdc0     fileManager.obj
 0002:0000cddc       ??_R1A@?0A@EA@QLabel@@8    1002cddc     fileManager.obj
 0002:0000cdf8       ??_R4QLabel@@6BQPaintDevice@@@ 1002cdf8     fileManager.obj
 0002:0000ce0c       ??_R1A@?0A@EA@QLayoutItem@@8 1002ce0c     fileManager.obj
 0002:0000ce28       ??_R3QLayoutItem@@8        1002ce28     fileManager.obj
 0002:0000ce38       ??_R2QLayoutItem@@8        1002ce38     fileManager.obj
 0002:0000ce40       ??_R4QVBoxLayout@@6BQObject@@@ 1002ce40     fileManager.obj
 0002:0000ce54       ??_R3QVBoxLayout@@8        1002ce54     fileManager.obj
 0002:0000ce64       ??_R2QVBoxLayout@@8        1002ce64     fileManager.obj
 0002:0000ce80       ??_R1A@?0A@EA@QVBoxLayout@@8 1002ce80     fileManager.obj
 0002:0000ce9c       ??_R1A@?0A@EA@QBoxLayout@@8 1002ce9c     fileManager.obj
 0002:0000ceb8       ??_R3QBoxLayout@@8         1002ceb8     fileManager.obj
 0002:0000cec8       ??_R2QBoxLayout@@8         1002cec8     fileManager.obj
 0002:0000cee0       ??_R1A@?0A@EA@QLayout@@8   1002cee0     fileManager.obj
 0002:0000cefc       ??_R3QLayout@@8            1002cefc     fileManager.obj
 0002:0000cf0c       ??_R2QLayout@@8            1002cf0c     fileManager.obj
 0002:0000cf20       ??_R1CI@?0A@EA@QLayoutItem@@8 1002cf20     fileManager.obj
 0002:0000cf3c       ??_R4QVBoxLayout@@6BQLayoutItem@@@ 1002cf3c     fileManager.obj
 0002:0000cf50       ??_R4QListView@@6BQObject@@@ 1002cf50     fileManager.obj
 0002:0000cf64       ??_R4QListView@@6BQPaintDevice@@@ 1002cf64     fileManager.obj
 0002:0000cf78       ??_R4QListViewItem@@6B@    1002cf78     fileManager.obj
 0002:0000cf8c       ??_R3QListViewItem@@8      1002cf8c     fileManager.obj
 0002:0000cf9c       ??_R2QListViewItem@@8      1002cf9c     fileManager.obj
 0002:0000cfa8       ??_R1A@?0A@EA@QListViewItem@@8 1002cfa8     fileManager.obj
 0002:0000cfc4       ??_R4QSplitter@@6BQObject@@@ 1002cfc4     fileManager.obj
 0002:0000cfd8       ??_R3QSplitter@@8          1002cfd8     fileManager.obj
 0002:0000cfe8       ??_R2QSplitter@@8          1002cfe8     fileManager.obj
 0002:0000d004       ??_R1A@?0A@EA@QSplitter@@8 1002d004     fileManager.obj
 0002:0000d020       ??_R4QSplitter@@6BQPaintDevice@@@ 1002d020     fileManager.obj
 0002:0000d034       ??_R4QGuardedPtrPrivate@@6B@ 1002d034     fileManager.obj
 0002:0000d048       ??_R3QGuardedPtrPrivate@@8 1002d048     fileManager.obj
 0002:0000d058       ??_R2QGuardedPtrPrivate@@8 1002d058     fileManager.obj
 0002:0000d06c       ??_R1A@?0A@EA@QGuardedPtrPrivate@@8 1002d06c     fileManager.obj
 0002:0000d088       ??_R1CI@?0A@EA@QShared@@8  1002d088     fileManager.obj
 0002:0000d0a4       ??_R4QDockWindowList@@6B@  1002d0a4     fileManager.obj
 0002:0000d0b8       ??_R3QDockWindowList@@8    1002d0b8     fileManager.obj
 0002:0000d0c8       ??_R2QDockWindowList@@8    1002d0c8     fileManager.obj
 0002:0000d0dc       ??_R1A@?0A@EA@QDockWindowList@@8 1002d0dc     fileManager.obj
 0002:0000d0f8       ??_R1A@?0A@EA@?$QPtrList@VQDockWindow@@@@8 1002d0f8     fileManager.obj
 0002:0000d114       ??_R3?$QPtrList@VQDockWindow@@@@8 1002d114     fileManager.obj
 0002:0000d124       ??_R2?$QPtrList@VQDockWindow@@@@8 1002d124     fileManager.obj
 0002:0000d134       ??_R4QPopupMenuList@@6B@   1002d134     fileManager.obj
 0002:0000d148       ??_R3QPopupMenuList@@8     1002d148     fileManager.obj
 0002:0000d158       ??_R2QPopupMenuList@@8     1002d158     fileManager.obj
 0002:0000d16c       ??_R1A@?0A@EA@QPopupMenuList@@8 1002d16c     fileManager.obj
 0002:0000d188       ??_R1A@?0A@EA@?$QPtrList@VQPopupMenu@@@@8 1002d188     fileManager.obj
 0002:0000d1a4       ??_R3?$QPtrList@VQPopupMenu@@@@8 1002d1a4     fileManager.obj
 0002:0000d1b4       ??_R2?$QPtrList@VQPopupMenu@@@@8 1002d1b4     fileManager.obj
 0002:0000d1c4       ??_R4?$QPtrList@VQPopupMenu@@@@6B@ 1002d1c4     fileManager.obj
 0002:0000d1d8       ??_R4config_plugin_base@@6BQObject@@@ 1002d1d8     fileManager.obj
 0002:0000d1ec       ??_R3config_plugin_base@@8 1002d1ec     fileManager.obj
 0002:0000d1fc       ??_R2config_plugin_base@@8 1002d1fc     fileManager.obj
 0002:0000d214       ??_R1A@?0A@EA@config_plugin_base@@8 1002d214     fileManager.obj
 0002:0000d230       ??_R4config_plugin_base@@6BQPaintDevice@@@ 1002d230     fileManager.obj
 0002:0000d244       ??_R4fileManager@@6BQObject@@@ 1002d244     fileManager.obj
 0002:0000d258       ??_R3fileManager@@8        1002d258     fileManager.obj
 0002:0000d268       ??_R2fileManager@@8        1002d268     fileManager.obj
 0002:0000d284       ??_R1A@?0A@EA@fileManager@@8 1002d284     fileManager.obj
 0002:0000d2a0       ??_R4fileManager@@6BQPaintDevice@@@ 1002d2a0     fileManager.obj
 0002:0000d2b4       ??_R4QWidget@@6BQObject@@@ 1002d2b4     frombasedialog.obj
 0002:0000d2c8       ??_R4QWidget@@6BQPaintDevice@@@ 1002d2c8     frombasedialog.obj
 0002:0000d2dc       ??_R4QHBoxLayout@@6BQObject@@@ 1002d2dc     frombasedialog.obj
 0002:0000d2f0       ??_R3QHBoxLayout@@8        1002d2f0     frombasedialog.obj
 0002:0000d300       ??_R2QHBoxLayout@@8        1002d300     frombasedialog.obj
 0002:0000d31c       ??_R1A@?0A@EA@QHBoxLayout@@8 1002d31c     frombasedialog.obj
 0002:0000d338       ??_R4QHBoxLayout@@6BQLayoutItem@@@ 1002d338     frombasedialog.obj
 0002:0000d34c       ??_R4QListBox@@6BQObject@@@ 1002d34c     frombasedialog.obj
 0002:0000d360       ??_R3QListBox@@8           1002d360     frombasedialog.obj
 0002:0000d370       ??_R2QListBox@@8           1002d370     frombasedialog.obj
 0002:0000d390       ??_R1A@?0A@EA@QListBox@@8  1002d390     frombasedialog.obj
 0002:0000d3ac       ??_R4QListBox@@6BQPaintDevice@@@ 1002d3ac     frombasedialog.obj
 0002:0000d3c0       ??_R4QPushButton@@6BQObject@@@ 1002d3c0     frombasedialog.obj
 0002:0000d3d4       ??_R3QPushButton@@8        1002d3d4     frombasedialog.obj
 0002:0000d3e4       ??_R2QPushButton@@8        1002d3e4     frombasedialog.obj
 0002:0000d400       ??_R1A@?0A@EA@QPushButton@@8 1002d400     frombasedialog.obj
 0002:0000d41c       ??_R1A@?0A@EA@QButton@@8   1002d41c     frombasedialog.obj
 0002:0000d438       ??_R3QButton@@8            1002d438     frombasedialog.obj
 0002:0000d448       ??_R2QButton@@8            1002d448     frombasedialog.obj
 0002:0000d460       ??_R4QPushButton@@6BQPaintDevice@@@ 1002d460     frombasedialog.obj
 0002:0000d474       ??_R4QGroupBox@@6BQObject@@@ 1002d474     frombasedialog.obj
 0002:0000d488       ??_R3QGroupBox@@8          1002d488     frombasedialog.obj
 0002:0000d498       ??_R2QGroupBox@@8          1002d498     frombasedialog.obj
 0002:0000d4b4       ??_R1A@?0A@EA@QGroupBox@@8 1002d4b4     frombasedialog.obj
 0002:0000d4d0       ??_R4QGroupBox@@6BQPaintDevice@@@ 1002d4d0     frombasedialog.obj
 0002:0000d4e4       ??_R4QLineEdit@@6BQObject@@@ 1002d4e4     frombasedialog.obj
 0002:0000d4f8       ??_R3QLineEdit@@8          1002d4f8     frombasedialog.obj
 0002:0000d508       ??_R2QLineEdit@@8          1002d508     frombasedialog.obj
 0002:0000d524       ??_R1A@?0A@EA@QLineEdit@@8 1002d524     frombasedialog.obj
 0002:0000d540       ??_R4QLineEdit@@6BQPaintDevice@@@ 1002d540     frombasedialog.obj
 0002:0000d554       ??_R4QFrame@@6BQObject@@@  1002d554     frombasedialog.obj
 0002:0000d568       ??_R4QFrame@@6BQPaintDevice@@@ 1002d568     frombasedialog.obj
 0002:0000d57c       ??_R4fromBaseDialogBase@@6BQObject@@@ 1002d57c     frombasedialog.obj
 0002:0000d590       ??_R3fromBaseDialogBase@@8 1002d590     frombasedialog.obj
 0002:0000d5a0       ??_R2fromBaseDialogBase@@8 1002d5a0     frombasedialog.obj
 0002:0000d5b8       ??_R1A@?0A@EA@fromBaseDialogBase@@8 1002d5b8     frombasedialog.obj
 0002:0000d5d4       ??_R4fromBaseDialogBase@@6BQPaintDevice@@@ 1002d5d4     frombasedialog.obj
 0002:0000d5e8       ??_R4QSpacerItem@@6B@      1002d5e8     frombasedialog.obj
 0002:0000d5fc       ??_R3QSpacerItem@@8        1002d5fc     frombasedialog.obj
 0002:0000d60c       ??_R2QSpacerItem@@8        1002d60c     frombasedialog.obj
 0002:0000d618       ??_R1A@?0A@EA@QSpacerItem@@8 1002d618     frombasedialog.obj
 0002:0000d634       ??_R4fromBaseDialog@@6BQObject@@@ 1002d634     frombasedialogimpl.obj
 0002:0000d648       ??_R3fromBaseDialog@@8     1002d648     frombasedialogimpl.obj
 0002:0000d658       ??_R2fromBaseDialog@@8     1002d658     frombasedialogimpl.obj
 0002:0000d674       ??_R1A@?0A@EA@fromBaseDialog@@8 1002d674     frombasedialogimpl.obj
 0002:0000d690       ??_R4fromBaseDialog@@6BQPaintDevice@@@ 1002d690     frombasedialogimpl.obj
 0002:0000d6a4       ??_R4launchCustomTable@@6BQObject@@@ 1002d6a4     launchCustomTable.obj
 0002:0000d6b8       ??_R3launchCustomTable@@8  1002d6b8     launchCustomTable.obj
 0002:0000d6c8       ??_R2launchCustomTable@@8  1002d6c8     launchCustomTable.obj
 0002:0000d6f0       ??_R1A@?0A@EA@launchCustomTable@@8 1002d6f0     launchCustomTable.obj
 0002:0000d70c       ??_R1A@?0A@EA@cfg_Table@@8 1002d70c     launchCustomTable.obj
 0002:0000d728       ??_R3cfg_Table@@8          1002d728     launchCustomTable.obj
 0002:0000d738       ??_R2cfg_Table@@8          1002d738     launchCustomTable.obj
 0002:0000d75c       ??_R1A@?0A@EA@QTable@@8    1002d75c     launchCustomTable.obj
 0002:0000d778       ??_R3QTable@@8             1002d778     launchCustomTable.obj
 0002:0000d788       ??_R2QTable@@8             1002d788     launchCustomTable.obj
 0002:0000d7a8       ??_R4launchCustomTable@@6BQPaintDevice@@@ 1002d7a8     launchCustomTable.obj
 0002:0000d7bc       ??_R4QToolBar@@6BQObject@@@ 1002d7bc     launchEditor.obj
 0002:0000d7d0       ??_R3QToolBar@@8           1002d7d0     launchEditor.obj
 0002:0000d7e0       ??_R2QToolBar@@8           1002d7e0     launchEditor.obj
 0002:0000d800       ??_R1A@?0A@EA@QToolBar@@8  1002d800     launchEditor.obj
 0002:0000d81c       ??_R1A@?0A@EA@QDockWindow@@8 1002d81c     launchEditor.obj
 0002:0000d838       ??_R3QDockWindow@@8        1002d838     launchEditor.obj
 0002:0000d848       ??_R2QDockWindow@@8        1002d848     launchEditor.obj
 0002:0000d864       ??_R4QToolBar@@6BQPaintDevice@@@ 1002d864     launchEditor.obj
 0002:0000d878       ??_R4QPopupMenu@@6BQObject@@@ 1002d878     launchEditor.obj
 0002:0000d88c       ??_R3QPopupMenu@@8         1002d88c     launchEditor.obj
 0002:0000d89c       ??_R2QPopupMenu@@8         1002d89c     launchEditor.obj
 0002:0000d8bc       ??_R1A@?0A@EA@QPopupMenu@@8 1002d8bc     launchEditor.obj
 0002:0000d8d8       ??_R1IM@?0A@EA@QMenuData@@8 1002d8d8     launchEditor.obj
 0002:0000d8f4       ??_R3QMenuData@@8          1002d8f4     launchEditor.obj
 0002:0000d904       ??_R2QMenuData@@8          1002d904     launchEditor.obj
 0002:0000d90c       ??_R1A@?0A@EA@QMenuData@@8 1002d90c     launchEditor.obj
 0002:0000d928       ??_R4QPopupMenu@@6BQPaintDevice@@@ 1002d928     launchEditor.obj
 0002:0000d93c       ??_R4QPopupMenu@@6B@       1002d93c     launchEditor.obj
 0002:0000d950       ??_R4QDockWindow@@6BQObject@@@ 1002d950     launchEditor.obj
 0002:0000d964       ??_R4QDockWindow@@6BQPaintDevice@@@ 1002d964     launchEditor.obj
 0002:0000d978       ??_R4QAction@@6B@          1002d978     launchEditor.obj
 0002:0000d98c       ??_R3QAction@@8            1002d98c     launchEditor.obj
 0002:0000d99c       ??_R2QAction@@8            1002d99c     launchEditor.obj
 0002:0000d9ac       ??_R1A@?0A@EA@QAction@@8   1002d9ac     launchEditor.obj
 0002:0000d9c8       ??_R1A@?0A@EA@QGDict@@8    1002d9c8     launchEditor.obj
 0002:0000d9e4       ??_R3QGDict@@8             1002d9e4     launchEditor.obj
 0002:0000d9f4       ??_R2QGDict@@8             1002d9f4     launchEditor.obj
 0002:0000da00       ??_R4launchEditor@@6BQObject@@@ 1002da00     launchEditor.obj
 0002:0000da14       ??_R3launchEditor@@8       1002da14     launchEditor.obj
 0002:0000da24       ??_R2launchEditor@@8       1002da24     launchEditor.obj
 0002:0000da40       ??_R1A@?0A@EA@launchEditor@@8 1002da40     launchEditor.obj
 0002:0000da5c       ??_R4launchEditor@@6BQPaintDevice@@@ 1002da5c     launchEditor.obj
 0002:0000da70       ??_R4?$QDict@VQAction@@@@6B@ 1002da70     launchEditor.obj
 0002:0000da84       ??_R3?$QDict@VQAction@@@@8 1002da84     launchEditor.obj
 0002:0000da94       ??_R2?$QDict@VQAction@@@@8 1002da94     launchEditor.obj
 0002:0000daa4       ??_R1A@?0A@EA@?$QDict@VQAction@@@@8 1002daa4     launchEditor.obj
 0002:0000dac0       ??_R4QCheckTableItem@@6B@  1002dac0     launcheditordlgimpl.obj
 0002:0000dad4       ??_R3QCheckTableItem@@8    1002dad4     launcheditordlgimpl.obj
 0002:0000dae4       ??_R2QCheckTableItem@@8    1002dae4     launcheditordlgimpl.obj
 0002:0000daf4       ??_R1A@?0A@EA@QCheckTableItem@@8 1002daf4     launcheditordlgimpl.obj
 0002:0000db10       ??_R1A@?0A@EA@QTableItem@@8 1002db10     launcheditordlgimpl.obj
 0002:0000db2c       ??_R3QTableItem@@8         1002db2c     launcheditordlgimpl.obj
 0002:0000db3c       ??_R2QTableItem@@8         1002db3c     launcheditordlgimpl.obj
 0002:0000db48       ??_R4launchEditorDlg@@6BQObject@@@ 1002db48     launcheditordlgimpl.obj
 0002:0000db5c       ??_R3launchEditorDlg@@8    1002db5c     launcheditordlgimpl.obj
 0002:0000db6c       ??_R2launchEditorDlg@@8    1002db6c     launcheditordlgimpl.obj
 0002:0000db88       ??_R1A@?0A@EA@launchEditorDlg@@8 1002db88     launcheditordlgimpl.obj
 0002:0000dba4       ??_R1A@?0A@EA@launchEditorDlgBase@@8 1002dba4     launcheditordlgimpl.obj
 0002:0000dbc0       ??_R3launchEditorDlgBase@@8 1002dbc0     launcheditordlgimpl.obj
 0002:0000dbd0       ??_R2launchEditorDlgBase@@8 1002dbd0     launcheditordlgimpl.obj
 0002:0000dbe8       ??_R4launchEditorDlg@@6BQPaintDevice@@@ 1002dbe8     launcheditordlgimpl.obj
 0002:0000dbfc       ??_R4config_plugin_desc_base@@6B@ 1002dbfc     plugindesc.obj
 0002:0000dc10       ??_R3config_plugin_desc_base@@8 1002dc10     plugindesc.obj
 0002:0000dc20       ??_R2config_plugin_desc_base@@8 1002dc20     plugindesc.obj
 0002:0000dc28       ??_R1A@?0A@EA@config_plugin_desc_base@@8 1002dc28     plugindesc.obj
 0002:0000dc44       ??_R4plugindesc@@6B@       1002dc44     plugindesc.obj
 0002:0000dc58       ??_R3plugindesc@@8         1002dc58     plugindesc.obj
 0002:0000dc68       ??_R2plugindesc@@8         1002dc68     plugindesc.obj
 0002:0000dc74       ??_R1A@?0A@EA@plugindesc@@8 1002dc74     plugindesc.obj
 0002:0000dc90       ??_R4testPlugin@@6BQObject@@@ 1002dc90     testPlugin.obj
 0002:0000dca4       ??_R3testPlugin@@8         1002dca4     testPlugin.obj
 0002:0000dcb4       ??_R2testPlugin@@8         1002dcb4     testPlugin.obj
 0002:0000dcd0       ??_R1A@?0A@EA@testPlugin@@8 1002dcd0     testPlugin.obj
 0002:0000dcec       ??_R4testPlugin@@6BQPaintDevice@@@ 1002dcec     testPlugin.obj
 0002:0000dd00       ??_R4testPluginFromBase@@6BQObject@@@ 1002dd00     testPluginFromBase.obj
 0002:0000dd14       ??_R3testPluginFromBase@@8 1002dd14     testPluginFromBase.obj
 0002:0000dd24       ??_R2testPluginFromBase@@8 1002dd24     testPluginFromBase.obj
 0002:0000dd44       ??_R1A@?0A@EA@testPluginFromBase@@8 1002dd44     testPluginFromBase.obj
 0002:0000dd60       ??_R1A@?0A@EA@pluginBase@@8 1002dd60     testPluginFromBase.obj
 0002:0000dd7c       ??_R3pluginBase@@8         1002dd7c     testPluginFromBase.obj
 0002:0000dd8c       ??_R2pluginBase@@8         1002dd8c     testPluginFromBase.obj
 0002:0000dda8       ??_R4testPluginFromBase@@6BQPaintDevice@@@ 1002dda8     testPluginFromBase.obj
 0002:0000ddbc       ??_R4workstationCustomTable@@6BQObject@@@ 1002ddbc     workstationCustomTable.obj
 0002:0000ddd0       ??_R3workstationCustomTable@@8 1002ddd0     workstationCustomTable.obj
 0002:0000dde0       ??_R2workstationCustomTable@@8 1002dde0     workstationCustomTable.obj
 0002:0000de08       ??_R1A@?0A@EA@workstationCustomTable@@8 1002de08     workstationCustomTable.obj
 0002:0000de24       ??_R4workstationCustomTable@@6BQPaintDevice@@@ 1002de24     workstationCustomTable.obj
 0002:0000de38       ??_R4workstationDockWindow@@6BQObject@@@ 1002de38     workstationdockwindowimpl.obj
 0002:0000de4c       ??_R3workstationDockWindow@@8 1002de4c     workstationdockwindowimpl.obj
 0002:0000de5c       ??_R2workstationDockWindow@@8 1002de5c     workstationdockwindowimpl.obj
 0002:0000de78       ??_R1A@?0A@EA@workstationDockWindow@@8 1002de78     workstationdockwindowimpl.obj
 0002:0000de94       ??_R1A@?0A@EA@workstationDockWindowBase@@8 1002de94     workstationdockwindowimpl.obj
 0002:0000deb0       ??_R3workstationDockWindowBase@@8 1002deb0     workstationdockwindowimpl.obj
 0002:0000dec0       ??_R2workstationDockWindowBase@@8 1002dec0     workstationdockwindowimpl.obj
 0002:0000ded8       ??_R4workstationDockWindow@@6BQPaintDevice@@@ 1002ded8     workstationdockwindowimpl.obj
 0002:0000deec       ??_R4workstationEditor@@6BQObject@@@ 1002deec     workstationEditor.obj
 0002:0000df00       ??_R3workstationEditor@@8  1002df00     workstationEditor.obj
 0002:0000df10       ??_R2workstationEditor@@8  1002df10     workstationEditor.obj
 0002:0000df2c       ??_R1A@?0A@EA@workstationEditor@@8 1002df2c     workstationEditor.obj
 0002:0000df48       ??_R4workstationEditor@@6BQPaintDevice@@@ 1002df48     workstationEditor.obj
 0002:0000df5c       ??_R4workstationEditorDlg@@6BQObject@@@ 1002df5c     workstationeditordlgimpl.obj
 0002:0000df70       ??_R3workstationEditorDlg@@8 1002df70     workstationeditordlgimpl.obj
 0002:0000df80       ??_R2workstationEditorDlg@@8 1002df80     workstationeditordlgimpl.obj
 0002:0000df9c       ??_R1A@?0A@EA@workstationEditorDlg@@8 1002df9c     workstationeditordlgimpl.obj
 0002:0000dfb8       ??_R1A@?0A@EA@workstationEditorDlgBase@@8 1002dfb8     workstationeditordlgimpl.obj
 0002:0000dfd4       ??_R3workstationEditorDlgBase@@8 1002dfd4     workstationeditordlgimpl.obj
 0002:0000dfe4       ??_R2workstationEditorDlgBase@@8 1002dfe4     workstationeditordlgimpl.obj
 0002:0000dffc       ??_R4workstationEditorDlg@@6BQPaintDevice@@@ 1002dffc     workstationeditordlgimpl.obj
 0002:0000e010       ??_R4workstationEditorNewWsDlg@@6BQObject@@@ 1002e010     workstationeditornewwsdlgimpl.obj
 0002:0000e024       ??_R3workstationEditorNewWsDlg@@8 1002e024     workstationeditornewwsdlgimpl.obj
 0002:0000e034       ??_R2workstationEditorNewWsDlg@@8 1002e034     workstationeditornewwsdlgimpl.obj
 0002:0000e054       ??_R1A@?0A@EA@workstationEditorNewWsDlg@@8 1002e054     workstationeditornewwsdlgimpl.obj
 0002:0000e070       ??_R1A@?0A@EA@workstationEditorNewWsDlgBase@@8 1002e070     workstationeditornewwsdlgimpl.obj
 0002:0000e08c       ??_R3workstationEditorNewWsDlgBase@@8 1002e08c     workstationeditornewwsdlgimpl.obj
 0002:0000e09c       ??_R2workstationEditorNewWsDlgBase@@8 1002e09c     workstationeditornewwsdlgimpl.obj
 0002:0000e0b8       ??_R1A@?0A@EA@QDialog@@8   1002e0b8     workstationeditornewwsdlgimpl.obj
 0002:0000e0d4       ??_R3QDialog@@8            1002e0d4     workstationeditornewwsdlgimpl.obj
 0002:0000e0e4       ??_R2QDialog@@8            1002e0e4     workstationeditornewwsdlgimpl.obj
 0002:0000e0fc       ??_R4workstationEditorNewWsDlg@@6BQPaintDevice@@@ 1002e0fc     workstationeditornewwsdlgimpl.obj
 0002:0000e110       ??_R4QComboBox@@6BQObject@@@ 1002e110     workstationUserTableItem.obj
 0002:0000e124       ??_R3QComboBox@@8          1002e124     workstationUserTableItem.obj
 0002:0000e134       ??_R2QComboBox@@8          1002e134     workstationUserTableItem.obj
 0002:0000e14c       ??_R1A@?0A@EA@QComboBox@@8 1002e14c     workstationUserTableItem.obj
 0002:0000e168       ??_R4QComboBox@@6BQPaintDevice@@@ 1002e168     workstationUserTableItem.obj
 0002:0000e17c       ??_R4workstationUserTableItem@@6B@ 1002e17c     workstationUserTableItem.obj
 0002:0000e190       ??_R3workstationUserTableItem@@8 1002e190     workstationUserTableItem.obj
 0002:0000e1a0       ??_R2workstationUserTableItem@@8 1002e1a0     workstationUserTableItem.obj
 0002:0000e1b0       ??_R1A@?0A@EA@workstationUserTableItem@@8 1002e1b0     workstationUserTableItem.obj
 0002:0000e1cc       ??_R4xml_listview@@6BQObject@@@ 1002e1cc     xml_listview.obj
 0002:0000e1e0       ??_R3xml_listview@@8       1002e1e0     xml_listview.obj
 0002:0000e1f0       ??_R2xml_listview@@8       1002e1f0     xml_listview.obj
 0002:0000e214       ??_R1A@?0A@EA@xml_listview@@8 1002e214     xml_listview.obj
 0002:0000e230       ??_R4xml_listview@@6BQPaintDevice@@@ 1002e230     xml_listview.obj
 0002:0000e244       ??_R4dialogBase@@6BQObject@@@ 1002e244     dialog.obj
 0002:0000e258       ??_R4dialogBase@@6BQPaintDevice@@@ 1002e258     dialog.obj
 0002:0000e26c       ??_R4QCheckBox@@6BQObject@@@ 1002e26c     launcheditordlg.obj
 0002:0000e280       ??_R3QCheckBox@@8          1002e280     launcheditordlg.obj
 0002:0000e290       ??_R2QCheckBox@@8          1002e290     launcheditordlg.obj
 0002:0000e2ac       ??_R1A@?0A@EA@QCheckBox@@8 1002e2ac     launcheditordlg.obj
 0002:0000e2c8       ??_R4QCheckBox@@6BQPaintDevice@@@ 1002e2c8     launcheditordlg.obj
 0002:0000e2dc       ??_R4launchEditorDlgBase@@6BQObject@@@ 1002e2dc     launcheditordlg.obj
 0002:0000e2f0       ??_R4launchEditorDlgBase@@6BQPaintDevice@@@ 1002e2f0     launcheditordlg.obj
 0002:0000e304       ??_R4QTabWidget@@6BQObject@@@ 1002e304     workstationdockwindow.obj
 0002:0000e318       ??_R3QTabWidget@@8         1002e318     workstationdockwindow.obj
 0002:0000e328       ??_R2QTabWidget@@8         1002e328     workstationdockwindow.obj
 0002:0000e340       ??_R1A@?0A@EA@QTabWidget@@8 1002e340     workstationdockwindow.obj
 0002:0000e35c       ??_R4QTabWidget@@6BQPaintDevice@@@ 1002e35c     workstationdockwindow.obj
 0002:0000e370       ??_R4workstationDockWindowBase@@6BQObject@@@ 1002e370     workstationdockwindow.obj
 0002:0000e384       ??_R4workstationDockWindowBase@@6BQPaintDevice@@@ 1002e384     workstationdockwindow.obj
 0002:0000e398       ??_R4workstationEditorDlgBase@@6BQObject@@@ 1002e398     workstationeditordlg.obj
 0002:0000e3ac       ??_R4workstationEditorDlgBase@@6BQPaintDevice@@@ 1002e3ac     workstationeditordlg.obj
 0002:0000e3c0       ??_R4QButtonGroup@@6BQObject@@@ 1002e3c0     workstationeditornewwsdlg.obj
 0002:0000e3d4       ??_R3QButtonGroup@@8       1002e3d4     workstationeditornewwsdlg.obj
 0002:0000e3e4       ??_R2QButtonGroup@@8       1002e3e4     workstationeditornewwsdlg.obj
 0002:0000e404       ??_R1A@?0A@EA@QButtonGroup@@8 1002e404     workstationeditornewwsdlg.obj
 0002:0000e420       ??_R4QButtonGroup@@6BQPaintDevice@@@ 1002e420     workstationeditornewwsdlg.obj
 0002:0000e434       ??_R4QRadioButton@@6BQObject@@@ 1002e434     workstationeditornewwsdlg.obj
 0002:0000e448       ??_R3QRadioButton@@8       1002e448     workstationeditornewwsdlg.obj
 0002:0000e458       ??_R2QRadioButton@@8       1002e458     workstationeditornewwsdlg.obj
 0002:0000e474       ??_R1A@?0A@EA@QRadioButton@@8 1002e474     workstationeditornewwsdlg.obj
 0002:0000e490       ??_R4QRadioButton@@6BQPaintDevice@@@ 1002e490     workstationeditornewwsdlg.obj
 0002:0000e4a4       ??_R4workstationEditorNewWsDlgBase@@6BQObject@@@ 1002e4a4     workstationeditornewwsdlg.obj
 0002:0000e4b8       ??_R4workstationEditorNewWsDlgBase@@6BQPaintDevice@@@ 1002e4b8     workstationeditornewwsdlg.obj
 0002:0000e4cc       ??_R4cfg_Table@@6BQObject@@@ 1002e4cc     cfg_widgets001:moc_cfg_Table.obj
 0002:0000e4e0       ??_R4cfg_Table@@6BQPaintDevice@@@ 1002e4e0     cfg_widgets001:moc_cfg_Table.obj
 0002:0000e4f4       ??_R4configFile@@6B@       1002e4f4     pluginBase:configFile.obj
 0002:0000e508       ??_R3configFile@@8         1002e508     pluginBase:configFile.obj
 0002:0000e518       ??_R2configFile@@8         1002e518     pluginBase:configFile.obj
 0002:0000e528       ??_R1A@?0A@EA@configFile@@8 1002e528     pluginBase:configFile.obj
 0002:0000e544       ??_R4pluginBase@@6BQObject@@@ 1002e544     pluginBase:pluginBase.obj
 0002:0000e558       ??_R4pluginBase@@6BQPaintDevice@@@ 1002e558     pluginBase:pluginBase.obj
 0002:0000e56c       ??_R4type_info@@6B@        1002e56c     MSVCRT:ti_inst.obj
 0002:0000e580       ??_R3type_info@@8          1002e580     MSVCRT:ti_inst.obj
 0002:0000e590       ??_R2type_info@@8          1002e590     MSVCRT:ti_inst.obj
 0002:0000e598       ??_R1A@?0A@EA@type_info@@8 1002e598     MSVCRT:ti_inst.obj
 0002:0000e5b4       ___rtc_iaa                 1002e5b4     MSVCRT:initsect.obj
 0002:0000e5b8       ___rtc_izz                 1002e5b8     MSVCRT:initsect.obj
 0002:0000e5bc       ___rtc_taa                 1002e5bc     MSVCRT:initsect.obj
 0002:0000e5c0       ___rtc_tzz                 1002e5c0     MSVCRT:initsect.obj
 0002:00012728       __IMPORT_DESCRIPTOR_config_icons 10032728     config_icons:config_icons.dll
 0002:0001273c       __IMPORT_DESCRIPTOR_qt-mt323 1003273c     qt-mt323:qt-mt323.dll
 0002:00012750       __IMPORT_DESCRIPTOR_KERNEL32 10032750     kernel32:KERNEL32.dll
 0002:00012764       __IMPORT_DESCRIPTOR_MSVCR120 10032764     MSVCRT:MSVCR120.dll
 0002:00012778       __NULL_IMPORT_DESCRIPTOR   10032778     config_icons:config_icons.dll
 0003:00000eb0       ___security_cookie         10040eb0     MSVCRT:gs_cookie.obj
 0003:00000eb4       ___security_cookie_complement 10040eb4     MSVCRT:gs_cookie.obj
 0003:00000ec0       ___native_dllmain_reason   10040ec0     MSVCRT:natstart.obj
 0003:00000ec4       ??_R0?AVdialog@@@8         10040ec4     dialogimpl.obj
 0003:00000edc       ??_R0?AVdialogBase@@@8     10040edc     dialogimpl.obj
 0003:00000ef8       ??_R0?AVQWidget@@@8        10040ef8     dialogimpl.obj
 0003:00000f10       ??_R0?AVQObject@@@8        10040f10     dialogimpl.obj
 0003:00000f28       ??_R0?AVQt@@@8             10040f28     dialogimpl.obj
 0003:00000f3c       ??_R0?AVQPaintDevice@@@8   10040f3c     dialogimpl.obj
 0003:00000f58       ??_R0?AVfileDrop@@@8       10040f58     fileDrop.obj
 0003:00000f70       ??_R0?AVQListView@@@8      10040f70     fileDrop.obj
 0003:00000f88       ??_R0?AVQScrollView@@@8    10040f88     fileDrop.obj
 0003:00000fa4       ??_R0?AVQFrame@@@8         10040fa4     fileDrop.obj
 0003:00000fbc       ??_R0?AUQShared@@@8        10040fbc     fileManager.obj
 0003:00000fd4       ??_R0?AVQGList@@@8         10040fd4     fileManager.obj
 0003:00000fec       ??_R0?AVQPtrCollection@@@8 10040fec     fileManager.obj
 0003:0000100c       ??_R0?AVQLabel@@@8         1004100c     fileManager.obj
 0003:00001024       ??_R0?AVQLayoutItem@@@8    10041024     fileManager.obj
 0003:00001040       ??_R0?AVQVBoxLayout@@@8    10041040     fileManager.obj
 0003:0000105c       ??_R0?AVQBoxLayout@@@8     1004105c     fileManager.obj
 0003:00001078       ??_R0?AVQLayout@@@8        10041078     fileManager.obj
 0003:00001090       ??_R0?AVQListViewItem@@@8  10041090     fileManager.obj
 0003:000010ac       ??_R0?AVQSplitter@@@8      100410ac     fileManager.obj
 0003:000010c4       ??_R0?AVQGuardedPtrPrivate@@@8 100410c4     fileManager.obj
 0003:000010e8       ??_R0?AVQDockWindowList@@@8 100410e8     fileManager.obj
 0003:00001108       ??_R0?AV?$QPtrList@VQDockWindow@@@@@8 10041108     fileManager.obj
 0003:00001130       ??_R0?AVQPopupMenuList@@@8 10041130     fileManager.obj
 0003:00001150       ??_R0?AV?$QPtrList@VQPopupMenu@@@@@8 10041150     fileManager.obj
 0003:00001178       ??_R0?AVconfig_plugin_base@@@8 10041178     fileManager.obj
 0003:0000119c       ??_R0?AVfileManager@@@8    1004119c     fileManager.obj
 0003:000011b8       ??_R0?AVQHBoxLayout@@@8    100411b8     frombasedialog.obj
 0003:000011d4       ??_R0?AVQListBox@@@8       100411d4     frombasedialog.obj
 0003:000011ec       ??_R0?AVQPushButton@@@8    100411ec     frombasedialog.obj
 0003:00001208       ??_R0?AVQButton@@@8        10041208     frombasedialog.obj
 0003:00001220       ??_R0?AVQGroupBox@@@8      10041220     frombasedialog.obj
 0003:00001238       ??_R0?AVQLineEdit@@@8      10041238     frombasedialog.obj
 0003:00001250       ??_R0?AVfromBaseDialogBase@@@8 10041250     frombasedialog.obj
 0003:00001274       ??_R0?AVQSpacerItem@@@8    10041274     frombasedialog.obj
 0003:00001290       ??_R0?AVfromBaseDialog@@@8 10041290     frombasedialogimpl.obj
 0003:000012b0       ??_R0?AVlaunchCustomTable@@@8 100412b0     launchCustomTable.obj
 0003:000012d0       ??_R0?AVcfg_Table@@@8      100412d0     launchCustomTable.obj
 0003:000012e8       ??_R0?AVQTable@@@8         100412e8     launchCustomTable.obj
 0003:00001300       ??_R0?AVQToolBar@@@8       10041300     launchEditor.obj
 0003:00001318       ??_R0?AVQDockWindow@@@8    10041318     launchEditor.obj
 0003:00001334       ??_R0?AVQPopupMenu@@@8     10041334     launchEditor.obj
 0003:00001350       ??_R0?AVQMenuData@@@8      10041350     launchEditor.obj
 0003:00001368       ??_R0?AVQAction@@@8        10041368     launchEditor.obj
 0003:00001380       ??_R0?AVQGDict@@@8         10041380     launchEditor.obj
 0003:00001398       ??_R0?AVlaunchEditor@@@8   10041398     launchEditor.obj
 0003:000013b4       ??_R0?AV?$QDict@VQAction@@@@@8 100413b4     launchEditor.obj
 0003:000013d8       ??_R0?AVQCheckTableItem@@@8 100413d8     launcheditordlgimpl.obj
 0003:000013f8       ??_R0?AVQTableItem@@@8     100413f8     launcheditordlgimpl.obj
 0003:00001414       ??_R0?AVlaunchEditorDlg@@@8 10041414     launcheditordlgimpl.obj
 0003:00001434       ??_R0?AVlaunchEditorDlgBase@@@8 10041434     launcheditordlgimpl.obj
 0003:00001458       ??_R0?AVconfig_plugin_desc_base@@@8 10041458     plugindesc.obj
 0003:00001480       ??_R0?AVplugindesc@@@8     10041480     plugindesc.obj
 0003:0000149c       ??_R0?AVtestPlugin@@@8     1004149c     testPlugin.obj
 0003:000014b8       ??_R0?AVtestPluginFromBase@@@8 100414b8     testPluginFromBase.obj
 0003:000014dc       ??_R0?AVpluginBase@@@8     100414dc     testPluginFromBase.obj
 0003:000014f8       ??_R0?AVworkstationCustomTable@@@8 100414f8     workstationCustomTable.obj
 0003:00001520       ??_R0?AVworkstationDockWindow@@@8 10041520     workstationdockwindowimpl.obj
 0003:00001544       ??_R0?AVworkstationDockWindowBase@@@8 10041544     workstationdockwindowimpl.obj
 0003:0000156c       ??_R0?AVworkstationEditor@@@8 1004156c     workstationEditor.obj
 0003:0000158c       ??_R0?AVworkstationEditorDlg@@@8 1004158c     workstationeditordlgimpl.obj
 0003:000015b0       ??_R0?AVworkstationEditorDlgBase@@@8 100415b0     workstationeditordlgimpl.obj
 0003:000015d8       ??_R0?AVworkstationEditorNewWsDlg@@@8 100415d8     workstationeditornewwsdlgimpl.obj
 0003:00001600       ??_R0?AVworkstationEditorNewWsDlgBase@@@8 10041600     workstationeditornewwsdlgimpl.obj
 0003:0000162c       ??_R0?AVQDialog@@@8        1004162c     workstationeditornewwsdlgimpl.obj
 0003:00001644       ??_R0?AVQComboBox@@@8      10041644     workstationUserTableItem.obj
 0003:0000165c       ??_R0?AVworkstationUserTableItem@@@8 1004165c     workstationUserTableItem.obj
 0003:00001684       ??_R0?AVxml_listview@@@8   10041684     xml_listview.obj
 0003:000016a0       ??_R0?AVQCheckBox@@@8      100416a0     launcheditordlg.obj
 0003:000016b8       ??_R0?AVQTabWidget@@@8     100416b8     workstationdockwindow.obj
 0003:000016d4       ??_R0?AVQButtonGroup@@@8   100416d4     workstationeditornewwsdlg.obj
 0003:000016f0       ??_R0?AVQRadioButton@@@8   100416f0     workstationeditornewwsdlg.obj
 0003:0000170c       ??_R0?AVconfigFile@@@8     1004170c     pluginBase:configFile.obj
 0003:00001728       ??_R0?AVtype_info@@@8      10041728     MSVCRT:ti_inst.obj
 0003:00001740       ?metaObj@dialogBase@@0PAVQMetaObject@@A 10041740     moc_dialog.obj
 0003:00001748       ?metaObj@dialog@@0PAVQMetaObject@@A 10041748     moc_dialogimpl.obj
 0003:00001750       ?metaObj@fileDrop@@0PAVQMetaObject@@A 10041750     moc_fileDrop.obj
 0003:0000176c       ?metaObj@fileManager@@0PAVQMetaObject@@A 1004176c     moc_fileManager.obj
 0003:00001798       ?metaObj@fromBaseDialogBase@@0PAVQMetaObject@@A 10041798     moc_frombasedialog.obj
 0003:000017a0       ?metaObj@fromBaseDialog@@0PAVQMetaObject@@A 100417a0     moc_frombasedialogimpl.obj
 0003:000017a8       ?metaObj@launchEditor@@0PAVQMetaObject@@A 100417a8     moc_launchEditor.obj
 0003:000017d4       ?metaObj@launchEditorDlgBase@@0PAVQMetaObject@@A 100417d4     moc_launcheditordlg.obj
 0003:000017dc       ?metaObj@launchEditorDlg@@0PAVQMetaObject@@A 100417dc     moc_launcheditordlgimpl.obj
 0003:00001818       ?metaObj@testPlugin@@0PAVQMetaObject@@A 10041818     moc_testPlugin.obj
 0003:00001844       ?metaObj@testPluginFromBase@@0PAVQMetaObject@@A 10041844     moc_testPluginFromBase.obj
 0003:0000184c       ?metaObj@workstationCustomTable@@0PAVQMetaObject@@A 1004184c     moc_workstationCustomTable.obj
 0003:00001858       ?metaObj@workstationDockWindowBase@@0PAVQMetaObject@@A 10041858     moc_workstationdockwindow.obj
 0003:00001860       ?metaObj@workstationDockWindow@@0PAVQMetaObject@@A 10041860     moc_workstationdockwindowimpl.obj
 0003:0000187c       ?metaObj@workstationEditor@@0PAVQMetaObject@@A 1004187c     moc_workstationeditor.obj
 0003:000018a8       ?metaObj@workstationEditorDlgBase@@0PAVQMetaObject@@A 100418a8     moc_workstationeditordlg.obj
 0003:000018b0       ?metaObj@workstationEditorDlg@@0PAVQMetaObject@@A 100418b0     moc_workstationeditordlgimpl.obj
 0003:000018dc       ?metaObj@workstationEditorNewWsDlgBase@@0PAVQMetaObject@@A 100418dc     moc_workstationeditornewwsdlg.obj
 0003:000018e4       ?metaObj@workstationEditorNewWsDlg@@0PAVQMetaObject@@A 100418e4     moc_workstationeditornewwsdlgimpl.obj
 0003:000018ec       ?metaObj@xml_listview@@0PAVQMetaObject@@A 100418ec     moc_xml_listview.obj
 0003:000018f8       ?metaObj@cfg_Table@@0PAVQMetaObject@@A 100418f8     cfg_widgets001:moc_cfg_Table.obj
 0003:00001914       ?metaObj@pluginBase@@0PAVQMetaObject@@A 10041914     pluginBase:moc_pluginBase.obj
 0003:00001940       ?metaObj@configFile@@0PAVQMetaObject@@A 10041940     pluginBase:moc_configFile.obj
 0003:00001c70       ?__type_info_root_node@@3U__type_info_node@@A 10041c70     MSVCRT:tncleanup.obj
 0003:00001c78       ___native_startup_lock     10041c78     <common>
 0003:00001c7c       ___native_startup_state    10041c7c     <common>
 0003:00001c80       ___dyn_tls_init_callback   10041c80     <common>
 0003:00001c84       ___onexitend               10041c84     <common>
 0003:00001c88       ___onexitbegin             10041c88     <common>

 entry point at        0001:0001992e

 Static symbols

 0001:00000000       ??__EcleanUp_dialogBase@@YAXXZ 10001000 f   moc_dialog.obj
 0001:00000021       ??__EcleanUp_dialog@@YAXXZ 10001021 f   moc_dialogimpl.obj
 0001:00000042       ??__EcleanUp_fileDrop@@YAXXZ 10001042 f   moc_fileDrop.obj
 0001:00000063       ??__EcleanUp_fileManager@@YAXXZ 10001063 f   moc_fileManager.obj
 0001:00000084       ??__EcleanUp_fromBaseDialogBase@@YAXXZ 10001084 f   moc_frombasedialog.obj
 0001:000000a5       ??__EcleanUp_fromBaseDialog@@YAXXZ 100010a5 f   moc_frombasedialogimpl.obj
 0001:000000c6       ??__EcleanUp_launchEditor@@YAXXZ 100010c6 f   moc_launchEditor.obj
 0001:000000e7       ??__EcleanUp_launchEditorDlgBase@@YAXXZ 100010e7 f   moc_launcheditordlg.obj
 0001:00000108       ??__EcleanUp_launchEditorDlg@@YAXXZ 10001108 f   moc_launcheditordlgimpl.obj
 0001:00000129       ??__EcleanUp_testPlugin@@YAXXZ 10001129 f   moc_testPlugin.obj
 0001:0000014a       ??__EcleanUp_testPluginFromBase@@YAXXZ 1000114a f   moc_testPluginFromBase.obj
 0001:0000016b       ??__EcleanUp_workstationCustomTable@@YAXXZ 1000116b f   moc_workstationCustomTable.obj
 0001:0000018c       ??__EcleanUp_workstationDockWindowBase@@YAXXZ 1000118c f   moc_workstationdockwindow.obj
 0001:000001ad       ??__EcleanUp_workstationDockWindow@@YAXXZ 100011ad f   moc_workstationdockwindowimpl.obj
 0001:000001ce       ??__EcleanUp_workstationEditor@@YAXXZ 100011ce f   moc_workstationeditor.obj
 0001:000001ef       ??__EcleanUp_workstationEditorDlgBase@@YAXXZ 100011ef f   moc_workstationeditordlg.obj
 0001:00000210       ??__EcleanUp_workstationEditorDlg@@YAXXZ 10001210 f   moc_workstationeditordlgimpl.obj
 0001:00000231       ??__EcleanUp_workstationEditorNewWsDlgBase@@YAXXZ 10001231 f   moc_workstationeditornewwsdlg.obj
 0001:00000252       ??__EcleanUp_workstationEditorNewWsDlg@@YAXXZ 10001252 f   moc_workstationeditornewwsdlgimpl.obj
 0001:00000273       ??__EcleanUp_xml_listview@@YAXXZ 10001273 f   moc_xml_listview.obj
 0001:00000294       ??__EcleanUp_cfg_Table@@YAXXZ 10001294 f   cfg_widgets001:moc_cfg_Table.obj
 0001:000002c0       ??__EcleanUp_pluginBase@@YAXXZ 100012c0 f   pluginBase:moc_pluginBase.obj
 0001:000002f0       ??__EcleanUp_configFile@@YAXXZ 100012f0 f   pluginBase:moc_configFile.obj
 0001:00012150       $LN23                      10013150     moc_launcheditordlgimpl.obj
 0001:00012478       $LN23                      10013478     moc_testPlugin.obj
 0001:00012642       $LN24                      10013642     moc_testPluginFromBase.obj
 0001:0001709c       $LN12                      1001809c     pluginBase:configFile.obj
 0001:00019490       $$000000                   1001a490     MSVCRT:chkstk.obj
 0001:000196eb       _pre_c_init                1001a6eb f   MSVCRT:crtdll.obj
 0001:00019951       ___DllMainCRTStartup       1001a951 f   MSVCRT:crtdll.obj
 0001:00019be0       $$000000                   1001abe0     MSVCRT:sehprolg4.obj
 0001:00019ef0       __unwindfunclet$??0fileDrop@@QAE@PAVQWidget@@PBD@Z$0 1001aef0 f   fileDrop.obj
 0001:00019ef0       __unwindfunclet$??1xml_listview@@UAE@XZ$0 1001aef0 f   fileDrop.obj
 0001:00019ef9       __ehhandler$??0fileDrop@@QAE@PAVQWidget@@PBD@Z 1001aef9 f   fileDrop.obj
 0001:00019ef9       __ehhandler$??1xml_listview@@UAE@XZ 1001aef9 f   fileDrop.obj
 0001:00019f14       __unwindfunclet$?contextMenuEvent@fileDrop@@UAEXPAVQContextMenuEvent@@@Z$0 1001af14 f   fileDrop.obj
 0001:00019f20       __unwindfunclet$?contextMenuEvent@fileDrop@@UAEXPAVQContextMenuEvent@@@Z$1 1001af20 f   fileDrop.obj
 0001:00019f29       __unwindfunclet$?contextMenuEvent@fileDrop@@UAEXPAVQContextMenuEvent@@@Z$2 1001af29 f   fileDrop.obj
 0001:00019f32       __unwindfunclet$?contextMenuEvent@fileDrop@@UAEXPAVQContextMenuEvent@@@Z$3 1001af32 f   fileDrop.obj
 0001:00019f3b       __ehhandler$?contextMenuEvent@fileDrop@@UAEXPAVQContextMenuEvent@@@Z 1001af3b f   fileDrop.obj
 0001:00019f59       __unwindfunclet$?dropEvent@fileDrop@@UAEXPAVQDropEvent@@@Z$0 1001af59 f   fileDrop.obj
 0001:00019f62       __unwindfunclet$?dropEvent@fileDrop@@UAEXPAVQDropEvent@@@Z$1 1001af62 f   fileDrop.obj
 0001:00019f6b       __ehhandler$?dropEvent@fileDrop@@UAEXPAVQDropEvent@@@Z 1001af6b f   fileDrop.obj
 0001:00019f86       __unwindfunclet$??0?$QGuardedPtr@VQPopupMenu@@@@QAE@XZ$0 1001af86 f   fileManager.obj
 0001:00019f86       __unwindfunclet$??4?$QGuardedPtr@VQPopupMenu@@@@QAEAAV0@PAVQPopupMenu@@@Z$0 1001af86 f   fileManager.obj
 0001:00019f86       __unwindfunclet$??4?$QGuardedPtr@VQDockWindow@@@@QAEAAV0@PAVQDockWindow@@@Z$0 1001af86 f   fileManager.obj
 0001:00019f86       __unwindfunclet$??0?$QGuardedPtr@VQDockWindow@@@@QAE@XZ$0 1001af86 f   fileManager.obj
 0001:00019f90       __ehhandler$??4?$QGuardedPtr@VQDockWindow@@@@QAEAAV0@PAVQDockWindow@@@Z 1001af90 f   fileManager.obj
 0001:00019f90       __ehhandler$??4?$QGuardedPtr@VQPopupMenu@@@@QAEAAV0@PAVQPopupMenu@@@Z 1001af90 f   fileManager.obj
 0001:00019f90       __ehhandler$??0?$QGuardedPtr@VQDockWindow@@@@QAE@XZ 1001af90 f   fileManager.obj
 0001:00019f90       __ehhandler$??0?$QGuardedPtr@VQPopupMenu@@@@QAE@XZ 1001af90 f   fileManager.obj
 0001:00019fab       __unwindfunclet$??0config_plugin_base@@QAE@ABVQString@@00@Z$0 1001afab f   fileManager.obj
 0001:00019fb4       __unwindfunclet$??0config_plugin_base@@QAE@ABVQString@@00@Z$1 1001afb4 f   fileManager.obj
 0001:00019fc0       __unwindfunclet$??0config_plugin_base@@QAE@ABVQString@@00@Z$2 1001afc0 f   fileManager.obj
 0001:00019fcc       __unwindfunclet$??0config_plugin_base@@QAE@ABVQString@@00@Z$3 1001afcc f   fileManager.obj
 0001:00019fd8       __ehhandler$??0config_plugin_base@@QAE@ABVQString@@00@Z 1001afd8 f   fileManager.obj
 0001:00019ff3       __unwindfunclet$??0fileManager@@QAE@ABVQString@@00@Z$0 1001aff3 f   fileManager.obj
 0001:00019ffb       __unwindfunclet$??0fileManager@@QAE@ABVQString@@00@Z$1 1001affb f   fileManager.obj
 0001:0001a006       __unwindfunclet$??0fileManager@@QAE@ABVQString@@00@Z$2 1001b006 f   fileManager.obj
 0001:0001a011       __unwindfunclet$??0fileManager@@QAE@ABVQString@@00@Z$3 1001b011 f   fileManager.obj
 0001:0001a01f       __unwindfunclet$??0fileManager@@QAE@ABVQString@@00@Z$4 1001b01f f   fileManager.obj
 0001:0001a02e       __unwindfunclet$??0fileManager@@QAE@ABVQString@@00@Z$5 1001b02e f   fileManager.obj
 0001:0001a03d       __unwindfunclet$??0fileManager@@QAE@ABVQString@@00@Z$6 1001b03d f   fileManager.obj
 0001:0001a046       __unwindfunclet$??0fileManager@@QAE@ABVQString@@00@Z$7 1001b046 f   fileManager.obj
 0001:0001a04f       __unwindfunclet$??0fileManager@@QAE@ABVQString@@00@Z$8 1001b04f f   fileManager.obj
 0001:0001a058       __unwindfunclet$??0fileManager@@QAE@ABVQString@@00@Z$9 1001b058 f   fileManager.obj
 0001:0001a062       __unwindfunclet$??0fileManager@@QAE@ABVQString@@00@Z$10 1001b062 f   fileManager.obj
 0001:0001a06c       __unwindfunclet$??0fileManager@@QAE@ABVQString@@00@Z$11 1001b06c f   fileManager.obj
 0001:0001a075       __unwindfunclet$??0fileManager@@QAE@ABVQString@@00@Z$12 1001b075 f   fileManager.obj
 0001:0001a07f       __unwindfunclet$??0fileManager@@QAE@ABVQString@@00@Z$13 1001b07f f   fileManager.obj
 0001:0001a089       __unwindfunclet$??0fileManager@@QAE@ABVQString@@00@Z$14 1001b089 f   fileManager.obj
 0001:0001a092       __unwindfunclet$??0fileManager@@QAE@ABVQString@@00@Z$15 1001b092 f   fileManager.obj
 0001:0001a09c       __unwindfunclet$??0fileManager@@QAE@ABVQString@@00@Z$16 1001b09c f   fileManager.obj
 0001:0001a0a5       __unwindfunclet$??0fileManager@@QAE@ABVQString@@00@Z$17 1001b0a5 f   fileManager.obj
 0001:0001a0ae       __unwindfunclet$??0fileManager@@QAE@ABVQString@@00@Z$18 1001b0ae f   fileManager.obj
 0001:0001a0b7       __ehhandler$??0fileManager@@QAE@ABVQString@@00@Z 1001b0b7 f   fileManager.obj
 0001:0001a0d2       __unwindfunclet$??1?$QPtrList@VQPopupMenu@@@@UAE@XZ$0 1001b0d2 f   fileManager.obj
 0001:0001a0db       __ehhandler$??1?$QPtrList@VQPopupMenu@@@@UAE@XZ 1001b0db f   fileManager.obj
 0001:0001a0f6       __unwindfunclet$??1QDockWindowList@@UAE@XZ$0 1001b0f6 f   fileManager.obj
 0001:0001a0ff       __unwindfunclet$??1QDockWindowList@@UAE@XZ$1 1001b0ff f   fileManager.obj
 0001:0001a108       __ehhandler$??1QDockWindowList@@UAE@XZ 1001b108 f   fileManager.obj
 0001:0001a123       __unwindfunclet$??1QPopupMenuList@@UAE@XZ$0 1001b123 f   fileManager.obj
 0001:0001a12b       __ehhandler$??1QPopupMenuList@@UAE@XZ 1001b12b f   fileManager.obj
 0001:0001a146       __unwindfunclet$??1config_plugin_base@@UAE@XZ$0 1001b146 f   fileManager.obj
 0001:0001a14f       __unwindfunclet$??1config_plugin_base@@UAE@XZ$1 1001b14f f   fileManager.obj
 0001:0001a15b       __unwindfunclet$??1config_plugin_base@@UAE@XZ$2 1001b15b f   fileManager.obj
 0001:0001a167       __ehhandler$??1config_plugin_base@@UAE@XZ 1001b167 f   fileManager.obj
 0001:0001a182       __unwindfunclet$??1fileManager@@UAE@XZ$0 1001b182 f   fileManager.obj
 0001:0001a18a       __unwindfunclet$??1fileManager@@UAE@XZ$1 1001b18a f   fileManager.obj
 0001:0001a195       __unwindfunclet$??1fileManager@@UAE@XZ$2 1001b195 f   fileManager.obj
 0001:0001a1a0       __unwindfunclet$??1fileManager@@UAE@XZ$3 1001b1a0 f   fileManager.obj
 0001:0001a1ae       __unwindfunclet$??1fileManager@@UAE@XZ$4 1001b1ae f   fileManager.obj
 0001:0001a1bd       __unwindfunclet$??1fileManager@@UAE@XZ$5 1001b1bd f   fileManager.obj
 0001:0001a1cc       __ehhandler$??1fileManager@@UAE@XZ 1001b1cc f   fileManager.obj
 0001:0001a1e7       __unwindfunclet$?about@config_plugin_base@@UAE?AVQString@@XZ$0 1001b1e7 f   fileManager.obj
 0001:0001a1f0       __unwindfunclet$?about@config_plugin_base@@UAE?AVQString@@XZ$1 1001b1f0 f   fileManager.obj
 0001:0001a20a       __ehhandler$?about@config_plugin_base@@UAE?AVQString@@XZ 1001b20a f   fileManager.obj
 0001:0001a225       __unwindfunclet$?copyFile@fileManager@@AAEXABVQString@@0@Z$0 1001b225 f   fileManager.obj
 0001:0001a231       __unwindfunclet$?copyFile@fileManager@@AAEXABVQString@@0@Z$1 1001b231 f   fileManager.obj
 0001:0001a23d       __unwindfunclet$?copyFile@fileManager@@AAEXABVQString@@0@Z$2 1001b23d f   fileManager.obj
 0001:0001a249       __unwindfunclet$?copyFile@fileManager@@AAEXABVQString@@0@Z$3 1001b249 f   fileManager.obj
 0001:0001a255       __unwindfunclet$?copyFile@fileManager@@AAEXABVQString@@0@Z$4 1001b255 f   fileManager.obj
 0001:0001a261       __ehhandler$?copyFile@fileManager@@AAEXABVQString@@0@Z 1001b261 f   fileManager.obj
 0001:0001a289       __unwindfunclet$?dirChanged@fileManager@@QAEXPAVQListViewItem@@@Z$0 1001b289 f   fileManager.obj
 0001:0001a292       __unwindfunclet$?dirChanged@fileManager@@QAEXPAVQListViewItem@@@Z$1 1001b292 f   fileManager.obj
 0001:0001a29b       __unwindfunclet$?dirChanged@fileManager@@QAEXPAVQListViewItem@@@Z$2 1001b29b f   fileManager.obj
 0001:0001a2a4       __ehhandler$?dirChanged@fileManager@@QAEXPAVQListViewItem@@@Z 1001b2a4 f   fileManager.obj
 0001:0001a2bf       __unwindfunclet$?doFileList@fileManager@@QAEXVQStringList@@@Z$0 1001b2bf f   fileManager.obj
 0001:0001a2c8       __unwindfunclet$?doFileList@fileManager@@QAEXVQStringList@@@Z$1 1001b2c8 f   fileManager.obj
 0001:0001a2d1       __unwindfunclet$?doFileList@fileManager@@QAEXVQStringList@@@Z$2 1001b2d1 f   fileManager.obj
 0001:0001a2da       __unwindfunclet$?doFileList@fileManager@@QAEXVQStringList@@@Z$3 1001b2da f   fileManager.obj
 0001:0001a2e3       __unwindfunclet$?doFileList@fileManager@@QAEXVQStringList@@@Z$4 1001b2e3 f   fileManager.obj
 0001:0001a2ec       __unwindfunclet$?doFileList@fileManager@@QAEXVQStringList@@@Z$6 1001b2ec f   fileManager.obj
 0001:0001a2f5       __unwindfunclet$?doFileList@fileManager@@QAEXVQStringList@@@Z$8 1001b2f5 f   fileManager.obj
 0001:0001a2fe       __unwindfunclet$?doFileList@fileManager@@QAEXVQStringList@@@Z$9 1001b2fe f   fileManager.obj
 0001:0001a307       __unwindfunclet$?doFileList@fileManager@@QAEXVQStringList@@@Z$10 1001b307 f   fileManager.obj
 0001:0001a310       __ehhandler$?doFileList@fileManager@@QAEXVQStringList@@@Z 1001b310 f   fileManager.obj
 0001:0001a32b       __unwindfunclet$?reply@fileManager@@UAEXPAVresponse@@@Z$0 1001b32b f   fileManager.obj
 0001:0001a334       __unwindfunclet$?reply@fileManager@@UAEXPAVresponse@@@Z$1 1001b334 f   fileManager.obj
 0001:0001a33d       __unwindfunclet$?reply@fileManager@@UAEXPAVresponse@@@Z$2 1001b33d f   fileManager.obj
 0001:0001a346       __unwindfunclet$?reply@fileManager@@UAEXPAVresponse@@@Z$3 1001b346 f   fileManager.obj
 0001:0001a34f       __unwindfunclet$?reply@fileManager@@UAEXPAVresponse@@@Z$4 1001b34f f   fileManager.obj
 0001:0001a358       __unwindfunclet$?reply@fileManager@@UAEXPAVresponse@@@Z$5 1001b358 f   fileManager.obj
 0001:0001a364       __unwindfunclet$?reply@fileManager@@UAEXPAVresponse@@@Z$6 1001b364 f   fileManager.obj
 0001:0001a36d       __unwindfunclet$?reply@fileManager@@UAEXPAVresponse@@@Z$7 1001b36d f   fileManager.obj
 0001:0001a376       __unwindfunclet$?reply@fileManager@@UAEXPAVresponse@@@Z$8 1001b376 f   fileManager.obj
 0001:0001a37f       __unwindfunclet$?reply@fileManager@@UAEXPAVresponse@@@Z$9 1001b37f f   fileManager.obj
 0001:0001a38b       __unwindfunclet$?reply@fileManager@@UAEXPAVresponse@@@Z$10 1001b38b f   fileManager.obj
 0001:0001a394       __unwindfunclet$?reply@fileManager@@UAEXPAVresponse@@@Z$11 1001b394 f   fileManager.obj
 0001:0001a39d       __unwindfunclet$?reply@fileManager@@UAEXPAVresponse@@@Z$12 1001b39d f   fileManager.obj
 0001:0001a3a6       __unwindfunclet$?reply@fileManager@@UAEXPAVresponse@@@Z$13 1001b3a6 f   fileManager.obj
 0001:0001a3b2       __unwindfunclet$?reply@fileManager@@UAEXPAVresponse@@@Z$14 1001b3b2 f   fileManager.obj
 0001:0001a3bb       __unwindfunclet$?reply@fileManager@@UAEXPAVresponse@@@Z$15 1001b3bb f   fileManager.obj
 0001:0001a3c4       __unwindfunclet$?reply@fileManager@@UAEXPAVresponse@@@Z$16 1001b3c4 f   fileManager.obj
 0001:0001a3cd       __unwindfunclet$?reply@fileManager@@UAEXPAVresponse@@@Z$18 1001b3cd f   fileManager.obj
 0001:0001a3d6       __unwindfunclet$?reply@fileManager@@UAEXPAVresponse@@@Z$20 1001b3d6 f   fileManager.obj
 0001:0001a3df       __unwindfunclet$?reply@fileManager@@UAEXPAVresponse@@@Z$21 1001b3df f   fileManager.obj
 0001:0001a3eb       __unwindfunclet$?reply@fileManager@@UAEXPAVresponse@@@Z$22 1001b3eb f   fileManager.obj
 0001:0001a3f7       __unwindfunclet$?reply@fileManager@@UAEXPAVresponse@@@Z$23 1001b3f7 f   fileManager.obj
 0001:0001a400       __unwindfunclet$?reply@fileManager@@UAEXPAVresponse@@@Z$24 1001b400 f   fileManager.obj
 0001:0001a409       __unwindfunclet$?reply@fileManager@@UAEXPAVresponse@@@Z$25 1001b409 f   fileManager.obj
 0001:0001a412       __unwindfunclet$?reply@fileManager@@UAEXPAVresponse@@@Z$27 1001b412 f   fileManager.obj
 0001:0001a41b       __unwindfunclet$?reply@fileManager@@UAEXPAVresponse@@@Z$28 1001b41b f   fileManager.obj
 0001:0001a424       __unwindfunclet$?reply@fileManager@@UAEXPAVresponse@@@Z$29 1001b424 f   fileManager.obj
 0001:0001a42d       __unwindfunclet$?reply@fileManager@@UAEXPAVresponse@@@Z$30 1001b42d f   fileManager.obj
 0001:0001a436       __unwindfunclet$?reply@fileManager@@UAEXPAVresponse@@@Z$31 1001b436 f   fileManager.obj
 0001:0001a440       __unwindfunclet$?reply@fileManager@@UAEXPAVresponse@@@Z$32 1001b440 f   fileManager.obj
 0001:0001a449       __unwindfunclet$?reply@fileManager@@UAEXPAVresponse@@@Z$33 1001b449 f   fileManager.obj
 0001:0001a452       __unwindfunclet$?reply@fileManager@@UAEXPAVresponse@@@Z$34 1001b452 f   fileManager.obj
 0001:0001a45b       __unwindfunclet$?reply@fileManager@@UAEXPAVresponse@@@Z$35 1001b45b f   fileManager.obj
 0001:0001a464       __unwindfunclet$?reply@fileManager@@UAEXPAVresponse@@@Z$36 1001b464 f   fileManager.obj
 0001:0001a46d       __unwindfunclet$?reply@fileManager@@UAEXPAVresponse@@@Z$37 1001b46d f   fileManager.obj
 0001:0001a476       __unwindfunclet$?reply@fileManager@@UAEXPAVresponse@@@Z$38 1001b476 f   fileManager.obj
 0001:0001a47f       __unwindfunclet$?reply@fileManager@@UAEXPAVresponse@@@Z$40 1001b47f f   fileManager.obj
 0001:0001a48b       __unwindfunclet$?reply@fileManager@@UAEXPAVresponse@@@Z$41 1001b48b f   fileManager.obj
 0001:0001a495       __unwindfunclet$?reply@fileManager@@UAEXPAVresponse@@@Z$42 1001b495 f   fileManager.obj
 0001:0001a49e       __unwindfunclet$?reply@fileManager@@UAEXPAVresponse@@@Z$43 1001b49e f   fileManager.obj
 0001:0001a4a7       __unwindfunclet$?reply@fileManager@@UAEXPAVresponse@@@Z$44 1001b4a7 f   fileManager.obj
 0001:0001a4b0       __unwindfunclet$?reply@fileManager@@UAEXPAVresponse@@@Z$45 1001b4b0 f   fileManager.obj
 0001:0001a4b9       __unwindfunclet$?reply@fileManager@@UAEXPAVresponse@@@Z$46 1001b4b9 f   fileManager.obj
 0001:0001a4c2       __unwindfunclet$?reply@fileManager@@UAEXPAVresponse@@@Z$47 1001b4c2 f   fileManager.obj
 0001:0001a4cb       __unwindfunclet$?reply@fileManager@@UAEXPAVresponse@@@Z$48 1001b4cb f   fileManager.obj
 0001:0001a4d4       __unwindfunclet$?reply@fileManager@@UAEXPAVresponse@@@Z$50 1001b4d4 f   fileManager.obj
 0001:0001a4e0       __unwindfunclet$?reply@fileManager@@UAEXPAVresponse@@@Z$51 1001b4e0 f   fileManager.obj
 0001:0001a4e9       __unwindfunclet$?reply@fileManager@@UAEXPAVresponse@@@Z$52 1001b4e9 f   fileManager.obj
 0001:0001a4f2       __unwindfunclet$?reply@fileManager@@UAEXPAVresponse@@@Z$53 1001b4f2 f   fileManager.obj
 0001:0001a4fc       __unwindfunclet$?reply@fileManager@@UAEXPAVresponse@@@Z$54 1001b4fc f   fileManager.obj
 0001:0001a516       __unwindfunclet$?reply@fileManager@@UAEXPAVresponse@@@Z$55 1001b516 f   fileManager.obj
 0001:0001a530       __unwindfunclet$?reply@fileManager@@UAEXPAVresponse@@@Z$56 1001b530 f   fileManager.obj
 0001:0001a54a       __unwindfunclet$?reply@fileManager@@UAEXPAVresponse@@@Z$57 1001b54a f   fileManager.obj
 0001:0001a564       __unwindfunclet$?reply@fileManager@@UAEXPAVresponse@@@Z$58 1001b564 f   fileManager.obj
 0001:0001a570       __unwindfunclet$?reply@fileManager@@UAEXPAVresponse@@@Z$59 1001b570 f   fileManager.obj
 0001:0001a579       __unwindfunclet$?reply@fileManager@@UAEXPAVresponse@@@Z$60 1001b579 f   fileManager.obj
 0001:0001a582       __unwindfunclet$?reply@fileManager@@UAEXPAVresponse@@@Z$61 1001b582 f   fileManager.obj
 0001:0001a58b       __unwindfunclet$?reply@fileManager@@UAEXPAVresponse@@@Z$62 1001b58b f   fileManager.obj
 0001:0001a594       __unwindfunclet$?reply@fileManager@@UAEXPAVresponse@@@Z$63 1001b594 f   fileManager.obj
 0001:0001a5ae       __unwindfunclet$?reply@fileManager@@UAEXPAVresponse@@@Z$64 1001b5ae f   fileManager.obj
 0001:0001a5b7       __unwindfunclet$?reply@fileManager@@UAEXPAVresponse@@@Z$65 1001b5b7 f   fileManager.obj
 0001:0001a5c0       __unwindfunclet$?reply@fileManager@@UAEXPAVresponse@@@Z$67 1001b5c0 f   fileManager.obj
 0001:0001a5cc       __ehhandler$?reply@fileManager@@UAEXPAVresponse@@@Z 1001b5cc f   fileManager.obj
 0001:0001a5ea       __unwindfunclet$??0fromBaseDialogBase@@QAE@PAVQWidget@@PBDI@Z$0 1001b5ea f   frombasedialog.obj
 0001:0001a5f3       __unwindfunclet$??0fromBaseDialogBase@@QAE@PAVQWidget@@PBDI@Z$1 1001b5f3 f   frombasedialog.obj
 0001:0001a5fd       __unwindfunclet$??0fromBaseDialogBase@@QAE@PAVQWidget@@PBDI@Z$2 1001b5fd f   frombasedialog.obj
 0001:0001a607       __unwindfunclet$??0fromBaseDialogBase@@QAE@PAVQWidget@@PBDI@Z$3 1001b607 f   frombasedialog.obj
 0001:0001a611       __unwindfunclet$??0fromBaseDialogBase@@QAE@PAVQWidget@@PBDI@Z$4 1001b611 f   frombasedialog.obj
 0001:0001a61b       __unwindfunclet$??0fromBaseDialogBase@@QAE@PAVQWidget@@PBDI@Z$5 1001b61b f   frombasedialog.obj
 0001:0001a625       __unwindfunclet$??0fromBaseDialogBase@@QAE@PAVQWidget@@PBDI@Z$6 1001b625 f   frombasedialog.obj
 0001:0001a62f       __unwindfunclet$??0fromBaseDialogBase@@QAE@PAVQWidget@@PBDI@Z$7 1001b62f f   frombasedialog.obj
 0001:0001a639       __unwindfunclet$??0fromBaseDialogBase@@QAE@PAVQWidget@@PBDI@Z$8 1001b639 f   frombasedialog.obj
 0001:0001a643       __unwindfunclet$??0fromBaseDialogBase@@QAE@PAVQWidget@@PBDI@Z$9 1001b643 f   frombasedialog.obj
 0001:0001a64d       __unwindfunclet$??0fromBaseDialogBase@@QAE@PAVQWidget@@PBDI@Z$10 1001b64d f   frombasedialog.obj
 0001:0001a657       __unwindfunclet$??0fromBaseDialogBase@@QAE@PAVQWidget@@PBDI@Z$11 1001b657 f   frombasedialog.obj
 0001:0001a661       __unwindfunclet$??0fromBaseDialogBase@@QAE@PAVQWidget@@PBDI@Z$12 1001b661 f   frombasedialog.obj
 0001:0001a66b       __unwindfunclet$??0fromBaseDialogBase@@QAE@PAVQWidget@@PBDI@Z$13 1001b66b f   frombasedialog.obj
 0001:0001a675       __unwindfunclet$??0fromBaseDialogBase@@QAE@PAVQWidget@@PBDI@Z$14 1001b675 f   frombasedialog.obj
 0001:0001a67f       __unwindfunclet$??0fromBaseDialogBase@@QAE@PAVQWidget@@PBDI@Z$15 1001b67f f   frombasedialog.obj
 0001:0001a689       __unwindfunclet$??0fromBaseDialogBase@@QAE@PAVQWidget@@PBDI@Z$16 1001b689 f   frombasedialog.obj
 0001:0001a693       __unwindfunclet$??0fromBaseDialogBase@@QAE@PAVQWidget@@PBDI@Z$17 1001b693 f   frombasedialog.obj
 0001:0001a69d       __unwindfunclet$??0fromBaseDialogBase@@QAE@PAVQWidget@@PBDI@Z$18 1001b69d f   frombasedialog.obj
 0001:0001a6a7       __unwindfunclet$??0fromBaseDialogBase@@QAE@PAVQWidget@@PBDI@Z$19 1001b6a7 f   frombasedialog.obj
 0001:0001a6b1       __unwindfunclet$??0fromBaseDialogBase@@QAE@PAVQWidget@@PBDI@Z$20 1001b6b1 f   frombasedialog.obj
 0001:0001a6bb       __unwindfunclet$??0fromBaseDialogBase@@QAE@PAVQWidget@@PBDI@Z$21 1001b6bb f   frombasedialog.obj
 0001:0001a6c5       __unwindfunclet$??0fromBaseDialogBase@@QAE@PAVQWidget@@PBDI@Z$22 1001b6c5 f   frombasedialog.obj
 0001:0001a6cf       __unwindfunclet$??0fromBaseDialogBase@@QAE@PAVQWidget@@PBDI@Z$23 1001b6cf f   frombasedialog.obj
 0001:0001a6d9       __unwindfunclet$??0fromBaseDialogBase@@QAE@PAVQWidget@@PBDI@Z$24 1001b6d9 f   frombasedialog.obj
 0001:0001a6e3       __unwindfunclet$??0fromBaseDialogBase@@QAE@PAVQWidget@@PBDI@Z$25 1001b6e3 f   frombasedialog.obj
 0001:0001a6ed       __unwindfunclet$??0fromBaseDialogBase@@QAE@PAVQWidget@@PBDI@Z$26 1001b6ed f   frombasedialog.obj
 0001:0001a6f7       __unwindfunclet$??0fromBaseDialogBase@@QAE@PAVQWidget@@PBDI@Z$27 1001b6f7 f   frombasedialog.obj
 0001:0001a701       __unwindfunclet$??0fromBaseDialogBase@@QAE@PAVQWidget@@PBDI@Z$28 1001b701 f   frombasedialog.obj
 0001:0001a70b       __unwindfunclet$??0fromBaseDialogBase@@QAE@PAVQWidget@@PBDI@Z$29 1001b70b f   frombasedialog.obj
 0001:0001a715       __unwindfunclet$??0fromBaseDialogBase@@QAE@PAVQWidget@@PBDI@Z$30 1001b715 f   frombasedialog.obj
 0001:0001a71f       __unwindfunclet$??0fromBaseDialogBase@@QAE@PAVQWidget@@PBDI@Z$31 1001b71f f   frombasedialog.obj
 0001:0001a729       __unwindfunclet$??0fromBaseDialogBase@@QAE@PAVQWidget@@PBDI@Z$32 1001b729 f   frombasedialog.obj
 0001:0001a733       __unwindfunclet$??0fromBaseDialogBase@@QAE@PAVQWidget@@PBDI@Z$33 1001b733 f   frombasedialog.obj
 0001:0001a73d       __unwindfunclet$??0fromBaseDialogBase@@QAE@PAVQWidget@@PBDI@Z$34 1001b73d f   frombasedialog.obj
 0001:0001a747       __unwindfunclet$??0fromBaseDialogBase@@QAE@PAVQWidget@@PBDI@Z$35 1001b747 f   frombasedialog.obj
 0001:0001a751       __unwindfunclet$??0fromBaseDialogBase@@QAE@PAVQWidget@@PBDI@Z$36 1001b751 f   frombasedialog.obj
 0001:0001a75b       __unwindfunclet$??0fromBaseDialogBase@@QAE@PAVQWidget@@PBDI@Z$37 1001b75b f   frombasedialog.obj
 0001:0001a765       __unwindfunclet$??0fromBaseDialogBase@@QAE@PAVQWidget@@PBDI@Z$38 1001b765 f   frombasedialog.obj
 0001:0001a76f       __unwindfunclet$??0fromBaseDialogBase@@QAE@PAVQWidget@@PBDI@Z$39 1001b76f f   frombasedialog.obj
 0001:0001a779       __unwindfunclet$??0fromBaseDialogBase@@QAE@PAVQWidget@@PBDI@Z$40 1001b779 f   frombasedialog.obj
 0001:0001a783       __unwindfunclet$??0fromBaseDialogBase@@QAE@PAVQWidget@@PBDI@Z$41 1001b783 f   frombasedialog.obj
 0001:0001a78d       __unwindfunclet$??0fromBaseDialogBase@@QAE@PAVQWidget@@PBDI@Z$42 1001b78d f   frombasedialog.obj
 0001:0001a797       __unwindfunclet$??0fromBaseDialogBase@@QAE@PAVQWidget@@PBDI@Z$43 1001b797 f   frombasedialog.obj
 0001:0001a7a1       __unwindfunclet$??0fromBaseDialogBase@@QAE@PAVQWidget@@PBDI@Z$44 1001b7a1 f   frombasedialog.obj
 0001:0001a7ab       __unwindfunclet$??0fromBaseDialogBase@@QAE@PAVQWidget@@PBDI@Z$45 1001b7ab f   frombasedialog.obj
 0001:0001a7b5       __unwindfunclet$??0fromBaseDialogBase@@QAE@PAVQWidget@@PBDI@Z$46 1001b7b5 f   frombasedialog.obj
 0001:0001a7bf       __unwindfunclet$??0fromBaseDialogBase@@QAE@PAVQWidget@@PBDI@Z$47 1001b7bf f   frombasedialog.obj
 0001:0001a7c9       __unwindfunclet$??0fromBaseDialogBase@@QAE@PAVQWidget@@PBDI@Z$48 1001b7c9 f   frombasedialog.obj
 0001:0001a7d3       __unwindfunclet$??0fromBaseDialogBase@@QAE@PAVQWidget@@PBDI@Z$49 1001b7d3 f   frombasedialog.obj
 0001:0001a7dd       __unwindfunclet$??0fromBaseDialogBase@@QAE@PAVQWidget@@PBDI@Z$50 1001b7dd f   frombasedialog.obj
 0001:0001a7e7       __unwindfunclet$??0fromBaseDialogBase@@QAE@PAVQWidget@@PBDI@Z$51 1001b7e7 f   frombasedialog.obj
 0001:0001a7f1       __unwindfunclet$??0fromBaseDialogBase@@QAE@PAVQWidget@@PBDI@Z$52 1001b7f1 f   frombasedialog.obj
 0001:0001a7fb       __unwindfunclet$??0fromBaseDialogBase@@QAE@PAVQWidget@@PBDI@Z$53 1001b7fb f   frombasedialog.obj
 0001:0001a805       __unwindfunclet$??0fromBaseDialogBase@@QAE@PAVQWidget@@PBDI@Z$54 1001b805 f   frombasedialog.obj
 0001:0001a80f       __ehhandler$??0fromBaseDialogBase@@QAE@PAVQWidget@@PBDI@Z 1001b80f f   frombasedialog.obj
 0001:0001a82a       __unwindfunclet$?languageChange@fromBaseDialogBase@@MAEXXZ$0 1001b82a f   frombasedialog.obj
 0001:0001a833       __unwindfunclet$?languageChange@fromBaseDialogBase@@MAEXXZ$1 1001b833 f   frombasedialog.obj
 0001:0001a83c       __unwindfunclet$?languageChange@fromBaseDialogBase@@MAEXXZ$2 1001b83c f   frombasedialog.obj
 0001:0001a845       __unwindfunclet$?languageChange@fromBaseDialogBase@@MAEXXZ$3 1001b845 f   frombasedialog.obj
 0001:0001a84e       __unwindfunclet$?languageChange@fromBaseDialogBase@@MAEXXZ$4 1001b84e f   frombasedialog.obj
 0001:0001a857       __unwindfunclet$?languageChange@fromBaseDialogBase@@MAEXXZ$5 1001b857 f   frombasedialog.obj
 0001:0001a860       __unwindfunclet$?languageChange@fromBaseDialogBase@@MAEXXZ$6 1001b860 f   frombasedialog.obj
 0001:0001a869       __unwindfunclet$?languageChange@fromBaseDialogBase@@MAEXXZ$7 1001b869 f   frombasedialog.obj
 0001:0001a872       __unwindfunclet$?languageChange@fromBaseDialogBase@@MAEXXZ$8 1001b872 f   frombasedialog.obj
 0001:0001a87b       __unwindfunclet$?languageChange@fromBaseDialogBase@@MAEXXZ$9 1001b87b f   frombasedialog.obj
 0001:0001a884       __unwindfunclet$?languageChange@fromBaseDialogBase@@MAEXXZ$10 1001b884 f   frombasedialog.obj
 0001:0001a88d       __unwindfunclet$?languageChange@fromBaseDialogBase@@MAEXXZ$11 1001b88d f   frombasedialog.obj
 0001:0001a896       __unwindfunclet$?languageChange@fromBaseDialogBase@@MAEXXZ$12 1001b896 f   frombasedialog.obj
 0001:0001a89f       __unwindfunclet$?languageChange@fromBaseDialogBase@@MAEXXZ$13 1001b89f f   frombasedialog.obj
 0001:0001a8a8       __unwindfunclet$?languageChange@fromBaseDialogBase@@MAEXXZ$14 1001b8a8 f   frombasedialog.obj
 0001:0001a8b1       __unwindfunclet$?languageChange@fromBaseDialogBase@@MAEXXZ$15 1001b8b1 f   frombasedialog.obj
 0001:0001a8ba       __unwindfunclet$?languageChange@fromBaseDialogBase@@MAEXXZ$16 1001b8ba f   frombasedialog.obj
 0001:0001a8c3       __unwindfunclet$?languageChange@fromBaseDialogBase@@MAEXXZ$17 1001b8c3 f   frombasedialog.obj
 0001:0001a8cc       __unwindfunclet$?languageChange@fromBaseDialogBase@@MAEXXZ$18 1001b8cc f   frombasedialog.obj
 0001:0001a8d5       __unwindfunclet$?languageChange@fromBaseDialogBase@@MAEXXZ$19 1001b8d5 f   frombasedialog.obj
 0001:0001a8de       __unwindfunclet$?languageChange@fromBaseDialogBase@@MAEXXZ$20 1001b8de f   frombasedialog.obj
 0001:0001a8e7       __unwindfunclet$?languageChange@fromBaseDialogBase@@MAEXXZ$21 1001b8e7 f   frombasedialog.obj
 0001:0001a8f0       __unwindfunclet$?languageChange@fromBaseDialogBase@@MAEXXZ$22 1001b8f0 f   frombasedialog.obj
 0001:0001a8f9       __unwindfunclet$?languageChange@fromBaseDialogBase@@MAEXXZ$23 1001b8f9 f   frombasedialog.obj
 0001:0001a902       __ehhandler$?languageChange@fromBaseDialogBase@@MAEXXZ 1001b902 f   frombasedialog.obj
 0001:0001a91d       __unwindfunclet$??0launchCustomTable@@QAE@PAVQWidget@@PBD@Z$0 1001b91d f   launchCustomTable.obj
 0001:0001a925       __unwindfunclet$??0launchCustomTable@@QAE@PAVQWidget@@PBD@Z$1 1001b925 f   launchCustomTable.obj
 0001:0001a92e       __unwindfunclet$??0launchCustomTable@@QAE@PAVQWidget@@PBD@Z$2 1001b92e f   launchCustomTable.obj
 0001:0001a937       __unwindfunclet$??0launchCustomTable@@QAE@PAVQWidget@@PBD@Z$3 1001b937 f   launchCustomTable.obj
 0001:0001a940       __unwindfunclet$??0launchCustomTable@@QAE@PAVQWidget@@PBD@Z$4 1001b940 f   launchCustomTable.obj
 0001:0001a949       __unwindfunclet$??0launchCustomTable@@QAE@PAVQWidget@@PBD@Z$5 1001b949 f   launchCustomTable.obj
 0001:0001a952       __unwindfunclet$??0launchCustomTable@@QAE@PAVQWidget@@PBD@Z$6 1001b952 f   launchCustomTable.obj
 0001:0001a95b       __ehhandler$??0launchCustomTable@@QAE@PAVQWidget@@PBD@Z 1001b95b f   launchCustomTable.obj
 0001:0001a976       __unwindfunclet$??0launchEditor@@QAE@ABVQString@@00@Z$0 1001b976 f   launchEditor.obj
 0001:0001a97e       __unwindfunclet$??0launchEditor@@QAE@ABVQString@@00@Z$1 1001b97e f   launchEditor.obj
 0001:0001a989       __unwindfunclet$??0launchEditor@@QAE@ABVQString@@00@Z$2 1001b989 f   launchEditor.obj
 0001:0001a994       __unwindfunclet$??0launchEditor@@QAE@ABVQString@@00@Z$3 1001b994 f   launchEditor.obj
 0001:0001a9a2       __unwindfunclet$??0launchEditor@@QAE@ABVQString@@00@Z$4 1001b9a2 f   launchEditor.obj
 0001:0001a9b0       __unwindfunclet$??0launchEditor@@QAE@ABVQString@@00@Z$5 1001b9b0 f   launchEditor.obj
 0001:0001a9b9       __unwindfunclet$??0launchEditor@@QAE@ABVQString@@00@Z$6 1001b9b9 f   launchEditor.obj
 0001:0001a9c3       __unwindfunclet$??0launchEditor@@QAE@ABVQString@@00@Z$7 1001b9c3 f   launchEditor.obj
 0001:0001a9cd       __unwindfunclet$??0launchEditor@@QAE@ABVQString@@00@Z$8 1001b9cd f   launchEditor.obj
 0001:0001a9d7       __unwindfunclet$??0launchEditor@@QAE@ABVQString@@00@Z$9 1001b9d7 f   launchEditor.obj
 0001:0001a9e0       __unwindfunclet$??0launchEditor@@QAE@ABVQString@@00@Z$10 1001b9e0 f   launchEditor.obj
 0001:0001a9e9       __unwindfunclet$??0launchEditor@@QAE@ABVQString@@00@Z$11 1001b9e9 f   launchEditor.obj
 0001:0001a9f3       __unwindfunclet$??0launchEditor@@QAE@ABVQString@@00@Z$12 1001b9f3 f   launchEditor.obj
 0001:0001a9fc       __unwindfunclet$??0launchEditor@@QAE@ABVQString@@00@Z$13 1001b9fc f   launchEditor.obj
 0001:0001aa06       __unwindfunclet$??0launchEditor@@QAE@ABVQString@@00@Z$14 1001ba06 f   launchEditor.obj
 0001:0001aa10       __unwindfunclet$??0launchEditor@@QAE@ABVQString@@00@Z$15 1001ba10 f   launchEditor.obj
 0001:0001aa2a       __unwindfunclet$??0launchEditor@@QAE@ABVQString@@00@Z$16 1001ba2a f   launchEditor.obj
 0001:0001aa44       __unwindfunclet$??0launchEditor@@QAE@ABVQString@@00@Z$17 1001ba44 f   launchEditor.obj
 0001:0001aa5e       __unwindfunclet$??0launchEditor@@QAE@ABVQString@@00@Z$18 1001ba5e f   launchEditor.obj
 0001:0001aa78       __unwindfunclet$??0launchEditor@@QAE@ABVQString@@00@Z$20 1001ba78 f   launchEditor.obj
 0001:0001aa81       __unwindfunclet$??0launchEditor@@QAE@ABVQString@@00@Z$21 1001ba81 f   launchEditor.obj
 0001:0001aa8a       __unwindfunclet$??0launchEditor@@QAE@ABVQString@@00@Z$22 1001ba8a f   launchEditor.obj
 0001:0001aa93       __unwindfunclet$??0launchEditor@@QAE@ABVQString@@00@Z$23 1001ba93 f   launchEditor.obj
 0001:0001aa9d       __unwindfunclet$??0launchEditor@@QAE@ABVQString@@00@Z$24 1001ba9d f   launchEditor.obj
 0001:0001aab7       __unwindfunclet$??0launchEditor@@QAE@ABVQString@@00@Z$25 1001bab7 f   launchEditor.obj
 0001:0001aad1       __unwindfunclet$??0launchEditor@@QAE@ABVQString@@00@Z$26 1001bad1 f   launchEditor.obj
 0001:0001aaeb       __unwindfunclet$??0launchEditor@@QAE@ABVQString@@00@Z$27 1001baeb f   launchEditor.obj
 0001:0001ab0a       __unwindfunclet$??0launchEditor@@QAE@ABVQString@@00@Z$29 1001bb0a f   launchEditor.obj
 0001:0001ab13       __unwindfunclet$??0launchEditor@@QAE@ABVQString@@00@Z$30 1001bb13 f   launchEditor.obj
 0001:0001ab1c       __unwindfunclet$??0launchEditor@@QAE@ABVQString@@00@Z$31 1001bb1c f   launchEditor.obj
 0001:0001ab25       __unwindfunclet$??0launchEditor@@QAE@ABVQString@@00@Z$32 1001bb25 f   launchEditor.obj
 0001:0001ab2f       __unwindfunclet$??0launchEditor@@QAE@ABVQString@@00@Z$33 1001bb2f f   launchEditor.obj
 0001:0001ab4e       __unwindfunclet$??0launchEditor@@QAE@ABVQString@@00@Z$34 1001bb4e f   launchEditor.obj
 0001:0001ab6d       __unwindfunclet$??0launchEditor@@QAE@ABVQString@@00@Z$35 1001bb6d f   launchEditor.obj
 0001:0001ab8c       __unwindfunclet$??0launchEditor@@QAE@ABVQString@@00@Z$36 1001bb8c f   launchEditor.obj
 0001:0001abab       __unwindfunclet$??0launchEditor@@QAE@ABVQString@@00@Z$38 1001bbab f   launchEditor.obj
 0001:0001abb4       __unwindfunclet$??0launchEditor@@QAE@ABVQString@@00@Z$39 1001bbb4 f   launchEditor.obj
 0001:0001abbd       __unwindfunclet$??0launchEditor@@QAE@ABVQString@@00@Z$40 1001bbbd f   launchEditor.obj
 0001:0001abc6       __unwindfunclet$??0launchEditor@@QAE@ABVQString@@00@Z$41 1001bbc6 f   launchEditor.obj
 0001:0001abcf       __unwindfunclet$??0launchEditor@@QAE@ABVQString@@00@Z$42 1001bbcf f   launchEditor.obj
 0001:0001abd8       __unwindfunclet$??0launchEditor@@QAE@ABVQString@@00@Z$43 1001bbd8 f   launchEditor.obj
 0001:0001abe1       __ehhandler$??0launchEditor@@QAE@ABVQString@@00@Z 1001bbe1 f   launchEditor.obj
 0001:0001abfc       __unwindfunclet$??1?$QDict@VQAction@@@@UAE@XZ$0 1001bbfc f   launchEditor.obj
 0001:0001ac05       __ehhandler$??1?$QDict@VQAction@@@@UAE@XZ 1001bc05 f   launchEditor.obj
 0001:0001ac20       __unwindfunclet$?about@workstationEditor@@UAE?AVQString@@XZ$0 1001bc20 f   launchEditor.obj
 0001:0001ac20       __unwindfunclet$?about@launchEditor@@UAE?AVQString@@XZ$0 1001bc20 f   launchEditor.obj
 0001:0001ac29       __unwindfunclet$?about@workstationEditor@@UAE?AVQString@@XZ$1 1001bc29 f   launchEditor.obj
 0001:0001ac29       __unwindfunclet$?about@launchEditor@@UAE?AVQString@@XZ$1 1001bc29 f   launchEditor.obj
 0001:0001ac32       __unwindfunclet$?about@launchEditor@@UAE?AVQString@@XZ$2 1001bc32 f   launchEditor.obj
 0001:0001ac32       __unwindfunclet$?about@workstationEditor@@UAE?AVQString@@XZ$2 1001bc32 f   launchEditor.obj
 0001:0001ac3b       __unwindfunclet$?about@launchEditor@@UAE?AVQString@@XZ$3 1001bc3b f   launchEditor.obj
 0001:0001ac3b       __unwindfunclet$?about@workstationEditor@@UAE?AVQString@@XZ$3 1001bc3b f   launchEditor.obj
 0001:0001ac44       __unwindfunclet$?about@launchEditor@@UAE?AVQString@@XZ$4 1001bc44 f   launchEditor.obj
 0001:0001ac44       __unwindfunclet$?about@workstationEditor@@UAE?AVQString@@XZ$4 1001bc44 f   launchEditor.obj
 0001:0001ac5e       __ehhandler$?about@workstationEditor@@UAE?AVQString@@XZ 1001bc5e f   launchEditor.obj
 0001:0001ac5e       __ehhandler$?about@launchEditor@@UAE?AVQString@@XZ 1001bc5e f   launchEditor.obj
 0001:0001ac79       __unwindfunclet$?activate@launchEditor@@UAEX_N@Z$0 1001bc79 f   launchEditor.obj
 0001:0001ac82       __unwindfunclet$?activate@launchEditor@@UAEX_N@Z$2 1001bc82 f   launchEditor.obj
 0001:0001ac8b       __unwindfunclet$?activate@launchEditor@@UAEX_N@Z$4 1001bc8b f   launchEditor.obj
 0001:0001ac94       __unwindfunclet$?activate@launchEditor@@UAEX_N@Z$5 1001bc94 f   launchEditor.obj
 0001:0001ac9d       __unwindfunclet$?activate@launchEditor@@UAEX_N@Z$6 1001bc9d f   launchEditor.obj
 0001:0001aca6       __unwindfunclet$?activate@launchEditor@@UAEX_N@Z$7 1001bca6 f   launchEditor.obj
 0001:0001acaf       __unwindfunclet$?activate@launchEditor@@UAEX_N@Z$8 1001bcaf f   launchEditor.obj
 0001:0001acb8       __ehhandler$?activate@launchEditor@@UAEX_N@Z 1001bcb8 f   launchEditor.obj
 0001:0001acd3       __unwindfunclet$?menus@launchEditor@@UAE?AVQPopupMenuList@@XZ$0 1001bcd3 f   launchEditor.obj
 0001:0001acd3       __unwindfunclet$?menus@workstationEditor@@UAE?AVQPopupMenuList@@XZ$0 1001bcd3 f   launchEditor.obj
 0001:0001acec       __ehhandler$?menus@workstationEditor@@UAE?AVQPopupMenuList@@XZ 1001bcec f   launchEditor.obj
 0001:0001acec       __ehhandler$?menus@launchEditor@@UAE?AVQPopupMenuList@@XZ 1001bcec f   launchEditor.obj
 0001:0001ad07       __unwindfunclet$?navigateToWs@launchEditor@@AAEXH@Z$0 1001bd07 f   launchEditor.obj
 0001:0001ad10       __unwindfunclet$?navigateToWs@launchEditor@@AAEXH@Z$1 1001bd10 f   launchEditor.obj
 0001:0001ad19       __ehhandler$?navigateToWs@launchEditor@@AAEXH@Z 1001bd19 f   launchEditor.obj
 0001:0001ad34       __unwindfunclet$?reply@launchEditor@@UAEXPAVresponse@@@Z$0 1001bd34 f   launchEditor.obj
 0001:0001ad3d       __unwindfunclet$?reply@launchEditor@@UAEXPAVresponse@@@Z$1 1001bd3d f   launchEditor.obj
 0001:0001ad46       __unwindfunclet$?reply@launchEditor@@UAEXPAVresponse@@@Z$2 1001bd46 f   launchEditor.obj
 0001:0001ad4f       __unwindfunclet$?reply@launchEditor@@UAEXPAVresponse@@@Z$3 1001bd4f f   launchEditor.obj
 0001:0001ad58       __unwindfunclet$?reply@launchEditor@@UAEXPAVresponse@@@Z$4 1001bd58 f   launchEditor.obj
 0001:0001ad61       __unwindfunclet$?reply@launchEditor@@UAEXPAVresponse@@@Z$5 1001bd61 f   launchEditor.obj
 0001:0001ad6a       __unwindfunclet$?reply@launchEditor@@UAEXPAVresponse@@@Z$6 1001bd6a f   launchEditor.obj
 0001:0001ad73       __unwindfunclet$?reply@launchEditor@@UAEXPAVresponse@@@Z$7 1001bd73 f   launchEditor.obj
 0001:0001ad7c       __unwindfunclet$?reply@launchEditor@@UAEXPAVresponse@@@Z$8 1001bd7c f   launchEditor.obj
 0001:0001ad85       __unwindfunclet$?reply@launchEditor@@UAEXPAVresponse@@@Z$9 1001bd85 f   launchEditor.obj
 0001:0001ad8e       __unwindfunclet$?reply@launchEditor@@UAEXPAVresponse@@@Z$10 1001bd8e f   launchEditor.obj
 0001:0001ad97       __unwindfunclet$?reply@launchEditor@@UAEXPAVresponse@@@Z$11 1001bd97 f   launchEditor.obj
 0001:0001ada0       __unwindfunclet$?reply@launchEditor@@UAEXPAVresponse@@@Z$12 1001bda0 f   launchEditor.obj
 0001:0001ada9       __unwindfunclet$?reply@launchEditor@@UAEXPAVresponse@@@Z$13 1001bda9 f   launchEditor.obj
 0001:0001adb2       __ehhandler$?reply@launchEditor@@UAEXPAVresponse@@@Z 1001bdb2 f   launchEditor.obj
 0001:0001adcd       __unwindfunclet$?toolbars@launchEditor@@UAE?AVQDockWindowList@@XZ$0 1001bdcd f   launchEditor.obj
 0001:0001adcd       __unwindfunclet$?toolbars@workstationEditor@@UAE?AVQDockWindowList@@XZ$0 1001bdcd f   launchEditor.obj
 0001:0001ade6       __ehhandler$?toolbars@workstationEditor@@UAE?AVQDockWindowList@@XZ 1001bde6 f   launchEditor.obj
 0001:0001ade6       __ehhandler$?toolbars@launchEditor@@UAE?AVQDockWindowList@@XZ 1001bde6 f   launchEditor.obj
 0001:0001ae01       __unwindfunclet$?workstationChanged@launchEditor@@AAEXPAVQListViewItem@@@Z$0 1001be01 f   launchEditor.obj
 0001:0001ae0a       __unwindfunclet$?workstationChanged@launchEditor@@AAEXPAVQListViewItem@@@Z$1 1001be0a f   launchEditor.obj
 0001:0001ae13       __ehhandler$?workstationChanged@launchEditor@@AAEXPAVQListViewItem@@@Z 1001be13 f   launchEditor.obj
 0001:0001ae2e       __unwindfunclet$??0launchEditorDlg@@QAE@ABVQString@@PAVQWidget@@PBDI@Z$0 1001be2e f   launcheditordlgimpl.obj
 0001:0001ae36       __unwindfunclet$??0launchEditorDlg@@QAE@ABVQString@@PAVQWidget@@PBDI@Z$1 1001be36 f   launcheditordlgimpl.obj
 0001:0001ae45       __unwindfunclet$??0launchEditorDlg@@QAE@ABVQString@@PAVQWidget@@PBDI@Z$2 1001be45 f   launcheditordlgimpl.obj
 0001:0001ae4e       __unwindfunclet$??0launchEditorDlg@@QAE@ABVQString@@PAVQWidget@@PBDI@Z$3 1001be4e f   launcheditordlgimpl.obj
 0001:0001ae57       __unwindfunclet$??0launchEditorDlg@@QAE@ABVQString@@PAVQWidget@@PBDI@Z$4 1001be57 f   launcheditordlgimpl.obj
 0001:0001ae60       __unwindfunclet$??0launchEditorDlg@@QAE@ABVQString@@PAVQWidget@@PBDI@Z$5 1001be60 f   launcheditordlgimpl.obj
 0001:0001ae69       __unwindfunclet$??0launchEditorDlg@@QAE@ABVQString@@PAVQWidget@@PBDI@Z$6 1001be69 f   launcheditordlgimpl.obj
 0001:0001ae72       __unwindfunclet$??0launchEditorDlg@@QAE@ABVQString@@PAVQWidget@@PBDI@Z$7 1001be72 f   launcheditordlgimpl.obj
 0001:0001ae7b       __unwindfunclet$??0launchEditorDlg@@QAE@ABVQString@@PAVQWidget@@PBDI@Z$8 1001be7b f   launcheditordlgimpl.obj
 0001:0001ae84       __unwindfunclet$??0launchEditorDlg@@QAE@ABVQString@@PAVQWidget@@PBDI@Z$9 1001be84 f   launcheditordlgimpl.obj
 0001:0001ae8d       __unwindfunclet$??0launchEditorDlg@@QAE@ABVQString@@PAVQWidget@@PBDI@Z$10 1001be8d f   launcheditordlgimpl.obj
 0001:0001ae96       __unwindfunclet$??0launchEditorDlg@@QAE@ABVQString@@PAVQWidget@@PBDI@Z$11 1001be96 f   launcheditordlgimpl.obj
 0001:0001ae9f       __ehhandler$??0launchEditorDlg@@QAE@ABVQString@@PAVQWidget@@PBDI@Z 1001be9f f   launcheditordlgimpl.obj
 0001:0001aeba       __unwindfunclet$??1launchEditorDlg@@UAE@XZ$0 1001beba f   launcheditordlgimpl.obj
 0001:0001aec2       __ehhandler$??1launchEditorDlg@@UAE@XZ 1001bec2 f   launcheditordlgimpl.obj
 0001:0001aedd       __unwindfunclet$?createLaunchElement@launchEditorDlg@@QAE?AVQDomElement@@ABVQString@@AAVQDomDocument@@@Z$0 1001bedd f   launcheditordlgimpl.obj
 0001:0001aee6       __unwindfunclet$?createLaunchElement@launchEditorDlg@@QAE?AVQDomElement@@ABVQString@@AAVQDomDocument@@@Z$1 1001bee6 f   launcheditordlgimpl.obj
 0001:0001af00       __unwindfunclet$?createLaunchElement@launchEditorDlg@@QAE?AVQDomElement@@ABVQString@@AAVQDomDocument@@@Z$2 1001bf00 f   launcheditordlgimpl.obj
 0001:0001af09       __unwindfunclet$?createLaunchElement@launchEditorDlg@@QAE?AVQDomElement@@ABVQString@@AAVQDomDocument@@@Z$3 1001bf09 f   launcheditordlgimpl.obj
 0001:0001af12       __unwindfunclet$?createLaunchElement@launchEditorDlg@@QAE?AVQDomElement@@ABVQString@@AAVQDomDocument@@@Z$4 1001bf12 f   launcheditordlgimpl.obj
 0001:0001af1b       __unwindfunclet$?createLaunchElement@launchEditorDlg@@QAE?AVQDomElement@@ABVQString@@AAVQDomDocument@@@Z$5 1001bf1b f   launcheditordlgimpl.obj
 0001:0001af24       __unwindfunclet$?createLaunchElement@launchEditorDlg@@QAE?AVQDomElement@@ABVQString@@AAVQDomDocument@@@Z$6 1001bf24 f   launcheditordlgimpl.obj
 0001:0001af2d       __unwindfunclet$?createLaunchElement@launchEditorDlg@@QAE?AVQDomElement@@ABVQString@@AAVQDomDocument@@@Z$7 1001bf2d f   launcheditordlgimpl.obj
 0001:0001af36       __unwindfunclet$?createLaunchElement@launchEditorDlg@@QAE?AVQDomElement@@ABVQString@@AAVQDomDocument@@@Z$8 1001bf36 f   launcheditordlgimpl.obj
 0001:0001af3f       __unwindfunclet$?createLaunchElement@launchEditorDlg@@QAE?AVQDomElement@@ABVQString@@AAVQDomDocument@@@Z$9 1001bf3f f   launcheditordlgimpl.obj
 0001:0001af48       __unwindfunclet$?createLaunchElement@launchEditorDlg@@QAE?AVQDomElement@@ABVQString@@AAVQDomDocument@@@Z$10 1001bf48 f   launcheditordlgimpl.obj
 0001:0001af51       __unwindfunclet$?createLaunchElement@launchEditorDlg@@QAE?AVQDomElement@@ABVQString@@AAVQDomDocument@@@Z$12 1001bf51 f   launcheditordlgimpl.obj
 0001:0001af5a       __unwindfunclet$?createLaunchElement@launchEditorDlg@@QAE?AVQDomElement@@ABVQString@@AAVQDomDocument@@@Z$13 1001bf5a f   launcheditordlgimpl.obj
 0001:0001af63       __unwindfunclet$?createLaunchElement@launchEditorDlg@@QAE?AVQDomElement@@ABVQString@@AAVQDomDocument@@@Z$15 1001bf63 f   launcheditordlgimpl.obj
 0001:0001af6c       __unwindfunclet$?createLaunchElement@launchEditorDlg@@QAE?AVQDomElement@@ABVQString@@AAVQDomDocument@@@Z$16 1001bf6c f   launcheditordlgimpl.obj
 0001:0001af75       __unwindfunclet$?createLaunchElement@launchEditorDlg@@QAE?AVQDomElement@@ABVQString@@AAVQDomDocument@@@Z$18 1001bf75 f   launcheditordlgimpl.obj
 0001:0001af7e       __unwindfunclet$?createLaunchElement@launchEditorDlg@@QAE?AVQDomElement@@ABVQString@@AAVQDomDocument@@@Z$19 1001bf7e f   launcheditordlgimpl.obj
 0001:0001af87       __unwindfunclet$?createLaunchElement@launchEditorDlg@@QAE?AVQDomElement@@ABVQString@@AAVQDomDocument@@@Z$20 1001bf87 f   launcheditordlgimpl.obj
 0001:0001af90       __unwindfunclet$?createLaunchElement@launchEditorDlg@@QAE?AVQDomElement@@ABVQString@@AAVQDomDocument@@@Z$21 1001bf90 f   launcheditordlgimpl.obj
 0001:0001af99       __ehhandler$?createLaunchElement@launchEditorDlg@@QAE?AVQDomElement@@ABVQString@@AAVQDomDocument@@@Z 1001bf99 f   launcheditordlgimpl.obj
 0001:0001afb4       __unwindfunclet$?doAdd@launchEditorDlg@@QAEXXZ$0 1001bfb4 f   launcheditordlgimpl.obj
 0001:0001afbd       __unwindfunclet$?doAdd@launchEditorDlg@@QAEXXZ$1 1001bfbd f   launcheditordlgimpl.obj
 0001:0001afc6       __unwindfunclet$?doAdd@launchEditorDlg@@QAEXXZ$2 1001bfc6 f   launcheditordlgimpl.obj
 0001:0001afcf       __unwindfunclet$?doAdd@launchEditorDlg@@QAEXXZ$3 1001bfcf f   launcheditordlgimpl.obj
 0001:0001afd8       __unwindfunclet$?doAdd@launchEditorDlg@@QAEXXZ$4 1001bfd8 f   launcheditordlgimpl.obj
 0001:0001afe2       __unwindfunclet$?doAdd@launchEditorDlg@@QAEXXZ$5 1001bfe2 f   launcheditordlgimpl.obj
 0001:0001affc       __unwindfunclet$?doAdd@launchEditorDlg@@QAEXXZ$6 1001bffc f   launcheditordlgimpl.obj
 0001:0001b005       __ehhandler$?doAdd@launchEditorDlg@@QAEXXZ 1001c005 f   launcheditordlgimpl.obj
 0001:0001b020       __unwindfunclet$?doDuplicate@launchEditorDlg@@QAEXXZ$0 1001c020 f   launcheditordlgimpl.obj
 0001:0001b029       __unwindfunclet$?doDuplicate@launchEditorDlg@@QAEXXZ$1 1001c029 f   launcheditordlgimpl.obj
 0001:0001b032       __unwindfunclet$?doDuplicate@launchEditorDlg@@QAEXXZ$2 1001c032 f   launcheditordlgimpl.obj
 0001:0001b03b       __unwindfunclet$?doDuplicate@launchEditorDlg@@QAEXXZ$3 1001c03b f   launcheditordlgimpl.obj
 0001:0001b044       __unwindfunclet$?doDuplicate@launchEditorDlg@@QAEXXZ$4 1001c044 f   launcheditordlgimpl.obj
 0001:0001b04e       __unwindfunclet$?doDuplicate@launchEditorDlg@@QAEXXZ$5 1001c04e f   launcheditordlgimpl.obj
 0001:0001b068       __unwindfunclet$?doDuplicate@launchEditorDlg@@QAEXXZ$6 1001c068 f   launcheditordlgimpl.obj
 0001:0001b071       __ehhandler$?doDuplicate@launchEditorDlg@@QAEXXZ 1001c071 f   launcheditordlgimpl.obj
 0001:0001b08c       __unwindfunclet$?doMoveUp@launchEditorDlg@@QAEXXZ$0 1001c08c f   launcheditordlgimpl.obj
 0001:0001b08c       __unwindfunclet$?doMoveDown@launchEditorDlg@@QAEXXZ$0 1001c08c f   launcheditordlgimpl.obj
 0001:0001b08c       __unwindfunclet$?doRemove@workstationEditorDlg@@AAEXXZ$0 1001c08c f   launcheditordlgimpl.obj
 0001:0001b095       __ehhandler$?doRemove@workstationEditorDlg@@AAEXXZ 1001c095 f   launcheditordlgimpl.obj
 0001:0001b095       __ehhandler$?doMoveUp@launchEditorDlg@@QAEXXZ 1001c095 f   launcheditordlgimpl.obj
 0001:0001b095       __ehhandler$?doMoveDown@launchEditorDlg@@QAEXXZ 1001c095 f   launcheditordlgimpl.obj
 0001:0001b0b0       __unwindfunclet$?load@launchEditorDlg@@QAE_NABVQString@@H@Z$0 1001c0b0 f   launcheditordlgimpl.obj
 0001:0001b0b9       __unwindfunclet$?load@launchEditorDlg@@QAE_NABVQString@@H@Z$1 1001c0b9 f   launcheditordlgimpl.obj
 0001:0001b0c2       __unwindfunclet$?load@launchEditorDlg@@QAE_NABVQString@@H@Z$2 1001c0c2 f   launcheditordlgimpl.obj
 0001:0001b0cb       __unwindfunclet$?load@launchEditorDlg@@QAE_NABVQString@@H@Z$3 1001c0cb f   launcheditordlgimpl.obj
 0001:0001b0d4       __unwindfunclet$?load@launchEditorDlg@@QAE_NABVQString@@H@Z$4 1001c0d4 f   launcheditordlgimpl.obj
 0001:0001b0dd       __unwindfunclet$?load@launchEditorDlg@@QAE_NABVQString@@H@Z$5 1001c0dd f   launcheditordlgimpl.obj
 0001:0001b0e9       __unwindfunclet$?load@launchEditorDlg@@QAE_NABVQString@@H@Z$6 1001c0e9 f   launcheditordlgimpl.obj
 0001:0001b0f2       __unwindfunclet$?load@launchEditorDlg@@QAE_NABVQString@@H@Z$7 1001c0f2 f   launcheditordlgimpl.obj
 0001:0001b0fb       __unwindfunclet$?load@launchEditorDlg@@QAE_NABVQString@@H@Z$8 1001c0fb f   launcheditordlgimpl.obj
 0001:0001b104       __unwindfunclet$?load@launchEditorDlg@@QAE_NABVQString@@H@Z$9 1001c104 f   launcheditordlgimpl.obj
 0001:0001b10d       __unwindfunclet$?load@launchEditorDlg@@QAE_NABVQString@@H@Z$10 1001c10d f   launcheditordlgimpl.obj
 0001:0001b116       __unwindfunclet$?load@launchEditorDlg@@QAE_NABVQString@@H@Z$11 1001c116 f   launcheditordlgimpl.obj
 0001:0001b11f       __unwindfunclet$?load@launchEditorDlg@@QAE_NABVQString@@H@Z$12 1001c11f f   launcheditordlgimpl.obj
 0001:0001b128       __unwindfunclet$?load@launchEditorDlg@@QAE_NABVQString@@H@Z$33 1001c128 f   launcheditordlgimpl.obj
 0001:0001b131       __unwindfunclet$?load@launchEditorDlg@@QAE_NABVQString@@H@Z$13 1001c131 f   launcheditordlgimpl.obj
 0001:0001b13a       __unwindfunclet$?load@launchEditorDlg@@QAE_NABVQString@@H@Z$14 1001c13a f   launcheditordlgimpl.obj
 0001:0001b143       __unwindfunclet$?load@launchEditorDlg@@QAE_NABVQString@@H@Z$15 1001c143 f   launcheditordlgimpl.obj
 0001:0001b14c       __unwindfunclet$?load@launchEditorDlg@@QAE_NABVQString@@H@Z$16 1001c14c f   launcheditordlgimpl.obj
 0001:0001b155       __unwindfunclet$?load@launchEditorDlg@@QAE_NABVQString@@H@Z$17 1001c155 f   launcheditordlgimpl.obj
 0001:0001b15e       __unwindfunclet$?load@launchEditorDlg@@QAE_NABVQString@@H@Z$18 1001c15e f   launcheditordlgimpl.obj
 0001:0001b167       __unwindfunclet$?load@launchEditorDlg@@QAE_NABVQString@@H@Z$19 1001c167 f   launcheditordlgimpl.obj
 0001:0001b170       __unwindfunclet$?load@launchEditorDlg@@QAE_NABVQString@@H@Z$20 1001c170 f   launcheditordlgimpl.obj
 0001:0001b179       __unwindfunclet$?load@launchEditorDlg@@QAE_NABVQString@@H@Z$21 1001c179 f   launcheditordlgimpl.obj
 0001:0001b182       __unwindfunclet$?load@launchEditorDlg@@QAE_NABVQString@@H@Z$22 1001c182 f   launcheditordlgimpl.obj
 0001:0001b18b       __unwindfunclet$?load@launchEditorDlg@@QAE_NABVQString@@H@Z$23 1001c18b f   launcheditordlgimpl.obj
 0001:0001b194       __unwindfunclet$?load@launchEditorDlg@@QAE_NABVQString@@H@Z$24 1001c194 f   launcheditordlgimpl.obj
 0001:0001b19d       __unwindfunclet$?load@launchEditorDlg@@QAE_NABVQString@@H@Z$25 1001c19d f   launcheditordlgimpl.obj
 0001:0001b1a6       __unwindfunclet$?load@launchEditorDlg@@QAE_NABVQString@@H@Z$26 1001c1a6 f   launcheditordlgimpl.obj
 0001:0001b1af       __unwindfunclet$?load@launchEditorDlg@@QAE_NABVQString@@H@Z$27 1001c1af f   launcheditordlgimpl.obj
 0001:0001b1b8       __unwindfunclet$?load@launchEditorDlg@@QAE_NABVQString@@H@Z$28 1001c1b8 f   launcheditordlgimpl.obj
 0001:0001b1c5       __unwindfunclet$?load@launchEditorDlg@@QAE_NABVQString@@H@Z$29 1001c1c5 f   launcheditordlgimpl.obj
 0001:0001b1df       __unwindfunclet$?load@launchEditorDlg@@QAE_NABVQString@@H@Z$30 1001c1df f   launcheditordlgimpl.obj
 0001:0001b1e8       __unwindfunclet$?load@launchEditorDlg@@QAE_NABVQString@@H@Z$31 1001c1e8 f   launcheditordlgimpl.obj
 0001:0001b1f1       __unwindfunclet$?load@launchEditorDlg@@QAE_NABVQString@@H@Z$32 1001c1f1 f   launcheditordlgimpl.obj
 0001:0001b1fa       __ehhandler$?load@launchEditorDlg@@QAE_NABVQString@@H@Z 1001c1fa f   launcheditordlgimpl.obj
 0001:0001b218       __unwindfunclet$?save@launchEditorDlg@@QAEXH@Z$0 1001c218 f   launcheditordlgimpl.obj
 0001:0001b221       __unwindfunclet$?save@launchEditorDlg@@QAEXH@Z$1 1001c221 f   launcheditordlgimpl.obj
 0001:0001b22a       __unwindfunclet$?save@launchEditorDlg@@QAEXH@Z$2 1001c22a f   launcheditordlgimpl.obj
 0001:0001b233       __unwindfunclet$?save@launchEditorDlg@@QAEXH@Z$3 1001c233 f   launcheditordlgimpl.obj
 0001:0001b23f       __unwindfunclet$?save@launchEditorDlg@@QAEXH@Z$4 1001c23f f   launcheditordlgimpl.obj
 0001:0001b248       __unwindfunclet$?save@launchEditorDlg@@QAEXH@Z$5 1001c248 f   launcheditordlgimpl.obj
 0001:0001b251       __unwindfunclet$?save@launchEditorDlg@@QAEXH@Z$6 1001c251 f   launcheditordlgimpl.obj
 0001:0001b25a       __unwindfunclet$?save@launchEditorDlg@@QAEXH@Z$7 1001c25a f   launcheditordlgimpl.obj
 0001:0001b263       __unwindfunclet$?save@launchEditorDlg@@QAEXH@Z$8 1001c263 f   launcheditordlgimpl.obj
 0001:0001b26c       __unwindfunclet$?save@launchEditorDlg@@QAEXH@Z$9 1001c26c f   launcheditordlgimpl.obj
 0001:0001b275       __unwindfunclet$?save@launchEditorDlg@@QAEXH@Z$10 1001c275 f   launcheditordlgimpl.obj
 0001:0001b27e       __unwindfunclet$?save@launchEditorDlg@@QAEXH@Z$11 1001c27e f   launcheditordlgimpl.obj
 0001:0001b287       __unwindfunclet$?save@launchEditorDlg@@QAEXH@Z$12 1001c287 f   launcheditordlgimpl.obj
 0001:0001b290       __unwindfunclet$?save@launchEditorDlg@@QAEXH@Z$13 1001c290 f   launcheditordlgimpl.obj
 0001:0001b299       __unwindfunclet$?save@launchEditorDlg@@QAEXH@Z$15 1001c299 f   launcheditordlgimpl.obj
 0001:0001b2a2       __unwindfunclet$?save@launchEditorDlg@@QAEXH@Z$16 1001c2a2 f   launcheditordlgimpl.obj
 0001:0001b2ab       __unwindfunclet$?save@launchEditorDlg@@QAEXH@Z$17 1001c2ab f   launcheditordlgimpl.obj
 0001:0001b2b4       __unwindfunclet$?save@launchEditorDlg@@QAEXH@Z$18 1001c2b4 f   launcheditordlgimpl.obj
 0001:0001b2bd       __unwindfunclet$?save@launchEditorDlg@@QAEXH@Z$20 1001c2bd f   launcheditordlgimpl.obj
 0001:0001b2c6       __unwindfunclet$?save@launchEditorDlg@@QAEXH@Z$21 1001c2c6 f   launcheditordlgimpl.obj
 0001:0001b2cf       __unwindfunclet$?save@launchEditorDlg@@QAEXH@Z$22 1001c2cf f   launcheditordlgimpl.obj
 0001:0001b2db       __unwindfunclet$?save@launchEditorDlg@@QAEXH@Z$23 1001c2db f   launcheditordlgimpl.obj
 0001:0001b2e7       __ehhandler$?save@launchEditorDlg@@QAEXH@Z 1001c2e7 f   launcheditordlgimpl.obj
 0001:0001b305       __unwindfunclet$?tableValueChanged@workstationEditorDlg@@AAEXHH@Z$0 1001c305 f   launcheditordlgimpl.obj
 0001:0001b305       __unwindfunclet$?tableValueChanged@launchEditorDlg@@QAEXHH@Z$0 1001c305 f   launcheditordlgimpl.obj
 0001:0001b30e       __ehhandler$?tableValueChanged@workstationEditorDlg@@AAEXHH@Z 1001c30e f   launcheditordlgimpl.obj
 0001:0001b30e       __ehhandler$?tableValueChanged@launchEditorDlg@@QAEXHH@Z 1001c30e f   launcheditordlgimpl.obj
 0001:0001b329       __unwindfunclet$?create@plugindesc@@UAEPAVconfig_plugin_base@@ABVQString@@00@Z$0 1001c329 f   plugindesc.obj
 0001:0001b333       __unwindfunclet$?create@plugindesc@@UAEPAVconfig_plugin_base@@ABVQString@@00@Z$1 1001c333 f   plugindesc.obj
 0001:0001b33d       __unwindfunclet$?create@plugindesc@@UAEPAVconfig_plugin_base@@ABVQString@@00@Z$2 1001c33d f   plugindesc.obj
 0001:0001b347       __unwindfunclet$?create@plugindesc@@UAEPAVconfig_plugin_base@@ABVQString@@00@Z$3 1001c347 f   plugindesc.obj
 0001:0001b351       __unwindfunclet$?create@plugindesc@@UAEPAVconfig_plugin_base@@ABVQString@@00@Z$4 1001c351 f   plugindesc.obj
 0001:0001b35b       __ehhandler$?create@plugindesc@@UAEPAVconfig_plugin_base@@ABVQString@@00@Z 1001c35b f   plugindesc.obj
 0001:0001b376       __unwindfunclet$?keys@plugindesc@@UAE?AVQStringList@@ABVQString@@0@Z$0 1001c376 f   plugindesc.obj
 0001:0001b390       __unwindfunclet$?keys@plugindesc@@UAE?AVQStringList@@ABVQString@@0@Z$1 1001c390 f   plugindesc.obj
 0001:0001b399       __unwindfunclet$?keys@plugindesc@@UAE?AVQStringList@@ABVQString@@0@Z$2 1001c399 f   plugindesc.obj
 0001:0001b3a2       __unwindfunclet$?keys@plugindesc@@UAE?AVQStringList@@ABVQString@@0@Z$3 1001c3a2 f   plugindesc.obj
 0001:0001b3ab       __unwindfunclet$?keys@plugindesc@@UAE?AVQStringList@@ABVQString@@0@Z$4 1001c3ab f   plugindesc.obj
 0001:0001b3b4       __unwindfunclet$?keys@plugindesc@@UAE?AVQStringList@@ABVQString@@0@Z$5 1001c3b4 f   plugindesc.obj
 0001:0001b3bd       __unwindfunclet$?keys@plugindesc@@UAE?AVQStringList@@ABVQString@@0@Z$6 1001c3bd f   plugindesc.obj
 0001:0001b3c6       __ehhandler$?keys@plugindesc@@UAE?AVQStringList@@ABVQString@@0@Z 1001c3c6 f   plugindesc.obj
 0001:0001b3e1       __unwindfunclet$??0testPlugin@@QAE@ABVQString@@00@Z$0 1001c3e1 f   testPlugin.obj
 0001:0001b3ec       __unwindfunclet$??0testPlugin@@QAE@ABVQString@@00@Z$1 1001c3ec f   testPlugin.obj
 0001:0001b3fa       __unwindfunclet$??0testPlugin@@QAE@ABVQString@@00@Z$2 1001c3fa f   testPlugin.obj
 0001:0001b408       __unwindfunclet$??0testPlugin@@QAE@ABVQString@@00@Z$3 1001c408 f   testPlugin.obj
 0001:0001b419       __unwindfunclet$??0testPlugin@@QAE@ABVQString@@00@Z$4 1001c419 f   testPlugin.obj
 0001:0001b42a       __unwindfunclet$??0testPlugin@@QAE@ABVQString@@00@Z$5 1001c42a f   testPlugin.obj
 0001:0001b436       __unwindfunclet$??0testPlugin@@QAE@ABVQString@@00@Z$6 1001c436 f   testPlugin.obj
 0001:0001b443       __unwindfunclet$??0testPlugin@@QAE@ABVQString@@00@Z$7 1001c443 f   testPlugin.obj
 0001:0001b44f       __unwindfunclet$??0testPlugin@@QAE@ABVQString@@00@Z$8 1001c44f f   testPlugin.obj
 0001:0001b45b       __unwindfunclet$??0testPlugin@@QAE@ABVQString@@00@Z$9 1001c45b f   testPlugin.obj
 0001:0001b467       __unwindfunclet$??0testPlugin@@QAE@ABVQString@@00@Z$10 1001c467 f   testPlugin.obj
 0001:0001b473       __unwindfunclet$??0testPlugin@@QAE@ABVQString@@00@Z$11 1001c473 f   testPlugin.obj
 0001:0001b47f       __unwindfunclet$??0testPlugin@@QAE@ABVQString@@00@Z$12 1001c47f f   testPlugin.obj
 0001:0001b48b       __unwindfunclet$??0testPlugin@@QAE@ABVQString@@00@Z$13 1001c48b f   testPlugin.obj
 0001:0001b497       __unwindfunclet$??0testPlugin@@QAE@ABVQString@@00@Z$14 1001c497 f   testPlugin.obj
 0001:0001b4a3       __unwindfunclet$??0testPlugin@@QAE@ABVQString@@00@Z$15 1001c4a3 f   testPlugin.obj
 0001:0001b4af       __unwindfunclet$??0testPlugin@@QAE@ABVQString@@00@Z$16 1001c4af f   testPlugin.obj
 0001:0001b4bb       __unwindfunclet$??0testPlugin@@QAE@ABVQString@@00@Z$17 1001c4bb f   testPlugin.obj
 0001:0001b4c7       __unwindfunclet$??0testPlugin@@QAE@ABVQString@@00@Z$18 1001c4c7 f   testPlugin.obj
 0001:0001b4d3       __unwindfunclet$??0testPlugin@@QAE@ABVQString@@00@Z$19 1001c4d3 f   testPlugin.obj
 0001:0001b4df       __unwindfunclet$??0testPlugin@@QAE@ABVQString@@00@Z$20 1001c4df f   testPlugin.obj
 0001:0001b4eb       __unwindfunclet$??0testPlugin@@QAE@ABVQString@@00@Z$21 1001c4eb f   testPlugin.obj
 0001:0001b4f7       __unwindfunclet$??0testPlugin@@QAE@ABVQString@@00@Z$22 1001c4f7 f   testPlugin.obj
 0001:0001b503       __unwindfunclet$??0testPlugin@@QAE@ABVQString@@00@Z$23 1001c503 f   testPlugin.obj
 0001:0001b50f       __unwindfunclet$??0testPlugin@@QAE@ABVQString@@00@Z$24 1001c50f f   testPlugin.obj
 0001:0001b51b       __unwindfunclet$??0testPlugin@@QAE@ABVQString@@00@Z$25 1001c51b f   testPlugin.obj
 0001:0001b527       __unwindfunclet$??0testPlugin@@QAE@ABVQString@@00@Z$27 1001c527 f   testPlugin.obj
 0001:0001b534       __unwindfunclet$??0testPlugin@@QAE@ABVQString@@00@Z$28 1001c534 f   testPlugin.obj
 0001:0001b540       __unwindfunclet$??0testPlugin@@QAE@ABVQString@@00@Z$29 1001c540 f   testPlugin.obj
 0001:0001b54d       __unwindfunclet$??0testPlugin@@QAE@ABVQString@@00@Z$30 1001c54d f   testPlugin.obj
 0001:0001b55a       __unwindfunclet$??0testPlugin@@QAE@ABVQString@@00@Z$31 1001c55a f   testPlugin.obj
 0001:0001b566       __unwindfunclet$??0testPlugin@@QAE@ABVQString@@00@Z$32 1001c566 f   testPlugin.obj
 0001:0001b573       __unwindfunclet$??0testPlugin@@QAE@ABVQString@@00@Z$33 1001c573 f   testPlugin.obj
 0001:0001b580       __unwindfunclet$??0testPlugin@@QAE@ABVQString@@00@Z$34 1001c580 f   testPlugin.obj
 0001:0001b58c       __unwindfunclet$??0testPlugin@@QAE@ABVQString@@00@Z$35 1001c58c f   testPlugin.obj
 0001:0001b598       __unwindfunclet$??0testPlugin@@QAE@ABVQString@@00@Z$36 1001c598 f   testPlugin.obj
 0001:0001b5a4       __unwindfunclet$??0testPlugin@@QAE@ABVQString@@00@Z$37 1001c5a4 f   testPlugin.obj
 0001:0001b5b0       __unwindfunclet$??0testPlugin@@QAE@ABVQString@@00@Z$38 1001c5b0 f   testPlugin.obj
 0001:0001b5bc       __unwindfunclet$??0testPlugin@@QAE@ABVQString@@00@Z$39 1001c5bc f   testPlugin.obj
 0001:0001b5c8       __unwindfunclet$??0testPlugin@@QAE@ABVQString@@00@Z$40 1001c5c8 f   testPlugin.obj
 0001:0001b5d4       __unwindfunclet$??0testPlugin@@QAE@ABVQString@@00@Z$41 1001c5d4 f   testPlugin.obj
 0001:0001b5e1       __unwindfunclet$??0testPlugin@@QAE@ABVQString@@00@Z$42 1001c5e1 f   testPlugin.obj
 0001:0001b5ed       __unwindfunclet$??0testPlugin@@QAE@ABVQString@@00@Z$43 1001c5ed f   testPlugin.obj
 0001:0001b5fa       __unwindfunclet$??0testPlugin@@QAE@ABVQString@@00@Z$44 1001c5fa f   testPlugin.obj
 0001:0001b607       __unwindfunclet$??0testPlugin@@QAE@ABVQString@@00@Z$45 1001c607 f   testPlugin.obj
 0001:0001b62a       __unwindfunclet$??0testPlugin@@QAE@ABVQString@@00@Z$46 1001c62a f   testPlugin.obj
 0001:0001b64d       __unwindfunclet$??0testPlugin@@QAE@ABVQString@@00@Z$47 1001c64d f   testPlugin.obj
 0001:0001b670       __unwindfunclet$??0testPlugin@@QAE@ABVQString@@00@Z$48 1001c670 f   testPlugin.obj
 0001:0001b693       __unwindfunclet$??0testPlugin@@QAE@ABVQString@@00@Z$50 1001c693 f   testPlugin.obj
 0001:0001b69f       __unwindfunclet$??0testPlugin@@QAE@ABVQString@@00@Z$51 1001c69f f   testPlugin.obj
 0001:0001b6ab       __unwindfunclet$??0testPlugin@@QAE@ABVQString@@00@Z$52 1001c6ab f   testPlugin.obj
 0001:0001b6b7       __unwindfunclet$??0testPlugin@@QAE@ABVQString@@00@Z$53 1001c6b7 f   testPlugin.obj
 0001:0001b6c4       __unwindfunclet$??0testPlugin@@QAE@ABVQString@@00@Z$54 1001c6c4 f   testPlugin.obj
 0001:0001b6e7       __unwindfunclet$??0testPlugin@@QAE@ABVQString@@00@Z$55 1001c6e7 f   testPlugin.obj
 0001:0001b70a       __unwindfunclet$??0testPlugin@@QAE@ABVQString@@00@Z$56 1001c70a f   testPlugin.obj
 0001:0001b72d       __unwindfunclet$??0testPlugin@@QAE@ABVQString@@00@Z$57 1001c72d f   testPlugin.obj
 0001:0001b755       __unwindfunclet$??0testPlugin@@QAE@ABVQString@@00@Z$59 1001c755 f   testPlugin.obj
 0001:0001b761       __unwindfunclet$??0testPlugin@@QAE@ABVQString@@00@Z$60 1001c761 f   testPlugin.obj
 0001:0001b76d       __unwindfunclet$??0testPlugin@@QAE@ABVQString@@00@Z$61 1001c76d f   testPlugin.obj
 0001:0001b779       __unwindfunclet$??0testPlugin@@QAE@ABVQString@@00@Z$62 1001c779 f   testPlugin.obj
 0001:0001b786       __unwindfunclet$??0testPlugin@@QAE@ABVQString@@00@Z$63 1001c786 f   testPlugin.obj
 0001:0001b7ae       __unwindfunclet$??0testPlugin@@QAE@ABVQString@@00@Z$64 1001c7ae f   testPlugin.obj
 0001:0001b7d6       __unwindfunclet$??0testPlugin@@QAE@ABVQString@@00@Z$65 1001c7d6 f   testPlugin.obj
 0001:0001b7fe       __unwindfunclet$??0testPlugin@@QAE@ABVQString@@00@Z$66 1001c7fe f   testPlugin.obj
 0001:0001b826       __unwindfunclet$??0testPlugin@@QAE@ABVQString@@00@Z$68 1001c826 f   testPlugin.obj
 0001:0001b832       __unwindfunclet$??0testPlugin@@QAE@ABVQString@@00@Z$69 1001c832 f   testPlugin.obj
 0001:0001b83e       __unwindfunclet$??0testPlugin@@QAE@ABVQString@@00@Z$70 1001c83e f   testPlugin.obj
 0001:0001b84b       __unwindfunclet$??0testPlugin@@QAE@ABVQString@@00@Z$71 1001c84b f   testPlugin.obj
 0001:0001b873       __unwindfunclet$??0testPlugin@@QAE@ABVQString@@00@Z$72 1001c873 f   testPlugin.obj
 0001:0001b89b       __unwindfunclet$??0testPlugin@@QAE@ABVQString@@00@Z$73 1001c89b f   testPlugin.obj
 0001:0001b8c3       __unwindfunclet$??0testPlugin@@QAE@ABVQString@@00@Z$74 1001c8c3 f   testPlugin.obj
 0001:0001b8eb       __unwindfunclet$??0testPlugin@@QAE@ABVQString@@00@Z$76 1001c8eb f   testPlugin.obj
 0001:0001b8f7       __unwindfunclet$??0testPlugin@@QAE@ABVQString@@00@Z$77 1001c8f7 f   testPlugin.obj
 0001:0001b903       __unwindfunclet$??0testPlugin@@QAE@ABVQString@@00@Z$78 1001c903 f   testPlugin.obj
 0001:0001b90f       __ehhandler$??0testPlugin@@QAE@ABVQString@@00@Z 1001c90f f   testPlugin.obj
 0001:0001b937       __unwindfunclet$??1launchEditor@@UAE@XZ$0 1001c937 f   testPlugin.obj
 0001:0001b937       __unwindfunclet$??1testPlugin@@UAE@XZ$0 1001c937 f   testPlugin.obj
 0001:0001b93f       __unwindfunclet$??1launchEditor@@UAE@XZ$1 1001c93f f   testPlugin.obj
 0001:0001b93f       __unwindfunclet$??1testPlugin@@UAE@XZ$1 1001c93f f   testPlugin.obj
 0001:0001b94a       __unwindfunclet$??1testPlugin@@UAE@XZ$2 1001c94a f   testPlugin.obj
 0001:0001b94a       __unwindfunclet$??1launchEditor@@UAE@XZ$2 1001c94a f   testPlugin.obj
 0001:0001b955       __unwindfunclet$??1launchEditor@@UAE@XZ$3 1001c955 f   testPlugin.obj
 0001:0001b955       __unwindfunclet$??1testPlugin@@UAE@XZ$3 1001c955 f   testPlugin.obj
 0001:0001b963       __unwindfunclet$??1launchEditor@@UAE@XZ$4 1001c963 f   testPlugin.obj
 0001:0001b963       __unwindfunclet$??1testPlugin@@UAE@XZ$4 1001c963 f   testPlugin.obj
 0001:0001b971       __ehhandler$??1launchEditor@@UAE@XZ 1001c971 f   testPlugin.obj
 0001:0001b971       __ehhandler$??1testPlugin@@UAE@XZ 1001c971 f   testPlugin.obj
 0001:0001b98c       __unwindfunclet$?activate@testPlugin@@UAEX_N@Z$1 1001c98c f   testPlugin.obj
 0001:0001b98c       __unwindfunclet$?timerEvent@fileManager@@EAEXPAVQTimerEvent@@@Z$0 1001c98c f   testPlugin.obj
 0001:0001b98c       __unwindfunclet$?activate@fileManager@@UAEX_N@Z$0 1001c98c f   testPlugin.obj
 0001:0001b995       __ehhandler$?activate@fileManager@@UAEX_N@Z 1001c995 f   testPlugin.obj
 0001:0001b995       __ehhandler$?timerEvent@fileManager@@EAEXPAVQTimerEvent@@@Z 1001c995 f   testPlugin.obj
 0001:0001b995       __ehhandler$?activate@testPlugin@@UAEX_N@Z 1001c995 f   testPlugin.obj
 0001:0001b9b0       __unwindfunclet$?closeEvent@testPlugin@@UAEXPAVQCloseEvent@@@Z$1 1001c9b0 f   testPlugin.obj
 0001:0001b9b9       __unwindfunclet$?closeEvent@testPlugin@@UAEXPAVQCloseEvent@@@Z$2 1001c9b9 f   testPlugin.obj
 0001:0001b9c2       __unwindfunclet$?closeEvent@testPlugin@@UAEXPAVQCloseEvent@@@Z$3 1001c9c2 f   testPlugin.obj
 0001:0001b9cb       __unwindfunclet$?closeEvent@testPlugin@@UAEXPAVQCloseEvent@@@Z$4 1001c9cb f   testPlugin.obj
 0001:0001b9d4       __unwindfunclet$?closeEvent@testPlugin@@UAEXPAVQCloseEvent@@@Z$5 1001c9d4 f   testPlugin.obj
 0001:0001b9dd       __unwindfunclet$?closeEvent@testPlugin@@UAEXPAVQCloseEvent@@@Z$6 1001c9dd f   testPlugin.obj
 0001:0001b9e6       __unwindfunclet$?closeEvent@testPlugin@@UAEXPAVQCloseEvent@@@Z$7 1001c9e6 f   testPlugin.obj
 0001:0001b9ef       __ehhandler$?closeEvent@testPlugin@@UAEXPAVQCloseEvent@@@Z 1001c9ef f   testPlugin.obj
 0001:0001ba10       __unwindfunclet$?db@testPlugin@@AAEXVQString@@@Z$0 1001ca10 f   testPlugin.obj
 0001:0001ba10       __unwindfunclet$?db@testPluginFromBase@@AAEXVQString@@@Z$0 1001ca10 f   testPlugin.obj
 0001:0001ba10       __unwindfunclet$?lviFind@fileManager@@AAEPAVQListViewItem@@PAV2@ABVQString@@@Z$0 1001ca10 f   testPlugin.obj
 0001:0001ba10       __unwindfunclet$?lock@configFile@@QAE_N_N@Z$2 1001ca10 f   testPlugin.obj
 0001:0001ba19       __ehhandler$?lviFind@fileManager@@AAEPAVQListViewItem@@PAV2@ABVQString@@@Z 1001ca19 f   testPlugin.obj
 0001:0001ba19       __ehhandler$?db@testPlugin@@AAEXVQString@@@Z 1001ca19 f   testPlugin.obj
 0001:0001ba19       __ehhandler$?lock@configFile@@QAE_N_N@Z 1001ca19 f   testPlugin.obj
 0001:0001ba19       __ehhandler$?db@testPluginFromBase@@AAEXVQString@@@Z 1001ca19 f   testPlugin.obj
 0001:0001ba34       __unwindfunclet$?rebootoptionchanged@launchEditorDlg@@QAEXXZ$0 1001ca34 f   testPlugin.obj
 0001:0001ba34       __unwindfunclet$?closeEvent@launchEditor@@UAEXPAVQCloseEvent@@@Z$0 1001ca34 f   testPlugin.obj
 0001:0001ba34       __unwindfunclet$?doRemove@launchEditorDlg@@QAEXXZ$0 1001ca34 f   testPlugin.obj
 0001:0001ba34       __unwindfunclet$?apply@testPlugin@@UAEXXZ$1 1001ca34 f   testPlugin.obj
 0001:0001ba34       __unwindfunclet$?navigateWSEditor@launchEditor@@AAEXXZ$0 1001ca34 f   testPlugin.obj
 0001:0001ba34       __unwindfunclet$?csiValueChanged@launchEditorDlg@@QAEXABVQString@@@Z$0 1001ca34 f   testPlugin.obj
 0001:0001ba34       __unwindfunclet$?apply@launchEditor@@UAEXXZ$0 1001ca34 f   testPlugin.obj
 0001:0001ba34       __unwindfunclet$?checkoutDir@testPlugin@@AAEXXZ$0 1001ca34 f   testPlugin.obj
 0001:0001ba34       __unwindfunclet$?downloadFile@testPlugin@@AAEXXZ$0 1001ca34 f   testPlugin.obj
 0001:0001ba34       __unwindfunclet$?checkoutFile@testPlugin@@AAEXXZ$0 1001ca34 f   testPlugin.obj
 0001:0001ba34       __unwindfunclet$?lockFile@testPlugin@@AAEXXZ$0 1001ca34 f   testPlugin.obj
 0001:0001ba34       __unwindfunclet$?doDirty@testPlugin@@AAEXXZ$0 1001ca34 f   testPlugin.obj
 0001:0001ba34       __unwindfunclet$?uploadFile@testPlugin@@AAEXXZ$0 1001ca34 f   testPlugin.obj
 0001:0001ba34       __unwindfunclet$?doHelp@testPlugin@@AAEXXZ$0 1001ca34 f   testPlugin.obj
 0001:0001ba34       __unwindfunclet$?unlockFile@testPlugin@@AAEXXZ$0 1001ca34 f   testPlugin.obj
 0001:0001ba34       __unwindfunclet$?doNavigate@testPlugin@@AAEXXZ$0 1001ca34 f   testPlugin.obj
 0001:0001ba34       __unwindfunclet$?unlockDir@testPlugin@@AAEXXZ$0 1001ca34 f   testPlugin.obj
 0001:0001ba34       __unwindfunclet$?uploadDir@testPlugin@@AAEXXZ$0 1001ca34 f   testPlugin.obj
 0001:0001ba34       __unwindfunclet$?downloadDir@testPlugin@@AAEXXZ$0 1001ca34 f   testPlugin.obj
 0001:0001ba34       __unwindfunclet$?dir@testPlugin@@AAEXXZ$0 1001ca34 f   testPlugin.obj
 0001:0001ba3d       __ehhandler$?downloadDir@testPlugin@@AAEXXZ 1001ca3d f   testPlugin.obj
 0001:0001ba3d       __ehhandler$?doRemove@launchEditorDlg@@QAEXXZ 1001ca3d f   testPlugin.obj
 0001:0001ba3d       __ehhandler$?unlockDir@testPlugin@@AAEXXZ 1001ca3d f   testPlugin.obj
 0001:0001ba3d       __ehhandler$?doHelp@testPlugin@@AAEXXZ 1001ca3d f   testPlugin.obj
 0001:0001ba3d       __ehhandler$?unlockFile@testPlugin@@AAEXXZ 1001ca3d f   testPlugin.obj
 0001:0001ba3d       __ehhandler$?doDirty@testPlugin@@AAEXXZ 1001ca3d f   testPlugin.obj
 0001:0001ba3d       __ehhandler$?uploadFile@testPlugin@@AAEXXZ 1001ca3d f   testPlugin.obj
 0001:0001ba3d       __ehhandler$?closeEvent@launchEditor@@UAEXPAVQCloseEvent@@@Z 1001ca3d f   testPlugin.obj
 0001:0001ba3d       __ehhandler$?checkoutFile@testPlugin@@AAEXXZ 1001ca3d f   testPlugin.obj
 0001:0001ba3d       __ehhandler$?lockFile@testPlugin@@AAEXXZ 1001ca3d f   testPlugin.obj
 0001:0001ba3d       __ehhandler$?checkoutDir@testPlugin@@AAEXXZ 1001ca3d f   testPlugin.obj
 0001:0001ba3d       __ehhandler$?downloadFile@testPlugin@@AAEXXZ 1001ca3d f   testPlugin.obj
 0001:0001ba3d       __ehhandler$?dir@testPlugin@@AAEXXZ 1001ca3d f   testPlugin.obj
 0001:0001ba3d       __ehhandler$?apply@testPlugin@@UAEXXZ 1001ca3d f   testPlugin.obj
 0001:0001ba3d       __ehhandler$?navigateWSEditor@launchEditor@@AAEXXZ 1001ca3d f   testPlugin.obj
 0001:0001ba3d       __ehhandler$?rebootoptionchanged@launchEditorDlg@@QAEXXZ 1001ca3d f   testPlugin.obj
 0001:0001ba3d       __ehhandler$?doNavigate@testPlugin@@AAEXXZ 1001ca3d f   testPlugin.obj
 0001:0001ba3d       __ehhandler$?csiValueChanged@launchEditorDlg@@QAEXABVQString@@@Z 1001ca3d f   testPlugin.obj
 0001:0001ba3d       __ehhandler$?apply@launchEditor@@UAEXXZ 1001ca3d f   testPlugin.obj
 0001:0001ba3d       __ehhandler$?uploadDir@testPlugin@@AAEXXZ 1001ca3d f   testPlugin.obj
 0001:0001ba58       __unwindfunclet$?menus@testPlugin@@UAE?AVQPopupMenuList@@XZ$1 1001ca58 f   testPlugin.obj
 0001:0001ba71       __ehhandler$?menus@testPlugin@@UAE?AVQPopupMenuList@@XZ 1001ca71 f   testPlugin.obj
 0001:0001ba8c       __unwindfunclet$?reply@testPlugin@@UAEXPAVresponse@@@Z$0 1001ca8c f   testPlugin.obj
 0001:0001ba95       __unwindfunclet$?reply@testPlugin@@UAEXPAVresponse@@@Z$1 1001ca95 f   testPlugin.obj
 0001:0001ba9e       __unwindfunclet$?reply@testPlugin@@UAEXPAVresponse@@@Z$2 1001ca9e f   testPlugin.obj
 0001:0001baa7       __unwindfunclet$?reply@testPlugin@@UAEXPAVresponse@@@Z$3 1001caa7 f   testPlugin.obj
 0001:0001bab0       __unwindfunclet$?reply@testPlugin@@UAEXPAVresponse@@@Z$4 1001cab0 f   testPlugin.obj
 0001:0001bab9       __unwindfunclet$?reply@testPlugin@@UAEXPAVresponse@@@Z$5 1001cab9 f   testPlugin.obj
 0001:0001bac2       __unwindfunclet$?reply@testPlugin@@UAEXPAVresponse@@@Z$6 1001cac2 f   testPlugin.obj
 0001:0001bacb       __unwindfunclet$?reply@testPlugin@@UAEXPAVresponse@@@Z$7 1001cacb f   testPlugin.obj
 0001:0001bad4       __unwindfunclet$?reply@testPlugin@@UAEXPAVresponse@@@Z$9 1001cad4 f   testPlugin.obj
 0001:0001badd       __ehhandler$?reply@testPlugin@@UAEXPAVresponse@@@Z 1001cadd f   testPlugin.obj
 0001:0001baf8       __unwindfunclet$?toolbars@testPlugin@@UAE?AVQDockWindowList@@XZ$1 1001caf8 f   testPlugin.obj
 0001:0001bb11       __ehhandler$?toolbars@testPlugin@@UAE?AVQDockWindowList@@XZ 1001cb11 f   testPlugin.obj
 0001:0001bb2c       __unwindfunclet$??0testPluginFromBase@@QAE@ABVQString@@00@Z$0 1001cb2c f   testPluginFromBase.obj
 0001:0001bb34       __unwindfunclet$??0testPluginFromBase@@QAE@ABVQString@@00@Z$1 1001cb34 f   testPluginFromBase.obj
 0001:0001bb3e       __unwindfunclet$??0testPluginFromBase@@QAE@ABVQString@@00@Z$3 1001cb3e f   testPluginFromBase.obj
 0001:0001bb48       __unwindfunclet$??0testPluginFromBase@@QAE@ABVQString@@00@Z$4 1001cb48 f   testPluginFromBase.obj
 0001:0001bb51       __unwindfunclet$??0testPluginFromBase@@QAE@ABVQString@@00@Z$5 1001cb51 f   testPluginFromBase.obj
 0001:0001bb5b       __unwindfunclet$??0testPluginFromBase@@QAE@ABVQString@@00@Z$6 1001cb5b f   testPluginFromBase.obj
 0001:0001bb65       __unwindfunclet$??0testPluginFromBase@@QAE@ABVQString@@00@Z$7 1001cb65 f   testPluginFromBase.obj
 0001:0001bb6e       __unwindfunclet$??0testPluginFromBase@@QAE@ABVQString@@00@Z$8 1001cb6e f   testPluginFromBase.obj
 0001:0001bb78       __unwindfunclet$??0testPluginFromBase@@QAE@ABVQString@@00@Z$9 1001cb78 f   testPluginFromBase.obj
 0001:0001bb82       __unwindfunclet$??0testPluginFromBase@@QAE@ABVQString@@00@Z$10 1001cb82 f   testPluginFromBase.obj
 0001:0001bb8b       __unwindfunclet$??0testPluginFromBase@@QAE@ABVQString@@00@Z$11 1001cb8b f   testPluginFromBase.obj
 0001:0001bb94       __unwindfunclet$??0testPluginFromBase@@QAE@ABVQString@@00@Z$12 1001cb94 f   testPluginFromBase.obj
 0001:0001bb9d       __unwindfunclet$??0testPluginFromBase@@QAE@ABVQString@@00@Z$13 1001cb9d f   testPluginFromBase.obj
 0001:0001bba6       __unwindfunclet$??0testPluginFromBase@@QAE@ABVQString@@00@Z$14 1001cba6 f   testPluginFromBase.obj
 0001:0001bbaf       __unwindfunclet$??0testPluginFromBase@@QAE@ABVQString@@00@Z$15 1001cbaf f   testPluginFromBase.obj
 0001:0001bbb8       __unwindfunclet$??0testPluginFromBase@@QAE@ABVQString@@00@Z$16 1001cbb8 f   testPluginFromBase.obj
 0001:0001bbc1       __unwindfunclet$??0testPluginFromBase@@QAE@ABVQString@@00@Z$17 1001cbc1 f   testPluginFromBase.obj
 0001:0001bbcb       __unwindfunclet$??0testPluginFromBase@@QAE@ABVQString@@00@Z$18 1001cbcb f   testPluginFromBase.obj
 0001:0001bbd4       __unwindfunclet$??0testPluginFromBase@@QAE@ABVQString@@00@Z$19 1001cbd4 f   testPluginFromBase.obj
 0001:0001bbde       __unwindfunclet$??0testPluginFromBase@@QAE@ABVQString@@00@Z$20 1001cbde f   testPluginFromBase.obj
 0001:0001bbe6       __unwindfunclet$??0testPluginFromBase@@QAE@ABVQString@@00@Z$21 1001cbe6 f   testPluginFromBase.obj
 0001:0001bbf0       __unwindfunclet$??0testPluginFromBase@@QAE@ABVQString@@00@Z$22 1001cbf0 f   testPluginFromBase.obj
 0001:0001bc0a       __unwindfunclet$??0testPluginFromBase@@QAE@ABVQString@@00@Z$23 1001cc0a f   testPluginFromBase.obj
 0001:0001bc24       __unwindfunclet$??0testPluginFromBase@@QAE@ABVQString@@00@Z$24 1001cc24 f   testPluginFromBase.obj
 0001:0001bc3e       __unwindfunclet$??0testPluginFromBase@@QAE@ABVQString@@00@Z$25 1001cc3e f   testPluginFromBase.obj
 0001:0001bc58       __unwindfunclet$??0testPluginFromBase@@QAE@ABVQString@@00@Z$27 1001cc58 f   testPluginFromBase.obj
 0001:0001bc61       __unwindfunclet$??0testPluginFromBase@@QAE@ABVQString@@00@Z$28 1001cc61 f   testPluginFromBase.obj
 0001:0001bc6a       __unwindfunclet$??0testPluginFromBase@@QAE@ABVQString@@00@Z$29 1001cc6a f   testPluginFromBase.obj
 0001:0001bc73       __unwindfunclet$??0testPluginFromBase@@QAE@ABVQString@@00@Z$30 1001cc73 f   testPluginFromBase.obj
 0001:0001bc7d       __unwindfunclet$??0testPluginFromBase@@QAE@ABVQString@@00@Z$31 1001cc7d f   testPluginFromBase.obj
 0001:0001bc97       __unwindfunclet$??0testPluginFromBase@@QAE@ABVQString@@00@Z$32 1001cc97 f   testPluginFromBase.obj
 0001:0001bcb1       __unwindfunclet$??0testPluginFromBase@@QAE@ABVQString@@00@Z$33 1001ccb1 f   testPluginFromBase.obj
 0001:0001bccb       __unwindfunclet$??0testPluginFromBase@@QAE@ABVQString@@00@Z$34 1001cccb f   testPluginFromBase.obj
 0001:0001bcea       __unwindfunclet$??0testPluginFromBase@@QAE@ABVQString@@00@Z$36 1001ccea f   testPluginFromBase.obj
 0001:0001bcf3       __unwindfunclet$??0testPluginFromBase@@QAE@ABVQString@@00@Z$37 1001ccf3 f   testPluginFromBase.obj
 0001:0001bcfc       __unwindfunclet$??0testPluginFromBase@@QAE@ABVQString@@00@Z$38 1001ccfc f   testPluginFromBase.obj
 0001:0001bd05       __unwindfunclet$??0testPluginFromBase@@QAE@ABVQString@@00@Z$39 1001cd05 f   testPluginFromBase.obj
 0001:0001bd0f       __unwindfunclet$??0testPluginFromBase@@QAE@ABVQString@@00@Z$40 1001cd0f f   testPluginFromBase.obj
 0001:0001bd2e       __unwindfunclet$??0testPluginFromBase@@QAE@ABVQString@@00@Z$41 1001cd2e f   testPluginFromBase.obj
 0001:0001bd4d       __unwindfunclet$??0testPluginFromBase@@QAE@ABVQString@@00@Z$42 1001cd4d f   testPluginFromBase.obj
 0001:0001bd6c       __unwindfunclet$??0testPluginFromBase@@QAE@ABVQString@@00@Z$43 1001cd6c f   testPluginFromBase.obj
 0001:0001bd8b       __unwindfunclet$??0testPluginFromBase@@QAE@ABVQString@@00@Z$45 1001cd8b f   testPluginFromBase.obj
 0001:0001bd94       __unwindfunclet$??0testPluginFromBase@@QAE@ABVQString@@00@Z$46 1001cd94 f   testPluginFromBase.obj
 0001:0001bd9d       __unwindfunclet$??0testPluginFromBase@@QAE@ABVQString@@00@Z$47 1001cd9d f   testPluginFromBase.obj
 0001:0001bda7       __unwindfunclet$??0testPluginFromBase@@QAE@ABVQString@@00@Z$48 1001cda7 f   testPluginFromBase.obj
 0001:0001bdc6       __unwindfunclet$??0testPluginFromBase@@QAE@ABVQString@@00@Z$49 1001cdc6 f   testPluginFromBase.obj
 0001:0001bde5       __unwindfunclet$??0testPluginFromBase@@QAE@ABVQString@@00@Z$50 1001cde5 f   testPluginFromBase.obj
 0001:0001be04       __unwindfunclet$??0testPluginFromBase@@QAE@ABVQString@@00@Z$51 1001ce04 f   testPluginFromBase.obj
 0001:0001be23       __unwindfunclet$??0testPluginFromBase@@QAE@ABVQString@@00@Z$53 1001ce23 f   testPluginFromBase.obj
 0001:0001be2c       __unwindfunclet$??0testPluginFromBase@@QAE@ABVQString@@00@Z$54 1001ce2c f   testPluginFromBase.obj
 0001:0001be35       __unwindfunclet$??0testPluginFromBase@@QAE@ABVQString@@00@Z$55 1001ce35 f   testPluginFromBase.obj
 0001:0001be3e       __ehhandler$??0testPluginFromBase@@QAE@ABVQString@@00@Z 1001ce3e f   testPluginFromBase.obj
 0001:0001be59       __unwindfunclet$?dirS@testPluginFromBase@@AAEXXZ$1 1001ce59 f   testPluginFromBase.obj
 0001:0001be62       __unwindfunclet$?dirS@testPluginFromBase@@AAEXXZ$3 1001ce62 f   testPluginFromBase.obj
 0001:0001be6b       __unwindfunclet$?dirS@testPluginFromBase@@AAEXXZ$4 1001ce6b f   testPluginFromBase.obj
 0001:0001be74       __unwindfunclet$?dirS@testPluginFromBase@@AAEXXZ$8 1001ce74 f   testPluginFromBase.obj
 0001:0001be7d       __unwindfunclet$?dirS@testPluginFromBase@@AAEXXZ$9 1001ce7d f   testPluginFromBase.obj
 0001:0001be86       __unwindfunclet$?dirS@testPluginFromBase@@AAEXXZ$10 1001ce86 f   testPluginFromBase.obj
 0001:0001be8f       __unwindfunclet$?dirS@testPluginFromBase@@AAEXXZ$11 1001ce8f f   testPluginFromBase.obj
 0001:0001be98       __ehhandler$?dirS@testPluginFromBase@@AAEXXZ 1001ce98 f   testPluginFromBase.obj
 0001:0001beb3       __unwindfunclet$?doDirtyS@testPluginFromBase@@AAEXXZ$1 1001ceb3 f   testPluginFromBase.obj
 0001:0001beb3       __unwindfunclet$?doCleanS@testPluginFromBase@@AAEXXZ$1 1001ceb3 f   testPluginFromBase.obj
 0001:0001bebc       __unwindfunclet$?doDirtyS@testPluginFromBase@@AAEXXZ$2 1001cebc f   testPluginFromBase.obj
 0001:0001bebc       __unwindfunclet$?doCleanS@testPluginFromBase@@AAEXXZ$2 1001cebc f   testPluginFromBase.obj
 0001:0001bec5       __ehhandler$?doCleanS@testPluginFromBase@@AAEXXZ 1001cec5 f   testPluginFromBase.obj
 0001:0001bec5       __ehhandler$?doDirtyS@testPluginFromBase@@AAEXXZ 1001cec5 f   testPluginFromBase.obj
 0001:0001bee0       __unwindfunclet$?init@testPluginFromBase@@MAEXXZ$2 1001cee0 f   testPluginFromBase.obj
 0001:0001bee0       __unwindfunclet$?clipBoardDataChanged@cfg_Table@@IAEXXZ$0 1001cee0 f   testPluginFromBase.obj
 0001:0001bee9       __ehhandler$?clipBoardDataChanged@cfg_Table@@IAEXXZ 1001cee9 f   testPluginFromBase.obj
 0001:0001bee9       __ehhandler$?init@testPluginFromBase@@MAEXXZ 1001cee9 f   testPluginFromBase.obj
 0001:0001bf04       __unwindfunclet$?saveFile@testPluginFromBase@@MAEXVQString@@@Z$0 1001cf04 f   testPluginFromBase.obj
 0001:0001bf04       __unwindfunclet$?loadFile@testPluginFromBase@@MAEXVQString@@@Z$0 1001cf04 f   testPluginFromBase.obj
 0001:0001bf0d       __unwindfunclet$?saveFile@testPluginFromBase@@MAEXVQString@@@Z$1 1001cf0d f   testPluginFromBase.obj
 0001:0001bf0d       __unwindfunclet$?loadFile@testPluginFromBase@@MAEXVQString@@@Z$1 1001cf0d f   testPluginFromBase.obj
 0001:0001bf16       __ehhandler$?loadFile@testPluginFromBase@@MAEXVQString@@@Z 1001cf16 f   testPluginFromBase.obj
 0001:0001bf16       __ehhandler$?saveFile@testPluginFromBase@@MAEXVQString@@@Z 1001cf16 f   testPluginFromBase.obj
 0001:0001bf31       __unwindfunclet$?checkoutFileS@testPluginFromBase@@AAEXXZ$1 1001cf31 f   testPluginFromBase.obj
 0001:0001bf31       __unwindfunclet$?downloadFileS@testPluginFromBase@@AAEXXZ$1 1001cf31 f   testPluginFromBase.obj
 0001:0001bf31       __unwindfunclet$?downloadDirS@testPluginFromBase@@AAEXXZ$2 1001cf31 f   testPluginFromBase.obj
 0001:0001bf31       __unwindfunclet$?unlockFileS@testPluginFromBase@@AAEXXZ$1 1001cf31 f   testPluginFromBase.obj
 0001:0001bf31       __unwindfunclet$?lockFileS@testPluginFromBase@@AAEXXZ$1 1001cf31 f   testPluginFromBase.obj
 0001:0001bf31       __unwindfunclet$?unlockDirS@testPluginFromBase@@AAEXXZ$2 1001cf31 f   testPluginFromBase.obj
 0001:0001bf31       __unwindfunclet$?uploadFileS@testPluginFromBase@@AAEXXZ$1 1001cf31 f   testPluginFromBase.obj
 0001:0001bf31       __unwindfunclet$?uploadDirS@testPluginFromBase@@AAEXXZ$2 1001cf31 f   testPluginFromBase.obj
 0001:0001bf31       __unwindfunclet$?checkoutDirS@testPluginFromBase@@AAEXXZ$2 1001cf31 f   testPluginFromBase.obj
 0001:0001bf3a       __unwindfunclet$?unlockFileS@testPluginFromBase@@AAEXXZ$2 1001cf3a f   testPluginFromBase.obj
 0001:0001bf3a       __unwindfunclet$?downloadDirS@testPluginFromBase@@AAEXXZ$3 1001cf3a f   testPluginFromBase.obj
 0001:0001bf3a       __unwindfunclet$?checkoutFileS@testPluginFromBase@@AAEXXZ$2 1001cf3a f   testPluginFromBase.obj
 0001:0001bf3a       __unwindfunclet$?uploadFileS@testPluginFromBase@@AAEXXZ$2 1001cf3a f   testPluginFromBase.obj
 0001:0001bf3a       __unwindfunclet$?lockFileS@testPluginFromBase@@AAEXXZ$2 1001cf3a f   testPluginFromBase.obj
 0001:0001bf3a       __unwindfunclet$?unlockDirS@testPluginFromBase@@AAEXXZ$3 1001cf3a f   testPluginFromBase.obj
 0001:0001bf3a       __unwindfunclet$?uploadDirS@testPluginFromBase@@AAEXXZ$3 1001cf3a f   testPluginFromBase.obj
 0001:0001bf3a       __unwindfunclet$?checkoutDirS@testPluginFromBase@@AAEXXZ$3 1001cf3a f   testPluginFromBase.obj
 0001:0001bf3a       __unwindfunclet$?downloadFileS@testPluginFromBase@@AAEXXZ$2 1001cf3a f   testPluginFromBase.obj
 0001:0001bf43       __unwindfunclet$?downloadFileS@testPluginFromBase@@AAEXXZ$5 1001cf43 f   testPluginFromBase.obj
 0001:0001bf43       __unwindfunclet$?checkoutDirS@testPluginFromBase@@AAEXXZ$6 1001cf43 f   testPluginFromBase.obj
 0001:0001bf43       __unwindfunclet$?uploadFileS@testPluginFromBase@@AAEXXZ$5 1001cf43 f   testPluginFromBase.obj
 0001:0001bf43       __unwindfunclet$?checkoutFileS@testPluginFromBase@@AAEXXZ$5 1001cf43 f   testPluginFromBase.obj
 0001:0001bf43       __unwindfunclet$?unlockFileS@testPluginFromBase@@AAEXXZ$5 1001cf43 f   testPluginFromBase.obj
 0001:0001bf43       __unwindfunclet$?uploadDirS@testPluginFromBase@@AAEXXZ$6 1001cf43 f   testPluginFromBase.obj
 0001:0001bf43       __unwindfunclet$?unlockDirS@testPluginFromBase@@AAEXXZ$6 1001cf43 f   testPluginFromBase.obj
 0001:0001bf43       __unwindfunclet$?downloadDirS@testPluginFromBase@@AAEXXZ$6 1001cf43 f   testPluginFromBase.obj
 0001:0001bf43       __unwindfunclet$?lockFileS@testPluginFromBase@@AAEXXZ$5 1001cf43 f   testPluginFromBase.obj
 0001:0001bf4c       __unwindfunclet$?downloadDirS@testPluginFromBase@@AAEXXZ$7 1001cf4c f   testPluginFromBase.obj
 0001:0001bf4c       __unwindfunclet$?unlockFileS@testPluginFromBase@@AAEXXZ$6 1001cf4c f   testPluginFromBase.obj
 0001:0001bf4c       __unwindfunclet$?uploadDirS@testPluginFromBase@@AAEXXZ$7 1001cf4c f   testPluginFromBase.obj
 0001:0001bf4c       __unwindfunclet$?uploadFileS@testPluginFromBase@@AAEXXZ$6 1001cf4c f   testPluginFromBase.obj
 0001:0001bf4c       __unwindfunclet$?checkoutFileS@testPluginFromBase@@AAEXXZ$6 1001cf4c f   testPluginFromBase.obj
 0001:0001bf4c       __unwindfunclet$?lockFileS@testPluginFromBase@@AAEXXZ$6 1001cf4c f   testPluginFromBase.obj
 0001:0001bf4c       __unwindfunclet$?checkoutDirS@testPluginFromBase@@AAEXXZ$7 1001cf4c f   testPluginFromBase.obj
 0001:0001bf4c       __unwindfunclet$?unlockDirS@testPluginFromBase@@AAEXXZ$7 1001cf4c f   testPluginFromBase.obj
 0001:0001bf4c       __unwindfunclet$?downloadFileS@testPluginFromBase@@AAEXXZ$6 1001cf4c f   testPluginFromBase.obj
 0001:0001bf55       __unwindfunclet$?uploadDirS@testPluginFromBase@@AAEXXZ$8 1001cf55 f   testPluginFromBase.obj
 0001:0001bf55       __unwindfunclet$?downloadDirS@testPluginFromBase@@AAEXXZ$8 1001cf55 f   testPluginFromBase.obj
 0001:0001bf55       __unwindfunclet$?checkoutDirS@testPluginFromBase@@AAEXXZ$8 1001cf55 f   testPluginFromBase.obj
 0001:0001bf55       __unwindfunclet$?unlockDirS@testPluginFromBase@@AAEXXZ$8 1001cf55 f   testPluginFromBase.obj
 0001:0001bf55       __unwindfunclet$?checkoutFileS@testPluginFromBase@@AAEXXZ$7 1001cf55 f   testPluginFromBase.obj
 0001:0001bf55       __unwindfunclet$?unlockFileS@testPluginFromBase@@AAEXXZ$7 1001cf55 f   testPluginFromBase.obj
 0001:0001bf55       __unwindfunclet$?lockFileS@testPluginFromBase@@AAEXXZ$7 1001cf55 f   testPluginFromBase.obj
 0001:0001bf55       __unwindfunclet$?uploadFileS@testPluginFromBase@@AAEXXZ$7 1001cf55 f   testPluginFromBase.obj
 0001:0001bf55       __unwindfunclet$?downloadFileS@testPluginFromBase@@AAEXXZ$7 1001cf55 f   testPluginFromBase.obj
 0001:0001bf5e       __unwindfunclet$?uploadFileS@testPluginFromBase@@AAEXXZ$8 1001cf5e f   testPluginFromBase.obj
 0001:0001bf5e       __unwindfunclet$?lockFileS@testPluginFromBase@@AAEXXZ$8 1001cf5e f   testPluginFromBase.obj
 0001:0001bf5e       __unwindfunclet$?downloadDirS@testPluginFromBase@@AAEXXZ$9 1001cf5e f   testPluginFromBase.obj
 0001:0001bf5e       __unwindfunclet$?unlockFileS@testPluginFromBase@@AAEXXZ$8 1001cf5e f   testPluginFromBase.obj
 0001:0001bf5e       __unwindfunclet$?checkoutFileS@testPluginFromBase@@AAEXXZ$8 1001cf5e f   testPluginFromBase.obj
 0001:0001bf5e       __unwindfunclet$?unlockDirS@testPluginFromBase@@AAEXXZ$9 1001cf5e f   testPluginFromBase.obj
 0001:0001bf5e       __unwindfunclet$?checkoutDirS@testPluginFromBase@@AAEXXZ$9 1001cf5e f   testPluginFromBase.obj
 0001:0001bf5e       __unwindfunclet$?uploadDirS@testPluginFromBase@@AAEXXZ$9 1001cf5e f   testPluginFromBase.obj
 0001:0001bf5e       __unwindfunclet$?downloadFileS@testPluginFromBase@@AAEXXZ$8 1001cf5e f   testPluginFromBase.obj
 0001:0001bf67       __ehhandler$?lockFileS@testPluginFromBase@@AAEXXZ 1001cf67 f   testPluginFromBase.obj
 0001:0001bf67       __ehhandler$?downloadFileS@testPluginFromBase@@AAEXXZ 1001cf67 f   testPluginFromBase.obj
 0001:0001bf67       __ehhandler$?checkoutDirS@testPluginFromBase@@AAEXXZ 1001cf67 f   testPluginFromBase.obj
 0001:0001bf67       __ehhandler$?downloadDirS@testPluginFromBase@@AAEXXZ 1001cf67 f   testPluginFromBase.obj
 0001:0001bf67       __ehhandler$?unlockDirS@testPluginFromBase@@AAEXXZ 1001cf67 f   testPluginFromBase.obj
 0001:0001bf67       __ehhandler$?unlockFileS@testPluginFromBase@@AAEXXZ 1001cf67 f   testPluginFromBase.obj
 0001:0001bf67       __ehhandler$?uploadFileS@testPluginFromBase@@AAEXXZ 1001cf67 f   testPluginFromBase.obj
 0001:0001bf67       __ehhandler$?checkoutFileS@testPluginFromBase@@AAEXXZ 1001cf67 f   testPluginFromBase.obj
 0001:0001bf67       __ehhandler$?uploadDirS@testPluginFromBase@@AAEXXZ 1001cf67 f   testPluginFromBase.obj
 0001:0001bf82       __unwindfunclet$??0workstationCustomTable@@QAE@PAVQWidget@@PBD@Z$0 1001cf82 f   workstationCustomTable.obj
 0001:0001bf8a       __unwindfunclet$??0workstationCustomTable@@QAE@PAVQWidget@@PBD@Z$1 1001cf8a f   workstationCustomTable.obj
 0001:0001bf93       __unwindfunclet$??0workstationCustomTable@@QAE@PAVQWidget@@PBD@Z$2 1001cf93 f   workstationCustomTable.obj
 0001:0001bf9c       __unwindfunclet$??0workstationCustomTable@@QAE@PAVQWidget@@PBD@Z$3 1001cf9c f   workstationCustomTable.obj
 0001:0001bfa5       __unwindfunclet$??0workstationCustomTable@@QAE@PAVQWidget@@PBD@Z$4 1001cfa5 f   workstationCustomTable.obj
 0001:0001bfae       __ehhandler$??0workstationCustomTable@@QAE@PAVQWidget@@PBD@Z 1001cfae f   workstationCustomTable.obj
 0001:0001bfc9       __unwindfunclet$??0workstationDockWindow@@QAE@PAVQWidget@@PBDI@Z$0 1001cfc9 f   workstationdockwindowimpl.obj
 0001:0001bfd1       __unwindfunclet$??0workstationDockWindow@@QAE@PAVQWidget@@PBDI@Z$1 1001cfd1 f   workstationdockwindowimpl.obj
 0001:0001bfda       __unwindfunclet$??0workstationDockWindow@@QAE@PAVQWidget@@PBDI@Z$2 1001cfda f   workstationdockwindowimpl.obj
 0001:0001bfe3       __unwindfunclet$??0workstationDockWindow@@QAE@PAVQWidget@@PBDI@Z$3 1001cfe3 f   workstationdockwindowimpl.obj
 0001:0001bfec       __unwindfunclet$??0workstationDockWindow@@QAE@PAVQWidget@@PBDI@Z$4 1001cfec f   workstationdockwindowimpl.obj
 0001:0001bff5       __unwindfunclet$??0workstationDockWindow@@QAE@PAVQWidget@@PBDI@Z$5 1001cff5 f   workstationdockwindowimpl.obj
 0001:0001bffe       __unwindfunclet$??0workstationDockWindow@@QAE@PAVQWidget@@PBDI@Z$6 1001cffe f   workstationdockwindowimpl.obj
 0001:0001c007       __ehhandler$??0workstationDockWindow@@QAE@PAVQWidget@@PBDI@Z 1001d007 f   workstationdockwindowimpl.obj
 0001:0001c022       __unwindfunclet$??0workstationEditor@@QAE@ABVQString@@00@Z$0 1001d022 f   workstationEditor.obj
 0001:0001c02a       __unwindfunclet$??0workstationEditor@@QAE@ABVQString@@00@Z$1 1001d02a f   workstationEditor.obj
 0001:0001c035       __unwindfunclet$??0workstationEditor@@QAE@ABVQString@@00@Z$2 1001d035 f   workstationEditor.obj
 0001:0001c040       __unwindfunclet$??0workstationEditor@@QAE@ABVQString@@00@Z$3 1001d040 f   workstationEditor.obj
 0001:0001c04e       __unwindfunclet$??0workstationEditor@@QAE@ABVQString@@00@Z$4 1001d04e f   workstationEditor.obj
 0001:0001c05c       __unwindfunclet$??0workstationEditor@@QAE@ABVQString@@00@Z$5 1001d05c f   workstationEditor.obj
 0001:0001c06b       __unwindfunclet$??0workstationEditor@@QAE@ABVQString@@00@Z$6 1001d06b f   workstationEditor.obj
 0001:0001c074       __unwindfunclet$??0workstationEditor@@QAE@ABVQString@@00@Z$7 1001d074 f   workstationEditor.obj
 0001:0001c07e       __unwindfunclet$??0workstationEditor@@QAE@ABVQString@@00@Z$8 1001d07e f   workstationEditor.obj
 0001:0001c088       __unwindfunclet$??0workstationEditor@@QAE@ABVQString@@00@Z$9 1001d088 f   workstationEditor.obj
 0001:0001c091       __unwindfunclet$??0workstationEditor@@QAE@ABVQString@@00@Z$10 1001d091 f   workstationEditor.obj
 0001:0001c09b       __unwindfunclet$??0workstationEditor@@QAE@ABVQString@@00@Z$11 1001d09b f   workstationEditor.obj
 0001:0001c0a5       __unwindfunclet$??0workstationEditor@@QAE@ABVQString@@00@Z$12 1001d0a5 f   workstationEditor.obj
 0001:0001c0bf       __unwindfunclet$??0workstationEditor@@QAE@ABVQString@@00@Z$13 1001d0bf f   workstationEditor.obj
 0001:0001c0d9       __unwindfunclet$??0workstationEditor@@QAE@ABVQString@@00@Z$14 1001d0d9 f   workstationEditor.obj
 0001:0001c0f3       __unwindfunclet$??0workstationEditor@@QAE@ABVQString@@00@Z$15 1001d0f3 f   workstationEditor.obj
 0001:0001c10d       __unwindfunclet$??0workstationEditor@@QAE@ABVQString@@00@Z$17 1001d10d f   workstationEditor.obj
 0001:0001c116       __unwindfunclet$??0workstationEditor@@QAE@ABVQString@@00@Z$18 1001d116 f   workstationEditor.obj
 0001:0001c11f       __unwindfunclet$??0workstationEditor@@QAE@ABVQString@@00@Z$19 1001d11f f   workstationEditor.obj
 0001:0001c128       __unwindfunclet$??0workstationEditor@@QAE@ABVQString@@00@Z$20 1001d128 f   workstationEditor.obj
 0001:0001c132       __unwindfunclet$??0workstationEditor@@QAE@ABVQString@@00@Z$21 1001d132 f   workstationEditor.obj
 0001:0001c14c       __unwindfunclet$??0workstationEditor@@QAE@ABVQString@@00@Z$22 1001d14c f   workstationEditor.obj
 0001:0001c166       __unwindfunclet$??0workstationEditor@@QAE@ABVQString@@00@Z$23 1001d166 f   workstationEditor.obj
 0001:0001c180       __unwindfunclet$??0workstationEditor@@QAE@ABVQString@@00@Z$24 1001d180 f   workstationEditor.obj
 0001:0001c19f       __unwindfunclet$??0workstationEditor@@QAE@ABVQString@@00@Z$26 1001d19f f   workstationEditor.obj
 0001:0001c1a8       __unwindfunclet$??0workstationEditor@@QAE@ABVQString@@00@Z$27 1001d1a8 f   workstationEditor.obj
 0001:0001c1b1       __unwindfunclet$??0workstationEditor@@QAE@ABVQString@@00@Z$28 1001d1b1 f   workstationEditor.obj
 0001:0001c1ba       __unwindfunclet$??0workstationEditor@@QAE@ABVQString@@00@Z$29 1001d1ba f   workstationEditor.obj
 0001:0001c1c3       __unwindfunclet$??0workstationEditor@@QAE@ABVQString@@00@Z$30 1001d1c3 f   workstationEditor.obj
 0001:0001c1cc       __ehhandler$??0workstationEditor@@QAE@ABVQString@@00@Z 1001d1cc f   workstationEditor.obj
 0001:0001c1e7       __unwindfunclet$??1workstationEditor@@UAE@XZ$0 1001d1e7 f   workstationEditor.obj
 0001:0001c1ef       __unwindfunclet$??1workstationEditor@@UAE@XZ$1 1001d1ef f   workstationEditor.obj
 0001:0001c1fa       __unwindfunclet$??1workstationEditor@@UAE@XZ$2 1001d1fa f   workstationEditor.obj
 0001:0001c205       __unwindfunclet$??1workstationEditor@@UAE@XZ$3 1001d205 f   workstationEditor.obj
 0001:0001c213       __unwindfunclet$??1workstationEditor@@UAE@XZ$4 1001d213 f   workstationEditor.obj
 0001:0001c221       __unwindfunclet$??1workstationEditor@@UAE@XZ$5 1001d221 f   workstationEditor.obj
 0001:0001c230       __ehhandler$??1workstationEditor@@UAE@XZ 1001d230 f   workstationEditor.obj
 0001:0001c24b       __unwindfunclet$?activate@workstationEditor@@UAEX_N@Z$0 1001d24b f   workstationEditor.obj
 0001:0001c254       __unwindfunclet$?activate@workstationEditor@@UAEX_N@Z$2 1001d254 f   workstationEditor.obj
 0001:0001c25d       __unwindfunclet$?activate@workstationEditor@@UAEX_N@Z$4 1001d25d f   workstationEditor.obj
 0001:0001c266       __unwindfunclet$?activate@workstationEditor@@UAEX_N@Z$5 1001d266 f   workstationEditor.obj
 0001:0001c26f       __unwindfunclet$?activate@workstationEditor@@UAEX_N@Z$6 1001d26f f   workstationEditor.obj
 0001:0001c278       __unwindfunclet$?activate@workstationEditor@@UAEX_N@Z$7 1001d278 f   workstationEditor.obj
 0001:0001c281       __ehhandler$?activate@workstationEditor@@UAEX_N@Z 1001d281 f   workstationEditor.obj
 0001:0001c29c       __unwindfunclet$?apply@workstationEditor@@UAEXXZ$0 1001d29c f   workstationEditor.obj
 0001:0001c2a5       __unwindfunclet$?apply@workstationEditor@@UAEXXZ$2 1001d2a5 f   workstationEditor.obj
 0001:0001c2ae       __unwindfunclet$?apply@workstationEditor@@UAEXXZ$4 1001d2ae f   workstationEditor.obj
 0001:0001c2b7       __ehhandler$?apply@workstationEditor@@UAEXXZ 1001d2b7 f   workstationEditor.obj
 0001:0001c2d2       __unwindfunclet$?closeEvent@workstationEditor@@UAEXPAVQCloseEvent@@@Z$0 1001d2d2 f   workstationEditor.obj
 0001:0001c2db       __unwindfunclet$?closeEvent@workstationEditor@@UAEXPAVQCloseEvent@@@Z$2 1001d2db f   workstationEditor.obj
 0001:0001c2e4       __ehhandler$?closeEvent@workstationEditor@@UAEXPAVQCloseEvent@@@Z 1001d2e4 f   workstationEditor.obj
 0001:0001c2ff       __unwindfunclet$?reply@workstationEditor@@UAEXPAVresponse@@@Z$0 1001d2ff f   workstationEditor.obj
 0001:0001c308       __unwindfunclet$?reply@workstationEditor@@UAEXPAVresponse@@@Z$1 1001d308 f   workstationEditor.obj
 0001:0001c311       __unwindfunclet$?reply@workstationEditor@@UAEXPAVresponse@@@Z$2 1001d311 f   workstationEditor.obj
 0001:0001c31a       __unwindfunclet$?reply@workstationEditor@@UAEXPAVresponse@@@Z$3 1001d31a f   workstationEditor.obj
 0001:0001c323       __unwindfunclet$?reply@workstationEditor@@UAEXPAVresponse@@@Z$4 1001d323 f   workstationEditor.obj
 0001:0001c32c       __unwindfunclet$?reply@workstationEditor@@UAEXPAVresponse@@@Z$5 1001d32c f   workstationEditor.obj
 0001:0001c335       __unwindfunclet$?reply@workstationEditor@@UAEXPAVresponse@@@Z$6 1001d335 f   workstationEditor.obj
 0001:0001c33e       __unwindfunclet$?reply@workstationEditor@@UAEXPAVresponse@@@Z$7 1001d33e f   workstationEditor.obj
 0001:0001c347       __unwindfunclet$?reply@workstationEditor@@UAEXPAVresponse@@@Z$8 1001d347 f   workstationEditor.obj
 0001:0001c350       __unwindfunclet$?reply@workstationEditor@@UAEXPAVresponse@@@Z$9 1001d350 f   workstationEditor.obj
 0001:0001c359       __unwindfunclet$?reply@workstationEditor@@UAEXPAVresponse@@@Z$10 1001d359 f   workstationEditor.obj
 0001:0001c362       __unwindfunclet$?reply@workstationEditor@@UAEXPAVresponse@@@Z$11 1001d362 f   workstationEditor.obj
 0001:0001c36b       __unwindfunclet$?reply@workstationEditor@@UAEXPAVresponse@@@Z$12 1001d36b f   workstationEditor.obj
 0001:0001c374       __unwindfunclet$?reply@workstationEditor@@UAEXPAVresponse@@@Z$13 1001d374 f   workstationEditor.obj
 0001:0001c37d       __ehhandler$?reply@workstationEditor@@UAEXPAVresponse@@@Z 1001d37d f   workstationEditor.obj
 0001:0001c398       __unwindfunclet$??0workstationEditorDlg@@QAE@ABVQString@@PAVQWidget@@PBDI@Z$0 1001d398 f   workstationeditordlgimpl.obj
 0001:0001c3a0       __unwindfunclet$??0workstationEditorDlg@@QAE@ABVQString@@PAVQWidget@@PBDI@Z$1 1001d3a0 f   workstationeditordlgimpl.obj
 0001:0001c3af       __unwindfunclet$??0workstationEditorDlg@@QAE@ABVQString@@PAVQWidget@@PBDI@Z$2 1001d3af f   workstationeditordlgimpl.obj
 0001:0001c3b8       __unwindfunclet$??0workstationEditorDlg@@QAE@ABVQString@@PAVQWidget@@PBDI@Z$3 1001d3b8 f   workstationeditordlgimpl.obj
 0001:0001c3c1       __unwindfunclet$??0workstationEditorDlg@@QAE@ABVQString@@PAVQWidget@@PBDI@Z$4 1001d3c1 f   workstationeditordlgimpl.obj
 0001:0001c3ca       __unwindfunclet$??0workstationEditorDlg@@QAE@ABVQString@@PAVQWidget@@PBDI@Z$5 1001d3ca f   workstationeditordlgimpl.obj
 0001:0001c3d3       __ehhandler$??0workstationEditorDlg@@QAE@ABVQString@@PAVQWidget@@PBDI@Z 1001d3d3 f   workstationeditordlgimpl.obj
 0001:0001c3ee       __unwindfunclet$??1workstationEditorDlg@@UAE@XZ$0 1001d3ee f   workstationeditordlgimpl.obj
 0001:0001c3f6       __ehhandler$??1workstationEditorDlg@@UAE@XZ 1001d3f6 f   workstationeditordlgimpl.obj
 0001:0001c411       __unwindfunclet$?doAdd@workstationEditorDlg@@AAEXXZ$0 1001d411 f   workstationeditordlgimpl.obj
 0001:0001c41c       __unwindfunclet$?doAdd@workstationEditorDlg@@AAEXXZ$1 1001d41c f   workstationeditordlgimpl.obj
 0001:0001c425       __unwindfunclet$?doAdd@workstationEditorDlg@@AAEXXZ$2 1001d425 f   workstationeditordlgimpl.obj
 0001:0001c42e       __unwindfunclet$?doAdd@workstationEditorDlg@@AAEXXZ$3 1001d42e f   workstationeditordlgimpl.obj
 0001:0001c437       __unwindfunclet$?doAdd@workstationEditorDlg@@AAEXXZ$4 1001d437 f   workstationeditordlgimpl.obj
 0001:0001c440       __unwindfunclet$?doAdd@workstationEditorDlg@@AAEXXZ$5 1001d440 f   workstationeditordlgimpl.obj
 0001:0001c449       __unwindfunclet$?doAdd@workstationEditorDlg@@AAEXXZ$6 1001d449 f   workstationeditordlgimpl.obj
 0001:0001c452       __unwindfunclet$?doAdd@workstationEditorDlg@@AAEXXZ$7 1001d452 f   workstationeditordlgimpl.obj
 0001:0001c45b       __unwindfunclet$?doAdd@workstationEditorDlg@@AAEXXZ$8 1001d45b f   workstationeditordlgimpl.obj
 0001:0001c465       __unwindfunclet$?doAdd@workstationEditorDlg@@AAEXXZ$9 1001d465 f   workstationeditordlgimpl.obj
 0001:0001c47f       __unwindfunclet$?doAdd@workstationEditorDlg@@AAEXXZ$10 1001d47f f   workstationeditordlgimpl.obj
 0001:0001c488       __unwindfunclet$?doAdd@workstationEditorDlg@@AAEXXZ$12 1001d488 f   workstationeditordlgimpl.obj
 0001:0001c491       __unwindfunclet$?doAdd@workstationEditorDlg@@AAEXXZ$13 1001d491 f   workstationeditordlgimpl.obj
 0001:0001c49a       __unwindfunclet$?doAdd@workstationEditorDlg@@AAEXXZ$14 1001d49a f   workstationeditordlgimpl.obj
 0001:0001c4a3       __ehhandler$?doAdd@workstationEditorDlg@@AAEXXZ 1001d4a3 f   workstationeditordlgimpl.obj
 0001:0001c4c1       __unwindfunclet$?load@workstationEditorDlg@@QAE_NABVQString@@@Z$0 1001d4c1 f   workstationeditordlgimpl.obj
 0001:0001c4ca       __unwindfunclet$?load@workstationEditorDlg@@QAE_NABVQString@@@Z$1 1001d4ca f   workstationeditordlgimpl.obj
 0001:0001c4d3       __unwindfunclet$?load@workstationEditorDlg@@QAE_NABVQString@@@Z$2 1001d4d3 f   workstationeditordlgimpl.obj
 0001:0001c4dc       __unwindfunclet$?load@workstationEditorDlg@@QAE_NABVQString@@@Z$3 1001d4dc f   workstationeditordlgimpl.obj
 0001:0001c4e8       __unwindfunclet$?load@workstationEditorDlg@@QAE_NABVQString@@@Z$4 1001d4e8 f   workstationeditordlgimpl.obj
 0001:0001c4f1       __unwindfunclet$?load@workstationEditorDlg@@QAE_NABVQString@@@Z$5 1001d4f1 f   workstationeditordlgimpl.obj
 0001:0001c4fa       __unwindfunclet$?load@workstationEditorDlg@@QAE_NABVQString@@@Z$6 1001d4fa f   workstationeditordlgimpl.obj
 0001:0001c503       __unwindfunclet$?load@workstationEditorDlg@@QAE_NABVQString@@@Z$7 1001d503 f   workstationeditordlgimpl.obj
 0001:0001c50c       __unwindfunclet$?load@workstationEditorDlg@@QAE_NABVQString@@@Z$8 1001d50c f   workstationeditordlgimpl.obj
 0001:0001c515       __unwindfunclet$?load@workstationEditorDlg@@QAE_NABVQString@@@Z$9 1001d515 f   workstationeditordlgimpl.obj
 0001:0001c51e       __unwindfunclet$?load@workstationEditorDlg@@QAE_NABVQString@@@Z$10 1001d51e f   workstationeditordlgimpl.obj
 0001:0001c527       __unwindfunclet$?load@workstationEditorDlg@@QAE_NABVQString@@@Z$11 1001d527 f   workstationeditordlgimpl.obj
 0001:0001c530       __unwindfunclet$?load@workstationEditorDlg@@QAE_NABVQString@@@Z$12 1001d530 f   workstationeditordlgimpl.obj
 0001:0001c53a       __unwindfunclet$?load@workstationEditorDlg@@QAE_NABVQString@@@Z$13 1001d53a f   workstationeditordlgimpl.obj
 0001:0001c554       __unwindfunclet$?load@workstationEditorDlg@@QAE_NABVQString@@@Z$14 1001d554 f   workstationeditordlgimpl.obj
 0001:0001c56e       __unwindfunclet$?load@workstationEditorDlg@@QAE_NABVQString@@@Z$15 1001d56e f   workstationeditordlgimpl.obj
 0001:0001c577       __ehhandler$?load@workstationEditorDlg@@QAE_NABVQString@@@Z 1001d577 f   workstationeditordlgimpl.obj
 0001:0001c595       __unwindfunclet$?newBNCSSystemIni@workstationEditorDlg@@AAEXH_N0@Z$0 1001d595 f   workstationeditordlgimpl.obj
 0001:0001c59e       __unwindfunclet$?newBNCSSystemIni@workstationEditorDlg@@AAEXH_N0@Z$1 1001d59e f   workstationeditordlgimpl.obj
 0001:0001c5a7       __unwindfunclet$?newBNCSSystemIni@workstationEditorDlg@@AAEXH_N0@Z$2 1001d5a7 f   workstationeditordlgimpl.obj
 0001:0001c5b0       __unwindfunclet$?newBNCSSystemIni@workstationEditorDlg@@AAEXH_N0@Z$3 1001d5b0 f   workstationeditordlgimpl.obj
 0001:0001c5b9       __unwindfunclet$?newBNCSSystemIni@workstationEditorDlg@@AAEXH_N0@Z$4 1001d5b9 f   workstationeditordlgimpl.obj
 0001:0001c5c2       __unwindfunclet$?newBNCSSystemIni@workstationEditorDlg@@AAEXH_N0@Z$5 1001d5c2 f   workstationeditordlgimpl.obj
 0001:0001c5cb       __unwindfunclet$?newBNCSSystemIni@workstationEditorDlg@@AAEXH_N0@Z$6 1001d5cb f   workstationeditordlgimpl.obj
 0001:0001c5d4       __unwindfunclet$?newBNCSSystemIni@workstationEditorDlg@@AAEXH_N0@Z$7 1001d5d4 f   workstationeditordlgimpl.obj
 0001:0001c5dd       __unwindfunclet$?newBNCSSystemIni@workstationEditorDlg@@AAEXH_N0@Z$8 1001d5dd f   workstationeditordlgimpl.obj
 0001:0001c5e6       __ehhandler$?newBNCSSystemIni@workstationEditorDlg@@AAEXH_N0@Z 1001d5e6 f   workstationeditordlgimpl.obj
 0001:0001c601       __unwindfunclet$?save@workstationEditorDlg@@QAEXXZ$0 1001d601 f   workstationeditordlgimpl.obj
 0001:0001c60a       __unwindfunclet$?save@workstationEditorDlg@@QAEXXZ$1 1001d60a f   workstationeditordlgimpl.obj
 0001:0001c616       __unwindfunclet$?save@workstationEditorDlg@@QAEXXZ$2 1001d616 f   workstationeditordlgimpl.obj
 0001:0001c61f       __unwindfunclet$?save@workstationEditorDlg@@QAEXXZ$3 1001d61f f   workstationeditordlgimpl.obj
 0001:0001c628       __unwindfunclet$?save@workstationEditorDlg@@QAEXXZ$4 1001d628 f   workstationeditordlgimpl.obj
 0001:0001c631       __unwindfunclet$?save@workstationEditorDlg@@QAEXXZ$5 1001d631 f   workstationeditordlgimpl.obj
 0001:0001c63a       __unwindfunclet$?save@workstationEditorDlg@@QAEXXZ$6 1001d63a f   workstationeditordlgimpl.obj
 0001:0001c643       __unwindfunclet$?save@workstationEditorDlg@@QAEXXZ$7 1001d643 f   workstationeditordlgimpl.obj
 0001:0001c64c       __unwindfunclet$?save@workstationEditorDlg@@QAEXXZ$8 1001d64c f   workstationeditordlgimpl.obj
 0001:0001c655       __unwindfunclet$?save@workstationEditorDlg@@QAEXXZ$9 1001d655 f   workstationeditordlgimpl.obj
 0001:0001c65e       __unwindfunclet$?save@workstationEditorDlg@@QAEXXZ$10 1001d65e f   workstationeditordlgimpl.obj
 0001:0001c667       __ehhandler$?save@workstationEditorDlg@@QAEXXZ 1001d667 f   workstationeditordlgimpl.obj
 0001:0001c685       __unwindfunclet$?toXML@@YA?AVQString@@ABV1@@Z$0 1001d685 f   workstationeditordlgimpl.obj
 0001:0001c69f       __unwindfunclet$?toXML@@YA?AVQString@@ABV1@@Z$1 1001d69f f   workstationeditordlgimpl.obj
 0001:0001c6a8       __unwindfunclet$?toXML@@YA?AVQString@@ABV1@@Z$2 1001d6a8 f   workstationeditordlgimpl.obj
 0001:0001c6b1       __unwindfunclet$?toXML@@YA?AVQString@@ABV1@@Z$3 1001d6b1 f   workstationeditordlgimpl.obj
 0001:0001c6ba       __unwindfunclet$?toXML@@YA?AVQString@@ABV1@@Z$4 1001d6ba f   workstationeditordlgimpl.obj
 0001:0001c6c3       __unwindfunclet$?toXML@@YA?AVQString@@ABV1@@Z$5 1001d6c3 f   workstationeditordlgimpl.obj
 0001:0001c6cc       __unwindfunclet$?toXML@@YA?AVQString@@ABV1@@Z$6 1001d6cc f   workstationeditordlgimpl.obj
 0001:0001c6d5       __unwindfunclet$?toXML@@YA?AVQString@@ABV1@@Z$7 1001d6d5 f   workstationeditordlgimpl.obj
 0001:0001c6de       __unwindfunclet$?toXML@@YA?AVQString@@ABV1@@Z$8 1001d6de f   workstationeditordlgimpl.obj
 0001:0001c6e7       __unwindfunclet$?toXML@@YA?AVQString@@ABV1@@Z$9 1001d6e7 f   workstationeditordlgimpl.obj
 0001:0001c6f0       __unwindfunclet$?toXML@@YA?AVQString@@ABV1@@Z$10 1001d6f0 f   workstationeditordlgimpl.obj
 0001:0001c6f9       __ehhandler$?toXML@@YA?AVQString@@ABV1@@Z 1001d6f9 f   workstationeditordlgimpl.obj
 0001:0001c714       __unwindfunclet$??0workstationEditorNewWsDlg@@QAE@ABVQString@@PAVQWidget@@PBD_NI@Z$0 1001d714 f   workstationeditornewwsdlgimpl.obj
 0001:0001c71c       __unwindfunclet$??0workstationEditorNewWsDlg@@QAE@ABVQString@@PAVQWidget@@PBD_NI@Z$1 1001d71c f   workstationeditornewwsdlgimpl.obj
 0001:0001c72b       __unwindfunclet$??0workstationEditorNewWsDlg@@QAE@ABVQString@@PAVQWidget@@PBD_NI@Z$2 1001d72b f   workstationeditornewwsdlgimpl.obj
 0001:0001c73a       __ehhandler$??0workstationEditorNewWsDlg@@QAE@ABVQString@@PAVQWidget@@PBD_NI@Z 1001d73a f   workstationeditornewwsdlgimpl.obj
 0001:0001c755       __unwindfunclet$??1workstationEditorNewWsDlg@@UAE@XZ$0 1001d755 f   workstationeditornewwsdlgimpl.obj
 0001:0001c75d       __unwindfunclet$??1workstationEditorNewWsDlg@@UAE@XZ$1 1001d75d f   workstationeditornewwsdlgimpl.obj
 0001:0001c76c       __ehhandler$??1workstationEditorNewWsDlg@@UAE@XZ 1001d76c f   workstationeditornewwsdlgimpl.obj
 0001:0001c787       __unwindfunclet$?accept@workstationEditorNewWsDlg@@UAEXXZ$0 1001d787 f   workstationeditornewwsdlgimpl.obj
 0001:0001c790       __unwindfunclet$?accept@workstationEditorNewWsDlg@@UAEXXZ$1 1001d790 f   workstationeditornewwsdlgimpl.obj
 0001:0001c799       __unwindfunclet$?accept@workstationEditorNewWsDlg@@UAEXXZ$2 1001d799 f   workstationeditornewwsdlgimpl.obj
 0001:0001c7a2       __unwindfunclet$?accept@workstationEditorNewWsDlg@@UAEXXZ$4 1001d7a2 f   workstationeditornewwsdlgimpl.obj
 0001:0001c7ab       __unwindfunclet$?accept@workstationEditorNewWsDlg@@UAEXXZ$5 1001d7ab f   workstationeditornewwsdlgimpl.obj
 0001:0001c7b4       __ehhandler$?accept@workstationEditorNewWsDlg@@UAEXXZ 1001d7b4 f   workstationeditornewwsdlgimpl.obj
 0001:0001c7cf       __unwindfunclet$?loadUsers@workstationEditorNewWsDlg@@AAEXXZ$0 1001d7cf f   workstationeditornewwsdlgimpl.obj
 0001:0001c7d8       __unwindfunclet$?loadUsers@workstationEditorNewWsDlg@@AAEXXZ$1 1001d7d8 f   workstationeditornewwsdlgimpl.obj
 0001:0001c7e1       __unwindfunclet$?loadUsers@workstationEditorNewWsDlg@@AAEXXZ$2 1001d7e1 f   workstationeditornewwsdlgimpl.obj
 0001:0001c7ea       __unwindfunclet$?loadUsers@workstationEditorNewWsDlg@@AAEXXZ$3 1001d7ea f   workstationeditornewwsdlgimpl.obj
 0001:0001c7f3       __unwindfunclet$?loadUsers@workstationEditorNewWsDlg@@AAEXXZ$4 1001d7f3 f   workstationeditornewwsdlgimpl.obj
 0001:0001c7fc       __unwindfunclet$?loadUsers@workstationEditorNewWsDlg@@AAEXXZ$5 1001d7fc f   workstationeditornewwsdlgimpl.obj
 0001:0001c805       __unwindfunclet$?loadUsers@workstationEditorNewWsDlg@@AAEXXZ$6 1001d805 f   workstationeditornewwsdlgimpl.obj
 0001:0001c80e       __unwindfunclet$?loadUsers@workstationEditorNewWsDlg@@AAEXXZ$7 1001d80e f   workstationeditornewwsdlgimpl.obj
 0001:0001c817       __unwindfunclet$?loadUsers@workstationEditorNewWsDlg@@AAEXXZ$8 1001d817 f   workstationeditornewwsdlgimpl.obj
 0001:0001c820       __unwindfunclet$?loadUsers@workstationEditorNewWsDlg@@AAEXXZ$9 1001d820 f   workstationeditornewwsdlgimpl.obj
 0001:0001c829       __ehhandler$?loadUsers@workstationEditorNewWsDlg@@AAEXXZ 1001d829 f   workstationeditornewwsdlgimpl.obj
 0001:0001c844       __unwindfunclet$??0workstationUserTableItem@@QAE@ABVQString@@PAVQTable@@W4EditType@QTableItem@@0@Z$0 1001d844 f   workstationUserTableItem.obj
 0001:0001c84d       __unwindfunclet$??0workstationUserTableItem@@QAE@ABVQString@@PAVQTable@@W4EditType@QTableItem@@0@Z$1 1001d84d f   workstationUserTableItem.obj
 0001:0001c859       __ehhandler$??0workstationUserTableItem@@QAE@ABVQString@@PAVQTable@@W4EditType@QTableItem@@0@Z 1001d859 f   workstationUserTableItem.obj
 0001:0001c874       __unwindfunclet$??1workstationUserTableItem@@UAE@XZ$0 1001d874 f   workstationUserTableItem.obj
 0001:0001c87d       __ehhandler$??1workstationUserTableItem@@UAE@XZ 1001d87d f   workstationUserTableItem.obj
 0001:0001c898       __unwindfunclet$?createEditor@workstationUserTableItem@@UBEPAVQWidget@@XZ$0 1001d898 f   workstationUserTableItem.obj
 0001:0001c8a2       __unwindfunclet$?createEditor@workstationUserTableItem@@UBEPAVQWidget@@XZ$1 1001d8a2 f   workstationUserTableItem.obj
 0001:0001c8ab       __unwindfunclet$?createEditor@workstationUserTableItem@@UBEPAVQWidget@@XZ$2 1001d8ab f   workstationUserTableItem.obj
 0001:0001c8b4       __unwindfunclet$?createEditor@workstationUserTableItem@@UBEPAVQWidget@@XZ$3 1001d8b4 f   workstationUserTableItem.obj
 0001:0001c8bd       __unwindfunclet$?createEditor@workstationUserTableItem@@UBEPAVQWidget@@XZ$4 1001d8bd f   workstationUserTableItem.obj
 0001:0001c8c6       __unwindfunclet$?createEditor@workstationUserTableItem@@UBEPAVQWidget@@XZ$5 1001d8c6 f   workstationUserTableItem.obj
 0001:0001c8cf       __unwindfunclet$?createEditor@workstationUserTableItem@@UBEPAVQWidget@@XZ$6 1001d8cf f   workstationUserTableItem.obj
 0001:0001c8d8       __unwindfunclet$?createEditor@workstationUserTableItem@@UBEPAVQWidget@@XZ$7 1001d8d8 f   workstationUserTableItem.obj
 0001:0001c8e1       __unwindfunclet$?createEditor@workstationUserTableItem@@UBEPAVQWidget@@XZ$8 1001d8e1 f   workstationUserTableItem.obj
 0001:0001c8ea       __unwindfunclet$?createEditor@workstationUserTableItem@@UBEPAVQWidget@@XZ$9 1001d8ea f   workstationUserTableItem.obj
 0001:0001c8f3       __unwindfunclet$?createEditor@workstationUserTableItem@@UBEPAVQWidget@@XZ$10 1001d8f3 f   workstationUserTableItem.obj
 0001:0001c8fc       __unwindfunclet$?createEditor@workstationUserTableItem@@UBEPAVQWidget@@XZ$11 1001d8fc f   workstationUserTableItem.obj
 0001:0001c905       __unwindfunclet$?createEditor@workstationUserTableItem@@UBEPAVQWidget@@XZ$12 1001d905 f   workstationUserTableItem.obj
 0001:0001c90e       __ehhandler$?createEditor@workstationUserTableItem@@UBEPAVQWidget@@XZ 1001d90e f   workstationUserTableItem.obj
 0001:0001c929       __unwindfunclet$?setContentFromEditor@workstationUserTableItem@@UAEXPAVQWidget@@@Z$0 1001d929 f   workstationUserTableItem.obj
 0001:0001c929       __unwindfunclet$?navigate@testPlugin@@UAEXABVQString@@0@Z$0 1001d929 f   workstationUserTableItem.obj
 0001:0001c932       __ehhandler$?navigate@testPlugin@@UAEXABVQString@@0@Z 1001d932 f   workstationUserTableItem.obj
 0001:0001c932       __ehhandler$?setContentFromEditor@workstationUserTableItem@@UAEXPAVQWidget@@@Z 1001d932 f   workstationUserTableItem.obj
 0001:0001c94d       __unwindfunclet$?createDirectory@xfer@@QAEXAAVQString@@@Z$0 1001d94d f   xfer.obj
 0001:0001c956       __unwindfunclet$?createDirectory@xfer@@QAEXAAVQString@@@Z$1 1001d956 f   xfer.obj
 0001:0001c95f       __unwindfunclet$?createDirectory@xfer@@QAEXAAVQString@@@Z$2 1001d95f f   xfer.obj
 0001:0001c968       __unwindfunclet$?createDirectory@xfer@@QAEXAAVQString@@@Z$3 1001d968 f   xfer.obj
 0001:0001c971       __unwindfunclet$?createDirectory@xfer@@QAEXAAVQString@@@Z$4 1001d971 f   xfer.obj
 0001:0001c97a       __unwindfunclet$?createDirectory@xfer@@QAEXAAVQString@@@Z$5 1001d97a f   xfer.obj
 0001:0001c983       __ehhandler$?createDirectory@xfer@@QAEXAAVQString@@@Z 1001d983 f   xfer.obj
 0001:0001c99e       __unwindfunclet$?setFileDate@xfer@@QAE_NABVQString@@AAVQDateTime@@@Z$0 1001d99e f   xfer.obj
 0001:0001c9a7       __unwindfunclet$?setFileDate@xfer@@QAE_NABVQString@@AAVQDateTime@@@Z$1 1001d9a7 f   xfer.obj
 0001:0001c9b0       __unwindfunclet$?setFileDate@xfer@@QAE_NABVQString@@AAVQDateTime@@@Z$2 1001d9b0 f   xfer.obj
 0001:0001c9b9       __ehhandler$?setFileDate@xfer@@QAE_NABVQString@@AAVQDateTime@@@Z 1001d9b9 f   xfer.obj
 0001:0001c9de       __unwindfunclet$??0xml_listview@@QAE@PAVQWidget@@PBDI@Z$0 1001d9de f   xml_listview.obj
 0001:0001c9e7       __unwindfunclet$??0xml_listview@@QAE@PAVQWidget@@PBDI@Z$1 1001d9e7 f   xml_listview.obj
 0001:0001c9f6       __ehhandler$??0xml_listview@@QAE@PAVQWidget@@PBDI@Z 1001d9f6 f   xml_listview.obj
 0001:0001ca11       __unwindfunclet$?load@xml_listview@@QAEXABVQString@@@Z$0 1001da11 f   xml_listview.obj
 0001:0001ca1a       __unwindfunclet$?load@xml_listview@@QAEXABVQString@@@Z$1 1001da1a f   xml_listview.obj
 0001:0001ca23       __unwindfunclet$?load@xml_listview@@QAEXABVQString@@@Z$2 1001da23 f   xml_listview.obj
 0001:0001ca2f       __unwindfunclet$?load@xml_listview@@QAEXABVQString@@@Z$3 1001da2f f   xml_listview.obj
 0001:0001ca39       __unwindfunclet$?load@xml_listview@@QAEXABVQString@@@Z$4 1001da39 f   xml_listview.obj
 0001:0001ca42       __unwindfunclet$?load@xml_listview@@QAEXABVQString@@@Z$5 1001da42 f   xml_listview.obj
 0001:0001ca4b       __unwindfunclet$?load@xml_listview@@QAEXABVQString@@@Z$6 1001da4b f   xml_listview.obj
 0001:0001ca54       __unwindfunclet$?load@xml_listview@@QAEXABVQString@@@Z$7 1001da54 f   xml_listview.obj
 0001:0001ca5d       __unwindfunclet$?load@xml_listview@@QAEXABVQString@@@Z$8 1001da5d f   xml_listview.obj
 0001:0001ca66       __unwindfunclet$?load@xml_listview@@QAEXABVQString@@@Z$9 1001da66 f   xml_listview.obj
 0001:0001ca6f       __unwindfunclet$?load@xml_listview@@QAEXABVQString@@@Z$10 1001da6f f   xml_listview.obj
 0001:0001ca78       __unwindfunclet$?load@xml_listview@@QAEXABVQString@@@Z$12 1001da78 f   xml_listview.obj
 0001:0001ca81       __unwindfunclet$?load@xml_listview@@QAEXABVQString@@@Z$13 1001da81 f   xml_listview.obj
 0001:0001ca8b       __unwindfunclet$?load@xml_listview@@QAEXABVQString@@@Z$14 1001da8b f   xml_listview.obj
 0001:0001ca94       __unwindfunclet$?load@xml_listview@@QAEXABVQString@@@Z$15 1001da94 f   xml_listview.obj
 0001:0001ca9d       __unwindfunclet$?load@xml_listview@@QAEXABVQString@@@Z$16 1001da9d f   xml_listview.obj
 0001:0001caa6       __unwindfunclet$?load@xml_listview@@QAEXABVQString@@@Z$17 1001daa6 f   xml_listview.obj
 0001:0001caaf       __unwindfunclet$?load@xml_listview@@QAEXABVQString@@@Z$18 1001daaf f   xml_listview.obj
 0001:0001cab8       __unwindfunclet$?load@xml_listview@@QAEXABVQString@@@Z$19 1001dab8 f   xml_listview.obj
 0001:0001cac1       __unwindfunclet$?load@xml_listview@@QAEXABVQString@@@Z$20 1001dac1 f   xml_listview.obj
 0001:0001caca       __unwindfunclet$?load@xml_listview@@QAEXABVQString@@@Z$22 1001daca f   xml_listview.obj
 0001:0001cad3       __unwindfunclet$?load@xml_listview@@QAEXABVQString@@@Z$23 1001dad3 f   xml_listview.obj
 0001:0001cadc       __unwindfunclet$?load@xml_listview@@QAEXABVQString@@@Z$24 1001dadc f   xml_listview.obj
 0001:0001cae5       __unwindfunclet$?load@xml_listview@@QAEXABVQString@@@Z$25 1001dae5 f   xml_listview.obj
 0001:0001caee       __unwindfunclet$?load@xml_listview@@QAEXABVQString@@@Z$44 1001daee f   xml_listview.obj
 0001:0001caf8       __unwindfunclet$?load@xml_listview@@QAEXABVQString@@@Z$45 1001daf8 f   xml_listview.obj
 0001:0001cb01       __unwindfunclet$?load@xml_listview@@QAEXABVQString@@@Z$46 1001db01 f   xml_listview.obj
 0001:0001cb0a       __unwindfunclet$?load@xml_listview@@QAEXABVQString@@@Z$47 1001db0a f   xml_listview.obj
 0001:0001cb13       __unwindfunclet$?load@xml_listview@@QAEXABVQString@@@Z$48 1001db13 f   xml_listview.obj
 0001:0001cb1c       __unwindfunclet$?load@xml_listview@@QAEXABVQString@@@Z$49 1001db1c f   xml_listview.obj
 0001:0001cb25       __unwindfunclet$?load@xml_listview@@QAEXABVQString@@@Z$50 1001db25 f   xml_listview.obj
 0001:0001cb2e       __unwindfunclet$?load@xml_listview@@QAEXABVQString@@@Z$51 1001db2e f   xml_listview.obj
 0001:0001cb37       __unwindfunclet$?load@xml_listview@@QAEXABVQString@@@Z$35 1001db37 f   xml_listview.obj
 0001:0001cb41       __unwindfunclet$?load@xml_listview@@QAEXABVQString@@@Z$36 1001db41 f   xml_listview.obj
 0001:0001cb4a       __unwindfunclet$?load@xml_listview@@QAEXABVQString@@@Z$37 1001db4a f   xml_listview.obj
 0001:0001cb53       __unwindfunclet$?load@xml_listview@@QAEXABVQString@@@Z$38 1001db53 f   xml_listview.obj
 0001:0001cb5c       __unwindfunclet$?load@xml_listview@@QAEXABVQString@@@Z$39 1001db5c f   xml_listview.obj
 0001:0001cb65       __unwindfunclet$?load@xml_listview@@QAEXABVQString@@@Z$40 1001db65 f   xml_listview.obj
 0001:0001cb6e       __unwindfunclet$?load@xml_listview@@QAEXABVQString@@@Z$41 1001db6e f   xml_listview.obj
 0001:0001cb77       __unwindfunclet$?load@xml_listview@@QAEXABVQString@@@Z$42 1001db77 f   xml_listview.obj
 0001:0001cb80       __unwindfunclet$?load@xml_listview@@QAEXABVQString@@@Z$26 1001db80 f   xml_listview.obj
 0001:0001cb8a       __unwindfunclet$?load@xml_listview@@QAEXABVQString@@@Z$27 1001db8a f   xml_listview.obj
 0001:0001cb93       __unwindfunclet$?load@xml_listview@@QAEXABVQString@@@Z$28 1001db93 f   xml_listview.obj
 0001:0001cb9c       __unwindfunclet$?load@xml_listview@@QAEXABVQString@@@Z$29 1001db9c f   xml_listview.obj
 0001:0001cba5       __unwindfunclet$?load@xml_listview@@QAEXABVQString@@@Z$30 1001dba5 f   xml_listview.obj
 0001:0001cbae       __unwindfunclet$?load@xml_listview@@QAEXABVQString@@@Z$31 1001dbae f   xml_listview.obj
 0001:0001cbb7       __unwindfunclet$?load@xml_listview@@QAEXABVQString@@@Z$32 1001dbb7 f   xml_listview.obj
 0001:0001cbc0       __unwindfunclet$?load@xml_listview@@QAEXABVQString@@@Z$33 1001dbc0 f   xml_listview.obj
 0001:0001cbc9       __unwindfunclet$?load@xml_listview@@QAEXABVQString@@@Z$53 1001dbc9 f   xml_listview.obj
 0001:0001cbd3       __unwindfunclet$?load@xml_listview@@QAEXABVQString@@@Z$54 1001dbd3 f   xml_listview.obj
 0001:0001cbdc       __unwindfunclet$?load@xml_listview@@QAEXABVQString@@@Z$55 1001dbdc f   xml_listview.obj
 0001:0001cbe5       __unwindfunclet$?load@xml_listview@@QAEXABVQString@@@Z$56 1001dbe5 f   xml_listview.obj
 0001:0001cbee       __unwindfunclet$?load@xml_listview@@QAEXABVQString@@@Z$57 1001dbee f   xml_listview.obj
 0001:0001cbf7       __unwindfunclet$?load@xml_listview@@QAEXABVQString@@@Z$58 1001dbf7 f   xml_listview.obj
 0001:0001cc00       __unwindfunclet$?load@xml_listview@@QAEXABVQString@@@Z$59 1001dc00 f   xml_listview.obj
 0001:0001cc09       __unwindfunclet$?load@xml_listview@@QAEXABVQString@@@Z$60 1001dc09 f   xml_listview.obj
 0001:0001cc12       __unwindfunclet$?load@xml_listview@@QAEXABVQString@@@Z$80 1001dc12 f   xml_listview.obj
 0001:0001cc1c       __unwindfunclet$?load@xml_listview@@QAEXABVQString@@@Z$81 1001dc1c f   xml_listview.obj
 0001:0001cc25       __unwindfunclet$?load@xml_listview@@QAEXABVQString@@@Z$82 1001dc25 f   xml_listview.obj
 0001:0001cc2e       __unwindfunclet$?load@xml_listview@@QAEXABVQString@@@Z$83 1001dc2e f   xml_listview.obj
 0001:0001cc37       __unwindfunclet$?load@xml_listview@@QAEXABVQString@@@Z$84 1001dc37 f   xml_listview.obj
 0001:0001cc40       __unwindfunclet$?load@xml_listview@@QAEXABVQString@@@Z$85 1001dc40 f   xml_listview.obj
 0001:0001cc49       __unwindfunclet$?load@xml_listview@@QAEXABVQString@@@Z$86 1001dc49 f   xml_listview.obj
 0001:0001cc52       __unwindfunclet$?load@xml_listview@@QAEXABVQString@@@Z$87 1001dc52 f   xml_listview.obj
 0001:0001cc5b       __unwindfunclet$?load@xml_listview@@QAEXABVQString@@@Z$71 1001dc5b f   xml_listview.obj
 0001:0001cc65       __unwindfunclet$?load@xml_listview@@QAEXABVQString@@@Z$72 1001dc65 f   xml_listview.obj
 0001:0001cc6e       __unwindfunclet$?load@xml_listview@@QAEXABVQString@@@Z$73 1001dc6e f   xml_listview.obj
 0001:0001cc77       __unwindfunclet$?load@xml_listview@@QAEXABVQString@@@Z$74 1001dc77 f   xml_listview.obj
 0001:0001cc80       __unwindfunclet$?load@xml_listview@@QAEXABVQString@@@Z$75 1001dc80 f   xml_listview.obj
 0001:0001cc89       __unwindfunclet$?load@xml_listview@@QAEXABVQString@@@Z$76 1001dc89 f   xml_listview.obj
 0001:0001cc92       __unwindfunclet$?load@xml_listview@@QAEXABVQString@@@Z$77 1001dc92 f   xml_listview.obj
 0001:0001cc9b       __unwindfunclet$?load@xml_listview@@QAEXABVQString@@@Z$78 1001dc9b f   xml_listview.obj
 0001:0001cca4       __unwindfunclet$?load@xml_listview@@QAEXABVQString@@@Z$62 1001dca4 f   xml_listview.obj
 0001:0001ccae       __unwindfunclet$?load@xml_listview@@QAEXABVQString@@@Z$63 1001dcae f   xml_listview.obj
 0001:0001ccb7       __unwindfunclet$?load@xml_listview@@QAEXABVQString@@@Z$64 1001dcb7 f   xml_listview.obj
 0001:0001ccc0       __unwindfunclet$?load@xml_listview@@QAEXABVQString@@@Z$65 1001dcc0 f   xml_listview.obj
 0001:0001ccc9       __unwindfunclet$?load@xml_listview@@QAEXABVQString@@@Z$66 1001dcc9 f   xml_listview.obj
 0001:0001ccd2       __unwindfunclet$?load@xml_listview@@QAEXABVQString@@@Z$67 1001dcd2 f   xml_listview.obj
 0001:0001ccdb       __unwindfunclet$?load@xml_listview@@QAEXABVQString@@@Z$68 1001dcdb f   xml_listview.obj
 0001:0001cce4       __unwindfunclet$?load@xml_listview@@QAEXABVQString@@@Z$69 1001dce4 f   xml_listview.obj
 0001:0001cced       __unwindfunclet$?load@xml_listview@@QAEXABVQString@@@Z$89 1001dced f   xml_listview.obj
 0001:0001ccf6       __unwindfunclet$?load@xml_listview@@QAEXABVQString@@@Z$117 1001dcf6 f   xml_listview.obj
 0001:0001cd00       __unwindfunclet$?load@xml_listview@@QAEXABVQString@@@Z$118 1001dd00 f   xml_listview.obj
 0001:0001cd09       __unwindfunclet$?load@xml_listview@@QAEXABVQString@@@Z$119 1001dd09 f   xml_listview.obj
 0001:0001cd12       __unwindfunclet$?load@xml_listview@@QAEXABVQString@@@Z$120 1001dd12 f   xml_listview.obj
 0001:0001cd1b       __unwindfunclet$?load@xml_listview@@QAEXABVQString@@@Z$121 1001dd1b f   xml_listview.obj
 0001:0001cd24       __unwindfunclet$?load@xml_listview@@QAEXABVQString@@@Z$122 1001dd24 f   xml_listview.obj
 0001:0001cd2d       __unwindfunclet$?load@xml_listview@@QAEXABVQString@@@Z$123 1001dd2d f   xml_listview.obj
 0001:0001cd36       __unwindfunclet$?load@xml_listview@@QAEXABVQString@@@Z$124 1001dd36 f   xml_listview.obj
 0001:0001cd3f       __unwindfunclet$?load@xml_listview@@QAEXABVQString@@@Z$108 1001dd3f f   xml_listview.obj
 0001:0001cd49       __unwindfunclet$?load@xml_listview@@QAEXABVQString@@@Z$109 1001dd49 f   xml_listview.obj
 0001:0001cd52       __unwindfunclet$?load@xml_listview@@QAEXABVQString@@@Z$110 1001dd52 f   xml_listview.obj
 0001:0001cd5b       __unwindfunclet$?load@xml_listview@@QAEXABVQString@@@Z$111 1001dd5b f   xml_listview.obj
 0001:0001cd64       __unwindfunclet$?load@xml_listview@@QAEXABVQString@@@Z$112 1001dd64 f   xml_listview.obj
 0001:0001cd6d       __unwindfunclet$?load@xml_listview@@QAEXABVQString@@@Z$113 1001dd6d f   xml_listview.obj
 0001:0001cd76       __unwindfunclet$?load@xml_listview@@QAEXABVQString@@@Z$114 1001dd76 f   xml_listview.obj
 0001:0001cd7f       __unwindfunclet$?load@xml_listview@@QAEXABVQString@@@Z$115 1001dd7f f   xml_listview.obj
 0001:0001cd88       __unwindfunclet$?load@xml_listview@@QAEXABVQString@@@Z$99 1001dd88 f   xml_listview.obj
 0001:0001cd92       __unwindfunclet$?load@xml_listview@@QAEXABVQString@@@Z$100 1001dd92 f   xml_listview.obj
 0001:0001cd9b       __unwindfunclet$?load@xml_listview@@QAEXABVQString@@@Z$101 1001dd9b f   xml_listview.obj
 0001:0001cda4       __unwindfunclet$?load@xml_listview@@QAEXABVQString@@@Z$102 1001dda4 f   xml_listview.obj
 0001:0001cdad       __unwindfunclet$?load@xml_listview@@QAEXABVQString@@@Z$103 1001ddad f   xml_listview.obj
 0001:0001cdb6       __unwindfunclet$?load@xml_listview@@QAEXABVQString@@@Z$104 1001ddb6 f   xml_listview.obj
 0001:0001cdbf       __unwindfunclet$?load@xml_listview@@QAEXABVQString@@@Z$105 1001ddbf f   xml_listview.obj
 0001:0001cdc8       __unwindfunclet$?load@xml_listview@@QAEXABVQString@@@Z$106 1001ddc8 f   xml_listview.obj
 0001:0001cdd1       __unwindfunclet$?load@xml_listview@@QAEXABVQString@@@Z$90 1001ddd1 f   xml_listview.obj
 0001:0001cddb       __unwindfunclet$?load@xml_listview@@QAEXABVQString@@@Z$91 1001dddb f   xml_listview.obj
 0001:0001cde4       __unwindfunclet$?load@xml_listview@@QAEXABVQString@@@Z$92 1001dde4 f   xml_listview.obj
 0001:0001cded       __unwindfunclet$?load@xml_listview@@QAEXABVQString@@@Z$93 1001dded f   xml_listview.obj
 0001:0001cdf6       __unwindfunclet$?load@xml_listview@@QAEXABVQString@@@Z$94 1001ddf6 f   xml_listview.obj
 0001:0001cdff       __unwindfunclet$?load@xml_listview@@QAEXABVQString@@@Z$95 1001ddff f   xml_listview.obj
 0001:0001ce08       __unwindfunclet$?load@xml_listview@@QAEXABVQString@@@Z$96 1001de08 f   xml_listview.obj
 0001:0001ce11       __unwindfunclet$?load@xml_listview@@QAEXABVQString@@@Z$97 1001de11 f   xml_listview.obj
 0001:0001ce1a       __unwindfunclet$?load@xml_listview@@QAEXABVQString@@@Z$126 1001de1a f   xml_listview.obj
 0001:0001ce23       __ehhandler$?load@xml_listview@@QAEXABVQString@@@Z 1001de23 f   xml_listview.obj
 0001:0001ce41       __unwindfunclet$??0dialogBase@@QAE@PAVQWidget@@PBDI@Z$0 1001de41 f   dialog.obj
 0001:0001ce4a       __unwindfunclet$??0dialogBase@@QAE@PAVQWidget@@PBDI@Z$1 1001de4a f   dialog.obj
 0001:0001ce54       __unwindfunclet$??0dialogBase@@QAE@PAVQWidget@@PBDI@Z$2 1001de54 f   dialog.obj
 0001:0001ce5e       __unwindfunclet$??0dialogBase@@QAE@PAVQWidget@@PBDI@Z$3 1001de5e f   dialog.obj
 0001:0001ce68       __unwindfunclet$??0dialogBase@@QAE@PAVQWidget@@PBDI@Z$4 1001de68 f   dialog.obj
 0001:0001ce72       __unwindfunclet$??0dialogBase@@QAE@PAVQWidget@@PBDI@Z$5 1001de72 f   dialog.obj
 0001:0001ce7c       __unwindfunclet$??0dialogBase@@QAE@PAVQWidget@@PBDI@Z$6 1001de7c f   dialog.obj
 0001:0001ce86       __unwindfunclet$??0dialogBase@@QAE@PAVQWidget@@PBDI@Z$7 1001de86 f   dialog.obj
 0001:0001ce90       __unwindfunclet$??0dialogBase@@QAE@PAVQWidget@@PBDI@Z$8 1001de90 f   dialog.obj
 0001:0001ce9a       __unwindfunclet$??0dialogBase@@QAE@PAVQWidget@@PBDI@Z$9 1001de9a f   dialog.obj
 0001:0001cea4       __unwindfunclet$??0dialogBase@@QAE@PAVQWidget@@PBDI@Z$10 1001dea4 f   dialog.obj
 0001:0001ceae       __unwindfunclet$??0dialogBase@@QAE@PAVQWidget@@PBDI@Z$11 1001deae f   dialog.obj
 0001:0001ceb8       __unwindfunclet$??0dialogBase@@QAE@PAVQWidget@@PBDI@Z$12 1001deb8 f   dialog.obj
 0001:0001cec2       __unwindfunclet$??0dialogBase@@QAE@PAVQWidget@@PBDI@Z$13 1001dec2 f   dialog.obj
 0001:0001cecc       __unwindfunclet$??0dialogBase@@QAE@PAVQWidget@@PBDI@Z$14 1001decc f   dialog.obj
 0001:0001ced6       __unwindfunclet$??0dialogBase@@QAE@PAVQWidget@@PBDI@Z$15 1001ded6 f   dialog.obj
 0001:0001cee0       __unwindfunclet$??0dialogBase@@QAE@PAVQWidget@@PBDI@Z$16 1001dee0 f   dialog.obj
 0001:0001ceea       __unwindfunclet$??0dialogBase@@QAE@PAVQWidget@@PBDI@Z$17 1001deea f   dialog.obj
 0001:0001cef4       __unwindfunclet$??0dialogBase@@QAE@PAVQWidget@@PBDI@Z$18 1001def4 f   dialog.obj
 0001:0001cefe       __unwindfunclet$??0dialogBase@@QAE@PAVQWidget@@PBDI@Z$19 1001defe f   dialog.obj
 0001:0001cf08       __unwindfunclet$??0dialogBase@@QAE@PAVQWidget@@PBDI@Z$20 1001df08 f   dialog.obj
 0001:0001cf12       __unwindfunclet$??0dialogBase@@QAE@PAVQWidget@@PBDI@Z$21 1001df12 f   dialog.obj
 0001:0001cf1c       __unwindfunclet$??0dialogBase@@QAE@PAVQWidget@@PBDI@Z$22 1001df1c f   dialog.obj
 0001:0001cf26       __unwindfunclet$??0dialogBase@@QAE@PAVQWidget@@PBDI@Z$23 1001df26 f   dialog.obj
 0001:0001cf30       __unwindfunclet$??0dialogBase@@QAE@PAVQWidget@@PBDI@Z$24 1001df30 f   dialog.obj
 0001:0001cf3a       __unwindfunclet$??0dialogBase@@QAE@PAVQWidget@@PBDI@Z$25 1001df3a f   dialog.obj
 0001:0001cf44       __unwindfunclet$??0dialogBase@@QAE@PAVQWidget@@PBDI@Z$26 1001df44 f   dialog.obj
 0001:0001cf4e       __unwindfunclet$??0dialogBase@@QAE@PAVQWidget@@PBDI@Z$27 1001df4e f   dialog.obj
 0001:0001cf58       __unwindfunclet$??0dialogBase@@QAE@PAVQWidget@@PBDI@Z$28 1001df58 f   dialog.obj
 0001:0001cf62       __unwindfunclet$??0dialogBase@@QAE@PAVQWidget@@PBDI@Z$29 1001df62 f   dialog.obj
 0001:0001cf6c       __unwindfunclet$??0dialogBase@@QAE@PAVQWidget@@PBDI@Z$30 1001df6c f   dialog.obj
 0001:0001cf76       __unwindfunclet$??0dialogBase@@QAE@PAVQWidget@@PBDI@Z$31 1001df76 f   dialog.obj
 0001:0001cf80       __unwindfunclet$??0dialogBase@@QAE@PAVQWidget@@PBDI@Z$32 1001df80 f   dialog.obj
 0001:0001cf8a       __unwindfunclet$??0dialogBase@@QAE@PAVQWidget@@PBDI@Z$33 1001df8a f   dialog.obj
 0001:0001cf94       __unwindfunclet$??0dialogBase@@QAE@PAVQWidget@@PBDI@Z$34 1001df94 f   dialog.obj
 0001:0001cf9e       __unwindfunclet$??0dialogBase@@QAE@PAVQWidget@@PBDI@Z$35 1001df9e f   dialog.obj
 0001:0001cfa8       __unwindfunclet$??0dialogBase@@QAE@PAVQWidget@@PBDI@Z$36 1001dfa8 f   dialog.obj
 0001:0001cfb2       __unwindfunclet$??0dialogBase@@QAE@PAVQWidget@@PBDI@Z$37 1001dfb2 f   dialog.obj
 0001:0001cfbc       __unwindfunclet$??0dialogBase@@QAE@PAVQWidget@@PBDI@Z$38 1001dfbc f   dialog.obj
 0001:0001cfc6       __unwindfunclet$??0dialogBase@@QAE@PAVQWidget@@PBDI@Z$39 1001dfc6 f   dialog.obj
 0001:0001cfd0       __unwindfunclet$??0dialogBase@@QAE@PAVQWidget@@PBDI@Z$40 1001dfd0 f   dialog.obj
 0001:0001cfda       __unwindfunclet$??0dialogBase@@QAE@PAVQWidget@@PBDI@Z$41 1001dfda f   dialog.obj
 0001:0001cfe4       __unwindfunclet$??0dialogBase@@QAE@PAVQWidget@@PBDI@Z$42 1001dfe4 f   dialog.obj
 0001:0001cfee       __unwindfunclet$??0dialogBase@@QAE@PAVQWidget@@PBDI@Z$43 1001dfee f   dialog.obj
 0001:0001cff8       __unwindfunclet$??0dialogBase@@QAE@PAVQWidget@@PBDI@Z$44 1001dff8 f   dialog.obj
 0001:0001d002       __unwindfunclet$??0dialogBase@@QAE@PAVQWidget@@PBDI@Z$45 1001e002 f   dialog.obj
 0001:0001d00c       __unwindfunclet$??0dialogBase@@QAE@PAVQWidget@@PBDI@Z$46 1001e00c f   dialog.obj
 0001:0001d016       __unwindfunclet$??0dialogBase@@QAE@PAVQWidget@@PBDI@Z$47 1001e016 f   dialog.obj
 0001:0001d020       __unwindfunclet$??0dialogBase@@QAE@PAVQWidget@@PBDI@Z$48 1001e020 f   dialog.obj
 0001:0001d02a       __unwindfunclet$??0dialogBase@@QAE@PAVQWidget@@PBDI@Z$49 1001e02a f   dialog.obj
 0001:0001d034       __unwindfunclet$??0dialogBase@@QAE@PAVQWidget@@PBDI@Z$50 1001e034 f   dialog.obj
 0001:0001d03e       __unwindfunclet$??0dialogBase@@QAE@PAVQWidget@@PBDI@Z$51 1001e03e f   dialog.obj
 0001:0001d048       __unwindfunclet$??0dialogBase@@QAE@PAVQWidget@@PBDI@Z$52 1001e048 f   dialog.obj
 0001:0001d052       __ehhandler$??0dialogBase@@QAE@PAVQWidget@@PBDI@Z 1001e052 f   dialog.obj
 0001:0001d06d       __unwindfunclet$?languageChange@dialogBase@@MAEXXZ$0 1001e06d f   dialog.obj
 0001:0001d076       __unwindfunclet$?languageChange@dialogBase@@MAEXXZ$1 1001e076 f   dialog.obj
 0001:0001d07f       __unwindfunclet$?languageChange@dialogBase@@MAEXXZ$2 1001e07f f   dialog.obj
 0001:0001d088       __unwindfunclet$?languageChange@dialogBase@@MAEXXZ$3 1001e088 f   dialog.obj
 0001:0001d091       __unwindfunclet$?languageChange@dialogBase@@MAEXXZ$4 1001e091 f   dialog.obj
 0001:0001d09a       __unwindfunclet$?languageChange@dialogBase@@MAEXXZ$5 1001e09a f   dialog.obj
 0001:0001d0a3       __unwindfunclet$?languageChange@dialogBase@@MAEXXZ$6 1001e0a3 f   dialog.obj
 0001:0001d0ac       __unwindfunclet$?languageChange@dialogBase@@MAEXXZ$7 1001e0ac f   dialog.obj
 0001:0001d0b5       __unwindfunclet$?languageChange@dialogBase@@MAEXXZ$8 1001e0b5 f   dialog.obj
 0001:0001d0be       __unwindfunclet$?languageChange@dialogBase@@MAEXXZ$9 1001e0be f   dialog.obj
 0001:0001d0c7       __unwindfunclet$?languageChange@dialogBase@@MAEXXZ$10 1001e0c7 f   dialog.obj
 0001:0001d0d0       __unwindfunclet$?languageChange@dialogBase@@MAEXXZ$11 1001e0d0 f   dialog.obj
 0001:0001d0d9       __unwindfunclet$?languageChange@dialogBase@@MAEXXZ$12 1001e0d9 f   dialog.obj
 0001:0001d0e2       __unwindfunclet$?languageChange@dialogBase@@MAEXXZ$13 1001e0e2 f   dialog.obj
 0001:0001d0eb       __unwindfunclet$?languageChange@dialogBase@@MAEXXZ$14 1001e0eb f   dialog.obj
 0001:0001d0f4       __unwindfunclet$?languageChange@dialogBase@@MAEXXZ$15 1001e0f4 f   dialog.obj
 0001:0001d0fd       __unwindfunclet$?languageChange@dialogBase@@MAEXXZ$16 1001e0fd f   dialog.obj
 0001:0001d106       __unwindfunclet$?languageChange@dialogBase@@MAEXXZ$17 1001e106 f   dialog.obj
 0001:0001d10f       __unwindfunclet$?languageChange@dialogBase@@MAEXXZ$18 1001e10f f   dialog.obj
 0001:0001d118       __unwindfunclet$?languageChange@dialogBase@@MAEXXZ$19 1001e118 f   dialog.obj
 0001:0001d121       __unwindfunclet$?languageChange@dialogBase@@MAEXXZ$20 1001e121 f   dialog.obj
 0001:0001d12a       __unwindfunclet$?languageChange@dialogBase@@MAEXXZ$21 1001e12a f   dialog.obj
 0001:0001d133       __unwindfunclet$?languageChange@dialogBase@@MAEXXZ$22 1001e133 f   dialog.obj
 0001:0001d13c       __ehhandler$?languageChange@dialogBase@@MAEXXZ 1001e13c f   dialog.obj
 0001:0001d157       __unwindfunclet$??0launchEditorDlgBase@@QAE@PAVQWidget@@PBDI@Z$0 1001e157 f   launcheditordlg.obj
 0001:0001d160       __unwindfunclet$??0launchEditorDlgBase@@QAE@PAVQWidget@@PBDI@Z$1 1001e160 f   launcheditordlg.obj
 0001:0001d16f       __unwindfunclet$??0launchEditorDlgBase@@QAE@PAVQWidget@@PBDI@Z$2 1001e16f f   launcheditordlg.obj
 0001:0001d179       __unwindfunclet$??0launchEditorDlgBase@@QAE@PAVQWidget@@PBDI@Z$3 1001e179 f   launcheditordlg.obj
 0001:0001d183       __unwindfunclet$??0launchEditorDlgBase@@QAE@PAVQWidget@@PBDI@Z$4 1001e183 f   launcheditordlg.obj
 0001:0001d18d       __unwindfunclet$??0launchEditorDlgBase@@QAE@PAVQWidget@@PBDI@Z$5 1001e18d f   launcheditordlg.obj
 0001:0001d197       __unwindfunclet$??0launchEditorDlgBase@@QAE@PAVQWidget@@PBDI@Z$6 1001e197 f   launcheditordlg.obj
 0001:0001d1a1       __unwindfunclet$??0launchEditorDlgBase@@QAE@PAVQWidget@@PBDI@Z$7 1001e1a1 f   launcheditordlg.obj
 0001:0001d1ab       __unwindfunclet$??0launchEditorDlgBase@@QAE@PAVQWidget@@PBDI@Z$8 1001e1ab f   launcheditordlg.obj
 0001:0001d1b5       __unwindfunclet$??0launchEditorDlgBase@@QAE@PAVQWidget@@PBDI@Z$9 1001e1b5 f   launcheditordlg.obj
 0001:0001d1bf       __unwindfunclet$??0launchEditorDlgBase@@QAE@PAVQWidget@@PBDI@Z$10 1001e1bf f   launcheditordlg.obj
 0001:0001d1c8       __unwindfunclet$??0launchEditorDlgBase@@QAE@PAVQWidget@@PBDI@Z$11 1001e1c8 f   launcheditordlg.obj
 0001:0001d1d2       __unwindfunclet$??0launchEditorDlgBase@@QAE@PAVQWidget@@PBDI@Z$12 1001e1d2 f   launcheditordlg.obj
 0001:0001d1dc       __unwindfunclet$??0launchEditorDlgBase@@QAE@PAVQWidget@@PBDI@Z$13 1001e1dc f   launcheditordlg.obj
 0001:0001d1e5       __unwindfunclet$??0launchEditorDlgBase@@QAE@PAVQWidget@@PBDI@Z$14 1001e1e5 f   launcheditordlg.obj
 0001:0001d1ef       __unwindfunclet$??0launchEditorDlgBase@@QAE@PAVQWidget@@PBDI@Z$15 1001e1ef f   launcheditordlg.obj
 0001:0001d1f9       __unwindfunclet$??0launchEditorDlgBase@@QAE@PAVQWidget@@PBDI@Z$16 1001e1f9 f   launcheditordlg.obj
 0001:0001d203       __unwindfunclet$??0launchEditorDlgBase@@QAE@PAVQWidget@@PBDI@Z$17 1001e203 f   launcheditordlg.obj
 0001:0001d20d       __unwindfunclet$??0launchEditorDlgBase@@QAE@PAVQWidget@@PBDI@Z$18 1001e20d f   launcheditordlg.obj
 0001:0001d217       __unwindfunclet$??0launchEditorDlgBase@@QAE@PAVQWidget@@PBDI@Z$19 1001e217 f   launcheditordlg.obj
 0001:0001d221       __unwindfunclet$??0launchEditorDlgBase@@QAE@PAVQWidget@@PBDI@Z$20 1001e221 f   launcheditordlg.obj
 0001:0001d22b       __unwindfunclet$??0launchEditorDlgBase@@QAE@PAVQWidget@@PBDI@Z$21 1001e22b f   launcheditordlg.obj
 0001:0001d235       __unwindfunclet$??0launchEditorDlgBase@@QAE@PAVQWidget@@PBDI@Z$22 1001e235 f   launcheditordlg.obj
 0001:0001d23f       __unwindfunclet$??0launchEditorDlgBase@@QAE@PAVQWidget@@PBDI@Z$23 1001e23f f   launcheditordlg.obj
 0001:0001d249       __unwindfunclet$??0launchEditorDlgBase@@QAE@PAVQWidget@@PBDI@Z$24 1001e249 f   launcheditordlg.obj
 0001:0001d253       __unwindfunclet$??0launchEditorDlgBase@@QAE@PAVQWidget@@PBDI@Z$25 1001e253 f   launcheditordlg.obj
 0001:0001d25d       __unwindfunclet$??0launchEditorDlgBase@@QAE@PAVQWidget@@PBDI@Z$26 1001e25d f   launcheditordlg.obj
 0001:0001d267       __unwindfunclet$??0launchEditorDlgBase@@QAE@PAVQWidget@@PBDI@Z$27 1001e267 f   launcheditordlg.obj
 0001:0001d271       __unwindfunclet$??0launchEditorDlgBase@@QAE@PAVQWidget@@PBDI@Z$28 1001e271 f   launcheditordlg.obj
 0001:0001d27b       __unwindfunclet$??0launchEditorDlgBase@@QAE@PAVQWidget@@PBDI@Z$29 1001e27b f   launcheditordlg.obj
 0001:0001d285       __unwindfunclet$??0launchEditorDlgBase@@QAE@PAVQWidget@@PBDI@Z$30 1001e285 f   launcheditordlg.obj
 0001:0001d28f       __unwindfunclet$??0launchEditorDlgBase@@QAE@PAVQWidget@@PBDI@Z$31 1001e28f f   launcheditordlg.obj
 0001:0001d299       __unwindfunclet$??0launchEditorDlgBase@@QAE@PAVQWidget@@PBDI@Z$32 1001e299 f   launcheditordlg.obj
 0001:0001d2a3       __ehhandler$??0launchEditorDlgBase@@QAE@PAVQWidget@@PBDI@Z 1001e2a3 f   launcheditordlg.obj
 0001:0001d2be       __unwindfunclet$?languageChange@launchEditorDlgBase@@MAEXXZ$0 1001e2be f   launcheditordlg.obj
 0001:0001d2c7       __unwindfunclet$?languageChange@launchEditorDlgBase@@MAEXXZ$1 1001e2c7 f   launcheditordlg.obj
 0001:0001d2d0       __unwindfunclet$?languageChange@launchEditorDlgBase@@MAEXXZ$2 1001e2d0 f   launcheditordlg.obj
 0001:0001d2d9       __unwindfunclet$?languageChange@launchEditorDlgBase@@MAEXXZ$3 1001e2d9 f   launcheditordlg.obj
 0001:0001d2e2       __unwindfunclet$?languageChange@launchEditorDlgBase@@MAEXXZ$4 1001e2e2 f   launcheditordlg.obj
 0001:0001d2eb       __unwindfunclet$?languageChange@launchEditorDlgBase@@MAEXXZ$5 1001e2eb f   launcheditordlg.obj
 0001:0001d2f4       __unwindfunclet$?languageChange@launchEditorDlgBase@@MAEXXZ$6 1001e2f4 f   launcheditordlg.obj
 0001:0001d2fd       __unwindfunclet$?languageChange@launchEditorDlgBase@@MAEXXZ$7 1001e2fd f   launcheditordlg.obj
 0001:0001d306       __unwindfunclet$?languageChange@launchEditorDlgBase@@MAEXXZ$8 1001e306 f   launcheditordlg.obj
 0001:0001d30f       __unwindfunclet$?languageChange@launchEditorDlgBase@@MAEXXZ$9 1001e30f f   launcheditordlg.obj
 0001:0001d318       __unwindfunclet$?languageChange@launchEditorDlgBase@@MAEXXZ$10 1001e318 f   launcheditordlg.obj
 0001:0001d321       __unwindfunclet$?languageChange@launchEditorDlgBase@@MAEXXZ$11 1001e321 f   launcheditordlg.obj
 0001:0001d32a       __unwindfunclet$?languageChange@launchEditorDlgBase@@MAEXXZ$12 1001e32a f   launcheditordlg.obj
 0001:0001d333       __unwindfunclet$?languageChange@launchEditorDlgBase@@MAEXXZ$13 1001e333 f   launcheditordlg.obj
 0001:0001d33c       __unwindfunclet$?languageChange@launchEditorDlgBase@@MAEXXZ$14 1001e33c f   launcheditordlg.obj
 0001:0001d345       __unwindfunclet$?languageChange@launchEditorDlgBase@@MAEXXZ$15 1001e345 f   launcheditordlg.obj
 0001:0001d34e       __unwindfunclet$?languageChange@launchEditorDlgBase@@MAEXXZ$16 1001e34e f   launcheditordlg.obj
 0001:0001d357       __unwindfunclet$?languageChange@launchEditorDlgBase@@MAEXXZ$17 1001e357 f   launcheditordlg.obj
 0001:0001d360       __unwindfunclet$?languageChange@launchEditorDlgBase@@MAEXXZ$18 1001e360 f   launcheditordlg.obj
 0001:0001d369       __unwindfunclet$?languageChange@launchEditorDlgBase@@MAEXXZ$19 1001e369 f   launcheditordlg.obj
 0001:0001d372       __unwindfunclet$?languageChange@launchEditorDlgBase@@MAEXXZ$20 1001e372 f   launcheditordlg.obj
 0001:0001d37b       __unwindfunclet$?languageChange@launchEditorDlgBase@@MAEXXZ$21 1001e37b f   launcheditordlg.obj
 0001:0001d384       __unwindfunclet$?languageChange@launchEditorDlgBase@@MAEXXZ$22 1001e384 f   launcheditordlg.obj
 0001:0001d38d       __unwindfunclet$?languageChange@launchEditorDlgBase@@MAEXXZ$23 1001e38d f   launcheditordlg.obj
 0001:0001d396       __unwindfunclet$?languageChange@launchEditorDlgBase@@MAEXXZ$24 1001e396 f   launcheditordlg.obj
 0001:0001d39f       __unwindfunclet$?languageChange@launchEditorDlgBase@@MAEXXZ$25 1001e39f f   launcheditordlg.obj
 0001:0001d3a8       __unwindfunclet$?languageChange@launchEditorDlgBase@@MAEXXZ$26 1001e3a8 f   launcheditordlg.obj
 0001:0001d3b1       __unwindfunclet$?languageChange@launchEditorDlgBase@@MAEXXZ$27 1001e3b1 f   launcheditordlg.obj
 0001:0001d3ba       __unwindfunclet$?languageChange@launchEditorDlgBase@@MAEXXZ$28 1001e3ba f   launcheditordlg.obj
 0001:0001d3c3       __unwindfunclet$?languageChange@launchEditorDlgBase@@MAEXXZ$29 1001e3c3 f   launcheditordlg.obj
 0001:0001d3cc       __unwindfunclet$?languageChange@launchEditorDlgBase@@MAEXXZ$30 1001e3cc f   launcheditordlg.obj
 0001:0001d3d5       __unwindfunclet$?languageChange@launchEditorDlgBase@@MAEXXZ$31 1001e3d5 f   launcheditordlg.obj
 0001:0001d3de       __unwindfunclet$?languageChange@launchEditorDlgBase@@MAEXXZ$32 1001e3de f   launcheditordlg.obj
 0001:0001d3e7       __unwindfunclet$?languageChange@launchEditorDlgBase@@MAEXXZ$33 1001e3e7 f   launcheditordlg.obj
 0001:0001d3f0       __unwindfunclet$?languageChange@launchEditorDlgBase@@MAEXXZ$34 1001e3f0 f   launcheditordlg.obj
 0001:0001d3f9       __unwindfunclet$?languageChange@launchEditorDlgBase@@MAEXXZ$35 1001e3f9 f   launcheditordlg.obj
 0001:0001d402       __unwindfunclet$?languageChange@launchEditorDlgBase@@MAEXXZ$36 1001e402 f   launcheditordlg.obj
 0001:0001d40b       __unwindfunclet$?languageChange@launchEditorDlgBase@@MAEXXZ$37 1001e40b f   launcheditordlg.obj
 0001:0001d414       __unwindfunclet$?languageChange@launchEditorDlgBase@@MAEXXZ$38 1001e414 f   launcheditordlg.obj
 0001:0001d41d       __ehhandler$?languageChange@launchEditorDlgBase@@MAEXXZ 1001e41d f   launcheditordlg.obj
 0001:0001d438       __unwindfunclet$?fileList@fileDrop@@IAEXVQStringList@@@Z$0 1001e438 f   moc_fileDrop.obj
 0001:0001d441       __unwindfunclet$?fileList@fileDrop@@IAEXVQStringList@@@Z$1 1001e441 f   moc_fileDrop.obj
 0001:0001d455       __ehhandler$?fileList@fileDrop@@IAEXVQStringList@@@Z 1001e455 f   moc_fileDrop.obj
 0001:0001d47a       __unwindfunclet$?command@testPlugin@@IAEXVQString@@0@Z$0 1001e47a f   moc_launcheditordlgimpl.obj
 0001:0001d47a       __unwindfunclet$?command@workstationEditor@@IAEXVQString@@0@Z$0 1001e47a f   moc_launcheditordlgimpl.obj
 0001:0001d47a       __unwindfunclet$?command@fileManager@@IAEXVQString@@0@Z$0 1001e47a f   moc_launcheditordlgimpl.obj
 0001:0001d47a       __unwindfunclet$?command@launchEditor@@IAEXVQString@@0@Z$0 1001e47a f   moc_launcheditordlgimpl.obj
 0001:0001d47a       __unwindfunclet$?command@launchEditorDlg@@IAEXVQString@@0@Z$0 1001e47a f   moc_launcheditordlgimpl.obj
 0001:0001d47a       __unwindfunclet$?command@workstationEditorDlg@@IAEXVQString@@0@Z$0 1001e47a f   moc_launcheditordlgimpl.obj
 0001:0001d483       __unwindfunclet$?command@workstationEditorDlg@@IAEXVQString@@0@Z$1 1001e483 f   moc_launcheditordlgimpl.obj
 0001:0001d483       __unwindfunclet$?command@fileManager@@IAEXVQString@@0@Z$1 1001e483 f   moc_launcheditordlgimpl.obj
 0001:0001d483       __unwindfunclet$?command@launchEditor@@IAEXVQString@@0@Z$1 1001e483 f   moc_launcheditordlgimpl.obj
 0001:0001d483       __unwindfunclet$?command@workstationEditor@@IAEXVQString@@0@Z$1 1001e483 f   moc_launcheditordlgimpl.obj
 0001:0001d483       __unwindfunclet$?command@testPlugin@@IAEXVQString@@0@Z$1 1001e483 f   moc_launcheditordlgimpl.obj
 0001:0001d483       __unwindfunclet$?command@launchEditorDlg@@IAEXVQString@@0@Z$1 1001e483 f   moc_launcheditordlgimpl.obj
 0001:0001d48c       __unwindfunclet$?command@launchEditor@@IAEXVQString@@0@Z$2 1001e48c f   moc_launcheditordlgimpl.obj
 0001:0001d48c       __unwindfunclet$?command@testPlugin@@IAEXVQString@@0@Z$2 1001e48c f   moc_launcheditordlgimpl.obj
 0001:0001d48c       __unwindfunclet$?command@workstationEditorDlg@@IAEXVQString@@0@Z$2 1001e48c f   moc_launcheditordlgimpl.obj
 0001:0001d48c       __unwindfunclet$?command@launchEditorDlg@@IAEXVQString@@0@Z$2 1001e48c f   moc_launcheditordlgimpl.obj
 0001:0001d48c       __unwindfunclet$?command@fileManager@@IAEXVQString@@0@Z$2 1001e48c f   moc_launcheditordlgimpl.obj
 0001:0001d48c       __unwindfunclet$?command@workstationEditor@@IAEXVQString@@0@Z$2 1001e48c f   moc_launcheditordlgimpl.obj
 0001:0001d4a0       __ehhandler$?command@fileManager@@IAEXVQString@@0@Z 1001e4a0 f   moc_launcheditordlgimpl.obj
 0001:0001d4a0       __ehhandler$?command@workstationEditorDlg@@IAEXVQString@@0@Z 1001e4a0 f   moc_launcheditordlgimpl.obj
 0001:0001d4a0       __ehhandler$?command@launchEditor@@IAEXVQString@@0@Z 1001e4a0 f   moc_launcheditordlgimpl.obj
 0001:0001d4a0       __ehhandler$?command@workstationEditor@@IAEXVQString@@0@Z 1001e4a0 f   moc_launcheditordlgimpl.obj
 0001:0001d4a0       __ehhandler$?command@launchEditorDlg@@IAEXVQString@@0@Z 1001e4a0 f   moc_launcheditordlgimpl.obj
 0001:0001d4a0       __ehhandler$?command@testPlugin@@IAEXVQString@@0@Z 1001e4a0 f   moc_launcheditordlgimpl.obj
 0001:0001d4c5       __unwindfunclet$?startDrag@xml_listview@@IAEXPAVQListViewItem@@@Z$0 1001e4c5 f   moc_workstationdockwindowimpl.obj
 0001:0001d4c5       __unwindfunclet$?selectionChanged@workstationDockWindow@@IAEXPAVQListViewItem@@@Z$0 1001e4c5 f   moc_workstationdockwindowimpl.obj
 0001:0001d4d9       __ehhandler$?startDrag@xml_listview@@IAEXPAVQListViewItem@@@Z 1001e4d9 f   moc_workstationdockwindowimpl.obj
 0001:0001d4d9       __ehhandler$?selectionChanged@workstationDockWindow@@IAEXPAVQListViewItem@@@Z 1001e4d9 f   moc_workstationdockwindowimpl.obj
 0001:0001d4fe       __unwindfunclet$?qt_emit@workstationEditorDlg@@UAE_NHPAUQUObject@@@Z$0 1001e4fe f   moc_workstationeditordlgimpl.obj
 0001:0001d4fe       __unwindfunclet$?qt_emit@launchEditorDlg@@UAE_NHPAUQUObject@@@Z$0 1001e4fe f   moc_workstationeditordlgimpl.obj
 0001:0001d4fe       __unwindfunclet$?qt_emit@fileManager@@UAE_NHPAUQUObject@@@Z$0 1001e4fe f   moc_workstationeditordlgimpl.obj
 0001:0001d4fe       __unwindfunclet$?qt_emit@launchEditor@@UAE_NHPAUQUObject@@@Z$0 1001e4fe f   moc_workstationeditordlgimpl.obj
 0001:0001d4fe       __unwindfunclet$?qt_emit@testPlugin@@UAE_NHPAUQUObject@@@Z$0 1001e4fe f   moc_workstationeditordlgimpl.obj
 0001:0001d4fe       __unwindfunclet$?qt_emit@workstationEditor@@UAE_NHPAUQUObject@@@Z$0 1001e4fe f   moc_workstationeditordlgimpl.obj
 0001:0001d507       __ehhandler$?qt_emit@launchEditor@@UAE_NHPAUQUObject@@@Z 1001e507 f   moc_workstationeditordlgimpl.obj
 0001:0001d507       __ehhandler$?qt_emit@launchEditorDlg@@UAE_NHPAUQUObject@@@Z 1001e507 f   moc_workstationeditordlgimpl.obj
 0001:0001d507       __ehhandler$?qt_emit@testPlugin@@UAE_NHPAUQUObject@@@Z 1001e507 f   moc_workstationeditordlgimpl.obj
 0001:0001d507       __ehhandler$?qt_emit@fileManager@@UAE_NHPAUQUObject@@@Z 1001e507 f   moc_workstationeditordlgimpl.obj
 0001:0001d507       __ehhandler$?qt_emit@workstationEditorDlg@@UAE_NHPAUQUObject@@@Z 1001e507 f   moc_workstationeditordlgimpl.obj
 0001:0001d507       __ehhandler$?qt_emit@workstationEditor@@UAE_NHPAUQUObject@@@Z 1001e507 f   moc_workstationeditordlgimpl.obj
 0001:0001d522       __unwindfunclet$??0workstationDockWindowBase@@QAE@PAVQWidget@@PBDI@Z$0 1001e522 f   workstationdockwindow.obj
 0001:0001d52b       __unwindfunclet$??0workstationDockWindowBase@@QAE@PAVQWidget@@PBDI@Z$1 1001e52b f   workstationdockwindow.obj
 0001:0001d53a       __unwindfunclet$??0workstationDockWindowBase@@QAE@PAVQWidget@@PBDI@Z$2 1001e53a f   workstationdockwindow.obj
 0001:0001d544       __unwindfunclet$??0workstationDockWindowBase@@QAE@PAVQWidget@@PBDI@Z$3 1001e544 f   workstationdockwindow.obj
 0001:0001d54e       __unwindfunclet$??0workstationDockWindowBase@@QAE@PAVQWidget@@PBDI@Z$4 1001e54e f   workstationdockwindow.obj
 0001:0001d558       __unwindfunclet$??0workstationDockWindowBase@@QAE@PAVQWidget@@PBDI@Z$5 1001e558 f   workstationdockwindow.obj
 0001:0001d562       __unwindfunclet$??0workstationDockWindowBase@@QAE@PAVQWidget@@PBDI@Z$6 1001e562 f   workstationdockwindow.obj
 0001:0001d56c       __unwindfunclet$??0workstationDockWindowBase@@QAE@PAVQWidget@@PBDI@Z$7 1001e56c f   workstationdockwindow.obj
 0001:0001d575       __ehhandler$??0workstationDockWindowBase@@QAE@PAVQWidget@@PBDI@Z 1001e575 f   workstationdockwindow.obj
 0001:0001d590       __unwindfunclet$??1workstationEditorDlgBase@@UAE@XZ$0 1001e590 f   workstationdockwindow.obj
 0001:0001d590       __unwindfunclet$??1workstationDockWindowBase@@UAE@XZ$0 1001e590 f   workstationdockwindow.obj
 0001:0001d590       __unwindfunclet$??1launchEditorDlgBase@@UAE@XZ$0 1001e590 f   workstationdockwindow.obj
 0001:0001d599       __ehhandler$??1workstationDockWindowBase@@UAE@XZ 1001e599 f   workstationdockwindow.obj
 0001:0001d599       __ehhandler$??1launchEditorDlgBase@@UAE@XZ 1001e599 f   workstationdockwindow.obj
 0001:0001d599       __ehhandler$??1workstationEditorDlgBase@@UAE@XZ 1001e599 f   workstationdockwindow.obj
 0001:0001d5b4       __unwindfunclet$?languageChange@workstationDockWindowBase@@MAEXXZ$0 1001e5b4 f   workstationdockwindow.obj
 0001:0001d5bd       __unwindfunclet$?languageChange@workstationDockWindowBase@@MAEXXZ$1 1001e5bd f   workstationdockwindow.obj
 0001:0001d5c6       __ehhandler$?languageChange@workstationDockWindowBase@@MAEXXZ 1001e5c6 f   workstationdockwindow.obj
 0001:0001d5e1       __unwindfunclet$??0workstationEditorDlgBase@@QAE@PAVQWidget@@PBDI@Z$0 1001e5e1 f   workstationeditordlg.obj
 0001:0001d5ea       __unwindfunclet$??0workstationEditorDlgBase@@QAE@PAVQWidget@@PBDI@Z$1 1001e5ea f   workstationeditordlg.obj
 0001:0001d5f9       __unwindfunclet$??0workstationEditorDlgBase@@QAE@PAVQWidget@@PBDI@Z$2 1001e5f9 f   workstationeditordlg.obj
 0001:0001d603       __unwindfunclet$??0workstationEditorDlgBase@@QAE@PAVQWidget@@PBDI@Z$3 1001e603 f   workstationeditordlg.obj
 0001:0001d60d       __unwindfunclet$??0workstationEditorDlgBase@@QAE@PAVQWidget@@PBDI@Z$4 1001e60d f   workstationeditordlg.obj
 0001:0001d617       __unwindfunclet$??0workstationEditorDlgBase@@QAE@PAVQWidget@@PBDI@Z$5 1001e617 f   workstationeditordlg.obj
 0001:0001d621       __unwindfunclet$??0workstationEditorDlgBase@@QAE@PAVQWidget@@PBDI@Z$6 1001e621 f   workstationeditordlg.obj
 0001:0001d62b       __unwindfunclet$??0workstationEditorDlgBase@@QAE@PAVQWidget@@PBDI@Z$7 1001e62b f   workstationeditordlg.obj
 0001:0001d635       __unwindfunclet$??0workstationEditorDlgBase@@QAE@PAVQWidget@@PBDI@Z$8 1001e635 f   workstationeditordlg.obj
 0001:0001d63f       __unwindfunclet$??0workstationEditorDlgBase@@QAE@PAVQWidget@@PBDI@Z$9 1001e63f f   workstationeditordlg.obj
 0001:0001d649       __ehhandler$??0workstationEditorDlgBase@@QAE@PAVQWidget@@PBDI@Z 1001e649 f   workstationeditordlg.obj
 0001:0001d664       __unwindfunclet$?languageChange@workstationEditorDlgBase@@MAEXXZ$0 1001e664 f   workstationeditordlg.obj
 0001:0001d66d       __unwindfunclet$?languageChange@workstationEditorDlgBase@@MAEXXZ$1 1001e66d f   workstationeditordlg.obj
 0001:0001d676       __unwindfunclet$?languageChange@workstationEditorDlgBase@@MAEXXZ$2 1001e676 f   workstationeditordlg.obj
 0001:0001d67f       __unwindfunclet$?languageChange@workstationEditorDlgBase@@MAEXXZ$3 1001e67f f   workstationeditordlg.obj
 0001:0001d688       __unwindfunclet$?languageChange@workstationEditorDlgBase@@MAEXXZ$4 1001e688 f   workstationeditordlg.obj
 0001:0001d691       __unwindfunclet$?languageChange@workstationEditorDlgBase@@MAEXXZ$5 1001e691 f   workstationeditordlg.obj
 0001:0001d69a       __unwindfunclet$?languageChange@workstationEditorDlgBase@@MAEXXZ$6 1001e69a f   workstationeditordlg.obj
 0001:0001d6a3       __unwindfunclet$?languageChange@workstationEditorDlgBase@@MAEXXZ$7 1001e6a3 f   workstationeditordlg.obj
 0001:0001d6ac       __ehhandler$?languageChange@workstationEditorDlgBase@@MAEXXZ 1001e6ac f   workstationeditordlg.obj
 0001:0001d6c7       __unwindfunclet$??0workstationEditorNewWsDlgBase@@QAE@PAVQWidget@@PBD_NI@Z$0 1001e6c7 f   workstationeditornewwsdlg.obj
 0001:0001d6d0       __unwindfunclet$??0workstationEditorNewWsDlgBase@@QAE@PAVQWidget@@PBD_NI@Z$1 1001e6d0 f   workstationeditornewwsdlg.obj
 0001:0001d6da       __unwindfunclet$??0workstationEditorNewWsDlgBase@@QAE@PAVQWidget@@PBD_NI@Z$2 1001e6da f   workstationeditornewwsdlg.obj
 0001:0001d6e4       __unwindfunclet$??0workstationEditorNewWsDlgBase@@QAE@PAVQWidget@@PBD_NI@Z$3 1001e6e4 f   workstationeditornewwsdlg.obj
 0001:0001d6ee       __unwindfunclet$??0workstationEditorNewWsDlgBase@@QAE@PAVQWidget@@PBD_NI@Z$4 1001e6ee f   workstationeditornewwsdlg.obj
 0001:0001d6f8       __unwindfunclet$??0workstationEditorNewWsDlgBase@@QAE@PAVQWidget@@PBD_NI@Z$5 1001e6f8 f   workstationeditornewwsdlg.obj
 0001:0001d702       __unwindfunclet$??0workstationEditorNewWsDlgBase@@QAE@PAVQWidget@@PBD_NI@Z$6 1001e702 f   workstationeditornewwsdlg.obj
 0001:0001d70c       __unwindfunclet$??0workstationEditorNewWsDlgBase@@QAE@PAVQWidget@@PBD_NI@Z$7 1001e70c f   workstationeditornewwsdlg.obj
 0001:0001d716       __unwindfunclet$??0workstationEditorNewWsDlgBase@@QAE@PAVQWidget@@PBD_NI@Z$8 1001e716 f   workstationeditornewwsdlg.obj
 0001:0001d720       __unwindfunclet$??0workstationEditorNewWsDlgBase@@QAE@PAVQWidget@@PBD_NI@Z$9 1001e720 f   workstationeditornewwsdlg.obj
 0001:0001d72a       __unwindfunclet$??0workstationEditorNewWsDlgBase@@QAE@PAVQWidget@@PBD_NI@Z$10 1001e72a f   workstationeditornewwsdlg.obj
 0001:0001d734       __unwindfunclet$??0workstationEditorNewWsDlgBase@@QAE@PAVQWidget@@PBD_NI@Z$11 1001e734 f   workstationeditornewwsdlg.obj
 0001:0001d73e       __unwindfunclet$??0workstationEditorNewWsDlgBase@@QAE@PAVQWidget@@PBD_NI@Z$12 1001e73e f   workstationeditornewwsdlg.obj
 0001:0001d748       __unwindfunclet$??0workstationEditorNewWsDlgBase@@QAE@PAVQWidget@@PBD_NI@Z$13 1001e748 f   workstationeditornewwsdlg.obj
 0001:0001d752       __unwindfunclet$??0workstationEditorNewWsDlgBase@@QAE@PAVQWidget@@PBD_NI@Z$14 1001e752 f   workstationeditornewwsdlg.obj
 0001:0001d75c       __unwindfunclet$??0workstationEditorNewWsDlgBase@@QAE@PAVQWidget@@PBD_NI@Z$15 1001e75c f   workstationeditornewwsdlg.obj
 0001:0001d766       __unwindfunclet$??0workstationEditorNewWsDlgBase@@QAE@PAVQWidget@@PBD_NI@Z$16 1001e766 f   workstationeditornewwsdlg.obj
 0001:0001d770       __unwindfunclet$??0workstationEditorNewWsDlgBase@@QAE@PAVQWidget@@PBD_NI@Z$17 1001e770 f   workstationeditornewwsdlg.obj
 0001:0001d77a       __unwindfunclet$??0workstationEditorNewWsDlgBase@@QAE@PAVQWidget@@PBD_NI@Z$18 1001e77a f   workstationeditornewwsdlg.obj
 0001:0001d784       __unwindfunclet$??0workstationEditorNewWsDlgBase@@QAE@PAVQWidget@@PBD_NI@Z$19 1001e784 f   workstationeditornewwsdlg.obj
 0001:0001d78e       __unwindfunclet$??0workstationEditorNewWsDlgBase@@QAE@PAVQWidget@@PBD_NI@Z$20 1001e78e f   workstationeditornewwsdlg.obj
 0001:0001d798       __unwindfunclet$??0workstationEditorNewWsDlgBase@@QAE@PAVQWidget@@PBD_NI@Z$21 1001e798 f   workstationeditornewwsdlg.obj
 0001:0001d7a2       __unwindfunclet$??0workstationEditorNewWsDlgBase@@QAE@PAVQWidget@@PBD_NI@Z$22 1001e7a2 f   workstationeditornewwsdlg.obj
 0001:0001d7ac       __unwindfunclet$??0workstationEditorNewWsDlgBase@@QAE@PAVQWidget@@PBD_NI@Z$23 1001e7ac f   workstationeditornewwsdlg.obj
 0001:0001d7b6       __unwindfunclet$??0workstationEditorNewWsDlgBase@@QAE@PAVQWidget@@PBD_NI@Z$24 1001e7b6 f   workstationeditornewwsdlg.obj
 0001:0001d7c0       __unwindfunclet$??0workstationEditorNewWsDlgBase@@QAE@PAVQWidget@@PBD_NI@Z$25 1001e7c0 f   workstationeditornewwsdlg.obj
 0001:0001d7ca       __ehhandler$??0workstationEditorNewWsDlgBase@@QAE@PAVQWidget@@PBD_NI@Z 1001e7ca f   workstationeditornewwsdlg.obj
 0001:0001d7e5       __unwindfunclet$?languageChange@workstationEditorNewWsDlgBase@@MAEXXZ$0 1001e7e5 f   workstationeditornewwsdlg.obj
 0001:0001d7ee       __unwindfunclet$?languageChange@workstationEditorNewWsDlgBase@@MAEXXZ$1 1001e7ee f   workstationeditornewwsdlg.obj
 0001:0001d7f7       __unwindfunclet$?languageChange@workstationEditorNewWsDlgBase@@MAEXXZ$2 1001e7f7 f   workstationeditornewwsdlg.obj
 0001:0001d800       __unwindfunclet$?languageChange@workstationEditorNewWsDlgBase@@MAEXXZ$3 1001e800 f   workstationeditornewwsdlg.obj
 0001:0001d809       __unwindfunclet$?languageChange@workstationEditorNewWsDlgBase@@MAEXXZ$4 1001e809 f   workstationeditornewwsdlg.obj
 0001:0001d812       __unwindfunclet$?languageChange@workstationEditorNewWsDlgBase@@MAEXXZ$5 1001e812 f   workstationeditornewwsdlg.obj
 0001:0001d81b       __unwindfunclet$?languageChange@workstationEditorNewWsDlgBase@@MAEXXZ$6 1001e81b f   workstationeditornewwsdlg.obj
 0001:0001d824       __unwindfunclet$?languageChange@workstationEditorNewWsDlgBase@@MAEXXZ$7 1001e824 f   workstationeditornewwsdlg.obj
 0001:0001d82d       __unwindfunclet$?languageChange@workstationEditorNewWsDlgBase@@MAEXXZ$8 1001e82d f   workstationeditornewwsdlg.obj
 0001:0001d836       __unwindfunclet$?languageChange@workstationEditorNewWsDlgBase@@MAEXXZ$9 1001e836 f   workstationeditornewwsdlg.obj
 0001:0001d83f       __unwindfunclet$?languageChange@workstationEditorNewWsDlgBase@@MAEXXZ$10 1001e83f f   workstationeditornewwsdlg.obj
 0001:0001d848       __ehhandler$?languageChange@workstationEditorNewWsDlgBase@@MAEXXZ 1001e848 f   workstationeditornewwsdlg.obj
 0001:0001d863       __unwindfunclet$??0cfg_Table@@QAE@PAVQWidget@@PBD@Z$0 1001e863 f   cfg_widgets001:cfg_Table.obj
 0001:0001d86c       __ehhandler$??0cfg_Table@@QAE@PAVQWidget@@PBD@Z 1001e86c f   cfg_widgets001:cfg_Table.obj
 0001:0001d887       __unwindfunclet$?copyToClipboard@cfg_Table@@QAEXXZ$0 1001e887 f   cfg_widgets001:cfg_Table.obj
 0001:0001d890       __unwindfunclet$?copyToClipboard@cfg_Table@@QAEXXZ$1 1001e890 f   cfg_widgets001:cfg_Table.obj
 0001:0001d899       __unwindfunclet$?copyToClipboard@cfg_Table@@QAEXXZ$2 1001e899 f   cfg_widgets001:cfg_Table.obj
 0001:0001d8a2       __ehhandler$?copyToClipboard@cfg_Table@@QAEXXZ 1001e8a2 f   cfg_widgets001:cfg_Table.obj
 0001:0001d8bd       __unwindfunclet$?deleteItems@cfg_Table@@QAEXXZ$0 1001e8bd f   cfg_widgets001:cfg_Table.obj
 0001:0001d8c6       __ehhandler$?deleteItems@cfg_Table@@QAEXXZ 1001e8c6 f   cfg_widgets001:cfg_Table.obj
 0001:0001d8e1       __unwindfunclet$?fillUndoBuffer@cfg_Table@@AAEXXZ$0 1001e8e1 f   cfg_widgets001:cfg_Table.obj
 0001:0001d8eb       __unwindfunclet$?fillUndoBuffer@cfg_Table@@AAEXXZ$1 1001e8eb f   cfg_widgets001:cfg_Table.obj
 0001:0001d8f4       __unwindfunclet$?fillUndoBuffer@cfg_Table@@AAEXXZ$2 1001e8f4 f   cfg_widgets001:cfg_Table.obj
 0001:0001d8fd       __unwindfunclet$?fillUndoBuffer@cfg_Table@@AAEXXZ$3 1001e8fd f   cfg_widgets001:cfg_Table.obj
 0001:0001d906       __ehhandler$?fillUndoBuffer@cfg_Table@@AAEXXZ 1001e906 f   cfg_widgets001:cfg_Table.obj
 0001:0001d921       __unwindfunclet$?pasteClipboard@cfg_Table@@QAEXXZ$0 1001e921 f   cfg_widgets001:cfg_Table.obj
 0001:0001d92a       __unwindfunclet$?pasteClipboard@cfg_Table@@QAEXXZ$1 1001e92a f   cfg_widgets001:cfg_Table.obj
 0001:0001d933       __unwindfunclet$?pasteClipboard@cfg_Table@@QAEXXZ$2 1001e933 f   cfg_widgets001:cfg_Table.obj
 0001:0001d93c       __unwindfunclet$?pasteClipboard@cfg_Table@@QAEXXZ$3 1001e93c f   cfg_widgets001:cfg_Table.obj
 0001:0001d945       __unwindfunclet$?pasteClipboard@cfg_Table@@QAEXXZ$4 1001e945 f   cfg_widgets001:cfg_Table.obj
 0001:0001d94e       __unwindfunclet$?pasteClipboard@cfg_Table@@QAEXXZ$5 1001e94e f   cfg_widgets001:cfg_Table.obj
 0001:0001d957       __unwindfunclet$?pasteClipboard@cfg_Table@@QAEXXZ$6 1001e957 f   cfg_widgets001:cfg_Table.obj
 0001:0001d960       __unwindfunclet$?pasteClipboard@cfg_Table@@QAEXXZ$7 1001e960 f   cfg_widgets001:cfg_Table.obj
 0001:0001d969       __unwindfunclet$?pasteClipboard@cfg_Table@@QAEXXZ$8 1001e969 f   cfg_widgets001:cfg_Table.obj
 0001:0001d972       __unwindfunclet$?pasteClipboard@cfg_Table@@QAEXXZ$9 1001e972 f   cfg_widgets001:cfg_Table.obj
 0001:0001d97b       __unwindfunclet$?pasteClipboard@cfg_Table@@QAEXXZ$10 1001e97b f   cfg_widgets001:cfg_Table.obj
 0001:0001d984       __unwindfunclet$?pasteClipboard@cfg_Table@@QAEXXZ$11 1001e984 f   cfg_widgets001:cfg_Table.obj
 0001:0001d98d       __unwindfunclet$?pasteClipboard@cfg_Table@@QAEXXZ$12 1001e98d f   cfg_widgets001:cfg_Table.obj
 0001:0001d996       __unwindfunclet$?pasteClipboard@cfg_Table@@QAEXXZ$13 1001e996 f   cfg_widgets001:cfg_Table.obj
 0001:0001d99f       __ehhandler$?pasteClipboard@cfg_Table@@QAEXXZ 1001e99f f   cfg_widgets001:cfg_Table.obj
 0001:0001d9ba       __unwindfunclet$?undoPaste@cfg_Table@@QAEXXZ$0 1001e9ba f   cfg_widgets001:cfg_Table.obj
 0001:0001d9c3       __unwindfunclet$?undoPaste@cfg_Table@@QAEXXZ$1 1001e9c3 f   cfg_widgets001:cfg_Table.obj
 0001:0001d9cc       __unwindfunclet$?undoPaste@cfg_Table@@QAEXXZ$2 1001e9cc f   cfg_widgets001:cfg_Table.obj
 0001:0001d9d5       __ehhandler$?undoPaste@cfg_Table@@QAEXXZ 1001e9d5 f   cfg_widgets001:cfg_Table.obj
 0001:0001d9f0       __unwindfunclet$??0configFile@@QAE@PAVpluginBase@@VQString@@_N@Z$0 1001e9f0 f   pluginBase:configFile.obj
 0001:0001d9f9       __unwindfunclet$??0configFile@@QAE@PAVpluginBase@@VQString@@_N@Z$1 1001e9f9 f   pluginBase:configFile.obj
 0001:0001da02       __unwindfunclet$??0configFile@@QAE@PAVpluginBase@@VQString@@_N@Z$2 1001ea02 f   pluginBase:configFile.obj
 0001:0001da0e       __unwindfunclet$??0configFile@@QAE@PAVpluginBase@@VQString@@_N@Z$3 1001ea0e f   pluginBase:configFile.obj
 0001:0001da1a       __unwindfunclet$??0configFile@@QAE@PAVpluginBase@@VQString@@_N@Z$4 1001ea1a f   pluginBase:configFile.obj
 0001:0001da26       __ehhandler$??0configFile@@QAE@PAVpluginBase@@VQString@@_N@Z 1001ea26 f   pluginBase:configFile.obj
 0001:0001da50       __unwindfunclet$??1configFile@@UAE@XZ$0 1001ea50 f   pluginBase:configFile.obj
 0001:0001da50       __unwindfunclet$??_GconfigFile@@UAEPAXI@Z$0 1001ea50 f   pluginBase:configFile.obj
 0001:0001da59       __unwindfunclet$??1configFile@@UAE@XZ$1 1001ea59 f   pluginBase:configFile.obj
 0001:0001da59       __unwindfunclet$??_GconfigFile@@UAEPAXI@Z$1 1001ea59 f   pluginBase:configFile.obj
 0001:0001da65       __unwindfunclet$??_GconfigFile@@UAEPAXI@Z$2 1001ea65 f   pluginBase:configFile.obj
 0001:0001da65       __unwindfunclet$??1configFile@@UAE@XZ$2 1001ea65 f   pluginBase:configFile.obj
 0001:0001da71       __ehhandler$??_GconfigFile@@UAEPAXI@Z 1001ea71 f   pluginBase:configFile.obj
 0001:0001da71       __ehhandler$??1configFile@@UAE@XZ 1001ea71 f   pluginBase:configFile.obj
 0001:0001da90       __unwindfunclet$??BconfigFile@@QAE?AVQFileInfo@@XZ$0 1001ea90 f   pluginBase:configFile.obj
 0001:0001da99       __unwindfunclet$??BconfigFile@@QAE?AVQFileInfo@@XZ$1 1001ea99 f   pluginBase:configFile.obj
 0001:0001dab3       __ehhandler$??BconfigFile@@QAE?AVQFileInfo@@XZ 1001eab3 f   pluginBase:configFile.obj
 0001:0001dad0       __unwindfunclet$?dirList@configFile@@QAE_NAAVQStringList@@@Z$9 1001ead0 f   pluginBase:configFile.obj
 0001:0001dad9       __unwindfunclet$?dirList@configFile@@QAE_NAAVQStringList@@@Z$10 1001ead9 f   pluginBase:configFile.obj
 0001:0001dae2       __unwindfunclet$?dirList@configFile@@QAE_NAAVQStringList@@@Z$1 1001eae2 f   pluginBase:configFile.obj
 0001:0001daeb       __unwindfunclet$?dirList@configFile@@QAE_NAAVQStringList@@@Z$2 1001eaeb f   pluginBase:configFile.obj
 0001:0001daf4       __unwindfunclet$?dirList@configFile@@QAE_NAAVQStringList@@@Z$3 1001eaf4 f   pluginBase:configFile.obj
 0001:0001dafd       __unwindfunclet$?dirList@configFile@@QAE_NAAVQStringList@@@Z$4 1001eafd f   pluginBase:configFile.obj
 0001:0001db06       __unwindfunclet$?dirList@configFile@@QAE_NAAVQStringList@@@Z$5 1001eb06 f   pluginBase:configFile.obj
 0001:0001db0f       __unwindfunclet$?dirList@configFile@@QAE_NAAVQStringList@@@Z$6 1001eb0f f   pluginBase:configFile.obj
 0001:0001db18       __unwindfunclet$?dirList@configFile@@QAE_NAAVQStringList@@@Z$7 1001eb18 f   pluginBase:configFile.obj
 0001:0001db21       __unwindfunclet$?dirList@configFile@@QAE_NAAVQStringList@@@Z$8 1001eb21 f   pluginBase:configFile.obj
 0001:0001db2a       __ehhandler$?dirList@configFile@@QAE_NAAVQStringList@@@Z 1001eb2a f   pluginBase:configFile.obj
 0001:0001db50       __unwindfunclet$?getLocalPath@configFile@@QAE?AVQString@@XZ$0 1001eb50 f   pluginBase:configFile.obj
 0001:0001db59       __unwindfunclet$?getLocalPath@configFile@@QAE?AVQString@@XZ$1 1001eb59 f   pluginBase:configFile.obj
 0001:0001db62       __unwindfunclet$?getLocalPath@configFile@@QAE?AVQString@@XZ$2 1001eb62 f   pluginBase:configFile.obj
 0001:0001db6b       __unwindfunclet$?getLocalPath@configFile@@QAE?AVQString@@XZ$3 1001eb6b f   pluginBase:configFile.obj
 0001:0001db85       __ehhandler$?getLocalPath@configFile@@QAE?AVQString@@XZ 1001eb85 f   pluginBase:configFile.obj
 0001:0001dba0       __unwindfunclet$?getModTime@configFile@@QAE?AVQDateTime@@XZ$0 1001eba0 f   pluginBase:configFile.obj
 0001:0001dba9       __unwindfunclet$?getModTime@configFile@@QAE?AVQDateTime@@XZ$1 1001eba9 f   pluginBase:configFile.obj
 0001:0001dbb2       __ehhandler$?getModTime@configFile@@QAE?AVQDateTime@@XZ 1001ebb2 f   pluginBase:configFile.obj
 0001:0001dbd0       __unwindfunclet$?reply@configFile@@MAEXPAVresponse@@@Z$1 1001ebd0 f   pluginBase:configFile.obj
 0001:0001dbd9       __ehhandler$?reply@configFile@@MAEXPAVresponse@@@Z 1001ebd9 f   pluginBase:configFile.obj
 0001:0001dc00       __unwindfunclet$?sendCommand@configFile@@IAEXVQString@@@Z$0 1001ec00 f   pluginBase:configFile.obj
 0001:0001dc09       __unwindfunclet$?sendCommand@configFile@@IAEXVQString@@@Z$1 1001ec09 f   pluginBase:configFile.obj
 0001:0001dc12       __ehhandler$?sendCommand@configFile@@IAEXVQString@@@Z 1001ec12 f   pluginBase:configFile.obj
 0001:0001dc30       __unwindfunclet$?setDirty@configFile@@QAE_NXZ$1 1001ec30 f   pluginBase:configFile.obj
 0001:0001dc39       __unwindfunclet$?setDirty@configFile@@QAE_NXZ$2 1001ec39 f   pluginBase:configFile.obj
 0001:0001dc42       __ehhandler$?setDirty@configFile@@QAE_NXZ 1001ec42 f   pluginBase:configFile.obj
 0001:0001dc60       __unwindfunclet$?timerEvent@configFile@@MAEXPAVQTimerEvent@@@Z$1 1001ec60 f   pluginBase:configFile.obj
 0001:0001dc69       __ehhandler$?timerEvent@configFile@@MAEXPAVQTimerEvent@@@Z 1001ec69 f   pluginBase:configFile.obj
 0001:0001dc90       __unwindfunclet$?unlock@configFile@@QAE_N_N@Z$1 1001ec90 f   pluginBase:configFile.obj
 0001:0001dc99       __unwindfunclet$?unlock@configFile@@QAE_N_N@Z$2 1001ec99 f   pluginBase:configFile.obj
 0001:0001dca2       __ehhandler$?unlock@configFile@@QAE_N_N@Z 1001eca2 f   pluginBase:configFile.obj
 0001:0001dcc0       __unwindfunclet$??0?$QMapNode@VQString@@VconfigFile@@@@QAE@ABU0@@Z$1 1001ecc0 f   pluginBase:pluginBase.obj
 0001:0001dccb       __unwindfunclet$??0?$QMapNode@VQString@@VconfigFile@@@@QAE@ABU0@@Z$2 1001eccb f   pluginBase:pluginBase.obj
 0001:0001dcd7       __ehhandler$??0?$QMapNode@VQString@@VconfigFile@@@@QAE@ABU0@@Z 1001ecd7 f   pluginBase:pluginBase.obj
 0001:0001dd00       __unwindfunclet$??0?$QMapPrivate@VQString@@VconfigFile@@@@QAE@PBV0@@Z$0 1001ed00 f   pluginBase:pluginBase.obj
 0001:0001dd0b       __unwindfunclet$??0?$QMapPrivate@VQString@@VconfigFile@@@@QAE@PBV0@@Z$2 1001ed0b f   pluginBase:pluginBase.obj
 0001:0001dd16       __ehhandler$??0?$QMapPrivate@VQString@@VconfigFile@@@@QAE@PBV0@@Z 1001ed16 f   pluginBase:pluginBase.obj
 0001:0001dd40       __unwindfunclet$??0?$QMapPrivate@VQString@@VconfigFile@@@@QAE@XZ$0 1001ed40 f   pluginBase:pluginBase.obj
 0001:0001dd4b       __unwindfunclet$??0?$QMapPrivate@VQString@@VconfigFile@@@@QAE@XZ$2 1001ed4b f   pluginBase:pluginBase.obj
 0001:0001dd56       __ehhandler$??0?$QMapPrivate@VQString@@VconfigFile@@@@QAE@XZ 1001ed56 f   pluginBase:pluginBase.obj
 0001:0001dd80       __unwindfunclet$??0pluginBase@@QAE@ABVQString@@00@Z$0 1001ed80 f   pluginBase:pluginBase.obj
 0001:0001dd88       __unwindfunclet$??0pluginBase@@QAE@ABVQString@@00@Z$4 1001ed88 f   pluginBase:pluginBase.obj
 0001:0001dd93       __unwindfunclet$??0pluginBase@@QAE@ABVQString@@00@Z$1 1001ed93 f   pluginBase:pluginBase.obj
 0001:0001dd9e       __unwindfunclet$??0pluginBase@@QAE@ABVQString@@00@Z$2 1001ed9e f   pluginBase:pluginBase.obj
 0001:0001ddac       __ehhandler$??0pluginBase@@QAE@ABVQString@@00@Z 1001edac f   pluginBase:pluginBase.obj
 0001:0001ddd0       __unwindfunclet$??1?$QMapNode@VQString@@VconfigFile@@@@QAE@XZ$0 1001edd0 f   pluginBase:pluginBase.obj
 0001:0001dddb       __unwindfunclet$??1?$QMapNode@VQString@@VconfigFile@@@@QAE@XZ$2 1001eddb f   pluginBase:pluginBase.obj
 0001:0001dde4       __unwindfunclet$??1?$QMapNode@VQString@@VconfigFile@@@@QAE@XZ$3 1001ede4 f   pluginBase:pluginBase.obj
 0001:0001ddf0       __unwindfunclet$??1?$QMapNode@VQString@@VconfigFile@@@@QAE@XZ$4 1001edf0 f   pluginBase:pluginBase.obj
 0001:0001ddfc       __ehhandler$??1?$QMapNode@VQString@@VconfigFile@@@@QAE@XZ 1001edfc f   pluginBase:pluginBase.obj
 0001:0001de20       __unwindfunclet$??1pluginBase@@UAE@XZ$0 1001ee20 f   pluginBase:pluginBase.obj
 0001:0001de28       __unwindfunclet$??1pluginBase@@UAE@XZ$1 1001ee28 f   pluginBase:pluginBase.obj
 0001:0001de33       __unwindfunclet$??1pluginBase@@UAE@XZ$2 1001ee33 f   pluginBase:pluginBase.obj
 0001:0001de41       __unwindfunclet$??1pluginBase@@UAE@XZ$3 1001ee41 f   pluginBase:pluginBase.obj
 0001:0001de4f       __unwindfunclet$??1pluginBase@@UAE@XZ$4 1001ee4f f   pluginBase:pluginBase.obj
 0001:0001de57       __unwindfunclet$??1pluginBase@@UAE@XZ$5 1001ee57 f   pluginBase:pluginBase.obj
 0001:0001de60       __unwindfunclet$??1pluginBase@@UAE@XZ$6 1001ee60 f   pluginBase:pluginBase.obj
 0001:0001de69       __unwindfunclet$??1pluginBase@@UAE@XZ$7 1001ee69 f   pluginBase:pluginBase.obj
 0001:0001de72       __unwindfunclet$??1pluginBase@@UAE@XZ$8 1001ee72 f   pluginBase:pluginBase.obj
 0001:0001de7d       __unwindfunclet$??1pluginBase@@UAE@XZ$10 1001ee7d f   pluginBase:pluginBase.obj
 0001:0001de86       __unwindfunclet$??1pluginBase@@UAE@XZ$11 1001ee86 f   pluginBase:pluginBase.obj
 0001:0001de92       __unwindfunclet$??1pluginBase@@UAE@XZ$12 1001ee92 f   pluginBase:pluginBase.obj
 0001:0001de9e       __unwindfunclet$??1pluginBase@@UAE@XZ$14 1001ee9e f   pluginBase:pluginBase.obj
 0001:0001dea7       __unwindfunclet$??1pluginBase@@UAE@XZ$15 1001eea7 f   pluginBase:pluginBase.obj
 0001:0001deb3       __unwindfunclet$??1pluginBase@@UAE@XZ$16 1001eeb3 f   pluginBase:pluginBase.obj
 0001:0001debf       __ehhandler$??1pluginBase@@UAE@XZ 1001eebf f   pluginBase:pluginBase.obj
 0001:0001dee0       __unwindfunclet$??A?$QMap@VQString@@VconfigFile@@@@QAEAAVconfigFile@@ABVQString@@@Z$2 1001eee0 f   pluginBase:pluginBase.obj
 0001:0001deeb       __unwindfunclet$??A?$QMap@VQString@@VconfigFile@@@@QAEAAVconfigFile@@ABVQString@@@Z$1 1001eeeb f   pluginBase:pluginBase.obj
 0001:0001def3       __unwindfunclet$??A?$QMap@VQString@@VconfigFile@@@@QAEAAVconfigFile@@ABVQString@@@Z$3 1001eef3 f   pluginBase:pluginBase.obj
 0001:0001defc       __unwindfunclet$??A?$QMap@VQString@@VconfigFile@@@@QAEAAVconfigFile@@ABVQString@@@Z$4 1001eefc f   pluginBase:pluginBase.obj
 0001:0001df05       __unwindfunclet$??A?$QMap@VQString@@VconfigFile@@@@QAEAAVconfigFile@@ABVQString@@@Z$5 1001ef05 f   pluginBase:pluginBase.obj
 0001:0001df0e       __ehhandler$??A?$QMap@VQString@@VconfigFile@@@@QAEAAVconfigFile@@ABVQString@@@Z 1001ef0e f   pluginBase:pluginBase.obj
 0001:0001df30       __unwindfunclet$?clear@?$QMapPrivate@VQString@@VconfigFile@@@@QAEXPAU?$QMapNode@VQString@@VconfigFile@@@@@Z$0 1001ef30 f   pluginBase:pluginBase.obj
 0001:0001df3b       __unwindfunclet$?clear@?$QMapPrivate@VQString@@VconfigFile@@@@QAEXPAU?$QMapNode@VQString@@VconfigFile@@@@@Z$2 1001ef3b f   pluginBase:pluginBase.obj
 0001:0001df44       __unwindfunclet$?clear@?$QMapPrivate@VQString@@VconfigFile@@@@QAEXPAU?$QMapNode@VQString@@VconfigFile@@@@@Z$3 1001ef44 f   pluginBase:pluginBase.obj
 0001:0001df50       __unwindfunclet$?clear@?$QMapPrivate@VQString@@VconfigFile@@@@QAEXPAU?$QMapNode@VQString@@VconfigFile@@@@@Z$4 1001ef50 f   pluginBase:pluginBase.obj
 0001:0001df5c       __ehhandler$?clear@?$QMapPrivate@VQString@@VconfigFile@@@@QAEXPAU?$QMapNode@VQString@@VconfigFile@@@@@Z 1001ef5c f   pluginBase:pluginBase.obj
 0001:0001df80       __unwindfunclet$?copy@?$QMapPrivate@VQString@@VconfigFile@@@@QAEPAU?$QMapNode@VQString@@VconfigFile@@@@PAU2@@Z$0 1001ef80 f   pluginBase:pluginBase.obj
 0001:0001df8b       __ehhandler$?copy@?$QMapPrivate@VQString@@VconfigFile@@@@QAEPAU?$QMapNode@VQString@@VconfigFile@@@@PAU2@@Z 1001ef8b f   pluginBase:pluginBase.obj
 0001:0001dfb0       __unwindfunclet$?file@pluginBase@@QAEAAVconfigFile@@VQString@@@Z$0 1001efb0 f   pluginBase:pluginBase.obj
 0001:0001dfb9       __unwindfunclet$?file@pluginBase@@QAEAAVconfigFile@@VQString@@@Z$3 1001efb9 f   pluginBase:pluginBase.obj
 0001:0001dfc1       __unwindfunclet$?file@pluginBase@@QAEAAVconfigFile@@VQString@@@Z$4 1001efc1 f   pluginBase:pluginBase.obj
 0001:0001dfca       __unwindfunclet$?file@pluginBase@@QAEAAVconfigFile@@VQString@@@Z$5 1001efca f   pluginBase:pluginBase.obj
 0001:0001dfd3       __unwindfunclet$?file@pluginBase@@QAEAAVconfigFile@@VQString@@@Z$6 1001efd3 f   pluginBase:pluginBase.obj
 0001:0001dfdc       __ehhandler$?file@pluginBase@@QAEAAVconfigFile@@VQString@@@Z 1001efdc f   pluginBase:pluginBase.obj
 0001:0001e000       __unwindfunclet$?insert@?$QMap@VQString@@VconfigFile@@@@QAE?AV?$QMapIterator@VQString@@VconfigFile@@@@ABVQString@@ABVconfigFile@@_N@Z$0 1001f000 f   pluginBase:pluginBase.obj
 0001:0001e00b       __ehhandler$?insert@?$QMap@VQString@@VconfigFile@@@@QAE?AV?$QMapIterator@VQString@@VconfigFile@@@@ABVQString@@ABVconfigFile@@_N@Z 1001f00b f   pluginBase:pluginBase.obj
 0001:0001e030       __unwindfunclet$?insert@?$QMapPrivate@VQString@@VconfigFile@@@@QAE?AV?$QMapIterator@VQString@@VconfigFile@@@@PAUQMapNodeBase@@0ABVQString@@@Z$0 1001f030 f   pluginBase:pluginBase.obj
 0001:0001e03b       __unwindfunclet$?insert@?$QMapPrivate@VQString@@VconfigFile@@@@QAE?AV?$QMapIterator@VQString@@VconfigFile@@@@PAUQMapNodeBase@@0ABVQString@@@Z$2 1001f03b f   pluginBase:pluginBase.obj
 0001:0001e046       __unwindfunclet$?insert@?$QMapPrivate@VQString@@VconfigFile@@@@QAE?AV?$QMapIterator@VQString@@VconfigFile@@@@PAUQMapNodeBase@@0ABVQString@@@Z$3 1001f046 f   pluginBase:pluginBase.obj
 0001:0001e052       __ehhandler$?insert@?$QMapPrivate@VQString@@VconfigFile@@@@QAE?AV?$QMapIterator@VQString@@VconfigFile@@@@PAUQMapNodeBase@@0ABVQString@@@Z 1001f052 f   pluginBase:pluginBase.obj
 0001:0001e070       __unwindfunclet$?isDirty@pluginBase@@EAE_NXZ$0 1001f070 f   pluginBase:pluginBase.obj
 0001:0001e070       __unwindfunclet$?uploadAllFiles@pluginBase@@AAEXXZ$0 1001f070 f   pluginBase:pluginBase.obj
 0001:0001e070       __unwindfunclet$?releaseAllLocks@pluginBase@@AAEXXZ$0 1001f070 f   pluginBase:pluginBase.obj
 0001:0001e07b       __unwindfunclet$?uploadAllFiles@pluginBase@@AAEXXZ$1 1001f07b f   pluginBase:pluginBase.obj
 0001:0001e07b       __unwindfunclet$?isDirty@pluginBase@@EAE_NXZ$1 1001f07b f   pluginBase:pluginBase.obj
 0001:0001e07b       __unwindfunclet$?releaseAllLocks@pluginBase@@AAEXXZ$1 1001f07b f   pluginBase:pluginBase.obj
 0001:0001e086       __ehhandler$?releaseAllLocks@pluginBase@@AAEXXZ 1001f086 f   pluginBase:pluginBase.obj
 0001:0001e086       __ehhandler$?isDirty@pluginBase@@EAE_NXZ 1001f086 f   pluginBase:pluginBase.obj
 0001:0001e086       __ehhandler$?uploadAllFiles@pluginBase@@AAEXXZ 1001f086 f   pluginBase:pluginBase.obj
 0001:0001e0b0       __unwindfunclet$?loadModdedFiles@pluginBase@@AAEXXZ$0 1001f0b0 f   pluginBase:pluginBase.obj
 0001:0001e0b0       __unwindfunclet$?saveAllFiles@pluginBase@@AAEXXZ$0 1001f0b0 f   pluginBase:pluginBase.obj
 0001:0001e0b0       __unwindfunclet$?waitForAllFiles@pluginBase@@QAE_NXZ$0 1001f0b0 f   pluginBase:pluginBase.obj
 0001:0001e0bb       __unwindfunclet$?loadModdedFiles@pluginBase@@AAEXXZ$1 1001f0bb f   pluginBase:pluginBase.obj
 0001:0001e0bb       __unwindfunclet$?saveAllFiles@pluginBase@@AAEXXZ$1 1001f0bb f   pluginBase:pluginBase.obj
 0001:0001e0bb       __unwindfunclet$?waitForAllFiles@pluginBase@@QAE_NXZ$1 1001f0bb f   pluginBase:pluginBase.obj
 0001:0001e0c6       __ehhandler$?saveAllFiles@pluginBase@@AAEXXZ 1001f0c6 f   pluginBase:pluginBase.obj
 0001:0001e0c6       __ehhandler$?waitForAllFiles@pluginBase@@QAE_NXZ 1001f0c6 f   pluginBase:pluginBase.obj
 0001:0001e0c6       __ehhandler$?loadModdedFiles@pluginBase@@AAEXXZ 1001f0c6 f   pluginBase:pluginBase.obj
 0001:0001e0f0       __unwindfunclet$?sendCommand@pluginBase@@AAEXVQString@@0@Z$0 1001f0f0 f   pluginBase:pluginBase.obj
 0001:0001e0f9       __unwindfunclet$?sendCommand@pluginBase@@AAEXVQString@@0@Z$1 1001f0f9 f   pluginBase:pluginBase.obj
 0001:0001e102       __unwindfunclet$?sendCommand@pluginBase@@AAEXVQString@@0@Z$2 1001f102 f   pluginBase:pluginBase.obj
 0001:0001e10b       __ehhandler$?sendCommand@pluginBase@@AAEXVQString@@0@Z 1001f10b f   pluginBase:pluginBase.obj
 0001:0001e130       __unwindfunclet$?command@pluginBase@@IAEXVQString@@0@Z$0 1001f130 f   pluginBase:moc_pluginBase.obj
 0001:0001e139       __unwindfunclet$?command@pluginBase@@IAEXVQString@@0@Z$1 1001f139 f   pluginBase:moc_pluginBase.obj
 0001:0001e142       __unwindfunclet$?command@pluginBase@@IAEXVQString@@0@Z$2 1001f142 f   pluginBase:moc_pluginBase.obj
 0001:0001e156       __ehhandler$?command@pluginBase@@IAEXVQString@@0@Z 1001f156 f   pluginBase:moc_pluginBase.obj
 0001:0001e180       __unwindfunclet$?qt_emit@pluginBase@@UAE_NHPAUQUObject@@@Z$0 1001f180 f   pluginBase:moc_pluginBase.obj
 0001:0001e189       __ehhandler$?qt_emit@pluginBase@@UAE_NHPAUQUObject@@@Z 1001f189 f   pluginBase:moc_pluginBase.obj
 0001:0001e1b0       ??__FcleanUp_dialogBase@@YAXXZ 1001f1b0 f   moc_dialog.obj
 0001:0001e1bb       ??__FcleanUp_dialog@@YAXXZ 1001f1bb f   moc_dialogimpl.obj
 0001:0001e1c6       ??__FcleanUp_fileDrop@@YAXXZ 1001f1c6 f   moc_fileDrop.obj
 0001:0001e1d1       ??__FcleanUp_fileManager@@YAXXZ 1001f1d1 f   moc_fileManager.obj
 0001:0001e1dc       ??__FcleanUp_fromBaseDialogBase@@YAXXZ 1001f1dc f   moc_frombasedialog.obj
 0001:0001e1e7       ??__FcleanUp_fromBaseDialog@@YAXXZ 1001f1e7 f   moc_frombasedialogimpl.obj
 0001:0001e1f2       ??__FcleanUp_launchEditor@@YAXXZ 1001f1f2 f   moc_launchEditor.obj
 0001:0001e1fd       ??__FcleanUp_launchEditorDlgBase@@YAXXZ 1001f1fd f   moc_launcheditordlg.obj
 0001:0001e208       ??__FcleanUp_launchEditorDlg@@YAXXZ 1001f208 f   moc_launcheditordlgimpl.obj
 0001:0001e213       ??__FcleanUp_testPlugin@@YAXXZ 1001f213 f   moc_testPlugin.obj
 0001:0001e21e       ??__FcleanUp_testPluginFromBase@@YAXXZ 1001f21e f   moc_testPluginFromBase.obj
 0001:0001e229       ??__FcleanUp_workstationCustomTable@@YAXXZ 1001f229 f   moc_workstationCustomTable.obj
 0001:0001e234       ??__FcleanUp_workstationDockWindowBase@@YAXXZ 1001f234 f   moc_workstationdockwindow.obj
 0001:0001e23f       ??__FcleanUp_workstationDockWindow@@YAXXZ 1001f23f f   moc_workstationdockwindowimpl.obj
 0001:0001e24a       ??__FcleanUp_workstationEditor@@YAXXZ 1001f24a f   moc_workstationeditor.obj
 0001:0001e255       ??__FcleanUp_workstationEditorDlgBase@@YAXXZ 1001f255 f   moc_workstationeditordlg.obj
 0001:0001e260       ??__FcleanUp_workstationEditorDlg@@YAXXZ 1001f260 f   moc_workstationeditordlgimpl.obj
 0001:0001e26b       ??__FcleanUp_workstationEditorNewWsDlgBase@@YAXXZ 1001f26b f   moc_workstationeditornewwsdlg.obj
 0001:0001e276       ??__FcleanUp_workstationEditorNewWsDlg@@YAXXZ 1001f276 f   moc_workstationeditornewwsdlgimpl.obj
 0001:0001e281       ??__FcleanUp_xml_listview@@YAXXZ 1001f281 f   moc_xml_listview.obj
 0001:0001e28c       ??__FcleanUp_cfg_Table@@YAXXZ 1001f28c f   cfg_widgets001:moc_cfg_Table.obj
 0001:0001e2a0       ??__FcleanUp_pluginBase@@YAXXZ 1001f2a0 f   pluginBase:moc_pluginBase.obj
 0001:0001e2b0       ??__FcleanUp_configFile@@YAXXZ 1001f2b0 f   pluginBase:moc_configFile.obj
 0002:000012a4       _cleanUp_dialogBase$initializer$ 100212a4     moc_dialog.obj
 0002:000012a8       _cleanUp_dialog$initializer$ 100212a8     moc_dialogimpl.obj
 0002:000012ac       _cleanUp_fileDrop$initializer$ 100212ac     moc_fileDrop.obj
 0002:000012b0       _cleanUp_fileManager$initializer$ 100212b0     moc_fileManager.obj
 0002:000012b4       _cleanUp_fromBaseDialogBase$initializer$ 100212b4     moc_frombasedialog.obj
 0002:000012b8       _cleanUp_fromBaseDialog$initializer$ 100212b8     moc_frombasedialogimpl.obj
 0002:000012bc       _cleanUp_launchEditor$initializer$ 100212bc     moc_launchEditor.obj
 0002:000012c0       _cleanUp_launchEditorDlgBase$initializer$ 100212c0     moc_launcheditordlg.obj
 0002:000012c4       _cleanUp_launchEditorDlg$initializer$ 100212c4     moc_launcheditordlgimpl.obj
 0002:000012c8       _cleanUp_testPlugin$initializer$ 100212c8     moc_testPlugin.obj
 0002:000012cc       _cleanUp_testPluginFromBase$initializer$ 100212cc     moc_testPluginFromBase.obj
 0002:000012d0       _cleanUp_workstationCustomTable$initializer$ 100212d0     moc_workstationCustomTable.obj
 0002:000012d4       _cleanUp_workstationDockWindowBase$initializer$ 100212d4     moc_workstationdockwindow.obj
 0002:000012d8       _cleanUp_workstationDockWindow$initializer$ 100212d8     moc_workstationdockwindowimpl.obj
 0002:000012dc       _cleanUp_workstationEditor$initializer$ 100212dc     moc_workstationeditor.obj
 0002:000012e0       _cleanUp_workstationEditorDlgBase$initializer$ 100212e0     moc_workstationeditordlg.obj
 0002:000012e4       _cleanUp_workstationEditorDlg$initializer$ 100212e4     moc_workstationeditordlgimpl.obj
 0002:000012e8       _cleanUp_workstationEditorNewWsDlgBase$initializer$ 100212e8     moc_workstationeditornewwsdlg.obj
 0002:000012ec       _cleanUp_workstationEditorNewWsDlg$initializer$ 100212ec     moc_workstationeditornewwsdlgimpl.obj
 0002:000012f0       _cleanUp_xml_listview$initializer$ 100212f0     moc_xml_listview.obj
 0002:000012f4       _cleanUp_cfg_Table$initializer$ 100212f4     cfg_widgets001:moc_cfg_Table.obj
 0002:000012f8       _cleanUp_pluginBase$initializer$ 100212f8     pluginBase:moc_pluginBase.obj
 0002:000012fc       _cleanUp_configFile$initializer$ 100212fc     pluginBase:moc_configFile.obj
 0002:00001308       _pcinit                    10021308     MSVCRT:crtdll.obj
 0002:0000130c       _pinit                     1002130c     MSVCRT:atonexit.obj
 0002:0000a53c       ?slot_0@?3??staticMetaObject@dialogBase@@SAPAVQMetaObject@@XZ@4UQUMethod@@B 1002a53c     moc_dialog.obj
 0002:0000a558       ?slot_tbl@?3??staticMetaObject@dialogBase@@SAPAVQMetaObject@@XZ@4QBUQMetaData@@B 1002a558     moc_dialog.obj
 0002:0000a58c       ?slot_0@?3??staticMetaObject@fileDrop@@SAPAVQMetaObject@@XZ@4UQUMethod@@B 1002a58c     moc_fileDrop.obj
 0002:0000a5a4       ?slot_tbl@?3??staticMetaObject@fileDrop@@SAPAVQMetaObject@@XZ@4QBUQMetaData@@B 1002a5a4     moc_fileDrop.obj
 0002:0000a5c0       ?signal_0@?3??staticMetaObject@fileDrop@@SAPAVQMetaObject@@XZ@4UQUMethod@@B 1002a5c0     moc_fileDrop.obj
 0002:0000a5d8       ?signal_tbl@?3??staticMetaObject@fileDrop@@SAPAVQMetaObject@@XZ@4QBUQMetaData@@B 1002a5d8     moc_fileDrop.obj
 0002:0000a61c       ?slot_0@?3??staticMetaObject@fileManager@@SAPAVQMetaObject@@XZ@4UQUMethod@@B 1002a61c     moc_fileManager.obj
 0002:0000a63c       ?slot_1@?3??staticMetaObject@fileManager@@SAPAVQMetaObject@@XZ@4UQUMethod@@B 1002a63c     moc_fileManager.obj
 0002:0000a654       ?slot_tbl@?3??staticMetaObject@fileManager@@SAPAVQMetaObject@@XZ@4QBUQMetaData@@B 1002a654     moc_fileManager.obj
 0002:0000a6a0       ?signal_0@?3??staticMetaObject@fileManager@@SAPAVQMetaObject@@XZ@4UQUMethod@@B 1002a6a0     moc_fileManager.obj
 0002:0000a6b4       ?signal_tbl@?3??staticMetaObject@fileManager@@SAPAVQMetaObject@@XZ@4QBUQMetaData@@B 1002a6b4     moc_fileManager.obj
 0002:0000a6dc       ?slot_0@?3??staticMetaObject@fromBaseDialogBase@@SAPAVQMetaObject@@XZ@4UQUMethod@@B 1002a6dc     moc_frombasedialog.obj
 0002:0000a6e8       ?slot_tbl@?3??staticMetaObject@fromBaseDialogBase@@SAPAVQMetaObject@@XZ@4QBUQMetaData@@B 1002a6e8     moc_frombasedialog.obj
 0002:0000a714       ?slot_0@?3??staticMetaObject@launchEditor@@SAPAVQMetaObject@@XZ@4UQUMethod@@B 1002a714     moc_launchEditor.obj
 0002:0000a734       ?slot_1@?3??staticMetaObject@launchEditor@@SAPAVQMetaObject@@XZ@4UQUMethod@@B 1002a734     moc_launchEditor.obj
 0002:0000a754       ?slot_tbl@?3??staticMetaObject@launchEditor@@SAPAVQMetaObject@@XZ@4QBUQMetaData@@B 1002a754     moc_launchEditor.obj
 0002:0000a7a4       ?signal_0@?3??staticMetaObject@launchEditor@@SAPAVQMetaObject@@XZ@4UQUMethod@@B 1002a7a4     moc_launchEditor.obj
 0002:0000a7b0       ?signal_tbl@?3??staticMetaObject@launchEditor@@SAPAVQMetaObject@@XZ@4QBUQMetaData@@B 1002a7b0     moc_launchEditor.obj
 0002:0000a7bc       ?slot_0@?3??staticMetaObject@launchEditorDlgBase@@SAPAVQMetaObject@@XZ@4UQUMethod@@B 1002a7bc     moc_launcheditordlg.obj
 0002:0000a7c8       ?slot_tbl@?3??staticMetaObject@launchEditorDlgBase@@SAPAVQMetaObject@@XZ@4QBUQMetaData@@B 1002a7c8     moc_launcheditordlg.obj
 0002:0000a7d4       ?slot_0@?3??staticMetaObject@launchEditorDlg@@SAPAVQMetaObject@@XZ@4UQUMethod@@B 1002a7d4     moc_launcheditordlgimpl.obj
 0002:0000a7ec       ?slot_1@?3??staticMetaObject@launchEditorDlg@@SAPAVQMetaObject@@XZ@4UQUMethod@@B 1002a7ec     moc_launcheditordlgimpl.obj
 0002:0000a800       ?slot_2@?3??staticMetaObject@launchEditorDlg@@SAPAVQMetaObject@@XZ@4UQUMethod@@B 1002a800     moc_launcheditordlgimpl.obj
 0002:0000a818       ?slot_3@?3??staticMetaObject@launchEditorDlg@@SAPAVQMetaObject@@XZ@4UQUMethod@@B 1002a818     moc_launcheditordlgimpl.obj
 0002:0000a830       ?slot_4@?3??staticMetaObject@launchEditorDlg@@SAPAVQMetaObject@@XZ@4UQUMethod@@B 1002a830     moc_launcheditordlgimpl.obj
 0002:0000a850       ?slot_5@?3??staticMetaObject@launchEditorDlg@@SAPAVQMetaObject@@XZ@4UQUMethod@@B 1002a850     moc_launcheditordlgimpl.obj
 0002:0000a870       ?slot_6@?3??staticMetaObject@launchEditorDlg@@SAPAVQMetaObject@@XZ@4UQUMethod@@B 1002a870     moc_launcheditordlgimpl.obj
 0002:0000a88c       ?slot_7@?3??staticMetaObject@launchEditorDlg@@SAPAVQMetaObject@@XZ@4UQUMethod@@B 1002a88c     moc_launcheditordlgimpl.obj
 0002:0000a8b0       ?slot_tbl@?3??staticMetaObject@launchEditorDlg@@SAPAVQMetaObject@@XZ@4QBUQMetaData@@B 1002a8b0     moc_launcheditordlgimpl.obj
 0002:0000a9a4       ?signal_0@?3??staticMetaObject@launchEditorDlg@@SAPAVQMetaObject@@XZ@4UQUMethod@@B 1002a9a4     moc_launcheditordlgimpl.obj
 0002:0000a9b0       ?signal_tbl@?3??staticMetaObject@launchEditorDlg@@SAPAVQMetaObject@@XZ@4QBUQMetaData@@B 1002a9b0     moc_launcheditordlgimpl.obj
 0002:0000a9c8       ?slot_0@?3??staticMetaObject@testPlugin@@SAPAVQMetaObject@@XZ@4UQUMethod@@B 1002a9c8     moc_testPlugin.obj
 0002:0000a9d4       ?slot_1@?3??staticMetaObject@testPlugin@@SAPAVQMetaObject@@XZ@4UQUMethod@@B 1002a9d4     moc_testPlugin.obj
 0002:0000a9e0       ?slot_2@?3??staticMetaObject@testPlugin@@SAPAVQMetaObject@@XZ@4UQUMethod@@B 1002a9e0     moc_testPlugin.obj
 0002:0000a9ec       ?slot_3@?3??staticMetaObject@testPlugin@@SAPAVQMetaObject@@XZ@4UQUMethod@@B 1002a9ec     moc_testPlugin.obj
 0002:0000a9f8       ?slot_4@?3??staticMetaObject@testPlugin@@SAPAVQMetaObject@@XZ@4UQUMethod@@B 1002a9f8     moc_testPlugin.obj
 0002:0000aa04       ?slot_5@?3??staticMetaObject@testPlugin@@SAPAVQMetaObject@@XZ@4UQUMethod@@B 1002aa04     moc_testPlugin.obj
 0002:0000aa10       ?slot_6@?3??staticMetaObject@testPlugin@@SAPAVQMetaObject@@XZ@4UQUMethod@@B 1002aa10     moc_testPlugin.obj
 0002:0000aa1c       ?slot_7@?3??staticMetaObject@testPlugin@@SAPAVQMetaObject@@XZ@4UQUMethod@@B 1002aa1c     moc_testPlugin.obj
 0002:0000aa28       ?slot_8@?3??staticMetaObject@testPlugin@@SAPAVQMetaObject@@XZ@4UQUMethod@@B 1002aa28     moc_testPlugin.obj
 0002:0000aa34       ?slot_9@?3??staticMetaObject@testPlugin@@SAPAVQMetaObject@@XZ@4UQUMethod@@B 1002aa34     moc_testPlugin.obj
 0002:0000aa40       ?slot_10@?3??staticMetaObject@testPlugin@@SAPAVQMetaObject@@XZ@4UQUMethod@@B 1002aa40     moc_testPlugin.obj
 0002:0000aa4c       ?slot_11@?3??staticMetaObject@testPlugin@@SAPAVQMetaObject@@XZ@4UQUMethod@@B 1002aa4c     moc_testPlugin.obj
 0002:0000aa64       ?slot_12@?3??staticMetaObject@testPlugin@@SAPAVQMetaObject@@XZ@4UQUMethod@@B 1002aa64     moc_testPlugin.obj
 0002:0000aa78       ?slot_13@?3??staticMetaObject@testPlugin@@SAPAVQMetaObject@@XZ@4UQUMethod@@B 1002aa78     moc_testPlugin.obj
 0002:0000aa90       ?slot_tbl@?3??staticMetaObject@testPlugin@@SAPAVQMetaObject@@XZ@4QBUQMetaData@@B 1002aa90     moc_testPlugin.obj
 0002:0000abf8       ?signal_0@?3??staticMetaObject@testPlugin@@SAPAVQMetaObject@@XZ@4UQUMethod@@B 1002abf8     moc_testPlugin.obj
 0002:0000ac04       ?signal_tbl@?3??staticMetaObject@testPlugin@@SAPAVQMetaObject@@XZ@4QBUQMetaData@@B 1002ac04     moc_testPlugin.obj
 0002:0000ac24       ?slot_0@?3??staticMetaObject@testPluginFromBase@@SAPAVQMetaObject@@XZ@4UQUMethod@@B 1002ac24     moc_testPluginFromBase.obj
 0002:0000ac40       ?slot_1@?3??staticMetaObject@testPluginFromBase@@SAPAVQMetaObject@@XZ@4UQUMethod@@B 1002ac40     moc_testPluginFromBase.obj
 0002:0000ac58       ?slot_2@?3??staticMetaObject@testPluginFromBase@@SAPAVQMetaObject@@XZ@4UQUMethod@@B 1002ac58     moc_testPluginFromBase.obj
 0002:0000ac70       ?slot_3@?3??staticMetaObject@testPluginFromBase@@SAPAVQMetaObject@@XZ@4UQUMethod@@B 1002ac70     moc_testPluginFromBase.obj
 0002:0000ac88       ?slot_4@?3??staticMetaObject@testPluginFromBase@@SAPAVQMetaObject@@XZ@4UQUMethod@@B 1002ac88     moc_testPluginFromBase.obj
 0002:0000aca0       ?slot_5@?3??staticMetaObject@testPluginFromBase@@SAPAVQMetaObject@@XZ@4UQUMethod@@B 1002aca0     moc_testPluginFromBase.obj
 0002:0000acb8       ?slot_6@?3??staticMetaObject@testPluginFromBase@@SAPAVQMetaObject@@XZ@4UQUMethod@@B 1002acb8     moc_testPluginFromBase.obj
 0002:0000acd4       ?slot_7@?3??staticMetaObject@testPluginFromBase@@SAPAVQMetaObject@@XZ@4UQUMethod@@B 1002acd4     moc_testPluginFromBase.obj
 0002:0000acec       ?slot_8@?3??staticMetaObject@testPluginFromBase@@SAPAVQMetaObject@@XZ@4UQUMethod@@B 1002acec     moc_testPluginFromBase.obj
 0002:0000ad08       ?slot_9@?3??staticMetaObject@testPluginFromBase@@SAPAVQMetaObject@@XZ@4UQUMethod@@B 1002ad08     moc_testPluginFromBase.obj
 0002:0000ad24       ?slot_10@?3??staticMetaObject@testPluginFromBase@@SAPAVQMetaObject@@XZ@4UQUMethod@@B 1002ad24     moc_testPluginFromBase.obj
 0002:0000ad38       ?slot_11@?3??staticMetaObject@testPluginFromBase@@SAPAVQMetaObject@@XZ@4UQUMethod@@B 1002ad38     moc_testPluginFromBase.obj
 0002:0000ad50       ?slot_12@?3??staticMetaObject@testPluginFromBase@@SAPAVQMetaObject@@XZ@4UQUMethod@@B 1002ad50     moc_testPluginFromBase.obj
 0002:0000ad64       ?slot_13@?3??staticMetaObject@testPluginFromBase@@SAPAVQMetaObject@@XZ@4UQUMethod@@B 1002ad64     moc_testPluginFromBase.obj
 0002:0000ad7c       ?slot_14@?3??staticMetaObject@testPluginFromBase@@SAPAVQMetaObject@@XZ@4UQUMethod@@B 1002ad7c     moc_testPluginFromBase.obj
 0002:0000ad98       ?slot_tbl@?3??staticMetaObject@testPluginFromBase@@SAPAVQMetaObject@@XZ@4QBUQMetaData@@B 1002ad98     moc_testPluginFromBase.obj
 0002:0000af38       ?slot_0@?3??staticMetaObject@workstationCustomTable@@SAPAVQMetaObject@@XZ@4UQUMethod@@B 1002af38     moc_workstationCustomTable.obj
 0002:0000af54       ?slot_1@?3??staticMetaObject@workstationCustomTable@@SAPAVQMetaObject@@XZ@4UQUMethod@@B 1002af54     moc_workstationCustomTable.obj
 0002:0000af68       ?slot_2@?3??staticMetaObject@workstationCustomTable@@SAPAVQMetaObject@@XZ@4UQUMethod@@B 1002af68     moc_workstationCustomTable.obj
 0002:0000af74       ?slot_3@?3??staticMetaObject@workstationCustomTable@@SAPAVQMetaObject@@XZ@4UQUMethod@@B 1002af74     moc_workstationCustomTable.obj
 0002:0000af8c       ?slot_tbl@?3??staticMetaObject@workstationCustomTable@@SAPAVQMetaObject@@XZ@4QBUQMetaData@@B 1002af8c     moc_workstationCustomTable.obj
 0002:0000b020       ?slot_0@?3??staticMetaObject@workstationDockWindowBase@@SAPAVQMetaObject@@XZ@4UQUMethod@@B 1002b020     moc_workstationdockwindow.obj
 0002:0000b02c       ?slot_tbl@?3??staticMetaObject@workstationDockWindowBase@@SAPAVQMetaObject@@XZ@4QBUQMetaData@@B 1002b02c     moc_workstationdockwindow.obj
 0002:0000b050       ?signal_0@?3??staticMetaObject@workstationDockWindow@@SAPAVQMetaObject@@XZ@4UQUMethod@@B 1002b050     moc_workstationdockwindowimpl.obj
 0002:0000b070       ?signal_tbl@?3??staticMetaObject@workstationDockWindow@@SAPAVQMetaObject@@XZ@4QBUQMetaData@@B 1002b070     moc_workstationdockwindowimpl.obj
 0002:0000b0b4       ?signal_0@?3??staticMetaObject@workstationEditor@@SAPAVQMetaObject@@XZ@4UQUMethod@@B 1002b0b4     moc_workstationeditor.obj
 0002:0000b0c0       ?signal_tbl@?3??staticMetaObject@workstationEditor@@SAPAVQMetaObject@@XZ@4QBUQMetaData@@B 1002b0c0     moc_workstationeditor.obj
 0002:0000b0e8       ?slot_0@?3??staticMetaObject@workstationEditorDlgBase@@SAPAVQMetaObject@@XZ@4UQUMethod@@B 1002b0e8     moc_workstationeditordlg.obj
 0002:0000b0f4       ?slot_tbl@?3??staticMetaObject@workstationEditorDlgBase@@SAPAVQMetaObject@@XZ@4QBUQMetaData@@B 1002b0f4     moc_workstationeditordlg.obj
 0002:0000b118       ?slot_0@?3??staticMetaObject@workstationEditorDlg@@SAPAVQMetaObject@@XZ@4UQUMethod@@B 1002b118     moc_workstationeditordlgimpl.obj
 0002:0000b124       ?slot_1@?3??staticMetaObject@workstationEditorDlg@@SAPAVQMetaObject@@XZ@4UQUMethod@@B 1002b124     moc_workstationeditordlgimpl.obj
 0002:0000b130       ?slot_2@?3??staticMetaObject@workstationEditorDlg@@SAPAVQMetaObject@@XZ@4UQUMethod@@B 1002b130     moc_workstationeditordlgimpl.obj
 0002:0000b13c       ?slot_tbl@?3??staticMetaObject@workstationEditorDlg@@SAPAVQMetaObject@@XZ@4QBUQMetaData@@B 1002b13c     moc_workstationeditordlgimpl.obj
 0002:0000b160       ?signal_0@?3??staticMetaObject@workstationEditorDlg@@SAPAVQMetaObject@@XZ@4UQUMethod@@B 1002b160     moc_workstationeditordlgimpl.obj
 0002:0000b16c       ?signal_tbl@?3??staticMetaObject@workstationEditorDlg@@SAPAVQMetaObject@@XZ@4QBUQMetaData@@B 1002b16c     moc_workstationeditordlgimpl.obj
 0002:0000b198       ?slot_0@?3??staticMetaObject@workstationEditorNewWsDlgBase@@SAPAVQMetaObject@@XZ@4UQUMethod@@B 1002b198     moc_workstationeditornewwsdlg.obj
 0002:0000b1a4       ?slot_tbl@?3??staticMetaObject@workstationEditorNewWsDlgBase@@SAPAVQMetaObject@@XZ@4QBUQMetaData@@B 1002b1a4     moc_workstationeditornewwsdlg.obj
 0002:0000b1dc       ?signal_0@?3??staticMetaObject@xml_listview@@SAPAVQMetaObject@@XZ@4UQUMethod@@B 1002b1dc     moc_xml_listview.obj
 0002:0000b1f4       ?signal_tbl@?3??staticMetaObject@xml_listview@@SAPAVQMetaObject@@XZ@4QBUQMetaData@@B 1002b1f4     moc_xml_listview.obj
 0002:0000c3b0       ?slot_0@?3??staticMetaObject@cfg_Table@@SAPAVQMetaObject@@XZ@4UQUMethod@@B 1002c3b0     cfg_widgets001:moc_cfg_Table.obj
 0002:0000c3c8       ?slot_1@?3??staticMetaObject@cfg_Table@@SAPAVQMetaObject@@XZ@4UQUMethod@@B 1002c3c8     cfg_widgets001:moc_cfg_Table.obj
 0002:0000c3e4       ?slot_2@?3??staticMetaObject@cfg_Table@@SAPAVQMetaObject@@XZ@4UQUMethod@@B 1002c3e4     cfg_widgets001:moc_cfg_Table.obj
 0002:0000c3fc       ?slot_3@?3??staticMetaObject@cfg_Table@@SAPAVQMetaObject@@XZ@4UQUMethod@@B 1002c3fc     cfg_widgets001:moc_cfg_Table.obj
 0002:0000c418       ?slot_4@?3??staticMetaObject@cfg_Table@@SAPAVQMetaObject@@XZ@4UQUMethod@@B 1002c418     cfg_widgets001:moc_cfg_Table.obj
 0002:0000c43c       ?slot_tbl@?3??staticMetaObject@cfg_Table@@SAPAVQMetaObject@@XZ@4QBUQMetaData@@B 1002c43c     cfg_widgets001:moc_cfg_Table.obj
 0002:0000c4d4       ?signal_0@?3??staticMetaObject@cfg_Table@@SAPAVQMetaObject@@XZ@4UQUMethod@@B 1002c4d4     cfg_widgets001:moc_cfg_Table.obj
 0002:0000c4ec       ?signal_1@?3??staticMetaObject@cfg_Table@@SAPAVQMetaObject@@XZ@4UQUMethod@@B 1002c4ec     cfg_widgets001:moc_cfg_Table.obj
 0002:0000c50c       ?signal_tbl@?3??staticMetaObject@cfg_Table@@SAPAVQMetaObject@@XZ@4QBUQMetaData@@B 1002c50c     cfg_widgets001:moc_cfg_Table.obj
 0002:0000c95c       ?signal_0@?3??staticMetaObject@pluginBase@@SAPAVQMetaObject@@XZ@4UQUMethod@@B 1002c95c     pluginBase:moc_pluginBase.obj
 0002:0000c968       ?signal_tbl@?3??staticMetaObject@pluginBase@@SAPAVQMetaObject@@XZ@4QBUQMetaData@@B 1002c968     pluginBase:moc_pluginBase.obj
 0002:0000c98c       _GS_ExceptionPointers      1002c98c     MSVCRT:gs_report.obj
 0002:0000e5c8       __unwindtable$??1xml_listview@@UAE@XZ 1002e5c8     fileDrop.obj
 0002:0000e5c8       __unwindtable$??0fileDrop@@QAE@PAVQWidget@@PBD@Z 1002e5c8     fileDrop.obj
 0002:0000e5d0       __ehfuncinfo$??1xml_listview@@UAE@XZ 1002e5d0     fileDrop.obj
 0002:0000e5d0       __ehfuncinfo$??0fileDrop@@QAE@PAVQWidget@@PBD@Z 1002e5d0     fileDrop.obj
 0002:0000e5f4       __unwindtable$?dropEvent@fileDrop@@UAEXPAVQDropEvent@@@Z 1002e5f4     fileDrop.obj
 0002:0000e604       __ehfuncinfo$?dropEvent@fileDrop@@UAEXPAVQDropEvent@@@Z 1002e604     fileDrop.obj
 0002:0000e628       __unwindtable$?contextMenuEvent@fileDrop@@UAEXPAVQContextMenuEvent@@@Z 1002e628     fileDrop.obj
 0002:0000e648       __ehfuncinfo$?contextMenuEvent@fileDrop@@UAEXPAVQContextMenuEvent@@@Z 1002e648     fileDrop.obj
 0002:0000e66c       __unwindtable$??1QDockWindowList@@UAE@XZ 1002e66c     fileManager.obj
 0002:0000e67c       __ehfuncinfo$??1QDockWindowList@@UAE@XZ 1002e67c     fileManager.obj
 0002:0000e6a0       __unwindtable$??1?$QPtrList@VQPopupMenu@@@@UAE@XZ 1002e6a0     fileManager.obj
 0002:0000e6a8       __ehfuncinfo$??1?$QPtrList@VQPopupMenu@@@@UAE@XZ 1002e6a8     fileManager.obj
 0002:0000e6cc       __unwindtable$??1QPopupMenuList@@UAE@XZ 1002e6cc     fileManager.obj
 0002:0000e6d4       __ehfuncinfo$??1QPopupMenuList@@UAE@XZ 1002e6d4     fileManager.obj
 0002:0000e6f8       __unwindtable$??0config_plugin_base@@QAE@ABVQString@@00@Z 1002e6f8     fileManager.obj
 0002:0000e718       __ehfuncinfo$??0config_plugin_base@@QAE@ABVQString@@00@Z 1002e718     fileManager.obj
 0002:0000e73c       __unwindtable$??1config_plugin_base@@UAE@XZ 1002e73c     fileManager.obj
 0002:0000e754       __ehfuncinfo$??1config_plugin_base@@UAE@XZ 1002e754     fileManager.obj
 0002:0000e778       __unwindtable$?about@config_plugin_base@@UAE?AVQString@@XZ 1002e778     fileManager.obj
 0002:0000e788       __ehfuncinfo$?about@config_plugin_base@@UAE?AVQString@@XZ 1002e788     fileManager.obj
 0002:0000e7ac       __ehfuncinfo$??0fileManager@@QAE@ABVQString@@00@Z 1002e7ac     fileManager.obj
 0002:0000e7d0       __unwindtable$??0fileManager@@QAE@ABVQString@@00@Z 1002e7d0     fileManager.obj
 0002:0000e868       __ehfuncinfo$??1fileManager@@UAE@XZ 1002e868     fileManager.obj
 0002:0000e88c       __unwindtable$??1fileManager@@UAE@XZ 1002e88c     fileManager.obj
 0002:0000e8bc       __ehfuncinfo$?reply@fileManager@@UAEXPAVresponse@@@Z 1002e8bc     fileManager.obj
 0002:0000e8e0       __unwindtable$?reply@fileManager@@UAEXPAVresponse@@@Z 1002e8e0     fileManager.obj
 0002:0000eb18       __unwindtable$??0?$QGuardedPtr@VQDockWindow@@@@QAE@XZ 1002eb18     fileManager.obj
 0002:0000eb18       __unwindtable$??4?$QGuardedPtr@VQDockWindow@@@@QAEAAV0@PAVQDockWindow@@@Z 1002eb18     fileManager.obj
 0002:0000eb18       __unwindtable$??0?$QGuardedPtr@VQPopupMenu@@@@QAE@XZ 1002eb18     fileManager.obj
 0002:0000eb18       __unwindtable$??4?$QGuardedPtr@VQPopupMenu@@@@QAEAAV0@PAVQPopupMenu@@@Z 1002eb18     fileManager.obj
 0002:0000eb20       __ehfuncinfo$??4?$QGuardedPtr@VQDockWindow@@@@QAEAAV0@PAVQDockWindow@@@Z 1002eb20     fileManager.obj
 0002:0000eb20       __ehfuncinfo$??0?$QGuardedPtr@VQDockWindow@@@@QAE@XZ 1002eb20     fileManager.obj
 0002:0000eb20       __ehfuncinfo$??0?$QGuardedPtr@VQPopupMenu@@@@QAE@XZ 1002eb20     fileManager.obj
 0002:0000eb20       __ehfuncinfo$??4?$QGuardedPtr@VQPopupMenu@@@@QAEAAV0@PAVQPopupMenu@@@Z 1002eb20     fileManager.obj
 0002:0000eb44       __ehfuncinfo$?copyFile@fileManager@@AAEXABVQString@@0@Z 1002eb44     fileManager.obj
 0002:0000eb68       __unwindtable$?copyFile@fileManager@@AAEXABVQString@@0@Z 1002eb68     fileManager.obj
 0002:0000eb90       __unwindtable$?dirChanged@fileManager@@QAEXPAVQListViewItem@@@Z 1002eb90     fileManager.obj
 0002:0000eba8       __ehfuncinfo$?dirChanged@fileManager@@QAEXPAVQListViewItem@@@Z 1002eba8     fileManager.obj
 0002:0000ebcc       __ehfuncinfo$?doFileList@fileManager@@QAEXVQStringList@@@Z 1002ebcc     fileManager.obj
 0002:0000ebf0       __unwindtable$?doFileList@fileManager@@QAEXVQStringList@@@Z 1002ebf0     fileManager.obj
 0002:0000ec38       __ehfuncinfo$??0fromBaseDialogBase@@QAE@PAVQWidget@@PBDI@Z 1002ec38     frombasedialog.obj
 0002:0000ec5c       __unwindtable$??0fromBaseDialogBase@@QAE@PAVQWidget@@PBDI@Z 1002ec5c     frombasedialog.obj
 0002:0000ee14       __ehfuncinfo$?languageChange@fromBaseDialogBase@@MAEXXZ 1002ee14     frombasedialog.obj
 0002:0000ee38       __unwindtable$?languageChange@fromBaseDialogBase@@MAEXXZ 1002ee38     frombasedialog.obj
 0002:0000eef8       __ehfuncinfo$??0launchCustomTable@@QAE@PAVQWidget@@PBD@Z 1002eef8     launchCustomTable.obj
 0002:0000ef1c       __unwindtable$??0launchCustomTable@@QAE@PAVQWidget@@PBD@Z 1002ef1c     launchCustomTable.obj
 0002:0000ef54       __ehfuncinfo$??0launchEditor@@QAE@ABVQString@@00@Z 1002ef54     launchEditor.obj
 0002:0000ef78       __unwindtable$??0launchEditor@@QAE@ABVQString@@00@Z 1002ef78     launchEditor.obj
 0002:0000f120       __unwindtable$?toolbars@workstationEditor@@UAE?AVQDockWindowList@@XZ 1002f120     launchEditor.obj
 0002:0000f120       __unwindtable$?toolbars@launchEditor@@UAE?AVQDockWindowList@@XZ 1002f120     launchEditor.obj
 0002:0000f128       __ehfuncinfo$?toolbars@workstationEditor@@UAE?AVQDockWindowList@@XZ 1002f128     launchEditor.obj
 0002:0000f128       __ehfuncinfo$?toolbars@launchEditor@@UAE?AVQDockWindowList@@XZ 1002f128     launchEditor.obj
 0002:0000f14c       __unwindtable$?menus@launchEditor@@UAE?AVQPopupMenuList@@XZ 1002f14c     launchEditor.obj
 0002:0000f14c       __unwindtable$?menus@workstationEditor@@UAE?AVQPopupMenuList@@XZ 1002f14c     launchEditor.obj
 0002:0000f154       __ehfuncinfo$?menus@launchEditor@@UAE?AVQPopupMenuList@@XZ 1002f154     launchEditor.obj
 0002:0000f154       __ehfuncinfo$?menus@workstationEditor@@UAE?AVQPopupMenuList@@XZ 1002f154     launchEditor.obj
 0002:0000f178       __ehfuncinfo$?reply@launchEditor@@UAEXPAVresponse@@@Z 1002f178     launchEditor.obj
 0002:0000f19c       __unwindtable$?reply@launchEditor@@UAEXPAVresponse@@@Z 1002f19c     launchEditor.obj
 0002:0000f20c       __ehfuncinfo$?activate@launchEditor@@UAEX_N@Z 1002f20c     launchEditor.obj
 0002:0000f230       __unwindtable$?activate@launchEditor@@UAEX_N@Z 1002f230     launchEditor.obj
 0002:0000f268       __ehfuncinfo$?about@workstationEditor@@UAE?AVQString@@XZ 1002f268     launchEditor.obj
 0002:0000f268       __ehfuncinfo$?about@launchEditor@@UAE?AVQString@@XZ 1002f268     launchEditor.obj
 0002:0000f28c       __unwindtable$?about@workstationEditor@@UAE?AVQString@@XZ 1002f28c     launchEditor.obj
 0002:0000f28c       __unwindtable$?about@launchEditor@@UAE?AVQString@@XZ 1002f28c     launchEditor.obj
 0002:0000f2b4       __unwindtable$??1?$QDict@VQAction@@@@UAE@XZ 1002f2b4     launchEditor.obj
 0002:0000f2bc       __ehfuncinfo$??1?$QDict@VQAction@@@@UAE@XZ 1002f2bc     launchEditor.obj
 0002:0000f2e0       __unwindtable$?navigateToWs@launchEditor@@AAEXH@Z 1002f2e0     launchEditor.obj
 0002:0000f2f0       __ehfuncinfo$?navigateToWs@launchEditor@@AAEXH@Z 1002f2f0     launchEditor.obj
 0002:0000f314       __unwindtable$?workstationChanged@launchEditor@@AAEXPAVQListViewItem@@@Z 1002f314     launchEditor.obj
 0002:0000f324       __ehfuncinfo$?workstationChanged@launchEditor@@AAEXPAVQListViewItem@@@Z 1002f324     launchEditor.obj
 0002:0000f348       __ehfuncinfo$??0launchEditorDlg@@QAE@ABVQString@@PAVQWidget@@PBDI@Z 1002f348     launcheditordlgimpl.obj
 0002:0000f36c       __unwindtable$??0launchEditorDlg@@QAE@ABVQString@@PAVQWidget@@PBDI@Z 1002f36c     launcheditordlgimpl.obj
 0002:0000f3cc       __unwindtable$??1launchEditorDlg@@UAE@XZ 1002f3cc     launcheditordlgimpl.obj
 0002:0000f3d4       __ehfuncinfo$??1launchEditorDlg@@UAE@XZ 1002f3d4     launcheditordlgimpl.obj
 0002:0000f3f8       __ehfuncinfo$?load@launchEditorDlg@@QAE_NABVQString@@H@Z 1002f3f8     launcheditordlgimpl.obj
 0002:0000f41c       __unwindtable$?load@launchEditorDlg@@QAE_NABVQString@@H@Z 1002f41c     launcheditordlgimpl.obj
 0002:0000f544       __ehfuncinfo$?save@launchEditorDlg@@QAEXH@Z 1002f544     launcheditordlgimpl.obj
 0002:0000f568       __unwindtable$?save@launchEditorDlg@@QAEXH@Z 1002f568     launcheditordlgimpl.obj
 0002:0000f650       __ehfuncinfo$?createLaunchElement@launchEditorDlg@@QAE?AVQDomElement@@ABVQString@@AAVQDomDocument@@@Z 1002f650     launcheditordlgimpl.obj
 0002:0000f674       __unwindtable$?createLaunchElement@launchEditorDlg@@QAE?AVQDomElement@@ABVQString@@AAVQDomDocument@@@Z 1002f674     launcheditordlgimpl.obj
 0002:0000f714       __ehfuncinfo$?doDuplicate@launchEditorDlg@@QAEXXZ 1002f714     launcheditordlgimpl.obj
 0002:0000f738       __unwindtable$?doDuplicate@launchEditorDlg@@QAEXXZ 1002f738     launcheditordlgimpl.obj
 0002:0000f778       __ehfuncinfo$?doAdd@launchEditorDlg@@QAEXXZ 1002f778     launcheditordlgimpl.obj
 0002:0000f79c       __unwindtable$?doAdd@launchEditorDlg@@QAEXXZ 1002f79c     launcheditordlgimpl.obj
 0002:0000f7dc       __unwindtable$?doRemove@workstationEditorDlg@@AAEXXZ 1002f7dc     launcheditordlgimpl.obj
 0002:0000f7dc       __unwindtable$?doMoveUp@launchEditorDlg@@QAEXXZ 1002f7dc     launcheditordlgimpl.obj
 0002:0000f7dc       __unwindtable$?doMoveDown@launchEditorDlg@@QAEXXZ 1002f7dc     launcheditordlgimpl.obj
 0002:0000f7e4       __ehfuncinfo$?doMoveUp@launchEditorDlg@@QAEXXZ 1002f7e4     launcheditordlgimpl.obj
 0002:0000f7e4       __ehfuncinfo$?doMoveDown@launchEditorDlg@@QAEXXZ 1002f7e4     launcheditordlgimpl.obj
 0002:0000f7e4       __ehfuncinfo$?doRemove@workstationEditorDlg@@AAEXXZ 1002f7e4     launcheditordlgimpl.obj
 0002:0000f808       __unwindtable$?tableValueChanged@workstationEditorDlg@@AAEXHH@Z 1002f808     launcheditordlgimpl.obj
 0002:0000f808       __unwindtable$?tableValueChanged@launchEditorDlg@@QAEXHH@Z 1002f808     launcheditordlgimpl.obj
 0002:0000f810       __ehfuncinfo$?tableValueChanged@workstationEditorDlg@@AAEXHH@Z 1002f810     launcheditordlgimpl.obj
 0002:0000f810       __ehfuncinfo$?tableValueChanged@launchEditorDlg@@QAEXHH@Z 1002f810     launcheditordlgimpl.obj
 0002:0000f834       __ehfuncinfo$?keys@plugindesc@@UAE?AVQStringList@@ABVQString@@0@Z 1002f834     plugindesc.obj
 0002:0000f858       __unwindtable$?keys@plugindesc@@UAE?AVQStringList@@ABVQString@@0@Z 1002f858     plugindesc.obj
 0002:0000f890       __ehfuncinfo$?create@plugindesc@@UAEPAVconfig_plugin_base@@ABVQString@@00@Z 1002f890     plugindesc.obj
 0002:0000f8b4       __unwindtable$?create@plugindesc@@UAEPAVconfig_plugin_base@@ABVQString@@00@Z 1002f8b4     plugindesc.obj
 0002:0000f8dc       __ehfuncinfo$??0testPlugin@@QAE@ABVQString@@00@Z 1002f8dc     testPlugin.obj
 0002:0000f900       __unwindtable$??0testPlugin@@QAE@ABVQString@@00@Z 1002f900     testPlugin.obj
 0002:0000fbd8       __ehfuncinfo$??1testPlugin@@UAE@XZ 1002fbd8     testPlugin.obj
 0002:0000fbd8       __ehfuncinfo$??1launchEditor@@UAE@XZ 1002fbd8     testPlugin.obj
 0002:0000fbfc       __unwindtable$??1launchEditor@@UAE@XZ 1002fbfc     testPlugin.obj
 0002:0000fbfc       __unwindtable$??1testPlugin@@UAE@XZ 1002fbfc     testPlugin.obj
 0002:0000fc24       __unwindtable$?toolbars@testPlugin@@UAE?AVQDockWindowList@@XZ 1002fc24     testPlugin.obj
 0002:0000fc2c       __ehfuncinfo$?toolbars@testPlugin@@UAE?AVQDockWindowList@@XZ 1002fc2c     testPlugin.obj
 0002:0000fc50       __unwindtable$?menus@testPlugin@@UAE?AVQPopupMenuList@@XZ 1002fc50     testPlugin.obj
 0002:0000fc58       __ehfuncinfo$?menus@testPlugin@@UAE?AVQPopupMenuList@@XZ 1002fc58     testPlugin.obj
 0002:0000fc7c       __ehfuncinfo$?reply@testPlugin@@UAEXPAVresponse@@@Z 1002fc7c     testPlugin.obj
 0002:0000fca0       __unwindtable$?reply@testPlugin@@UAEXPAVresponse@@@Z 1002fca0     testPlugin.obj
 0002:0000fce8       __unwindtable$?timerEvent@fileManager@@EAEXPAVQTimerEvent@@@Z 1002fce8     testPlugin.obj
 0002:0000fce8       __unwindtable$?activate@testPlugin@@UAEX_N@Z 1002fce8     testPlugin.obj
 0002:0000fce8       __unwindtable$?activate@fileManager@@UAEX_N@Z 1002fce8     testPlugin.obj
 0002:0000fcf0       __ehfuncinfo$?activate@fileManager@@UAEX_N@Z 1002fcf0     testPlugin.obj
 0002:0000fcf0       __ehfuncinfo$?timerEvent@fileManager@@EAEXPAVQTimerEvent@@@Z 1002fcf0     testPlugin.obj
 0002:0000fcf0       __ehfuncinfo$?activate@testPlugin@@UAEX_N@Z 1002fcf0     testPlugin.obj
 0002:0000fd14       __ehfuncinfo$?closeEvent@testPlugin@@UAEXPAVQCloseEvent@@@Z 1002fd14     testPlugin.obj
 0002:0000fd38       __unwindtable$?closeEvent@testPlugin@@UAEXPAVQCloseEvent@@@Z 1002fd38     testPlugin.obj
 0002:0000fd78       __unwindtable$?lock@configFile@@QAE_N_N@Z 1002fd78     testPlugin.obj
 0002:0000fd78       __unwindtable$?db@testPluginFromBase@@AAEXVQString@@@Z 1002fd78     testPlugin.obj
 0002:0000fd78       __unwindtable$?db@testPlugin@@AAEXVQString@@@Z 1002fd78     testPlugin.obj
 0002:0000fd78       __unwindtable$?lviFind@fileManager@@AAEPAVQListViewItem@@PAV2@ABVQString@@@Z 1002fd78     testPlugin.obj
 0002:0000fd80       __ehfuncinfo$?db@testPlugin@@AAEXVQString@@@Z 1002fd80     testPlugin.obj
 0002:0000fd80       __ehfuncinfo$?db@testPluginFromBase@@AAEXVQString@@@Z 1002fd80     testPlugin.obj
 0002:0000fd80       __ehfuncinfo$?lock@configFile@@QAE_N_N@Z 1002fd80     testPlugin.obj
 0002:0000fd80       __ehfuncinfo$?lviFind@fileManager@@AAEPAVQListViewItem@@PAV2@ABVQString@@@Z 1002fd80     testPlugin.obj
 0002:0000fda4       __unwindtable$?csiValueChanged@launchEditorDlg@@QAEXABVQString@@@Z 1002fda4     testPlugin.obj
 0002:0000fda4       __unwindtable$?doHelp@testPlugin@@AAEXXZ 1002fda4     testPlugin.obj
 0002:0000fda4       __unwindtable$?lockFile@testPlugin@@AAEXXZ 1002fda4     testPlugin.obj
 0002:0000fda4       __unwindtable$?doDirty@testPlugin@@AAEXXZ 1002fda4     testPlugin.obj
 0002:0000fda4       __unwindtable$?closeEvent@launchEditor@@UAEXPAVQCloseEvent@@@Z 1002fda4     testPlugin.obj
 0002:0000fda4       __unwindtable$?downloadFile@testPlugin@@AAEXXZ 1002fda4     testPlugin.obj
 0002:0000fda4       __unwindtable$?apply@launchEditor@@UAEXXZ 1002fda4     testPlugin.obj
 0002:0000fda4       __unwindtable$?doNavigate@testPlugin@@AAEXXZ 1002fda4     testPlugin.obj
 0002:0000fda4       __unwindtable$?navigateWSEditor@launchEditor@@AAEXXZ 1002fda4     testPlugin.obj
 0002:0000fda4       __unwindtable$?apply@testPlugin@@UAEXXZ 1002fda4     testPlugin.obj
 0002:0000fda4       __unwindtable$?dir@testPlugin@@AAEXXZ 1002fda4     testPlugin.obj
 0002:0000fda4       __unwindtable$?checkoutFile@testPlugin@@AAEXXZ 1002fda4     testPlugin.obj
 0002:0000fda4       __unwindtable$?uploadFile@testPlugin@@AAEXXZ 1002fda4     testPlugin.obj
 0002:0000fda4       __unwindtable$?doRemove@launchEditorDlg@@QAEXXZ 1002fda4     testPlugin.obj
 0002:0000fda4       __unwindtable$?unlockFile@testPlugin@@AAEXXZ 1002fda4     testPlugin.obj
 0002:0000fda4       __unwindtable$?checkoutDir@testPlugin@@AAEXXZ 1002fda4     testPlugin.obj
 0002:0000fda4       __unwindtable$?rebootoptionchanged@launchEditorDlg@@QAEXXZ 1002fda4     testPlugin.obj
 0002:0000fda4       __unwindtable$?unlockDir@testPlugin@@AAEXXZ 1002fda4     testPlugin.obj
 0002:0000fda4       __unwindtable$?uploadDir@testPlugin@@AAEXXZ 1002fda4     testPlugin.obj
 0002:0000fda4       __unwindtable$?downloadDir@testPlugin@@AAEXXZ 1002fda4     testPlugin.obj
 0002:0000fdac       __ehfuncinfo$?downloadDir@testPlugin@@AAEXXZ 1002fdac     testPlugin.obj
 0002:0000fdac       __ehfuncinfo$?uploadDir@testPlugin@@AAEXXZ 1002fdac     testPlugin.obj
 0002:0000fdac       __ehfuncinfo$?unlockDir@testPlugin@@AAEXXZ 1002fdac     testPlugin.obj
 0002:0000fdac       __ehfuncinfo$?unlockFile@testPlugin@@AAEXXZ 1002fdac     testPlugin.obj
 0002:0000fdac       __ehfuncinfo$?navigateWSEditor@launchEditor@@AAEXXZ 1002fdac     testPlugin.obj
 0002:0000fdac       __ehfuncinfo$?apply@launchEditor@@UAEXXZ 1002fdac     testPlugin.obj
 0002:0000fdac       __ehfuncinfo$?closeEvent@launchEditor@@UAEXPAVQCloseEvent@@@Z 1002fdac     testPlugin.obj
 0002:0000fdac       __ehfuncinfo$?doDirty@testPlugin@@AAEXXZ 1002fdac     testPlugin.obj
 0002:0000fdac       __ehfuncinfo$?lockFile@testPlugin@@AAEXXZ 1002fdac     testPlugin.obj
 0002:0000fdac       __ehfuncinfo$?rebootoptionchanged@launchEditorDlg@@QAEXXZ 1002fdac     testPlugin.obj
 0002:0000fdac       __ehfuncinfo$?csiValueChanged@launchEditorDlg@@QAEXABVQString@@@Z 1002fdac     testPlugin.obj
 0002:0000fdac       __ehfuncinfo$?doHelp@testPlugin@@AAEXXZ 1002fdac     testPlugin.obj
 0002:0000fdac       __ehfuncinfo$?downloadFile@testPlugin@@AAEXXZ 1002fdac     testPlugin.obj
 0002:0000fdac       __ehfuncinfo$?doNavigate@testPlugin@@AAEXXZ 1002fdac     testPlugin.obj
 0002:0000fdac       __ehfuncinfo$?apply@testPlugin@@UAEXXZ 1002fdac     testPlugin.obj
 0002:0000fdac       __ehfuncinfo$?dir@testPlugin@@AAEXXZ 1002fdac     testPlugin.obj
 0002:0000fdac       __ehfuncinfo$?doRemove@launchEditorDlg@@QAEXXZ 1002fdac     testPlugin.obj
 0002:0000fdac       __ehfuncinfo$?checkoutDir@testPlugin@@AAEXXZ 1002fdac     testPlugin.obj
 0002:0000fdac       __ehfuncinfo$?uploadFile@testPlugin@@AAEXXZ 1002fdac     testPlugin.obj
 0002:0000fdac       __ehfuncinfo$?checkoutFile@testPlugin@@AAEXXZ 1002fdac     testPlugin.obj
 0002:0000fdd0       __ehfuncinfo$??0testPluginFromBase@@QAE@ABVQString@@00@Z 1002fdd0     testPluginFromBase.obj
 0002:0000fdf4       __unwindtable$??0testPluginFromBase@@QAE@ABVQString@@00@Z 1002fdf4     testPluginFromBase.obj
 0002:0001000c       __unwindtable$?loadFile@testPluginFromBase@@MAEXVQString@@@Z 1003000c     testPluginFromBase.obj
 0002:0001000c       __unwindtable$?saveFile@testPluginFromBase@@MAEXVQString@@@Z 1003000c     testPluginFromBase.obj
 0002:0001001c       __ehfuncinfo$?loadFile@testPluginFromBase@@MAEXVQString@@@Z 1003001c     testPluginFromBase.obj
 0002:0001001c       __ehfuncinfo$?saveFile@testPluginFromBase@@MAEXVQString@@@Z 1003001c     testPluginFromBase.obj
 0002:00010040       __unwindtable$?init@testPluginFromBase@@MAEXXZ 10030040     testPluginFromBase.obj
 0002:00010040       __unwindtable$?clipBoardDataChanged@cfg_Table@@IAEXXZ 10030040     testPluginFromBase.obj
 0002:00010048       __ehfuncinfo$?init@testPluginFromBase@@MAEXXZ 10030048     testPluginFromBase.obj
 0002:00010048       __ehfuncinfo$?clipBoardDataChanged@cfg_Table@@IAEXXZ 10030048     testPluginFromBase.obj
 0002:0001006c       __ehfuncinfo$?lockFileS@testPluginFromBase@@AAEXXZ 1003006c     testPluginFromBase.obj
 0002:0001006c       __ehfuncinfo$?checkoutFileS@testPluginFromBase@@AAEXXZ 1003006c     testPluginFromBase.obj
 0002:0001006c       __ehfuncinfo$?downloadDirS@testPluginFromBase@@AAEXXZ 1003006c     testPluginFromBase.obj
 0002:0001006c       __ehfuncinfo$?uploadFileS@testPluginFromBase@@AAEXXZ 1003006c     testPluginFromBase.obj
 0002:0001006c       __ehfuncinfo$?unlockDirS@testPluginFromBase@@AAEXXZ 1003006c     testPluginFromBase.obj
 0002:0001006c       __ehfuncinfo$?uploadDirS@testPluginFromBase@@AAEXXZ 1003006c     testPluginFromBase.obj
 0002:0001006c       __ehfuncinfo$?unlockFileS@testPluginFromBase@@AAEXXZ 1003006c     testPluginFromBase.obj
 0002:0001006c       __ehfuncinfo$?checkoutDirS@testPluginFromBase@@AAEXXZ 1003006c     testPluginFromBase.obj
 0002:0001006c       __ehfuncinfo$?downloadFileS@testPluginFromBase@@AAEXXZ 1003006c     testPluginFromBase.obj
 0002:00010090       __unwindtable$?uploadDirS@testPluginFromBase@@AAEXXZ 10030090     testPluginFromBase.obj
 0002:00010090       __unwindtable$?checkoutFileS@testPluginFromBase@@AAEXXZ 10030090     testPluginFromBase.obj
 0002:00010090       __unwindtable$?uploadFileS@testPluginFromBase@@AAEXXZ 10030090     testPluginFromBase.obj
 0002:00010090       __unwindtable$?downloadFileS@testPluginFromBase@@AAEXXZ 10030090     testPluginFromBase.obj
 0002:00010090       __unwindtable$?unlockFileS@testPluginFromBase@@AAEXXZ 10030090     testPluginFromBase.obj
 0002:00010090       __unwindtable$?lockFileS@testPluginFromBase@@AAEXXZ 10030090     testPluginFromBase.obj
 0002:00010090       __unwindtable$?checkoutDirS@testPluginFromBase@@AAEXXZ 10030090     testPluginFromBase.obj
 0002:00010090       __unwindtable$?downloadDirS@testPluginFromBase@@AAEXXZ 10030090     testPluginFromBase.obj
 0002:00010090       __unwindtable$?unlockDirS@testPluginFromBase@@AAEXXZ 10030090     testPluginFromBase.obj
 0002:000100c0       __ehfuncinfo$?dirS@testPluginFromBase@@AAEXXZ 100300c0     testPluginFromBase.obj
 0002:000100e4       __unwindtable$?dirS@testPluginFromBase@@AAEXXZ 100300e4     testPluginFromBase.obj
 0002:0001011c       __unwindtable$?doDirtyS@testPluginFromBase@@AAEXXZ 1003011c     testPluginFromBase.obj
 0002:0001011c       __unwindtable$?doCleanS@testPluginFromBase@@AAEXXZ 1003011c     testPluginFromBase.obj
 0002:0001012c       __ehfuncinfo$?doCleanS@testPluginFromBase@@AAEXXZ 1003012c     testPluginFromBase.obj
 0002:0001012c       __ehfuncinfo$?doDirtyS@testPluginFromBase@@AAEXXZ 1003012c     testPluginFromBase.obj
 0002:00010150       __ehfuncinfo$??0workstationCustomTable@@QAE@PAVQWidget@@PBD@Z 10030150     workstationCustomTable.obj
 0002:00010174       __unwindtable$??0workstationCustomTable@@QAE@PAVQWidget@@PBD@Z 10030174     workstationCustomTable.obj
 0002:0001019c       __ehfuncinfo$??0workstationDockWindow@@QAE@PAVQWidget@@PBDI@Z 1003019c     workstationdockwindowimpl.obj
 0002:000101c0       __unwindtable$??0workstationDockWindow@@QAE@PAVQWidget@@PBDI@Z 100301c0     workstationdockwindowimpl.obj
 0002:000101f8       __ehfuncinfo$??0workstationEditor@@QAE@ABVQString@@00@Z 100301f8     workstationEditor.obj
 0002:0001021c       __unwindtable$??0workstationEditor@@QAE@ABVQString@@00@Z 1003021c     workstationEditor.obj
 0002:00010344       __ehfuncinfo$??1workstationEditor@@UAE@XZ 10030344     workstationEditor.obj
 0002:00010368       __unwindtable$??1workstationEditor@@UAE@XZ 10030368     workstationEditor.obj
 0002:00010398       __ehfuncinfo$?reply@workstationEditor@@UAEXPAVresponse@@@Z 10030398     workstationEditor.obj
 0002:000103bc       __unwindtable$?reply@workstationEditor@@UAEXPAVresponse@@@Z 100303bc     workstationEditor.obj
 0002:0001042c       __ehfuncinfo$?activate@workstationEditor@@UAEX_N@Z 1003042c     workstationEditor.obj
 0002:00010450       __unwindtable$?activate@workstationEditor@@UAEX_N@Z 10030450     workstationEditor.obj
 0002:00010480       __unwindtable$?closeEvent@workstationEditor@@UAEXPAVQCloseEvent@@@Z 10030480     workstationEditor.obj
 0002:00010490       __ehfuncinfo$?closeEvent@workstationEditor@@UAEXPAVQCloseEvent@@@Z 10030490     workstationEditor.obj
 0002:000104b4       __unwindtable$?apply@workstationEditor@@UAEXXZ 100304b4     workstationEditor.obj
 0002:000104cc       __ehfuncinfo$?apply@workstationEditor@@UAEXXZ 100304cc     workstationEditor.obj
 0002:000104f0       __ehfuncinfo$??0workstationEditorDlg@@QAE@ABVQString@@PAVQWidget@@PBDI@Z 100304f0     workstationeditordlgimpl.obj
 0002:00010514       __unwindtable$??0workstationEditorDlg@@QAE@ABVQString@@PAVQWidget@@PBDI@Z 10030514     workstationeditordlgimpl.obj
 0002:00010544       __unwindtable$??1workstationEditorDlg@@UAE@XZ 10030544     workstationeditordlgimpl.obj
 0002:0001054c       __ehfuncinfo$??1workstationEditorDlg@@UAE@XZ 1003054c     workstationeditordlgimpl.obj
 0002:00010570       __ehfuncinfo$?save@workstationEditorDlg@@QAEXXZ 10030570     workstationeditordlgimpl.obj
 0002:00010594       __unwindtable$?save@workstationEditorDlg@@QAEXXZ 10030594     workstationeditordlgimpl.obj
 0002:00010604       __ehfuncinfo$?load@workstationEditorDlg@@QAE_NABVQString@@@Z 10030604     workstationeditordlgimpl.obj
 0002:00010628       __unwindtable$?load@workstationEditorDlg@@QAE_NABVQString@@@Z 10030628     workstationeditordlgimpl.obj
 0002:000106c8       __ehfuncinfo$?newBNCSSystemIni@workstationEditorDlg@@AAEXH_N0@Z 100306c8     workstationeditordlgimpl.obj
 0002:000106ec       __unwindtable$?newBNCSSystemIni@workstationEditorDlg@@AAEXH_N0@Z 100306ec     workstationeditordlgimpl.obj
 0002:00010744       __ehfuncinfo$?doAdd@workstationEditorDlg@@AAEXXZ 10030744     workstationeditordlgimpl.obj
 0002:00010768       __unwindtable$?doAdd@workstationEditorDlg@@AAEXXZ 10030768     workstationeditordlgimpl.obj
 0002:000107e0       __ehfuncinfo$?toXML@@YA?AVQString@@ABV1@@Z 100307e0     workstationeditordlgimpl.obj
 0002:00010804       __unwindtable$?toXML@@YA?AVQString@@ABV1@@Z 10030804     workstationeditordlgimpl.obj
 0002:0001085c       __unwindtable$??0workstationEditorNewWsDlg@@QAE@ABVQString@@PAVQWidget@@PBD_NI@Z 1003085c     workstationeditornewwsdlgimpl.obj
 0002:00010874       __ehfuncinfo$??0workstationEditorNewWsDlg@@QAE@ABVQString@@PAVQWidget@@PBD_NI@Z 10030874     workstationeditornewwsdlgimpl.obj
 0002:00010898       __unwindtable$??1workstationEditorNewWsDlg@@UAE@XZ 10030898     workstationeditornewwsdlgimpl.obj
 0002:000108a8       __ehfuncinfo$??1workstationEditorNewWsDlg@@UAE@XZ 100308a8     workstationeditornewwsdlgimpl.obj
 0002:000108cc       __ehfuncinfo$?accept@workstationEditorNewWsDlg@@UAEXXZ 100308cc     workstationeditornewwsdlgimpl.obj
 0002:000108f0       __unwindtable$?accept@workstationEditorNewWsDlg@@UAEXXZ 100308f0     workstationeditornewwsdlgimpl.obj
 0002:00010918       __ehfuncinfo$?loadUsers@workstationEditorNewWsDlg@@AAEXXZ 10030918     workstationeditornewwsdlgimpl.obj
 0002:0001093c       __unwindtable$?loadUsers@workstationEditorNewWsDlg@@AAEXXZ 1003093c     workstationeditornewwsdlgimpl.obj
 0002:0001099c       __unwindtable$??0workstationUserTableItem@@QAE@ABVQString@@PAVQTable@@W4EditType@QTableItem@@0@Z 1003099c     workstationUserTableItem.obj
 0002:000109ac       __ehfuncinfo$??0workstationUserTableItem@@QAE@ABVQString@@PAVQTable@@W4EditType@QTableItem@@0@Z 100309ac     workstationUserTableItem.obj
 0002:000109d0       __unwindtable$??1workstationUserTableItem@@UAE@XZ 100309d0     workstationUserTableItem.obj
 0002:000109d8       __ehfuncinfo$??1workstationUserTableItem@@UAE@XZ 100309d8     workstationUserTableItem.obj
 0002:000109fc       __ehfuncinfo$?createEditor@workstationUserTableItem@@UBEPAVQWidget@@XZ 100309fc     workstationUserTableItem.obj
 0002:00010a20       __unwindtable$?createEditor@workstationUserTableItem@@UBEPAVQWidget@@XZ 10030a20     workstationUserTableItem.obj
 0002:00010a98       __unwindtable$?navigate@testPlugin@@UAEXABVQString@@0@Z 10030a98     workstationUserTableItem.obj
 0002:00010a98       __unwindtable$?setContentFromEditor@workstationUserTableItem@@UAEXPAVQWidget@@@Z 10030a98     workstationUserTableItem.obj
 0002:00010aa0       __ehfuncinfo$?setContentFromEditor@workstationUserTableItem@@UAEXPAVQWidget@@@Z 10030aa0     workstationUserTableItem.obj
 0002:00010aa0       __ehfuncinfo$?navigate@testPlugin@@UAEXABVQString@@0@Z 10030aa0     workstationUserTableItem.obj
 0002:00010ac4       __ehfuncinfo$?createDirectory@xfer@@QAEXAAVQString@@@Z 10030ac4     xfer.obj
 0002:00010ae8       __unwindtable$?createDirectory@xfer@@QAEXAAVQString@@@Z 10030ae8     xfer.obj
 0002:00010b28       __unwindtable$?setFileDate@xfer@@QAE_NABVQString@@AAVQDateTime@@@Z 10030b28     xfer.obj
 0002:00010b40       __ehfuncinfo$?setFileDate@xfer@@QAE_NABVQString@@AAVQDateTime@@@Z 10030b40     xfer.obj
 0002:00010b64       __unwindtable$??0xml_listview@@QAE@PAVQWidget@@PBDI@Z 10030b64     xml_listview.obj
 0002:00010b74       __ehfuncinfo$??0xml_listview@@QAE@PAVQWidget@@PBDI@Z 10030b74     xml_listview.obj
 0002:00010b98       __ehfuncinfo$?load@xml_listview@@QAEXABVQString@@@Z 10030b98     xml_listview.obj
 0002:00010bbc       __unwindtable$?load@xml_listview@@QAEXABVQString@@@Z 10030bbc     xml_listview.obj
 0002:00010f54       __ehfuncinfo$??0dialogBase@@QAE@PAVQWidget@@PBDI@Z 10030f54     dialog.obj
 0002:00010f78       __unwindtable$??0dialogBase@@QAE@PAVQWidget@@PBDI@Z 10030f78     dialog.obj
 0002:00011120       __ehfuncinfo$?languageChange@dialogBase@@MAEXXZ 10031120     dialog.obj
 0002:00011144       __unwindtable$?languageChange@dialogBase@@MAEXXZ 10031144     dialog.obj
 0002:000111fc       __ehfuncinfo$??0launchEditorDlgBase@@QAE@PAVQWidget@@PBDI@Z 100311fc     launcheditordlg.obj
 0002:00011220       __unwindtable$??0launchEditorDlgBase@@QAE@PAVQWidget@@PBDI@Z 10031220     launcheditordlg.obj
 0002:00011328       __ehfuncinfo$?languageChange@launchEditorDlgBase@@MAEXXZ 10031328     launcheditordlg.obj
 0002:0001134c       __unwindtable$?languageChange@launchEditorDlgBase@@MAEXXZ 1003134c     launcheditordlg.obj
 0002:00011484       __unwindtable$?fileList@fileDrop@@IAEXVQStringList@@@Z 10031484     moc_fileDrop.obj
 0002:00011494       __ehfuncinfo$?fileList@fileDrop@@IAEXVQStringList@@@Z 10031494     moc_fileDrop.obj
 0002:000114b8       __unwindtable$?command@testPlugin@@IAEXVQString@@0@Z 100314b8     moc_launcheditordlgimpl.obj
 0002:000114b8       __unwindtable$?command@workstationEditorDlg@@IAEXVQString@@0@Z 100314b8     moc_launcheditordlgimpl.obj
 0002:000114b8       __unwindtable$?command@launchEditorDlg@@IAEXVQString@@0@Z 100314b8     moc_launcheditordlgimpl.obj
 0002:000114b8       __unwindtable$?command@launchEditor@@IAEXVQString@@0@Z 100314b8     moc_launcheditordlgimpl.obj
 0002:000114b8       __unwindtable$?command@workstationEditor@@IAEXVQString@@0@Z 100314b8     moc_launcheditordlgimpl.obj
 0002:000114b8       __unwindtable$?command@fileManager@@IAEXVQString@@0@Z 100314b8     moc_launcheditordlgimpl.obj
 0002:000114d0       __ehfuncinfo$?command@fileManager@@IAEXVQString@@0@Z 100314d0     moc_launcheditordlgimpl.obj
 0002:000114d0       __ehfuncinfo$?command@launchEditorDlg@@IAEXVQString@@0@Z 100314d0     moc_launcheditordlgimpl.obj
 0002:000114d0       __ehfuncinfo$?command@workstationEditorDlg@@IAEXVQString@@0@Z 100314d0     moc_launcheditordlgimpl.obj
 0002:000114d0       __ehfuncinfo$?command@testPlugin@@IAEXVQString@@0@Z 100314d0     moc_launcheditordlgimpl.obj
 0002:000114d0       __ehfuncinfo$?command@launchEditor@@IAEXVQString@@0@Z 100314d0     moc_launcheditordlgimpl.obj
 0002:000114d0       __ehfuncinfo$?command@workstationEditor@@IAEXVQString@@0@Z 100314d0     moc_launcheditordlgimpl.obj
 0002:000114f4       __unwindtable$?selectionChanged@workstationDockWindow@@IAEXPAVQListViewItem@@@Z 100314f4     moc_workstationdockwindowimpl.obj
 0002:000114f4       __unwindtable$?startDrag@xml_listview@@IAEXPAVQListViewItem@@@Z 100314f4     moc_workstationdockwindowimpl.obj
 0002:000114fc       __ehfuncinfo$?selectionChanged@workstationDockWindow@@IAEXPAVQListViewItem@@@Z 100314fc     moc_workstationdockwindowimpl.obj
 0002:000114fc       __ehfuncinfo$?startDrag@xml_listview@@IAEXPAVQListViewItem@@@Z 100314fc     moc_workstationdockwindowimpl.obj
 0002:00011520       __unwindtable$?qt_emit@launchEditorDlg@@UAE_NHPAUQUObject@@@Z 10031520     moc_workstationeditordlgimpl.obj
 0002:00011520       __unwindtable$?qt_emit@fileManager@@UAE_NHPAUQUObject@@@Z 10031520     moc_workstationeditordlgimpl.obj
 0002:00011520       __unwindtable$?qt_emit@launchEditor@@UAE_NHPAUQUObject@@@Z 10031520     moc_workstationeditordlgimpl.obj
 0002:00011520       __unwindtable$?qt_emit@workstationEditor@@UAE_NHPAUQUObject@@@Z 10031520     moc_workstationeditordlgimpl.obj
 0002:00011520       __unwindtable$?qt_emit@workstationEditorDlg@@UAE_NHPAUQUObject@@@Z 10031520     moc_workstationeditordlgimpl.obj
 0002:00011520       __unwindtable$?qt_emit@testPlugin@@UAE_NHPAUQUObject@@@Z 10031520     moc_workstationeditordlgimpl.obj
 0002:00011528       __ehfuncinfo$?qt_emit@launchEditor@@UAE_NHPAUQUObject@@@Z 10031528     moc_workstationeditordlgimpl.obj
 0002:00011528       __ehfuncinfo$?qt_emit@testPlugin@@UAE_NHPAUQUObject@@@Z 10031528     moc_workstationeditordlgimpl.obj
 0002:00011528       __ehfuncinfo$?qt_emit@workstationEditorDlg@@UAE_NHPAUQUObject@@@Z 10031528     moc_workstationeditordlgimpl.obj
 0002:00011528       __ehfuncinfo$?qt_emit@workstationEditor@@UAE_NHPAUQUObject@@@Z 10031528     moc_workstationeditordlgimpl.obj
 0002:00011528       __ehfuncinfo$?qt_emit@launchEditorDlg@@UAE_NHPAUQUObject@@@Z 10031528     moc_workstationeditordlgimpl.obj
 0002:00011528       __ehfuncinfo$?qt_emit@fileManager@@UAE_NHPAUQUObject@@@Z 10031528     moc_workstationeditordlgimpl.obj
 0002:0001154c       __ehfuncinfo$??0workstationDockWindowBase@@QAE@PAVQWidget@@PBDI@Z 1003154c     workstationdockwindow.obj
 0002:00011570       __unwindtable$??0workstationDockWindowBase@@QAE@PAVQWidget@@PBDI@Z 10031570     workstationdockwindow.obj
 0002:000115b0       __unwindtable$??1workstationEditorDlgBase@@UAE@XZ 100315b0     workstationdockwindow.obj
 0002:000115b0       __unwindtable$??1launchEditorDlgBase@@UAE@XZ 100315b0     workstationdockwindow.obj
 0002:000115b0       __unwindtable$??1workstationDockWindowBase@@UAE@XZ 100315b0     workstationdockwindow.obj
 0002:000115b8       __ehfuncinfo$??1workstationEditorDlgBase@@UAE@XZ 100315b8     workstationdockwindow.obj
 0002:000115b8       __ehfuncinfo$??1launchEditorDlgBase@@UAE@XZ 100315b8     workstationdockwindow.obj
 0002:000115b8       __ehfuncinfo$??1workstationDockWindowBase@@UAE@XZ 100315b8     workstationdockwindow.obj
 0002:000115dc       __unwindtable$?languageChange@workstationDockWindowBase@@MAEXXZ 100315dc     workstationdockwindow.obj
 0002:000115ec       __ehfuncinfo$?languageChange@workstationDockWindowBase@@MAEXXZ 100315ec     workstationdockwindow.obj
 0002:00011610       __ehfuncinfo$??0workstationEditorDlgBase@@QAE@PAVQWidget@@PBDI@Z 10031610     workstationeditordlg.obj
 0002:00011634       __unwindtable$??0workstationEditorDlgBase@@QAE@PAVQWidget@@PBDI@Z 10031634     workstationeditordlg.obj
 0002:00011684       __ehfuncinfo$?languageChange@workstationEditorDlgBase@@MAEXXZ 10031684     workstationeditordlg.obj
 0002:000116a8       __unwindtable$?languageChange@workstationEditorDlgBase@@MAEXXZ 100316a8     workstationeditordlg.obj
 0002:000116e8       __ehfuncinfo$??0workstationEditorNewWsDlgBase@@QAE@PAVQWidget@@PBD_NI@Z 100316e8     workstationeditornewwsdlg.obj
 0002:0001170c       __unwindtable$??0workstationEditorNewWsDlgBase@@QAE@PAVQWidget@@PBD_NI@Z 1003170c     workstationeditornewwsdlg.obj
 0002:000117dc       __ehfuncinfo$?languageChange@workstationEditorNewWsDlgBase@@MAEXXZ 100317dc     workstationeditornewwsdlg.obj
 0002:00011800       __unwindtable$?languageChange@workstationEditorNewWsDlgBase@@MAEXXZ 10031800     workstationeditornewwsdlg.obj
 0002:00011858       __unwindtable$??0cfg_Table@@QAE@PAVQWidget@@PBD@Z 10031858     cfg_widgets001:cfg_Table.obj
 0002:00011860       __ehfuncinfo$??0cfg_Table@@QAE@PAVQWidget@@PBD@Z 10031860     cfg_widgets001:cfg_Table.obj
 0002:00011884       __unwindtable$?deleteItems@cfg_Table@@QAEXXZ 10031884     cfg_widgets001:cfg_Table.obj
 0002:0001188c       __ehfuncinfo$?deleteItems@cfg_Table@@QAEXXZ 1003188c     cfg_widgets001:cfg_Table.obj
 0002:000118b0       __unwindtable$?copyToClipboard@cfg_Table@@QAEXXZ 100318b0     cfg_widgets001:cfg_Table.obj
 0002:000118c8       __ehfuncinfo$?copyToClipboard@cfg_Table@@QAEXXZ 100318c8     cfg_widgets001:cfg_Table.obj
 0002:000118ec       __unwindtable$?undoPaste@cfg_Table@@QAEXXZ 100318ec     cfg_widgets001:cfg_Table.obj
 0002:00011904       __ehfuncinfo$?undoPaste@cfg_Table@@QAEXXZ 10031904     cfg_widgets001:cfg_Table.obj
 0002:00011928       __ehfuncinfo$?pasteClipboard@cfg_Table@@QAEXXZ 10031928     cfg_widgets001:cfg_Table.obj
 0002:0001194c       __unwindtable$?pasteClipboard@cfg_Table@@QAEXXZ 1003194c     cfg_widgets001:cfg_Table.obj
 0002:000119bc       __unwindtable$?fillUndoBuffer@cfg_Table@@AAEXXZ 100319bc     cfg_widgets001:cfg_Table.obj
 0002:000119dc       __ehfuncinfo$?fillUndoBuffer@cfg_Table@@AAEXXZ 100319dc     cfg_widgets001:cfg_Table.obj
 0002:00011a00       __ehfuncinfo$??0configFile@@QAE@PAVpluginBase@@VQString@@_N@Z 10031a00     pluginBase:configFile.obj
 0002:00011a24       __unwindtable$??0configFile@@QAE@PAVpluginBase@@VQString@@_N@Z 10031a24     pluginBase:configFile.obj
 0002:00011a4c       __unwindtable$??_GconfigFile@@UAEPAXI@Z 10031a4c     pluginBase:configFile.obj
 0002:00011a4c       __unwindtable$??1configFile@@UAE@XZ 10031a4c     pluginBase:configFile.obj
 0002:00011a64       __ehfuncinfo$??_GconfigFile@@UAEPAXI@Z 10031a64     pluginBase:configFile.obj
 0002:00011a64       __ehfuncinfo$??1configFile@@UAE@XZ 10031a64     pluginBase:configFile.obj
 0002:00011a88       __unwindtable$??BconfigFile@@QAE?AVQFileInfo@@XZ 10031a88     pluginBase:configFile.obj
 0002:00011a98       __ehfuncinfo$??BconfigFile@@QAE?AVQFileInfo@@XZ 10031a98     pluginBase:configFile.obj
 0002:00011abc       __unwindtable$?getLocalPath@configFile@@QAE?AVQString@@XZ 10031abc     pluginBase:configFile.obj
 0002:00011adc       __ehfuncinfo$?getLocalPath@configFile@@QAE?AVQString@@XZ 10031adc     pluginBase:configFile.obj
 0002:00011b00       __unwindtable$?unlock@configFile@@QAE_N_N@Z 10031b00     pluginBase:configFile.obj
 0002:00011b10       __ehfuncinfo$?unlock@configFile@@QAE_N_N@Z 10031b10     pluginBase:configFile.obj
 0002:00011b34       __ehfuncinfo$?dirList@configFile@@QAE_NAAVQStringList@@@Z 10031b34     pluginBase:configFile.obj
 0002:00011b58       __unwindtable$?dirList@configFile@@QAE_NAAVQStringList@@@Z 10031b58     pluginBase:configFile.obj
 0002:00011bb8       __unwindtable$?setDirty@configFile@@QAE_NXZ 10031bb8     pluginBase:configFile.obj
 0002:00011bc8       __ehfuncinfo$?setDirty@configFile@@QAE_NXZ 10031bc8     pluginBase:configFile.obj
 0002:00011bec       __unwindtable$?getModTime@configFile@@QAE?AVQDateTime@@XZ 10031bec     pluginBase:configFile.obj
 0002:00011c04       __ehfuncinfo$?getModTime@configFile@@QAE?AVQDateTime@@XZ 10031c04     pluginBase:configFile.obj
 0002:00011c28       __unwindtable$?sendCommand@configFile@@IAEXVQString@@@Z 10031c28     pluginBase:configFile.obj
 0002:00011c38       __ehfuncinfo$?sendCommand@configFile@@IAEXVQString@@@Z 10031c38     pluginBase:configFile.obj
 0002:00011c5c       __unwindtable$?timerEvent@configFile@@MAEXPAVQTimerEvent@@@Z 10031c5c     pluginBase:configFile.obj
 0002:00011c64       __ehfuncinfo$?timerEvent@configFile@@MAEXPAVQTimerEvent@@@Z 10031c64     pluginBase:configFile.obj
 0002:00011c88       __unwindtable$?reply@configFile@@MAEXPAVresponse@@@Z 10031c88     pluginBase:configFile.obj
 0002:00011c90       __ehfuncinfo$?reply@configFile@@MAEXPAVresponse@@@Z 10031c90     pluginBase:configFile.obj
 0002:00011cb4       __unwindtable$??0pluginBase@@QAE@ABVQString@@00@Z 10031cb4     pluginBase:pluginBase.obj
 0002:00011cd4       __ehfuncinfo$??0pluginBase@@QAE@ABVQString@@00@Z 10031cd4     pluginBase:pluginBase.obj
 0002:00011cf8       __ehfuncinfo$??1pluginBase@@UAE@XZ 10031cf8     pluginBase:pluginBase.obj
 0002:00011d1c       __unwindtable$??1pluginBase@@UAE@XZ 10031d1c     pluginBase:pluginBase.obj
 0002:00011d94       __ehfuncinfo$?file@pluginBase@@QAEAAVconfigFile@@VQString@@@Z 10031d94     pluginBase:pluginBase.obj
 0002:00011db8       __unwindtable$?file@pluginBase@@QAEAAVconfigFile@@VQString@@@Z 10031db8     pluginBase:pluginBase.obj
 0002:00011de0       __unwindtable$?uploadAllFiles@pluginBase@@AAEXXZ 10031de0     pluginBase:pluginBase.obj
 0002:00011de0       __unwindtable$?releaseAllLocks@pluginBase@@AAEXXZ 10031de0     pluginBase:pluginBase.obj
 0002:00011de0       __unwindtable$?isDirty@pluginBase@@EAE_NXZ 10031de0     pluginBase:pluginBase.obj
 0002:00011df0       __ehfuncinfo$?releaseAllLocks@pluginBase@@AAEXXZ 10031df0     pluginBase:pluginBase.obj
 0002:00011df0       __ehfuncinfo$?uploadAllFiles@pluginBase@@AAEXXZ 10031df0     pluginBase:pluginBase.obj
 0002:00011df0       __ehfuncinfo$?isDirty@pluginBase@@EAE_NXZ 10031df0     pluginBase:pluginBase.obj
 0002:00011e14       __unwindtable$?sendCommand@pluginBase@@AAEXVQString@@0@Z 10031e14     pluginBase:pluginBase.obj
 0002:00011e2c       __ehfuncinfo$?sendCommand@pluginBase@@AAEXVQString@@0@Z 10031e2c     pluginBase:pluginBase.obj
 0002:00011e50       __unwindtable$?waitForAllFiles@pluginBase@@QAE_NXZ 10031e50     pluginBase:pluginBase.obj
 0002:00011e50       __unwindtable$?saveAllFiles@pluginBase@@AAEXXZ 10031e50     pluginBase:pluginBase.obj
 0002:00011e50       __unwindtable$?loadModdedFiles@pluginBase@@AAEXXZ 10031e50     pluginBase:pluginBase.obj
 0002:00011e60       __ehfuncinfo$?waitForAllFiles@pluginBase@@QAE_NXZ 10031e60     pluginBase:pluginBase.obj
 0002:00011e60       __ehfuncinfo$?saveAllFiles@pluginBase@@AAEXXZ 10031e60     pluginBase:pluginBase.obj
 0002:00011e60       __ehfuncinfo$?loadModdedFiles@pluginBase@@AAEXXZ 10031e60     pluginBase:pluginBase.obj
 0002:00011e84       __ehfuncinfo$??A?$QMap@VQString@@VconfigFile@@@@QAEAAVconfigFile@@ABVQString@@@Z 10031e84     pluginBase:pluginBase.obj
 0002:00011ea8       __unwindtable$??A?$QMap@VQString@@VconfigFile@@@@QAEAAVconfigFile@@ABVQString@@@Z 10031ea8     pluginBase:pluginBase.obj
 0002:00011ed0       __unwindtable$?insert@?$QMap@VQString@@VconfigFile@@@@QAE?AV?$QMapIterator@VQString@@VconfigFile@@@@ABVQString@@ABVconfigFile@@_N@Z 10031ed0     pluginBase:pluginBase.obj
 0002:00011ed8       __ehfuncinfo$?insert@?$QMap@VQString@@VconfigFile@@@@QAE?AV?$QMapIterator@VQString@@VconfigFile@@@@ABVQString@@ABVconfigFile@@_N@Z 10031ed8     pluginBase:pluginBase.obj
 0002:00011efc       __unwindtable$??0?$QMapPrivate@VQString@@VconfigFile@@@@QAE@XZ 10031efc     pluginBase:pluginBase.obj
 0002:00011f0c       __ehfuncinfo$??0?$QMapPrivate@VQString@@VconfigFile@@@@QAE@XZ 10031f0c     pluginBase:pluginBase.obj
 0002:00011f30       __unwindtable$??0?$QMapPrivate@VQString@@VconfigFile@@@@QAE@PBV0@@Z 10031f30     pluginBase:pluginBase.obj
 0002:00011f40       __ehfuncinfo$??0?$QMapPrivate@VQString@@VconfigFile@@@@QAE@PBV0@@Z 10031f40     pluginBase:pluginBase.obj
 0002:00011f64       __unwindtable$?copy@?$QMapPrivate@VQString@@VconfigFile@@@@QAEPAU?$QMapNode@VQString@@VconfigFile@@@@PAU2@@Z 10031f64     pluginBase:pluginBase.obj
 0002:00011f6c       __ehfuncinfo$?copy@?$QMapPrivate@VQString@@VconfigFile@@@@QAEPAU?$QMapNode@VQString@@VconfigFile@@@@PAU2@@Z 10031f6c     pluginBase:pluginBase.obj
 0002:00011f90       __unwindtable$?clear@?$QMapPrivate@VQString@@VconfigFile@@@@QAEXPAU?$QMapNode@VQString@@VconfigFile@@@@@Z 10031f90     pluginBase:pluginBase.obj
 0002:00011fb0       __ehfuncinfo$?clear@?$QMapPrivate@VQString@@VconfigFile@@@@QAEXPAU?$QMapNode@VQString@@VconfigFile@@@@@Z 10031fb0     pluginBase:pluginBase.obj
 0002:00011fd4       __unwindtable$?insert@?$QMapPrivate@VQString@@VconfigFile@@@@QAE?AV?$QMapIterator@VQString@@VconfigFile@@@@PAUQMapNodeBase@@0ABVQString@@@Z 10031fd4     pluginBase:pluginBase.obj
 0002:00011fec       __ehfuncinfo$?insert@?$QMapPrivate@VQString@@VconfigFile@@@@QAE?AV?$QMapIterator@VQString@@VconfigFile@@@@PAUQMapNodeBase@@0ABVQString@@@Z 10031fec     pluginBase:pluginBase.obj
 0002:00012010       __unwindtable$??0?$QMapNode@VQString@@VconfigFile@@@@QAE@ABU0@@Z 10032010     pluginBase:pluginBase.obj
 0002:00012020       __ehfuncinfo$??0?$QMapNode@VQString@@VconfigFile@@@@QAE@ABU0@@Z 10032020     pluginBase:pluginBase.obj
 0002:00012044       __unwindtable$??1?$QMapNode@VQString@@VconfigFile@@@@QAE@XZ 10032044     pluginBase:pluginBase.obj
 0002:00012064       __ehfuncinfo$??1?$QMapNode@VQString@@VconfigFile@@@@QAE@XZ 10032064     pluginBase:pluginBase.obj
 0002:00012088       __unwindtable$?qt_emit@pluginBase@@UAE_NHPAUQUObject@@@Z 10032088     pluginBase:moc_pluginBase.obj
 0002:00012090       __ehfuncinfo$?qt_emit@pluginBase@@UAE_NHPAUQUObject@@@Z 10032090     pluginBase:moc_pluginBase.obj
 0002:000120b4       __unwindtable$?command@pluginBase@@IAEXVQString@@0@Z 100320b4     pluginBase:moc_pluginBase.obj
 0002:000120cc       __ehfuncinfo$?command@pluginBase@@IAEXVQString@@0@Z 100320cc     pluginBase:moc_pluginBase.obj
 0002:000120f0       __sehtable$__onexit        100320f0     MSVCRT:atonexit.obj
 0002:00012110       __sehtable$??_L@YGXPAXIHP6EX0@Z1@Z 10032110     MSVCRT:ehvecctr.obj
 0002:00012130       __sehtable$??_M@YGXPAXIHP6EX0@Z@Z 10032130     MSVCRT:ehvecdtr.obj
 0002:00012150       __sehtable$?__ArrayUnwind@@YGXPAXIHP6EX0@Z@Z 10032150     MSVCRT:ehvecdtr.obj
 0002:00012170       __sehtable$___DllMainCRTStartup 10032170     MSVCRT:crtdll.obj
 0002:00012198       __sehtable$__IsNonwritableInCurrentImage 10032198     MSVCRT:pesect.obj
 0002:000121c0       .edata                     100321c0     testPlugin.exp
 0002:000121e8       rgpv                       100321e8     testPlugin.exp
 0002:0001225c       rgszName                   1003225c     testPlugin.exp
 0002:000122d0       rgwOrd                     100322d0     testPlugin.exp
 0002:0001230a       szName                     1003230a     testPlugin.exp
 0002:00012319       $N00001                    10032319     testPlugin.exp
 0002:00012333       $N00002                    10032333     testPlugin.exp
 0002:00012357       $N00003                    10032357     testPlugin.exp
 0002:0001236c       $N00004                    1003236c     testPlugin.exp
 0002:0001238a       $N00005                    1003238a     testPlugin.exp
 0002:000123a6       $N00006                    100323a6     testPlugin.exp
 0002:000123c7       $N00007                    100323c7     testPlugin.exp
 0002:000123dd       $N00008                    100323dd     testPlugin.exp
 0002:000123fc       $N00009                    100323fc     testPlugin.exp
 0002:00012424       $N00010                    10032424     testPlugin.exp
 0002:0001244c       $N00011                    1003244c     testPlugin.exp
 0002:0001246f       $N00012                    1003246f     testPlugin.exp
 0002:0001248d       $N00013                    1003248d     testPlugin.exp
 0002:000124ac       $N00014                    100324ac     testPlugin.exp
 0002:000124ce       $N00015                    100324ce     testPlugin.exp
 0002:000124f5       $N00016                    100324f5     testPlugin.exp
 0002:00012522       $N00017                    10032522     testPlugin.exp
 0002:00012544       $N00018                    10032544     testPlugin.exp
 0002:0001256a       $N00019                    1003256a     testPlugin.exp
 0002:0001258a       $N00020                    1003258a     testPlugin.exp
 0002:000125b4       $N00021                    100325b4     testPlugin.exp
 0002:000125e0       $N00022                    100325e0     testPlugin.exp
 0002:0001260f       $N00023                    1003260f     testPlugin.exp
 0002:00012650       $N00024                    10032650     testPlugin.exp
 0002:00012682       $N00025                    10032682     testPlugin.exp
 0002:000126a6       $N00026                    100326a6     testPlugin.exp
 0002:000126ce       $N00027                    100326ce     testPlugin.exp
 0002:000126eb       $N00028                    100326eb     testPlugin.exp
 0002:0001270b       $N00029                    1003270b     testPlugin.exp
 0002:00013a4c       .idata$6                   10033a4c     config_icons:config_icons.dll
 0002:0001f582       .idata$6                   1003f582     qt-mt323:qt-mt323.dll
 0002:0001f60a       .idata$6                   1003f60a     kernel32:KERNEL32.dll
 0002:0001f664       .idata$6                   1003f664     MSVCRT:MSVCR120.dll
 0003:00000000       _folder                    10040000     fileManager.obj
 0003:00000058       _filesave                  10040058     fileManager.obj
 0003:000000a8       _copy                      100400a8     fileManager.obj
 0003:00000100       _paste                     10040100     fileManager.obj
 0003:00000168       _undo                      10040168     fileManager.obj
 0003:000001b8       _paste                     100401b8     launchEditor.obj
 0003:00000220       _undo                      10040220     launchEditor.obj
 0003:00000270       _filesave                  10040270     launchEditor.obj
 0003:000002c0       _copy                      100402c0     launchEditor.obj
 0003:00000318       _filemanager               10040318     plugindesc.obj
 0003:00000680       _filesave                  10040680     plugindesc.obj
 0003:000006d0       _launch                    100406d0     plugindesc.obj
 0003:00000748       _workstations              10040748     plugindesc.obj
 0003:000009a8       _filesave                  100409a8     testPlugin.obj
 0003:000009f8       _copy                      100409f8     testPlugin.obj
 0003:00000a50       _paste                     10040a50     testPlugin.obj
 0003:00000ab8       _undo                      10040ab8     testPlugin.obj
 0003:00000b08       _filesave                  10040b08     testPluginFromBase.obj
 0003:00000b58       _copy                      10040b58     testPluginFromBase.obj
 0003:00000bb0       _paste                     10040bb0     testPluginFromBase.obj
 0003:00000c18       _undo                      10040c18     testPluginFromBase.obj
 0003:00000c68       _filesave                  10040c68     workstationEditor.obj
 0003:00000cb8       _copy                      10040cb8     workstationEditor.obj
 0003:00000d10       _paste                     10040d10     workstationEditor.obj
 0003:00000d78       _undo                      10040d78     workstationEditor.obj
 0003:00000dc8       ?param_slot_0@?3??staticMetaObject@fileManager@@SAPAVQMetaObject@@XZ@4QBUQUParameter@@B 10040dc8     moc_fileManager.obj
 0003:00000dd8       ?param_slot_1@?3??staticMetaObject@fileManager@@SAPAVQMetaObject@@XZ@4QBUQUParameter@@B 10040dd8     moc_fileManager.obj
 0003:00000de8       ?param_slot_0@?3??staticMetaObject@launchEditor@@SAPAVQMetaObject@@XZ@4QBUQUParameter@@B 10040de8     moc_launchEditor.obj
 0003:00000df8       ?param_slot_5@?3??staticMetaObject@launchEditorDlg@@SAPAVQMetaObject@@XZ@4QBUQUParameter@@B 10040df8     moc_launcheditordlgimpl.obj
 0003:00000e18       ?param_slot_0@?3??staticMetaObject@workstationCustomTable@@SAPAVQMetaObject@@XZ@4QBUQUParameter@@B 10040e18     moc_workstationCustomTable.obj
 0003:00000e28       ?param_slot_1@?3??staticMetaObject@workstationCustomTable@@SAPAVQMetaObject@@XZ@4QBUQUParameter@@B 10040e28     moc_workstationCustomTable.obj
 0003:00000e48       ?param_slot_2@?3??staticMetaObject@workstationCustomTable@@SAPAVQMetaObject@@XZ@4QBUQUParameter@@B 10040e48     moc_workstationCustomTable.obj
 0003:00000e78       ?param_slot_0@?3??staticMetaObject@workstationEditorDlg@@SAPAVQMetaObject@@XZ@4QBUQUParameter@@B 10040e78     moc_workstationeditordlgimpl.obj
 0003:00000e98       ?param_signal_0@?3??staticMetaObject@xml_listview@@SAPAVQMetaObject@@XZ@4QBUQUParameter@@B 10040e98     moc_xml_listview.obj
 0003:00001744       _cleanUp_dialogBase        10041744     moc_dialog.obj
 0003:0000174c       _cleanUp_dialog            1004174c     moc_dialogimpl.obj
 0003:00001754       _cleanUp_fileDrop          10041754     moc_fileDrop.obj
 0003:00001758       ?param_signal_0@?3??staticMetaObject@fileDrop@@SAPAVQMetaObject@@XZ@4QBUQUParameter@@B 10041758     moc_fileDrop.obj
 0003:00001768       ?$S1@?3??staticMetaObject@fileDrop@@SAPAVQMetaObject@@XZ@4IA 10041768     moc_fileDrop.obj
 0003:00001770       _cleanUp_fileManager       10041770     moc_fileManager.obj
 0003:00001774       ?$S1@?3??staticMetaObject@fileManager@@SAPAVQMetaObject@@XZ@4IA 10041774     moc_fileManager.obj
 0003:00001778       ?param_signal_0@?3??staticMetaObject@fileManager@@SAPAVQMetaObject@@XZ@4QBUQUParameter@@B 10041778     moc_fileManager.obj
 0003:0000179c       _cleanUp_fromBaseDialogBase 1004179c     moc_frombasedialog.obj
 0003:000017a4       _cleanUp_fromBaseDialog    100417a4     moc_frombasedialogimpl.obj
 0003:000017ac       _cleanUp_launchEditor      100417ac     moc_launchEditor.obj
 0003:000017b0       ?$S1@?3??staticMetaObject@launchEditor@@SAPAVQMetaObject@@XZ@4IA 100417b0     moc_launchEditor.obj
 0003:000017b4       ?param_signal_0@?3??staticMetaObject@launchEditor@@SAPAVQMetaObject@@XZ@4QBUQUParameter@@B 100417b4     moc_launchEditor.obj
 0003:000017d8       _cleanUp_launchEditorDlgBase 100417d8     moc_launcheditordlg.obj
 0003:000017e0       _cleanUp_launchEditorDlg   100417e0     moc_launcheditordlgimpl.obj
 0003:000017e4       ?$S1@?3??staticMetaObject@launchEditorDlg@@SAPAVQMetaObject@@XZ@4IA 100417e4     moc_launcheditordlgimpl.obj
 0003:000017e8       ?param_slot_6@?3??staticMetaObject@launchEditorDlg@@SAPAVQMetaObject@@XZ@4QBUQUParameter@@B 100417e8     moc_launcheditordlgimpl.obj
 0003:000017f8       ?param_signal_0@?3??staticMetaObject@launchEditorDlg@@SAPAVQMetaObject@@XZ@4QBUQUParameter@@B 100417f8     moc_launcheditordlgimpl.obj
 0003:0000181c       _cleanUp_testPlugin        1004181c     moc_testPlugin.obj
 0003:00001820       ?param_signal_0@?3??staticMetaObject@testPlugin@@SAPAVQMetaObject@@XZ@4QBUQUParameter@@B 10041820     moc_testPlugin.obj
 0003:00001840       ?$S1@?3??staticMetaObject@testPlugin@@SAPAVQMetaObject@@XZ@4IA 10041840     moc_testPlugin.obj
 0003:00001848       _cleanUp_testPluginFromBase 10041848     moc_testPluginFromBase.obj
 0003:00001850       _cleanUp_workstationCustomTable 10041850     moc_workstationCustomTable.obj
 0003:00001854       ?$S1@?3??staticMetaObject@workstationCustomTable@@SAPAVQMetaObject@@XZ@4IA 10041854     moc_workstationCustomTable.obj
 0003:0000185c       _cleanUp_workstationDockWindowBase 1004185c     moc_workstationdockwindow.obj
 0003:00001864       _cleanUp_workstationDockWindow 10041864     moc_workstationdockwindowimpl.obj
 0003:00001868       ?param_signal_0@?3??staticMetaObject@workstationDockWindow@@SAPAVQMetaObject@@XZ@4QBUQUParameter@@B 10041868     moc_workstationdockwindowimpl.obj
 0003:00001878       ?$S1@?3??staticMetaObject@workstationDockWindow@@SAPAVQMetaObject@@XZ@4IA 10041878     moc_workstationdockwindowimpl.obj
 0003:00001880       _cleanUp_workstationEditor 10041880     moc_workstationeditor.obj
 0003:00001884       ?param_signal_0@?3??staticMetaObject@workstationEditor@@SAPAVQMetaObject@@XZ@4QBUQUParameter@@B 10041884     moc_workstationeditor.obj
 0003:000018a4       ?$S1@?3??staticMetaObject@workstationEditor@@SAPAVQMetaObject@@XZ@4IA 100418a4     moc_workstationeditor.obj
 0003:000018ac       _cleanUp_workstationEditorDlgBase 100418ac     moc_workstationeditordlg.obj
 0003:000018b4       _cleanUp_workstationEditorDlg 100418b4     moc_workstationeditordlgimpl.obj
 0003:000018b8       ?$S1@?3??staticMetaObject@workstationEditorDlg@@SAPAVQMetaObject@@XZ@4IA 100418b8     moc_workstationeditordlgimpl.obj
 0003:000018bc       ?param_signal_0@?3??staticMetaObject@workstationEditorDlg@@SAPAVQMetaObject@@XZ@4QBUQUParameter@@B 100418bc     moc_workstationeditordlgimpl.obj
 0003:000018e0       _cleanUp_workstationEditorNewWsDlgBase 100418e0     moc_workstationeditornewwsdlg.obj
 0003:000018e8       _cleanUp_workstationEditorNewWsDlg 100418e8     moc_workstationeditornewwsdlgimpl.obj
 0003:000018f0       _cleanUp_xml_listview      100418f0     moc_xml_listview.obj
 0003:000018f4       ?$S1@?3??staticMetaObject@xml_listview@@SAPAVQMetaObject@@XZ@4IA 100418f4     moc_xml_listview.obj
 0003:000018fc       _cleanUp_cfg_Table         100418fc     cfg_widgets001:moc_cfg_Table.obj
 0003:00001900       ?param_signal_1@?3??staticMetaObject@cfg_Table@@SAPAVQMetaObject@@XZ@4QBUQUParameter@@B 10041900     cfg_widgets001:moc_cfg_Table.obj
 0003:00001910       ?$S1@?3??staticMetaObject@cfg_Table@@SAPAVQMetaObject@@XZ@4IA 10041910     cfg_widgets001:moc_cfg_Table.obj
 0003:00001918       _cleanUp_pluginBase        10041918     pluginBase:moc_pluginBase.obj
 0003:0000191c       ?param_signal_0@?3??staticMetaObject@pluginBase@@SAPAVQMetaObject@@XZ@4QBUQUParameter@@B 1004191c     pluginBase:moc_pluginBase.obj
 0003:0000193c       ?$S1@?3??staticMetaObject@pluginBase@@SAPAVQMetaObject@@XZ@4IA 1004193c     pluginBase:moc_pluginBase.obj
 0003:00001944       _cleanUp_configFile        10041944     pluginBase:moc_configFile.obj
 0003:00001948       ___proc_attached           10041948     MSVCRT:crtdll.obj
 0003:00001950       _GS_ExceptionRecord        10041950     MSVCRT:gs_report.obj
 0003:000019a0       _GS_ContextRecord          100419a0     MSVCRT:gs_report.obj
 0003:00001c6c       _DebuggerWasPresent        10041c6c     MSVCRT:gs_report.obj
 0004:000000a0       $R000000                   100420a0     Script1.res
 0004:00000528       $R000488                   10042528     Script1.res
